 wzSound

 Timestamp is 56cd51e8 (Wed Feb 24 15:47:04 2016)

 Preferred load address is 10000000

 Start         Length     Name                   Class
 0001:00000000 00077dccH .text                   CODE
 0001:00077dd0 00000a84H .text$x                 CODE
 0001:00078860 0000023cH .text$yc                CODE
 0001:00078aa0 000000eaH .text$yd                CODE
 0002:00000000 00000230H .idata$5                DATA
 0002:00000230 00000004H .CRT$XCA                DATA
 0002:00000234 00000034H .CRT$XCU                DATA
 0002:00000268 00000004H .CRT$XCZ                DATA
 0002:0000026c 00000004H .CRT$XIA                DATA
 0002:00000270 00000014H .CRT$XIC                DATA
 0002:00000284 00000004H .CRT$XIZ                DATA
 0002:00000288 00000004H .CRT$XPA                DATA
 0002:0000028c 00000004H .CRT$XPX                DATA
 0002:00000290 00000004H .CRT$XPXA               DATA
 0002:00000294 00000004H .CRT$XPZ                DATA
 0002:00000298 00000004H .CRT$XTA                DATA
 0002:0000029c 00000004H .CRT$XTZ                DATA
 0002:000002a0 000d9610H .rdata                  DATA
 0002:000d98b0 00000060H .rdata$debug            DATA
 0002:000d9910 0000034cH .rdata$r                DATA
 0002:000d9c5c 00000004H .rtc$IAA                DATA
 0002:000d9c60 00000004H .rtc$IZZ                DATA
 0002:000d9c64 00000004H .rtc$TAA                DATA
 0002:000d9c68 00000004H .rtc$TZZ                DATA
 0002:000d9c70 0000186cH .xdata$x                DATA
 0002:000db4dc 00000064H .idata$2                DATA
 0002:000db540 00000014H .idata$3                DATA
 0002:000db554 00000230H .idata$4                DATA
 0002:000db784 000009deH .idata$6                DATA
 0002:000dc170 00000a32H .edata                  DATA
 0003:00000000 00011450H .data                   DATA
 0003:00011460 000e1940H .bss                    DATA
 0004:00000000 00000058H .rsrc$01                DATA
 0004:00000060 000002f8H .rsrc$02                DATA

  Address         Publics by Value              Rva+Base       Lib:Object

 0000:00000000       ___safe_se_handler_count   00000000     <absolute>
 0000:00000000       ___safe_se_handler_table   00000000     <absolute>
 0000:00000000       __except_list              00000000     <absolute>
 0000:00000000       ___ImageBase               10000000     <linker-defined>
 0001:00000000       ?GetUncompressedAvgDataRate@WaveFile@@QAEIXZ 10001000 f i audiostr.obj
 0001:00000010       ?GetPDS@AudioStreamServices@@QAEPAUIDirectSound8@@XZ 10001010 f i audiostr.obj
 0001:00000020       ?Is_Playing@AudioStream@@QAEHXZ 10001020 f i audiostr.obj
 0001:00000030       ?Is_Paused@AudioStream@@QAEHXZ 10001030 f i audiostr.obj
 0001:00000040       ?Is_Past_Limit@AudioStream@@QAEHXZ 10001040 f i audiostr.obj
 0001:00000050       ?Set_Default_Volume@AudioStream@@QAEXJ@Z 10001050 f i audiostr.obj
 0001:00000060       ?Get_Default_Volume@AudioStream@@QAEJXZ 10001060 f i audiostr.obj
 0001:00000070       ?Set_Base_Volume@AudioStream@@QAEXM@Z 10001070 f i audiostr.obj
 0001:00000080       ?Get_Base_Volume@AudioStream@@QAEMXZ 10001080 f i audiostr.obj
 0001:00000090       ?Is_looping@AudioStream@@QAEHXZ 10001090 f i audiostr.obj
 0001:000000a0       ?Set_looping@AudioStream@@QAEXH@Z 100010a0 f i audiostr.obj
 0001:000000b0       ?Constructor@AudioStreamServices@@QAEXXZ 100010b0 f   audiostr.obj
 0001:000000c0       ?Initialize@AudioStreamServices@@QAEHXZ 100010c0 f   audiostr.obj
 0001:000000e0       ??0AudioStream@@QAE@XZ     100010e0 f   audiostr.obj
 0001:00000100       ??1AudioStream@@QAE@XZ     10001100 f   audiostr.obj
 0001:00000110       ?Init_Data@AudioStream@@QAEXXZ 10001110 f   audiostr.obj
 0001:00000180       ?GetMaxWriteSize@AudioStream@@IAEKXZ 10001180 f   audiostr.obj
 0001:000001d0       ?Set_Sample_Cutoff@AudioStream@@QAEXI@Z 100011d0 f   audiostr.obj
 0001:000001f0       ?Get_Samples_Committed@AudioStream@@QAEIXZ 100011f0 f   audiostr.obj
 0001:00000210       ?Fade_and_Destroy@AudioStream@@QAEXXZ 10001210 f   audiostr.obj
 0001:00000220       ?Fade_and_Stop@AudioStream@@QAEXXZ 10001220 f   audiostr.obj
 0001:00000230       ?Set_Volume@AudioStream@@QAEXJ@Z 10001230 f   audiostr.obj
 0001:00000270       ?Get_Volume@AudioStream@@QAEJXZ 10001270 f   audiostr.obj
 0001:00000280       ?constructor@Timer@@QAEXXZ 10001280 f   audiostr.obj
 0001:00000290       ?destructor@Timer@@QAEXXZ  10001290 f   audiostr.obj
 0001:000002b0       ?TimeProc@Timer@@KGXIIKKK@Z 100012b0 f   audiostr.obj
 0001:000002c0       ?Init@WaveFile@@QAEXXZ     100012c0 f   audiostr.obj
 0001:000002f0       ?Close@WaveFile@@QAEXXZ    100012f0 f   audiostr.obj
 0001:00000350       ?Cue@WaveFile@@QAEHXZ      10001350 f   audiostr.obj
 0001:000003b0       ?Read@WaveFile@@QAEHPAEIH@Z 100013b0 f   audiostr.obj
 0001:000004e0       ?GetSilenceData@WaveFile@@QAEEXZ 100014e0 f   audiostr.obj
 0001:00000510       ?audiostream_init@@YAXXZ   10001510 f   audiostr.obj
 0001:00000570       ?audiostream_is_playing@@YAHH@Z 10001570 f   audiostr.obj
 0001:000005a0       ?audiostream_set_volume_all@@YAXMH@Z 100015a0 f   audiostr.obj
 0001:00000630       ?audiostream_set_volume@@YAXHM@Z 10001630 f   audiostr.obj
 0001:00000680       ?audiostream_is_paused@@YAHH@Z 10001680 f   audiostr.obj
 0001:000006b0       ?audiostream_set_looping@@YAXHH@Z 100016b0 f   audiostr.obj
 0001:000006e0       ?audiostream_set_sample_cutoff@@YAXHI@Z 100016e0 f   audiostr.obj
 0001:00000720       ?audiostream_get_samples_committed@@YAIH@Z 10001720 f   audiostr.obj
 0001:00000760       ?audiostream_done_reading@@YAHH@Z 10001760 f   audiostr.obj
 0001:00000790       ?audiostream_is_inited@@YAHXZ 10001790 f   audiostr.obj
 0001:000007a0       ?WriteWaveData@AudioStream@@IAEHIPAIH@Z 100017a0 f   audiostr.obj
 0001:00000920       ?WriteSilence@AudioStream@@IAEHI@Z 10001920 f   audiostr.obj
 0001:00000a10       ?Cue@AudioStream@@IAEXXZ   10001a10 f   audiostr.obj
 0001:00000a80       ?Stop@AudioStream@@QAEXH@Z 10001a80 f   audiostr.obj
 0001:00000ac0       ?Stop_and_Rewind@AudioStream@@QAEXXZ 10001ac0 f   audiostr.obj
 0001:00000b00       ?Create@Timer@@QAEHIIKP6AHK@Z@Z 10001b00 f   audiostr.obj
 0001:00000b50       ?Open@WaveFile@@QAEHPAD@Z  10001b50 f   audiostr.obj
 0001:00000e60       ?audiostream_stop@@YAXHHH@Z 10001e60 f   audiostr.obj
 0001:00000eb0       ?audiostream_pause@@YAXH@Z 10001eb0 f   audiostr.obj
 0001:00000ef0       ?audiostream_pause_all@@YAXH@Z 10001ef0 f   audiostr.obj
 0001:00000f50       ?Create@AudioStream@@QAEHPADHPAVAudioStreamServices@@@Z 10001f50 f   audiostr.obj
 0001:00001090       ?Destroy@AudioStream@@QAEHXZ 10002090 f   audiostr.obj
 0001:00001130       ?ServiceBuffer@AudioStream@@IAEHXZ 10002130 f   audiostr.obj
 0001:000013a0       ?TimerCallback@AudioStream@@KAHK@Z 100023a0 f   audiostr.obj
 0001:000013b0       ?audiostream_close@@YAXXZ  100023b0 f   audiostr.obj
 0001:00001400       ?audiostream_open@@YAHPADHMH@Z 10002400 f   audiostr.obj
 0001:000014a0       ?audiostream_close_file@@YAXHH@Z 100024a0 f   audiostr.obj
 0001:000014e0       ?audiostream_close_all@@YAXHH@Z 100024e0 f   audiostr.obj
 0001:00001540       ?Play@AudioStream@@QAEXJH@Z 10002540 f   audiostr.obj
 0001:00001630       ?audiostream_play@@YAXHMHH@Z 10002630 f   audiostr.obj
 0001:000016a0       ?audiostream_unpause@@YAXH@Z 100026a0 f   audiostr.obj
 0001:000016e0       ?audiostream_unpause_all@@YAXH@Z 100026e0 f   audiostr.obj
 0001:00001740       ?_Getcont@_Aux_cont@std@@QBEPBV_Container_base_aux@2@XZ 10002740 f i ds.obj
 0001:00001750       ??0_Iterator_base_aux@std@@QAE@XZ 10002750 f i ds.obj
 0001:00001760       ?_Set_container@_Iterator_base_aux@std@@QAEXQBV_Container_base_aux@2@@Z 10002760 f i ds.obj
 0001:00001770       ?_Getmycont@_Iterator_base_aux@std@@QBEPBV_Container_base_aux@2@XZ 10002770 f i ds.obj
 0001:00001780       ?_Same_container@_Iterator_base_aux@std@@QBE_NABV12@@Z 10002780 f i ds.obj
 0001:000017a0       ?_Has_container@_Iterator_base_aux@std@@QBE_NXZ 100027a0 f i ds.obj
 0001:000017b0       _logf                      100027b0 f i ds.obj
 0001:000017d0       ?log@@YAMM@Z               100027d0 f i ds.obj
 0001:000017f0       ?ds_is_3d_buffer@@YAHPAUIDirectSoundBuffer@@@Z 100027f0 f   ds.obj
 0001:00001830       ?ds_is_3d_buffer@@YAHHH@Z  10002830 f   ds.obj
 0001:00001880       ?ds_build_vol_lookup@@YAXXZ 10002880 f   ds.obj
 0001:00001900       ?ds_convert_volume@@YAHM@Z 10002900 f   ds.obj
 0001:00001930       ?ds_get_percentage_vol@@YAMH@Z 10002930 f   ds.obj
 0001:00001950       ?ds_parse_sound@@YAHPAUCFILE@@PAPAEPAIPAPAUtWAVEFORMATEX@@PAUOggVorbis_File@@@Z 10002950 f   ds.obj
 0001:00001b10       ?ds_get_sid@@YAHXZ         10002b10 f   ds.obj
 0001:00001b70       ?ds_get_hid@@YAHXZ         10002b70 f   ds.obj
 0001:00001bd0       ?ds_init_software_buffers@@YAXXZ 10002bd0 f   ds.obj
 0001:00001c00       ?ds_init_hardware_buffers@@YAXXZ 10002c00 f   ds.obj
 0001:00001c30       ?ds_init_buffers@@YAXXZ    10002c30 f   ds.obj
 0001:00001c80       ?ds_get_soundcard_caps@@YAXPAU_DSCAPS@@@Z 10002c80 f   ds.obj
 0001:00001cb0       ?ds_show_caps@@YAXPAU_DSCAPS@@@Z 10002cb0 f   ds.obj
 0001:00001cc0       ?ds_get_primary_format@@YAXPAUtWAVEFORMATEX@@KG@Z 10002cc0 f   ds.obj
 0001:00001d10       ?ds_dll_get_functions@@YAXXZ 10002d10 f   ds.obj
 0001:00001d30       ?ds_dll_load@@YAHXZ        10002d30 f   ds.obj
 0001:00001d70       ?ds_init_property_set@@YAHKG@Z 10002d70 f   ds.obj
 0001:00001eb0       ?get_DSERR_text@@YAPADH@Z  10002eb0 f   ds.obj
 0001:00002000       ?ds_close_channel@@YAXH@Z  10003000 f   ds.obj
 0001:000020c0       ?ds_close_all_channels@@YAXXZ 100030c0 f   ds.obj
 0001:000020f0       ?ds_unload_buffer@@YAXHH@Z 100030f0 f   ds.obj
 0001:00002160       ?ds_close_software_buffers@@YAXXZ 10003160 f   ds.obj
 0001:00002190       ?ds_close_hardware_buffers@@YAXXZ 10003190 f   ds.obj
 0001:000021c0       ?ds_close_buffers@@YAXXZ   100031c0 f   ds.obj
 0001:00002220       ?ds_close@@YAXXZ           10003220 f   ds.obj
 0001:00002300       ?ds_get_3d_interface@@YAXPAUIDirectSoundBuffer@@PAPAUIDirectSound3DBuffer@@@Z 10003300 f   ds.obj
 0001:00002340       ?ds_get_free_channel@@YAHHHH@Z 10003340 f   ds.obj
 0001:00002510       ?ds_channel_dup@@YAHPAUIDirectSoundBuffer@@HH@Z 10003510 f   ds.obj
 0001:00002580       ?ds_restore_buffer@@YAXPAUIDirectSoundBuffer@@@Z 10003580 f   ds.obj
 0001:00002590       ?ds_create_buffer@@YAHHHHH@Z 10003590 f   ds.obj
 0001:000026f0       ?ds_lock_data@@YAHHPAEH@Z  100036f0 f   ds.obj
 0001:000027c0       ?ds_stop_easy@@YAXH@Z      100037c0 f   ds.obj
 0001:000027e0       ?ds_play_easy@@YAHHH@Z     100037e0 f   ds.obj
 0001:00002820       ?ds_play@@YAHHHHHHHH_NH@Z  10003820 f   ds.obj
 0001:000029d0       ?ds_is_channel_playing@@YAHH@Z 100039d0 f   ds.obj
 0001:00002a10       ?ds_stop_channel@@YAXH@Z   10003a10 f   ds.obj
 0001:00002a20       ?ds_stop_channel_all@@YAXXZ 10003a20 f   ds.obj
 0001:00002a60       ?ds_pause_channel@@YAXH@Z  10003a60 f   ds.obj
 0001:00002ae0       ?ds_pause_channel_all@@YAXXZ 10003ae0 f   ds.obj
 0001:00002b20       ?ds_unpause_channel@@YAXH@Z 10003b20 f   ds.obj
 0001:00002b90       ?ds_unpause_channel_all@@YAXXZ 10003b90 f   ds.obj
 0001:00002bd0       ?ds_set_pan@@YAXHH@Z       10003bd0 f   ds.obj
 0001:00002c20       ?ds_get_pitch@@YAHH@Z      10003c20 f   ds.obj
 0001:00002c80       ?ds_set_pitch@@YAXHH@Z     10003c80 f   ds.obj
 0001:00002ce0       ?ds_chg_loop_status@@YAXHH@Z 10003ce0 f   ds.obj
 0001:00002d40       ?ds3d_play@@YAHPAUgame_snd@@HHHPAUvector@@1HHHHHHHPAUSND_DIRECTION@@@Z 10003d40 f   ds.obj
 0001:00002f50       ?ds_set_position@@YAXHK@Z  10003f50 f   ds.obj
 0001:00002f70       ?ds_get_play_position@@YAKH@Z 10003f70 f   ds.obj
 0001:00002fb0       ?ds_get_write_position@@YAKH@Z 10003fb0 f   ds.obj
 0001:00002ff0       ?ds_get_channel_size@@YAHH@Z 10003ff0 f   ds.obj
 0001:00003050       ?ds_get_number_channels@@YAHXZ 10004050 f   ds.obj
 0001:000030b0       ?ds_get_data@@YAHHPAD@Z    100040b0 f   ds.obj
 0001:00003160       ?ds_get_size@@YAHHPAH@Z    10004160 f   ds.obj
 0001:000031c0       ?ds_using_ds3d@@YAHXZ      100041c0 f   ds.obj
 0001:000031d0       ?ds_get_primary_buffer_interface@@YAIXZ 100041d0 f   ds.obj
 0001:000031e0       ?ds_get_dsound_interface@@YAIXZ 100041e0 f   ds.obj
 0001:000031f0       ?ds_get_property_set_interface@@YAIXZ 100041f0 f   ds.obj
 0001:00003200       ?ds_eax_set_environment@@YAHK@Z 10004200 f   ds.obj
 0001:00003240       ?ds_eax_set_preset@@YAHK@Z 10004240 f   ds.obj
 0001:00003280       ?ds_eax_set_all@@YAHKMMM@Z 10004280 f   ds.obj
 0001:000032e0       ?ds_eax_get_all@@YAHPAUEAX_REVERBPROPERTIES@@@Z 100042e0 f   ds.obj
 0001:00003320       ?ds_eax_close@@YAXXZ       10004320 f   ds.obj
 0001:00003340       ?ds_eax_init@@YAHXZ        10004340 f   ds.obj
 0001:000033e0       ?ds_eax_is_inited@@YAHXZ   100043e0 f   ds.obj
 0001:000033f0       ?ds_do_frame@@YAXXZ        100043f0 f   ds.obj
 0001:00003460       ??8const_iterator@?$_Tree@V?$_Tmap_traits@HUgame_snd@@U?$less@H@std@@V?$allocator@U?$pair@$$CBHUgame_snd@@@std@@@3@$0A@@std@@@std@@QBE_NABV012@@Z 10004460 f i ds.obj
 0001:00003490       ??R?$less@H@std@@QBE_NABH0@Z 10004490 f i ds.obj
 0001:000034b0       ?_Mynode@const_iterator@?$_Tree@V?$_Tmap_traits@HUgame_snd@@U?$less@H@std@@V?$allocator@U?$pair@$$CBHUgame_snd@@@std@@@3@$0A@@std@@@std@@QBEPAU_Node@?$_Tree_nod@V?$_Tmap_traits@HUgame_snd@@U?$less@H@std@@V?$allocator@U?$pair@$$CBHUgame_snd@@@std@@@3@$0A@@std@@@3@XZ 100044b0 f i ds.obj
 0001:000034c0       ?_Myval@?$_Tree@V?$_Tmap_traits@HUgame_snd@@U?$less@H@std@@V?$allocator@U?$pair@$$CBHUgame_snd@@@std@@@3@$0A@@std@@@std@@KAAAU?$pair@$$CBHUgame_snd@@@2@PAU_Node@?$_Tree_nod@V?$_Tmap_traits@HUgame_snd@@U?$less@H@std@@V?$allocator@U?$pair@$$CBHUgame_snd@@@std@@@3@$0A@@std@@@2@@Z 100044c0 f i ds.obj
 0001:000034d0       ?_Kfn@?$_Tmap_traits@HUgame_snd@@U?$less@H@std@@V?$allocator@U?$pair@$$CBHUgame_snd@@@std@@@3@$0A@@std@@SAABHABU?$pair@$$CBHUgame_snd@@@2@@Z 100044d0 f i ds.obj
 0001:000034e0       ??Dconst_iterator@?$_Tree@V?$_Tmap_traits@HUgame_snd@@U?$less@H@std@@V?$allocator@U?$pair@$$CBHUgame_snd@@@std@@@3@$0A@@std@@@std@@QBEABU?$pair@$$CBHUgame_snd@@@2@XZ 100044e0 f i ds.obj
 0001:00003510       ??0?$_Iterator_with_base@Ubidirectional_iterator_tag@std@@U?$pair@$$CBHUgame_snd@@@2@HPBU32@ABU32@V_Iterator_base_aux@2@@std@@QAE@XZ 10004510 f i ds.obj
 0001:00003520       ?_Isnil@?$_Tree@V?$_Tmap_traits@HUgame_snd@@U?$less@H@std@@V?$allocator@U?$pair@$$CBHUgame_snd@@@std@@@3@$0A@@std@@@std@@KAAADPAU_Node@?$_Tree_nod@V?$_Tmap_traits@HUgame_snd@@U?$less@H@std@@V?$allocator@U?$pair@$$CBHUgame_snd@@@std@@@3@$0A@@std@@@2@@Z 10004520 f i ds.obj
 0001:00003530       ?_Left@?$_Tree@V?$_Tmap_traits@HUgame_snd@@U?$less@H@std@@V?$allocator@U?$pair@$$CBHUgame_snd@@@std@@@3@$0A@@std@@@std@@KAAAPAU_Node@?$_Tree_nod@V?$_Tmap_traits@HUgame_snd@@U?$less@H@std@@V?$allocator@U?$pair@$$CBHUgame_snd@@@std@@@3@$0A@@std@@@2@PAU342@@Z 10004530 f i ds.obj
 0001:00003540       ?_Right@?$_Tree@V?$_Tmap_traits@HUgame_snd@@U?$less@H@std@@V?$allocator@U?$pair@$$CBHUgame_snd@@@std@@@3@$0A@@std@@@std@@KAAAPAU_Node@?$_Tree_nod@V?$_Tmap_traits@HUgame_snd@@U?$less@H@std@@V?$allocator@U?$pair@$$CBHUgame_snd@@@std@@@3@$0A@@std@@@2@PAU342@@Z 10004540 f i ds.obj
 0001:00003550       ?_Parent@?$_Tree@V?$_Tmap_traits@HUgame_snd@@U?$less@H@std@@V?$allocator@U?$pair@$$CBHUgame_snd@@@std@@@3@$0A@@std@@@std@@KAAAPAU_Node@?$_Tree_nod@V?$_Tmap_traits@HUgame_snd@@U?$less@H@std@@V?$allocator@U?$pair@$$CBHUgame_snd@@@std@@@3@$0A@@std@@@2@PAU342@@Z 10004550 f i ds.obj
 0001:00003560       ??$CAP@M@@YAXAAMMM@Z       10004560 f i ds.obj
 0001:00003590       ?ds_load_buffer@@YAHPAH00PAXPAUsound_info@@H@Z 10004590 f   ds.obj
 0001:00003980       ?ds_init_channels@@YAXXZ   10004980 f   ds.obj
 0001:00003a60       ?ds_init@@YAHHIG@Z         10004a60 f   ds.obj
 0001:00003c80       ?ds_get_channel@@YAHH@Z    10004c80 f   ds.obj
 0001:00003d00       ?ds_find_channel@@YAPAUchannel@@HPAH@Z 10004d00 f   ds.obj
 0001:00003da0       ?ds_eax_set_volume@@YAHM@Z 10004da0 f   ds.obj
 0001:00003e00       ?ds_eax_set_decay_time@@YAHM@Z 10004e00 f   ds.obj
 0001:00003e70       ?ds_eax_set_damping@@YAHM@Z 10004e70 f   ds.obj
 0001:00003ee0       ?_Key@?$_Tree@V?$_Tmap_traits@HUgame_snd@@U?$less@H@std@@V?$allocator@U?$pair@$$CBHUgame_snd@@@std@@@3@$0A@@std@@@std@@KAABHPAU_Node@?$_Tree_nod@V?$_Tmap_traits@HUgame_snd@@U?$less@H@std@@V?$allocator@U?$pair@$$CBHUgame_snd@@@std@@@3@$0A@@std@@@2@@Z 10004ee0 f i ds.obj
 0001:00003ef0       ??Diterator@?$_Tree@V?$_Tmap_traits@HUgame_snd@@U?$less@H@std@@V?$allocator@U?$pair@$$CBHUgame_snd@@@std@@@3@$0A@@std@@@std@@QBEAAU?$pair@$$CBHUgame_snd@@@2@XZ 10004ef0 f i ds.obj
 0001:00003f20       ??0?$_Bidit@U?$pair@$$CBHUgame_snd@@@std@@HPBU12@ABU12@@std@@QAE@XZ 10004f20 f i ds.obj
 0001:00003f30       ?_Root@?$_Tree@V?$_Tmap_traits@HUgame_snd@@U?$less@H@std@@V?$allocator@U?$pair@$$CBHUgame_snd@@@std@@@3@$0A@@std@@@std@@IBEAAPAU_Node@?$_Tree_nod@V?$_Tmap_traits@HUgame_snd@@U?$less@H@std@@V?$allocator@U?$pair@$$CBHUgame_snd@@@std@@@3@$0A@@std@@@2@XZ 10004f30 f i ds.obj
 0001:00003f40       ??Citerator@?$_Tree@V?$_Tmap_traits@HUgame_snd@@U?$less@H@std@@V?$allocator@U?$pair@$$CBHUgame_snd@@@std@@@3@$0A@@std@@@std@@QBEPAU?$pair@$$CBHUgame_snd@@@2@XZ 10004f40 f i ds.obj
 0001:00003f70       ?_Lbound@?$_Tree@V?$_Tmap_traits@HUgame_snd@@U?$less@H@std@@V?$allocator@U?$pair@$$CBHUgame_snd@@@std@@@3@$0A@@std@@@std@@IBEPAU_Node@?$_Tree_nod@V?$_Tmap_traits@HUgame_snd@@U?$less@H@std@@V?$allocator@U?$pair@$$CBHUgame_snd@@@std@@@3@$0A@@std@@@2@ABH@Z 10004f70 f i ds.obj
 0001:00003fa0       ??0const_iterator@?$_Tree@V?$_Tmap_traits@HUgame_snd@@U?$less@H@std@@V?$allocator@U?$pair@$$CBHUgame_snd@@@std@@@3@$0A@@std@@@std@@QAE@PAU_Node@?$_Tree_nod@V?$_Tmap_traits@HUgame_snd@@U?$less@H@std@@V?$allocator@U?$pair@$$CBHUgame_snd@@@std@@@3@$0A@@std@@@2@PBV12@@Z 10004fa0 f i ds.obj
 0001:00003fd0       ??0iterator@?$_Tree@V?$_Tmap_traits@HUgame_snd@@U?$less@H@std@@V?$allocator@U?$pair@$$CBHUgame_snd@@@std@@@3@$0A@@std@@@std@@QAE@PAU_Node@?$_Tree_nod@V?$_Tmap_traits@HUgame_snd@@U?$less@H@std@@V?$allocator@U?$pair@$$CBHUgame_snd@@@std@@@3@$0A@@std@@@2@PBV12@@Z 10004fd0 f i ds.obj
 0001:00004000       ?end@?$_Tree@V?$_Tmap_traits@HUgame_snd@@U?$less@H@std@@V?$allocator@U?$pair@$$CBHUgame_snd@@@std@@@3@$0A@@std@@@std@@QAE?AViterator@12@XZ 10005000 f i ds.obj
 0001:00004020       ?lower_bound@?$_Tree@V?$_Tmap_traits@HUgame_snd@@U?$less@H@std@@V?$allocator@U?$pair@$$CBHUgame_snd@@@std@@@3@$0A@@std@@@std@@QAE?AViterator@12@ABH@Z 10005020 f i ds.obj
 0001:00004060       ?find@?$_Tree@V?$_Tmap_traits@HUgame_snd@@U?$less@H@std@@V?$allocator@U?$pair@$$CBHUgame_snd@@@std@@@3@$0A@@std@@@std@@QAE?AViterator@12@ABH@Z 10005060 f i ds.obj
 0001:000040d0       ?ds_set_volume@@YAXHH@Z    100050d0 f   ds.obj
 0001:000041d0       ?ds_set_volume_all@@YAXH@Z 100051d0 f   ds.obj
 0001:00004210       ?ds3d_update_buffer@@YAHHPAUgame_snd@@MMPAUvector@@1@Z 10005210 f   ds3d.obj
 0001:00004370       ?ds3d_set_sound_cone@@YAHHPAUvector@@HHH@Z 10005370 f   ds3d.obj
 0001:00004420       ?ds3d_update_listener@@YAHPAUvector@@0PAUmatrix@@MMM@Z 10005420 f   ds3d.obj
 0001:00004550       ?ds3d_init_listener@@YAHXZ 10005550 f   ds3d.obj
 0001:00004580       ?ds3d_close_listener@@YAXXZ 10005580 f   ds3d.obj
 0001:000045a0       ?ds3d_init@@YAHH@Z         100055a0 f   ds3d.obj
 0001:00004660       ?ds3d_close@@YAXXZ         10005660 f   ds3d.obj
 0001:00004690       ?assign@?$char_traits@D@std@@SAXAADABD@Z 10005690 f i sound.obj
 0001:000046a0       ?length@?$char_traits@D@std@@SAIPBD@Z 100056a0 f i sound.obj
 0001:000046c0       ?_Copy_s@?$char_traits@D@std@@SAPADPADIPBDI@Z 100056c0 f i sound.obj
 0001:000046f0       ?_Move_s@?$char_traits@D@std@@SAPADPADIPBDI@Z 100056f0 f i sound.obj
 0001:00004720       ??0_Aux_cont@std@@QAE@QBV_Container_base_aux@1@@Z 10005720 f i sound.obj
 0001:00004730       ??0_Container_base_aux@std@@QAE@XZ 10005730 f i sound.obj
 0001:00004740       ??1_Container_base_aux@std@@QAE@XZ 10005740 f i sound.obj
 0001:00004750       ??0bad_alloc@std@@QAE@PBD@Z 10005750 f i sound.obj
 0001:00004770       ??1bad_alloc@std@@UAE@XZ   10005770 f i sound.obj
 0001:00004780       ??_Gbad_alloc@std@@UAEPAXI@Z 10005780 f i sound.obj
 0001:00004780       ??_Ebad_alloc@std@@UAEPAXI@Z 10005780 f i sound.obj
 0001:000047b0       ??2@YAPAXIPAX@Z            100057b0 f i sound.obj
 0001:000047c0       ??3@YAXPAX0@Z              100057c0 f i sound.obj
 0001:000047d0       ??0sound@@QAE@XZ           100057d0 f i sound.obj
 0001:00004800       ?sound_cache_reset@@YAXXZ  10005800 f   sound.obj
 0001:00004820       ?sound_cache_maintain_milliseconds_set@@YAXH@Z 10005820 f   sound.obj
 0001:00004830       ?sound_cache_maintain_milliseconds_get@@YAHXZ 10005830 f   sound.obj
 0001:00004840       ?sound_cache_on@@YAXXZ     10005840 f   sound.obj
 0001:00004850       ?sound_cache_off@@YAXXZ    10005850 f   sound.obj
 0001:00004860       ?sound_cache_is@@YA_NXZ    10005860 f   sound.obj
 0001:00004870       ?ds_priority@@YAHH@Z       10005870 f   sound.obj
 0001:000048b0       ?snd_clear@@YAXXZ          100058b0 f   sound.obj
 0001:000048c0       ?snd_init@@YAHHIG@Z        100058c0 f   sound.obj
 0001:00004970       ?snd_unload@@YAXPAUsound@@@Z 10005970 f   sound.obj
 0001:000049b0       ?snd_update_3d_source_orientation@@YAXHPAUvector@@HHM@Z 100059b0 f   sound.obj
 0001:00004a00       ?snd_stop@@YAXH@Z          10005a00 f   sound.obj
 0001:00004a30       ?snd_pause@@YAXH@Z         10005a30 f   sound.obj
 0001:00004a60       ?snd_pause_all@@YAXXZ      10005a60 f   sound.obj
 0001:00004a70       ?snd_unpause@@YAXH@Z       10005a70 f   sound.obj
 0001:00004aa0       ?snd_unpause_all@@YAXXZ    10005aa0 f   sound.obj
 0001:00004ab0       ?snd_set_volume@@YAXHM@Z   10005ab0 f   sound.obj
 0001:00004b00       ?snd_set_volume_all@@YAXM@Z 10005b00 f   sound.obj
 0001:00004b40       ?snd_set_pan@@YAXHM@Z      10005b40 f   sound.obj
 0001:00004b80       ?snd_get_pitch@@YAHH@Z     10005b80 f   sound.obj
 0001:00004bb0       ?snd_set_pitch@@YAXHH@Z    10005bb0 f   sound.obj
 0001:00004be0       ?snd_is_playing@@YAHH@Z    10005be0 f   sound.obj
 0001:00004c20       ?snd_chg_loop_status@@YAXHH@Z 10005c20 f   sound.obj
 0001:00004c50       ?snd_stop_all@@YAXXZ       10005c50 f   sound.obj
 0001:00004c60       ?sound_get_ds@@YAIXZ       10005c60 f   sound.obj
 0001:00004c70       ?snd_is_inited@@YAHXZ      10005c70 f   sound.obj
 0001:00004c80       ?snd_update_listener@@YAXPAUvector@@0PAUmatrix@@MMM@Z 10005c80 f   sound.obj
 0001:00004cc0       ?snd_num_playing@@YAHXZ    10005cc0 f   sound.obj
 0001:00004cd0       ?snd_stop_any_sound@@YAXXZ 10005cd0 f   sound.obj
 0001:00004d00       ?sound_env_set@@YAHPAUsound_env@@@Z 10005d00 f   sound.obj
 0001:00004d60       ?sound_env_set_preset@@YAHK@Z 10005d60 f   sound.obj
 0001:00004d70       ?sound_env_get@@YAHPAUsound_env@@@Z 10005d70 f   sound.obj
 0001:00004db0       ?sound_env_disable@@YAHXZ  10005db0 f   sound.obj
 0001:00004de0       ?sound_env_supported@@YAHXZ 10005de0 f   sound.obj
 0001:00004df0       ?sound_check_channel@@YAXXZ 10005df0 f   sound.obj
 0001:00004e00       ?size@?$basic_string@DU?$char_traits@D@std@@V?$allocator@D@2@@std@@QBEIXZ 10005e00 f i sound.obj
 0001:00004e10       ?size@?$_Tree@V?$_Tmap_traits@HUsound@@U?$less@H@std@@V?$allocator@U?$pair@$$CBHUsound@@@std@@@3@$0A@@std@@@std@@QBEIXZ 10005e10 f i sound.obj
 0001:00004e20       ?_Myptr@?$basic_string@DU?$char_traits@D@std@@V?$allocator@D@2@@std@@IBEPBDXZ 10005e20 f i sound.obj
 0001:00004e30       ?_Color@?$_Tree@V?$_Tmap_traits@HUsound@@U?$less@H@std@@V?$allocator@U?$pair@$$CBHUsound@@@std@@@3@$0A@@std@@@std@@KAAADPAU_Node@?$_Tree_nod@V?$_Tmap_traits@HUsound@@U?$less@H@std@@V?$allocator@U?$pair@$$CBHUsound@@@std@@@3@$0A@@std@@@2@@Z 10005e30 f i sound.obj
 0001:00004e40       ?_Isnil@?$_Tree@V?$_Tmap_traits@HUsound@@U?$less@H@std@@V?$allocator@U?$pair@$$CBHUsound@@@std@@@3@$0A@@std@@@std@@KAAADPAU_Node@?$_Tree_nod@V?$_Tmap_traits@HUsound@@U?$less@H@std@@V?$allocator@U?$pair@$$CBHUsound@@@std@@@3@$0A@@std@@@2@@Z 10005e40 f i sound.obj
 0001:00004e50       ?_Left@?$_Tree@V?$_Tmap_traits@HUsound@@U?$less@H@std@@V?$allocator@U?$pair@$$CBHUsound@@@std@@@3@$0A@@std@@@std@@KAAAPAU_Node@?$_Tree_nod@V?$_Tmap_traits@HUsound@@U?$less@H@std@@V?$allocator@U?$pair@$$CBHUsound@@@std@@@3@$0A@@std@@@2@PAU342@@Z 10005e50 f i sound.obj
 0001:00004e60       ?_Parent@?$_Tree@V?$_Tmap_traits@HUsound@@U?$less@H@std@@V?$allocator@U?$pair@$$CBHUsound@@@std@@@3@$0A@@std@@@std@@KAAAPAU_Node@?$_Tree_nod@V?$_Tmap_traits@HUsound@@U?$less@H@std@@V?$allocator@U?$pair@$$CBHUsound@@@std@@@3@$0A@@std@@@2@PAU342@@Z 10005e60 f i sound.obj
 0001:00004e70       ?_Right@?$_Tree@V?$_Tmap_traits@HUsound@@U?$less@H@std@@V?$allocator@U?$pair@$$CBHUsound@@@std@@@3@$0A@@std@@@std@@KAAAPAU_Node@?$_Tree_nod@V?$_Tmap_traits@HUsound@@U?$less@H@std@@V?$allocator@U?$pair@$$CBHUsound@@@std@@@3@$0A@@std@@@2@PAU342@@Z 10005e70 f i sound.obj
 0001:00004e80       ?_Lmost@?$_Tree@V?$_Tmap_traits@HUsound@@U?$less@H@std@@V?$allocator@U?$pair@$$CBHUsound@@@std@@@3@$0A@@std@@@std@@IBEAAPAU_Node@?$_Tree_nod@V?$_Tmap_traits@HUsound@@U?$less@H@std@@V?$allocator@U?$pair@$$CBHUsound@@@std@@@3@$0A@@std@@@2@XZ 10005e80 f i sound.obj
 0001:00004e90       ?_Max@?$_Tree@V?$_Tmap_traits@HUsound@@U?$less@H@std@@V?$allocator@U?$pair@$$CBHUsound@@@std@@@3@$0A@@std@@@std@@KAPAU_Node@?$_Tree_nod@V?$_Tmap_traits@HUsound@@U?$less@H@std@@V?$allocator@U?$pair@$$CBHUsound@@@std@@@3@$0A@@std@@@2@PAU342@@Z 10005e90 f i sound.obj
 0001:00004eb0       ?_Min@?$_Tree@V?$_Tmap_traits@HUsound@@U?$less@H@std@@V?$allocator@U?$pair@$$CBHUsound@@@std@@@3@$0A@@std@@@std@@KAPAU_Node@?$_Tree_nod@V?$_Tmap_traits@HUsound@@U?$less@H@std@@V?$allocator@U?$pair@$$CBHUsound@@@std@@@3@$0A@@std@@@2@PAU342@@Z 10005eb0 f i sound.obj
 0001:00004ed0       ?_Rmost@?$_Tree@V?$_Tmap_traits@HUsound@@U?$less@H@std@@V?$allocator@U?$pair@$$CBHUsound@@@std@@@3@$0A@@std@@@std@@IBEAAPAU_Node@?$_Tree_nod@V?$_Tmap_traits@HUsound@@U?$less@H@std@@V?$allocator@U?$pair@$$CBHUsound@@@std@@@3@$0A@@std@@@2@XZ 10005ed0 f i sound.obj
 0001:00004ee0       ?_Root@?$_Tree@V?$_Tmap_traits@HUsound@@U?$less@H@std@@V?$allocator@U?$pair@$$CBHUsound@@@std@@@3@$0A@@std@@@std@@IBEAAPAU_Node@?$_Tree_nod@V?$_Tmap_traits@HUsound@@U?$less@H@std@@V?$allocator@U?$pair@$$CBHUsound@@@std@@@3@$0A@@std@@@2@XZ 10005ee0 f i sound.obj
 0001:00004ef0       ?_Rrotate@?$_Tree@V?$_Tmap_traits@HUsound@@U?$less@H@std@@V?$allocator@U?$pair@$$CBHUsound@@@std@@@3@$0A@@std@@@std@@IAEXPAU_Node@?$_Tree_nod@V?$_Tmap_traits@HUsound@@U?$less@H@std@@V?$allocator@U?$pair@$$CBHUsound@@@std@@@3@$0A@@std@@@2@@Z 10005ef0 f i sound.obj
 0001:00004f50       ??0?$allocator@U?$pair@$$CBHUsound@@@std@@@std@@QAE@XZ 10005f50 f i sound.obj
 0001:00004f60       ?deallocate@?$allocator@U_Node@?$_Tree_nod@V?$_Tmap_traits@HUsound@@U?$less@H@std@@V?$allocator@U?$pair@$$CBHUsound@@@std@@@3@$0A@@std@@@std@@@std@@QAEXPAU_Node@?$_Tree_nod@V?$_Tmap_traits@HUsound@@U?$less@H@std@@V?$allocator@U?$pair@$$CBHUsound@@@std@@@3@$0A@@std@@@2@I@Z 10005f60 f i sound.obj
 0001:00004f70       ??8const_iterator@?$_Tree@V?$_Tmap_traits@HUsound@@U?$less@H@std@@V?$allocator@U?$pair@$$CBHUsound@@@std@@@3@$0A@@std@@@std@@QBE_NABV012@@Z 10005f70 f i sound.obj
 0001:00004fa0       ?_Mynode@const_iterator@?$_Tree@V?$_Tmap_traits@HUsound@@U?$less@H@std@@V?$allocator@U?$pair@$$CBHUsound@@@std@@@3@$0A@@std@@@std@@QBEPAU_Node@?$_Tree_nod@V?$_Tmap_traits@HUsound@@U?$less@H@std@@V?$allocator@U?$pair@$$CBHUsound@@@std@@@3@$0A@@std@@@3@XZ 10005fa0 f i sound.obj
 0001:00004fb0       ??0?$pair@$$CBHUsound@@@std@@QAE@ABHABUsound@@@Z 10005fb0 f i sound.obj
 0001:00004fd0       ?_Myptr@?$basic_string@DU?$char_traits@D@std@@V?$allocator@D@2@@std@@IAEPADXZ 10005fd0 f i sound.obj
 0001:00004fe0       ??0?$allocator@D@std@@QAE@XZ 10005fe0 f i sound.obj
 0001:00004ff0       ??0?$allocator@D@std@@QAE@ABV01@@Z 10005ff0 f i sound.obj
 0001:00005000       ?deallocate@?$allocator@D@std@@QAEXPADI@Z 10006000 f i sound.obj
 0001:00005010       ?deallocate@?$allocator@V_Aux_cont@std@@@std@@QAEXPAV_Aux_cont@2@I@Z 10006010 f i sound.obj
 0001:00005020       ?_Myval@?$_Tree@V?$_Tmap_traits@HUsound@@U?$less@H@std@@V?$allocator@U?$pair@$$CBHUsound@@@std@@@3@$0A@@std@@@std@@KAAAU?$pair@$$CBHUsound@@@2@PAU_Node@?$_Tree_nod@V?$_Tmap_traits@HUsound@@U?$less@H@std@@V?$allocator@U?$pair@$$CBHUsound@@@std@@@3@$0A@@std@@@2@@Z 10006020 f i sound.obj
 0001:00005030       ?_Kfn@?$_Tmap_traits@HUsound@@U?$less@H@std@@V?$allocator@U?$pair@$$CBHUsound@@@std@@@3@$0A@@std@@SAABHABU?$pair@$$CBHUsound@@@2@@Z 10006030 f i sound.obj
 0001:00005040       ??0?$allocator@U?$pair@$$CBHUsound@@@std@@@std@@QAE@ABV01@@Z 10006040 f i sound.obj
 0001:00005050       ??Dconst_iterator@?$_Tree@V?$_Tmap_traits@HUsound@@U?$less@H@std@@V?$allocator@U?$pair@$$CBHUsound@@@std@@@3@$0A@@std@@@std@@QBEABU?$pair@$$CBHUsound@@@2@XZ 10006050 f i sound.obj
 0001:00005080       ?_Inc@const_iterator@?$_Tree@V?$_Tmap_traits@HUsound@@U?$less@H@std@@V?$allocator@U?$pair@$$CBHUsound@@@std@@@3@$0A@@std@@@std@@QAEXXZ 10006080 f i sound.obj
 0001:00005100       ??0?$_Iterator_with_base@Ubidirectional_iterator_tag@std@@U?$pair@$$CBHUsound@@@2@HPBU32@ABU32@V_Iterator_base_aux@2@@std@@QAE@XZ 10006100 f i sound.obj
 0001:00005110       ?_Dec@const_iterator@?$_Tree@V?$_Tmap_traits@HUsound@@U?$less@H@std@@V?$allocator@U?$pair@$$CBHUsound@@@std@@@3@$0A@@std@@@std@@QAEXXZ 10006110 f i sound.obj
 0001:000051b0       ??0?$pair@Viterator@?$_Tree@V?$_Tmap_traits@HUsound@@U?$less@H@std@@V?$allocator@U?$pair@$$CBHUsound@@@std@@@3@$0A@@std@@@std@@V123@@std@@QAE@ABViterator@?$_Tree@V?$_Tmap_traits@HUsound@@U?$less@H@std@@V?$allocator@U?$pair@$$CBHUsound@@@std@@@3@$0A@@std@@@1@0@Z 100061b0 f i sound.obj
 0001:000051e0       ??0?$pair@Viterator@?$_Tree@V?$_Tmap_traits@HUsound@@U?$less@H@std@@V?$allocator@U?$pair@$$CBHUsound@@@std@@@3@$0A@@std@@@std@@_N@std@@QAE@ABViterator@?$_Tree@V?$_Tmap_traits@HUsound@@U?$less@H@std@@V?$allocator@U?$pair@$$CBHUsound@@@std@@@3@$0A@@std@@@1@AB_N@Z 100061e0 f i sound.obj
 0001:00005200       ?_Inside@?$basic_string@DU?$char_traits@D@std@@V?$allocator@D@2@@std@@IAE_NPBD@Z 10006200 f i sound.obj
 0001:00005240       ?max_size@?$allocator@D@std@@QBEIXZ 10006240 f i sound.obj
 0001:00005250       ?max_size@?$allocator@U?$pair@$$CBHUsound@@@std@@@std@@QBEIXZ 10006250 f i sound.obj
 0001:00005260       ??0_Node@?$_Tree_nod@V?$_Tmap_traits@HUsound@@U?$less@H@std@@V?$allocator@U?$pair@$$CBHUsound@@@std@@@3@$0A@@std@@@std@@QAE@PAU012@00ABU?$pair@$$CBHUsound@@@2@D@Z 10006260 f i sound.obj
 0001:000052a0       ??$swap@D@std@@YAXAAD0@Z   100062a0 f i sound.obj
 0001:000052c0       ??$_Destroy@U_Node@?$_Tree_nod@V?$_Tmap_traits@HUsound@@U?$less@H@std@@V?$allocator@U?$pair@$$CBHUsound@@@std@@@3@$0A@@std@@@std@@@std@@YAXPAU_Node@?$_Tree_nod@V?$_Tmap_traits@HUsound@@U?$less@H@std@@V?$allocator@U?$pair@$$CBHUsound@@@std@@@3@$0A@@std@@@0@@Z 100062c0 f i sound.obj
 0001:000052d0       ??$_Destroy@PAU_Node@?$_Tree_nod@V?$_Tmap_traits@HUsound@@U?$less@H@std@@V?$allocator@U?$pair@$$CBHUsound@@@std@@@3@$0A@@std@@@std@@@std@@YAXPAPAU_Node@?$_Tree_nod@V?$_Tmap_traits@HUsound@@U?$less@H@std@@V?$allocator@U?$pair@$$CBHUsound@@@std@@@3@$0A@@std@@@0@@Z 100062d0 f i sound.obj
 0001:000052e0       ??$?0U?$pair@$$CBHUsound@@@std@@@?$allocator@PAU_Node@?$_Tree_nod@V?$_Tmap_traits@HUsound@@U?$less@H@std@@V?$allocator@U?$pair@$$CBHUsound@@@std@@@3@$0A@@std@@@std@@@std@@QAE@ABV?$allocator@U?$pair@$$CBHUsound@@@std@@@1@@Z 100062e0 f i sound.obj
 0001:000052f0       ??$_Allocate@D@std@@YAPADIPAD@Z 100062f0 f i sound.obj
 0001:00005350       ??$?0U?$pair@$$CBHUsound@@@std@@@?$allocator@U_Node@?$_Tree_nod@V?$_Tmap_traits@HUsound@@U?$less@H@std@@V?$allocator@U?$pair@$$CBHUsound@@@std@@@3@$0A@@std@@@std@@@std@@QAE@ABV?$allocator@U?$pair@$$CBHUsound@@@std@@@1@@Z 10006350 f i sound.obj
 0001:00005360       ??$_Allocate@U_Node@?$_Tree_nod@V?$_Tmap_traits@HUsound@@U?$less@H@std@@V?$allocator@U?$pair@$$CBHUsound@@@std@@@3@$0A@@std@@@std@@@std@@YAPAU_Node@?$_Tree_nod@V?$_Tmap_traits@HUsound@@U?$less@H@std@@V?$allocator@U?$pair@$$CBHUsound@@@std@@@3@$0A@@std@@@0@IPAU120@@Z 10006360 f i sound.obj
 0001:000053c0       ??$_Construct@PAU_Node@?$_Tree_nod@V?$_Tmap_traits@HUsound@@U?$less@H@std@@V?$allocator@U?$pair@$$CBHUsound@@@std@@@3@$0A@@std@@@std@@PAU123@@std@@YAXPAPAU_Node@?$_Tree_nod@V?$_Tmap_traits@HUsound@@U?$less@H@std@@V?$allocator@U?$pair@$$CBHUsound@@@std@@@3@$0A@@std@@@0@ABQAU120@@Z 100063c0 f i sound.obj
 0001:000053e0       ??$?0U?$pair@$$CBHUsound@@@std@@@?$allocator@V_Aux_cont@std@@@std@@QAE@ABV?$allocator@U?$pair@$$CBHUsound@@@std@@@1@@Z 100063e0 f i sound.obj
 0001:000053f0       ??$_Allocate@V_Aux_cont@std@@@std@@YAPAV_Aux_cont@0@IPAV10@@Z 100063f0 f i sound.obj
 0001:00005450       ??0bad_alloc@std@@QAE@ABV01@@Z 10006450 f i sound.obj
 0001:00005470       ??$_Iter_cat@Viterator@?$_Tree@V?$_Tmap_traits@HUsound@@U?$less@H@std@@V?$allocator@U?$pair@$$CBHUsound@@@std@@@3@$0A@@std@@@std@@@std@@YA?AUbidirectional_iterator_tag@0@ABViterator@?$_Tree@V?$_Tmap_traits@HUsound@@U?$less@H@std@@V?$allocator@U?$pair@$$CBHUsound@@@std@@@3@$0A@@std@@@0@@Z 10006470 f i sound.obj
 0001:00005480       ??$_Char_traits_cat@U?$char_traits@D@std@@@std@@YA?AU_Secure_char_traits_tag@0@XZ 10006480 f i sound.obj
 0001:00005490       ??$copy_s@U?$char_traits@D@std@@@_Traits_helper@std@@YAPADPADIPBDIU_Secure_char_traits_tag@1@@Z 10006490 f i sound.obj
 0001:000054c0       ??$move_s@U?$char_traits@D@std@@@_Traits_helper@std@@YAPADPADIPBDIU_Secure_char_traits_tag@1@@Z 100064c0 f i sound.obj
 0001:000054f0       ?sound_size@@YAHXZ         100064f0 f   sound.obj
 0001:00005500       ??9const_iterator@?$_Tree@V?$_Tmap_traits@HUsound@@U?$less@H@std@@V?$allocator@U?$pair@$$CBHUsound@@@std@@@3@$0A@@std@@@std@@QBE_NABV012@@Z 10006500 f i sound.obj
 0001:00005530       ??9const_iterator@?$_Tree@V?$_Tmap_traits@HUgame_snd@@U?$less@H@std@@V?$allocator@U?$pair@$$CBHUgame_snd@@@std@@@3@$0A@@std@@@std@@QBE_NABV012@@Z 10006530 f i sound.obj
 0001:00005560       ??0?$_String_val@DV?$allocator@D@std@@@std@@QAE@ABV01@@Z 10006560 f i sound.obj
 0001:00005570       ?_Key@?$_Tree@V?$_Tmap_traits@HUsound@@U?$less@H@std@@V?$allocator@U?$pair@$$CBHUsound@@@std@@@3@$0A@@std@@@std@@KAABHPAU_Node@?$_Tree_nod@V?$_Tmap_traits@HUsound@@U?$less@H@std@@V?$allocator@U?$pair@$$CBHUsound@@@std@@@3@$0A@@std@@@2@@Z 10006570 f i sound.obj
 0001:00005580       ?_Lrotate@?$_Tree@V?$_Tmap_traits@HUsound@@U?$less@H@std@@V?$allocator@U?$pair@$$CBHUsound@@@std@@@3@$0A@@std@@@std@@IAEXPAU_Node@?$_Tree_nod@V?$_Tmap_traits@HUsound@@U?$less@H@std@@V?$allocator@U?$pair@$$CBHUsound@@@std@@@3@$0A@@std@@@2@@Z 10006580 f i sound.obj
 0001:000055e0       ??1?$_Container_base_aux_alloc_real@V?$allocator@U?$pair@$$CBHUsound@@@std@@@std@@@std@@IAE@XZ 100065e0 f i sound.obj
 0001:000055f0       ?destroy@?$allocator@U_Node@?$_Tree_nod@V?$_Tmap_traits@HUsound@@U?$less@H@std@@V?$allocator@U?$pair@$$CBHUsound@@@std@@@3@$0A@@std@@@std@@@std@@QAEXPAU_Node@?$_Tree_nod@V?$_Tmap_traits@HUsound@@U?$less@H@std@@V?$allocator@U?$pair@$$CBHUsound@@@std@@@3@$0A@@std@@@2@@Z 100065f0 f i sound.obj
 0001:00005600       ??Diterator@?$_Tree@V?$_Tmap_traits@HUsound@@U?$less@H@std@@V?$allocator@U?$pair@$$CBHUsound@@@std@@@3@$0A@@std@@@std@@QBEAAU?$pair@$$CBHUsound@@@2@XZ 10006600 f i sound.obj
 0001:00005630       ??Econst_iterator@?$_Tree@V?$_Tmap_traits@HUsound@@U?$less@H@std@@V?$allocator@U?$pair@$$CBHUsound@@@std@@@3@$0A@@std@@@std@@QAEAAV012@XZ 10006630 f i sound.obj
 0001:00005640       ?_Eos@?$basic_string@DU?$char_traits@D@std@@V?$allocator@D@2@@std@@IAEXI@Z 10006640 f i sound.obj
 0001:00005660       ??0?$_String_val@DV?$allocator@D@std@@@std@@IAE@V?$allocator@D@1@@Z 10006660 f i sound.obj
 0001:00005670       ?_Lbound@?$_Tree@V?$_Tmap_traits@HUsound@@U?$less@H@std@@V?$allocator@U?$pair@$$CBHUsound@@@std@@@3@$0A@@std@@@std@@IBEPAU_Node@?$_Tree_nod@V?$_Tmap_traits@HUsound@@U?$less@H@std@@V?$allocator@U?$pair@$$CBHUsound@@@std@@@3@$0A@@std@@@2@ABH@Z 10006670 f i sound.obj
 0001:000056a0       ?destroy@?$allocator@PAU_Node@?$_Tree_nod@V?$_Tmap_traits@HUsound@@U?$less@H@std@@V?$allocator@U?$pair@$$CBHUsound@@@std@@@3@$0A@@std@@@std@@@std@@QAEXPAPAU_Node@?$_Tree_nod@V?$_Tmap_traits@HUsound@@U?$less@H@std@@V?$allocator@U?$pair@$$CBHUsound@@@std@@@3@$0A@@std@@@2@@Z 100066a0 f i sound.obj
 0001:000056b0       ??Econst_iterator@?$_Tree@V?$_Tmap_traits@HUsound@@U?$less@H@std@@V?$allocator@U?$pair@$$CBHUsound@@@std@@@3@$0A@@std@@@std@@QAE?AV012@H@Z 100066b0 f i sound.obj
 0001:000056d0       ??Fconst_iterator@?$_Tree@V?$_Tmap_traits@HUsound@@U?$less@H@std@@V?$allocator@U?$pair@$$CBHUsound@@@std@@@3@$0A@@std@@@std@@QAEAAV012@XZ 100066d0 f i sound.obj
 0001:000056e0       ??0?$_Bidit@U?$pair@$$CBHUsound@@@std@@HPBU12@ABU12@@std@@QAE@XZ 100066e0 f i sound.obj
 0001:000056f0       ?max_size@?$basic_string@DU?$char_traits@D@std@@V?$allocator@D@2@@std@@QBEIXZ 100066f0 f i sound.obj
 0001:00005700       ?max_size@?$_Tree@V?$_Tmap_traits@HUsound@@U?$less@H@std@@V?$allocator@U?$pair@$$CBHUsound@@@std@@@3@$0A@@std@@@std@@QBEIXZ 10006700 f i sound.obj
 0001:00005710       ??Fiterator@?$_Tree@V?$_Tmap_traits@HUsound@@U?$less@H@std@@V?$allocator@U?$pair@$$CBHUsound@@@std@@@3@$0A@@std@@@std@@QAEAAV012@XZ 10006710 f i sound.obj
 0001:00005720       ?allocate@?$allocator@D@std@@QAEPADI@Z 10006720 f i sound.obj
 0001:00005740       ?allocate@?$allocator@U_Node@?$_Tree_nod@V?$_Tmap_traits@HUsound@@U?$less@H@std@@V?$allocator@U?$pair@$$CBHUsound@@@std@@@3@$0A@@std@@@std@@@std@@QAEPAU_Node@?$_Tree_nod@V?$_Tmap_traits@HUsound@@U?$less@H@std@@V?$allocator@U?$pair@$$CBHUsound@@@std@@@3@$0A@@std@@@2@I@Z 10006740 f i sound.obj
 0001:00005760       ?construct@?$allocator@PAU_Node@?$_Tree_nod@V?$_Tmap_traits@HUsound@@U?$less@H@std@@V?$allocator@U?$pair@$$CBHUsound@@@std@@@3@$0A@@std@@@std@@@std@@QAEXPAPAU_Node@?$_Tree_nod@V?$_Tmap_traits@HUsound@@U?$less@H@std@@V?$allocator@U?$pair@$$CBHUsound@@@std@@@3@$0A@@std@@@2@ABQAU342@@Z 10006760 f i sound.obj
 0001:00005780       ?allocate@?$allocator@V_Aux_cont@std@@@std@@QAEPAV_Aux_cont@2@I@Z 10006780 f i sound.obj
 0001:000057a0       ??$copy_s@U?$char_traits@D@std@@@_Traits_helper@std@@YAPADPADIPBDI@Z 100067a0 f i sound.obj
 0001:000057d0       ??$move_s@U?$char_traits@D@std@@@_Traits_helper@std@@YAPADPADIPBDI@Z 100067d0 f i sound.obj
 0001:00005800       ??Citerator@?$_Tree@V?$_Tmap_traits@HUsound@@U?$less@H@std@@V?$allocator@U?$pair@$$CBHUsound@@@std@@@3@$0A@@std@@@std@@QBEPAU?$pair@$$CBHUsound@@@2@XZ 10006800 f i sound.obj
 0001:00005830       ??Eiterator@?$_Tree@V?$_Tmap_traits@HUsound@@U?$less@H@std@@V?$allocator@U?$pair@$$CBHUsound@@@std@@@3@$0A@@std@@@std@@QAEAAV012@XZ 10006830 f i sound.obj
 0001:00005840       ??1?$_Tmap_traits@HUsound@@U?$less@H@std@@V?$allocator@U?$pair@$$CBHUsound@@@std@@@3@$0A@@std@@QAE@XZ 10006840 f i sound.obj
 0001:00005850       ?_Tidy@?$basic_string@DU?$char_traits@D@std@@V?$allocator@D@2@@std@@IAEX_NI@Z 10006850 f i sound.obj
 0001:000058a0       ?_Erase@?$_Tree@V?$_Tmap_traits@HUsound@@U?$less@H@std@@V?$allocator@U?$pair@$$CBHUsound@@@std@@@3@$0A@@std@@@std@@IAEXPAU_Node@?$_Tree_nod@V?$_Tmap_traits@HUsound@@U?$less@H@std@@V?$allocator@U?$pair@$$CBHUsound@@@std@@@3@$0A@@std@@@2@@Z 100068a0 f i sound.obj
 0001:000058e0       ?erase@?$basic_string@DU?$char_traits@D@std@@V?$allocator@D@2@@std@@QAEAAV12@II@Z 100068e0 f i sound.obj
 0001:00005970       ??0const_iterator@?$_Tree@V?$_Tmap_traits@HUsound@@U?$less@H@std@@V?$allocator@U?$pair@$$CBHUsound@@@std@@@3@$0A@@std@@@std@@QAE@XZ 10006970 f i sound.obj
 0001:00005980       ??0const_iterator@?$_Tree@V?$_Tmap_traits@HUsound@@U?$less@H@std@@V?$allocator@U?$pair@$$CBHUsound@@@std@@@3@$0A@@std@@@std@@QAE@PAU_Node@?$_Tree_nod@V?$_Tmap_traits@HUsound@@U?$less@H@std@@V?$allocator@U?$pair@$$CBHUsound@@@std@@@3@$0A@@std@@@2@PBV12@@Z 10006980 f i sound.obj
 0001:000059b0       ?_Copy@?$basic_string@DU?$char_traits@D@std@@V?$allocator@D@2@@std@@IAEXII@Z 100069b0 f i sound.obj
 0001:00005af0       ?_Buynode@?$_Tree@V?$_Tmap_traits@HUsound@@U?$less@H@std@@V?$allocator@U?$pair@$$CBHUsound@@@std@@@3@$0A@@std@@@std@@IAEPAU_Node@?$_Tree_nod@V?$_Tmap_traits@HUsound@@U?$less@H@std@@V?$allocator@U?$pair@$$CBHUsound@@@std@@@3@$0A@@std@@@2@XZ 10006af0 f i sound.obj
 0001:00005b30       ?_Buynode@?$_Tree@V?$_Tmap_traits@HUsound@@U?$less@H@std@@V?$allocator@U?$pair@$$CBHUsound@@@std@@@3@$0A@@std@@@std@@IAEPAU_Node@?$_Tree_nod@V?$_Tmap_traits@HUsound@@U?$less@H@std@@V?$allocator@U?$pair@$$CBHUsound@@@std@@@3@$0A@@std@@@2@PAU342@00ABU?$pair@$$CBHUsound@@@2@D@Z 10006b30 f i sound.obj
 0001:00005b80       ??0?$_Container_base_aux_alloc_real@V?$allocator@U?$pair@$$CBHUsound@@@std@@@std@@@std@@IAE@V?$allocator@U?$pair@$$CBHUsound@@@std@@@1@@Z 10006b80 f i sound.obj
 0001:00005bb0       ??$_Distance2@Viterator@?$_Tree@V?$_Tmap_traits@HUsound@@U?$less@H@std@@V?$allocator@U?$pair@$$CBHUsound@@@std@@@3@$0A@@std@@@std@@I@std@@YAXViterator@?$_Tree@V?$_Tmap_traits@HUsound@@U?$less@H@std@@V?$allocator@U?$pair@$$CBHUsound@@@std@@@3@$0A@@std@@@0@0AAIUbidirectional_iterator_tag@0@@Z 10006bb0 f i sound.obj
 0001:00005bf0       ??1?$basic_string@DU?$char_traits@D@std@@V?$allocator@D@2@@std@@QAE@XZ 10006bf0 f i sound.obj
 0001:00005c20       ?clear@?$_Tree@V?$_Tmap_traits@HUsound@@U?$less@H@std@@V?$allocator@U?$pair@$$CBHUsound@@@std@@@3@$0A@@std@@@std@@QAEXXZ 10006c20 f i sound.obj
 0001:00005c50       ??1?$_Tree_nod@V?$_Tmap_traits@HUsound@@U?$less@H@std@@V?$allocator@U?$pair@$$CBHUsound@@@std@@@3@$0A@@std@@@std@@QAE@XZ 10006c50 f i sound.obj
 0001:00005c60       ??0iterator@?$_Tree@V?$_Tmap_traits@HUsound@@U?$less@H@std@@V?$allocator@U?$pair@$$CBHUsound@@@std@@@3@$0A@@std@@@std@@QAE@PAU_Node@?$_Tree_nod@V?$_Tmap_traits@HUsound@@U?$less@H@std@@V?$allocator@U?$pair@$$CBHUsound@@@std@@@3@$0A@@std@@@2@PBV12@@Z 10006c60 f i sound.obj
 0001:00005c90       ?_Grow@?$basic_string@DU?$char_traits@D@std@@V?$allocator@D@2@@std@@IAE_NI_N@Z 10006c90 f i sound.obj
 0001:00005d50       ?_Eqrange@?$_Tree@V?$_Tmap_traits@HUsound@@U?$less@H@std@@V?$allocator@U?$pair@$$CBHUsound@@@std@@@3@$0A@@std@@@std@@IAE?AU?$pair@Viterator@?$_Tree@V?$_Tmap_traits@HUsound@@U?$less@H@std@@V?$allocator@U?$pair@$$CBHUsound@@@std@@@3@$0A@@std@@@std@@V123@@2@ABH@Z 10006d50 f i sound.obj
 0001:00005df0       ?_Init@?$_Tree@V?$_Tmap_traits@HUsound@@U?$less@H@std@@V?$allocator@U?$pair@$$CBHUsound@@@std@@@3@$0A@@std@@@std@@IAEXXZ 10006df0 f i sound.obj
 0001:00005e20       ??0?$_Tmap_traits@HUsound@@U?$less@H@std@@V?$allocator@U?$pair@$$CBHUsound@@@std@@@3@$0A@@std@@QAE@U?$less@H@1@V?$allocator@U?$pair@$$CBHUsound@@@std@@@1@@Z 10006e20 f i sound.obj
 0001:00005e50       ??$_Distance@Viterator@?$_Tree@V?$_Tmap_traits@HUsound@@U?$less@H@std@@V?$allocator@U?$pair@$$CBHUsound@@@std@@@3@$0A@@std@@@std@@I@std@@YAXViterator@?$_Tree@V?$_Tmap_traits@HUsound@@U?$less@H@std@@V?$allocator@U?$pair@$$CBHUsound@@@std@@@3@$0A@@std@@@0@0AAI@Z 10006e50 f i sound.obj
 0001:00005e80       ??1logic_error@std@@UAE@XZ 10006e80 f i sound.obj
 0001:00005ec0       ?c_str@?$basic_string@DU?$char_traits@D@std@@V?$allocator@D@2@@std@@QBEPBDXZ 10006ec0 f i sound.obj
 0001:00005ed0       ?what@logic_error@std@@UBEPBDXZ 10006ed0 f i sound.obj
 0001:00005ee0       ??_Glogic_error@std@@UAEPAXI@Z 10006ee0 f i sound.obj
 0001:00005ee0       ??_Elogic_error@std@@UAEPAXI@Z 10006ee0 f i sound.obj
 0001:00005f30       ?begin@?$_Tree@V?$_Tmap_traits@HUsound@@U?$less@H@std@@V?$allocator@U?$pair@$$CBHUsound@@@std@@@3@$0A@@std@@@std@@QAE?AViterator@12@XZ 10006f30 f i sound.obj
 0001:00005f50       ?end@?$_Tree@V?$_Tmap_traits@HUsound@@U?$less@H@std@@V?$allocator@U?$pair@$$CBHUsound@@@std@@@3@$0A@@std@@@std@@QAE?AViterator@12@XZ 10006f50 f i sound.obj
 0001:00005f70       ??1?$_Tree_ptr@V?$_Tmap_traits@HUsound@@U?$less@H@std@@V?$allocator@U?$pair@$$CBHUsound@@@std@@@3@$0A@@std@@@std@@QAE@XZ 10006f70 f i sound.obj
 0001:00005f80       ?assign@?$basic_string@DU?$char_traits@D@std@@V?$allocator@D@2@@std@@QAEAAV12@ABV12@II@Z 10006f80 f i sound.obj
 0001:00006060       ?_Make_iter@?$_Tree@V?$_Tmap_traits@HUsound@@U?$less@H@std@@V?$allocator@U?$pair@$$CBHUsound@@@std@@@3@$0A@@std@@@std@@QBE?AViterator@12@Vconst_iterator@12@@Z 10007060 f i sound.obj
 0001:00006090       ?lower_bound@?$_Tree@V?$_Tmap_traits@HUsound@@U?$less@H@std@@V?$allocator@U?$pair@$$CBHUsound@@@std@@@3@$0A@@std@@@std@@QAE?AViterator@12@ABH@Z 10007090 f i sound.obj
 0001:000060d0       ?equal_range@?$_Tree@V?$_Tmap_traits@HUsound@@U?$less@H@std@@V?$allocator@U?$pair@$$CBHUsound@@@std@@@3@$0A@@std@@@std@@QAE?AU?$pair@Viterator@?$_Tree@V?$_Tmap_traits@HUsound@@U?$less@H@std@@V?$allocator@U?$pair@$$CBHUsound@@@std@@@3@$0A@@std@@@std@@V123@@2@ABH@Z 100070d0 f i sound.obj
 0001:000060f0       ?assign@?$basic_string@DU?$char_traits@D@std@@V?$allocator@D@2@@std@@QAEAAV12@PBDI@Z 100070f0 f i sound.obj
 0001:000061d0       ??0?$_Tree_nod@V?$_Tmap_traits@HUsound@@U?$less@H@std@@V?$allocator@U?$pair@$$CBHUsound@@@std@@@3@$0A@@std@@@std@@IAE@ABU?$less@H@1@V?$allocator@U?$pair@$$CBHUsound@@@std@@@1@@Z 100071d0 f i sound.obj
 0001:00006200       ?snd_unload_all@@YAXXZ     10007200 f   sound.obj
 0001:00006300       ?snd_close@@YAXXZ          10007300 f   sound.obj
 0001:00006340       ??0?$basic_string@DU?$char_traits@D@std@@V?$allocator@D@2@@std@@QAE@ABV01@@Z 10007340 f i sound.obj
 0001:00006370       ?find@?$_Tree@V?$_Tmap_traits@HUsound@@U?$less@H@std@@V?$allocator@U?$pair@$$CBHUsound@@@std@@@3@$0A@@std@@@std@@QAE?AViterator@12@ABH@Z 10007370 f i sound.obj
 0001:000063e0       ??1?$_Tree_val@V?$_Tmap_traits@HUsound@@U?$less@H@std@@V?$allocator@U?$pair@$$CBHUsound@@@std@@@3@$0A@@std@@@std@@QAE@XZ 100073e0 f i sound.obj
 0001:000063f0       ?assign@?$basic_string@DU?$char_traits@D@std@@V?$allocator@D@2@@std@@QAEAAV12@PBD@Z 100073f0 f i sound.obj
 0001:00006420       ??0?$_Tree_ptr@V?$_Tmap_traits@HUsound@@U?$less@H@std@@V?$allocator@U?$pair@$$CBHUsound@@@std@@@3@$0A@@std@@@std@@IAE@ABU?$less@H@1@V?$allocator@U?$pair@$$CBHUsound@@@std@@@1@@Z 10007420 f i sound.obj
 0001:00006450       ??0logic_error@std@@QAE@ABV?$basic_string@DU?$char_traits@D@std@@V?$allocator@D@2@@1@@Z 10007450 f i sound.obj
 0001:000064c0       ??0length_error@std@@QAE@ABV?$basic_string@DU?$char_traits@D@std@@V?$allocator@D@2@@1@@Z 100074c0 f i sound.obj
 0001:000064e0       ??1length_error@std@@UAE@XZ 100074e0 f i sound.obj
 0001:00006520       ??_Glength_error@std@@UAEPAXI@Z 10007520 f i sound.obj
 0001:00006520       ??_Elength_error@std@@UAEPAXI@Z 10007520 f i sound.obj
 0001:00006570       ??0out_of_range@std@@QAE@ABV?$basic_string@DU?$char_traits@D@std@@V?$allocator@D@2@@1@@Z 10007570 f i sound.obj
 0001:00006590       ??1out_of_range@std@@UAE@XZ 10007590 f i sound.obj
 0001:000065d0       ??_Gout_of_range@std@@UAEPAXI@Z 100075d0 f i sound.obj
 0001:000065d0       ??_Eout_of_range@std@@UAEPAXI@Z 100075d0 f i sound.obj
 0001:00006620       ?sound_get@@YAPAUsound@@H@Z 10007620 f   sound.obj
 0001:00006690       ?snd_update_3d_source_position@@YAXHPAUvector@@0MM@Z 10007690 f   sound.obj
 0001:00006740       ??0?$basic_string@DU?$char_traits@D@std@@V?$allocator@D@2@@std@@QAE@PBD@Z 10007740 f i sound.obj
 0001:00006780       ?_Insert@?$_Tree@V?$_Tmap_traits@HUsound@@U?$less@H@std@@V?$allocator@U?$pair@$$CBHUsound@@@std@@@3@$0A@@std@@@std@@IAE?AViterator@12@_NPAU_Node@?$_Tree_nod@V?$_Tmap_traits@HUsound@@U?$less@H@std@@V?$allocator@U?$pair@$$CBHUsound@@@std@@@3@$0A@@std@@@2@ABU?$pair@$$CBHUsound@@@2@@Z 10007780 f i sound.obj
 0001:00006990       ??0logic_error@std@@QAE@ABV01@@Z 10007990 f i sound.obj
 0001:00006a10       ??0length_error@std@@QAE@ABV01@@Z 10007a10 f i sound.obj
 0001:00006a30       ??0?$_Tree_val@V?$_Tmap_traits@HUsound@@U?$less@H@std@@V?$allocator@U?$pair@$$CBHUsound@@@std@@@3@$0A@@std@@@std@@IAE@ABU?$less@H@1@V?$allocator@U?$pair@$$CBHUsound@@@std@@@1@@Z 10007a30 f i sound.obj
 0001:00006a60       ?erase@?$_Tree@V?$_Tmap_traits@HUsound@@U?$less@H@std@@V?$allocator@U?$pair@$$CBHUsound@@@std@@@3@$0A@@std@@@std@@QAE?AViterator@12@Vconst_iterator@12@@Z 10007a60 f i sound.obj
 0001:00006db0       ??0out_of_range@std@@QAE@ABV01@@Z 10007db0 f i sound.obj
 0001:00006dd0       ??0?$_Tree@V?$_Tmap_traits@HUsound@@U?$less@H@std@@V?$allocator@U?$pair@$$CBHUsound@@@std@@@3@$0A@@std@@@std@@QAE@ABU?$less@H@1@ABV?$allocator@U?$pair@$$CBHUsound@@@std@@@1@@Z 10007dd0 f i sound.obj
 0001:00006e60       ?erase@?$_Tree@V?$_Tmap_traits@HUsound@@U?$less@H@std@@V?$allocator@U?$pair@$$CBHUsound@@@std@@@3@$0A@@std@@@std@@QAE?AViterator@12@Vconst_iterator@12@0@Z 10007e60 f i sound.obj
 0001:00006f40       ?_Tidy@?$_Tree@V?$_Tmap_traits@HUsound@@U?$less@H@std@@V?$allocator@U?$pair@$$CBHUsound@@@std@@@3@$0A@@std@@@std@@IAEXXZ 10007f40 f i sound.obj
 0001:00006f80       ?insert@?$_Tree@V?$_Tmap_traits@HUsound@@U?$less@H@std@@V?$allocator@U?$pair@$$CBHUsound@@@std@@@3@$0A@@std@@@std@@QAE?AU?$pair@Viterator@?$_Tree@V?$_Tmap_traits@HUsound@@U?$less@H@std@@V?$allocator@U?$pair@$$CBHUsound@@@std@@@3@$0A@@std@@@std@@_N@2@ABU?$pair@$$CBHUsound@@@2@@Z 10007f80 f i sound.obj
 0001:00007080       ?sound_update_cache@@YAXXZ 10008080 f   sound.obj
 0001:000072a0       ??1?$_Tree@V?$_Tmap_traits@HUsound@@U?$less@H@std@@V?$allocator@U?$pair@$$CBHUsound@@@std@@@3@$0A@@std@@@std@@QAE@XZ 100082a0 f i sound.obj
 0001:00007320       ?erase@?$_Tree@V?$_Tmap_traits@HUsound@@U?$less@H@std@@V?$allocator@U?$pair@$$CBHUsound@@@std@@@3@$0A@@std@@@std@@QAEIABH@Z 10008320 f i sound.obj
 0001:00007390       ?insert@?$_Tree@V?$_Tmap_traits@HUsound@@U?$less@H@std@@V?$allocator@U?$pair@$$CBHUsound@@@std@@@3@$0A@@std@@@std@@QAE?AViterator@12@Vconst_iterator@12@ABU?$pair@$$CBHUsound@@@2@@Z 10008390 f i sound.obj
 0001:00007570       ??1?$map@HUsound@@U?$less@H@std@@V?$allocator@U?$pair@$$CBHUsound@@@std@@@3@@std@@QAE@XZ 10008570 f i sound.obj
 0001:00007580       ?snd_unload@@YAHH@Z        10008580 f   sound.obj
 0001:000075c0       ??0?$map@HUsound@@U?$less@H@std@@V?$allocator@U?$pair@$$CBHUsound@@@std@@@3@@std@@QAE@XZ 100085c0 f i sound.obj
 0001:000075e0       ??A?$map@HUsound@@U?$less@H@std@@V?$allocator@U?$pair@$$CBHUsound@@@std@@@3@@std@@QAEAAUsound@@ABH@Z 100085e0 f i sound.obj
 0001:000076d0       ?snd_load@@YAPAUsound@@PAUgame_snd@@H@Z 100086d0 f   sound.obj
 0001:00007960       ?snd_play@@YAHPAUgame_snd@@MMH_NHH@Z 10008960 f   sound.obj
 0001:00007ab0       ?snd_get_3d_vol_and_pan@@YAHPAUgame_snd@@PAUvector@@PAM2M@Z 10008ab0 f   sound.obj
 0001:00007bc0       ?snd_play_looping@@YAHPAUgame_snd@@MHHMHH@Z 10008bc0 f   sound.obj
 0001:00007cd0       ?snd_play_3d@@YAHPAUgame_snd@@PAUvector@@1M1HMH1MHHPAUSND_DIRECTION@@MM@Z 10008cd0 f   sound.obj
 0001:00007fc0       ?snd_update_3d_pos@@YAXHPAUgame_snd@@PAUvector@@@Z 10008fc0 f   sound.obj
 0001:00008070       ?ogg_cfread@@YAIPAXII0@Z   10009070 f   ogg.obj
 0001:00008080       ?ogg_cfseek@@YAHPAX_JH@Z   10009080 f   ogg.obj
 0001:000080a0       ?ogg_cfclose@@YAHPAX@Z     100090a0 f   ogg.obj
 0001:000080b0       ?ogg_cftell@@YAJPAX@Z      100090b0 f   ogg.obj
 0001:000080c0       ?ogg_mmio_read@@YAIPAXII0@Z 100090c0 f   ogg.obj
 0001:000080e0       ?ogg_mmio_seek@@YAHPAX_JH@Z 100090e0 f   ogg.obj
 0001:00008100       ?ogg_mmio_close@@YAHPAX@Z  10009100 f   ogg.obj
 0001:00008110       ?ogg_mmio_tell@@YAJPAX@Z   10009110 f   ogg.obj
 0001:00008130       ?OGG_init@@YAHXZ           10009130 f   ogg.obj
 0001:00008160       ?ambi_init@@YAXXZ          10009160 f   ambientsnd.obj
 0001:00008170       ?ambi_close@@YAXXZ         10009170 f   ambientsnd.obj
 0001:00008180       ?ambi_stop_all@@YAXH@Z     10009180 f   ambientsnd.obj
 0001:00008190       ?ambi_pause_all@@YAXXZ     10009190 f   ambientsnd.obj
 0001:000081a0       ?ambi_unpause_all@@YAXXZ   100091a0 f   ambientsnd.obj
 0001:000081b0       ?ambi_set_volume_all@@YAXM@Z 100091b0 f   ambientsnd.obj
 0001:000081d0       ??8const_iterator@?$_Tree@V?$_Tmap_traits@HHU?$less@H@std@@V?$allocator@U?$pair@$$CBHH@std@@@2@$0A@@std@@@std@@QBE_NABV012@@Z 100091d0 f i ambientsnd.obj
 0001:00008200       ??8const_iterator@?$_Tree@V?$_Tmap_traits@HUAmbientSnd@@U?$less@H@std@@V?$allocator@U?$pair@$$CBHUAmbientSnd@@@std@@@3@$0A@@std@@@std@@QBE_NABV012@@Z 10009200 f i ambientsnd.obj
 0001:00008230       ??0?$allocator@U?$pair@$$CBHH@std@@@std@@QAE@XZ 10009230 f i ambientsnd.obj
 0001:00008240       ?_Mynode@const_iterator@?$_Tree@V?$_Tmap_traits@HHU?$less@H@std@@V?$allocator@U?$pair@$$CBHH@std@@@2@$0A@@std@@@std@@QBEPAU_Node@?$_Tree_nod@V?$_Tmap_traits@HHU?$less@H@std@@V?$allocator@U?$pair@$$CBHH@std@@@2@$0A@@std@@@3@XZ 10009240 f i ambientsnd.obj
 0001:00008250       ??0?$pair@$$CBHH@std@@QAE@ABH0@Z 10009250 f i ambientsnd.obj
 0001:00008270       ?_Mynode@const_iterator@?$_Tree@V?$_Tmap_traits@HUAmbientSnd@@U?$less@H@std@@V?$allocator@U?$pair@$$CBHUAmbientSnd@@@std@@@3@$0A@@std@@@std@@QBEPAU_Node@?$_Tree_nod@V?$_Tmap_traits@HUAmbientSnd@@U?$less@H@std@@V?$allocator@U?$pair@$$CBHUAmbientSnd@@@std@@@3@$0A@@std@@@3@XZ 10009270 f i ambientsnd.obj
 0001:00008280       ??0?$pair@$$CBHUAmbientSnd@@@std@@QAE@ABHABUAmbientSnd@@@Z 10009280 f i ambientsnd.obj
 0001:000082a0       ?_Isnil@?$_Tree@V?$_Tmap_traits@HHU?$less@H@std@@V?$allocator@U?$pair@$$CBHH@std@@@2@$0A@@std@@@std@@KAAADPAU_Node@?$_Tree_nod@V?$_Tmap_traits@HHU?$less@H@std@@V?$allocator@U?$pair@$$CBHH@std@@@2@$0A@@std@@@2@@Z 100092a0 f i ambientsnd.obj
 0001:000082b0       ?_Left@?$_Tree@V?$_Tmap_traits@HHU?$less@H@std@@V?$allocator@U?$pair@$$CBHH@std@@@2@$0A@@std@@@std@@KAAAPAU_Node@?$_Tree_nod@V?$_Tmap_traits@HHU?$less@H@std@@V?$allocator@U?$pair@$$CBHH@std@@@2@$0A@@std@@@2@PAU342@@Z 100092b0 f i ambientsnd.obj
 0001:000082c0       ?_Parent@?$_Tree@V?$_Tmap_traits@HHU?$less@H@std@@V?$allocator@U?$pair@$$CBHH@std@@@2@$0A@@std@@@std@@KAAAPAU_Node@?$_Tree_nod@V?$_Tmap_traits@HHU?$less@H@std@@V?$allocator@U?$pair@$$CBHH@std@@@2@$0A@@std@@@2@PAU342@@Z 100092c0 f i ambientsnd.obj
 0001:000082d0       ?_Right@?$_Tree@V?$_Tmap_traits@HHU?$less@H@std@@V?$allocator@U?$pair@$$CBHH@std@@@2@$0A@@std@@@std@@KAAAPAU_Node@?$_Tree_nod@V?$_Tmap_traits@HHU?$less@H@std@@V?$allocator@U?$pair@$$CBHH@std@@@2@$0A@@std@@@2@PAU342@@Z 100092d0 f i ambientsnd.obj
 0001:000082e0       ?_Myval@?$_Tree@V?$_Tmap_traits@HHU?$less@H@std@@V?$allocator@U?$pair@$$CBHH@std@@@2@$0A@@std@@@std@@KAAAU?$pair@$$CBHH@2@PAU_Node@?$_Tree_nod@V?$_Tmap_traits@HHU?$less@H@std@@V?$allocator@U?$pair@$$CBHH@std@@@2@$0A@@std@@@2@@Z 100092e0 f i ambientsnd.obj
 0001:000082f0       ?size@?$_Tree@V?$_Tmap_traits@HHU?$less@H@std@@V?$allocator@U?$pair@$$CBHH@std@@@2@$0A@@std@@@std@@QBEIXZ 100092f0 f i ambientsnd.obj
 0001:00008300       ?_Rmost@?$_Tree@V?$_Tmap_traits@HHU?$less@H@std@@V?$allocator@U?$pair@$$CBHH@std@@@2@$0A@@std@@@std@@IBEAAPAU_Node@?$_Tree_nod@V?$_Tmap_traits@HHU?$less@H@std@@V?$allocator@U?$pair@$$CBHH@std@@@2@$0A@@std@@@2@XZ 10009300 f i ambientsnd.obj
 0001:00008310       ?_Kfn@?$_Tmap_traits@HHU?$less@H@std@@V?$allocator@U?$pair@$$CBHH@std@@@2@$0A@@std@@SAABHABU?$pair@$$CBHH@2@@Z 10009310 f i ambientsnd.obj
 0001:00008320       ??0?$allocator@U?$pair@$$CBHH@std@@@std@@QAE@ABV01@@Z 10009320 f i ambientsnd.obj
 0001:00008330       ?deallocate@?$allocator@U_Node@?$_Tree_nod@V?$_Tmap_traits@HHU?$less@H@std@@V?$allocator@U?$pair@$$CBHH@std@@@2@$0A@@std@@@std@@@std@@QAEXPAU_Node@?$_Tree_nod@V?$_Tmap_traits@HHU?$less@H@std@@V?$allocator@U?$pair@$$CBHH@std@@@2@$0A@@std@@@2@I@Z 10009330 f i ambientsnd.obj
 0001:00008340       ?_Isnil@?$_Tree@V?$_Tmap_traits@HUAmbientSnd@@U?$less@H@std@@V?$allocator@U?$pair@$$CBHUAmbientSnd@@@std@@@3@$0A@@std@@@std@@KAAADPAU_Node@?$_Tree_nod@V?$_Tmap_traits@HUAmbientSnd@@U?$less@H@std@@V?$allocator@U?$pair@$$CBHUAmbientSnd@@@std@@@3@$0A@@std@@@2@@Z 10009340 f i ambientsnd.obj
 0001:00008350       ?_Right@?$_Tree@V?$_Tmap_traits@HUAmbientSnd@@U?$less@H@std@@V?$allocator@U?$pair@$$CBHUAmbientSnd@@@std@@@3@$0A@@std@@@std@@KAAAPAU_Node@?$_Tree_nod@V?$_Tmap_traits@HUAmbientSnd@@U?$less@H@std@@V?$allocator@U?$pair@$$CBHUAmbientSnd@@@std@@@3@$0A@@std@@@2@PAU342@@Z 10009350 f i ambientsnd.obj
 0001:00008360       ?_Myval@?$_Tree@V?$_Tmap_traits@HUAmbientSnd@@U?$less@H@std@@V?$allocator@U?$pair@$$CBHUAmbientSnd@@@std@@@3@$0A@@std@@@std@@KAAAU?$pair@$$CBHUAmbientSnd@@@2@PAU_Node@?$_Tree_nod@V?$_Tmap_traits@HUAmbientSnd@@U?$less@H@std@@V?$allocator@U?$pair@$$CBHUAmbientSnd@@@std@@@3@$0A@@std@@@2@@Z 10009360 f i ambientsnd.obj
 0001:00008370       ?size@?$_Tree@V?$_Tmap_traits@HUAmbientSnd@@U?$less@H@std@@V?$allocator@U?$pair@$$CBHUAmbientSnd@@@std@@@3@$0A@@std@@@std@@QBEIXZ 10009370 f i ambientsnd.obj
 0001:00008380       ?_Rmost@?$_Tree@V?$_Tmap_traits@HUAmbientSnd@@U?$less@H@std@@V?$allocator@U?$pair@$$CBHUAmbientSnd@@@std@@@3@$0A@@std@@@std@@IBEAAPAU_Node@?$_Tree_nod@V?$_Tmap_traits@HUAmbientSnd@@U?$less@H@std@@V?$allocator@U?$pair@$$CBHUAmbientSnd@@@std@@@3@$0A@@std@@@2@XZ 10009380 f i ambientsnd.obj
 0001:00008390       ?_Kfn@?$_Tmap_traits@HUAmbientSnd@@U?$less@H@std@@V?$allocator@U?$pair@$$CBHUAmbientSnd@@@std@@@3@$0A@@std@@SAABHABU?$pair@$$CBHUAmbientSnd@@@2@@Z 10009390 f i ambientsnd.obj
 0001:000083a0       ??Dconst_iterator@?$_Tree@V?$_Tmap_traits@HHU?$less@H@std@@V?$allocator@U?$pair@$$CBHH@std@@@2@$0A@@std@@@std@@QBEABU?$pair@$$CBHH@2@XZ 100093a0 f i ambientsnd.obj
 0001:000083d0       ??Dconst_iterator@?$_Tree@V?$_Tmap_traits@HUAmbientSnd@@U?$less@H@std@@V?$allocator@U?$pair@$$CBHUAmbientSnd@@@std@@@3@$0A@@std@@@std@@QBEABU?$pair@$$CBHUAmbientSnd@@@2@XZ 100093d0 f i ambientsnd.obj
 0001:00008400       ??0?$_Iterator_with_base@Ubidirectional_iterator_tag@std@@U?$pair@$$CBHH@2@HPBU32@ABU32@V_Iterator_base_aux@2@@std@@QAE@XZ 10009400 f i ambientsnd.obj
 0001:00008410       ??0?$_Iterator_with_base@Ubidirectional_iterator_tag@std@@U?$pair@$$CBHUAmbientSnd@@@2@HPBU32@ABU32@V_Iterator_base_aux@2@@std@@QAE@XZ 10009410 f i ambientsnd.obj
 0001:00008420       ?_Color@?$_Tree@V?$_Tmap_traits@HHU?$less@H@std@@V?$allocator@U?$pair@$$CBHH@std@@@2@$0A@@std@@@std@@KAAADPAU_Node@?$_Tree_nod@V?$_Tmap_traits@HHU?$less@H@std@@V?$allocator@U?$pair@$$CBHH@std@@@2@$0A@@std@@@2@@Z 10009420 f i ambientsnd.obj
 0001:00008430       ?_Lmost@?$_Tree@V?$_Tmap_traits@HHU?$less@H@std@@V?$allocator@U?$pair@$$CBHH@std@@@2@$0A@@std@@@std@@IBEAAPAU_Node@?$_Tree_nod@V?$_Tmap_traits@HHU?$less@H@std@@V?$allocator@U?$pair@$$CBHH@std@@@2@$0A@@std@@@2@XZ 10009430 f i ambientsnd.obj
 0001:00008440       ?_Root@?$_Tree@V?$_Tmap_traits@HHU?$less@H@std@@V?$allocator@U?$pair@$$CBHH@std@@@2@$0A@@std@@@std@@IBEAAPAU_Node@?$_Tree_nod@V?$_Tmap_traits@HHU?$less@H@std@@V?$allocator@U?$pair@$$CBHH@std@@@2@$0A@@std@@@2@XZ 10009440 f i ambientsnd.obj
 0001:00008450       ?_Rrotate@?$_Tree@V?$_Tmap_traits@HHU?$less@H@std@@V?$allocator@U?$pair@$$CBHH@std@@@2@$0A@@std@@@std@@IAEXPAU_Node@?$_Tree_nod@V?$_Tmap_traits@HHU?$less@H@std@@V?$allocator@U?$pair@$$CBHH@std@@@2@$0A@@std@@@2@@Z 10009450 f i ambientsnd.obj
 0001:000084b0       ?_Color@?$_Tree@V?$_Tmap_traits@HUAmbientSnd@@U?$less@H@std@@V?$allocator@U?$pair@$$CBHUAmbientSnd@@@std@@@3@$0A@@std@@@std@@KAAADPAU_Node@?$_Tree_nod@V?$_Tmap_traits@HUAmbientSnd@@U?$less@H@std@@V?$allocator@U?$pair@$$CBHUAmbientSnd@@@std@@@3@$0A@@std@@@2@@Z 100094b0 f i ambientsnd.obj
 0001:000084c0       ?_Left@?$_Tree@V?$_Tmap_traits@HUAmbientSnd@@U?$less@H@std@@V?$allocator@U?$pair@$$CBHUAmbientSnd@@@std@@@3@$0A@@std@@@std@@KAAAPAU_Node@?$_Tree_nod@V?$_Tmap_traits@HUAmbientSnd@@U?$less@H@std@@V?$allocator@U?$pair@$$CBHUAmbientSnd@@@std@@@3@$0A@@std@@@2@PAU342@@Z 100094c0 f i ambientsnd.obj
 0001:000084d0       ?_Parent@?$_Tree@V?$_Tmap_traits@HUAmbientSnd@@U?$less@H@std@@V?$allocator@U?$pair@$$CBHUAmbientSnd@@@std@@@3@$0A@@std@@@std@@KAAAPAU_Node@?$_Tree_nod@V?$_Tmap_traits@HUAmbientSnd@@U?$less@H@std@@V?$allocator@U?$pair@$$CBHUAmbientSnd@@@std@@@3@$0A@@std@@@2@PAU342@@Z 100094d0 f i ambientsnd.obj
 0001:000084e0       ?_Lmost@?$_Tree@V?$_Tmap_traits@HUAmbientSnd@@U?$less@H@std@@V?$allocator@U?$pair@$$CBHUAmbientSnd@@@std@@@3@$0A@@std@@@std@@IBEAAPAU_Node@?$_Tree_nod@V?$_Tmap_traits@HUAmbientSnd@@U?$less@H@std@@V?$allocator@U?$pair@$$CBHUAmbientSnd@@@std@@@3@$0A@@std@@@2@XZ 100094e0 f i ambientsnd.obj
 0001:000084f0       ?_Root@?$_Tree@V?$_Tmap_traits@HUAmbientSnd@@U?$less@H@std@@V?$allocator@U?$pair@$$CBHUAmbientSnd@@@std@@@3@$0A@@std@@@std@@IBEAAPAU_Node@?$_Tree_nod@V?$_Tmap_traits@HUAmbientSnd@@U?$less@H@std@@V?$allocator@U?$pair@$$CBHUAmbientSnd@@@std@@@3@$0A@@std@@@2@XZ 100094f0 f i ambientsnd.obj
 0001:00008500       ?_Rrotate@?$_Tree@V?$_Tmap_traits@HUAmbientSnd@@U?$less@H@std@@V?$allocator@U?$pair@$$CBHUAmbientSnd@@@std@@@3@$0A@@std@@@std@@IAEXPAU_Node@?$_Tree_nod@V?$_Tmap_traits@HUAmbientSnd@@U?$less@H@std@@V?$allocator@U?$pair@$$CBHUAmbientSnd@@@std@@@3@$0A@@std@@@2@@Z 10009500 f i ambientsnd.obj
 0001:00008560       ??9const_iterator@?$_Tree@V?$_Tmap_traits@HHU?$less@H@std@@V?$allocator@U?$pair@$$CBHH@std@@@2@$0A@@std@@@std@@QBE_NABV012@@Z 10009560 f i ambientsnd.obj
 0001:00008590       ??0?$pair@Viterator@?$_Tree@V?$_Tmap_traits@HHU?$less@H@std@@V?$allocator@U?$pair@$$CBHH@std@@@2@$0A@@std@@@std@@_N@std@@QAE@ABViterator@?$_Tree@V?$_Tmap_traits@HHU?$less@H@std@@V?$allocator@U?$pair@$$CBHH@std@@@2@$0A@@std@@@1@AB_N@Z 10009590 f i ambientsnd.obj
 0001:000085b0       ??0?$pair@Viterator@?$_Tree@V?$_Tmap_traits@HUAmbientSnd@@U?$less@H@std@@V?$allocator@U?$pair@$$CBHUAmbientSnd@@@std@@@3@$0A@@std@@@std@@_N@std@@QAE@ABViterator@?$_Tree@V?$_Tmap_traits@HUAmbientSnd@@U?$less@H@std@@V?$allocator@U?$pair@$$CBHUAmbientSnd@@@std@@@3@$0A@@std@@@1@AB_N@Z 100095b0 f i ambientsnd.obj
 0001:000085d0       ?_Max@?$_Tree@V?$_Tmap_traits@HHU?$less@H@std@@V?$allocator@U?$pair@$$CBHH@std@@@2@$0A@@std@@@std@@KAPAU_Node@?$_Tree_nod@V?$_Tmap_traits@HHU?$less@H@std@@V?$allocator@U?$pair@$$CBHH@std@@@2@$0A@@std@@@2@PAU342@@Z 100095d0 f i ambientsnd.obj
 0001:000085f0       ?_Min@?$_Tree@V?$_Tmap_traits@HHU?$less@H@std@@V?$allocator@U?$pair@$$CBHH@std@@@2@$0A@@std@@@std@@KAPAU_Node@?$_Tree_nod@V?$_Tmap_traits@HHU?$less@H@std@@V?$allocator@U?$pair@$$CBHH@std@@@2@$0A@@std@@@2@PAU342@@Z 100095f0 f i ambientsnd.obj
 0001:00008610       ?max_size@?$allocator@U?$pair@$$CBHH@std@@@std@@QBEIXZ 10009610 f i ambientsnd.obj
 0001:00008620       ?_Max@?$_Tree@V?$_Tmap_traits@HUAmbientSnd@@U?$less@H@std@@V?$allocator@U?$pair@$$CBHUAmbientSnd@@@std@@@3@$0A@@std@@@std@@KAPAU_Node@?$_Tree_nod@V?$_Tmap_traits@HUAmbientSnd@@U?$less@H@std@@V?$allocator@U?$pair@$$CBHUAmbientSnd@@@std@@@3@$0A@@std@@@2@PAU342@@Z 10009620 f i ambientsnd.obj
 0001:00008640       ?_Min@?$_Tree@V?$_Tmap_traits@HUAmbientSnd@@U?$less@H@std@@V?$allocator@U?$pair@$$CBHUAmbientSnd@@@std@@@3@$0A@@std@@@std@@KAPAU_Node@?$_Tree_nod@V?$_Tmap_traits@HUAmbientSnd@@U?$less@H@std@@V?$allocator@U?$pair@$$CBHUAmbientSnd@@@std@@@3@$0A@@std@@@2@PAU342@@Z 10009640 f i ambientsnd.obj
 0001:00008660       ?max_size@?$allocator@U?$pair@$$CBHUAmbientSnd@@@std@@@std@@QBEIXZ 10009660 f i ambientsnd.obj
 0001:00008670       ?deallocate@?$allocator@U_Node@?$_Tree_nod@V?$_Tmap_traits@HUAmbientSnd@@U?$less@H@std@@V?$allocator@U?$pair@$$CBHUAmbientSnd@@@std@@@3@$0A@@std@@@std@@@std@@QAEXPAU_Node@?$_Tree_nod@V?$_Tmap_traits@HUAmbientSnd@@U?$less@H@std@@V?$allocator@U?$pair@$$CBHUAmbientSnd@@@std@@@3@$0A@@std@@@2@I@Z 10009670 f i ambientsnd.obj
 0001:00008680       ??0_Node@?$_Tree_nod@V?$_Tmap_traits@HHU?$less@H@std@@V?$allocator@U?$pair@$$CBHH@std@@@2@$0A@@std@@@std@@QAE@PAU012@00ABU?$pair@$$CBHH@2@D@Z 10009680 f i ambientsnd.obj
 0001:000086c0       ??0_Node@?$_Tree_nod@V?$_Tmap_traits@HUAmbientSnd@@U?$less@H@std@@V?$allocator@U?$pair@$$CBHUAmbientSnd@@@std@@@3@$0A@@std@@@std@@QAE@PAU012@00ABU?$pair@$$CBHUAmbientSnd@@@2@D@Z 100096c0 f i ambientsnd.obj
 0001:00008700       ??$_Destroy@PAU_Node@?$_Tree_nod@V?$_Tmap_traits@HHU?$less@H@std@@V?$allocator@U?$pair@$$CBHH@std@@@2@$0A@@std@@@std@@@std@@YAXPAPAU_Node@?$_Tree_nod@V?$_Tmap_traits@HHU?$less@H@std@@V?$allocator@U?$pair@$$CBHH@std@@@2@$0A@@std@@@0@@Z 10009700 f i ambientsnd.obj
 0001:00008710       ??$?0U?$pair@$$CBHH@std@@@?$allocator@PAU_Node@?$_Tree_nod@V?$_Tmap_traits@HHU?$less@H@std@@V?$allocator@U?$pair@$$CBHH@std@@@2@$0A@@std@@@std@@@std@@QAE@ABV?$allocator@U?$pair@$$CBHH@std@@@1@@Z 10009710 f i ambientsnd.obj
 0001:00008720       ??$?0U?$pair@$$CBHH@std@@@?$allocator@U_Node@?$_Tree_nod@V?$_Tmap_traits@HHU?$less@H@std@@V?$allocator@U?$pair@$$CBHH@std@@@2@$0A@@std@@@std@@@std@@QAE@ABV?$allocator@U?$pair@$$CBHH@std@@@1@@Z 10009720 f i ambientsnd.obj
 0001:00008730       ??$_Allocate@U_Node@?$_Tree_nod@V?$_Tmap_traits@HHU?$less@H@std@@V?$allocator@U?$pair@$$CBHH@std@@@2@$0A@@std@@@std@@@std@@YAPAU_Node@?$_Tree_nod@V?$_Tmap_traits@HHU?$less@H@std@@V?$allocator@U?$pair@$$CBHH@std@@@2@$0A@@std@@@0@IPAU120@@Z 10009730 f i ambientsnd.obj
 0001:00008790       ??$_Destroy@U_Node@?$_Tree_nod@V?$_Tmap_traits@HHU?$less@H@std@@V?$allocator@U?$pair@$$CBHH@std@@@2@$0A@@std@@@std@@@std@@YAXPAU_Node@?$_Tree_nod@V?$_Tmap_traits@HHU?$less@H@std@@V?$allocator@U?$pair@$$CBHH@std@@@2@$0A@@std@@@0@@Z 10009790 f i ambientsnd.obj
 0001:000087a0       ??$_Construct@PAU_Node@?$_Tree_nod@V?$_Tmap_traits@HHU?$less@H@std@@V?$allocator@U?$pair@$$CBHH@std@@@2@$0A@@std@@@std@@PAU123@@std@@YAXPAPAU_Node@?$_Tree_nod@V?$_Tmap_traits@HHU?$less@H@std@@V?$allocator@U?$pair@$$CBHH@std@@@2@$0A@@std@@@0@ABQAU120@@Z 100097a0 f i ambientsnd.obj
 0001:000087c0       ??$_Allocate@U_Node@?$_Tree_nod@V?$_Tmap_traits@HUAmbientSnd@@U?$less@H@std@@V?$allocator@U?$pair@$$CBHUAmbientSnd@@@std@@@3@$0A@@std@@@std@@@std@@YAPAU_Node@?$_Tree_nod@V?$_Tmap_traits@HUAmbientSnd@@U?$less@H@std@@V?$allocator@U?$pair@$$CBHUAmbientSnd@@@std@@@3@$0A@@std@@@0@IPAU120@@Z 100097c0 f i ambientsnd.obj
 0001:00008820       ??$?0U?$pair@$$CBHH@std@@@?$allocator@V_Aux_cont@std@@@std@@QAE@ABV?$allocator@U?$pair@$$CBHH@std@@@1@@Z 10009820 f i ambientsnd.obj
 0001:00008830       ?_Key@?$_Tree@V?$_Tmap_traits@HHU?$less@H@std@@V?$allocator@U?$pair@$$CBHH@std@@@2@$0A@@std@@@std@@KAABHPAU_Node@?$_Tree_nod@V?$_Tmap_traits@HHU?$less@H@std@@V?$allocator@U?$pair@$$CBHH@std@@@2@$0A@@std@@@2@@Z 10009830 f i ambientsnd.obj
 0001:00008840       ??1?$_Container_base_aux_alloc_real@V?$allocator@U?$pair@$$CBHH@std@@@std@@@std@@IAE@XZ 10009840 f i ambientsnd.obj
 0001:00008850       ?_Key@?$_Tree@V?$_Tmap_traits@HUAmbientSnd@@U?$less@H@std@@V?$allocator@U?$pair@$$CBHUAmbientSnd@@@std@@@3@$0A@@std@@@std@@KAABHPAU_Node@?$_Tree_nod@V?$_Tmap_traits@HUAmbientSnd@@U?$less@H@std@@V?$allocator@U?$pair@$$CBHUAmbientSnd@@@std@@@3@$0A@@std@@@2@@Z 10009850 f i ambientsnd.obj
 0001:00008860       ??Diterator@?$_Tree@V?$_Tmap_traits@HHU?$less@H@std@@V?$allocator@U?$pair@$$CBHH@std@@@2@$0A@@std@@@std@@QBEAAU?$pair@$$CBHH@2@XZ 10009860 f i ambientsnd.obj
 0001:00008890       ??Diterator@?$_Tree@V?$_Tmap_traits@HUAmbientSnd@@U?$less@H@std@@V?$allocator@U?$pair@$$CBHUAmbientSnd@@@std@@@3@$0A@@std@@@std@@QBEAAU?$pair@$$CBHUAmbientSnd@@@2@XZ 10009890 f i ambientsnd.obj
 0001:000088c0       ?_Lbound@?$_Tree@V?$_Tmap_traits@HHU?$less@H@std@@V?$allocator@U?$pair@$$CBHH@std@@@2@$0A@@std@@@std@@IBEPAU_Node@?$_Tree_nod@V?$_Tmap_traits@HHU?$less@H@std@@V?$allocator@U?$pair@$$CBHH@std@@@2@$0A@@std@@@2@ABH@Z 100098c0 f i ambientsnd.obj
 0001:000088f0       ?destroy@?$allocator@PAU_Node@?$_Tree_nod@V?$_Tmap_traits@HHU?$less@H@std@@V?$allocator@U?$pair@$$CBHH@std@@@2@$0A@@std@@@std@@@std@@QAEXPAPAU_Node@?$_Tree_nod@V?$_Tmap_traits@HHU?$less@H@std@@V?$allocator@U?$pair@$$CBHH@std@@@2@$0A@@std@@@2@@Z 100098f0 f i ambientsnd.obj
 0001:00008900       ?_Lbound@?$_Tree@V?$_Tmap_traits@HUAmbientSnd@@U?$less@H@std@@V?$allocator@U?$pair@$$CBHUAmbientSnd@@@std@@@3@$0A@@std@@@std@@IBEPAU_Node@?$_Tree_nod@V?$_Tmap_traits@HUAmbientSnd@@U?$less@H@std@@V?$allocator@U?$pair@$$CBHUAmbientSnd@@@std@@@3@$0A@@std@@@2@ABH@Z 10009900 f i ambientsnd.obj
 0001:00008930       ??0?$_Bidit@U?$pair@$$CBHH@std@@HPBU12@ABU12@@std@@QAE@XZ 10009930 f i ambientsnd.obj
 0001:00008940       ??0?$_Bidit@U?$pair@$$CBHUAmbientSnd@@@std@@HPBU12@ABU12@@std@@QAE@XZ 10009940 f i ambientsnd.obj
 0001:00008950       ?max_size@?$_Tree@V?$_Tmap_traits@HHU?$less@H@std@@V?$allocator@U?$pair@$$CBHH@std@@@2@$0A@@std@@@std@@QBEIXZ 10009950 f i ambientsnd.obj
 0001:00008960       ?_Lrotate@?$_Tree@V?$_Tmap_traits@HHU?$less@H@std@@V?$allocator@U?$pair@$$CBHH@std@@@2@$0A@@std@@@std@@IAEXPAU_Node@?$_Tree_nod@V?$_Tmap_traits@HHU?$less@H@std@@V?$allocator@U?$pair@$$CBHH@std@@@2@$0A@@std@@@2@@Z 10009960 f i ambientsnd.obj
 0001:000089b0       ?max_size@?$_Tree@V?$_Tmap_traits@HUAmbientSnd@@U?$less@H@std@@V?$allocator@U?$pair@$$CBHUAmbientSnd@@@std@@@3@$0A@@std@@@std@@QBEIXZ 100099b0 f i ambientsnd.obj
 0001:000089c0       ?_Lrotate@?$_Tree@V?$_Tmap_traits@HUAmbientSnd@@U?$less@H@std@@V?$allocator@U?$pair@$$CBHUAmbientSnd@@@std@@@3@$0A@@std@@@std@@IAEXPAU_Node@?$_Tree_nod@V?$_Tmap_traits@HUAmbientSnd@@U?$less@H@std@@V?$allocator@U?$pair@$$CBHUAmbientSnd@@@std@@@3@$0A@@std@@@2@@Z 100099c0 f i ambientsnd.obj
 0001:00008a20       ?_Dec@const_iterator@?$_Tree@V?$_Tmap_traits@HHU?$less@H@std@@V?$allocator@U?$pair@$$CBHH@std@@@2@$0A@@std@@@std@@QAEXXZ 10009a20 f i ambientsnd.obj
 0001:00008ab0       ?_Inc@const_iterator@?$_Tree@V?$_Tmap_traits@HHU?$less@H@std@@V?$allocator@U?$pair@$$CBHH@std@@@2@$0A@@std@@@std@@QAEXXZ 10009ab0 f i ambientsnd.obj
 0001:00008b20       ?_Dec@const_iterator@?$_Tree@V?$_Tmap_traits@HUAmbientSnd@@U?$less@H@std@@V?$allocator@U?$pair@$$CBHUAmbientSnd@@@std@@@3@$0A@@std@@@std@@QAEXXZ 10009b20 f i ambientsnd.obj
 0001:00008bc0       ?_Inc@const_iterator@?$_Tree@V?$_Tmap_traits@HUAmbientSnd@@U?$less@H@std@@V?$allocator@U?$pair@$$CBHUAmbientSnd@@@std@@@3@$0A@@std@@@std@@QAEXXZ 10009bc0 f i ambientsnd.obj
 0001:00008c40       ?allocate@?$allocator@U_Node@?$_Tree_nod@V?$_Tmap_traits@HHU?$less@H@std@@V?$allocator@U?$pair@$$CBHH@std@@@2@$0A@@std@@@std@@@std@@QAEPAU_Node@?$_Tree_nod@V?$_Tmap_traits@HHU?$less@H@std@@V?$allocator@U?$pair@$$CBHH@std@@@2@$0A@@std@@@2@I@Z 10009c40 f i ambientsnd.obj
 0001:00008c60       ?destroy@?$allocator@U_Node@?$_Tree_nod@V?$_Tmap_traits@HHU?$less@H@std@@V?$allocator@U?$pair@$$CBHH@std@@@2@$0A@@std@@@std@@@std@@QAEXPAU_Node@?$_Tree_nod@V?$_Tmap_traits@HHU?$less@H@std@@V?$allocator@U?$pair@$$CBHH@std@@@2@$0A@@std@@@2@@Z 10009c60 f i ambientsnd.obj
 0001:00008c70       ?construct@?$allocator@PAU_Node@?$_Tree_nod@V?$_Tmap_traits@HHU?$less@H@std@@V?$allocator@U?$pair@$$CBHH@std@@@2@$0A@@std@@@std@@@std@@QAEXPAPAU_Node@?$_Tree_nod@V?$_Tmap_traits@HHU?$less@H@std@@V?$allocator@U?$pair@$$CBHH@std@@@2@$0A@@std@@@2@ABQAU342@@Z 10009c70 f i ambientsnd.obj
 0001:00008c90       ?allocate@?$allocator@U_Node@?$_Tree_nod@V?$_Tmap_traits@HUAmbientSnd@@U?$less@H@std@@V?$allocator@U?$pair@$$CBHUAmbientSnd@@@std@@@3@$0A@@std@@@std@@@std@@QAEPAU_Node@?$_Tree_nod@V?$_Tmap_traits@HUAmbientSnd@@U?$less@H@std@@V?$allocator@U?$pair@$$CBHUAmbientSnd@@@std@@@3@$0A@@std@@@2@I@Z 10009c90 f i ambientsnd.obj
 0001:00008cb0       ??Citerator@?$_Tree@V?$_Tmap_traits@HHU?$less@H@std@@V?$allocator@U?$pair@$$CBHH@std@@@2@$0A@@std@@@std@@QBEPAU?$pair@$$CBHH@2@XZ 10009cb0 f i ambientsnd.obj
 0001:00008ce0       ??Citerator@?$_Tree@V?$_Tmap_traits@HUAmbientSnd@@U?$less@H@std@@V?$allocator@U?$pair@$$CBHUAmbientSnd@@@std@@@3@$0A@@std@@@std@@QBEPAU?$pair@$$CBHUAmbientSnd@@@2@XZ 10009ce0 f i ambientsnd.obj
 0001:00008d10       ??1?$_Tmap_traits@HHU?$less@H@std@@V?$allocator@U?$pair@$$CBHH@std@@@2@$0A@@std@@QAE@XZ 10009d10 f i ambientsnd.obj
 0001:00008d20       ??0const_iterator@?$_Tree@V?$_Tmap_traits@HHU?$less@H@std@@V?$allocator@U?$pair@$$CBHH@std@@@2@$0A@@std@@@std@@QAE@XZ 10009d20 f i ambientsnd.obj
 0001:00008d30       ??0const_iterator@?$_Tree@V?$_Tmap_traits@HHU?$less@H@std@@V?$allocator@U?$pair@$$CBHH@std@@@2@$0A@@std@@@std@@QAE@PAU_Node@?$_Tree_nod@V?$_Tmap_traits@HHU?$less@H@std@@V?$allocator@U?$pair@$$CBHH@std@@@2@$0A@@std@@@2@PBV12@@Z 10009d30 f i ambientsnd.obj
 0001:00008d60       ??Econst_iterator@?$_Tree@V?$_Tmap_traits@HHU?$less@H@std@@V?$allocator@U?$pair@$$CBHH@std@@@2@$0A@@std@@@std@@QAEAAV012@XZ 10009d60 f i ambientsnd.obj
 0001:00008d70       ??Fconst_iterator@?$_Tree@V?$_Tmap_traits@HHU?$less@H@std@@V?$allocator@U?$pair@$$CBHH@std@@@2@$0A@@std@@@std@@QAEAAV012@XZ 10009d70 f i ambientsnd.obj
 0001:00008d80       ??0const_iterator@?$_Tree@V?$_Tmap_traits@HUAmbientSnd@@U?$less@H@std@@V?$allocator@U?$pair@$$CBHUAmbientSnd@@@std@@@3@$0A@@std@@@std@@QAE@XZ 10009d80 f i ambientsnd.obj
 0001:00008d90       ??0const_iterator@?$_Tree@V?$_Tmap_traits@HUAmbientSnd@@U?$less@H@std@@V?$allocator@U?$pair@$$CBHUAmbientSnd@@@std@@@3@$0A@@std@@@std@@QAE@PAU_Node@?$_Tree_nod@V?$_Tmap_traits@HUAmbientSnd@@U?$less@H@std@@V?$allocator@U?$pair@$$CBHUAmbientSnd@@@std@@@3@$0A@@std@@@2@PBV12@@Z 10009d90 f i ambientsnd.obj
 0001:00008dc0       ??Econst_iterator@?$_Tree@V?$_Tmap_traits@HUAmbientSnd@@U?$less@H@std@@V?$allocator@U?$pair@$$CBHUAmbientSnd@@@std@@@3@$0A@@std@@@std@@QAEAAV012@XZ 10009dc0 f i ambientsnd.obj
 0001:00008dd0       ??Fconst_iterator@?$_Tree@V?$_Tmap_traits@HUAmbientSnd@@U?$less@H@std@@V?$allocator@U?$pair@$$CBHUAmbientSnd@@@std@@@3@$0A@@std@@@std@@QAEAAV012@XZ 10009dd0 f i ambientsnd.obj
 0001:00008de0       ?_Buynode@?$_Tree@V?$_Tmap_traits@HHU?$less@H@std@@V?$allocator@U?$pair@$$CBHH@std@@@2@$0A@@std@@@std@@IAEPAU_Node@?$_Tree_nod@V?$_Tmap_traits@HHU?$less@H@std@@V?$allocator@U?$pair@$$CBHH@std@@@2@$0A@@std@@@2@XZ 10009de0 f i ambientsnd.obj
 0001:00008e20       ?_Buynode@?$_Tree@V?$_Tmap_traits@HHU?$less@H@std@@V?$allocator@U?$pair@$$CBHH@std@@@2@$0A@@std@@@std@@IAEPAU_Node@?$_Tree_nod@V?$_Tmap_traits@HHU?$less@H@std@@V?$allocator@U?$pair@$$CBHH@std@@@2@$0A@@std@@@2@PAU342@00ABU?$pair@$$CBHH@2@D@Z 10009e20 f i ambientsnd.obj
 0001:00008e60       ?_Buynode@?$_Tree@V?$_Tmap_traits@HUAmbientSnd@@U?$less@H@std@@V?$allocator@U?$pair@$$CBHUAmbientSnd@@@std@@@3@$0A@@std@@@std@@IAEPAU_Node@?$_Tree_nod@V?$_Tmap_traits@HUAmbientSnd@@U?$less@H@std@@V?$allocator@U?$pair@$$CBHUAmbientSnd@@@std@@@3@$0A@@std@@@2@PAU342@00ABU?$pair@$$CBHUAmbientSnd@@@2@D@Z 10009e60 f i ambientsnd.obj
 0001:00008eb0       ??Fiterator@?$_Tree@V?$_Tmap_traits@HHU?$less@H@std@@V?$allocator@U?$pair@$$CBHH@std@@@2@$0A@@std@@@std@@QAEAAV012@XZ 10009eb0 f i ambientsnd.obj
 0001:00008ec0       ??Econst_iterator@?$_Tree@V?$_Tmap_traits@HHU?$less@H@std@@V?$allocator@U?$pair@$$CBHH@std@@@2@$0A@@std@@@std@@QAE?AV012@H@Z 10009ec0 f i ambientsnd.obj
 0001:00008ee0       ??Fiterator@?$_Tree@V?$_Tmap_traits@HUAmbientSnd@@U?$less@H@std@@V?$allocator@U?$pair@$$CBHUAmbientSnd@@@std@@@3@$0A@@std@@@std@@QAEAAV012@XZ 10009ee0 f i ambientsnd.obj
 0001:00008ef0       ?_Erase@?$_Tree@V?$_Tmap_traits@HHU?$less@H@std@@V?$allocator@U?$pair@$$CBHH@std@@@2@$0A@@std@@@std@@IAEXPAU_Node@?$_Tree_nod@V?$_Tmap_traits@HHU?$less@H@std@@V?$allocator@U?$pair@$$CBHH@std@@@2@$0A@@std@@@2@@Z 10009ef0 f i ambientsnd.obj
 0001:00008f30       ??0?$_Container_base_aux_alloc_real@V?$allocator@U?$pair@$$CBHH@std@@@std@@@std@@IAE@V?$allocator@U?$pair@$$CBHH@std@@@1@@Z 10009f30 f i ambientsnd.obj
 0001:00008f60       ??1?$_Tree_nod@V?$_Tmap_traits@HHU?$less@H@std@@V?$allocator@U?$pair@$$CBHH@std@@@2@$0A@@std@@@std@@QAE@XZ 10009f60 f i ambientsnd.obj
 0001:00008f70       ??0iterator@?$_Tree@V?$_Tmap_traits@HHU?$less@H@std@@V?$allocator@U?$pair@$$CBHH@std@@@2@$0A@@std@@@std@@QAE@PAU_Node@?$_Tree_nod@V?$_Tmap_traits@HHU?$less@H@std@@V?$allocator@U?$pair@$$CBHH@std@@@2@$0A@@std@@@2@PBV12@@Z 10009f70 f i ambientsnd.obj
 0001:00008fa0       ??0iterator@?$_Tree@V?$_Tmap_traits@HUAmbientSnd@@U?$less@H@std@@V?$allocator@U?$pair@$$CBHUAmbientSnd@@@std@@@3@$0A@@std@@@std@@QAE@PAU_Node@?$_Tree_nod@V?$_Tmap_traits@HUAmbientSnd@@U?$less@H@std@@V?$allocator@U?$pair@$$CBHUAmbientSnd@@@std@@@3@$0A@@std@@@2@PBV12@@Z 10009fa0 f i ambientsnd.obj
 0001:00008fd0       ?begin@?$_Tree@V?$_Tmap_traits@HHU?$less@H@std@@V?$allocator@U?$pair@$$CBHH@std@@@2@$0A@@std@@@std@@QAE?AViterator@12@XZ 10009fd0 f i ambientsnd.obj
 0001:00008ff0       ?_Init@?$_Tree@V?$_Tmap_traits@HHU?$less@H@std@@V?$allocator@U?$pair@$$CBHH@std@@@2@$0A@@std@@@std@@IAEXXZ 10009ff0 f i ambientsnd.obj
 0001:00009020       ?begin@?$_Tree@V?$_Tmap_traits@HUAmbientSnd@@U?$less@H@std@@V?$allocator@U?$pair@$$CBHUAmbientSnd@@@std@@@3@$0A@@std@@@std@@QAE?AViterator@12@XZ 1000a020 f i ambientsnd.obj
 0001:00009040       ?_Make_iter@?$_Tree@V?$_Tmap_traits@HHU?$less@H@std@@V?$allocator@U?$pair@$$CBHH@std@@@2@$0A@@std@@@std@@QBE?AViterator@12@Vconst_iterator@12@@Z 1000a040 f i ambientsnd.obj
 0001:00009070       ?clear@?$_Tree@V?$_Tmap_traits@HHU?$less@H@std@@V?$allocator@U?$pair@$$CBHH@std@@@2@$0A@@std@@@std@@QAEXXZ 1000a070 f i ambientsnd.obj
 0001:000090a0       ??0?$_Tmap_traits@HHU?$less@H@std@@V?$allocator@U?$pair@$$CBHH@std@@@2@$0A@@std@@QAE@U?$less@H@1@V?$allocator@U?$pair@$$CBHH@std@@@1@@Z 1000a0a0 f i ambientsnd.obj
 0001:000090d0       ?end@?$_Tree@V?$_Tmap_traits@HHU?$less@H@std@@V?$allocator@U?$pair@$$CBHH@std@@@2@$0A@@std@@@std@@QAE?AViterator@12@XZ 1000a0d0 f i ambientsnd.obj
 0001:000090f0       ?end@?$_Tree@V?$_Tmap_traits@HUAmbientSnd@@U?$less@H@std@@V?$allocator@U?$pair@$$CBHUAmbientSnd@@@std@@@3@$0A@@std@@@std@@QAE?AViterator@12@XZ 1000a0f0 f i ambientsnd.obj
 0001:00009110       ??1?$_Tree_ptr@V?$_Tmap_traits@HHU?$less@H@std@@V?$allocator@U?$pair@$$CBHH@std@@@2@$0A@@std@@@std@@QAE@XZ 1000a110 f i ambientsnd.obj
 0001:00009120       ?lower_bound@?$_Tree@V?$_Tmap_traits@HHU?$less@H@std@@V?$allocator@U?$pair@$$CBHH@std@@@2@$0A@@std@@@std@@QAE?AViterator@12@ABH@Z 1000a120 f i ambientsnd.obj
 0001:00009160       ?lower_bound@?$_Tree@V?$_Tmap_traits@HUAmbientSnd@@U?$less@H@std@@V?$allocator@U?$pair@$$CBHUAmbientSnd@@@std@@@3@$0A@@std@@@std@@QAE?AViterator@12@ABH@Z 1000a160 f i ambientsnd.obj
 0001:000091a0       ??0?$_Tree_nod@V?$_Tmap_traits@HHU?$less@H@std@@V?$allocator@U?$pair@$$CBHH@std@@@2@$0A@@std@@@std@@IAE@ABU?$less@H@1@V?$allocator@U?$pair@$$CBHH@std@@@1@@Z 1000a1a0 f i ambientsnd.obj
 0001:000091d0       ?find@?$_Tree@V?$_Tmap_traits@HHU?$less@H@std@@V?$allocator@U?$pair@$$CBHH@std@@@2@$0A@@std@@@std@@QAE?AViterator@12@ABH@Z 1000a1d0 f i ambientsnd.obj
 0001:00009260       ?find@?$_Tree@V?$_Tmap_traits@HUAmbientSnd@@U?$less@H@std@@V?$allocator@U?$pair@$$CBHUAmbientSnd@@@std@@@3@$0A@@std@@@std@@QAE?AViterator@12@ABH@Z 1000a260 f i ambientsnd.obj
 0001:000092d0       ??1?$_Tree_val@V?$_Tmap_traits@HHU?$less@H@std@@V?$allocator@U?$pair@$$CBHH@std@@@2@$0A@@std@@@std@@QAE@XZ 1000a2d0 f i ambientsnd.obj
 0001:000092e0       ??0?$_Tree_ptr@V?$_Tmap_traits@HHU?$less@H@std@@V?$allocator@U?$pair@$$CBHH@std@@@2@$0A@@std@@@std@@IAE@ABU?$less@H@1@V?$allocator@U?$pair@$$CBHH@std@@@1@@Z 1000a2e0 f i ambientsnd.obj
 0001:00009380       ?ambi_pause@@YAXH@Z        1000a380 f   ambientsnd.obj
 0001:000093a0       ?ambi_unpause@@YAXH@Z      1000a3a0 f   ambientsnd.obj
 0001:000093c0       ?ambi_set_volume@@YAXHM@Z  1000a3c0 f   ambientsnd.obj
 0001:00009460       ?ambi_set_loop@@YAXHH@Z    1000a460 f   ambientsnd.obj
 0001:00009490       ?ambi_state@@YAHH@Z        1000a490 f   ambientsnd.obj
 0001:000094d0       ??0?$_Tree_val@V?$_Tmap_traits@HHU?$less@H@std@@V?$allocator@U?$pair@$$CBHH@std@@@2@$0A@@std@@@std@@IAE@ABU?$less@H@1@V?$allocator@U?$pair@$$CBHH@std@@@1@@Z 1000a4d0 f i ambientsnd.obj
 0001:00009500       ?erase@?$_Tree@V?$_Tmap_traits@HHU?$less@H@std@@V?$allocator@U?$pair@$$CBHH@std@@@2@$0A@@std@@@std@@QAE?AViterator@12@Vconst_iterator@12@@Z 1000a500 f i ambientsnd.obj
 0001:000097d0       ??0?$_Tree@V?$_Tmap_traits@HHU?$less@H@std@@V?$allocator@U?$pair@$$CBHH@std@@@2@$0A@@std@@@std@@QAE@ABU?$less@H@1@ABV?$allocator@U?$pair@$$CBHH@std@@@1@@Z 1000a7d0 f i ambientsnd.obj
 0001:00009860       ?erase@?$_Tree@V?$_Tmap_traits@HHU?$less@H@std@@V?$allocator@U?$pair@$$CBHH@std@@@2@$0A@@std@@@std@@QAE?AViterator@12@Vconst_iterator@12@0@Z 1000a860 f i ambientsnd.obj
 0001:00009940       ?_Insert@?$_Tree@V?$_Tmap_traits@HHU?$less@H@std@@V?$allocator@U?$pair@$$CBHH@std@@@2@$0A@@std@@@std@@IAE?AViterator@12@_NPAU_Node@?$_Tree_nod@V?$_Tmap_traits@HHU?$less@H@std@@V?$allocator@U?$pair@$$CBHH@std@@@2@$0A@@std@@@2@ABU?$pair@$$CBHH@2@@Z 1000a940 f i ambientsnd.obj
 0001:00009b40       ?_Insert@?$_Tree@V?$_Tmap_traits@HUAmbientSnd@@U?$less@H@std@@V?$allocator@U?$pair@$$CBHUAmbientSnd@@@std@@@3@$0A@@std@@@std@@IAE?AViterator@12@_NPAU_Node@?$_Tree_nod@V?$_Tmap_traits@HUAmbientSnd@@U?$less@H@std@@V?$allocator@U?$pair@$$CBHUAmbientSnd@@@std@@@3@$0A@@std@@@2@ABU?$pair@$$CBHUAmbientSnd@@@2@@Z 1000ab40 f i ambientsnd.obj
 0001:00009d50       ?_Tidy@?$_Tree@V?$_Tmap_traits@HHU?$less@H@std@@V?$allocator@U?$pair@$$CBHH@std@@@2@$0A@@std@@@std@@IAEXXZ 1000ad50 f i ambientsnd.obj
 0001:00009d90       ?insert@?$_Tree@V?$_Tmap_traits@HHU?$less@H@std@@V?$allocator@U?$pair@$$CBHH@std@@@2@$0A@@std@@@std@@QAE?AU?$pair@Viterator@?$_Tree@V?$_Tmap_traits@HHU?$less@H@std@@V?$allocator@U?$pair@$$CBHH@std@@@2@$0A@@std@@@std@@_N@2@ABU?$pair@$$CBHH@2@@Z 1000ad90 f i ambientsnd.obj
 0001:00009e80       ?insert@?$_Tree@V?$_Tmap_traits@HUAmbientSnd@@U?$less@H@std@@V?$allocator@U?$pair@$$CBHUAmbientSnd@@@std@@@3@$0A@@std@@@std@@QAE?AU?$pair@Viterator@?$_Tree@V?$_Tmap_traits@HUAmbientSnd@@U?$less@H@std@@V?$allocator@U?$pair@$$CBHUAmbientSnd@@@std@@@3@$0A@@std@@@std@@_N@2@ABU?$pair@$$CBHUAmbientSnd@@@2@@Z 1000ae80 f i ambientsnd.obj
 0001:00009f80       ??1?$_Tree@V?$_Tmap_traits@HHU?$less@H@std@@V?$allocator@U?$pair@$$CBHH@std@@@2@$0A@@std@@@std@@QAE@XZ 1000af80 f i ambientsnd.obj
 0001:0000a000       ?insert@?$_Tree@V?$_Tmap_traits@HHU?$less@H@std@@V?$allocator@U?$pair@$$CBHH@std@@@2@$0A@@std@@@std@@QAE?AViterator@12@Vconst_iterator@12@ABU?$pair@$$CBHH@2@@Z 1000b000 f i ambientsnd.obj
 0001:0000a1d0       ?insert@?$_Tree@V?$_Tmap_traits@HUAmbientSnd@@U?$less@H@std@@V?$allocator@U?$pair@$$CBHUAmbientSnd@@@std@@@3@$0A@@std@@@std@@QAE?AViterator@12@Vconst_iterator@12@ABU?$pair@$$CBHUAmbientSnd@@@2@@Z 1000b1d0 f i ambientsnd.obj
 0001:0000a3b0       ??1?$map@HHU?$less@H@std@@V?$allocator@U?$pair@$$CBHH@std@@@2@@std@@QAE@XZ 1000b3b0 f i ambientsnd.obj
 0001:0000a3c0       ??0?$map@HHU?$less@H@std@@V?$allocator@U?$pair@$$CBHH@std@@@2@@std@@QAE@XZ 1000b3c0 f i ambientsnd.obj
 0001:0000a3e0       ??A?$map@HHU?$less@H@std@@V?$allocator@U?$pair@$$CBHH@std@@@2@@std@@QAEAAHABH@Z 1000b3e0 f i ambientsnd.obj
 0001:0000a490       ??A?$map@HUAmbientSnd@@U?$less@H@std@@V?$allocator@U?$pair@$$CBHUAmbientSnd@@@std@@@3@@std@@QAEAAUAmbientSnd@@ABH@Z 1000b490 f i ambientsnd.obj
 0001:0000a560       ?ambi_start@@YAHHHHMHH@Z   1000b560 f   ambientsnd.obj
 0001:0000a670       ?ambi_stop@@YAXHH@Z        1000b670 f   ambientsnd.obj
 0001:0000a6c0       ?event_music_init@@YAHXZ   1000b6c0 f   eventmusic.obj
 0001:0000a6d0       ?event_music_close@@YAXXZ  1000b6d0 f   eventmusic.obj
 0001:0000a6e0       ?event_music_stop_all@@YAXH@Z 1000b6e0 f   eventmusic.obj
 0001:0000a6f0       ?event_music_pause_all@@YAXXZ 1000b6f0 f   eventmusic.obj
 0001:0000a700       ?event_music_unpause_all@@YAXXZ 1000b700 f   eventmusic.obj
 0001:0000a710       ?event_music_set_volume_all@@YAXM@Z 1000b710 f   eventmusic.obj
 0001:0000a7a0       ?event_music_stop@@YAXHH@Z 1000b7a0 f   eventmusic.obj
 0001:0000a7f0       ?event_music_pause@@YAXH@Z 1000b7f0 f   eventmusic.obj
 0001:0000a810       ?event_music_unpause@@YAXH@Z 1000b810 f   eventmusic.obj
 0001:0000a830       ?event_music_set_volume@@YAXHM@Z 1000b830 f   eventmusic.obj
 0001:0000a860       ?event_music_set_loop@@YAXHH@Z 1000b860 f   eventmusic.obj
 0001:0000a890       ?event_music_state@@YAHH@Z 1000b890 f   eventmusic.obj
 0001:0000a8d0       ?event_music_start@@YAHHMH@Z 1000b8d0 f   eventmusic.obj
 0001:0000a980       ?gamesnd_stop_iface@@YAXH@Z 1000b980 f   gamesnd.obj
 0001:0000a990       ?deallocate@?$allocator@U_Node@?$_Tree_nod@V?$_Tmap_traits@HUgame_snd@@U?$less@H@std@@V?$allocator@U?$pair@$$CBHUgame_snd@@@std@@@3@$0A@@std@@@std@@@std@@QAEXPAU_Node@?$_Tree_nod@V?$_Tmap_traits@HUgame_snd@@U?$less@H@std@@V?$allocator@U?$pair@$$CBHUgame_snd@@@std@@@3@$0A@@std@@@2@I@Z 1000b990 f i gamesnd.obj
 0001:0000a9a0       ?_Min@?$_Tree@V?$_Tmap_traits@HUgame_snd@@U?$less@H@std@@V?$allocator@U?$pair@$$CBHUgame_snd@@@std@@@3@$0A@@std@@@std@@KAPAU_Node@?$_Tree_nod@V?$_Tmap_traits@HUgame_snd@@U?$less@H@std@@V?$allocator@U?$pair@$$CBHUgame_snd@@@std@@@3@$0A@@std@@@2@PAU342@@Z 1000b9a0 f i gamesnd.obj
 0001:0000a9c0       ??$_Destroy@U_Node@?$_Tree_nod@V?$_Tmap_traits@HUgame_snd@@U?$less@H@std@@V?$allocator@U?$pair@$$CBHUgame_snd@@@std@@@3@$0A@@std@@@std@@@std@@YAXPAU_Node@?$_Tree_nod@V?$_Tmap_traits@HUgame_snd@@U?$less@H@std@@V?$allocator@U?$pair@$$CBHUgame_snd@@@std@@@3@$0A@@std@@@0@@Z 1000b9c0 f i gamesnd.obj
 0001:0000a9d0       ?_Lmost@?$_Tree@V?$_Tmap_traits@HUgame_snd@@U?$less@H@std@@V?$allocator@U?$pair@$$CBHUgame_snd@@@std@@@3@$0A@@std@@@std@@IBEAAPAU_Node@?$_Tree_nod@V?$_Tmap_traits@HUgame_snd@@U?$less@H@std@@V?$allocator@U?$pair@$$CBHUgame_snd@@@std@@@3@$0A@@std@@@2@XZ 1000b9d0 f i gamesnd.obj
 0001:0000a9e0       ?_Rmost@?$_Tree@V?$_Tmap_traits@HUgame_snd@@U?$less@H@std@@V?$allocator@U?$pair@$$CBHUgame_snd@@@std@@@3@$0A@@std@@@std@@IBEAAPAU_Node@?$_Tree_nod@V?$_Tmap_traits@HUgame_snd@@U?$less@H@std@@V?$allocator@U?$pair@$$CBHUgame_snd@@@std@@@3@$0A@@std@@@2@XZ 1000b9e0 f i gamesnd.obj
 0001:0000a9f0       ?destroy@?$allocator@U_Node@?$_Tree_nod@V?$_Tmap_traits@HUgame_snd@@U?$less@H@std@@V?$allocator@U?$pair@$$CBHUgame_snd@@@std@@@3@$0A@@std@@@std@@@std@@QAEXPAU_Node@?$_Tree_nod@V?$_Tmap_traits@HUgame_snd@@U?$less@H@std@@V?$allocator@U?$pair@$$CBHUgame_snd@@@std@@@3@$0A@@std@@@2@@Z 1000b9f0 f i gamesnd.obj
 0001:0000aa00       ?_Inc@const_iterator@?$_Tree@V?$_Tmap_traits@HUgame_snd@@U?$less@H@std@@V?$allocator@U?$pair@$$CBHUgame_snd@@@std@@@3@$0A@@std@@@std@@QAEXXZ 1000ba00 f i gamesnd.obj
 0001:0000aa80       ?_Erase@?$_Tree@V?$_Tmap_traits@HUgame_snd@@U?$less@H@std@@V?$allocator@U?$pair@$$CBHUgame_snd@@@std@@@3@$0A@@std@@@std@@IAEXPAU_Node@?$_Tree_nod@V?$_Tmap_traits@HUgame_snd@@U?$less@H@std@@V?$allocator@U?$pair@$$CBHUgame_snd@@@std@@@3@$0A@@std@@@2@@Z 1000ba80 f i gamesnd.obj
 0001:0000aac0       ??Econst_iterator@?$_Tree@V?$_Tmap_traits@HUgame_snd@@U?$less@H@std@@V?$allocator@U?$pair@$$CBHUgame_snd@@@std@@@3@$0A@@std@@@std@@QAEAAV012@XZ 1000bac0 f i gamesnd.obj
 0001:0000aad0       ?clear@?$_Tree@V?$_Tmap_traits@HUgame_snd@@U?$less@H@std@@V?$allocator@U?$pair@$$CBHUgame_snd@@@std@@@3@$0A@@std@@@std@@QAEXXZ 1000bad0 f i gamesnd.obj
 0001:0000ab00       ??Eiterator@?$_Tree@V?$_Tmap_traits@HUgame_snd@@U?$less@H@std@@V?$allocator@U?$pair@$$CBHUgame_snd@@@std@@@3@$0A@@std@@@std@@QAEAAV012@XZ 1000bb00 f i gamesnd.obj
 0001:0000ab10       ?gamesnd_init_sounds@@YAXXZ 1000bb10 f   gamesnd.obj
 0001:0000abb0       ?gamesnd_close@@YAXXZ      1000bbb0 f   gamesnd.obj
 0001:0000ac20       ?begin@?$_Tree@V?$_Tmap_traits@HUgame_snd@@U?$less@H@std@@V?$allocator@U?$pair@$$CBHUgame_snd@@@std@@@3@$0A@@std@@@std@@QAE?AViterator@12@XZ 1000bc20 f i gamesnd.obj
 0001:0000ac40       ?gamesnd_load_gameplay_sounds@@YAXXZ 1000bc40 f   gamesnd.obj
 0001:0000acc0       ?gamesnd_unload_gameplay_sounds@@YAXXZ 1000bcc0 f   gamesnd.obj
 0001:0000ad40       ?gamesnd_load_interface_sounds@@YAXXZ 1000bd40 f   gamesnd.obj
 0001:0000ade0       ?gamesnd_unload_interface_sounds@@YAXXZ 1000bde0 f   gamesnd.obj
 0001:0000ae60       ?gamesnd_play_iface@@YAHHM@Z 1000be60 f   gamesnd.obj
 0001:0000af00       ?compare@?$char_traits@D@std@@SAHPBD0I@Z 1000bf00 f i scriptparser.obj
 0001:0000afd0       ?gamesnd_parse_configtbl@@YAXPAD@Z 1000bfd0 f   scriptparser.obj
 0001:0000b1d0       ?empty@?$basic_string@DU?$char_traits@D@std@@V?$allocator@D@2@@std@@QBE_NXZ 1000c1d0 f i scriptparser.obj
 0001:0000b1e0       ?size@?$vector@V?$basic_string@DU?$char_traits@D@std@@V?$allocator@D@2@@std@@V?$allocator@V?$basic_string@DU?$char_traits@D@std@@V?$allocator@D@2@@std@@@2@@std@@QBEIXZ 1000c1e0 f i scriptparser.obj
 0001:0000b200       ??A?$vector@V?$basic_string@DU?$char_traits@D@std@@V?$allocator@D@2@@std@@V?$allocator@V?$basic_string@DU?$char_traits@D@std@@V?$allocator@D@2@@std@@@2@@std@@QAEAAV?$basic_string@DU?$char_traits@D@std@@V?$allocator@D@2@@1@I@Z 1000c200 f i scriptparser.obj
 0001:0000b240       ?size@?$vector@UST_CELLS@@V?$allocator@UST_CELLS@@@std@@@std@@QBEIXZ 1000c240 f i scriptparser.obj
 0001:0000b260       ??A?$vector@UST_CELLS@@V?$allocator@UST_CELLS@@@std@@@std@@QAEAAUST_CELLS@@I@Z 1000c260 f i scriptparser.obj
 0001:0000b2a0       ??0?$pair@$$CBHUgame_snd@@@std@@QAE@ABHABUgame_snd@@@Z 1000c2a0 f i scriptparser.obj
 0001:0000b2c0       ??0?$allocator@U?$pair@$$CBHUgame_snd@@@std@@@std@@QAE@XZ 1000c2c0 f i scriptparser.obj
 0001:0000b2d0       ??0?$allocator@U?$pair@$$CBHUAmbientSnd@@@std@@@std@@QAE@XZ 1000c2d0 f i scriptparser.obj
 0001:0000b2e0       ??0?$allocator@U?$pair@$$CBHUVoiceSnd@@@std@@@std@@QAE@XZ 1000c2e0 f i scriptparser.obj
 0001:0000b2f0       ??0?$allocator@UST_CELLS@@@std@@QAE@XZ 1000c2f0 f i scriptparser.obj
 0001:0000b300       ??0?$pair@Viterator@?$_Tree@V?$_Tmap_traits@HUgame_snd@@U?$less@H@std@@V?$allocator@U?$pair@$$CBHUgame_snd@@@std@@@3@$0A@@std@@@std@@_N@std@@QAE@ABViterator@?$_Tree@V?$_Tmap_traits@HUgame_snd@@U?$less@H@std@@V?$allocator@U?$pair@$$CBHUgame_snd@@@std@@@3@$0A@@std@@@1@AB_N@Z 1000c300 f i scriptparser.obj
 0001:0000b320       ?_Color@?$_Tree@V?$_Tmap_traits@HUgame_snd@@U?$less@H@std@@V?$allocator@U?$pair@$$CBHUgame_snd@@@std@@@3@$0A@@std@@@std@@KAAADPAU_Node@?$_Tree_nod@V?$_Tmap_traits@HUgame_snd@@U?$less@H@std@@V?$allocator@U?$pair@$$CBHUgame_snd@@@std@@@3@$0A@@std@@@2@@Z 1000c320 f i scriptparser.obj
 0001:0000b330       ?size@?$_Tree@V?$_Tmap_traits@HUgame_snd@@U?$less@H@std@@V?$allocator@U?$pair@$$CBHUgame_snd@@@std@@@3@$0A@@std@@@std@@QBEIXZ 1000c330 f i scriptparser.obj
 0001:0000b340       ??0?$allocator@U?$pair@$$CBHUgame_snd@@@std@@@std@@QAE@ABV01@@Z 1000c340 f i scriptparser.obj
 0001:0000b350       ??0?$allocator@U?$pair@$$CBHUAmbientSnd@@@std@@@std@@QAE@ABV01@@Z 1000c350 f i scriptparser.obj
 0001:0000b360       ?_Left@?$_Tree@V?$_Tmap_traits@HUVoiceSnd@@U?$less@H@std@@V?$allocator@U?$pair@$$CBHUVoiceSnd@@@std@@@3@$0A@@std@@@std@@KAAAPAU_Node@?$_Tree_nod@V?$_Tmap_traits@HUVoiceSnd@@U?$less@H@std@@V?$allocator@U?$pair@$$CBHUVoiceSnd@@@std@@@3@$0A@@std@@@2@PAU342@@Z 1000c360 f i scriptparser.obj
 0001:0000b370       ?_Parent@?$_Tree@V?$_Tmap_traits@HUVoiceSnd@@U?$less@H@std@@V?$allocator@U?$pair@$$CBHUVoiceSnd@@@std@@@3@$0A@@std@@@std@@KAAAPAU_Node@?$_Tree_nod@V?$_Tmap_traits@HUVoiceSnd@@U?$less@H@std@@V?$allocator@U?$pair@$$CBHUVoiceSnd@@@std@@@3@$0A@@std@@@2@PAU342@@Z 1000c370 f i scriptparser.obj
 0001:0000b380       ?_Right@?$_Tree@V?$_Tmap_traits@HUVoiceSnd@@U?$less@H@std@@V?$allocator@U?$pair@$$CBHUVoiceSnd@@@std@@@3@$0A@@std@@@std@@KAAAPAU_Node@?$_Tree_nod@V?$_Tmap_traits@HUVoiceSnd@@U?$less@H@std@@V?$allocator@U?$pair@$$CBHUVoiceSnd@@@std@@@3@$0A@@std@@@2@PAU342@@Z 1000c380 f i scriptparser.obj
 0001:0000b390       ??0?$allocator@U?$pair@$$CBHUVoiceSnd@@@std@@@std@@QAE@ABV01@@Z 1000c390 f i scriptparser.obj
 0001:0000b3a0       ?deallocate@?$allocator@U_Node@?$_Tree_nod@V?$_Tmap_traits@HUVoiceSnd@@U?$less@H@std@@V?$allocator@U?$pair@$$CBHUVoiceSnd@@@std@@@3@$0A@@std@@@std@@@std@@QAEXPAU_Node@?$_Tree_nod@V?$_Tmap_traits@HUVoiceSnd@@U?$less@H@std@@V?$allocator@U?$pair@$$CBHUVoiceSnd@@@std@@@3@$0A@@std@@@2@I@Z 1000c3a0 f i scriptparser.obj
 0001:0000b3b0       ??0?$allocator@UST_CELLS@@@std@@QAE@ABV01@@Z 1000c3b0 f i scriptparser.obj
 0001:0000b3c0       ?deallocate@?$allocator@UST_CELLS@@@std@@QAEXPAUST_CELLS@@I@Z 1000c3c0 f i scriptparser.obj
 0001:0000b3d0       ?max_size@?$allocator@U?$pair@$$CBHUgame_snd@@@std@@@std@@QBEIXZ 1000c3d0 f i scriptparser.obj
 0001:0000b3e0       ?_Isnil@?$_Tree@V?$_Tmap_traits@HUVoiceSnd@@U?$less@H@std@@V?$allocator@U?$pair@$$CBHUVoiceSnd@@@std@@@3@$0A@@std@@@std@@KAAADPAU_Node@?$_Tree_nod@V?$_Tmap_traits@HUVoiceSnd@@U?$less@H@std@@V?$allocator@U?$pair@$$CBHUVoiceSnd@@@std@@@3@$0A@@std@@@2@@Z 1000c3e0 f i scriptparser.obj
 0001:0000b3f0       ?_Lmost@?$_Tree@V?$_Tmap_traits@HUVoiceSnd@@U?$less@H@std@@V?$allocator@U?$pair@$$CBHUVoiceSnd@@@std@@@3@$0A@@std@@@std@@IBEAAPAU_Node@?$_Tree_nod@V?$_Tmap_traits@HUVoiceSnd@@U?$less@H@std@@V?$allocator@U?$pair@$$CBHUVoiceSnd@@@std@@@3@$0A@@std@@@2@XZ 1000c3f0 f i scriptparser.obj
 0001:0000b400       ?_Rmost@?$_Tree@V?$_Tmap_traits@HUVoiceSnd@@U?$less@H@std@@V?$allocator@U?$pair@$$CBHUVoiceSnd@@@std@@@3@$0A@@std@@@std@@IBEAAPAU_Node@?$_Tree_nod@V?$_Tmap_traits@HUVoiceSnd@@U?$less@H@std@@V?$allocator@U?$pair@$$CBHUVoiceSnd@@@std@@@3@$0A@@std@@@2@XZ 1000c400 f i scriptparser.obj
 0001:0000b410       ?_Root@?$_Tree@V?$_Tmap_traits@HUVoiceSnd@@U?$less@H@std@@V?$allocator@U?$pair@$$CBHUVoiceSnd@@@std@@@3@$0A@@std@@@std@@IBEAAPAU_Node@?$_Tree_nod@V?$_Tmap_traits@HUVoiceSnd@@U?$less@H@std@@V?$allocator@U?$pair@$$CBHUVoiceSnd@@@std@@@3@$0A@@std@@@2@XZ 1000c410 f i scriptparser.obj
 0001:0000b420       ?max_size@?$allocator@UST_CELLS@@@std@@QBEIXZ 1000c420 f i scriptparser.obj
 0001:0000b430       ??9const_iterator@?$_Tree@V?$_Tmap_traits@HUAmbientSnd@@U?$less@H@std@@V?$allocator@U?$pair@$$CBHUAmbientSnd@@@std@@@3@$0A@@std@@@std@@QBE_NABV012@@Z 1000c430 f i scriptparser.obj
 0001:0000b460       ??0_Node@?$_Tree_nod@V?$_Tmap_traits@HUgame_snd@@U?$less@H@std@@V?$allocator@U?$pair@$$CBHUgame_snd@@@std@@@3@$0A@@std@@@std@@QAE@PAU012@00ABU?$pair@$$CBHUgame_snd@@@2@D@Z 1000c460 f i scriptparser.obj
 0001:0000b4a0       ??8const_iterator@?$_Tree@V?$_Tmap_traits@HUVoiceSnd@@U?$less@H@std@@V?$allocator@U?$pair@$$CBHUVoiceSnd@@@std@@@3@$0A@@std@@@std@@QBE_NABV012@@Z 1000c4a0 f i scriptparser.obj
 0001:0000b4d0       ??9const_iterator@?$_Tree@V?$_Tmap_traits@HUVoiceSnd@@U?$less@H@std@@V?$allocator@U?$pair@$$CBHUVoiceSnd@@@std@@@3@$0A@@std@@@std@@QBE_NABV012@@Z 1000c4d0 f i scriptparser.obj
 0001:0000b500       ?_Max@?$_Tree@V?$_Tmap_traits@HUgame_snd@@U?$less@H@std@@V?$allocator@U?$pair@$$CBHUgame_snd@@@std@@@3@$0A@@std@@@std@@KAPAU_Node@?$_Tree_nod@V?$_Tmap_traits@HUgame_snd@@U?$less@H@std@@V?$allocator@U?$pair@$$CBHUgame_snd@@@std@@@3@$0A@@std@@@2@PAU342@@Z 1000c500 f i scriptparser.obj
 0001:0000b520       ?_Color@?$_Tree@V?$_Tmap_traits@HUVoiceSnd@@U?$less@H@std@@V?$allocator@U?$pair@$$CBHUVoiceSnd@@@std@@@3@$0A@@std@@@std@@KAAADPAU_Node@?$_Tree_nod@V?$_Tmap_traits@HUVoiceSnd@@U?$less@H@std@@V?$allocator@U?$pair@$$CBHUVoiceSnd@@@std@@@3@$0A@@std@@@2@@Z 1000c520 f i scriptparser.obj
 0001:0000b530       ?_Lrotate@?$_Tree@V?$_Tmap_traits@HUVoiceSnd@@U?$less@H@std@@V?$allocator@U?$pair@$$CBHUVoiceSnd@@@std@@@3@$0A@@std@@@std@@IAEXPAU_Node@?$_Tree_nod@V?$_Tmap_traits@HUVoiceSnd@@U?$less@H@std@@V?$allocator@U?$pair@$$CBHUVoiceSnd@@@std@@@3@$0A@@std@@@2@@Z 1000c530 f i scriptparser.obj
 0001:0000b590       ?_Max@?$_Tree@V?$_Tmap_traits@HUVoiceSnd@@U?$less@H@std@@V?$allocator@U?$pair@$$CBHUVoiceSnd@@@std@@@3@$0A@@std@@@std@@KAPAU_Node@?$_Tree_nod@V?$_Tmap_traits@HUVoiceSnd@@U?$less@H@std@@V?$allocator@U?$pair@$$CBHUVoiceSnd@@@std@@@3@$0A@@std@@@2@PAU342@@Z 1000c590 f i scriptparser.obj
 0001:0000b5b0       ?_Min@?$_Tree@V?$_Tmap_traits@HUVoiceSnd@@U?$less@H@std@@V?$allocator@U?$pair@$$CBHUVoiceSnd@@@std@@@3@$0A@@std@@@std@@KAPAU_Node@?$_Tree_nod@V?$_Tmap_traits@HUVoiceSnd@@U?$less@H@std@@V?$allocator@U?$pair@$$CBHUVoiceSnd@@@std@@@3@$0A@@std@@@2@PAU342@@Z 1000c5b0 f i scriptparser.obj
 0001:0000b5d0       ?_Rrotate@?$_Tree@V?$_Tmap_traits@HUVoiceSnd@@U?$less@H@std@@V?$allocator@U?$pair@$$CBHUVoiceSnd@@@std@@@3@$0A@@std@@@std@@IAEXPAU_Node@?$_Tree_nod@V?$_Tmap_traits@HUVoiceSnd@@U?$less@H@std@@V?$allocator@U?$pair@$$CBHUVoiceSnd@@@std@@@3@$0A@@std@@@2@@Z 1000c5d0 f i scriptparser.obj
 0001:0000b630       ?_Mynode@const_iterator@?$_Tree@V?$_Tmap_traits@HUVoiceSnd@@U?$less@H@std@@V?$allocator@U?$pair@$$CBHUVoiceSnd@@@std@@@3@$0A@@std@@@std@@QBEPAU_Node@?$_Tree_nod@V?$_Tmap_traits@HUVoiceSnd@@U?$less@H@std@@V?$allocator@U?$pair@$$CBHUVoiceSnd@@@std@@@3@$0A@@std@@@3@XZ 1000c630 f i scriptparser.obj
 0001:0000b640       ??0?$_Iterator_with_base@Ubidirectional_iterator_tag@std@@U?$pair@$$CBHUVoiceSnd@@@2@HPBU32@ABU32@V_Iterator_base_aux@2@@std@@QAE@XZ 1000c640 f i scriptparser.obj
 0001:0000b650       ?_Inc@const_iterator@?$_Tree@V?$_Tmap_traits@HUVoiceSnd@@U?$less@H@std@@V?$allocator@U?$pair@$$CBHUVoiceSnd@@@std@@@3@$0A@@std@@@std@@QAEXXZ 1000c650 f i scriptparser.obj
 0001:0000b6d0       ??$_Destroy@PAU_Node@?$_Tree_nod@V?$_Tmap_traits@HUgame_snd@@U?$less@H@std@@V?$allocator@U?$pair@$$CBHUgame_snd@@@std@@@3@$0A@@std@@@std@@@std@@YAXPAPAU_Node@?$_Tree_nod@V?$_Tmap_traits@HUgame_snd@@U?$less@H@std@@V?$allocator@U?$pair@$$CBHUgame_snd@@@std@@@3@$0A@@std@@@0@@Z 1000c6d0 f i scriptparser.obj
 0001:0000b6e0       ??$_Destroy@PAU_Node@?$_Tree_nod@V?$_Tmap_traits@HUAmbientSnd@@U?$less@H@std@@V?$allocator@U?$pair@$$CBHUAmbientSnd@@@std@@@3@$0A@@std@@@std@@@std@@YAXPAPAU_Node@?$_Tree_nod@V?$_Tmap_traits@HUAmbientSnd@@U?$less@H@std@@V?$allocator@U?$pair@$$CBHUAmbientSnd@@@std@@@3@$0A@@std@@@0@@Z 1000c6e0 f i scriptparser.obj
 0001:0000b6f0       ??$_Destroy@PAU_Node@?$_Tree_nod@V?$_Tmap_traits@HUVoiceSnd@@U?$less@H@std@@V?$allocator@U?$pair@$$CBHUVoiceSnd@@@std@@@3@$0A@@std@@@std@@@std@@YAXPAPAU_Node@?$_Tree_nod@V?$_Tmap_traits@HUVoiceSnd@@U?$less@H@std@@V?$allocator@U?$pair@$$CBHUVoiceSnd@@@std@@@3@$0A@@std@@@0@@Z 1000c6f0 f i scriptparser.obj
 0001:0000b700       ??$?0UST_CELLS@@@?$allocator@V_Aux_cont@std@@@std@@QAE@ABV?$allocator@UST_CELLS@@@1@@Z 1000c700 f i scriptparser.obj
 0001:0000b710       ??$_Allocate@UST_CELLS@@@std@@YAPAUST_CELLS@@IPAU1@@Z 1000c710 f i scriptparser.obj
 0001:0000b770       ??$?0U?$pair@$$CBHUgame_snd@@@std@@@?$allocator@PAU_Node@?$_Tree_nod@V?$_Tmap_traits@HUgame_snd@@U?$less@H@std@@V?$allocator@U?$pair@$$CBHUgame_snd@@@std@@@3@$0A@@std@@@std@@@std@@QAE@ABV?$allocator@U?$pair@$$CBHUgame_snd@@@std@@@1@@Z 1000c770 f i scriptparser.obj
 0001:0000b780       ??$_Allocate@U_Node@?$_Tree_nod@V?$_Tmap_traits@HUgame_snd@@U?$less@H@std@@V?$allocator@U?$pair@$$CBHUgame_snd@@@std@@@3@$0A@@std@@@std@@@std@@YAPAU_Node@?$_Tree_nod@V?$_Tmap_traits@HUgame_snd@@U?$less@H@std@@V?$allocator@U?$pair@$$CBHUgame_snd@@@std@@@3@$0A@@std@@@0@IPAU120@@Z 1000c780 f i scriptparser.obj
 0001:0000b7e0       ??$?0U?$pair@$$CBHUAmbientSnd@@@std@@@?$allocator@PAU_Node@?$_Tree_nod@V?$_Tmap_traits@HUAmbientSnd@@U?$less@H@std@@V?$allocator@U?$pair@$$CBHUAmbientSnd@@@std@@@3@$0A@@std@@@std@@@std@@QAE@ABV?$allocator@U?$pair@$$CBHUAmbientSnd@@@std@@@1@@Z 1000c7e0 f i scriptparser.obj
 0001:0000b7f0       ??$?0U?$pair@$$CBHUVoiceSnd@@@std@@@?$allocator@PAU_Node@?$_Tree_nod@V?$_Tmap_traits@HUVoiceSnd@@U?$less@H@std@@V?$allocator@U?$pair@$$CBHUVoiceSnd@@@std@@@3@$0A@@std@@@std@@@std@@QAE@ABV?$allocator@U?$pair@$$CBHUVoiceSnd@@@std@@@1@@Z 1000c7f0 f i scriptparser.obj
 0001:0000b800       ??$?0U?$pair@$$CBHUgame_snd@@@std@@@?$allocator@U_Node@?$_Tree_nod@V?$_Tmap_traits@HUgame_snd@@U?$less@H@std@@V?$allocator@U?$pair@$$CBHUgame_snd@@@std@@@3@$0A@@std@@@std@@@std@@QAE@ABV?$allocator@U?$pair@$$CBHUgame_snd@@@std@@@1@@Z 1000c800 f i scriptparser.obj
 0001:0000b810       ??$_Construct@PAU_Node@?$_Tree_nod@V?$_Tmap_traits@HUgame_snd@@U?$less@H@std@@V?$allocator@U?$pair@$$CBHUgame_snd@@@std@@@3@$0A@@std@@@std@@PAU123@@std@@YAXPAPAU_Node@?$_Tree_nod@V?$_Tmap_traits@HUgame_snd@@U?$less@H@std@@V?$allocator@U?$pair@$$CBHUgame_snd@@@std@@@3@$0A@@std@@@0@ABQAU120@@Z 1000c810 f i scriptparser.obj
 0001:0000b830       ??$?0U?$pair@$$CBHUAmbientSnd@@@std@@@?$allocator@U_Node@?$_Tree_nod@V?$_Tmap_traits@HUAmbientSnd@@U?$less@H@std@@V?$allocator@U?$pair@$$CBHUAmbientSnd@@@std@@@3@$0A@@std@@@std@@@std@@QAE@ABV?$allocator@U?$pair@$$CBHUAmbientSnd@@@std@@@1@@Z 1000c830 f i scriptparser.obj
 0001:0000b840       ??$_Destroy@U_Node@?$_Tree_nod@V?$_Tmap_traits@HUAmbientSnd@@U?$less@H@std@@V?$allocator@U?$pair@$$CBHUAmbientSnd@@@std@@@3@$0A@@std@@@std@@@std@@YAXPAU_Node@?$_Tree_nod@V?$_Tmap_traits@HUAmbientSnd@@U?$less@H@std@@V?$allocator@U?$pair@$$CBHUAmbientSnd@@@std@@@3@$0A@@std@@@0@@Z 1000c840 f i scriptparser.obj
 0001:0000b850       ??$_Construct@PAU_Node@?$_Tree_nod@V?$_Tmap_traits@HUAmbientSnd@@U?$less@H@std@@V?$allocator@U?$pair@$$CBHUAmbientSnd@@@std@@@3@$0A@@std@@@std@@PAU123@@std@@YAXPAPAU_Node@?$_Tree_nod@V?$_Tmap_traits@HUAmbientSnd@@U?$less@H@std@@V?$allocator@U?$pair@$$CBHUAmbientSnd@@@std@@@3@$0A@@std@@@0@ABQAU120@@Z 1000c850 f i scriptparser.obj
 0001:0000b870       ??$?0U?$pair@$$CBHUVoiceSnd@@@std@@@?$allocator@U_Node@?$_Tree_nod@V?$_Tmap_traits@HUVoiceSnd@@U?$less@H@std@@V?$allocator@U?$pair@$$CBHUVoiceSnd@@@std@@@3@$0A@@std@@@std@@@std@@QAE@ABV?$allocator@U?$pair@$$CBHUVoiceSnd@@@std@@@1@@Z 1000c870 f i scriptparser.obj
 0001:0000b880       ??$_Allocate@U_Node@?$_Tree_nod@V?$_Tmap_traits@HUVoiceSnd@@U?$less@H@std@@V?$allocator@U?$pair@$$CBHUVoiceSnd@@@std@@@3@$0A@@std@@@std@@@std@@YAPAU_Node@?$_Tree_nod@V?$_Tmap_traits@HUVoiceSnd@@U?$less@H@std@@V?$allocator@U?$pair@$$CBHUVoiceSnd@@@std@@@3@$0A@@std@@@0@IPAU120@@Z 1000c880 f i scriptparser.obj
 0001:0000b8e0       ??$_Destroy@U_Node@?$_Tree_nod@V?$_Tmap_traits@HUVoiceSnd@@U?$less@H@std@@V?$allocator@U?$pair@$$CBHUVoiceSnd@@@std@@@3@$0A@@std@@@std@@@std@@YAXPAU_Node@?$_Tree_nod@V?$_Tmap_traits@HUVoiceSnd@@U?$less@H@std@@V?$allocator@U?$pair@$$CBHUVoiceSnd@@@std@@@3@$0A@@std@@@0@@Z 1000c8e0 f i scriptparser.obj
 0001:0000b8f0       ??$_Construct@PAU_Node@?$_Tree_nod@V?$_Tmap_traits@HUVoiceSnd@@U?$less@H@std@@V?$allocator@U?$pair@$$CBHUVoiceSnd@@@std@@@3@$0A@@std@@@std@@PAU123@@std@@YAXPAPAU_Node@?$_Tree_nod@V?$_Tmap_traits@HUVoiceSnd@@U?$less@H@std@@V?$allocator@U?$pair@$$CBHUVoiceSnd@@@std@@@3@$0A@@std@@@0@ABQAU120@@Z 1000c8f0 f i scriptparser.obj
 0001:0000b910       ??$?0U?$pair@$$CBHUgame_snd@@@std@@@?$allocator@V_Aux_cont@std@@@std@@QAE@ABV?$allocator@U?$pair@$$CBHUgame_snd@@@std@@@1@@Z 1000c910 f i scriptparser.obj
 0001:0000b920       ??$?0U?$pair@$$CBHUAmbientSnd@@@std@@@?$allocator@V_Aux_cont@std@@@std@@QAE@ABV?$allocator@U?$pair@$$CBHUAmbientSnd@@@std@@@1@@Z 1000c920 f i scriptparser.obj
 0001:0000b930       ??$?0U?$pair@$$CBHUVoiceSnd@@@std@@@?$allocator@V_Aux_cont@std@@@std@@QAE@ABV?$allocator@U?$pair@$$CBHUVoiceSnd@@@std@@@1@@Z 1000c930 f i scriptparser.obj
 0001:0000b940       ??$_Ptr_cat@PAUST_CELLS@@PAU1@@std@@YA?AU_Nonscalar_ptr_iterator_tag@0@AAPAUST_CELLS@@0@Z 1000c940 f i scriptparser.obj
 0001:0000b950       ??1?$_Container_base_aux_alloc_real@V?$allocator@V?$basic_string@DU?$char_traits@D@std@@V?$allocator@D@2@@std@@@std@@@std@@IAE@XZ 1000c950 f i scriptparser.obj
 0001:0000b960       ?deallocate@?$allocator@V?$basic_string@DU?$char_traits@D@std@@V?$allocator@D@2@@std@@@std@@QAEXPAV?$basic_string@DU?$char_traits@D@std@@V?$allocator@D@2@@2@I@Z 1000c960 f i scriptparser.obj
 0001:0000b970       ??$_Ptr_cat@PAV?$basic_string@DU?$char_traits@D@std@@V?$allocator@D@2@@std@@PAV12@@std@@YA?AU_Nonscalar_ptr_iterator_tag@0@AAPAV?$basic_string@DU?$char_traits@D@std@@V?$allocator@D@2@@0@0@Z 1000c970 f i scriptparser.obj
 0001:0000b980       ?compare@?$basic_string@DU?$char_traits@D@std@@V?$allocator@D@2@@std@@QBEHIIPBDI@Z 1000c980 f i scriptparser.obj
 0001:0000b9f0       ??1?$_Container_base_aux_alloc_real@V?$allocator@U?$pair@$$CBHUgame_snd@@@std@@@std@@@std@@IAE@XZ 1000c9f0 f i scriptparser.obj
 0001:0000ba00       ??1?$_Container_base_aux_alloc_real@V?$allocator@U?$pair@$$CBHUAmbientSnd@@@std@@@std@@@std@@IAE@XZ 1000ca00 f i scriptparser.obj
 0001:0000ba10       ??1?$_Container_base_aux_alloc_real@V?$allocator@U?$pair@$$CBHUVoiceSnd@@@std@@@std@@@std@@IAE@XZ 1000ca10 f i scriptparser.obj
 0001:0000ba20       ??1?$_Container_base_aux_alloc_real@V?$allocator@UST_CELLS@@@std@@@std@@IAE@XZ 1000ca20 f i scriptparser.obj
 0001:0000ba30       ?max_size@?$_Tree@V?$_Tmap_traits@HUgame_snd@@U?$less@H@std@@V?$allocator@U?$pair@$$CBHUgame_snd@@@std@@@3@$0A@@std@@@std@@QBEIXZ 1000ca30 f i scriptparser.obj
 0001:0000ba40       ?_Lrotate@?$_Tree@V?$_Tmap_traits@HUgame_snd@@U?$less@H@std@@V?$allocator@U?$pair@$$CBHUgame_snd@@@std@@@3@$0A@@std@@@std@@IAEXPAU_Node@?$_Tree_nod@V?$_Tmap_traits@HUgame_snd@@U?$less@H@std@@V?$allocator@U?$pair@$$CBHUgame_snd@@@std@@@3@$0A@@std@@@2@@Z 1000ca40 f i scriptparser.obj
 0001:0000baa0       ?_Rrotate@?$_Tree@V?$_Tmap_traits@HUgame_snd@@U?$less@H@std@@V?$allocator@U?$pair@$$CBHUgame_snd@@@std@@@3@$0A@@std@@@std@@IAEXPAU_Node@?$_Tree_nod@V?$_Tmap_traits@HUgame_snd@@U?$less@H@std@@V?$allocator@U?$pair@$$CBHUgame_snd@@@std@@@3@$0A@@std@@@2@@Z 1000caa0 f i scriptparser.obj
 0001:0000bb00       ?destroy@?$allocator@PAU_Node@?$_Tree_nod@V?$_Tmap_traits@HUgame_snd@@U?$less@H@std@@V?$allocator@U?$pair@$$CBHUgame_snd@@@std@@@3@$0A@@std@@@std@@@std@@QAEXPAPAU_Node@?$_Tree_nod@V?$_Tmap_traits@HUgame_snd@@U?$less@H@std@@V?$allocator@U?$pair@$$CBHUgame_snd@@@std@@@3@$0A@@std@@@2@@Z 1000cb00 f i scriptparser.obj
 0001:0000bb10       ?destroy@?$allocator@PAU_Node@?$_Tree_nod@V?$_Tmap_traits@HUAmbientSnd@@U?$less@H@std@@V?$allocator@U?$pair@$$CBHUAmbientSnd@@@std@@@3@$0A@@std@@@std@@@std@@QAEXPAPAU_Node@?$_Tree_nod@V?$_Tmap_traits@HUAmbientSnd@@U?$less@H@std@@V?$allocator@U?$pair@$$CBHUAmbientSnd@@@std@@@3@$0A@@std@@@2@@Z 1000cb10 f i scriptparser.obj
 0001:0000bb20       ?destroy@?$allocator@PAU_Node@?$_Tree_nod@V?$_Tmap_traits@HUVoiceSnd@@U?$less@H@std@@V?$allocator@U?$pair@$$CBHUVoiceSnd@@@std@@@3@$0A@@std@@@std@@@std@@QAEXPAPAU_Node@?$_Tree_nod@V?$_Tmap_traits@HUVoiceSnd@@U?$less@H@std@@V?$allocator@U?$pair@$$CBHUVoiceSnd@@@std@@@3@$0A@@std@@@2@@Z 1000cb20 f i scriptparser.obj
 0001:0000bb30       ?max_size@?$vector@UST_CELLS@@V?$allocator@UST_CELLS@@@std@@@std@@QBEIXZ 1000cb30 f i scriptparser.obj
 0001:0000bb40       ?allocate@?$allocator@UST_CELLS@@@std@@QAEPAUST_CELLS@@I@Z 1000cb40 f i scriptparser.obj
 0001:0000bb60       ?allocate@?$allocator@U_Node@?$_Tree_nod@V?$_Tmap_traits@HUgame_snd@@U?$less@H@std@@V?$allocator@U?$pair@$$CBHUgame_snd@@@std@@@3@$0A@@std@@@std@@@std@@QAEPAU_Node@?$_Tree_nod@V?$_Tmap_traits@HUgame_snd@@U?$less@H@std@@V?$allocator@U?$pair@$$CBHUgame_snd@@@std@@@3@$0A@@std@@@2@I@Z 1000cb60 f i scriptparser.obj
 0001:0000bb80       ?_Dec@const_iterator@?$_Tree@V?$_Tmap_traits@HUgame_snd@@U?$less@H@std@@V?$allocator@U?$pair@$$CBHUgame_snd@@@std@@@3@$0A@@std@@@std@@QAEXXZ 1000cb80 f i scriptparser.obj
 0001:0000bc20       ?construct@?$allocator@PAU_Node@?$_Tree_nod@V?$_Tmap_traits@HUgame_snd@@U?$less@H@std@@V?$allocator@U?$pair@$$CBHUgame_snd@@@std@@@3@$0A@@std@@@std@@@std@@QAEXPAPAU_Node@?$_Tree_nod@V?$_Tmap_traits@HUgame_snd@@U?$less@H@std@@V?$allocator@U?$pair@$$CBHUgame_snd@@@std@@@3@$0A@@std@@@2@ABQAU342@@Z 1000cc20 f i scriptparser.obj
 0001:0000bc40       ?destroy@?$allocator@U_Node@?$_Tree_nod@V?$_Tmap_traits@HUAmbientSnd@@U?$less@H@std@@V?$allocator@U?$pair@$$CBHUAmbientSnd@@@std@@@3@$0A@@std@@@std@@@std@@QAEXPAU_Node@?$_Tree_nod@V?$_Tmap_traits@HUAmbientSnd@@U?$less@H@std@@V?$allocator@U?$pair@$$CBHUAmbientSnd@@@std@@@3@$0A@@std@@@2@@Z 1000cc40 f i scriptparser.obj
 0001:0000bc50       ?construct@?$allocator@PAU_Node@?$_Tree_nod@V?$_Tmap_traits@HUAmbientSnd@@U?$less@H@std@@V?$allocator@U?$pair@$$CBHUAmbientSnd@@@std@@@3@$0A@@std@@@std@@@std@@QAEXPAPAU_Node@?$_Tree_nod@V?$_Tmap_traits@HUAmbientSnd@@U?$less@H@std@@V?$allocator@U?$pair@$$CBHUAmbientSnd@@@std@@@3@$0A@@std@@@2@ABQAU342@@Z 1000cc50 f i scriptparser.obj
 0001:0000bc70       ?allocate@?$allocator@U_Node@?$_Tree_nod@V?$_Tmap_traits@HUVoiceSnd@@U?$less@H@std@@V?$allocator@U?$pair@$$CBHUVoiceSnd@@@std@@@3@$0A@@std@@@std@@@std@@QAEPAU_Node@?$_Tree_nod@V?$_Tmap_traits@HUVoiceSnd@@U?$less@H@std@@V?$allocator@U?$pair@$$CBHUVoiceSnd@@@std@@@3@$0A@@std@@@2@I@Z 1000cc70 f i scriptparser.obj
 0001:0000bc90       ?destroy@?$allocator@U_Node@?$_Tree_nod@V?$_Tmap_traits@HUVoiceSnd@@U?$less@H@std@@V?$allocator@U?$pair@$$CBHUVoiceSnd@@@std@@@3@$0A@@std@@@std@@@std@@QAEXPAU_Node@?$_Tree_nod@V?$_Tmap_traits@HUVoiceSnd@@U?$less@H@std@@V?$allocator@U?$pair@$$CBHUVoiceSnd@@@std@@@3@$0A@@std@@@2@@Z 1000cc90 f i scriptparser.obj
 0001:0000bca0       ?construct@?$allocator@PAU_Node@?$_Tree_nod@V?$_Tmap_traits@HUVoiceSnd@@U?$less@H@std@@V?$allocator@U?$pair@$$CBHUVoiceSnd@@@std@@@3@$0A@@std@@@std@@@std@@QAEXPAPAU_Node@?$_Tree_nod@V?$_Tmap_traits@HUVoiceSnd@@U?$less@H@std@@V?$allocator@U?$pair@$$CBHUVoiceSnd@@@std@@@3@$0A@@std@@@2@ABQAU342@@Z 1000cca0 f i scriptparser.obj
 0001:0000bcc0       ??Econst_iterator@?$_Tree@V?$_Tmap_traits@HUVoiceSnd@@U?$less@H@std@@V?$allocator@U?$pair@$$CBHUVoiceSnd@@@std@@@3@$0A@@std@@@std@@QAEAAV012@XZ 1000ccc0 f i scriptparser.obj
 0001:0000bcd0       ??0?$_Bidit@U?$pair@$$CBHUVoiceSnd@@@std@@HPBU12@ABU12@@std@@QAE@XZ 1000ccd0 f i scriptparser.obj
 0001:0000bce0       ??0?$_Container_base_aux_alloc_real@V?$allocator@U?$pair@$$CBHUgame_snd@@@std@@@std@@@std@@IAE@V?$allocator@U?$pair@$$CBHUgame_snd@@@std@@@1@@Z 1000cce0 f i scriptparser.obj
 0001:0000bd10       ??0?$_Container_base_aux_alloc_real@V?$allocator@U?$pair@$$CBHUAmbientSnd@@@std@@@std@@@std@@IAE@V?$allocator@U?$pair@$$CBHUAmbientSnd@@@std@@@1@@Z 1000cd10 f i scriptparser.obj
 0001:0000bd40       ??0?$_Container_base_aux_alloc_real@V?$allocator@U?$pair@$$CBHUVoiceSnd@@@std@@@std@@@std@@IAE@V?$allocator@U?$pair@$$CBHUVoiceSnd@@@std@@@1@@Z 1000cd40 f i scriptparser.obj
 0001:0000bd70       ??1?$_Vector_val@V?$basic_string@DU?$char_traits@D@std@@V?$allocator@D@2@@std@@V?$allocator@V?$basic_string@DU?$char_traits@D@std@@V?$allocator@D@2@@std@@@2@@std@@QAE@XZ 1000cd70 f i scriptparser.obj
 0001:0000bd80       ?compare@?$basic_string@DU?$char_traits@D@std@@V?$allocator@D@2@@std@@QBEHPBD@Z 1000cd80 f i scriptparser.obj
 0001:0000bdb0       ??1?$_Vector_val@UST_CELLS@@V?$allocator@UST_CELLS@@@std@@@std@@QAE@XZ 1000cdb0 f i scriptparser.obj
 0001:0000bdc0       ??1?$_Tmap_traits@HUgame_snd@@U?$less@H@std@@V?$allocator@U?$pair@$$CBHUgame_snd@@@std@@@3@$0A@@std@@QAE@XZ 1000cdc0 f i scriptparser.obj
 0001:0000bdd0       ??1?$_Tmap_traits@HUAmbientSnd@@U?$less@H@std@@V?$allocator@U?$pair@$$CBHUAmbientSnd@@@std@@@3@$0A@@std@@QAE@XZ 1000cdd0 f i scriptparser.obj
 0001:0000bde0       ??1?$_Tmap_traits@HUVoiceSnd@@U?$less@H@std@@V?$allocator@U?$pair@$$CBHUVoiceSnd@@@std@@@3@$0A@@std@@QAE@XZ 1000cde0 f i scriptparser.obj
 0001:0000bdf0       ?_Buynode@?$_Tree@V?$_Tmap_traits@HUgame_snd@@U?$less@H@std@@V?$allocator@U?$pair@$$CBHUgame_snd@@@std@@@3@$0A@@std@@@std@@IAEPAU_Node@?$_Tree_nod@V?$_Tmap_traits@HUgame_snd@@U?$less@H@std@@V?$allocator@U?$pair@$$CBHUgame_snd@@@std@@@3@$0A@@std@@@2@PAU342@00ABU?$pair@$$CBHUgame_snd@@@2@D@Z 1000cdf0 f i scriptparser.obj
 0001:0000be40       ??0?$_Container_base_aux_alloc_real@V?$allocator@UST_CELLS@@@std@@@std@@IAE@V?$allocator@UST_CELLS@@@1@@Z 1000ce40 f i scriptparser.obj
 0001:0000be70       ??0const_iterator@?$_Tree@V?$_Tmap_traits@HUgame_snd@@U?$less@H@std@@V?$allocator@U?$pair@$$CBHUgame_snd@@@std@@@3@$0A@@std@@@std@@QAE@XZ 1000ce70 f i scriptparser.obj
 0001:0000be80       ??Fconst_iterator@?$_Tree@V?$_Tmap_traits@HUgame_snd@@U?$less@H@std@@V?$allocator@U?$pair@$$CBHUgame_snd@@@std@@@3@$0A@@std@@@std@@QAEAAV012@XZ 1000ce80 f i scriptparser.obj
 0001:0000be90       ?_Buynode@?$_Tree@V?$_Tmap_traits@HUgame_snd@@U?$less@H@std@@V?$allocator@U?$pair@$$CBHUgame_snd@@@std@@@3@$0A@@std@@@std@@IAEPAU_Node@?$_Tree_nod@V?$_Tmap_traits@HUgame_snd@@U?$less@H@std@@V?$allocator@U?$pair@$$CBHUgame_snd@@@std@@@3@$0A@@std@@@2@XZ 1000ce90 f i scriptparser.obj
 0001:0000bed0       ?_Buynode@?$_Tree@V?$_Tmap_traits@HUAmbientSnd@@U?$less@H@std@@V?$allocator@U?$pair@$$CBHUAmbientSnd@@@std@@@3@$0A@@std@@@std@@IAEPAU_Node@?$_Tree_nod@V?$_Tmap_traits@HUAmbientSnd@@U?$less@H@std@@V?$allocator@U?$pair@$$CBHUAmbientSnd@@@std@@@3@$0A@@std@@@2@XZ 1000ced0 f i scriptparser.obj
 0001:0000bf10       ?_Buynode@?$_Tree@V?$_Tmap_traits@HUVoiceSnd@@U?$less@H@std@@V?$allocator@U?$pair@$$CBHUVoiceSnd@@@std@@@3@$0A@@std@@@std@@IAEPAU_Node@?$_Tree_nod@V?$_Tmap_traits@HUVoiceSnd@@U?$less@H@std@@V?$allocator@U?$pair@$$CBHUVoiceSnd@@@std@@@3@$0A@@std@@@2@XZ 1000cf10 f i scriptparser.obj
 0001:0000bf50       ??Econst_iterator@?$_Tree@V?$_Tmap_traits@HUgame_snd@@U?$less@H@std@@V?$allocator@U?$pair@$$CBHUgame_snd@@@std@@@3@$0A@@std@@@std@@QAE?AV012@H@Z 1000cf50 f i scriptparser.obj
 0001:0000bf70       ??Econst_iterator@?$_Tree@V?$_Tmap_traits@HUAmbientSnd@@U?$less@H@std@@V?$allocator@U?$pair@$$CBHUAmbientSnd@@@std@@@3@$0A@@std@@@std@@QAE?AV012@H@Z 1000cf70 f i scriptparser.obj
 0001:0000bf90       ??Econst_iterator@?$_Tree@V?$_Tmap_traits@HUVoiceSnd@@U?$less@H@std@@V?$allocator@U?$pair@$$CBHUVoiceSnd@@@std@@@3@$0A@@std@@@std@@QAE?AV012@H@Z 1000cf90 f i scriptparser.obj
 0001:0000bfb0       ?_Erase@?$_Tree@V?$_Tmap_traits@HUAmbientSnd@@U?$less@H@std@@V?$allocator@U?$pair@$$CBHUAmbientSnd@@@std@@@3@$0A@@std@@@std@@IAEXPAU_Node@?$_Tree_nod@V?$_Tmap_traits@HUAmbientSnd@@U?$less@H@std@@V?$allocator@U?$pair@$$CBHUAmbientSnd@@@std@@@3@$0A@@std@@@2@@Z 1000cfb0 f i scriptparser.obj
 0001:0000bff0       ?_Erase@?$_Tree@V?$_Tmap_traits@HUVoiceSnd@@U?$less@H@std@@V?$allocator@U?$pair@$$CBHUVoiceSnd@@@std@@@3@$0A@@std@@@std@@IAEXPAU_Node@?$_Tree_nod@V?$_Tmap_traits@HUVoiceSnd@@U?$less@H@std@@V?$allocator@U?$pair@$$CBHUVoiceSnd@@@std@@@3@$0A@@std@@@2@@Z 1000cff0 f i scriptparser.obj
 0001:0000c030       ??0const_iterator@?$_Tree@V?$_Tmap_traits@HUVoiceSnd@@U?$less@H@std@@V?$allocator@U?$pair@$$CBHUVoiceSnd@@@std@@@3@$0A@@std@@@std@@QAE@PAU_Node@?$_Tree_nod@V?$_Tmap_traits@HUVoiceSnd@@U?$less@H@std@@V?$allocator@U?$pair@$$CBHUVoiceSnd@@@std@@@3@$0A@@std@@@2@PBV12@@Z 1000d030 f i scriptparser.obj
 0001:0000c060       ??0?$_Tmap_traits@HUgame_snd@@U?$less@H@std@@V?$allocator@U?$pair@$$CBHUgame_snd@@@std@@@3@$0A@@std@@QAE@U?$less@H@1@V?$allocator@U?$pair@$$CBHUgame_snd@@@std@@@1@@Z 1000d060 f i scriptparser.obj
 0001:0000c090       ??0?$_Tmap_traits@HUAmbientSnd@@U?$less@H@std@@V?$allocator@U?$pair@$$CBHUAmbientSnd@@@std@@@3@$0A@@std@@QAE@U?$less@H@1@V?$allocator@U?$pair@$$CBHUAmbientSnd@@@std@@@1@@Z 1000d090 f i scriptparser.obj
 0001:0000c0c0       ??0?$_Tmap_traits@HUVoiceSnd@@U?$less@H@std@@V?$allocator@U?$pair@$$CBHUVoiceSnd@@@std@@@3@$0A@@std@@QAE@U?$less@H@1@V?$allocator@U?$pair@$$CBHUVoiceSnd@@@std@@@1@@Z 1000d0c0 f i scriptparser.obj
 0001:0000c0f0       ??$?8DU?$char_traits@D@std@@V?$allocator@D@1@@std@@YA_NPBDABV?$basic_string@DU?$char_traits@D@std@@V?$allocator@D@2@@0@@Z 1000d0f0 f i scriptparser.obj
 0001:0000c130       ??1?$_Tree_nod@V?$_Tmap_traits@HUgame_snd@@U?$less@H@std@@V?$allocator@U?$pair@$$CBHUgame_snd@@@std@@@3@$0A@@std@@@std@@QAE@XZ 1000d130 f i scriptparser.obj
 0001:0000c140       ??1?$_Tree_nod@V?$_Tmap_traits@HUAmbientSnd@@U?$less@H@std@@V?$allocator@U?$pair@$$CBHUAmbientSnd@@@std@@@3@$0A@@std@@@std@@QAE@XZ 1000d140 f i scriptparser.obj
 0001:0000c150       ??1?$_Tree_nod@V?$_Tmap_traits@HUVoiceSnd@@U?$less@H@std@@V?$allocator@U?$pair@$$CBHUVoiceSnd@@@std@@@3@$0A@@std@@@std@@QAE@XZ 1000d150 f i scriptparser.obj
 0001:0000c160       ??0?$_Vector_val@UST_CELLS@@V?$allocator@UST_CELLS@@@std@@@std@@IAE@V?$allocator@UST_CELLS@@@1@@Z 1000d160 f i scriptparser.obj
 0001:0000c190       ??Fiterator@?$_Tree@V?$_Tmap_traits@HUgame_snd@@U?$less@H@std@@V?$allocator@U?$pair@$$CBHUgame_snd@@@std@@@3@$0A@@std@@@std@@QAEAAV012@XZ 1000d190 f i scriptparser.obj
 0001:0000c1a0       ?_Init@?$_Tree@V?$_Tmap_traits@HUgame_snd@@U?$less@H@std@@V?$allocator@U?$pair@$$CBHUgame_snd@@@std@@@3@$0A@@std@@@std@@IAEXXZ 1000d1a0 f i scriptparser.obj
 0001:0000c1d0       ?_Init@?$_Tree@V?$_Tmap_traits@HUAmbientSnd@@U?$less@H@std@@V?$allocator@U?$pair@$$CBHUAmbientSnd@@@std@@@3@$0A@@std@@@std@@IAEXXZ 1000d1d0 f i scriptparser.obj
 0001:0000c200       ?_Init@?$_Tree@V?$_Tmap_traits@HUVoiceSnd@@U?$less@H@std@@V?$allocator@U?$pair@$$CBHUVoiceSnd@@@std@@@3@$0A@@std@@@std@@IAEXXZ 1000d200 f i scriptparser.obj
 0001:0000c230       ?_Make_iter@?$_Tree@V?$_Tmap_traits@HUgame_snd@@U?$less@H@std@@V?$allocator@U?$pair@$$CBHUgame_snd@@@std@@@3@$0A@@std@@@std@@QBE?AViterator@12@Vconst_iterator@12@@Z 1000d230 f i scriptparser.obj
 0001:0000c260       ?_Make_iter@?$_Tree@V?$_Tmap_traits@HUAmbientSnd@@U?$less@H@std@@V?$allocator@U?$pair@$$CBHUAmbientSnd@@@std@@@3@$0A@@std@@@std@@QBE?AViterator@12@Vconst_iterator@12@@Z 1000d260 f i scriptparser.obj
 0001:0000c290       ?clear@?$_Tree@V?$_Tmap_traits@HUAmbientSnd@@U?$less@H@std@@V?$allocator@U?$pair@$$CBHUAmbientSnd@@@std@@@3@$0A@@std@@@std@@QAEXXZ 1000d290 f i scriptparser.obj
 0001:0000c2c0       ?clear@?$_Tree@V?$_Tmap_traits@HUVoiceSnd@@U?$less@H@std@@V?$allocator@U?$pair@$$CBHUVoiceSnd@@@std@@@3@$0A@@std@@@std@@QAEXXZ 1000d2c0 f i scriptparser.obj
 0001:0000c2f0       ??0iterator@?$_Tree@V?$_Tmap_traits@HUVoiceSnd@@U?$less@H@std@@V?$allocator@U?$pair@$$CBHUVoiceSnd@@@std@@@3@$0A@@std@@@std@@QAE@PAU_Node@?$_Tree_nod@V?$_Tmap_traits@HUVoiceSnd@@U?$less@H@std@@V?$allocator@U?$pair@$$CBHUVoiceSnd@@@std@@@3@$0A@@std@@@2@PBV12@@Z 1000d2f0 f i scriptparser.obj
 0001:0000c320       ??0?$_Tree_nod@V?$_Tmap_traits@HUgame_snd@@U?$less@H@std@@V?$allocator@U?$pair@$$CBHUgame_snd@@@std@@@3@$0A@@std@@@std@@IAE@ABU?$less@H@1@V?$allocator@U?$pair@$$CBHUgame_snd@@@std@@@1@@Z 1000d320 f i scriptparser.obj
 0001:0000c350       ??0?$_Tree_nod@V?$_Tmap_traits@HUAmbientSnd@@U?$less@H@std@@V?$allocator@U?$pair@$$CBHUAmbientSnd@@@std@@@3@$0A@@std@@@std@@IAE@ABU?$less@H@1@V?$allocator@U?$pair@$$CBHUAmbientSnd@@@std@@@1@@Z 1000d350 f i scriptparser.obj
 0001:0000c380       ??0?$_Tree_nod@V?$_Tmap_traits@HUVoiceSnd@@U?$less@H@std@@V?$allocator@U?$pair@$$CBHUVoiceSnd@@@std@@@3@$0A@@std@@@std@@IAE@ABU?$less@H@1@V?$allocator@U?$pair@$$CBHUVoiceSnd@@@std@@@1@@Z 1000d380 f i scriptparser.obj
 0001:0000c3b0       ??_G?$basic_string@DU?$char_traits@D@std@@V?$allocator@D@2@@std@@QAEPAXI@Z 1000d3b0 f i scriptparser.obj
 0001:0000c3f0       ??1?$_Tree_ptr@V?$_Tmap_traits@HUgame_snd@@U?$less@H@std@@V?$allocator@U?$pair@$$CBHUgame_snd@@@std@@@3@$0A@@std@@@std@@QAE@XZ 1000d3f0 f i scriptparser.obj
 0001:0000c400       ??1?$_Tree_ptr@V?$_Tmap_traits@HUAmbientSnd@@U?$less@H@std@@V?$allocator@U?$pair@$$CBHUAmbientSnd@@@std@@@3@$0A@@std@@@std@@QAE@XZ 1000d400 f i scriptparser.obj
 0001:0000c410       ??1?$_Tree_ptr@V?$_Tmap_traits@HUVoiceSnd@@U?$less@H@std@@V?$allocator@U?$pair@$$CBHUVoiceSnd@@@std@@@3@$0A@@std@@@std@@QAE@XZ 1000d410 f i scriptparser.obj
 0001:0000c420       ?begin@?$_Tree@V?$_Tmap_traits@HUVoiceSnd@@U?$less@H@std@@V?$allocator@U?$pair@$$CBHUVoiceSnd@@@std@@@3@$0A@@std@@@std@@QAE?AViterator@12@XZ 1000d420 f i scriptparser.obj
 0001:0000c440       ?end@?$_Tree@V?$_Tmap_traits@HUVoiceSnd@@U?$less@H@std@@V?$allocator@U?$pair@$$CBHUVoiceSnd@@@std@@@3@$0A@@std@@@std@@QAE?AViterator@12@XZ 1000d440 f i scriptparser.obj
 0001:0000c460       ??0?$_Tree_ptr@V?$_Tmap_traits@HUgame_snd@@U?$less@H@std@@V?$allocator@U?$pair@$$CBHUgame_snd@@@std@@@3@$0A@@std@@@std@@IAE@ABU?$less@H@1@V?$allocator@U?$pair@$$CBHUgame_snd@@@std@@@1@@Z 1000d460 f i scriptparser.obj
 0001:0000c490       ??0?$_Tree_ptr@V?$_Tmap_traits@HUAmbientSnd@@U?$less@H@std@@V?$allocator@U?$pair@$$CBHUAmbientSnd@@@std@@@3@$0A@@std@@@std@@IAE@ABU?$less@H@1@V?$allocator@U?$pair@$$CBHUAmbientSnd@@@std@@@1@@Z 1000d490 f i scriptparser.obj
 0001:0000c4c0       ?_Make_iter@?$_Tree@V?$_Tmap_traits@HUVoiceSnd@@U?$less@H@std@@V?$allocator@U?$pair@$$CBHUVoiceSnd@@@std@@@3@$0A@@std@@@std@@QBE?AViterator@12@Vconst_iterator@12@@Z 1000d4c0 f i scriptparser.obj
 0001:0000c4f0       ??0?$_Tree_ptr@V?$_Tmap_traits@HUVoiceSnd@@U?$less@H@std@@V?$allocator@U?$pair@$$CBHUVoiceSnd@@@std@@@3@$0A@@std@@@std@@IAE@ABU?$less@H@1@V?$allocator@U?$pair@$$CBHUVoiceSnd@@@std@@@1@@Z 1000d4f0 f i scriptparser.obj
 0001:0000c520       ??$_Destroy@V?$basic_string@DU?$char_traits@D@std@@V?$allocator@D@2@@std@@@std@@YAXPAV?$basic_string@DU?$char_traits@D@std@@V?$allocator@D@2@@0@@Z 1000d520 f i scriptparser.obj
 0001:0000c550       ??1?$_Tree_val@V?$_Tmap_traits@HUgame_snd@@U?$less@H@std@@V?$allocator@U?$pair@$$CBHUgame_snd@@@std@@@3@$0A@@std@@@std@@QAE@XZ 1000d550 f i scriptparser.obj
 0001:0000c560       ??1?$_Tree_val@V?$_Tmap_traits@HUAmbientSnd@@U?$less@H@std@@V?$allocator@U?$pair@$$CBHUAmbientSnd@@@std@@@3@$0A@@std@@@std@@QAE@XZ 1000d560 f i scriptparser.obj
 0001:0000c570       ??1?$_Tree_val@V?$_Tmap_traits@HUVoiceSnd@@U?$less@H@std@@V?$allocator@U?$pair@$$CBHUVoiceSnd@@@std@@@3@$0A@@std@@@std@@QAE@XZ 1000d570 f i scriptparser.obj
 0001:0000c580       ?assign@?$basic_string@DU?$char_traits@D@std@@V?$allocator@D@2@@std@@QAEAAV12@ABV12@@Z 1000d580 f i scriptparser.obj
 0001:0000c5a0       ??0?$_Tree_val@V?$_Tmap_traits@HUgame_snd@@U?$less@H@std@@V?$allocator@U?$pair@$$CBHUgame_snd@@@std@@@3@$0A@@std@@@std@@IAE@ABU?$less@H@1@V?$allocator@U?$pair@$$CBHUgame_snd@@@std@@@1@@Z 1000d5a0 f i scriptparser.obj
 0001:0000c5d0       ??0?$_Tree_val@V?$_Tmap_traits@HUAmbientSnd@@U?$less@H@std@@V?$allocator@U?$pair@$$CBHUAmbientSnd@@@std@@@3@$0A@@std@@@std@@IAE@ABU?$less@H@1@V?$allocator@U?$pair@$$CBHUAmbientSnd@@@std@@@1@@Z 1000d5d0 f i scriptparser.obj
 0001:0000c600       ??0?$_Tree_val@V?$_Tmap_traits@HUVoiceSnd@@U?$less@H@std@@V?$allocator@U?$pair@$$CBHUVoiceSnd@@@std@@@3@$0A@@std@@@std@@IAE@ABU?$less@H@1@V?$allocator@U?$pair@$$CBHUVoiceSnd@@@std@@@1@@Z 1000d600 f i scriptparser.obj
 0001:0000c630       ?destroy@?$allocator@V?$basic_string@DU?$char_traits@D@std@@V?$allocator@D@2@@std@@@std@@QAEXPAV?$basic_string@DU?$char_traits@D@std@@V?$allocator@D@2@@2@@Z 1000d630 f i scriptparser.obj
 0001:0000c660       ??4?$basic_string@DU?$char_traits@D@std@@V?$allocator@D@2@@std@@QAEAAV01@ABV01@@Z 1000d660 f i scriptparser.obj
 0001:0000c680       ??0?$_Tree@V?$_Tmap_traits@HUgame_snd@@U?$less@H@std@@V?$allocator@U?$pair@$$CBHUgame_snd@@@std@@@3@$0A@@std@@@std@@QAE@ABU?$less@H@1@ABV?$allocator@U?$pair@$$CBHUgame_snd@@@std@@@1@@Z 1000d680 f i scriptparser.obj
 0001:0000c710       ?_Insert@?$_Tree@V?$_Tmap_traits@HUgame_snd@@U?$less@H@std@@V?$allocator@U?$pair@$$CBHUgame_snd@@@std@@@3@$0A@@std@@@std@@IAE?AViterator@12@_NPAU_Node@?$_Tree_nod@V?$_Tmap_traits@HUgame_snd@@U?$less@H@std@@V?$allocator@U?$pair@$$CBHUgame_snd@@@std@@@3@$0A@@std@@@2@ABU?$pair@$$CBHUgame_snd@@@2@@Z 1000d710 f i scriptparser.obj
 0001:0000c920       ??0?$_Tree@V?$_Tmap_traits@HUAmbientSnd@@U?$less@H@std@@V?$allocator@U?$pair@$$CBHUAmbientSnd@@@std@@@3@$0A@@std@@@std@@QAE@ABU?$less@H@1@ABV?$allocator@U?$pair@$$CBHUAmbientSnd@@@std@@@1@@Z 1000d920 f i scriptparser.obj
 0001:0000c9b0       ??0?$_Tree@V?$_Tmap_traits@HUVoiceSnd@@U?$less@H@std@@V?$allocator@U?$pair@$$CBHUVoiceSnd@@@std@@@3@$0A@@std@@@std@@QAE@ABU?$less@H@1@ABV?$allocator@U?$pair@$$CBHUVoiceSnd@@@std@@@1@@Z 1000d9b0 f i scriptparser.obj
 0001:0000ca40       ?_Xlen@?$vector@UST_CELLS@@V?$allocator@UST_CELLS@@@std@@@std@@KAXXZ 1000da40 f i scriptparser.obj
 0001:0000cac0       ?erase@?$_Tree@V?$_Tmap_traits@HUgame_snd@@U?$less@H@std@@V?$allocator@U?$pair@$$CBHUgame_snd@@@std@@@3@$0A@@std@@@std@@QAE?AViterator@12@Vconst_iterator@12@@Z 1000dac0 f i scriptparser.obj
 0001:0000ce10       ?erase@?$_Tree@V?$_Tmap_traits@HUAmbientSnd@@U?$less@H@std@@V?$allocator@U?$pair@$$CBHUAmbientSnd@@@std@@@3@$0A@@std@@@std@@QAE?AViterator@12@Vconst_iterator@12@@Z 1000de10 f i scriptparser.obj
 0001:0000d160       ?erase@?$_Tree@V?$_Tmap_traits@HUVoiceSnd@@U?$less@H@std@@V?$allocator@U?$pair@$$CBHUVoiceSnd@@@std@@@3@$0A@@std@@@std@@QAE?AViterator@12@Vconst_iterator@12@@Z 1000e160 f i scriptparser.obj
 0001:0000d4b0       ??$_Destroy_range@V?$allocator@V?$basic_string@DU?$char_traits@D@std@@V?$allocator@D@2@@std@@@std@@@std@@YAXPAV?$basic_string@DU?$char_traits@D@std@@V?$allocator@D@2@@0@0AAV?$allocator@V?$basic_string@DU?$char_traits@D@std@@V?$allocator@D@2@@std@@@0@U_Nonscalar_ptr_iterator_tag@0@@Z 1000e4b0 f i scriptparser.obj
 0001:0000d4f0       ?insert@?$_Tree@V?$_Tmap_traits@HUgame_snd@@U?$less@H@std@@V?$allocator@U?$pair@$$CBHUgame_snd@@@std@@@3@$0A@@std@@@std@@QAE?AU?$pair@Viterator@?$_Tree@V?$_Tmap_traits@HUgame_snd@@U?$less@H@std@@V?$allocator@U?$pair@$$CBHUgame_snd@@@std@@@3@$0A@@std@@@std@@_N@2@ABU?$pair@$$CBHUgame_snd@@@2@@Z 1000e4f0 f i scriptparser.obj
 0001:0000d5f0       ?insert@?$_Tree@V?$_Tmap_traits@HUgame_snd@@U?$less@H@std@@V?$allocator@U?$pair@$$CBHUgame_snd@@@std@@@3@$0A@@std@@@std@@QAE?AViterator@12@Vconst_iterator@12@ABU?$pair@$$CBHUgame_snd@@@2@@Z 1000e5f0 f i scriptparser.obj
 0001:0000d7d0       ?_Buy@?$vector@UST_CELLS@@V?$allocator@UST_CELLS@@@std@@@std@@IAE_NI@Z 1000e7d0 f i scriptparser.obj
 0001:0000d820       ?erase@?$_Tree@V?$_Tmap_traits@HUgame_snd@@U?$less@H@std@@V?$allocator@U?$pair@$$CBHUgame_snd@@@std@@@3@$0A@@std@@@std@@QAE?AViterator@12@Vconst_iterator@12@0@Z 1000e820 f i scriptparser.obj
 0001:0000d900       ?erase@?$_Tree@V?$_Tmap_traits@HUAmbientSnd@@U?$less@H@std@@V?$allocator@U?$pair@$$CBHUAmbientSnd@@@std@@@3@$0A@@std@@@std@@QAE?AViterator@12@Vconst_iterator@12@0@Z 1000e900 f i scriptparser.obj
 0001:0000d9e0       ?erase@?$_Tree@V?$_Tmap_traits@HUVoiceSnd@@U?$less@H@std@@V?$allocator@U?$pair@$$CBHUVoiceSnd@@@std@@@3@$0A@@std@@@std@@QAE?AViterator@12@Vconst_iterator@12@0@Z 1000e9e0 f i scriptparser.obj
 0001:0000dac0       ??$_Destroy_range@V?$allocator@V?$basic_string@DU?$char_traits@D@std@@V?$allocator@D@2@@std@@@std@@@std@@YAXPAV?$basic_string@DU?$char_traits@D@std@@V?$allocator@D@2@@0@0AAV?$allocator@V?$basic_string@DU?$char_traits@D@std@@V?$allocator@D@2@@std@@@0@@Z 1000eac0 f i scriptparser.obj
 0001:0000dae0       ??A?$map@HUgame_snd@@U?$less@H@std@@V?$allocator@U?$pair@$$CBHUgame_snd@@@std@@@3@@std@@QAEAAUgame_snd@@ABH@Z 1000eae0 f i scriptparser.obj
 0001:0000dbb0       ??0?$vector@UST_CELLS@@V?$allocator@UST_CELLS@@@std@@@std@@QAE@XZ 1000ebb0 f i scriptparser.obj
 0001:0000dc10       ?_Tidy@?$_Tree@V?$_Tmap_traits@HUgame_snd@@U?$less@H@std@@V?$allocator@U?$pair@$$CBHUgame_snd@@@std@@@3@$0A@@std@@@std@@IAEXXZ 1000ec10 f i scriptparser.obj
 0001:0000dc50       ?_Tidy@?$_Tree@V?$_Tmap_traits@HUAmbientSnd@@U?$less@H@std@@V?$allocator@U?$pair@$$CBHUAmbientSnd@@@std@@@3@$0A@@std@@@std@@IAEXXZ 1000ec50 f i scriptparser.obj
 0001:0000dc90       ?_Tidy@?$_Tree@V?$_Tmap_traits@HUVoiceSnd@@U?$less@H@std@@V?$allocator@U?$pair@$$CBHUVoiceSnd@@@std@@@3@$0A@@std@@@std@@IAEXXZ 1000ec90 f i scriptparser.obj
 0001:0000dcd0       ?_Destroy@?$vector@V?$basic_string@DU?$char_traits@D@std@@V?$allocator@D@2@@std@@V?$allocator@V?$basic_string@DU?$char_traits@D@std@@V?$allocator@D@2@@std@@@2@@std@@IAEXPAV?$basic_string@DU?$char_traits@D@std@@V?$allocator@D@2@@2@0@Z 1000ecd0 f i scriptparser.obj
 0001:0000dcf0       ?gamesnd_parse_soundtbl@@YAXPAD@Z 1000ecf0 f   scriptparser.obj
 0001:0000e330       ??1?$_Tree@V?$_Tmap_traits@HUgame_snd@@U?$less@H@std@@V?$allocator@U?$pair@$$CBHUgame_snd@@@std@@@3@$0A@@std@@@std@@QAE@XZ 1000f330 f i scriptparser.obj
 0001:0000e3b0       ??1?$_Tree@V?$_Tmap_traits@HUAmbientSnd@@U?$less@H@std@@V?$allocator@U?$pair@$$CBHUAmbientSnd@@@std@@@3@$0A@@std@@@std@@QAE@XZ 1000f3b0 f i scriptparser.obj
 0001:0000e430       ??1?$_Tree@V?$_Tmap_traits@HUVoiceSnd@@U?$less@H@std@@V?$allocator@U?$pair@$$CBHUVoiceSnd@@@std@@@3@$0A@@std@@@std@@QAE@XZ 1000f430 f i scriptparser.obj
 0001:0000e4b0       ?_Tidy@?$vector@V?$basic_string@DU?$char_traits@D@std@@V?$allocator@D@2@@std@@V?$allocator@V?$basic_string@DU?$char_traits@D@std@@V?$allocator@D@2@@std@@@2@@std@@IAEXXZ 1000f4b0 f i scriptparser.obj
 0001:0000e500       ??1?$map@HUgame_snd@@U?$less@H@std@@V?$allocator@U?$pair@$$CBHUgame_snd@@@std@@@3@@std@@QAE@XZ 1000f500 f i scriptparser.obj
 0001:0000e510       ??1?$map@HUAmbientSnd@@U?$less@H@std@@V?$allocator@U?$pair@$$CBHUAmbientSnd@@@std@@@3@@std@@QAE@XZ 1000f510 f i scriptparser.obj
 0001:0000e520       ??1?$map@HUVoiceSnd@@U?$less@H@std@@V?$allocator@U?$pair@$$CBHUVoiceSnd@@@std@@@3@@std@@QAE@XZ 1000f520 f i scriptparser.obj
 0001:0000e530       ?gamesnd_parse_musictbl@@YAXPAD@Z 1000f530 f   scriptparser.obj
 0001:0000e7d0       ?gamesnd_parse_voicetbl@@YAXPAD@Z 1000f7d0 f   scriptparser.obj
 0001:0000ea70       ??0?$map@HUgame_snd@@U?$less@H@std@@V?$allocator@U?$pair@$$CBHUgame_snd@@@std@@@3@@std@@QAE@XZ 1000fa70 f i scriptparser.obj
 0001:0000ea90       ??0?$map@HUAmbientSnd@@U?$less@H@std@@V?$allocator@U?$pair@$$CBHUAmbientSnd@@@std@@@3@@std@@QAE@XZ 1000fa90 f i scriptparser.obj
 0001:0000eab0       ??0?$map@HUVoiceSnd@@U?$less@H@std@@V?$allocator@U?$pair@$$CBHUVoiceSnd@@@std@@@3@@std@@QAE@XZ 1000fab0 f i scriptparser.obj
 0001:0000ead0       ??1?$vector@V?$basic_string@DU?$char_traits@D@std@@V?$allocator@D@2@@std@@V?$allocator@V?$basic_string@DU?$char_traits@D@std@@V?$allocator@D@2@@std@@@2@@std@@QAE@XZ 1000fad0 f i scriptparser.obj
 0001:0000eb20       ??1ST_CELLS@@QAE@XZ        1000fb20 f i scriptparser.obj
 0001:0000eb30       ??_GST_CELLS@@QAEPAXI@Z    1000fb30 f i scriptparser.obj
 0001:0000eb50       ??$_Destroy@UST_CELLS@@@std@@YAXPAUST_CELLS@@@Z 1000fb50 f i scriptparser.obj
 0001:0000eb60       ?destroy@?$allocator@UST_CELLS@@@std@@QAEXPAUST_CELLS@@@Z 1000fb60 f i scriptparser.obj
 0001:0000eb70       ??$_Destroy_range@V?$allocator@UST_CELLS@@@std@@@std@@YAXPAUST_CELLS@@0AAV?$allocator@UST_CELLS@@@0@U_Nonscalar_ptr_iterator_tag@0@@Z 1000fb70 f i scriptparser.obj
 0001:0000ebd0       ??$_Destroy_range@V?$allocator@UST_CELLS@@@std@@@std@@YAXPAUST_CELLS@@0AAV?$allocator@UST_CELLS@@@0@@Z 1000fbd0 f i scriptparser.obj
 0001:0000ebf0       ?_Destroy@?$vector@UST_CELLS@@V?$allocator@UST_CELLS@@@std@@@std@@IAEXPAUST_CELLS@@0@Z 1000fbf0 f i scriptparser.obj
 0001:0000ec10       ?_Tidy@?$vector@UST_CELLS@@V?$allocator@UST_CELLS@@@std@@@std@@IAEXXZ 1000fc10 f i scriptparser.obj
 0001:0000ec60       ??1?$vector@UST_CELLS@@V?$allocator@UST_CELLS@@@std@@@std@@QAE@XZ 1000fc60 f i scriptparser.obj
 0001:0000ecb0       ??0ST_ROWS@@QAE@XZ         1000fcb0 f i scriptparser.obj
 0001:0000ecc0       ??1ST_ROWS@@QAE@XZ         1000fcc0 f i scriptparser.obj
 0001:0000ecd0       ?gamesnd_parse_musictxt@@YAXPAD@Z 1000fcd0 f   scriptparser.obj
 0001:0000f270       ?gamesnd_parse_voicetxt@@YAXPAD@Z 10010270 f   scriptparser.obj
 0001:0000f7c0       ?gamesnd_parse_configtxt@@YAXPAD@Z 100107c0 f   scriptparser.obj
 0001:0000fc90       ?gamesnd_parse_config@@YAXPAD_N@Z 10010c90 f   scriptparser.obj
 0001:0000fcc0       ?gamesnd_parse_music@@YAXPAD_N@Z 10010cc0 f   scriptparser.obj
 0001:0000fcf0       ?gamesnd_parse_voice@@YAXPAD_N@Z 10010cf0 f   scriptparser.obj
 0001:0000fd20       ?gamesnd_parse_soundtxt@@YAXPAD@Z 10010d20 f   scriptparser.obj
 0001:00010a30       ?gamesnd_parse_sound@@YAXPAD_N@Z 10011a30 f   scriptparser.obj
 0001:00010a60       ?voice_init@@YAXXZ         10011a60 f   voicesnd.obj
 0001:00010a70       ?voice_close@@YAXXZ        10011a70 f   voicesnd.obj
 0001:00010a80       ?voice_stop_all@@YAXH@Z    10011a80 f   voicesnd.obj
 0001:00010a90       ?voice_pause_all@@YAXXZ    10011a90 f   voicesnd.obj
 0001:00010aa0       ?voice_unpause_all@@YAXXZ  10011aa0 f   voicesnd.obj
 0001:00010ab0       ?voice_set_volume_all@@YAXM@Z 10011ab0 f   voicesnd.obj
 0001:00010b40       ?voice_stop@@YAXHH@Z       10011b40 f   voicesnd.obj
 0001:00010b90       ?voice_pause@@YAXH@Z       10011b90 f   voicesnd.obj
 0001:00010bb0       ?voice_unpause@@YAXH@Z     10011bb0 f   voicesnd.obj
 0001:00010bd0       ?voice_set_volume@@YAXHM@Z 10011bd0 f   voicesnd.obj
 0001:00010c00       ?voice_set_loop@@YAXHH@Z   10011c00 f   voicesnd.obj
 0001:00010c30       ?voice_state@@YAHH@Z       10011c30 f   voicesnd.obj
 0001:00010c70       ?voice_start@@YAHHMH@Z     10011c70 f   voicesnd.obj
 0001:00010d20       ?timer_close@@YAXXZ        10011d20 f   timer.obj
 0001:00010d50       ?timer_init@@YAXXZ         10011d50 f   timer.obj
 0001:00010de0       ?timer_get_fixed_seconds@@YAJXZ 10011de0 f   timer.obj
 0001:00010e40       ?timer_get_fixed_secondsX@@YAJXZ 10011e40 f   timer.obj
 0001:00010e50       ?timer_get_approx_seconds@@YAJXZ 10011e50 f   timer.obj
 0001:00010e60       ?timer_get_milliseconds@@YAHXZ 10011e60 f   timer.obj
 0001:00010eb0       ?timer_get_microseconds@@YAHXZ 10011eb0 f   timer.obj
 0001:00010f00       ?timestamp_reset@@YAXXZ    10011f00 f   timer.obj
 0001:00010f10       ?timestamp_inc@@YAXM@Z     10011f10 f   timer.obj
 0001:00010f50       ?timestamp@@YAHH@Z         10011f50 f   timer.obj
 0001:00010f90       ?timestamp_until@@YAHH@Z   10011f90 f   timer.obj
 0001:00010fa0       ?timestamp@@YAHXZ          10011fa0 f   timer.obj
 0001:00010fb0       ?timestamp_has_time_elapsed@@YAHHH@Z 10011fb0 f   timer.obj
 0001:00010fd0       ?timing_event_lookup@@YAHPAD@Z 10011fd0 f   timer.obj
 0001:00010fe0       ?timing_frame_start@@YAXXZ 10011fe0 f   timer.obj
 0001:00010ff0       ?timing_frame_stop@@YAXXZ  10011ff0 f   timer.obj
 0001:00011000       ?timing_frame_total@@YAHXZ 10012000 f   timer.obj
 0001:00011010       ?timing_event_start@@YAXPAD@Z 10012010 f   timer.obj
 0001:00011020       ?timing_event_stop@@YAXPAD@Z 10012020 f   timer.obj
 0001:00011030       ?timing_event_total@@YAHPAD@Z 10012030 f   timer.obj
 0001:00011040       ?timing_event_pct@@YAMPAD@Z 10012040 f   timer.obj
 0001:00011180       ?amdInitialize@@YAHPAPAUHMIXER__@@0@Z 10012180 f   util_audiomixer.obj
 0001:000112f0       ?amdUninitialize@@YAHPAUHMIXER__@@@Z 100122f0 f   util_audiomixer.obj
 0001:00011310       ?amdGetMasterVolumeControl@@YAHPAUHMIXER__@@PAHPAK2@Z 10012310 f   util_audiomixer.obj
 0001:00011400       ?amdGetMasterVolumeValue@@YAHPAUHMIXER__@@HPAK@Z 10012400 f   util_audiomixer.obj
 0001:00011470       ?amdSetMasterVolumeValue@@YAHPAUHMIXER__@@HK@Z 10012470 f   util_audiomixer.obj
 0001:000114e0       ?amdGetMasterPanControl@@YAHPAUHMIXER__@@PAHPAJ2@Z 100124e0 f   util_audiomixer.obj
 0001:000115d0       ?amdGetMasterPanValue@@YAHPAUHMIXER__@@HPAJ@Z 100125d0 f   util_audiomixer.obj
 0001:00011640       ?amdSetMasterPanValue@@YAHPAUHMIXER__@@HJ@Z 10012640 f   util_audiomixer.obj
 0001:000116b0       ?amdGetMasterMuteControl@@YAHPAUHMIXER__@@PAH@Z 100126b0 f   util_audiomixer.obj
 0001:00011780       ?amdGetMasterMuteValue@@YAHPAUHMIXER__@@HPAJ@Z 10012780 f   util_audiomixer.obj
 0001:000117f0       ?amdSetMasterMuteValue@@YAHPAUHMIXER__@@HJ@Z 100127f0 f   util_audiomixer.obj
 0001:00011860       ?amdGetVolume@@YAXPAUHMIXER__@@HKKPAH1@Z 10012860 f   util_audiomixer.obj
 0001:00011940       ?amdSetVolume@@YAXPAUHMIXER__@@HKKHH@Z 10012940 f   util_audiomixer.obj
 0001:000119c0       ?amdGetWavVolumeControl@@YAHPAUHMIXER__@@PAHPAK2@Z 100129c0 f   util_audiomixer.obj
 0001:00011ab0       ?amdGetWavVolumeValue@@YAHPAUHMIXER__@@HPAK@Z 10012ab0 f   util_audiomixer.obj
 0001:00011b20       ?amdSetWavVolumeValue@@YAHPAUHMIXER__@@HK@Z 10012b20 f   util_audiomixer.obj
 0001:00011b90       ?amdGetWavPanControl@@YAHPAUHMIXER__@@PAHPAJ2@Z 10012b90 f   util_audiomixer.obj
 0001:00011c80       ?amdGetWavPanValue@@YAHPAUHMIXER__@@HPAJ@Z 10012c80 f   util_audiomixer.obj
 0001:00011cf0       ?amdSetWavPanValue@@YAHPAUHMIXER__@@HJ@Z 10012cf0 f   util_audiomixer.obj
 0001:00011d60       ?amdGetWavMuteControl@@YAHPAUHMIXER__@@PAH@Z 10012d60 f   util_audiomixer.obj
 0001:00011e30       ?amdGetWavMuteValue@@YAHPAUHMIXER__@@HPAJ@Z 10012e30 f   util_audiomixer.obj
 0001:00011ea0       ?amdSetWavMuteValue@@YAHPAUHMIXER__@@HJ@Z 10012ea0 f   util_audiomixer.obj
 0001:00011f10       ?amdGetMicInputVolumeControl@@YAHPAUHMIXER__@@PAHPAK22@Z 10012f10 f   util_audiomixer.obj
 0001:00012150       ?amdGetMicInputVolumeValue@@YAHPAUHMIXER__@@HPAKK@Z 10013150 f   util_audiomixer.obj
 0001:000121c0       ?amdSetMicInputVolumeValue@@YAHPAUHMIXER__@@PAHKK@Z 100131c0 f   util_audiomixer.obj
 0001:00012260       ?amdGetMicOutputVolumeControl@@YAHPAUHMIXER__@@PAHPAK2@Z 10013260 f   util_audiomixer.obj
 0001:000123f0       ?amdGetMicOutputVolumeValue@@YAHPAUHMIXER__@@HPAK@Z 100133f0 f   util_audiomixer.obj
 0001:00012460       ?amdSetMicOutputVolumeValue@@YAHPAUHMIXER__@@HK@Z 10013460 f   util_audiomixer.obj
 0001:000124d0       ?amdGetMicPanControl@@YAHPAUHMIXER__@@PAHPAJ2@Z 100134d0 f   util_audiomixer.obj
 0001:000125c0       ?amdGetMicPanValue@@YAHPAUHMIXER__@@HPAJ@Z 100135c0 f   util_audiomixer.obj
 0001:00012630       ?amdSetMicPanValue@@YAHPAUHMIXER__@@HJ@Z 10013630 f   util_audiomixer.obj
 0001:000126a0       ?amdGetMicOutputMuteControl@@YAHPAUHMIXER__@@PAH@Z 100136a0 f   util_audiomixer.obj
 0001:00012800       ?amdGetMicOutputMuteValue@@YAHPAUHMIXER__@@HPAJ@Z 10013800 f   util_audiomixer.obj
 0001:00012870       ?amdSetMicOutputMuteValue@@YAHPAUHMIXER__@@HJ@Z 10013870 f   util_audiomixer.obj
 0001:000128e0       ?SelectMic@@YAXPAUHMIXER__@@@Z 100138e0 f   util_audiomixer.obj
 0001:00012b70       __LOG                      10013b70 f   util_debug.obj
 0001:00012be0       __LOG2                     10013be0 f   util_debug.obj
 0001:00012cf0       _path_is_directory         10013cf0 f   util_shwapi.obj
 0001:00012d10       _get_program_path          10013d10 f   util_shwapi.obj
 0001:00012d50       _path_add_backslash        10013d50 f   util_shwapi.obj
 0001:00012d90       _path_is_relative          10013d90 f   util_shwapi.obj
 0001:00012e80       _path_remove_filespec      10013e80 f   util_shwapi.obj
 0001:00012ef0       _path_unquote              10013ef0 f   util_shwapi.obj
 0001:00012fc0       __offset                   10013fc0 f   util_shwapi.obj
 0001:00013000       __getat                    10014000 f   util_shwapi.obj
 0001:00013020       __strsize                  10014020 f   util_shwapi.obj
 0001:00013040       __strsizez                 10014040 f   util_shwapi.obj
 0001:00013050       __strzcpy                  10014050 f   util_shwapi.obj
 0001:00013090       __strzcat                  10014090 f   util_shwapi.obj
 0001:000130e0       __strzncpy                 100140e0 f   util_shwapi.obj
 0001:00013160       __strzncat                 10014160 f   util_shwapi.obj
 0001:000131d0       __setat                    100141d0 f   util_shwapi.obj
 0001:000131f0       __insert                   100141f0 f   util_shwapi.obj
 0001:00013230       __remove                   10014230 f   util_shwapi.obj
 0001:00013270       _replace_filename          10014270 f   util_shwapi.obj
 0001:00013370       _replace_extension         10014370 f   util_shwapi.obj
 0001:000134b0       _append_filename           100144b0 f   util_shwapi.obj
 0001:000135a0       _get_filename              100145a0 f   util_shwapi.obj
 0001:00013630       _get_extension             10014630 f   util_shwapi.obj
 0001:000136e0       _put_backslash             100146e0 f   util_shwapi.obj
 0001:00013750       _str_trim                  10014750 f   util_string.obj
 0001:00013790       _str_delete_substr         10014790 f   util_string.obj
 0001:000137e0       _STR_AllocSetString        100147e0 f   util_string.obj
 0001:00013840       _hexVal                    10014840 f   util_string.obj
 0001:00013880       _trimLeft                  10014880 f   util_string.obj
 0001:000138c0       _trimInet                  100148c0 f   util_string.obj
 0001:00013900       _trimRight                 10014900 f   util_string.obj
 0001:00013940       _trimDirSeparator          10014940 f   util_string.obj
 0001:00013980       _trim                      10014980 f   util_string.obj
 0001:000139a0       _splitPath                 100149a0 f   util_string.obj
 0001:00013a50       _getExtension              10014a50 f   util_string.obj
 0001:00013aa0       _translateEscapeString     10014aa0 f   util_string.obj
 0001:00013b90       _translateFilepath         10014b90 f   util_string.obj
 0001:00013bc0       ?cf_init_lowlevel_read_code@@YAXPAUCFILE@@HH@Z 10014bc0 f   cfile.obj
 0001:00013c20       ?cfeof@@YAHPAUCFILE@@@Z    10014c20 f   cfile.obj
 0001:00013c40       ?cftell@@YAHPAUCFILE@@@Z   10014c40 f   cfile.obj
 0001:00013c50       ?cfseek@@YAHPAUCFILE@@HH@Z 10014c50 f   cfile.obj
 0001:00013ce0       ?cfread@@YAHPAXHHPAUCFILE@@@Z 10014ce0 f   cfile.obj
 0001:00013da0       ?cfread_float@@YAMPAUCFILE@@M@Z 10014da0 f   cfile.obj
 0001:00013dd0       ?cfread_int@@YAHPAUCFILE@@H@Z 10014dd0 f   cfile.obj
 0001:00013e00       ?cfread_uint@@YAIPAUCFILE@@I@Z 10014e00 f   cfile.obj
 0001:00013e30       ?cfread_short@@YAFPAUCFILE@@F@Z 10014e30 f   cfile.obj
 0001:00013e60       ?cfread_ushort@@YAGPAUCFILE@@G@Z 10014e60 f   cfile.obj
 0001:00013e90       ?cfread_ubyte@@YAEPAUCFILE@@E@Z 10014e90 f   cfile.obj
 0001:00013ec0       ?cfread_char@@YADPAUCFILE@@D@Z 10014ec0 f   cfile.obj
 0001:00013ef0       ?cfread_string@@YAXPADHPAUCFILE@@@Z 10014ef0 f   cfile.obj
 0001:00013f30       ?cfread_string_len@@YAXPADHPAUCFILE@@@Z 10014f30 f   cfile.obj
 0001:00013f90       ?cfget_cfile_block@@YAPAUCFILE@@XZ 10014f90 f   cfile.obj
 0001:00013fe0       ?cffree_cfile_block@@YAXPAUCFILE@@@Z 10014fe0 f   cfile.obj
 0001:00014030       ?cfilelength@@YAHPAUCFILE@@@Z 10015030 f   cfile.obj
 0001:00014040       ?cfclose@@YAHPAUCFILE@@@Z  10015040 f   cfile.obj
 0001:00014090       ?cf_open_file_cfblock@@YAPAUCFILE@@PAU_iobuf@@H@Z 10015090 f   cfile.obj
 0001:000140c0       ?cf_open_vfs_cfblock@@YAPAUCFILE@@PAXH@Z 100150c0 f   cfile.obj
 0001:00014110       ?cfopen@@YAPAUCFILE@@PAD0H@Z 10015110 f   cfile.obj
 0001:000141b0       ?fixmul@@YAJJJ@Z           100151b0 f   fix.obj
 0001:000141c0       ?fixdiv@@YAJJJ@Z           100151c0 f   fix.obj
 0001:000141e0       ?fixmuldiv@@YAJJJJ@Z       100151e0 f   fix.obj
 0001:00014200       ?fl_isqrt_c@@YAMM@Z        10015200 f   floating.obj
 0001:00014230       ?fl_roundoff@@YAMMH@Z      10015230 f   floating.obj
 0001:00014280       ?frand@@YAMXZ              10015280 f   floating.obj
 0001:000142b0       ?frand_range@@YAMMM@Z      100152b0 f   floating.obj
 0001:000142f0       ?rand_chance@@YAHMM@Z      100152f0 f   floating.obj
 0001:000143a0       _acosf                     100153a0 f i vecmat.obj
 0001:000143c0       _asinf                     100153c0 f i vecmat.obj
 0001:000143e0       _atanf                     100153e0 f i vecmat.obj
 0001:00014400       _cosf                      10015400 f i vecmat.obj
 0001:00014420       _sinf                      10015420 f i vecmat.obj
 0001:00014440       _sqrtf                     10015440 f i vecmat.obj
 0001:00014460       ?acos@@YAMM@Z              10015460 f i vecmat.obj
 0001:00014480       ?asin@@YAMM@Z              10015480 f i vecmat.obj
 0001:000144a0       ?atan@@YAMM@Z              100154a0 f i vecmat.obj
 0001:000144c0       ?cos@@YAMM@Z               100154c0 f i vecmat.obj
 0001:000144e0       ?sin@@YAMM@Z               100154e0 f i vecmat.obj
 0001:00014500       ?sqrt@@YAMM@Z              10015500 f i vecmat.obj
 0001:00014520       ?atan2_safe@@YAMMM@Z       10015520 f   vecmat.obj
 0001:000145b0       ?asqrt@@YAMM@Z             100155b0 f   vecmat.obj
 0001:000145e0       ?vm_set_identity@@YAXPAUmatrix@@@Z 100155e0 f   vecmat.obj
 0001:00014610       ?vm_vec_add@@YAXPAUvector@@00@Z 10015610 f   vecmat.obj
 0001:00014640       ?vm_vec_sub@@YAXPAUvector@@00@Z 10015640 f   vecmat.obj
 0001:00014670       ?vm_vec_add2@@YAXPAUvector@@0@Z 10015670 f   vecmat.obj
 0001:000146a0       ?vm_vec_sub2@@YAXPAUvector@@0@Z 100156a0 f   vecmat.obj
 0001:000146d0       ?vm_vert2vec@@YAXPAUvertex@@PAUvector@@@Z 100156d0 f   vecmat.obj
 0001:000146f0       ?vm_vec2vert@@YAXPAUvector@@PAUvertex@@@Z 100156f0 f   vecmat.obj
 0001:00014710       ?vm_vec_avg_n@@YAPAUvector@@PAU1@HQAU1@@Z 10015710 f   vecmat.obj
 0001:00014840       ?vm_vec_avg@@YAPAUvector@@PAU1@00@Z 10015840 f   vecmat.obj
 0001:00014880       ?vm_vec_avg3@@YAPAUvector@@PAU1@000@Z 10015880 f   vecmat.obj
 0001:000148d0       ?vm_vec_avg4@@YAPAUvector@@PAU1@0000@Z 100158d0 f   vecmat.obj
 0001:00014920       ?vm_vec_scale@@YAXPAUvector@@M@Z 10015920 f   vecmat.obj
 0001:00014950       ?vm_vec_copy_scale@@YAXPAUvector@@0M@Z 10015950 f   vecmat.obj
 0001:00014980       ?vm_vec_scale_add@@YAXPAUvector@@00M@Z 10015980 f   vecmat.obj
 0001:000149c0       ?vm_vec_scale_add2@@YAXPAUvector@@0M@Z 100159c0 f   vecmat.obj
 0001:000149f0       ?vm_vec_scale_sub2@@YAXPAUvector@@0M@Z 100159f0 f   vecmat.obj
 0001:00014a30       ?vm_vec_scale2@@YAXPAUvector@@MM@Z 10015a30 f   vecmat.obj
 0001:00014a70       ?vm_vec_dotprod@@YAMPAUvector@@0@Z 10015a70 f   vecmat.obj
 0001:00014aa0       ?vm_vec_dot3@@YAMMMMPAUvector@@@Z 10015aa0 f   vecmat.obj
 0001:00014ad0       ?vm_vec_mag@@YAMPAUvector@@@Z 10015ad0 f   vecmat.obj
 0001:00014b30       ?vm_vec_mag_squared@@YAMPAUvector@@@Z 10015b30 f   vecmat.obj
 0001:00014b70       ?vm_vec_dist_squared@@YAMPAUvector@@0@Z 10015b70 f   vecmat.obj
 0001:00014bc0       ?vm_vec_dist@@YAMPAUvector@@0@Z 10015bc0 f   vecmat.obj
 0001:00014c00       ?vm_vec_mag_quick@@YAMPAUvector@@@Z 10015c00 f   vecmat.obj
 0001:00014cf0       ?vm_vec_dist_quick@@YAMPAUvector@@0@Z 10015cf0 f   vecmat.obj
 0001:00014d30       ?vm_vec_copy_normalize@@YAMPAUvector@@0@Z 10015d30 f   vecmat.obj
 0001:00014db0       ?vm_vec_normalize@@YAMPAUvector@@@Z 10015db0 f   vecmat.obj
 0001:00014dc0       ?vm_vec_normalize_safe@@YAMPAUvector@@@Z 10015dc0 f   vecmat.obj
 0001:00014e20       ?vm_vec_imag@@YAMPAUvector@@@Z 10015e20 f   vecmat.obj
 0001:00014e60       ?vm_vec_copy_normalize_quick@@YAMPAUvector@@0@Z 10015e60 f   vecmat.obj
 0001:00014ed0       ?vm_vec_normalize_quick@@YAMPAUvector@@@Z 10015ed0 f   vecmat.obj
 0001:00014f40       ?vm_vec_copy_normalize_quick_mag@@YAMPAUvector@@0@Z 10015f40 f   vecmat.obj
 0001:00014f80       ?vm_vec_normalize_quick_mag@@YAMPAUvector@@@Z 10015f80 f   vecmat.obj
 0001:00014fb0       ?vm_vec_normalized_dir@@YAMPAUvector@@00@Z 10015fb0 f   vecmat.obj
 0001:00014fe0       ?vm_vec_normalized_dir_quick@@YAMPAUvector@@00@Z 10015fe0 f   vecmat.obj
 0001:00015010       ?vm_vec_normalized_dir_quick_mag@@YAMPAUvector@@00@Z 10016010 f   vecmat.obj
 0001:00015060       ?vm_vec_crossprod@@YAPAUvector@@PAU1@00@Z 10016060 f   vecmat.obj
 0001:000150a0       ?vm_test_parallel@@YAHPAUvector@@0@Z 100160a0 f   vecmat.obj
 0001:00015110       ?vm_vec_perp@@YAPAUvector@@PAU1@000@Z 10016110 f   vecmat.obj
 0001:000151b0       ?vm_vec_delta_ang_norm@@YAMPAUvector@@00@Z 100161b0 f   vecmat.obj
 0001:00015270       ?sincos_2_matrix@@YAPAUmatrix@@PAU1@MMMMMM@Z 10016270 f   vecmat.obj
 0001:00015320       ?vm_angles_2_matrix@@YAPAUmatrix@@PAU1@PAUangles@@@Z 10016320 f   vecmat.obj
 0001:000153e0       ?vm_angle_2_matrix@@YAPAUmatrix@@PAU1@MH@Z 100163e0 f   vecmat.obj
 0001:000154f0       ?vm_vec_ang_2_matrix@@YAPAUmatrix@@PAU1@PAUvector@@M@Z 100164f0 f   vecmat.obj
 0001:000155a0       ?vm_vector_2_matrix@@YAPAUmatrix@@PAU1@PAUvector@@11@Z 100165a0 f   vecmat.obj
 0001:00015720       ?vm_vector_2_matrix_norm@@YAPAUmatrix@@PAU1@PAUvector@@11@Z 10016720 f   vecmat.obj
 0001:00015890       ?vm_vec_rotate@@YAPAUvector@@PAU1@0PAUmatrix@@@Z 10016890 f   vecmat.obj
 0001:000158f0       ?vm_vec_unrotate@@YAPAUvector@@PAU1@0PAUmatrix@@@Z 100168f0 f   vecmat.obj
 0001:00015950       ?vm_transpose_matrix@@YAPAUmatrix@@PAU1@@Z 10016950 f   vecmat.obj
 0001:000159a0       ?vm_copy_transpose_matrix@@YAPAUmatrix@@PAU1@0@Z 100169a0 f   vecmat.obj
 0001:000159e0       ?vm_matrix_x_matrix@@YAPAUmatrix@@PAU1@00@Z 100169e0 f   vecmat.obj
 0001:00015ad0       ?vm_extract_angles_matrix@@YAPAUangles@@PAU1@PAUmatrix@@@Z 10016ad0 f   vecmat.obj
 0001:00015c40       ?vm_extract_angles_vector_normalized@@YAPAUangles@@PAU1@PAUvector@@@Z 10016c40 f   vecmat.obj
 0001:00015ca0       ?vm_extract_angles_vector@@YAPAUangles@@PAU1@PAUvector@@@Z 10016ca0 f   vecmat.obj
 0001:00015cf0       ?vm_dist_to_plane@@YAMPAUvector@@00@Z 10016cf0 f   vecmat.obj
 0001:00015d40       ?vm_trackball@@YAXHHPAUmatrix@@@Z 10016d40 f   vecmat.obj
 0001:00015e70       ?vm_vec_outer_product@@YAXPAUmatrix@@PAUvector@@@Z 10016e70 f   vecmat.obj
 0001:00015ed0       ?find_nearest_point_on_line@@YAMPAUvector@@000@Z 10016ed0 f   vecmat.obj
 0001:000160a0       ?vm_orthogonalize_matrix@@YAXPAUmatrix@@@Z 100170a0 f   vecmat.obj
 0001:00016240       ?vm_fix_matrix@@YAXPAUmatrix@@@Z 10017240 f   vecmat.obj
 0001:00016410       ?vm_rotate_matrix_by_angles@@YAXPAUmatrix@@PAUangles@@@Z 10017410 f   vecmat.obj
 0001:00016460       ?vm_vec_dot_to_point@@YAMPAUvector@@00@Z 10017460 f   vecmat.obj
 0001:000164c0       ?compute_point_on_plane@@YAXPAUvector@@PAUplane@@0@Z 100174c0 f   vecmat.obj
 0001:00016570       ?vm_vec_rand_vec_quick@@YAXPAUvector@@@Z 10017570 f   vecmat.obj
 0001:000165f0       ?vm_rot_point_around_line@@YAXPAUvector@@0M00@Z 100175f0 f   vecmat.obj
 0001:00016870       ?vm_vec_cmp@@YAHPAUvector@@0@Z 10017870 f   vecmat.obj
 0001:000168c0       ?vm_matrix_cmp@@YAHPAUmatrix@@0@Z 100178c0 f   vecmat.obj
 0001:00016980       ?vm_interp_angle@@YAXPAMMM@Z 10017980 f   vecmat.obj
 0001:00016a60       ?vm_check_matrix_for_zeros@@YAHPAUmatrix@@@Z 10017a60 f   vecmat.obj
 0001:00016b30       ?vm_vec_same@@YAHPAUvector@@0@Z 10017b30 f   vecmat.obj
 0001:00016b70       ?vm_quaternion_rotate@@YAXPAUmatrix@@MPAUvector@@@Z 10017b70 f   vecmat.obj
 0001:00016c60       ?rotate_z@@YAXPAUmatrix@@M@Z 10017c60 f   vecmat.obj
 0001:00016cd0       ?vm_matrix_to_rot_axis_and_angle@@YAXPAUmatrix@@PAMPAUvector@@@Z 10017cd0 f   vecmat.obj
 0001:00016ec0       ?approach@@YAMMMMMMPAMH@Z  10017ec0 f   vecmat.obj
 0001:00017310       ?away@@YAMMMMMMPAMH@Z      10018310 f   vecmat.obj
 0001:00017430       ?vm_matrix_interpolate@@YAXPAUmatrix@@0PAUvector@@M0111H@Z 10018430 f   vecmat.obj
 0001:00017980       ?get_camera_limits@@YAXPAUmatrix@@0MPAUvector@@1@Z 10018980 f   vecmat.obj
 0001:00017ae0       ?vm_fvec_matrix_interpolate@@YAXPAUmatrix@@0PAUvector@@M0111H@Z 10018ae0 f   vecmat.obj
 0001:00018380       ?vm_forward_interpolate@@YAXPAUvector@@PAUmatrix@@0MM1000H@Z 10019380 f   vecmat.obj
 0001:00018a90       ?vm_find_bounding_sphere@@YAXPAUvector@@H0PAM@Z 10019a90 f   vecmat.obj
 0001:00019370       ?vm_rotate_vec_to_body@@YAPAUvector@@PAU1@0PAUmatrix@@@Z 1001a370 f   vecmat.obj
 0001:000193d0       ?vm_rotate_vec_to_world@@YAPAUvector@@PAU1@0PAUmatrix@@@Z 1001a3d0 f   vecmat.obj
 0001:00019430       ?vm_estimate_next_orientation@@YAXPAUmatrix@@00@Z 1001a430 f   vecmat.obj
 0001:000194b0       ?is_valid_vec@@YAHPAUvector@@@Z 1001a4b0 f   vecmat.obj
 0001:00019500       ?is_valid_matrix@@YAHPAUmatrix@@@Z 1001a500 f   vecmat.obj
 0001:00019540       ?vm_vec_interp_constant@@YAXPAUvector@@00M@Z 1001a540 f   vecmat.obj
 0001:000195f0       ?vm_vec_random_cone@@YAXPAUvector@@0MPAUmatrix@@@Z 1001a5f0 f   vecmat.obj
 0001:00019710       ?vm_vec_random_in_circle@@YAXPAUvector@@0PAUmatrix@@MH@Z 1001a710 f   vecmat.obj
 0001:000197c0       ?vm_vec_dist_to_line@@YAHPAUvector@@000PAM@Z 1001a7c0 f   vecmat.obj
 0001:00019900       ?vm_vec_dist_squared_to_line@@YAXPAUvector@@000PAM@Z 1001a900 f   vecmat.obj
 0001:00019a10       ?vm_vec_projection_parallel@@YAMPAUvector@@00@Z 1001aa10 f   vecmat.obj
 0001:00019a60       ?vm_vec_projection_onto_plane@@YAXPAUvector@@00@Z 1001aa60 f   vecmat.obj
 0001:00019ad0       ?vm_project_point_onto_plane@@YAXPAUvector@@000@Z 1001aad0 f   vecmat.obj
 0001:00019b70       ?vm_vec_normal@@YAPAUvector@@PAU1@000@Z 1001ab70 f   vecmat.obj
 0001:00019ba0       ?vm_vec_delta_ang@@YAMPAUvector@@00@Z 1001aba0 f   vecmat.obj
 0001:00019bf0       ?myrand@@YAHXZ             1001abf0 f   systemvars.obj
 0001:00019c00       ?ole2_bufread@@YAXPAUOLE2Stream@@@Z 1001ac00 f   ole.obj
 0001:00019c90       ?ole2_read@@YAHPAXJJPAUOLE2Stream@@@Z 1001ac90 f   ole.obj
 0001:00019d60       ?ole2_sopen@@YAPAUOLE2Stream@@PAUOLE2@@K@Z 1001ad60 f   ole.obj
 0001:00019db0       ?ole2_seek@@YAXPAUOLE2Stream@@K@Z 1001adb0 f   ole.obj
 0001:00019e10       ?ole2_fopen@@YAPAUOLE2Stream@@PAUOLE2@@PAD@Z 1001ae10 f   ole.obj
 0001:00019ed0       ?ole2_open@@YAPAUOLE2@@PAD@Z 1001aed0 f   ole.obj
 0001:0001a280       ?ole2_close@@YAXPAUOLE2@@@Z 1001b280 f   ole.obj
 0001:0001a2c0       ?ole2_fclose@@YAXPAUOLE2Stream@@@Z 1001b2c0 f   ole.obj
 0001:0001a2d0       ?find@?$char_traits@D@std@@SAPBDPBDIABD@Z 1001b2d0 f i xls.obj
 0001:0001a2f0       ?xls@@YAHXZ                1001b2f0 f   xls.obj
 0001:0001a300       ?xls_appendSST@@YAXPAUxlsWorkBook@@PAEK@Z 1001b300 f   xls.obj
 0001:0001a500       ?NumFromRk@@YANPAE@Z       1001b500 f   xls.obj
 0001:0001a550       ?xls_addSheet@@YAXPAUxlsWorkBook@@PAE@Z 1001b550 f   xls.obj
 0001:0001a5f0       ?xls_addRow@@YAXPAUxlsWorkSheet@@PAUROW@@@Z 1001b5f0 f   xls.obj
 0001:0001a650       ?xls_makeTable@@YAXPAUxlsWorkSheet@@@Z 1001b650 f   xls.obj
 0001:0001a750       ?xls_addCell@@YAXPAUxlsWorkSheet@@PAUBOF@@PAE@Z 1001b750 f   xls.obj
 0001:0001a970       ?xls_addFont@@YAXPAUxlsWorkBook@@PAUFONT@@@Z 1001b970 f   xls.obj
 0001:0001aa10       ?xls_addXF@@YAXPAUxlsWorkBook@@PAUXF@@@Z 1001ba10 f   xls.obj
 0001:0001aab0       ?xls_addColinfo@@YAXPAUxlsWorkSheet@@PAUCOLINFO@@@Z 1001bab0 f   xls.obj
 0001:0001ab30       ?xls_mergedCells@@YAXPAUxlsWorkSheet@@PAUBOF@@PAE@Z 1001bb30 f   xls.obj
 0001:0001ac30       ?xls_preparseWorkSheet@@YAXPAUxlsWorkSheet@@@Z 1001bc30 f   xls.obj
 0001:0001ad00       ?xls_formatColumn@@YAXPAUxlsWorkSheet@@@Z 1001bd00 f   xls.obj
 0001:0001add0       ?xls_parseWorkSheet@@YAXPAUxlsWorkSheet@@@Z 1001bdd0 f   xls.obj
 0001:0001afd0       ?xls_getWorkSheet@@YAPAUxlsWorkSheet@@PAUxlsWorkBook@@H@Z 1001bfd0 f   xls.obj
 0001:0001b010       ?xls_close@@YAXPAUxlsWorkBook@@@Z 1001c010 f   xls.obj
 0001:0001b040       ?capacity@?$vector@V?$basic_string@DU?$char_traits@D@std@@V?$allocator@D@2@@std@@V?$allocator@V?$basic_string@DU?$char_traits@D@std@@V?$allocator@D@2@@std@@@2@@std@@QBEIXZ 1001c040 f i xls.obj
 0001:0001b070       ??0?$allocator@V?$basic_string@DU?$char_traits@D@std@@V?$allocator@D@2@@std@@@std@@QAE@XZ 1001c070 f i xls.obj
 0001:0001b080       ?capacity@?$vector@UST_CELLS@@V?$allocator@UST_CELLS@@@std@@@std@@QBEIXZ 1001c080 f i xls.obj
 0001:0001b0a0       ??0?$allocator@V?$basic_string@DU?$char_traits@D@std@@V?$allocator@D@2@@std@@@std@@QAE@ABV01@@Z 1001c0a0 f i xls.obj
 0001:0001b0b0       ??G?$_Vector_const_iterator@V?$basic_string@DU?$char_traits@D@std@@V?$allocator@D@2@@std@@V?$allocator@V?$basic_string@DU?$char_traits@D@std@@V?$allocator@D@2@@std@@@2@@std@@QBEHABV01@@Z 1001c0b0 f i xls.obj
 0001:0001b0f0       ??G?$_Vector_const_iterator@UST_CELLS@@V?$allocator@UST_CELLS@@@std@@@std@@QBEHABV01@@Z 1001c0f0 f i xls.obj
 0001:0001b130       ?max_size@?$allocator@V?$basic_string@DU?$char_traits@D@std@@V?$allocator@D@2@@std@@@std@@QBEIXZ 1001c130 f i xls.obj
 0001:0001b140       ??0?$_Iterator_with_base@Urandom_access_iterator_tag@std@@V?$basic_string@DU?$char_traits@D@std@@V?$allocator@D@2@@2@HPBV32@ABV32@V_Iterator_base_aux@2@@std@@QAE@XZ 1001c140 f i xls.obj
 0001:0001b150       ??0?$_Iterator_with_base@Urandom_access_iterator_tag@std@@UST_CELLS@@HPBU3@ABU3@V_Iterator_base_aux@2@@std@@QAE@XZ 1001c150 f i xls.obj
 0001:0001b160       ??Y?$_Vector_const_iterator@V?$basic_string@DU?$char_traits@D@std@@V?$allocator@D@2@@std@@V?$allocator@V?$basic_string@DU?$char_traits@D@std@@V?$allocator@D@2@@std@@@2@@std@@QAEAAV01@H@Z 1001c160 f i xls.obj
 0001:0001b1c0       ??Y?$_Vector_const_iterator@UST_CELLS@@V?$allocator@UST_CELLS@@@std@@@std@@QAEAAV01@H@Z 1001c1c0 f i xls.obj
 0001:0001b210       ??$?0V?$basic_string@DU?$char_traits@D@std@@V?$allocator@D@2@@std@@@?$allocator@V_Aux_cont@std@@@std@@QAE@ABV?$allocator@V?$basic_string@DU?$char_traits@D@std@@V?$allocator@D@2@@std@@@1@@Z 1001c210 f i xls.obj
 0001:0001b220       ??$_Allocate@V?$basic_string@DU?$char_traits@D@std@@V?$allocator@D@2@@std@@@std@@YAPAV?$basic_string@DU?$char_traits@D@std@@V?$allocator@D@2@@0@IPAV10@@Z 1001c220 f i xls.obj
 0001:0001b290       ??$_Iter_random@PAV?$basic_string@DU?$char_traits@D@std@@V?$allocator@D@2@@std@@PAV12@@std@@YA?AUrandom_access_iterator_tag@0@ABQAV?$basic_string@DU?$char_traits@D@std@@V?$allocator@D@2@@0@0@Z 1001c290 f i xls.obj
 0001:0001b2a0       ??$_Move_cat@PAV?$basic_string@DU?$char_traits@D@std@@V?$allocator@D@2@@std@@@std@@YA?AU_Swap_move_tag@0@ABQAV?$basic_string@DU?$char_traits@D@std@@V?$allocator@D@2@@0@@Z 1001c2a0 f i xls.obj
 0001:0001b2b0       ??$_Iter_random@PAUST_CELLS@@PAU1@@std@@YA?AUrandom_access_iterator_tag@0@ABQAUST_CELLS@@0@Z 1001c2b0 f i xls.obj
 0001:0001b2c0       ??$_Move_cat@PAUST_CELLS@@@std@@YA?AU_Undefined_move_tag@0@ABQAUST_CELLS@@@Z 1001c2c0 f i xls.obj
 0001:0001b2d0       ??8?$_Vector_const_iterator@V?$basic_string@DU?$char_traits@D@std@@V?$allocator@D@2@@std@@V?$allocator@V?$basic_string@DU?$char_traits@D@std@@V?$allocator@D@2@@std@@@2@@std@@QBE_NABV01@@Z 1001c2d0 f i xls.obj
 0001:0001b300       ??$_Checked_base@PAV?$basic_string@DU?$char_traits@D@std@@V?$allocator@D@2@@std@@@std@@YAPAV?$basic_string@DU?$char_traits@D@std@@V?$allocator@D@2@@0@AAPAV10@U_Unchanged_checked_iterator_base_type_tag@0@@Z 1001c300 f i xls.obj
 0001:0001b310       ??$_Checked_base@PAUST_CELLS@@@std@@YAPAUST_CELLS@@AAPAU1@U_Unchanged_checked_iterator_base_type_tag@0@@Z 1001c310 f i xls.obj
 0001:0001b320       ??$_Ptr_cat@V?$_Vector_const_iterator@V?$basic_string@DU?$char_traits@D@std@@V?$allocator@D@2@@std@@V?$allocator@V?$basic_string@DU?$char_traits@D@std@@V?$allocator@D@2@@std@@@2@@std@@PAV?$basic_string@DU?$char_traits@D@std@@V?$allocator@D@2@@2@@std@@YA?AU_Nonscalar_ptr_iterator_tag@0@AAV?$_Vector_const_iterator@V?$basic_string@DU?$char_traits@D@std@@V?$allocator@D@2@@std@@V?$allocator@V?$basic_string@DU?$char_traits@D@std@@V?$allocator@D@2@@std@@@2@@0@AAPAV?$basic_string@DU?$char_traits@D@std@@V?$allocator@D@2@@0@@Z 1001c320 f i xls.obj
 0001:0001b330       ?_Checked_iterator_base@?$_Vector_const_iterator@V?$basic_string@DU?$char_traits@D@std@@V?$allocator@D@2@@std@@V?$allocator@V?$basic_string@DU?$char_traits@D@std@@V?$allocator@D@2@@std@@@2@@std@@QBEPBV?$basic_string@DU?$char_traits@D@std@@V?$allocator@D@2@@2@XZ 1001c330 f i xls.obj
 0001:0001b340       ??$?8DD@std@@YA_NABV?$allocator@D@0@0@Z 1001c340 f i xls.obj
 0001:0001b350       ?xls_addSST@@YAXPAUxlsWorkBook@@PAUSST@@K@Z 1001c350 f   xls.obj
 0001:0001b3a0       ?xls_parseWorkBook@@YAXPAUxlsWorkBook@@@Z 1001c3a0 f   xls.obj
 0001:0001b540       ?xls_open@@YAPAUxlsWorkBook@@PAD0@Z 1001c540 f   xls.obj
 0001:0001b600       ?find@?$basic_string@DU?$char_traits@D@std@@V?$allocator@D@2@@std@@QBEIPBDII@Z 1001c600 f i xls.obj
 0001:0001b6c0       ?get_allocator@?$basic_string@DU?$char_traits@D@std@@V?$allocator@D@2@@std@@QBE?AV?$allocator@D@2@XZ 1001c6c0 f i xls.obj
 0001:0001b6d0       ?max_size@?$vector@V?$basic_string@DU?$char_traits@D@std@@V?$allocator@D@2@@std@@V?$allocator@V?$basic_string@DU?$char_traits@D@std@@V?$allocator@D@2@@std@@@2@@std@@QBEIXZ 1001c6d0 f i xls.obj
 0001:0001b6e0       ?allocate@?$allocator@V?$basic_string@DU?$char_traits@D@std@@V?$allocator@D@2@@std@@@std@@QAEPAV?$basic_string@DU?$char_traits@D@std@@V?$allocator@D@2@@2@I@Z 1001c6e0 f i xls.obj
 0001:0001b700       ??Y?$_Vector_iterator@V?$basic_string@DU?$char_traits@D@std@@V?$allocator@D@2@@std@@V?$allocator@V?$basic_string@DU?$char_traits@D@std@@V?$allocator@D@2@@std@@@2@@std@@QAEAAV01@H@Z 1001c700 f i xls.obj
 0001:0001b720       ??Y?$_Vector_iterator@UST_CELLS@@V?$allocator@UST_CELLS@@@std@@@std@@QAEAAV01@H@Z 1001c720 f i xls.obj
 0001:0001b740       ??0?$_Ranit@V?$basic_string@DU?$char_traits@D@std@@V?$allocator@D@2@@std@@HPBV12@ABV12@@std@@QAE@XZ 1001c740 f i xls.obj
 0001:0001b750       ??0?$_Ranit@UST_CELLS@@HPBU1@ABU1@@std@@QAE@XZ 1001c750 f i xls.obj
 0001:0001b760       ??$_Checked_base@PAV?$basic_string@DU?$char_traits@D@std@@V?$allocator@D@2@@std@@@std@@YAPAV?$basic_string@DU?$char_traits@D@std@@V?$allocator@D@2@@0@AAPAV10@@Z 1001c760 f i xls.obj
 0001:0001b770       ??$_Checked_base@PAUST_CELLS@@@std@@YAPAUST_CELLS@@AAPAU1@@Z 1001c770 f i xls.obj
 0001:0001b780       ??9?$_Vector_const_iterator@V?$basic_string@DU?$char_traits@D@std@@V?$allocator@D@2@@std@@V?$allocator@V?$basic_string@DU?$char_traits@D@std@@V?$allocator@D@2@@std@@@2@@std@@QBE_NABV01@@Z 1001c780 f i xls.obj
 0001:0001b7b0       ??$_Checked_base@V?$_Vector_const_iterator@V?$basic_string@DU?$char_traits@D@std@@V?$allocator@D@2@@std@@V?$allocator@V?$basic_string@DU?$char_traits@D@std@@V?$allocator@D@2@@std@@@2@@std@@U_Different_checked_iterator_base_type_tag@2@@std@@YAPBV?$basic_string@DU?$char_traits@D@std@@V?$allocator@D@2@@0@AAV?$_Vector_const_iterator@V?$basic_string@DU?$char_traits@D@std@@V?$allocator@D@2@@std@@V?$allocator@V?$basic_string@DU?$char_traits@D@std@@V?$allocator@D@2@@std@@@2@@0@U_Different_checked_iterator_base_type_tag@0@@Z 1001c7b0 f i xls.obj
 0001:0001b7c0       ?find@?$basic_string@DU?$char_traits@D@std@@V?$allocator@D@2@@std@@QBEIPBDI@Z 1001c7c0 f i xls.obj
 0001:0001b7f0       ??0?$_Container_base_aux_alloc_real@V?$allocator@V?$basic_string@DU?$char_traits@D@std@@V?$allocator@D@2@@std@@@std@@@std@@IAE@V?$allocator@V?$basic_string@DU?$char_traits@D@std@@V?$allocator@D@2@@std@@@1@@Z 1001c7f0 f i xls.obj
 0001:0001b820       ??H?$_Vector_iterator@V?$basic_string@DU?$char_traits@D@std@@V?$allocator@D@2@@std@@V?$allocator@V?$basic_string@DU?$char_traits@D@std@@V?$allocator@D@2@@std@@@2@@std@@QBE?AV01@H@Z 1001c820 f i xls.obj
 0001:0001b860       ??H?$_Vector_iterator@UST_CELLS@@V?$allocator@UST_CELLS@@@std@@@std@@QBE?AV01@H@Z 1001c860 f i xls.obj
 0001:0001b8b0       ??0?$_Vector_const_iterator@V?$basic_string@DU?$char_traits@D@std@@V?$allocator@D@2@@std@@V?$allocator@V?$basic_string@DU?$char_traits@D@std@@V?$allocator@D@2@@std@@@2@@std@@QAE@PAV?$basic_string@DU?$char_traits@D@std@@V?$allocator@D@2@@1@PBV_Container_base_aux@1@@Z 1001c8b0 f i xls.obj
 0001:0001b8f0       ??0?$_Vector_const_iterator@UST_CELLS@@V?$allocator@UST_CELLS@@@std@@@std@@QAE@PAUST_CELLS@@PBV_Container_base_aux@1@@Z 1001c8f0 f i xls.obj
 0001:0001b930       ?begin@?$vector@V?$basic_string@DU?$char_traits@D@std@@V?$allocator@D@2@@std@@V?$allocator@V?$basic_string@DU?$char_traits@D@std@@V?$allocator@D@2@@std@@@2@@std@@QBE?AV?$_Vector_const_iterator@V?$basic_string@DU?$char_traits@D@std@@V?$allocator@D@2@@std@@V?$allocator@V?$basic_string@DU?$char_traits@D@std@@V?$allocator@D@2@@std@@@2@@2@XZ 1001c930 f i xls.obj
 0001:0001b960       ?end@?$vector@V?$basic_string@DU?$char_traits@D@std@@V?$allocator@D@2@@std@@V?$allocator@V?$basic_string@DU?$char_traits@D@std@@V?$allocator@D@2@@std@@@2@@std@@QBE?AV?$_Vector_const_iterator@V?$basic_string@DU?$char_traits@D@std@@V?$allocator@D@2@@std@@V?$allocator@V?$basic_string@DU?$char_traits@D@std@@V?$allocator@D@2@@std@@@2@@2@XZ 1001c960 f i xls.obj
 0001:0001b990       ??$_Checked_base@V?$_Vector_const_iterator@V?$basic_string@DU?$char_traits@D@std@@V?$allocator@D@2@@std@@V?$allocator@V?$basic_string@DU?$char_traits@D@std@@V?$allocator@D@2@@std@@@2@@std@@@std@@YAPBV?$basic_string@DU?$char_traits@D@std@@V?$allocator@D@2@@0@AAV?$_Vector_const_iterator@V?$basic_string@DU?$char_traits@D@std@@V?$allocator@D@2@@std@@V?$allocator@V?$basic_string@DU?$char_traits@D@std@@V?$allocator@D@2@@std@@@2@@0@@Z 1001c990 f i xls.obj
 0001:0001b9a0       ??0?$basic_string@DU?$char_traits@D@std@@V?$allocator@D@2@@std@@QAE@XZ 1001c9a0 f i xls.obj
 0001:0001b9c0       ??0?$_Vector_val@V?$basic_string@DU?$char_traits@D@std@@V?$allocator@D@2@@std@@V?$allocator@V?$basic_string@DU?$char_traits@D@std@@V?$allocator@D@2@@std@@@2@@std@@IAE@V?$allocator@V?$basic_string@DU?$char_traits@D@std@@V?$allocator@D@2@@std@@@1@@Z 1001c9c0 f i xls.obj
 0001:0001b9f0       ??0?$_Vector_iterator@V?$basic_string@DU?$char_traits@D@std@@V?$allocator@D@2@@std@@V?$allocator@V?$basic_string@DU?$char_traits@D@std@@V?$allocator@D@2@@std@@@2@@std@@QAE@PAV?$basic_string@DU?$char_traits@D@std@@V?$allocator@D@2@@1@PBV_Container_base_aux@1@@Z 1001c9f0 f i xls.obj
 0001:0001ba30       ??0?$_Vector_iterator@UST_CELLS@@V?$allocator@UST_CELLS@@@std@@@std@@QAE@PAUST_CELLS@@PBV_Container_base_aux@1@@Z 1001ca30 f i xls.obj
 0001:0001ba70       ?_Make_iter@?$vector@V?$basic_string@DU?$char_traits@D@std@@V?$allocator@D@2@@std@@V?$allocator@V?$basic_string@DU?$char_traits@D@std@@V?$allocator@D@2@@std@@@2@@std@@QBE?AV?$_Vector_iterator@V?$basic_string@DU?$char_traits@D@std@@V?$allocator@D@2@@std@@V?$allocator@V?$basic_string@DU?$char_traits@D@std@@V?$allocator@D@2@@std@@@2@@2@V?$_Vector_const_iterator@V?$basic_string@DU?$char_traits@D@std@@V?$allocator@D@2@@std@@V?$allocator@V?$basic_string@DU?$char_traits@D@std@@V?$allocator@D@2@@std@@@2@@2@@Z 1001ca70 f i xls.obj
 0001:0001bab0       ?IsRows@@YAHV?$basic_string@DU?$char_traits@D@std@@V?$allocator@D@2@@std@@@Z 1001cab0 f   xls.obj
 0001:0001bb20       ?end@?$vector@V?$basic_string@DU?$char_traits@D@std@@V?$allocator@D@2@@std@@V?$allocator@V?$basic_string@DU?$char_traits@D@std@@V?$allocator@D@2@@std@@@2@@std@@QAE?AV?$_Vector_iterator@V?$basic_string@DU?$char_traits@D@std@@V?$allocator@D@2@@std@@V?$allocator@V?$basic_string@DU?$char_traits@D@std@@V?$allocator@D@2@@std@@@2@@2@XZ 1001cb20 f i xls.obj
 0001:0001bb50       ?end@?$vector@UST_CELLS@@V?$allocator@UST_CELLS@@@std@@@std@@QAE?AV?$_Vector_iterator@UST_CELLS@@V?$allocator@UST_CELLS@@@std@@@2@XZ 1001cb50 f i xls.obj
 0001:0001bb80       ?append@?$basic_string@DU?$char_traits@D@std@@V?$allocator@D@2@@std@@QAEAAV12@ABV12@II@Z 1001cb80 f i xls.obj
 0001:0001bc80       ?append@?$basic_string@DU?$char_traits@D@std@@V?$allocator@D@2@@std@@QAEAAV12@PBDI@Z 1001cc80 f i xls.obj
 0001:0001bd90       ?begin@?$vector@V?$basic_string@DU?$char_traits@D@std@@V?$allocator@D@2@@std@@V?$allocator@V?$basic_string@DU?$char_traits@D@std@@V?$allocator@D@2@@std@@@2@@std@@QAE?AV?$_Vector_iterator@V?$basic_string@DU?$char_traits@D@std@@V?$allocator@D@2@@std@@V?$allocator@V?$basic_string@DU?$char_traits@D@std@@V?$allocator@D@2@@std@@@2@@2@XZ 1001cd90 f i xls.obj
 0001:0001bdc0       ?begin@?$vector@UST_CELLS@@V?$allocator@UST_CELLS@@@std@@@std@@QAE?AV?$_Vector_iterator@UST_CELLS@@V?$allocator@UST_CELLS@@@std@@@2@XZ 1001cdc0 f i xls.obj
 0001:0001bdf0       ??0?$basic_string@DU?$char_traits@D@std@@V?$allocator@D@2@@std@@QAE@ABV01@IIABV?$allocator@D@1@@Z 1001cdf0 f i xls.obj
 0001:0001be20       ?append@?$basic_string@DU?$char_traits@D@std@@V?$allocator@D@2@@std@@QAEAAV12@ABV12@@Z 1001ce20 f i xls.obj
 0001:0001be40       ?append@?$basic_string@DU?$char_traits@D@std@@V?$allocator@D@2@@std@@QAEAAV12@PBD@Z 1001ce40 f i xls.obj
 0001:0001be70       ??$_Construct@V?$basic_string@DU?$char_traits@D@std@@V?$allocator@D@2@@std@@V12@@std@@YAXPAV?$basic_string@DU?$char_traits@D@std@@V?$allocator@D@2@@0@ABV10@@Z 1001ce70 f i xls.obj
 0001:0001bee0       ??$_Copy_opt@PAV?$basic_string@DU?$char_traits@D@std@@V?$allocator@D@2@@std@@PAV12@Uforward_iterator_tag@2@@std@@YAPAV?$basic_string@DU?$char_traits@D@std@@V?$allocator@D@2@@0@PAV10@00Uforward_iterator_tag@0@U_Nonscalar_ptr_iterator_tag@0@U_Range_checked_iterator_tag@0@@Z 1001cee0 f i xls.obj
 0001:0001bf20       ?swap@?$basic_string@DU?$char_traits@D@std@@V?$allocator@D@2@@std@@QAEXAAV12@@Z 1001cf20 f i xls.obj
 0001:0001bfa0       ??4?$basic_string@DU?$char_traits@D@std@@V?$allocator@D@2@@std@@QAEAAV01@PBD@Z 1001cfa0 f i xls.obj
 0001:0001bfd0       ??Y?$basic_string@DU?$char_traits@D@std@@V?$allocator@D@2@@std@@QAEAAV01@ABV01@@Z 1001cfd0 f i xls.obj
 0001:0001bff0       ??Y?$basic_string@DU?$char_traits@D@std@@V?$allocator@D@2@@std@@QAEAAV01@PBD@Z 1001cff0 f i xls.obj
 0001:0001c020       ?substr@?$basic_string@DU?$char_traits@D@std@@V?$allocator@D@2@@std@@QBE?AV12@II@Z 1001d020 f i xls.obj
 0001:0001c060       ?_Xlen@?$vector@V?$basic_string@DU?$char_traits@D@std@@V?$allocator@D@2@@std@@V?$allocator@V?$basic_string@DU?$char_traits@D@std@@V?$allocator@D@2@@std@@@2@@std@@KAXXZ 1001d060 f i xls.obj
 0001:0001c0e0       ??$_Fill@PAV?$basic_string@DU?$char_traits@D@std@@V?$allocator@D@2@@std@@V12@@std@@YAXPAV?$basic_string@DU?$char_traits@D@std@@V?$allocator@D@2@@0@0ABV10@@Z 1001d0e0 f i xls.obj
 0001:0001c110       ?construct@?$allocator@V?$basic_string@DU?$char_traits@D@std@@V?$allocator@D@2@@std@@@std@@QAEXPAV?$basic_string@DU?$char_traits@D@std@@V?$allocator@D@2@@2@ABV32@@Z 1001d110 f i xls.obj
 0001:0001c130       ??$_Uninit_copy@PBV?$basic_string@DU?$char_traits@D@std@@V?$allocator@D@2@@std@@PAV12@V?$allocator@V?$basic_string@DU?$char_traits@D@std@@V?$allocator@D@2@@std@@@2@@std@@YAPAV?$basic_string@DU?$char_traits@D@std@@V?$allocator@D@2@@0@PBV10@0PAV10@AAV?$allocator@V?$basic_string@DU?$char_traits@D@std@@V?$allocator@D@2@@std@@@0@U_Nonscalar_ptr_iterator_tag@0@U_Range_checked_iterator_tag@0@@Z 1001d130 f i xls.obj
 0001:0001c1f0       ??$_Copy_opt@PAV?$basic_string@DU?$char_traits@D@std@@V?$allocator@D@2@@std@@PAV12@@std@@YAPAV?$basic_string@DU?$char_traits@D@std@@V?$allocator@D@2@@0@PAV10@00Urandom_access_iterator_tag@0@U_Nonscalar_ptr_iterator_tag@0@U_Range_checked_iterator_tag@0@@Z 1001d1f0 f i xls.obj
 0001:0001c250       ??$swap@DU?$char_traits@D@std@@V?$allocator@D@2@@std@@YAXAAV?$basic_string@DU?$char_traits@D@std@@V?$allocator@D@2@@0@0@Z 1001d250 f i xls.obj
 0001:0001c260       ??$_Uninit_copy@PAV?$basic_string@DU?$char_traits@D@std@@V?$allocator@D@2@@std@@PAV12@V?$allocator@V?$basic_string@DU?$char_traits@D@std@@V?$allocator@D@2@@std@@@2@@std@@YAPAV?$basic_string@DU?$char_traits@D@std@@V?$allocator@D@2@@0@PAV10@00AAV?$allocator@V?$basic_string@DU?$char_traits@D@std@@V?$allocator@D@2@@std@@@0@U_Nonscalar_ptr_iterator_tag@0@U_Range_checked_iterator_tag@0@@Z 1001d260 f i xls.obj
 0001:0001c320       ?_Buy@?$vector@V?$basic_string@DU?$char_traits@D@std@@V?$allocator@D@2@@std@@V?$allocator@V?$basic_string@DU?$char_traits@D@std@@V?$allocator@D@2@@std@@@2@@std@@IAE_NI@Z 1001d320 f i xls.obj
 0001:0001c380       ??$fill@PAV?$basic_string@DU?$char_traits@D@std@@V?$allocator@D@2@@std@@V12@@std@@YAXPAV?$basic_string@DU?$char_traits@D@std@@V?$allocator@D@2@@0@0ABV10@@Z 1001d380 f i xls.obj
 0001:0001c3b0       ??$_Uninit_fill_n@PAV?$basic_string@DU?$char_traits@D@std@@V?$allocator@D@2@@std@@IV12@V?$allocator@V?$basic_string@DU?$char_traits@D@std@@V?$allocator@D@2@@std@@@2@@std@@YAXPAV?$basic_string@DU?$char_traits@D@std@@V?$allocator@D@2@@0@IABV10@AAV?$allocator@V?$basic_string@DU?$char_traits@D@std@@V?$allocator@D@2@@std@@@0@U_Nonscalar_ptr_iterator_tag@0@U_Range_checked_iterator_tag@0@@Z 1001d3b0 f i xls.obj
 0001:0001c460       ??$unchecked_uninitialized_copy@V?$_Vector_const_iterator@V?$basic_string@DU?$char_traits@D@std@@V?$allocator@D@2@@std@@V?$allocator@V?$basic_string@DU?$char_traits@D@std@@V?$allocator@D@2@@std@@@2@@std@@PAV?$basic_string@DU?$char_traits@D@std@@V?$allocator@D@2@@2@V?$allocator@V?$basic_string@DU?$char_traits@D@std@@V?$allocator@D@2@@std@@@2@@stdext@@YAPAV?$basic_string@DU?$char_traits@D@std@@V?$allocator@D@2@@std@@V?$_Vector_const_iterator@V?$basic_string@DU?$char_traits@D@std@@V?$allocator@D@2@@std@@V?$allocator@V?$basic_string@DU?$char_traits@D@std@@V?$allocator@D@2@@std@@@2@@2@0PAV12@AAV?$allocator@V?$basic_string@DU?$char_traits@D@std@@V?$allocator@D@2@@std@@@2@@Z 1001d460 f i xls.obj
 0001:0001c490       ??$unchecked_copy@PAV?$basic_string@DU?$char_traits@D@std@@V?$allocator@D@2@@std@@PAV12@@stdext@@YAPAV?$basic_string@DU?$char_traits@D@std@@V?$allocator@D@2@@std@@PAV12@00@Z 1001d490 f i xls.obj
 0001:0001c4c0       ??$_Swap_adl@V?$basic_string@DU?$char_traits@D@std@@V?$allocator@D@2@@std@@@std@@YAXAAV?$basic_string@DU?$char_traits@D@std@@V?$allocator@D@2@@0@0@Z 1001d4c0 f i xls.obj
 0001:0001c4d0       ??$unchecked_uninitialized_copy@PAV?$basic_string@DU?$char_traits@D@std@@V?$allocator@D@2@@std@@PAV12@V?$allocator@V?$basic_string@DU?$char_traits@D@std@@V?$allocator@D@2@@std@@@2@@stdext@@YAPAV?$basic_string@DU?$char_traits@D@std@@V?$allocator@D@2@@std@@PAV12@00AAV?$allocator@V?$basic_string@DU?$char_traits@D@std@@V?$allocator@D@2@@std@@@2@@Z 1001d4d0 f i xls.obj
 0001:0001c500       ??0?$vector@V?$basic_string@DU?$char_traits@D@std@@V?$allocator@D@2@@std@@V?$allocator@V?$basic_string@DU?$char_traits@D@std@@V?$allocator@D@2@@std@@@2@@std@@QAE@XZ 1001d500 f i xls.obj
 0001:0001c560       ??$unchecked_uninitialized_fill_n@PAV?$basic_string@DU?$char_traits@D@std@@V?$allocator@D@2@@std@@IV12@V?$allocator@V?$basic_string@DU?$char_traits@D@std@@V?$allocator@D@2@@std@@@2@@stdext@@YAXPAV?$basic_string@DU?$char_traits@D@std@@V?$allocator@D@2@@std@@IABV12@AAV?$allocator@V?$basic_string@DU?$char_traits@D@std@@V?$allocator@D@2@@std@@@2@@Z 1001d560 f i xls.obj
 0001:0001c590       ??$_Ucopy@V?$_Vector_const_iterator@V?$basic_string@DU?$char_traits@D@std@@V?$allocator@D@2@@std@@V?$allocator@V?$basic_string@DU?$char_traits@D@std@@V?$allocator@D@2@@std@@@2@@std@@@?$vector@V?$basic_string@DU?$char_traits@D@std@@V?$allocator@D@2@@std@@V?$allocator@V?$basic_string@DU?$char_traits@D@std@@V?$allocator@D@2@@std@@@2@@std@@IAEPAV?$basic_string@DU?$char_traits@D@std@@V?$allocator@D@2@@1@V?$_Vector_const_iterator@V?$basic_string@DU?$char_traits@D@std@@V?$allocator@D@2@@std@@V?$allocator@V?$basic_string@DU?$char_traits@D@std@@V?$allocator@D@2@@std@@@2@@1@0PAV21@@Z 1001d590 f i xls.obj
 0001:0001c5c0       ?erase@?$vector@V?$basic_string@DU?$char_traits@D@std@@V?$allocator@D@2@@std@@V?$allocator@V?$basic_string@DU?$char_traits@D@std@@V?$allocator@D@2@@std@@@2@@std@@QAE?AV?$_Vector_iterator@V?$basic_string@DU?$char_traits@D@std@@V?$allocator@D@2@@std@@V?$allocator@V?$basic_string@DU?$char_traits@D@std@@V?$allocator@D@2@@std@@@2@@2@V?$_Vector_const_iterator@V?$basic_string@DU?$char_traits@D@std@@V?$allocator@D@2@@std@@V?$allocator@V?$basic_string@DU?$char_traits@D@std@@V?$allocator@D@2@@std@@@2@@2@0@Z 1001d5c0 f i xls.obj
 0001:0001c670       ??$_Uninit_move@PAV?$basic_string@DU?$char_traits@D@std@@V?$allocator@D@2@@std@@PAV12@V?$allocator@V?$basic_string@DU?$char_traits@D@std@@V?$allocator@D@2@@std@@@2@@std@@YAPAV?$basic_string@DU?$char_traits@D@std@@V?$allocator@D@2@@0@PAV10@00AAV?$allocator@V?$basic_string@DU?$char_traits@D@std@@V?$allocator@D@2@@std@@@0@U_Swap_move_tag@0@U_Range_checked_iterator_tag@0@@Z 1001d670 f i xls.obj
 0001:0001c760       ??$_Move_backward_opt@PAV?$basic_string@DU?$char_traits@D@std@@V?$allocator@D@2@@std@@PAV12@Uforward_iterator_tag@2@@std@@YAPAV?$basic_string@DU?$char_traits@D@std@@V?$allocator@D@2@@0@PAV10@00Uforward_iterator_tag@0@U_Swap_move_tag@0@U_Range_checked_iterator_tag@0@@Z 1001d760 f i xls.obj
 0001:0001c7a0       ??$_Ucopy@PAV?$basic_string@DU?$char_traits@D@std@@V?$allocator@D@2@@std@@@?$vector@V?$basic_string@DU?$char_traits@D@std@@V?$allocator@D@2@@std@@V?$allocator@V?$basic_string@DU?$char_traits@D@std@@V?$allocator@D@2@@std@@@2@@std@@IAEPAV?$basic_string@DU?$char_traits@D@std@@V?$allocator@D@2@@1@PAV21@00@Z 1001d7a0 f i xls.obj
 0001:0001c7d0       ?_Ufill@?$vector@V?$basic_string@DU?$char_traits@D@std@@V?$allocator@D@2@@std@@V?$allocator@V?$basic_string@DU?$char_traits@D@std@@V?$allocator@D@2@@std@@@2@@std@@IAEPAV?$basic_string@DU?$char_traits@D@std@@V?$allocator@D@2@@2@PAV32@IABV32@@Z 1001d7d0 f i xls.obj
 0001:0001c810       ??0?$vector@V?$basic_string@DU?$char_traits@D@std@@V?$allocator@D@2@@std@@V?$allocator@V?$basic_string@DU?$char_traits@D@std@@V?$allocator@D@2@@std@@@2@@std@@QAE@ABV01@@Z 1001d810 f i xls.obj
 0001:0001c900       ??$_Unchecked_uninitialized_move@PAV?$basic_string@DU?$char_traits@D@std@@V?$allocator@D@2@@std@@PAV12@V?$allocator@V?$basic_string@DU?$char_traits@D@std@@V?$allocator@D@2@@std@@@2@@stdext@@YAPAV?$basic_string@DU?$char_traits@D@std@@V?$allocator@D@2@@std@@PAV12@00AAV?$allocator@V?$basic_string@DU?$char_traits@D@std@@V?$allocator@D@2@@std@@@2@@Z 1001d900 f i xls.obj
 0001:0001c930       ??$_Move_backward_opt@PAV?$basic_string@DU?$char_traits@D@std@@V?$allocator@D@2@@std@@PAV12@@std@@YAPAV?$basic_string@DU?$char_traits@D@std@@V?$allocator@D@2@@0@PAV10@00Urandom_access_iterator_tag@0@U_Swap_move_tag@0@U_Range_checked_iterator_tag@0@@Z 1001d930 f i xls.obj
 0001:0001c990       ?clear@?$vector@V?$basic_string@DU?$char_traits@D@std@@V?$allocator@D@2@@std@@V?$allocator@V?$basic_string@DU?$char_traits@D@std@@V?$allocator@D@2@@std@@@2@@std@@QAEXXZ 1001d990 f i xls.obj
 0001:0001c9d0       ??0ST_CELLS@@QAE@ABU0@@Z   1001d9d0 f i xls.obj
 0001:0001c9f0       ??$_Umove@PAV?$basic_string@DU?$char_traits@D@std@@V?$allocator@D@2@@std@@@?$vector@V?$basic_string@DU?$char_traits@D@std@@V?$allocator@D@2@@std@@V?$allocator@V?$basic_string@DU?$char_traits@D@std@@V?$allocator@D@2@@std@@@2@@std@@IAEPAV?$basic_string@DU?$char_traits@D@std@@V?$allocator@D@2@@1@PAV21@00@Z 1001d9f0 f i xls.obj
 0001:0001ca20       ??$_Unchecked_move_backward@PAV?$basic_string@DU?$char_traits@D@std@@V?$allocator@D@2@@std@@PAV12@@stdext@@YAPAV?$basic_string@DU?$char_traits@D@std@@V?$allocator@D@2@@std@@PAV12@00@Z 1001da20 f i xls.obj
 0001:0001ca50       ??4?$vector@V?$basic_string@DU?$char_traits@D@std@@V?$allocator@D@2@@std@@V?$allocator@V?$basic_string@DU?$char_traits@D@std@@V?$allocator@D@2@@std@@@2@@std@@QAEAAV01@ABV01@@Z 1001da50 f i xls.obj
 0001:0001cbe0       ??$_Construct@UST_CELLS@@U1@@std@@YAXPAUST_CELLS@@ABU1@@Z 1001dbe0 f i xls.obj
 0001:0001cc40       ??0ST_CELLS@@QAE@XZ        1001dc40 f i xls.obj
 0001:0001cc50       ?_Insert_n@?$vector@V?$basic_string@DU?$char_traits@D@std@@V?$allocator@D@2@@std@@V?$allocator@V?$basic_string@DU?$char_traits@D@std@@V?$allocator@D@2@@std@@@2@@std@@IAEXV?$_Vector_const_iterator@V?$basic_string@DU?$char_traits@D@std@@V?$allocator@D@2@@std@@V?$allocator@V?$basic_string@DU?$char_traits@D@std@@V?$allocator@D@2@@std@@@2@@2@IABV?$basic_string@DU?$char_traits@D@std@@V?$allocator@D@2@@2@@Z 1001dc50 f i xls.obj
 0001:0001cff0       ??4ST_CELLS@@QAEAAU0@ABU0@@Z 1001dff0 f i xls.obj
 0001:0001d010       ?construct@?$allocator@UST_CELLS@@@std@@QAEXPAUST_CELLS@@ABU3@@Z 1001e010 f i xls.obj
 0001:0001d030       ??$_Copy_backward_opt@PAUST_CELLS@@PAU1@Uforward_iterator_tag@std@@@std@@YAPAUST_CELLS@@PAU1@00Uforward_iterator_tag@0@U_Nonscalar_ptr_iterator_tag@0@U_Range_checked_iterator_tag@0@@Z 1001e030 f i xls.obj
 0001:0001d070       ?insert@?$vector@V?$basic_string@DU?$char_traits@D@std@@V?$allocator@D@2@@std@@V?$allocator@V?$basic_string@DU?$char_traits@D@std@@V?$allocator@D@2@@std@@@2@@std@@QAE?AV?$_Vector_iterator@V?$basic_string@DU?$char_traits@D@std@@V?$allocator@D@2@@std@@V?$allocator@V?$basic_string@DU?$char_traits@D@std@@V?$allocator@D@2@@std@@@2@@2@V?$_Vector_const_iterator@V?$basic_string@DU?$char_traits@D@std@@V?$allocator@D@2@@std@@V?$allocator@V?$basic_string@DU?$char_traits@D@std@@V?$allocator@D@2@@std@@@2@@2@ABV?$basic_string@DU?$char_traits@D@std@@V?$allocator@D@2@@2@@Z 1001e070 f i xls.obj
 0001:0001d130       ??$_Fill@PAUST_CELLS@@U1@@std@@YAXPAUST_CELLS@@0ABU1@@Z 1001e130 f i xls.obj
 0001:0001d160       ??$_Copy_backward_opt@PAUST_CELLS@@PAU1@@std@@YAPAUST_CELLS@@PAU1@00Urandom_access_iterator_tag@0@U_Nonscalar_ptr_iterator_tag@0@U_Range_checked_iterator_tag@0@@Z 1001e160 f i xls.obj
 0001:0001d1b0       ?push_back@?$vector@V?$basic_string@DU?$char_traits@D@std@@V?$allocator@D@2@@std@@V?$allocator@V?$basic_string@DU?$char_traits@D@std@@V?$allocator@D@2@@std@@@2@@std@@QAEXABV?$basic_string@DU?$char_traits@D@std@@V?$allocator@D@2@@2@@Z 1001e1b0 f i xls.obj
 0001:0001d260       ??$fill@PAUST_CELLS@@U1@@std@@YAXPAUST_CELLS@@0ABU1@@Z 1001e260 f i xls.obj
 0001:0001d290       ??$_Move_backward_opt@PAUST_CELLS@@PAU1@Urandom_access_iterator_tag@std@@U_Undefined_move_tag@3@@std@@YAPAUST_CELLS@@PAU1@00Urandom_access_iterator_tag@0@U_Undefined_move_tag@0@U_Range_checked_iterator_tag@0@@Z 1001e290 f i xls.obj
 0001:0001d2c0       ??$_Uninit_copy@PAUST_CELLS@@PAU1@V?$allocator@UST_CELLS@@@std@@@std@@YAPAUST_CELLS@@PAU1@00AAV?$allocator@UST_CELLS@@@0@U_Nonscalar_ptr_iterator_tag@0@U_Range_checked_iterator_tag@0@@Z 1001e2c0 f i xls.obj
 0001:0001d360       ??$_Unchecked_move_backward@PAUST_CELLS@@PAU1@@stdext@@YAPAUST_CELLS@@PAU1@00@Z 1001e360 f i xls.obj
 0001:0001d390       ??$_Uninit_fill_n@PAUST_CELLS@@IU1@V?$allocator@UST_CELLS@@@std@@@std@@YAXPAUST_CELLS@@IABU1@AAV?$allocator@UST_CELLS@@@0@U_Nonscalar_ptr_iterator_tag@0@U_Range_checked_iterator_tag@0@@Z 1001e390 f i xls.obj
 0001:0001d430       ??$unchecked_uninitialized_copy@PAUST_CELLS@@PAU1@V?$allocator@UST_CELLS@@@std@@@stdext@@YAPAUST_CELLS@@PAU1@00AAV?$allocator@UST_CELLS@@@std@@@Z 1001e430 f i xls.obj
 0001:0001d460       ??$unchecked_uninitialized_fill_n@PAUST_CELLS@@IU1@V?$allocator@UST_CELLS@@@std@@@stdext@@YAXPAUST_CELLS@@IABU1@AAV?$allocator@UST_CELLS@@@std@@@Z 1001e460 f i xls.obj
 0001:0001d490       ??$_Uninit_move@PAUST_CELLS@@PAU1@V?$allocator@UST_CELLS@@@std@@U_Undefined_move_tag@3@@std@@YAPAUST_CELLS@@PAU1@00AAV?$allocator@UST_CELLS@@@0@U_Undefined_move_tag@0@U_Range_checked_iterator_tag@0@@Z 1001e490 f i xls.obj
 0001:0001d4c0       ?_Ufill@?$vector@UST_CELLS@@V?$allocator@UST_CELLS@@@std@@@std@@IAEPAUST_CELLS@@PAU3@IABU3@@Z 1001e4c0 f i xls.obj
 0001:0001d500       ??$_Unchecked_uninitialized_move@PAUST_CELLS@@PAU1@V?$allocator@UST_CELLS@@@std@@@stdext@@YAPAUST_CELLS@@PAU1@00AAV?$allocator@UST_CELLS@@@std@@@Z 1001e500 f i xls.obj
 0001:0001d530       ??$_Umove@PAUST_CELLS@@@?$vector@UST_CELLS@@V?$allocator@UST_CELLS@@@std@@@std@@IAEPAUST_CELLS@@PAU2@00@Z 1001e530 f i xls.obj
 0001:0001d560       ?_Insert_n@?$vector@UST_CELLS@@V?$allocator@UST_CELLS@@@std@@@std@@IAEXV?$_Vector_const_iterator@UST_CELLS@@V?$allocator@UST_CELLS@@@std@@@2@IABUST_CELLS@@@Z 1001e560 f i xls.obj
 0001:0001d920       ?insert@?$vector@UST_CELLS@@V?$allocator@UST_CELLS@@@std@@@std@@QAE?AV?$_Vector_iterator@UST_CELLS@@V?$allocator@UST_CELLS@@@std@@@2@V?$_Vector_const_iterator@UST_CELLS@@V?$allocator@UST_CELLS@@@std@@@2@ABUST_CELLS@@@Z 1001e920 f i xls.obj
 0001:0001d9f0       ?push_back@?$vector@UST_CELLS@@V?$allocator@UST_CELLS@@@std@@@std@@QAEXABUST_CELLS@@@Z 1001e9f0 f i xls.obj
 0001:0001da90       ?SetRow@@YAXV?$basic_string@DU?$char_traits@D@std@@V?$allocator@D@2@@std@@PAUST_ROWS@@@Z 1001ea90 f   xls.obj
 0001:0001dc00       ?SetRows@@YAXAAV?$basic_string@DU?$char_traits@D@std@@V?$allocator@D@2@@std@@PAUST_ROWS@@@Z 1001ec00 f   xls.obj
 0001:0001dd80       ?GetTxtFile@@YAHPADPAUST_ROWS@@@Z 1001ed80 f   xls.obj
 0001:0001e000       ?dumpbuf@@YAXPADJPAE@Z     1001f000 f   xlstool.obj
 0001:0001e030       ?verbose@@YAXPAD@Z         1001f030 f   xlstool.obj
 0001:0001e170       ?utf8_decode@@YAPADPBDHPAH0@Z 1001f170 f   xlstool.obj
 0001:0001e190       ?get_unicode@@YAPADPAEE@Z  1001f190 f   xlstool.obj
 0001:0001e220       ?xls_getColor@@YAKGG@Z     1001f220 f   xlstool.obj
 0001:0001e250       ?xls_showBookInfo@@YAXPAUxlsWorkBook@@@Z 1001f250 f   xlstool.obj
 0001:0001e480       ?xls_showBOF@@YAXPAUBOF@@@Z 1001f480 f   xlstool.obj
 0001:0001e4f0       ?xls_showBOUNDSHEET@@YAXPAUBOUNDSHEET@@@Z 1001f4f0 f   xlstool.obj
 0001:0001e590       ?xls_showROW@@YAXPAUst_row_data@@@Z 1001f590 f   xlstool.obj
 0001:0001e620       ?xls_showColinfo@@YAXPAUst_colinfo_data@@@Z 1001f620 f   xlstool.obj
 0001:0001e6f0       ?xls_showCell@@YAXPAUst_cell_data@@@Z 1001f6f0 f   xlstool.obj
 0001:0001e780       ?xls_showFont@@YAXPAUst_font_data@@@Z 1001f780 f   xlstool.obj
 0001:0001e820       ?xls_showXF@@YAXPAUst_xf_data@@@Z 1001f820 f   xlstool.obj
 0001:0001e8c0       ?xls_getfcell@@YAPADPAUxlsWorkBook@@PAUst_cell_data@@@Z 1001f8c0 f   xlstool.obj
 0001:0001eae0       ?xls_getCSS@@YAPADPAUxlsWorkBook@@@Z 1001fae0 f   xlstool.obj
 0001:0001ef00       ??0SND_SOURCEDESC@@QAE@XZ  1001ff00 f i wzSound.obj
 0001:0001ef30       _DllMain@12                1001ff30 f   wzSound.obj
 0001:0001ef40       ?wzsnd_init@@YAHPAUWZSNDINFO@@@Z 1001ff40 f   wzSound.obj
 0001:0001f430       ?wzsnd_reload_soundtable@@YAXXZ 10020430 f   wzSound.obj
 0001:0001f460       ?wzsnd_reload_musictable@@YAXXZ 10020460 f   wzSound.obj
 0001:0001f490       ?wzsnd_reload_voicetable@@YAXXZ 10020490 f   wzSound.obj
 0001:0001f4c0       ?wzsnd_uninit@@YAXXZ       100204c0 f   wzSound.obj
 0001:0001f5a0       ?wzsnd_load_gameplay@@YAXXZ 100205a0 f   wzSound.obj
 0001:0001f5c0       ?wzsnd_unload_gameplay@@YAXXZ 100205c0 f   wzSound.obj
 0001:0001f5e0       ?wzsnd_update_3d_source@@YAXHPAU_D3DVECTOR@@0PAUSND_SOURCEDESC@@@Z 100205e0 f   wzSound.obj
 0001:0001f650       ?wzsnd_update_listener@@YAXPAU_D3DVECTOR@@000@Z 10020650 f   wzSound.obj
 0001:0001f6e0       ?wzsnd_getState_sound@@YAHH@Z 100206e0 f   wzSound.obj
 0001:0001f700       ?wzsnd_stop@@YAXH@Z        10020700 f   wzSound.obj
 0001:0001f720       ?wzsnd_stop_all@@YAXXZ     10020720 f   wzSound.obj
 0001:0001f740       ?wzsnd_pause@@YAXH@Z       10020740 f   wzSound.obj
 0001:0001f760       ?wzsnd_pause_all@@YAXXZ    10020760 f   wzSound.obj
 0001:0001f780       ?wzsnd_unpause@@YAXH@Z     10020780 f   wzSound.obj
 0001:0001f7a0       ?wzsnd_unpause_all@@YAXXZ  100207a0 f   wzSound.obj
 0001:0001f7c0       ?wzsnd_set_volume@@YAXHM@Z 100207c0 f   wzSound.obj
 0001:0001f7f0       ?wzsnd_set_volume_all@@YAXM@Z 100207f0 f   wzSound.obj
 0001:0001f820       ?wzsnd_set_loop@@YAXHH@Z   10020820 f   wzSound.obj
 0001:0001f840       ?wzsnd_load_ui@@YAXXZ      10020840 f   wzSound.obj
 0001:0001f860       ?wzsnd_unload_ui@@YAXXZ    10020860 f   wzSound.obj
 0001:0001f880       ?wzsnd_play_ui@@YAHHM@Z    10020880 f   wzSound.obj
 0001:0001f8b0       ?wzsnd_stop_ui@@YAXH@Z     100208b0 f   wzSound.obj
 0001:0001f8c0       ?wzsnd_play_ambi@@YAHHHHMHH@Z 100208c0 f   wzSound.obj
 0001:0001f910       ?wzsnd_stop_ambi@@YAXHH@Z  10020910 f   wzSound.obj
 0001:0001f930       ?wzsnd_stop_all_ambi@@YAXH@Z 10020930 f   wzSound.obj
 0001:0001f950       ?wzsnd_pause_ambi@@YAXH@Z  10020950 f   wzSound.obj
 0001:0001f970       ?wzsnd_pause_all_ambi@@YAXXZ 10020970 f   wzSound.obj
 0001:0001f990       ?wzsnd_unpause_ambi@@YAXH@Z 10020990 f   wzSound.obj
 0001:0001f9b0       ?wzsnd_unpause_all_ambi@@YAXXZ 100209b0 f   wzSound.obj
 0001:0001f9d0       ?wzsnd_set_volume_ambi@@YAXHM@Z 100209d0 f   wzSound.obj
 0001:0001fa00       ?wzsnd_set_volume_all_ambi@@YAXM@Z 10020a00 f   wzSound.obj
 0001:0001fa30       ?wzsnd_set_loop_ambi@@YAXHH@Z 10020a30 f   wzSound.obj
 0001:0001fa50       ?wzsnd_getState_ambi@@YAHH@Z 10020a50 f   wzSound.obj
 0001:0001fa60       ?wzsnd_stop_voice@@YAXHH@Z 10020a60 f   wzSound.obj
 0001:0001fa80       ?wzsnd_stop_all_voice@@YAXH@Z 10020a80 f   wzSound.obj
 0001:0001faa0       ?wzsnd_pause_voice@@YAXH@Z 10020aa0 f   wzSound.obj
 0001:0001fac0       ?wzsnd_pause_all_voice@@YAXXZ 10020ac0 f   wzSound.obj
 0001:0001fae0       ?wzsnd_unpause_voice@@YAXH@Z 10020ae0 f   wzSound.obj
 0001:0001fb00       ?wzsnd_unpause_all_voice@@YAXXZ 10020b00 f   wzSound.obj
 0001:0001fb20       ?wzsnd_set_volume_voice@@YAXHM@Z 10020b20 f   wzSound.obj
 0001:0001fb50       ?wzsnd_set_volume_all_voice@@YAXM@Z 10020b50 f   wzSound.obj
 0001:0001fb80       ?wzsnd_set_loop_voice@@YAXHH@Z 10020b80 f   wzSound.obj
 0001:0001fba0       ?wzsnd_getState_voice@@YAHH@Z 10020ba0 f   wzSound.obj
 0001:0001fbc0       ?wzsnd_getState_bgm@@YAHH@Z 10020bc0 f   wzSound.obj
 0001:0001fbe0       ?wzsnd_stop_bgm@@YAXHH@Z   10020be0 f   wzSound.obj
 0001:0001fc10       ?wzsnd_stop_all_bgm@@YAXH@Z 10020c10 f   wzSound.obj
 0001:0001fc40       ?wzsnd_pause_bgm@@YAXH@Z   10020c40 f   wzSound.obj
 0001:0001fc60       ?wzsnd_pause_all_bgm@@YAXXZ 10020c60 f   wzSound.obj
 0001:0001fc80       ?wzsnd_unpause_bgm@@YAXH@Z 10020c80 f   wzSound.obj
 0001:0001fca0       ?wzsnd_unpause_all_bgm@@YAXXZ 10020ca0 f   wzSound.obj
 0001:0001fcc0       ?wzsnd_set_volume_bgm@@YAXHM@Z 10020cc0 f   wzSound.obj
 0001:0001fcf0       ?wzsnd_set_volume_all_bgm@@YAXM@Z 10020cf0 f   wzSound.obj
 0001:0001fd20       ?wzsnd_set_loop_bgm@@YAXHH@Z 10020d20 f   wzSound.obj
 0001:0001fd40       ?wzsnd_set_master_vol@@YAXHH@Z 10020d40 f   wzSound.obj
 0001:0001fd90       ?wzsnd_get_master_vol@@YAXPAH0@Z 10020d90 f   wzSound.obj
 0001:0001fde0       ?wzsnd_set_master_mute@@YAX_N@Z 10020de0 f   wzSound.obj
 0001:0001fe20       ?wzsnd_get_master_mute@@YA_NXZ 10020e20 f   wzSound.obj
 0001:0001fe60       ?wzsnd_set_wav_vol@@YAXHH@Z 10020e60 f   wzSound.obj
 0001:0001feb0       ?wzsnd_get_wav_vol@@YAXPAH0@Z 10020eb0 f   wzSound.obj
 0001:0001ff00       ?wzsnd_set_wav_mute@@YAX_N@Z 10020f00 f   wzSound.obj
 0001:0001ff40       ?wzsnd_get_wav_mute@@YA_NXZ 10020f40 f   wzSound.obj
 0001:0001ff80       ?wzsnd_set_mic_input_vol@@YAXK@Z 10020f80 f   wzSound.obj
 0001:0001ffd0       ?wzsnd_get_mic_input_vol@@YAXPAK@Z 10020fd0 f   wzSound.obj
 0001:00020080       ?wzsnd_set_mic_output_vol@@YAXK@Z 10021080 f   wzSound.obj
 0001:000200d0       ?wzsnd_get_mic_output_vol@@YAXPAK@Z 100210d0 f   wzSound.obj
 0001:00020170       ?wzsnd_set_mic_output_mute@@YAX_N@Z 10021170 f   wzSound.obj
 0001:000201b0       ?wzsnd_get_mic_output_mute@@YA_NXZ 100211b0 f   wzSound.obj
 0001:000201f0       ?wzsnd_env_set@@YAXPAUsound_env@@@Z 100211f0 f   wzSound.obj
 0001:00020210       ?wzsnd_env_set_preset@@YAXK@Z 10021210 f   wzSound.obj
 0001:00020230       ?wzsnd_env_get@@YAXPAUsound_env@@@Z 10021230 f   wzSound.obj
 0001:00020250       ?wzsnd_env_disable@@YAXXZ  10021250 f   wzSound.obj
 0001:00020270       ?wzsnd_env_supported@@YAHXZ 10021270 f   wzSound.obj
 0001:00020290       ?wzsnd_check_channel@@YAXXZ 10021290 f   wzSound.obj
 0001:000202a0       ?wzsnd_update_cache@@YAXXZ 100212a0 f   wzSound.obj
 0001:000202b0       ?wzsnd_cache_maintain_milliseconds_set@@YAXH@Z 100212b0 f   wzSound.obj
 0001:000202c0       ?wzsnd_cache_maintain_milliseconds_get@@YAHXZ 100212c0 f   wzSound.obj
 0001:000202d0       ?wzsnd_cache_on@@YAXXZ     100212d0 f   wzSound.obj
 0001:000202e0       ?wzsnd_cache_off@@YAXXZ    100212e0 f   wzSound.obj
 0001:000202f0       ?wzsnd_cache_is@@YA_NXZ    100212f0 f   wzSound.obj
 0001:00020300       ?wzsnd_cache_size@@YAHXZ   10021300 f   wzSound.obj
 0001:00020310       ??Eiterator@?$_Tree@V?$_Tmap_traits@HUAmbientSnd@@U?$less@H@std@@V?$allocator@U?$pair@$$CBHUAmbientSnd@@@std@@@3@$0A@@std@@@std@@QAEAAV012@XZ 10021310 f i wzSound.obj
 0001:00020320       ?wzsnd_get_interfacesoundtable@@YAHPAUsoundEntry@@@Z 10021320 f   wzSound.obj
 0001:000203f0       ?wzsnd_get_soundtable@@YAHPAUsoundEntry@@@Z 100213f0 f   wzSound.obj
 0001:000204b0       ?wzsnd_get_soundtableArray@@YAHPAUsoundEntry@@@Z 100214b0 f   wzSound.obj
 0001:00020570       ?wzsnd_get_ambienttable@@YAHPAUsoundEntry@@@Z 10021570 f   wzSound.obj
 0001:00020640       ?wzsnd_play@@YAHHHHMH@Z    10021640 f   wzSound.obj
 0001:00020720       ?wzsnd_play_3d@@YAHHPAU_D3DVECTOR@@00HHPAUSND_SOURCEDESC@@@Z 10021720 f   wzSound.obj
 0001:00020840       ?wzsnd_play_voice@@YAHHHMH@Z 10021840 f   wzSound.obj
 0001:00020890       ?wzsnd_play_bgm@@YAHHHMH@Z 10021890 f   wzSound.obj
 0001:000208d2       _InitializeCriticalSection@4 100218d2 f   kernel32:KERNEL32.dll
 0001:000208d8       _DeleteCriticalSection@4   100218d8 f   kernel32:KERNEL32.dll
 0001:000208de       _LeaveCriticalSection@4    100218de f   kernel32:KERNEL32.dll
 0001:000208e4       _EnterCriticalSection@4    100218e4 f   kernel32:KERNEL32.dll
 0001:000208ea       _GetCurrentDirectoryA@8    100218ea f   kernel32:KERNEL32.dll
 0001:000208f0       _InterlockedExchange@8     100218f0 f   kernel32:KERNEL32.dll
 0001:000208f6       _GetProcAddress@8          100218f6 f   kernel32:KERNEL32.dll
 0001:000208fc       _LoadLibraryA@4            100218fc f   kernel32:KERNEL32.dll
 0001:00020902       _FreeLibrary@4             10021902 f   kernel32:KERNEL32.dll
 0001:00020908       _Sleep@4                   10021908 f   kernel32:KERNEL32.dll
 0001:0002090e       _GetLastError@0            1002190e f   kernel32:KERNEL32.dll
 0001:00020914       _LocalFree@4               10021914 f   kernel32:KERNEL32.dll
 0001:0002091a       _LocalAlloc@8              1002191a f   kernel32:KERNEL32.dll
 0001:00020920       _OutputDebugStringA@4      10021920 f   kernel32:KERNEL32.dll
 0001:00020926       _GetFileAttributesA@4      10021926 f   kernel32:KERNEL32.dll
 0001:0002092c       _GetModuleFileNameA@12     1002192c f   kernel32:KERNEL32.dll
 0001:00020932       _GetDriveTypeA@4           10021932 f   kernel32:KERNEL32.dll
 0001:00020938       _MulDiv@12                 10021938 f   kernel32:KERNEL32.dll
 0001:0002093e       _GetDesktopWindow@0        1002193e f   user32:USER32.dll
 0001:00020944       _CoUninitialize@0          10021944 f   ole32:ole32.dll
 0001:0002094a       _CoInitialize@4            1002194a f   ole32:ole32.dll
 0001:00020950       ??0invalid_argument@std@@QAE@ABV?$basic_string@DU?$char_traits@D@std@@V?$allocator@D@2@@1@@Z 10021950 f i libcpmt:string.obj
 0001:0002096d       ??1invalid_argument@std@@UAE@XZ 1002196d f i libcpmt:string.obj
 0001:00020978       ??_Einvalid_argument@std@@UAEPAXI@Z 10021978 f i libcpmt:string.obj
 0001:00020978       ??_Ginvalid_argument@std@@UAEPAXI@Z 10021978 f i libcpmt:string.obj
 0001:0002099f       ?_Xlen@_String_base@std@@SAXXZ 1002199f f   libcpmt:string.obj
 0001:000209d7       ?_Xran@_String_base@std@@SAXXZ 100219d7 f   libcpmt:string.obj
 0001:00020a0f       ?_Xinvarg@_String_base@std@@SAXXZ 10021a0f f   libcpmt:string.obj
 0001:00020a47       ??0invalid_argument@std@@QAE@ABV01@@Z 10021a47 f i libcpmt:string.obj
 0001:00020a70       _ov_clear                  10021a70 f   vorbisfile_static:vorbisfile.obj
 0001:00020b70       _ov_open_callbacks         10021b70 f   vorbisfile_static:vorbisfile.obj
 0001:00021710       _ov_open                   10022710 f   vorbisfile_static:vorbisfile.obj
 0001:00021780       _ov_halfrate               10022780 f   vorbisfile_static:vorbisfile.obj
 0001:00021840       _ov_halfrate_p             10022840 f   vorbisfile_static:vorbisfile.obj
 0001:00021860       _ov_test_callbacks         10022860 f   vorbisfile_static:vorbisfile.obj
 0001:000218a0       _ov_test                   100228a0 f   vorbisfile_static:vorbisfile.obj
 0001:000218f0       _ov_test_open              100228f0 f   vorbisfile_static:vorbisfile.obj
 0001:00021910       _ov_streams                10022910 f   vorbisfile_static:vorbisfile.obj
 0001:00021920       _ov_seekable               10022920 f   vorbisfile_static:vorbisfile.obj
 0001:00021930       _ov_bitrate                10022930 f   vorbisfile_static:vorbisfile.obj
 0001:00021a90       _ov_bitrate_instant        10022a90 f   vorbisfile_static:vorbisfile.obj
 0001:00021b00       _ov_serialnumber           10022b00 f   vorbisfile_static:vorbisfile.obj
 0001:00021b40       _ov_raw_total              10022b40 f   vorbisfile_static:vorbisfile.obj
 0001:00021bc0       _ov_pcm_total              10022bc0 f   vorbisfile_static:vorbisfile.obj
 0001:00021c30       _ov_time_total             10022c30 f   vorbisfile_static:vorbisfile.obj
 0001:00021cc0       _ov_raw_seek               10022cc0 f   vorbisfile_static:vorbisfile.obj
 0001:00021fe0       _ov_pcm_seek_page          10022fe0 f   vorbisfile_static:vorbisfile.obj
 0001:000225d0       _ov_pcm_seek               100235d0 f   vorbisfile_static:vorbisfile.obj
 0001:00022c20       _ov_time_seek              10023c20 f   vorbisfile_static:vorbisfile.obj
 0001:00022d20       _ov_time_seek_page         10023d20 f   vorbisfile_static:vorbisfile.obj
 0001:00022e20       _ov_raw_tell               10023e20 f   vorbisfile_static:vorbisfile.obj
 0001:00022e40       _ov_pcm_tell               10023e40 f   vorbisfile_static:vorbisfile.obj
 0001:00022e60       _ov_time_tell              10023e60 f   vorbisfile_static:vorbisfile.obj
 0001:00022f50       _ov_info                   10023f50 f   vorbisfile_static:vorbisfile.obj
 0001:00022f90       _ov_comment                10023f90 f   vorbisfile_static:vorbisfile.obj
 0001:00022fd0       _ov_read                   10023fd0 f   vorbisfile_static:vorbisfile.obj
 0001:00023340       _ov_read_float             10024340 f   vorbisfile_static:vorbisfile.obj
 0001:000233e0       _ov_crosslap               100243e0 f   vorbisfile_static:vorbisfile.obj
 0001:000238b0       _ov_raw_seek_lap           100248b0 f   vorbisfile_static:vorbisfile.obj
 0001:00023a20       _ov_pcm_seek_lap           10024a20 f   vorbisfile_static:vorbisfile.obj
 0001:00023a40       _ov_pcm_seek_page_lap      10024a40 f   vorbisfile_static:vorbisfile.obj
 0001:00023a60       _ov_time_seek_lap          10024a60 f   vorbisfile_static:vorbisfile.obj
 0001:00023bd0       _ov_time_seek_page_lap     10024bd0 f   vorbisfile_static:vorbisfile.obj
 0001:00023bf0       _vorbis_comment_init       10024bf0 f   vorbisfile_static:info.obj
 0001:00023c10       _vorbis_comment_add        10024c10 f   vorbisfile_static:info.obj
 0001:00023cc0       _vorbis_comment_add_tag    10024cc0 f   vorbisfile_static:info.obj
 0001:00023d80       _vorbis_comment_query      10024d80 f   vorbisfile_static:info.obj
 0001:00023eb0       _vorbis_comment_query_count 10024eb0 f   vorbisfile_static:info.obj
 0001:00023f70       _vorbis_comment_clear      10024f70 f   vorbisfile_static:info.obj
 0001:00023fe0       _vorbis_info_blocksize     10024fe0 f   vorbisfile_static:info.obj
 0001:00024000       _vorbis_info_init          10025000 f   vorbisfile_static:info.obj
 0001:00024030       _vorbis_info_clear         10025030 f   vorbisfile_static:info.obj
 0001:000241a0       _vorbis_synthesis_headerin 100251a0 f   vorbisfile_static:info.obj
 0001:00024710       _vorbis_commentheader_out  10025710 f   vorbisfile_static:info.obj
 0001:000248a0       _vorbis_analysis_headerout 100258a0 f   vorbisfile_static:info.obj
 0001:00024de0       _vorbis_granule_time       10025de0 f   vorbisfile_static:info.obj
 0001:00024e10       _vorbis_block_init         10025e10 f   vorbisfile_static:block.obj
 0001:00024e60       __vorbis_block_alloc       10025e60 f   vorbisfile_static:block.obj
 0001:00024ed0       __vorbis_block_ripcord     10025ed0 f   vorbisfile_static:block.obj
 0001:00024f40       _vorbis_block_clear        10025f40 f   vorbisfile_static:block.obj
 0001:00024fa0       _vorbis_analysis_init      10025fa0 f   vorbisfile_static:block.obj
 0001:000253c0       _vorbis_dsp_clear          100263c0 f   vorbisfile_static:block.obj
 0001:000255f0       _vorbis_analysis_buffer    100265f0 f   vorbisfile_static:block.obj
 0001:000256c0       _vorbis_analysis_wrote     100266c0 f   vorbisfile_static:block.obj
 0001:00025920       _vorbis_analysis_blockout  10026920 f   vorbisfile_static:block.obj
 0001:00025c50       _vorbis_synthesis_restart  10026c50 f   vorbisfile_static:block.obj
 0001:00025cc0       _vorbis_synthesis_init     10026cc0 f   vorbisfile_static:block.obj
 0001:00025cf0       _vorbis_synthesis_blockin  10026cf0 f   vorbisfile_static:block.obj
 0001:00026340       _vorbis_synthesis_pcmout   10027340 f   vorbisfile_static:block.obj
 0001:000263a0       _vorbis_synthesis_read     100273a0 f   vorbisfile_static:block.obj
 0001:000263d0       _vorbis_synthesis_lapout   100273d0 f   vorbisfile_static:block.obj
 0001:000265d0       _vorbis_window             100275d0 f   vorbisfile_static:block.obj
 0001:00026610       _vorbis_synthesis          10027610 f   vorbisfile_static:synthesis.obj
 0001:00026760       _vorbis_synthesis_trackonly 10027760 f   vorbisfile_static:synthesis.obj
 0001:00026840       _vorbis_packet_blocksize   10027840 f   vorbisfile_static:synthesis.obj
 0001:000268c0       _vorbis_synthesis_halfrate 100278c0 f   vorbisfile_static:synthesis.obj
 0001:000268f0       _vorbis_synthesis_halfrate_p 100278f0 f   vorbisfile_static:synthesis.obj
 0001:00026900       _vorbis_analysis           10027900 f   vorbisfile_static:analysis.obj
 0001:00026990       __analysis_output_always   10027990 f   vorbisfile_static:analysis.obj
 0001:00026ae0       __analysis_output          10027ae0 f   vorbisfile_static:analysis.obj
 0001:00026b50       __vp_global_look           10027b50 f   vorbisfile_static:psy.obj
 0001:00026b80       __vp_global_free           10027b80 f   vorbisfile_static:psy.obj
 0001:00026ba0       __vi_gpsy_free             10027ba0 f   vorbisfile_static:psy.obj
 0001:00026bc0       __vi_psy_free              10027bc0 f   vorbisfile_static:psy.obj
 0001:00026be0       __vp_psy_init              10027be0 f   vorbisfile_static:psy.obj
 0001:00027930       __vp_psy_clear             10028930 f   vorbisfile_static:psy.obj
 0001:000279f0       __vp_remove_floor          100289f0 f   vorbisfile_static:psy.obj
 0001:00027a50       __vp_noisemask             10028a50 f   vorbisfile_static:psy.obj
 0001:00028110       __vp_tonemask              10029110 f   vorbisfile_static:psy.obj
 0001:00028600       __vp_offset_and_mix        10029600 f   vorbisfile_static:psy.obj
 0001:00028690       __vp_ampmax_decay          10029690 f   vorbisfile_static:psy.obj
 0001:000286e0       __vp_quantize_couple_memo  100296e0 f   vorbisfile_static:psy.obj
 0001:00028990       __vp_quantize_couple_sort  10029990 f   vorbisfile_static:psy.obj
 0001:00028b40       __vp_noise_normalize_sort  10029b40 f   vorbisfile_static:psy.obj
 0001:00028c10       __vp_noise_normalize       10029c10 f   vorbisfile_static:psy.obj
 0001:00028e80       __vp_couple                10029e80 f   vorbisfile_static:psy.obj
 0001:000293b0       __ilog                     1002a3b0 f   vorbisfile_static:sharedbook.obj
 0001:000293c0       __float32_pack             1002a3c0 f   vorbisfile_static:sharedbook.obj
 0001:00029450       __float32_unpack           1002a450 f   vorbisfile_static:sharedbook.obj
 0001:000294a0       __make_words               1002a4a0 f   vorbisfile_static:sharedbook.obj
 0001:00029620       __book_maptype1_quantvals  1002a620 f   vorbisfile_static:sharedbook.obj
 0001:00029690       __book_unquantize          1002a690 f   vorbisfile_static:sharedbook.obj
 0001:00029880       _vorbis_staticbook_clear   1002a880 f   vorbisfile_static:sharedbook.obj
 0001:00029950       _vorbis_staticbook_destroy 1002a950 f   vorbisfile_static:sharedbook.obj
 0001:00029970       _vorbis_book_clear         1002a970 f   vorbisfile_static:sharedbook.obj
 0001:000299d0       _vorbis_book_init_encode   1002a9d0 f   vorbisfile_static:sharedbook.obj
 0001:00029a30       _vorbis_book_init_decode   1002aa30 f   vorbisfile_static:sharedbook.obj
 0001:00029e80       __best                     1002ae80 f   vorbisfile_static:sharedbook.obj
 0001:0002a030       _vorbis_book_codeword      1002b030 f   vorbisfile_static:sharedbook.obj
 0001:0002a050       _vorbis_book_codelen       1002b050 f   vorbisfile_static:sharedbook.obj
 0001:0002a070       _vorbis_staticbook_pack    1002b070 f   vorbisfile_static:codebook.obj
 0001:0002a2c0       _vorbis_staticbook_unpack  1002b2c0 f   vorbisfile_static:codebook.obj
 0001:0002a500       _vorbis_book_encode        1002b500 f   vorbisfile_static:codebook.obj
 0001:0002a540       _vorbis_book_errorv        1002b540 f   vorbisfile_static:codebook.obj
 0001:0002a580       _vorbis_book_encodev       1002b580 f   vorbisfile_static:codebook.obj
 0001:0002a5d0       _vorbis_book_decode        1002b5d0 f   vorbisfile_static:codebook.obj
 0001:0002a760       _vorbis_book_decodevs_add  1002b760 f   vorbisfile_static:codebook.obj
 0001:0002a960       _vorbis_book_decodev_add   1002b960 f   vorbisfile_static:codebook.obj
 0001:0002acf0       _vorbis_book_decodev_set   1002bcf0 f   vorbisfile_static:codebook.obj
 0001:0002ae70       _vorbis_book_decodevv_add  1002be70 f   vorbisfile_static:codebook.obj
 0001:0002b030       _vorbis_bitrate_init       1002c030 f   vorbisfile_static:bitrate.obj
 0001:0002b230       _vorbis_bitrate_clear      1002c230 f   vorbisfile_static:bitrate.obj
 0001:0002b310       _vorbis_bitrate_managed    1002c310 f   vorbisfile_static:bitrate.obj
 0001:0002b330       _vorbis_bitrate_addblock   1002c330 f   vorbisfile_static:bitrate.obj
 0001:0002bfd0       _vorbis_bitrate_flushpacket 1002cfd0 f   vorbisfile_static:bitrate.obj
 0001:0002c090       __ve_envelope_init         1002d090 f   vorbisfile_static:envelope.obj
 0001:0002c230       __ve_envelope_clear        1002d230 f   vorbisfile_static:envelope.obj
 0001:0002c290       __ve_envelope_search       1002d290 f   vorbisfile_static:envelope.obj
 0001:0002c850       __ve_envelope_mark         1002d850 f   vorbisfile_static:envelope.obj
 0001:0002c910       __ve_envelope_shift        1002d910 f   vorbisfile_static:envelope.obj
 0001:0002c990       _drft_forward              1002d990 f   vorbisfile_static:smallft.obj
 0001:0002dd50       _drft_backward             1002ed50 f   vorbisfile_static:smallft.obj
 0001:0002f360       _drft_init                 10030360 f   vorbisfile_static:smallft.obj
 0001:0002f550       _drft_clear                10030550 f   vorbisfile_static:smallft.obj
 0001:0002f590       _mdct_init                 10030590 f   vorbisfile_static:mdct.obj
 0001:0002f770       _mdct_clear                10030770 f   vorbisfile_static:mdct.obj
 0001:0002f7b0       _mdct_backward             100307b0 f   vorbisfile_static:mdct.obj
 0001:00030370       _mdct_forward              10031370 f   vorbisfile_static:mdct.obj
 0001:000307f0       _vorbis_lpc_from_data      100317f0 f   vorbisfile_static:lpc.obj
 0001:000309a0       _vorbis_lpc_predict        100319a0 f   vorbisfile_static:lpc.obj
 0001:00030a70       __vorbis_window_get        10031a70 f   vorbisfile_static:window.obj
 0001:00030a80       __vorbis_apply_window      10031a80 f   vorbisfile_static:window.obj
 0001:00031c30       _res0_free_info            10032c30 f   vorbisfile_static:res0.obj
 0001:00031c50       _res0_free_look            10032c50 f   vorbisfile_static:res0.obj
 0001:00031cd0       _res0_pack                 10032cd0 f   vorbisfile_static:res0.obj
 0001:00031df0       _res0_unpack               10032df0 f   vorbisfile_static:res0.obj
 0001:00031f30       _res0_look                 10032f30 f   vorbisfile_static:res0.obj
 0001:00032110       _res0_inverse              10033110 f   vorbisfile_static:res0.obj
 0001:00032390       _res1_forward              10033390 f   vorbisfile_static:res0.obj
 0001:00032940       _res1_class                10033940 f   vorbisfile_static:res0.obj
 0001:00032bd0       _res1_inverse              10033bd0 f   vorbisfile_static:res0.obj
 0001:00032c30       _res2_class                10033c30 f   vorbisfile_static:res0.obj
 0001:00032e10       _res2_forward              10033e10 f   vorbisfile_static:res0.obj
 0001:00032f70       _res2_inverse              10033f70 f   vorbisfile_static:res0.obj
 0001:000337a0       _floor1_fit                100347a0 f   vorbisfile_static:floor1.obj
 0001:00034340       _floor1_interpolate_fit    10035340 f   vorbisfile_static:floor1.obj
 0001:000343f0       _floor1_encode             100353f0 f   vorbisfile_static:floor1.obj
 0001:000353d0       _vorbis_lsp_to_curve       100363d0 f   vorbisfile_static:lsp.obj
 0001:00035550       _vorbis_coslook            10036550 f   vorbisfile_static:lsp.obj
 0001:000355a0       _vorbis_invsqlook          100365a0 f   vorbisfile_static:lsp.obj
 0001:000355f0       _vorbis_invsq2explook      100365f0 f   vorbisfile_static:lsp.obj
 0001:00035600       _vorbis_fromdBlook         10036600 f   vorbisfile_static:lsp.obj
 0001:00035660       _vorbis_lpc_to_lsp         10036660 f   vorbisfile_static:lsp.obj
 0001:00035b80       __fpclear                  10036b80 f   LIBCMT:_fpinit_.obj
 0001:00035b81       __cfltcvt_init             10036b81 f   LIBCMT:_fpinit_.obj
 0001:00035be1       ___setfflag                10036be1 f   LIBCMT:_fpinit_.obj
 0001:00035bf6       __fpmath                   10036bf6 f   LIBCMT:_fpinit_.obj
 0001:00035c19       _free                      10036c19 f   LIBCMT:free.obj
 0001:00035cb0       _memcpy                    10036cb0 f   LIBCMT:memcpy.obj
 0001:00036020       _memset                    10037020 f   LIBCMT:memset.obj
 0001:0003609a       ??0_LocaleUpdate@@QAE@PAUlocaleinfo_struct@@@Z 1003709a f i LIBCMT:stricmp.obj
 0001:00036121       ??1_LocaleUpdate@@QAE@XZ   10037121 f i LIBCMT:stricmp.obj
 0001:0003612f       ?GetLocaleT@_LocaleUpdate@@QAEPAUlocaleinfo_struct@@XZ 1003712f f i LIBCMT:stricmp.obj
 0001:00036132       ___ascii_stricmp           10037132 f   LIBCMT:stricmp.obj
 0001:0003616b       __stricmp_l                1003716b f   LIBCMT:stricmp.obj
 0001:00036240       __stricmp                  10037240 f   LIBCMT:stricmp.obj
 0001:00036240       _stricmp                   10037240 f   LIBCMT:stricmp.obj
 0001:00036292       @__security_check_cookie@4 10037292 f   LIBCMT:secchk.obj
 0001:000362a1       _V6_HeapAlloc              100372a1 f   LIBCMT:malloc.obj
 0001:000362f0       __heap_alloc               100372f0 f i LIBCMT:malloc.obj
 0001:0003636a       _malloc                    1003736a f   LIBCMT:malloc.obj
 0001:000364ee       ___onexitinit              100374ee f   LIBCMT:onexit.obj
 0001:0003651f       __onexit                   1003751f f   LIBCMT:onexit.obj
 0001:0003655b       _atexit                    1003755b f   LIBCMT:onexit.obj
 0001:00036572       ??_L@YGXPAXIHP6EX0@Z1@Z    10037572 f   LIBCMT:ehvecctr.obj
 0001:000365e9       ?__ArrayUnwind@@YGXPAXIHP6EX0@Z@Z 100375e9 f   LIBCMT:ehvecdtr.obj
 0001:00036647       ??_M@YGXPAXIHP6EX0@Z@Z     10037647 f   LIBCMT:ehvecdtr.obj
 0001:000366b0       _log                       100376b0 f   LIBCMT:_log_.obj
 0001:000366f0       __CIlog                    100376f0 f   LIBCMT:_log_.obj
 0001:0003672b       __CIlog_default            1003772b f   LIBCMT:_log_.obj
 0001:0003673f       __log_default              1003773f     LIBCMT:_log_.obj
 0001:00036800       __ftol2_sse                10037800 f   LIBCMT:ftol2.obj
 0001:00036809       __ftol2_pentium4           10037809 f   LIBCMT:ftol2.obj
 0001:0003681c       __ftol2_sse_excpt          1003781c f   LIBCMT:ftol2.obj
 0001:00036836       __ftol2                    10037836 f   LIBCMT:ftol2.obj
 0001:000368b0       _pow                       100378b0 f   LIBCMT:_pow_.obj
 0001:000368f0       __CIpow                    100378f0 f   LIBCMT:_pow_.obj
 0001:0003692b       __CIpow_default            1003792b f   LIBCMT:_pow_.obj
 0001:00036944       __pow_default              10037944     LIBCMT:_pow_.obj
 0001:00036b3a       __initp_misc_invarg        10037b3a f   LIBCMT:invarg.obj
 0001:00036b49       __invoke_watson            10037b49 f   LIBCMT:invarg.obj
 0001:00036c71       __set_invalid_parameter_handler 10037c71 f   LIBCMT:invarg.obj
 0001:00036c98       __get_invalid_parameter_handler 10037c98 f   LIBCMT:invarg.obj
 0001:00036ca5       ?_invoke_watson@@YAXPBG00II@Z 10037ca5 f   LIBCMT:invarg.obj
 0001:00036cb0       __invalid_parameter        10037cb0 f   LIBCMT:invarg.obj
 0001:00036cd6       __invalid_parameter_noinfo 10037cd6 f   LIBCMT:invarg.obj
 0001:00036ce6       ?_invalid_parameter@@YAXPBG00II@Z 10037ce6 f   LIBCMT:invarg.obj
 0001:00036cf1       _memcpy_s                  10037cf1 f   LIBCMT:memcpy_s.obj
 0001:00036d6e       _memmove_s                 10037d6e f   LIBCMT:memmove_s.obj
 0001:00036dcb       ??0exception@std@@QAE@XZ   10037dcb f   LIBCMT:stdexcpt.obj
 0001:00036ddc       ??0exception@std@@QAE@ABQBD@Z 10037ddc f   LIBCMT:stdexcpt.obj
 0001:00036e2f       ??0exception@std@@QAE@ABQBDH@Z 10037e2f f   LIBCMT:stdexcpt.obj
 0001:00036e4c       ??0exception@std@@QAE@ABV01@@Z 10037e4c f   LIBCMT:stdexcpt.obj
 0001:00036ea9       ??4exception@std@@QAEAAV01@ABV01@@Z 10037ea9 f   LIBCMT:stdexcpt.obj
 0001:00036f04       ??1exception@std@@UAE@XZ   10037f04 f   LIBCMT:stdexcpt.obj
 0001:00036f1a       ?what@exception@std@@UBEPBDXZ 10037f1a f   LIBCMT:stdexcpt.obj
 0001:00036f27       ??0bad_cast@std@@QAE@PBD@Z 10037f27 f   LIBCMT:stdexcpt.obj
 0001:00036f45       ??0bad_cast@std@@QAE@ABV01@@Z 10037f45 f   LIBCMT:stdexcpt.obj
 0001:00036f62       ??1bad_cast@std@@UAE@XZ    10037f62 f   LIBCMT:stdexcpt.obj
 0001:00036f6d       ??0bad_typeid@std@@QAE@PBD@Z 10037f6d f   LIBCMT:stdexcpt.obj
 0001:00036f8b       ??0bad_typeid@std@@QAE@ABV01@@Z 10037f8b f   LIBCMT:stdexcpt.obj
 0001:00036fa8       ??1bad_typeid@std@@UAE@XZ  10037fa8 f   LIBCMT:stdexcpt.obj
 0001:00036fb3       ??0__non_rtti_object@std@@QAE@PBD@Z 10037fb3 f   LIBCMT:stdexcpt.obj
 0001:00036fd0       ??0__non_rtti_object@std@@QAE@ABV01@@Z 10037fd0 f   LIBCMT:stdexcpt.obj
 0001:00036fed       ??1__non_rtti_object@std@@UAE@XZ 10037fed f   LIBCMT:stdexcpt.obj
 0001:00036ff8       ??_Gexception@std@@UAEPAXI@Z 10037ff8 f i LIBCMT:stdexcpt.obj
 0001:00036ff8       ??_Eexception@std@@UAEPAXI@Z 10037ff8 f i LIBCMT:stdexcpt.obj
 0001:00037019       ??_Ebad_cast@std@@UAEPAXI@Z 10038019 f i LIBCMT:stdexcpt.obj
 0001:00037019       ??_Gbad_cast@std@@UAEPAXI@Z 10038019 f i LIBCMT:stdexcpt.obj
 0001:00037040       ??_Gbad_typeid@std@@UAEPAXI@Z 10038040 f i LIBCMT:stdexcpt.obj
 0001:00037040       ??_Ebad_typeid@std@@UAEPAXI@Z 10038040 f i LIBCMT:stdexcpt.obj
 0001:00037067       ??_G__non_rtti_object@std@@UAEPAXI@Z 10038067 f i LIBCMT:stdexcpt.obj
 0001:00037067       ??_E__non_rtti_object@std@@UAEPAXI@Z 10038067 f i LIBCMT:stdexcpt.obj
 0001:0003708e       ?name@type_info@@QBEPBDPAU__type_info_node@@@Z 1003808e f   LIBCMT:typinfo.obj
 0001:000370a2       ??1type_info@@UAE@XZ       100380a2 f   LIBCMT:typinfo.obj
 0001:000370b2       ??_Etype_info@@UAEPAXI@Z   100380b2 f i LIBCMT:typinfo.obj
 0001:000370b2       ??_Gtype_info@@UAEPAXI@Z   100380b2 f i LIBCMT:typinfo.obj
 0001:000370d3       ?_name_internal_method@type_info@@QBEPBDPAU__type_info_node@@@Z 100380d3 f   LIBCMT:typinfo.obj
 0001:000370e7       ?_type_info_dtor_internal_method@type_info@@QAEXXZ 100380e7 f   LIBCMT:typinfo.obj
 0001:000370f1       ??8type_info@@QBE_NABV0@@Z 100380f1 f   LIBCMT:typinfo.obj
 0001:00037111       ??9type_info@@QBE_NABV0@@Z 10038111 f   LIBCMT:typinfo.obj
 0001:00037132       ?before@type_info@@QBEHABV1@@Z 10038132 f   LIBCMT:typinfo.obj
 0001:00037156       ?raw_name@type_info@@QBEPBDXZ 10038156 f   LIBCMT:typinfo.obj
 0001:0003715a       ??0type_info@@AAE@ABV0@@Z  1003815a f   LIBCMT:typinfo.obj
 0001:00037165       ??4type_info@@AAEAAV0@ABV0@@Z 10038165 f   LIBCMT:typinfo.obj
 0001:0003716a       ??3@YAXPAX@Z               1003816a f   LIBCMT:delete.obj
 0001:00037175       ??0bad_alloc@std@@QAE@XZ   10038175 f i LIBCMT:new.obj
 0001:00037190       ??2@YAPAXI@Z               10038190 f   LIBCMT:new.obj
 0001:000371f5       __CxxThrowException@8      100381f5 f   LIBCMT:throw.obj
 0001:00037241       ?_JumpToContinuation@@YGXPAXPAUEHRegistrationNode@@@Z 10038241 f   LIBCMT:_trnsctrl_.obj
 0001:00037273       ?_CallMemberFunction0@@YGXPAX0@Z 10038273 f   LIBCMT:_trnsctrl_.obj
 0001:0003727a       ?_CallMemberFunction1@@YGXPAX00@Z 1003827a f   LIBCMT:_trnsctrl_.obj
 0001:00037281       ?_CallMemberFunction2@@YGXPAX00H@Z 10038281 f   LIBCMT:_trnsctrl_.obj
 0001:00037288       ?_UnwindNestedFrames@@YGXPAUEHRegistrationNode@@PAUEHExceptionRecord@@@Z 10038288 f   LIBCMT:_trnsctrl_.obj
 0001:000372dc       ___CxxFrameHandler         100382dc f   LIBCMT:_trnsctrl_.obj
 0001:00037312       ___CxxFrameHandler3        10038312 f   LIBCMT:_trnsctrl_.obj
 0001:00037348       ___CxxFrameHandler2        10038348 f   LIBCMT:_trnsctrl_.obj
 0001:0003737e       ___CxxLongjmpUnwind@4      1003837e f   LIBCMT:_trnsctrl_.obj
 0001:000373d0       ?_CallSETranslator@@YAHPAUEHExceptionRecord@@PAUEHRegistrationNode@@PAX2PBU_s_FuncInfo@@H1@Z 100383d0 f   LIBCMT:_trnsctrl_.obj
 0001:00037546       ?_GetRangeOfTrysToCheck@@YAPBU_s_TryBlockMapEntry@@PBU_s_FuncInfo@@HHPAI1@Z 10038546 f   LIBCMT:_trnsctrl_.obj
 0001:000375bb       __CreateFrameInfo          100385bb f   LIBCMT:_trnsctrl_.obj
 0001:000375e7       __IsExceptionObjectToBeDestroyed 100385e7 f   LIBCMT:_trnsctrl_.obj
 0001:0003760e       __FindAndUnlinkFrame       1003860e f   LIBCMT:_trnsctrl_.obj
 0001:00037660       ?_CallCatchBlock2@@YAPAXPAUEHRegistrationNode@@PBU_s_FuncInfo@@PAXHK@Z 10038660 f   LIBCMT:_trnsctrl_.obj
 0001:000376c0       _strncpy                   100386c0 f   LIBCMT:strncpy.obj
 0001:000377e4       _sprintf                   100387e4 f   LIBCMT:sprintf.obj
 0001:00037861       __sprintf_l                10038861 f   LIBCMT:sprintf.obj
 0001:0003787d       _sprintf_s                 1003887d f   LIBCMT:sprintf.obj
 0001:0003789b       __sprintf_s_l              1003889b f   LIBCMT:sprintf.obj
 0001:000378ba       __snprintf_s               100388ba f   LIBCMT:sprintf.obj
 0001:000378db       __snprintf_s_l             100388db f   LIBCMT:sprintf.obj
 0001:000378fd       __sprintf_p                100388fd f   LIBCMT:sprintf.obj
 0001:0003791b       __sprintf_p_l              1003891b f   LIBCMT:sprintf.obj
 0001:0003793a       __scprintf                 1003893a f   LIBCMT:sprintf.obj
 0001:0003794f       __scprintf_p               1003894f f   LIBCMT:sprintf.obj
 0001:00037964       __scprintf_l               10038964 f   LIBCMT:sprintf.obj
 0001:0003797d       __scprintf_p_l             1003897d f   LIBCMT:sprintf.obj
 0001:00037996       _atol                      10038996 f   LIBCMT:atox.obj
 0001:000379ac       __atol_l                   100389ac f   LIBCMT:atox.obj
 0001:000379c5       _atoi                      100389c5 f   LIBCMT:atox.obj
 0001:000379d0       __atoi_l                   100389d0 f   LIBCMT:atox.obj
 0001:000379db       __atoi64                   100389db f   LIBCMT:atox.obj
 0001:000379f1       __atoi64_l                 100389f1 f   LIBCMT:atox.obj
 0001:00037a0a       __atof_l                   10038a0a f   LIBCMT:atof.obj
 0001:00037ab5       _atof                      10038ab5 f   LIBCMT:atof.obj
 0001:00037ac8       ___strgtold12              10038ac8 f   LIBCMT:atof.obj
 0001:00037b0a       ___STRINGTOLD              10038b0a f   LIBCMT:atof.obj
 0001:00037b50       __alldiv                   10038b50 f   LIBCMT:lldiv.obj
 0001:00037bfa       __vsprintf_l               10038bfa f   LIBCMT:vsprintf.obj
 0001:00037c78       _vsprintf                  10038c78 f   LIBCMT:vsprintf.obj
 0001:00037c92       __vscprintf_helper         10038c92 f   LIBCMT:vsprintf.obj
 0001:00037ce9       __vscprintf                10038ce9 f   LIBCMT:vsprintf.obj
 0001:00037d05       __vscprintf_l              10038d05 f   LIBCMT:vsprintf.obj
 0001:00037d22       __vscprintf_p              10038d22 f   LIBCMT:vsprintf.obj
 0001:00037d3e       __vscprintf_p_l            10038d3e f   LIBCMT:vsprintf.obj
 0001:00037d60       __alloca_probe             10038d60     LIBCMT:chkstk.obj
 0001:00037d60       __chkstk                   10038d60 f   LIBCMT:chkstk.obj
 0001:00037da0       _strchr                    10038da0 f   LIBCMT:strchr.obj
 0001:00037da6       ___from_strstr_to_strchr   10038da6     LIBCMT:strchr.obj
 0001:00038050       __splitpath                10039050 f   LIBCMT:splitpat.obj
 0001:0003809c       __makepath                 1003909c f   LIBCMT:makepath.obj
 0001:000380c0       _memmove                   100390c0 f   LIBCMT:memmove.obj
 0001:00038430       _strstr                    10039430 f   LIBCMT:strstr.obj
 0001:000384b6       __fseek_nolock             100394b6 f   LIBCMT:fseek.obj
 0001:00038540       _fseek                     10039540 f   LIBCMT:fseek.obj
 0001:000385c5       __fread_nolock_s           100395c5 f   LIBCMT:fread.obj
 0001:000387cf       __fread_nolock             100397cf f   LIBCMT:fread.obj
 0001:000387ec       _fread_s                   100397ec f   LIBCMT:fread.obj
 0001:00038882       _fread                     10039882 f   LIBCMT:fread.obj
 0001:0003889f       __fclose_nolock            1003989f f   LIBCMT:fclose.obj
 0001:00038916       _fclose                    10039916 f   LIBCMT:fclose.obj
 0001:00038992       __fsopen                   10039992 f   LIBCMT:fopen.obj
 0001:00038a56       _fopen                     10039a56 f   LIBCMT:fopen.obj
 0001:00038a6d       _fopen_s                   10039a6d f   LIBCMT:fopen.obj
 0001:00038ac0       __allshr                   10039ac0 f   LIBCMT:llshr.obj
 0001:00038af0       __CIsqrt                   10039af0 f   LIBCMT:_sqrt_.obj
 0001:00038b04       _sqrt                      10039b04     LIBCMT:_sqrt_.obj
 0001:00038bb0       _acos                      10039bb0 f   LIBCMT:_acos_.obj
 0001:00038bf0       __CIacos                   10039bf0 f   LIBCMT:_acos_.obj
 0001:00038c2b       __CIacos_default           10039c2b f   LIBCMT:_acos_.obj
 0001:00038c3f       __acos_default             10039c3f     LIBCMT:_acos_.obj
 0001:00038d00       _asin                      10039d00 f   LIBCMT:_asin_.obj
 0001:00038d40       __CIasin                   10039d40 f   LIBCMT:_asin_.obj
 0001:00038d7b       __CIasin_default           10039d7b f   LIBCMT:_asin_.obj
 0001:00038d8f       __asin_default             10039d8f     LIBCMT:_asin_.obj
 0001:00038e50       _atan                      10039e50 f   LIBCMT:_atan_.obj
 0001:00038e90       __CIatan                   10039e90 f   LIBCMT:_atan_.obj
 0001:00038ecb       __CIatan_default           10039ecb f   LIBCMT:_atan_.obj
 0001:00038edf       __atan_default             10039edf     LIBCMT:_atan_.obj
 0001:00038f70       _cos                       10039f70 f   LIBCMT:_cos_.obj
 0001:00038fb0       __CIcos                    10039fb0 f   LIBCMT:_cos_.obj
 0001:00038feb       __CIcos_default            10039feb f   LIBCMT:_cos_.obj
 0001:00038fff       __cos_default              10039fff     LIBCMT:_cos_.obj
 0001:000390a0       _sin                       1003a0a0 f   LIBCMT:_sin_.obj
 0001:000390e0       __CIsin                    1003a0e0 f   LIBCMT:_sin_.obj
 0001:0003911b       __CIsin_default            1003a11b f   LIBCMT:_sin_.obj
 0001:0003912f       __sin_default              1003a12f     LIBCMT:_sin_.obj
 0001:000391c9       __copysign                 1003a1c9 f   LIBCMT:_ieeemisc_.obj
 0001:000391f1       __chgsign                  1003a1f1 f   LIBCMT:_ieeemisc_.obj
 0001:0003921e       __scalb                    1003a21e f   LIBCMT:_ieeemisc_.obj
 0001:00039238       __logb                     1003a238 f   LIBCMT:_ieeemisc_.obj
 0001:00039321       __nextafter                1003a321 f   LIBCMT:_ieeemisc_.obj
 0001:000395c9       __finite                   1003a5c9 f   LIBCMT:_ieeemisc_.obj
 0001:000395e5       __isnan                    1003a5e5 f   LIBCMT:_ieeemisc_.obj
 0001:00039619       __fpclass                  1003a619 f   LIBCMT:_ieeemisc_.obj
 0001:000396ad       _srand                     1003a6ad f   LIBCMT:rand.obj
 0001:000396bf       _rand                      1003a6bf f   LIBCMT:rand.obj
 0001:000396e1       _ldiv                      1003a6e1 f   LIBCMT:ldiv.obj
 0001:000396ef       _realloc                   1003a6ef f   LIBCMT:realloc.obj
 0001:0003990a       _printf                    1003a90a f   LIBCMT:printf.obj
 0001:000399b9       __printf_l                 1003a9b9 f   LIBCMT:printf.obj
 0001:000399d2       __printf_s_l               1003a9d2 f   LIBCMT:printf.obj
 0001:000399eb       _printf_s                  1003a9eb f   LIBCMT:printf.obj
 0001:00039a03       __printf_p_l               1003aa03 f   LIBCMT:printf.obj
 0001:00039a1c       __printf_p                 1003aa1c f   LIBCMT:printf.obj
 0001:00039a34       __set_printf_count_output  1003aa34 f   LIBCMT:printf.obj
 0001:00039a5e       __get_printf_count_output  1003aa5e f   LIBCMT:printf.obj
 0001:00039a80       _memchr                    1003aa80 f   LIBCMT:memchr.obj
 0001:00039b2d       __fwrite_nolock            1003ab2d f   LIBCMT:fwrite.obj
 0001:00039c8f       _fwrite                    1003ac8f f   LIBCMT:fwrite.obj
 0001:00039d11       __get_errno_from_oserr     1003ad11 f   LIBCMT:dosmap.obj
 0001:00039d53       __errno                    1003ad53 f   LIBCMT:dosmap.obj
 0001:00039d66       ___doserrno                1003ad66 f   LIBCMT:dosmap.obj
 0001:00039d79       __dosmaperr                1003ad79 f   LIBCMT:dosmap.obj
 0001:00039d9c       __set_errno                1003ad9c f   LIBCMT:dosmap.obj
 0001:00039dbd       __get_errno                1003adbd f   LIBCMT:dosmap.obj
 0001:00039dec       __set_doserrno             1003adec f   LIBCMT:dosmap.obj
 0001:00039e0d       __get_doserrno             1003ae0d f   LIBCMT:dosmap.obj
 0001:00039e3c       __CRT_INIT@12              1003ae3c f   LIBCMT:dllcrt0.obj
 0001:0003a067       __DllMainCRTStartup@12     1003b067 f   LIBCMT:dllcrt0.obj
 0001:0003a090       _strlen                    1003b090 f   LIBCMT:strlen.obj
 0001:0003a11b       __EH_prolog3               1003b11b f   LIBCMT:ehprolg3.obj
 0001:0003a14e       __EH_prolog3_catch         1003b14e f   LIBCMT:ehprolg3.obj
 0001:0003a184       __EH_prolog3_GS            1003b184 f   LIBCMT:ehprolg3.obj
 0001:0003a1ba       __EH_prolog3_catch_GS      1003b1ba f   LIBCMT:ehprolg3.obj
 0001:0003a1f3       __EH_epilog3               1003b1f3 f   LIBCMT:ehprolg3.obj
 0001:0003a207       __EH_epilog3_GS            1003b207 f   LIBCMT:ehprolg3.obj
 0001:0003a216       __EH_epilog3_catch_GS      1003b216 f   LIBCMT:ehprolg3.obj
 0001:0003a225       _calloc                    1003b225 f   LIBCMT:calloc.obj
 0001:0003a265       __ftell_nolock             1003b265 f   LIBCMT:ftell.obj
 0001:0003a402       _ftell                     1003b402 f   LIBCMT:ftell.obj
 0001:0003a470       _floor                     1003b470 f   LIBCMT:_floor_pentium4_.obj
 0001:0003a4b0       __floor_pentium4           1003b4b0 f   LIBCMT:_floor_pentium4_.obj
 0001:0003a5a0       __ftol                     1003b5a0 f   LIBCMT:_ftol_.obj
 0001:0003a5d0       __allmul                   1003b5d0 f   LIBCMT:llmul.obj
 0001:0003a604       __toupper                  1003b604 f   LIBCMT:toupper.obj
 0001:0003a611       __toupper_l                1003b611 f   LIBCMT:toupper.obj
 0001:0003a727       _toupper                   1003b727 f   LIBCMT:toupper.obj
 0001:0003a753       _fprintf                   1003b753 f   LIBCMT:fprintf.obj
 0001:0003a86f       __fprintf_l                1003b86f f   LIBCMT:fprintf.obj
 0001:0003a88b       __fprintf_s_l              1003b88b f   LIBCMT:fprintf.obj
 0001:0003a8a7       _fprintf_s                 1003b8a7 f   LIBCMT:fprintf.obj
 0001:0003a8c2       __fprintf_p_l              1003b8c2 f   LIBCMT:fprintf.obj
 0001:0003a8de       __fprintf_p                1003b8de f   LIBCMT:fprintf.obj
 0001:0003a8f9       __get_sys_err_msg          1003b8f9 f i LIBCMT:perror.obj
 0001:0003a921       _perror                    1003b921 f   LIBCMT:perror.obj
 0001:0003a9b0       _ceil                      1003b9b0 f   LIBCMT:_ceil_pentium4_.obj
 0001:0003a9f0       __ceil_pentium4            1003b9f0 f   LIBCMT:_ceil_pentium4_.obj
 0001:0003ab90       _qsort                     1003bb90 f   LIBCMT:qsort.obj
 0001:0003addd       _ldexp                     1003bddd f   LIBCMT:_ldexp_.obj
 0001:0003af8f       __crt_waiting_on_module_handle 1003bf8f f   LIBCMT:crt0dat.obj
 0001:0003afbf       __amsg_exit                1003bfbf f   LIBCMT:crt0dat.obj
 0001:0003afe8       ___crtCorExitProcess       1003bfe8 f   LIBCMT:crt0dat.obj
 0001:0003b013       ___crtExitProcess          1003c013 f   LIBCMT:crt0dat.obj
 0001:0003b02b       __lockexit                 1003c02b f   LIBCMT:crt0dat.obj
 0001:0003b034       __unlockexit               1003c034 f   LIBCMT:crt0dat.obj
 0001:0003b05a       __initterm_e               1003c05a f   LIBCMT:crt0dat.obj
 0001:0003b07e       __get_wpgmptr              1003c07e f   LIBCMT:crt0dat.obj
 0001:0003b0ba       __get_pgmptr               1003c0ba f   LIBCMT:crt0dat.obj
 0001:0003b0f6       __cinit                    1003c0f6 f   LIBCMT:crt0dat.obj
 0001:0003b2a7       _exit                      1003c2a7 f   LIBCMT:crt0dat.obj
 0001:0003b2bd       __exit                     1003c2bd f   LIBCMT:crt0dat.obj
 0001:0003b2d3       __cexit                    1003c2d3 f   LIBCMT:crt0dat.obj
 0001:0003b2e2       __c_exit                   1003c2e2 f   LIBCMT:crt0dat.obj
 0001:0003b2f1       __init_pointers            1003c2f1 f   LIBCMT:crt0dat.obj
 0001:0003b33f       _frexp                     1003c33f f   LIBCMT:_frexp_.obj
 0001:0003b41d       ?strrchr@@YAPADPADH@Z      1003c41d f i LIBCMT:cvt.obj
 0001:0003b428       __invoke_watson_if_error   1003c428 f i LIBCMT:cvt.obj
 0001:0003b44c       __forcdecpt_l              1003c44c f   LIBCMT:cvt.obj
 0001:0003b4bf       __cropzeros_l              1003c4bf f   LIBCMT:cvt.obj
 0001:0003b541       __positive                 1003c541 f   LIBCMT:cvt.obj
 0001:0003b55d       __fassign_l                1003c55d f   LIBCMT:cvt.obj
 0001:0003b59f       __fassign                  1003c59f f   LIBCMT:cvt.obj
 0001:0003b5d8       __forcdecpt                1003c5d8 f   LIBCMT:cvt.obj
 0001:0003b5eb       __cropzeros                1003c5eb f   LIBCMT:cvt.obj
 0001:0003b76d       __cftoe_l                  1003c76d f   LIBCMT:cvt.obj
 0001:0003b83d       __cftoe                    1003c83d f   LIBCMT:cvt.obj
 0001:0003b85d       __cftoa_l                  1003c85d f   LIBCMT:cvt.obj
 0001:0003bbd0       __cftoa                    1003cbd0 f   LIBCMT:cvt.obj
 0001:0003bce7       __cftof_l                  1003cce7 f   LIBCMT:cvt.obj
 0001:0003bda2       __cftof                    1003cda2 f   LIBCMT:cvt.obj
 0001:0003bdbf       __cftog_l                  1003cdbf f   LIBCMT:cvt.obj
 0001:0003beb9       __cftog                    1003ceb9 f   LIBCMT:cvt.obj
 0001:0003bed9       __cfltcvt_l                1003ced9 f   LIBCMT:cvt.obj
 0001:0003bf61       __cfltcvt                  1003cf61 f   LIBCMT:cvt.obj
 0001:0003bf84       __initp_misc_cfltcvt_tab   1003cf84 f   LIBCMT:cmiscdat.obj
 0001:0003bfa5       __setdefaultprecision      1003cfa5 f   LIBCMT:fp8.obj
 0001:0003bfd0       __ms_p5_test_fdiv          1003cfd0 f   LIBCMT:_testfdiv_.obj
 0001:0003c00e       __ms_p5_mp_test_fdiv       1003d00e f   LIBCMT:_testfdiv_.obj
 0001:0003c037       ___heap_select             1003d037 f   LIBCMT:heapinit.obj
 0001:0003c03b       __heap_init                1003d03b f   LIBCMT:heapinit.obj
 0001:0003c06b       __heap_term                1003d06b f   LIBCMT:heapinit.obj
 0001:0003c0df       __get_heap_handle          1003d0df f   LIBCMT:heapinit.obj
 0001:0003c0e5       __mtinitlocks              1003d0e5 f   LIBCMT:mlock.obj
 0001:0003c130       __mtdeletelocks            1003d130 f   LIBCMT:mlock.obj
 0001:0003c187       __unlock                   1003d187 f   LIBCMT:mlock.obj
 0001:0003c19e       __lockerr_exit             1003d19e f   LIBCMT:mlock.obj
 0001:0003c1b6       __mtinitlocknum            1003d1b6 f   LIBCMT:mlock.obj
 0001:0003c279       __lock                     1003d279 f   LIBCMT:mlock.obj
 0001:0003c2ac       __get_sbh_threshold        1003d2ac f   LIBCMT:sbheap.obj
 0001:0003c2cd       __set_amblksiz             1003d2cd f   LIBCMT:sbheap.obj
 0001:0003c318       __get_amblksiz             1003d318 f   LIBCMT:sbheap.obj
 0001:0003c359       ___sbh_heap_init           1003d359 f   LIBCMT:sbheap.obj
 0001:0003c3a7       ___sbh_find_block          1003d3a7 f   LIBCMT:sbheap.obj
 0001:0003c3d7       ___sbh_free_block          1003d3d7 f   LIBCMT:sbheap.obj
 0001:0003c6ed       ___sbh_alloc_new_region    1003d6ed f   LIBCMT:sbheap.obj
 0001:0003c79d       ___sbh_alloc_new_group     1003d79d f   LIBCMT:sbheap.obj
 0001:0003c8a5       ___sbh_resize_block        1003d8a5 f   LIBCMT:sbheap.obj
 0001:0003cb86       ___sbh_heapmin             1003db86 f   LIBCMT:sbheap.obj
 0001:0003cc53       ___sbh_heap_check          1003dc53 f   LIBCMT:sbheap.obj
 0001:0003cf37       __set_sbh_threshold        1003df37 f   LIBCMT:sbheap.obj
 0001:0003cfe6       ___sbh_alloc_block         1003dfe6 f   LIBCMT:sbheap.obj
 0001:0003d2cc       __SEH_prolog4              1003e2cc f   LIBCMT:sehprolg4.obj
 0001:0003d311       __SEH_epilog4              1003e311 f   LIBCMT:sehprolg4.obj
 0001:0003d360       __except_handler4          1003e360 f   LIBCMT:chandler4.obj
 0001:0003d573       __VEC_memcpy               1003e573 f   LIBCMT:p4_memcpy.obj
 0001:0003d6a6       __get_sse2_info            1003e6a6 f   LIBCMT:cpu_disp.obj
 0001:0003d708       ___sse2_available_init     1003e708 f   LIBCMT:cpu_disp.obj
 0001:0003d76c       __VEC_memzero              1003e76c f   LIBCMT:p4_memset.obj
 0001:0003da21       ___updatetmbcinfo          1003ea21 f   LIBCMT:mbctype.obj
 0001:0003db41       __setmbcp_nolock           1003eb41 f   LIBCMT:mbctype.obj
 0001:0003dd26       __getmbcp                  1003ed26 f   LIBCMT:mbctype.obj
 0001:0003dd64       __setmbcp                  1003ed64 f   LIBCMT:mbctype.obj
 0001:0003defe       ___initmbctable            1003eefe f   LIBCMT:mbctype.obj
 0001:0003df1c       ____setlc_active_func      1003ef1c f   LIBCMT:setlocal.obj
 0001:0003df22       ____unguarded_readlc_active_add_func 1003ef22 f   LIBCMT:setlocal.obj
 0001:0003df28       ___freetlocinfo            1003ef28 f   LIBCMT:setlocal.obj
 0001:0003e071       ___addlocaleref            1003f071 f   LIBCMT:setlocal.obj
 0001:0003e100       ___removelocaleref         1003f100 f   LIBCMT:setlocal.obj
 0001:0003e1fd       ___updatetlocinfo          1003f1fd f   LIBCMT:setlocal.obj
 0001:0003e273       __configthreadlocale       1003f273 f   LIBCMT:setlocal.obj
 0001:0003e330       __free_locale              1003f330 f   LIBCMT:setlocal.obj
 0001:0003e3f2       ___free_locale             1003f3f2 f   LIBCMT:setlocal.obj
 0001:0003e3fd       __get_current_locale       1003f3fd f   LIBCMT:setlocal.obj
 0001:0003e4ac       ___get_current_locale      1003f4ac f   LIBCMT:setlocal.obj
 0001:0003e4b1       ___init_dummy              1003f4b1 f   LIBCMT:setlocal.obj
 0001:0003e4b4       __strcats                  1003f4b4 f   LIBCMT:setlocal.obj
 0001:0003e4f4       ___lc_strtolc              1003f4f4 f   LIBCMT:setlocal.obj
 0001:0003e61d       ___lc_lctostr              1003f61d f   LIBCMT:setlocal.obj
 0001:0003e807       __expandlocale             1003f807 f   LIBCMT:setlocal.obj
 0001:0003ef55       __create_locale            1003ff55 f   LIBCMT:setlocal.obj
 0001:0003f04a       ___create_locale           1004004a f   LIBCMT:setlocal.obj
 0001:0003f055       _setlocale                 10040055 f   LIBCMT:setlocal.obj
 0001:0003f1c5       __crt_wait_module_handle   100401c5 f i LIBCMT:tidtable.obj
 0001:0003f1df       __encode_pointer           100401df f   LIBCMT:tidtable.obj
 0001:0003f251       __encoded_null             10040251 f   LIBCMT:tidtable.obj
 0001:0003f25a       __decode_pointer           1004025a f   LIBCMT:tidtable.obj
 0001:0003f2cc       ___crtTlsAlloc@4           100402cc f   LIBCMT:tidtable.obj
 0001:0003f2d5       ___fls_getvalue@4          100402d5 f   LIBCMT:tidtable.obj
 0001:0003f2ef       ___get_flsindex            100402ef f   LIBCMT:tidtable.obj
 0001:0003f2f5       ___set_flsgetvalue         100402f5 f   LIBCMT:tidtable.obj
 0001:0003f329       ___fls_setvalue@8          10040329 f   LIBCMT:tidtable.obj
 0001:0003f346       __mtterm                   10040346 f   LIBCMT:tidtable.obj
 0001:0003f383       __initptd                  10040383 f   LIBCMT:tidtable.obj
 0001:0003f46a       __getptd_noexit            1004046a f   LIBCMT:tidtable.obj
 0001:0003f4e3       __getptd                   100404e3 f   LIBCMT:tidtable.obj
 0001:0003f4fd       __freefls@4                100404fd f   LIBCMT:tidtable.obj
 0001:0003f62c       __freeptd                  1004062c f   LIBCMT:tidtable.obj
 0001:0003f69a       ___threadid                1004069a f   LIBCMT:tidtable.obj
 0001:0003f6a0       ___threadhandle            100406a0 f   LIBCMT:tidtable.obj
 0001:0003f6a6       __mtinit                   100406a6 f   LIBCMT:tidtable.obj
 0001:0003f833       __tolower                  10040833 f   LIBCMT:tolower.obj
 0001:0003f840       __tolower_l                10040840 f   LIBCMT:tolower.obj
 0001:0003f955       _tolower                   10040955 f   LIBCMT:tolower.obj
 0001:0003f981       ___report_gsfailure        10040981 f   LIBCMT:gs_report.obj
 0001:0003fa87       __NMSG_WRITE               10040a87 f   LIBCMT:crt0msg.obj
 0001:0003fc32       __GET_RTERRMSG             10040c32 f   LIBCMT:crt0msg.obj
 0001:0003fc58       __FF_MSGBANNER             10040c58 f   LIBCMT:crt0msg.obj
 0001:0003fc91       __initp_heap_handler       10040c91 f   LIBCMT:handler.obj
 0001:0003fca0       ?_set_new_handler@@YAP6AHI@ZP6AHI@Z@Z 10040ca0 f   LIBCMT:handler.obj
 0001:0003fcd6       ?_set_new_handler@@YAP6AHI@ZH@Z 10040cd6 f   LIBCMT:handler.obj
 0001:0003fcdf       ?_query_new_handler@@YAP6AHI@ZXZ 10040cdf f   LIBCMT:handler.obj
 0001:0003fcec       __callnewh                 10040cec f   LIBCMT:handler.obj
 0001:0003fd14       _wait_a_bit                10040d14 f i LIBCMT:crtheap.obj
 0001:0003fd3a       __set_malloc_crt_max_wait  10040d3a f   LIBCMT:crtheap.obj
 0001:0003fd4f       __malloc_crt               10040d4f f   LIBCMT:crtheap.obj
 0001:0003fd94       __calloc_crt               10040d94 f   LIBCMT:crtheap.obj
 0001:0003fde0       __realloc_crt              10040de0 f   LIBCMT:crtheap.obj
 0001:0003fe2e       __recalloc_crt             10040e2e f   LIBCMT:crtheap.obj
 0001:0003fe80       __msize                    10040e80 f   LIBCMT:msize.obj
 0001:0003ff23       ?terminate@@YAXXZ          10040f23 f   LIBCMT:hooks.obj
 0001:0003ff5c       ?unexpected@@YAXXZ         10040f5c f   LIBCMT:hooks.obj
 0001:0003ff6f       ?_inconsistency@@YAXXZ     10040f6f f   LIBCMT:hooks.obj
 0001:0003ffa7       __initp_eh_hooks           10040fa7 f   LIBCMT:hooks.obj
 0001:0003ffb8       __sse2_mathfcns_init       10040fb8 f   LIBCMT:_mathfcns_.obj
 0001:0003ffcc       __set_SSE2_enable          10040fcc f   LIBCMT:_mathfcns_.obj
 0001:0003fff0       __CIlog_pentium4           10040ff0 f   LIBCMT:_log_pentium4_.obj
 0001:00040008       __log_pentium4             10041008     LIBCMT:_log_pentium4_.obj
 0001:00040271       __fFEXP                    10041271     LIBCMT:_87tran_.obj
 0001:000402d8       __rtinfpopse               100412d8     LIBCMT:_87tran_.obj
 0001:000402da       __rtinfnpopse              100412da     LIBCMT:_87tran_.obj
 0001:000402ea       __fFLN                     100412ea     LIBCMT:_87tran_.obj
 0001:0004039f       __rtinfpop                 1004139f     LIBCMT:_87tran_.obj
 0001:000403a1       __rtinfnpop                100413a1     LIBCMT:_87tran_.obj
 0001:000403be       __ffexpm1                  100413be     LIBCMT:_87tran_.obj
 0001:00040470       __trandisp1                10041470 f   LIBCMT:_87disp_.obj
 0001:000404d7       __trandisp2                100414d7 f   LIBCMT:_87disp_.obj
 0001:00040563       __rttospopde               10041563     LIBCMT:_87disp_.obj
 0001:00040568       __rttospop                 10041568     LIBCMT:_87disp_.obj
 0001:0004056a       __rtnospop                 1004156a     LIBCMT:_87disp_.obj
 0001:0004056c       __rttosnpop                1004156c     LIBCMT:_87disp_.obj
 0001:0004056d       __rtnospopde               1004156d     LIBCMT:_87disp_.obj
 0001:00040574       __rtzeropop                10041574     LIBCMT:_87disp_.obj
 0001:00040576       __rtzeronpop               10041576     LIBCMT:_87disp_.obj
 0001:0004057b       __rtonepop                 1004157b     LIBCMT:_87disp_.obj
 0001:0004057d       __rtonenpop                1004157d     LIBCMT:_87disp_.obj
 0001:00040582       __tosnan1                  10041582     LIBCMT:_87disp_.obj
 0001:000405ad       __nosnan2                  100415ad     LIBCMT:_87disp_.obj
 0001:000405af       __tosnan2                  100415af     LIBCMT:_87disp_.obj
 0001:000405d7       __nan2                     100415d7     LIBCMT:_87disp_.obj
 0001:00040616       __rtindfpop                10041616     LIBCMT:_87disp_.obj
 0001:00040618       __rtindfnpop               10041618     LIBCMT:_87disp_.obj
 0001:00040629       __rttosnpopde              10041629     LIBCMT:_87disp_.obj
 0001:00040633       __rtchsifneg               10041633     LIBCMT:_87disp_.obj
 0001:00040640       __twoToTOS                 10041640 f   LIBCMT:_common_.obj
 0001:00040655       __load_CW                  10041655 f   LIBCMT:_common_.obj
 0001:0004066c       __convertTOStoQNaN         1004166c f   LIBCMT:_common_.obj
 0001:00040685       __fload_withFB             10041685 f   LIBCMT:_common_.obj
 0001:000406c8       __checkTOS_withFB          100416c8 f   LIBCMT:_common_.obj
 0001:000406de       __fast_exit                100416de f   LIBCMT:_common_.obj
 0001:000406eb       __math_exit                100416eb f   LIBCMT:_common_.obj
 0001:00040715       __check_overflow_exit      10041715 f   LIBCMT:_common_.obj
 0001:00040729       __check_range_exit         10041729 f   LIBCMT:_common_.obj
 0001:000407d0       __startTwoArgErrorHandling 100417d0 f   LIBCMT:_genexcep_.obj
 0001:000407e7       __startOneArgErrorHandling 100417e7 f   LIBCMT:_genexcep_.obj
 0001:00040830       __CIpow_pentium4           10041830 f   LIBCMT:_pow_pentium4_.obj
 0001:00040849       __pow_pentium4             10041849     LIBCMT:_pow_pentium4_.obj
 0001:00041390       __d_inttype                10042390 f   LIBCMT:_powhlp_.obj
 0001:000413f6       __powhlp                   100423f6 f   LIBCMT:_powhlp_.obj
 0001:00041536       __crt_debugger_hook        10042536 f   LIBCMT:dbghook.obj
 0001:0004153e       _strcpy_s                  1004253e f   LIBCMT:strcpy_s.obj
 0001:000415a6       ?_Type_info_dtor@type_info@@CAXPAV1@@Z 100425a6 f   LIBCMT:typname.obj
 0001:00041616       ?_Name_base@type_info@@CAPBDPBV1@PAU__type_info_node@@@Z 10042616 f   LIBCMT:typname.obj
 0001:0004170b       ?_Type_info_dtor_internal@type_info@@CAXPAV1@@Z 1004270b f   LIBCMT:typname.obj
 0001:0004177b       ___unDNameHelper           1004277b f   LIBCMT:typname.obj
 0001:000417ae       ?_Name_base_internal@type_info@@CAPBDPBV1@PAU__type_info_node@@@Z 100427ae f   LIBCMT:typname.obj
 0001:000418bd       ___clean_type_info_names_internal 100428bd f   LIBCMT:typname.obj
 0001:00041910       _strcmp                    10042910 f   LIBCMT:strcmp.obj
 0001:00041998       ??0bad_exception@std@@QAE@PBD@Z 10042998 f i LIBCMT:frame.obj
 0001:000419b6       ??1bad_exception@std@@UAE@XZ 100429b6 f i LIBCMT:frame.obj
 0001:000419c1       ??_Ebad_exception@std@@UAEPAXI@Z 100429c1 f i LIBCMT:frame.obj
 0001:000419c1       ??_Gbad_exception@std@@UAEPAXI@Z 100429c1 f i LIBCMT:frame.obj
 0001:000419e8       ___TypeMatch               100429e8 f   LIBCMT:frame.obj
 0001:00041a47       ___FrameUnwindFilter       10042a47 f   LIBCMT:frame.obj
 0001:00041a90       ___FrameUnwindToState      10042a90 f   LIBCMT:frame.obj
 0001:00041bb6       ___DestructExceptionObject 10042bb6 f   LIBCMT:frame.obj
 0001:00041c0b       ___AdjustPointer           10042c0b f   LIBCMT:frame.obj
 0001:00041c34       ?__uncaught_exception@@YA_NXZ 10042c34 f   LIBCMT:frame.obj
 0001:00041c47       ___CxxRegisterExceptionObject 10042c47 f   LIBCMT:frame.obj
 0001:00041cfe       ___CxxDetectRethrow        10042cfe f   LIBCMT:frame.obj
 0001:00041d50       ___CxxUnregisterExceptionObject 10042d50 f   LIBCMT:frame.obj
 0001:00041e8f       ___CxxQueryExceptionSize   10042e8f f   LIBCMT:frame.obj
 0001:00041e93       ___CxxCallUnwindDtor       10042e93 f   LIBCMT:frame.obj
 0001:00041ec5       ___CxxCallUnwindDelDtor    10042ec5 f   LIBCMT:frame.obj
 0001:00041ef8       ___CxxCallUnwindStdDelDtor 10042ef8 f   LIBCMT:frame.obj
 0001:00041f2a       ___CxxCallUnwindVecDtor    10042f2a f   LIBCMT:frame.obj
 0001:0004205b       ?_is_exception_typeof@@YAHABVtype_info@@PAU_EXCEPTION_POINTERS@@@Z 1004305b f   LIBCMT:frame.obj
 0001:0004227d       ___BuildCatchObjectHelper  1004327d f   LIBCMT:frame.obj
 0001:000423fc       ___BuildCatchObject        100433fc f   LIBCMT:frame.obj
 0001:0004248e       ___CxxExceptionFilter      1004348e f   LIBCMT:frame.obj
 0001:00042a7c       ??0bad_exception@std@@QAE@ABV01@@Z 10043a7c f i LIBCMT:frame.obj
 0001:00042a99       ___InternalCxxFrameHandler 10043a99 f   LIBCMT:frame.obj
 0001:00042b80       __CallSettingFrame@12      10043b80 f   LIBCMT:lowhelpr.obj
 0001:00042ba7       __NLG_Return               10043ba7     LIBCMT:lowhelpr.obj
 0001:00042bcc       __flsbuf                   10043bcc f   LIBCMT:_flsbuf.obj
 0001:00042dd6       _get_int_arg               10043dd6 f i LIBCMT:output.obj
 0001:00042de8       _get_int64_arg             10043de8 f i LIBCMT:output.obj
 0001:00042dfd       _get_short_arg             10043dfd f i LIBCMT:output.obj
 0001:00042e10       __output_l                 10043e10 f   LIBCMT:output.obj
 0001:000439a8       __vsnprintf_helper         100449a8 f   LIBCMT:vsnprnc.obj
 0001:00043a74       __vsnprintf_c              10044a74 f   LIBCMT:vsnprnc.obj
 0001:00043a9d       __vsnprintf_c_l            10044a9d f   LIBCMT:vsnprnc.obj
 0001:00043ac7       __vsprintf_s_l             10044ac7 f   LIBCMT:vsnprnc.obj
 0001:00043b4f       _vsprintf_s                10044b4f f   LIBCMT:vsnprnc.obj
 0001:00043b6c       __vsnprintf_s_l            10044b6c f   LIBCMT:vsnprnc.obj
 0001:00043c73       __vsnprintf_s              10044c73 f   LIBCMT:vsnprnc.obj
 0001:00043c93       __vsprintf_p               10044c93 f   LIBCMT:vsnprnc.obj
 0001:00043cbc       __vsprintf_p_l             10044cbc f   LIBCMT:vsnprnc.obj
 0001:00043f15       _strtol                    10044f15 f   LIBCMT:strtol.obj
 0001:00043f40       __strtol_l                 10044f40 f   LIBCMT:strtol.obj
 0001:00043f5d       _strtoul                   10044f5d f   LIBCMT:strtol.obj
 0001:00043f89       __strtoul_l                10044f89 f   LIBCMT:strtol.obj
 0001:0004423d       __strtoi64                 1004523d f   LIBCMT:strtoq.obj
 0001:00044268       __strtoi64_l               10045268 f   LIBCMT:strtoq.obj
 0001:00044285       __strtoui64                10045285 f   LIBCMT:strtoq.obj
 0001:000442b1       __strtoui64_l              100452b1 f   LIBCMT:strtoq.obj
 0001:000442ce       __fltin2                   100452ce f   LIBCMT:_cfin_.obj
 0001:00044375       __isctype_l                10045375 f   LIBCMT:isctype.obj
 0001:0004442d       __isctype                  1004542d f   LIBCMT:isctype.obj
 0001:0004445f       ___addl                    1004545f f i LIBCMT:_strgtold_.obj
 0001:00044483       ___shl_12                  10045483 f i LIBCMT:_strgtold_.obj
 0001:000444b6       ___shr_12                  100454b6 f i LIBCMT:_strgtold_.obj
 0001:000444e8       ___ld12mul                 100454e8 f i LIBCMT:_strgtold_.obj
 0001:00044763       ___multtenpow12            10045763 f i LIBCMT:_strgtold_.obj
 0001:00044a68       ___strgtold12_l            10045a68 f   LIBCMT:_strgtold_.obj
 0001:00045160       ___STRINGTOLD_L            10046160 f   LIBCMT:_strgtold_.obj
 0001:000451bb       __validate_param_reuseA    100461bb f   LIBCMT:outputp.obj
 0001:0004538c       _get_crtdouble_arg         1004638c f i LIBCMT:outputp.obj
 0001:000453a1       __output_p_l               100463a1 f   LIBCMT:outputp.obj
 0001:000466b4       __ismbbkalnum_l            100476b4 f   LIBCMT:ismbbyte.obj
 0001:000466cd       __ismbbkalnum              100476cd f   LIBCMT:ismbbyte.obj
 0001:000466e5       __ismbbkprint_l            100476e5 f   LIBCMT:ismbbyte.obj
 0001:000466fe       __ismbbkprint              100476fe f   LIBCMT:ismbbyte.obj
 0001:00046716       __ismbbkpunct_l            10047716 f   LIBCMT:ismbbyte.obj
 0001:0004672f       __ismbbkpunct              1004772f f   LIBCMT:ismbbyte.obj
 0001:00046747       __ismbbalnum_l             10047747 f   LIBCMT:ismbbyte.obj
 0001:00046763       __ismbbalnum               10047763 f   LIBCMT:ismbbyte.obj
 0001:0004677e       __ismbbalpha_l             1004777e f   LIBCMT:ismbbyte.obj
 0001:0004679a       __ismbbalpha               1004779a f   LIBCMT:ismbbyte.obj
 0001:000467b5       __ismbbgraph_l             100477b5 f   LIBCMT:ismbbyte.obj
 0001:000467d1       __ismbbgraph               100477d1 f   LIBCMT:ismbbyte.obj
 0001:000467ec       __ismbbprint_l             100477ec f   LIBCMT:ismbbyte.obj
 0001:00046808       __ismbbprint               10047808 f   LIBCMT:ismbbyte.obj
 0001:00046823       __ismbbpunct_l             10047823 f   LIBCMT:ismbbyte.obj
 0001:0004683c       __ismbbpunct               1004783c f   LIBCMT:ismbbyte.obj
 0001:00046854       __ismbblead_l              10047854 f   LIBCMT:ismbbyte.obj
 0001:0004686d       __ismbblead                1004786d f   LIBCMT:ismbbyte.obj
 0001:00046885       __ismbbtrail_l             10047885 f   LIBCMT:ismbbyte.obj
 0001:0004689e       __ismbbtrail               1004789e f   LIBCMT:ismbbyte.obj
 0001:000468b6       __ismbbkana_l              100478b6 f   LIBCMT:ismbbyte.obj
 0001:0004690b       __ismbbkana                1004790b f   LIBCMT:ismbbyte.obj
 0001:0004691e       __mbsnbcpy_s               1004791e f   LIBCMT:mbsnbcpy_s.obj
 0001:0004693b       __makepath_s               1004793b f   LIBCMT:makepath_s.obj
 0001:00046a44       __lseek_nolock             10047a44 f   LIBCMT:lseek.obj
 0001:00046ab9       __lseek                    10047ab9 f   LIBCMT:lseek.obj
 0001:00046b95       _fileno                    10047b95 f   LIBCMT:fileno.obj
 0001:00046b95       __fileno                   10047b95 f   LIBCMT:fileno.obj
 0001:00046bc7       __flush                    10047bc7 f   LIBCMT:fflush.obj
 0001:00046c2f       __fflush_nolock            10047c2f f   LIBCMT:fflush.obj
 0001:00046d51       _fflush                    10047d51 f   LIBCMT:fflush.obj
 0001:00046da4       __flushall                 10047da4 f   LIBCMT:fflush.obj
 0001:00046dad       ___iob_func                10047dad f   LIBCMT:_file.obj
 0001:00046db3       ___initstdio               10047db3 f   LIBCMT:_file.obj
 0001:00046e64       ___endstdio                10047e64 f   LIBCMT:_file.obj
 0001:00046e84       __lock_file                10047e84 f   LIBCMT:_file.obj
 0001:00046ec5       __lock_file2               10047ec5 f   LIBCMT:_file.obj
 0001:00046ef7       __unlock_file              10047ef7 f   LIBCMT:_file.obj
 0001:00046f33       __unlock_file2             10047f33 f   LIBCMT:_file.obj
 0001:00046f62       __filbuf                   10047f62 f   LIBCMT:_filbuf.obj
 0001:0004708d       __read_nolock              1004808d f   LIBCMT:read.obj
 0001:0004764f       __read                     1004864f f   LIBCMT:read.obj
 0001:0004774c       __close_nolock             1004874c f   LIBCMT:close.obj
 0001:000477e8       __close                    100487e8 f   LIBCMT:close.obj
 0001:000478b5       __freebuf                  100488b5 f   LIBCMT:_freebuf.obj
 0001:000478e6       __openfile                 100488e6 f   LIBCMT:_open.obj
 0001:00047baf       __getstream                10048baf f   LIBCMT:stream.obj
 0001:00047ce8       __local_unwind4            10048ce8 f   LIBCMT:exsup4.obj
 0001:00047dbe       __seh_longjmp_unwind4@4    10048dbe f   LIBCMT:exsup4.obj
 0001:00047dda       @_EH4_CallFilterFunc@8     10048dda f   LIBCMT:exsup4.obj
 0001:00047df1       @_EH4_TransferToHandler@8  10048df1 f   LIBCMT:exsup4.obj
 0001:00047e0a       @_EH4_GlobalUnwind@4       10048e0a f   LIBCMT:exsup4.obj
 0001:00047e24       @_EH4_LocalUnwind@16       10048e24 f   LIBCMT:exsup4.obj
 0001:00047e40       __CIacos_pentium4          10048e40 f   LIBCMT:_acos_pentium4_.obj
 0001:00047e58       __acos_pentium4            10048e58     LIBCMT:_acos_pentium4_.obj
 0001:000483a0       __CIasin_pentium4          100493a0 f   LIBCMT:_asin_pentium4_.obj
 0001:000483b8       __asin_pentium4            100493b8     LIBCMT:_asin_pentium4_.obj
 0001:00048920       __CIatan_pentium4          10049920 f   LIBCMT:_atan_pentium4_.obj
 0001:00048938       __atan_pentium4            10049938     LIBCMT:_atan_pentium4_.obj
 0001:00048c10       __CIcos_pentium4           10049c10 f   LIBCMT:_cos_pentium4_.obj
 0001:00048c28       __cos_pentium4             10049c28     LIBCMT:_cos_pentium4_.obj
 0001:00048dc0       __CIsin_pentium4           10049dc0 f   LIBCMT:_sin_pentium4_.obj
 0001:00048dd8       __sin_pentium4             10049dd8     LIBCMT:_sin_pentium4_.obj
 0001:00048f88       __set_exp                  10049f88 f   LIBCMT:_util_.obj
 0001:00048fb4       __get_exp                  10049fb4 f   LIBCMT:_util_.obj
 0001:00048fcc       __add_exp                  10049fcc f   LIBCMT:_util_.obj
 0001:00048ff9       __set_bexp                 10049ff9 f   LIBCMT:_util_.obj
 0001:00049020       __sptype                   1004a020 f   LIBCMT:_util_.obj
 0001:00049080       __decomp                   1004a080 f   LIBCMT:_util_.obj
 0001:00049139       __raise_exc_ex             1004a139 f   LIBCMT:_fpexcept_.obj
 0001:00049415       __raise_exc                1004a415 f   LIBCMT:_fpexcept_.obj
 0001:00049438       __raise_excf               1004a438 f   LIBCMT:_fpexcept_.obj
 0001:0004945b       __handle_exc               1004a45b f   LIBCMT:_fpexcept_.obj
 0001:0004963d       __set_errno_from_matherr   1004a63d f   LIBCMT:_fpexcept_.obj
 0001:00049690       __errcode                  1004a690 f   LIBCMT:_fpexcept_.obj
 0001:000496c4       __umatherr                 1004a6c4 f   LIBCMT:_fpexcept_.obj
 0001:00049764       __handle_qnan1             1004a764 f   LIBCMT:_fpexcept_.obj
 0001:000497b9       __handle_qnan2             1004a7b9 f   LIBCMT:_fpexcept_.obj
 0001:0004981a       __except1                  1004a81a f   LIBCMT:_fpexcept_.obj
 0001:000498e3       __except2                  1004a8e3 f   LIBCMT:_fpexcept_.obj
 0001:000499bb       __statfp                   1004a9bb f   LIBCMT:_fpctrl_.obj
 0001:000499cb       __clrfp                    1004a9cb f   LIBCMT:_fpctrl_.obj
 0001:000499dc       __ctrlfp                   1004a9dc f   LIBCMT:_fpctrl_.obj
 0001:00049a05       __set_statfp               1004aa05 f   LIBCMT:_fpctrl_.obj
 0001:00049a5d       ___get_fpsr_sse2           1004aa5d f   LIBCMT:_fpctrl_.obj
 0001:00049a7b       ___set_fpsr_sse2           1004aa7b f   LIBCMT:_fpctrl_.obj
 0001:00049aed       ___fclrf_sse2              1004aaed f   LIBCMT:_fpctrl_.obj
 0001:00049b0a       ___statfp_sse2             1004ab0a f   LIBCMT:_fpctrl_.obj
 0001:00049b1d       ___clrfp_sse2              1004ab1d f   LIBCMT:_fpctrl_.obj
 0001:00049b35       ___ctrlfp_sse2             1004ab35 f   LIBCMT:_fpctrl_.obj
 0001:00049b6c       ___set_statfp_sse2         1004ab6c f   LIBCMT:_fpctrl_.obj
 0001:00049b87       __stbuf                    1004ab87 f   LIBCMT:_sftbuf.obj
 0001:00049c23       __ftbuf                    1004ac23 f   LIBCMT:_sftbuf.obj
 0001:00049c57       _vprintf_helper            1004ac57 f   LIBCMT:vprintf.obj
 0001:00049ce7       __vprintf_l                1004ace7 f   LIBCMT:vprintf.obj
 0001:00049d04       __vprintf_s_l              1004ad04 f   LIBCMT:vprintf.obj
 0001:00049d21       __vprintf_p_l              1004ad21 f   LIBCMT:vprintf.obj
 0001:00049d3e       _vprintf                   1004ad3e f   LIBCMT:vprintf.obj
 0001:00049d5a       _vprintf_s                 1004ad5a f   LIBCMT:vprintf.obj
 0001:00049d76       __vprintf_p                1004ad76 f   LIBCMT:vprintf.obj
 0001:00049d92       __write_nolock             1004ad92 f   LIBCMT:write.obj
 0001:0004a4c5       __write                    1004b4c5 f   LIBCMT:write.obj
 0001:0004a5a1       __ioinit                   1004b5a1 f   LIBCMT:ioinit.obj
 0001:0004a7f5       __ioterm                   1004b7f5 f   LIBCMT:ioinit.obj
 0001:0004a843       __setenvp                  1004b843 f   LIBCMT:stdenvp.obj
 0001:0004a921       __set_pgmptr               1004b921 f i LIBCMT:stdargv.obj
 0001:0004aaca       __setargv                  1004baca f   LIBCMT:stdargv.obj
 0001:0004ab85       ___crtGetEnvironmentStringsA 1004bb85 f   LIBCMT:a_env.obj
 0001:0004acbc       __RTC_Initialize           1004bcbc f   LIBCMT:_initsect_.obj
 0001:0004ace2       __RTC_Terminate            1004bce2 f   LIBCMT:_initsect_.obj
 0001:0004ad08       __initp_misc_winxfltr      1004bd08 f   LIBCMT:winxfltr.obj
 0001:0004ad3e       __XcptFilter               1004bd3e f   LIBCMT:winxfltr.obj
 0001:0004ae9e       ___CppXcptFilter           1004be9e f   LIBCMT:winxfltr.obj
 0001:0004aebe       ___security_init_cookie    1004bebe f   LIBCMT:gs_support.obj
 0001:0004af54       __calloc_impl              1004bf54 f   LIBCMT:calloc_impl.obj
 0001:0004b072       ___libm_setusermatherr     1004c072 f   LIBCMT:_libm_error_.obj
 0001:0004b0a0       ___libm_error_support      1004c0a0 f   LIBCMT:_libm_error_.obj
 0001:0004b350       __floor_default            1004c350 f   LIBCMT:_floor_.obj
 0001:0004b425       __MarkAllocaS              1004c425 f i LIBCMT:a_map.obj
 0001:0004b43b       __freea                    1004c43b f i LIBCMT:a_map.obj
 0001:0004b81e       ___crtLCMapStringA         1004c81e f   LIBCMT:a_map.obj
 0001:0004b863       __isleadbyte_l             1004c863 f i LIBCMT:_wctype.obj
 0001:0004b89b       _isleadbyte                1004c89b f i LIBCMT:_wctype.obj
 0001:0004b8ae       __iswalpha_l               1004c8ae f i LIBCMT:_wctype.obj
 0001:0004b8c8       _iswalpha                  1004c8c8 f i LIBCMT:_wctype.obj
 0001:0004b8de       __iswupper_l               1004c8de f i LIBCMT:_wctype.obj
 0001:0004b8f5       _iswupper                  1004c8f5 f i LIBCMT:_wctype.obj
 0001:0004b908       __iswlower_l               1004c908 f i LIBCMT:_wctype.obj
 0001:0004b91f       _iswlower                  1004c91f f i LIBCMT:_wctype.obj
 0001:0004b932       __iswdigit_l               1004c932 f i LIBCMT:_wctype.obj
 0001:0004b949       _iswdigit                  1004c949 f i LIBCMT:_wctype.obj
 0001:0004b95c       __iswxdigit_l              1004c95c f i LIBCMT:_wctype.obj
 0001:0004b976       _iswxdigit                 1004c976 f i LIBCMT:_wctype.obj
 0001:0004b98c       __iswspace_l               1004c98c f i LIBCMT:_wctype.obj
 0001:0004b9a3       _iswspace                  1004c9a3 f i LIBCMT:_wctype.obj
 0001:0004b9b6       __iswpunct_l               1004c9b6 f i LIBCMT:_wctype.obj
 0001:0004b9cd       _iswpunct                  1004c9cd f i LIBCMT:_wctype.obj
 0001:0004b9e0       __iswalnum_l               1004c9e0 f i LIBCMT:_wctype.obj
 0001:0004b9fa       _iswalnum                  1004c9fa f i LIBCMT:_wctype.obj
 0001:0004ba10       __iswprint_l               1004ca10 f i LIBCMT:_wctype.obj
 0001:0004ba2a       _iswprint                  1004ca2a f i LIBCMT:_wctype.obj
 0001:0004ba40       __iswgraph_l               1004ca40 f i LIBCMT:_wctype.obj
 0001:0004ba5a       _iswgraph                  1004ca5a f i LIBCMT:_wctype.obj
 0001:0004ba70       __iswcntrl_l               1004ca70 f i LIBCMT:_wctype.obj
 0001:0004ba87       _iswcntrl                  1004ca87 f i LIBCMT:_wctype.obj
 0001:0004ba9a       _iswascii                  1004ca9a f i LIBCMT:_wctype.obj
 0001:0004baae       __iswcsym_l                1004caae f i LIBCMT:_wctype.obj
 0001:0004bad8       ___iswcsym                 1004cad8 f i LIBCMT:_wctype.obj
 0001:0004bafe       __iswcsymf_l               1004cafe f i LIBCMT:_wctype.obj
 0001:0004bb28       ___iswcsymf                1004cb28 f i LIBCMT:_wctype.obj
 0001:0004bb4e       _vfprintf_helper           1004cb4e f   LIBCMT:vfprintf.obj
 0001:0004bc69       __vfprintf_l               1004cc69 f   LIBCMT:vfprintf.obj
 0001:0004bc89       __vfprintf_s_l             1004cc89 f   LIBCMT:vfprintf.obj
 0001:0004bca9       __vfprintf_p_l             1004cca9 f   LIBCMT:vfprintf.obj
 0001:0004bcc9       _vfprintf                  1004ccc9 f   LIBCMT:vfprintf.obj
 0001:0004bce8       _vfprintf_s                1004cce8 f   LIBCMT:vfprintf.obj
 0001:0004bd07       __vfprintf_p               1004cd07 f   LIBCMT:vfprintf.obj
 0001:0004bd26       ___sys_nerr                1004cd26 f   LIBCMT:syserr.obj
 0001:0004bd2c       ___sys_errlist             1004cd2c f   LIBCMT:syserr.obj
 0001:0004bd32       __set_osfhnd               1004cd32 f   LIBCMT:osfinfo.obj
 0001:0004bdb3       __free_osfhnd              1004cdb3 f   LIBCMT:osfinfo.obj
 0001:0004be39       __get_osfhandle            1004ce39 f   LIBCMT:osfinfo.obj
 0001:0004beb0       ___lock_fhandle            1004ceb0 f   LIBCMT:osfinfo.obj
 0001:0004bf50       __unlock_fhandle           1004cf50 f   LIBCMT:osfinfo.obj
 0001:0004bf77       __alloc_osfhnd             1004cf77 f   LIBCMT:osfinfo.obj
 0001:0004c111       __open_osfhandle           1004d111 f   LIBCMT:osfinfo.obj
 0001:0004c227       __ceil_default             1004d227 f   LIBCMT:_ceil_.obj
 0001:0004c300       __ValidateImageBase        1004d300 f   LIBCMT:pesect.obj
 0001:0004c340       __FindPESection            1004d340 f   LIBCMT:pesect.obj
 0001:0004c390       __IsNonwritableInCurrentImage 1004d390 f   LIBCMT:pesect.obj
 0001:0004c44d       __initp_misc_winsig        1004d44d f   LIBCMT:winsig.obj
 0001:0004c53d       ___get_sigabrt             1004d53d f   LIBCMT:winsig.obj
 0001:0004c54a       ___fpecode                 1004d54a f   LIBCMT:winsig.obj
 0001:0004c553       ___pxcptinfoptrs           1004d553 f   LIBCMT:winsig.obj
 0001:0004c55c       _signal                    1004d55c f   LIBCMT:winsig.obj
 0001:0004c799       _raise                     1004d799 f   LIBCMT:winsig.obj
 0001:0004c949       __initp_misc_rand_s        1004d949 f   LIBCMT:rand_s.obj
 0001:0004c958       _rand_s                    1004d958 f   LIBCMT:rand_s.obj
 0001:0004ca60       ___getlocaleinfo           1004da60 f   LIBCMT:inithelp.obj
 0001:0004cbdf       __initp_misc_purevirt      1004dbdf f   LIBCMT:inithelp.obj
 0001:0004cbee       __initp_misc_initcrit      1004dbee f   LIBCMT:initcrit.obj
 0001:0004cbfd       ___crtInitCritSecAndSpinCount 1004dbfd f   LIBCMT:initcrit.obj
 0001:0004cc60       _strrchr                   1004dc60 f   LIBCMT:strrchr.obj
 0001:0004cc8d       __isalpha_l                1004dc8d f i LIBCMT:_ctype.obj
 0001:0004cce3       _isalpha                   1004dce3 f i LIBCMT:_ctype.obj
 0001:0004cd13       __isupper_l                1004dd13 f i LIBCMT:_ctype.obj
 0001:0004cd64       _isupper                   1004dd64 f i LIBCMT:_ctype.obj
 0001:0004cd92       __islower_l                1004dd92 f i LIBCMT:_ctype.obj
 0001:0004cde3       _islower                   1004dde3 f i LIBCMT:_ctype.obj
 0001:0004ce11       __isdigit_l                1004de11 f i LIBCMT:_ctype.obj
 0001:0004ce62       _isdigit                   1004de62 f i LIBCMT:_ctype.obj
 0001:0004ce90       __isxdigit_l               1004de90 f i LIBCMT:_ctype.obj
 0001:0004cee6       _isxdigit                  1004dee6 f i LIBCMT:_ctype.obj
 0001:0004cf16       __isspace_l                1004df16 f i LIBCMT:_ctype.obj
 0001:0004cf67       _isspace                   1004df67 f i LIBCMT:_ctype.obj
 0001:0004cf95       __ispunct_l                1004df95 f i LIBCMT:_ctype.obj
 0001:0004cfe6       _ispunct                   1004dfe6 f i LIBCMT:_ctype.obj
 0001:0004d014       __isalnum_l                1004e014 f i LIBCMT:_ctype.obj
 0001:0004d06a       _isalnum                   1004e06a f i LIBCMT:_ctype.obj
 0001:0004d09a       __isprint_l                1004e09a f i LIBCMT:_ctype.obj
 0001:0004d0f0       _isprint                   1004e0f0 f i LIBCMT:_ctype.obj
 0001:0004d120       __isgraph_l                1004e120 f i LIBCMT:_ctype.obj
 0001:0004d176       _isgraph                   1004e176 f i LIBCMT:_ctype.obj
 0001:0004d1a6       __iscntrl_l                1004e1a6 f i LIBCMT:_ctype.obj
 0001:0004d1f7       _iscntrl                   1004e1f7 f i LIBCMT:_ctype.obj
 0001:0004d225       ___isascii                 1004e225 f i LIBCMT:_ctype.obj
 0001:0004d237       ___toascii                 1004e237 f i LIBCMT:_ctype.obj
 0001:0004d244       __iscsymf_l                1004e244 f i LIBCMT:_ctype.obj
 0001:0004d267       ___iscsymf                 1004e267 f i LIBCMT:_ctype.obj
 0001:0004d286       __iscsym_l                 1004e286 f i LIBCMT:_ctype.obj
 0001:0004d2a9       ___iscsym                  1004e2a9 f i LIBCMT:_ctype.obj
 0001:0004d2ca       __atodbl_l                 1004e2ca f   LIBCMT:atodbl.obj
 0001:0004d372       __atodbl                   1004e372 f   LIBCMT:atodbl.obj
 0001:0004d389       __atoldbl_l                1004e389 f   LIBCMT:atodbl.obj
 0001:0004d432       __atoldbl                  1004e432 f   LIBCMT:atodbl.obj
 0001:0004d449       __atoflt_l                 1004e449 f   LIBCMT:atodbl.obj
 0001:0004d4f1       __atoflt                   1004e4f1 f   LIBCMT:atodbl.obj
 0001:0004d508       __set_output_format        1004e508 f   LIBCMT:outputformat.obj
 0001:0004d544       __get_output_format        1004e544 f   LIBCMT:outputformat.obj
 0001:0004d54a       __fptostr                  1004e54a f   LIBCMT:_fptostr.obj
 0001:0004d609       ___dtold                   1004e609 f   LIBCMT:_cfout_.obj
 0001:0004d6c6       __fltout2                  1004e6c6 f   LIBCMT:_cfout_.obj
 0001:0004d760       __alldvrm                  1004e760 f   LIBCMT:lldvrm.obj
 0001:0004d840       __aullshr                  1004e840 f   LIBCMT:ullshr.obj
 0001:0004d85f       __fptrap                   1004e85f f   LIBCMT:crt0fp.obj
 0001:0004d868       __controlfp_s              1004e868 f   LIBCMT:_contrlfp_.obj
 0001:0004da8e       ___crtGetStringTypeA       1004ea8e f   LIBCMT:a_str.obj
 0001:0004dad0       ___pwctype_func            1004ead0 f   LIBCMT:ctype.obj
 0001:0004dad6       ___pctype_func             1004ead6 f   LIBCMT:ctype.obj
 0001:0004df1a       ___free_lc_time            1004ef1a f   LIBCMT:inittime.obj
 0001:0004e0af       ___init_time               1004f0af f   LIBCMT:inittime.obj
 0001:0004e15b       ___free_lconv_num          1004f15b f   LIBCMT:initnum.obj
 0001:0004e1a0       ___init_numeric            1004f1a0 f   LIBCMT:initnum.obj
 0001:0004e39d       ___free_lconv_mon          1004f39d f   LIBCMT:initmon.obj
 0001:0004e42b       ___init_monetary           1004f42b f   LIBCMT:initmon.obj
 0001:0004e6f1       ___init_ctype              1004f6f1 f   LIBCMT:initctyp.obj
 0001:0004ea93       ____mb_cur_max_func        1004fa93 f   LIBCMT:initctyp.obj
 0001:0004eabc       ____mb_cur_max_l_func      1004fabc f   LIBCMT:initctyp.obj
 0001:0004ead8       ____lc_codepage_func       1004fad8 f   LIBCMT:initctyp.obj
 0001:0004eafe       ____lc_collate_cp_func     1004fafe f   LIBCMT:initctyp.obj
 0001:0004eb24       ____lc_handle_func         1004fb24 f   LIBCMT:initctyp.obj
 0001:0004eb4a       ___init_collate            1004fb4a f   LIBCMT:initcoll.obj
 0001:0004eb4d       __Getdays_l                1004fb4d f   LIBCMT:strftime.obj
 0001:0004ec4d       __Getdays                  1004fc4d f   LIBCMT:strftime.obj
 0001:0004ec56       __Getmonths_l              1004fc56 f   LIBCMT:strftime.obj
 0001:0004ed56       __Getmonths                1004fd56 f   LIBCMT:strftime.obj
 0001:0004ed5f       __Gettnames_l              1004fd5f f   LIBCMT:strftime.obj
 0001:0004f0b6       __Gettnames                100500b6 f   LIBCMT:strftime.obj
 0001:0004f9d9       __Strftime_l               100509d9 f   LIBCMT:strftime.obj
 0001:0004fb7d       __strftime_l               10050b7d f   LIBCMT:strftime.obj
 0001:0004fb9d       _strftime                  10050b9d f   LIBCMT:strftime.obj
 0001:0004fbbc       __Strftime                 10050bbc f   LIBCMT:strftime.obj
 0001:0004fbdc       _localeconv                10050bdc f   LIBCMT:lconv.obj
 0001:0004fc02       _strcat_s                  10050c02 f   LIBCMT:strcat_s.obj
 0001:0004fc80       _strcspn                   10050c80 f   LIBCMT:strcspn.obj
 0001:0004fcc6       _strncpy_s                 10050cc6 f   LIBCMT:strncpy_s.obj
 0001:00050376       ___get_qualified_locale    10051376 f   LIBCMT:getqloc.obj
 0001:00051add       _memcmp                    10052add f   LIBCMT:memcmp.obj
 0001:0005315d       _strncmp                   1005415d f   LIBCMT:strncmp.obj
 0001:00053220       _strpbrk                   10054220 f   LIBCMT:strpbrk.obj
 0001:00053260       ___crtMessageBoxA          10054260 f   LIBCMT:crtmbox.obj
 0001:000533c9       __set_error_mode           100543c9 f   LIBCMT:errmode.obj
 0001:00053414       ___set_app_type            10054414 f   LIBCMT:errmode.obj
 0001:00053423       ___get_app_type            10054423 f   LIBCMT:errmode.obj
 0001:00053429       __recalloc                 10054429 f   LIBCMT:recalloc.obj
 0001:000534a4       _abort                     100544a4 f   LIBCMT:abort.obj
 0001:000535bb       __set_abort_behavior       100545bb f   LIBCMT:abort.obj
 0001:000535e0       _fdiv_main_routine         100545e0 f   LIBCMT:_adj_fdiv_.obj
 0001:000536f7       __adj_fdiv_r               100546f7 f   LIBCMT:_adj_fdiv_.obj
 0001:00053b96       __fdivp_sti_st             10054b96 f   LIBCMT:_adj_fdiv_.obj
 0001:00053ba9       __fdivrp_sti_st            10054ba9 f   LIBCMT:_adj_fdiv_.obj
 0001:00053bbc       __adj_fdiv_m32             10054bbc f   LIBCMT:_adj_fdiv_.obj
 0001:00053c08       __adj_fdiv_m64             10054c08 f   LIBCMT:_adj_fdiv_.obj
 0001:00053c54       __adj_fdiv_m16i            10054c54 f   LIBCMT:_adj_fdiv_.obj
 0001:00053c88       __adj_fdiv_m32i            10054c88 f   LIBCMT:_adj_fdiv_.obj
 0001:00053cbc       __adj_fdivr_m32            10054cbc f   LIBCMT:_adj_fdiv_.obj
 0001:00053d08       __adj_fdivr_m64            10054d08 f   LIBCMT:_adj_fdiv_.obj
 0001:00053d54       __adj_fdivr_m16i           10054d54 f   LIBCMT:_adj_fdiv_.obj
 0001:00053d88       __adj_fdivr_m32i           10054d88 f   LIBCMT:_adj_fdiv_.obj
 0001:00053dbc       __safe_fdiv                10054dbc f   LIBCMT:_adj_fdiv_.obj
 0001:00053dd1       __safe_fdivr               10054dd1 f   LIBCMT:_adj_fdiv_.obj
 0001:00053de6       __fprem_common             10054de6 f   LIBCMT:_adj_fdiv_.obj
 0001:00053fec       __adj_fprem                10054fec f   LIBCMT:_adj_fdiv_.obj
 0001:0005409e       __fprem1_common            1005509e f   LIBCMT:_adj_fdiv_.obj
 0001:000542a4       __adj_fprem1               100552a4 f   LIBCMT:_adj_fdiv_.obj
 0001:00054359       __safe_fprem               10055359 f   LIBCMT:_adj_fdiv_.obj
 0001:0005435f       __safe_fprem1              1005535f f   LIBCMT:_adj_fdiv_.obj
 0001:00054365       __adj_fpatan               10055365 f   LIBCMT:_adj_fdiv_.obj
 0001:00054368       __adj_fptan                10055368 f   LIBCMT:_adj_fdiv_.obj
 0001:0005436b       __87except                 1005536b f   LIBCMT:_87except_.obj
 0001:000544aa       __frnd                     100554aa f   LIBCMT:_frnd_.obj
 0001:000544be       ??0Block@HeapManager@@QAE@XZ 100554be f i LIBCMT:undname.obj
 0001:000544c4       ?Constructor@HeapManager@@QAEXP6APAXI@ZP6AXPAX@Z@Z 100554c4 f i LIBCMT:undname.obj
 0001:000544e3       ?Destructor@HeapManager@@QAEXXZ 100554e3 f i LIBCMT:undname.obj
 0001:0005450b       ?getNumberOfDimensions@UnDecorator@@CAHXZ 1005550b f   LIBCMT:undname.obj
 0001:0005456e       ?getTypeEncoding@UnDecorator@@CAHXZ 1005556e f i LIBCMT:undname.obj
 0001:00054a5a       ?doUnderScore@UnDecorator@@SAHXZ 10055a5a f i LIBCMT:undname.obj
 0001:00054a65       ?doMSKeywords@UnDecorator@@SAHXZ 10055a65 f i LIBCMT:undname.obj
 0001:00054a72       ?doPtr64@UnDecorator@@SAHXZ 10055a72 f i LIBCMT:undname.obj
 0001:00054a80       ?doFunctionReturns@UnDecorator@@SAHXZ 10055a80 f i LIBCMT:undname.obj
 0001:00054a8e       ?doAllocationModel@UnDecorator@@SAHXZ 10055a8e f i LIBCMT:undname.obj
 0001:00054a9c       ?doAllocationLanguage@UnDecorator@@SAHXZ 10055a9c f i LIBCMT:undname.obj
 0001:00054aaa       ?doThisTypes@UnDecorator@@SAHXZ 10055aaa f i LIBCMT:undname.obj
 0001:00054abc       ?doAccessSpecifiers@UnDecorator@@SAHXZ 10055abc f i LIBCMT:undname.obj
 0001:00054aca       ?doThrowTypes@UnDecorator@@SAHXZ 10055aca f i LIBCMT:undname.obj
 0001:00054ad8       ?doMemberTypes@UnDecorator@@SAHXZ 10055ad8 f i LIBCMT:undname.obj
 0001:00054ae6       ?doNameOnly@UnDecorator@@SAHXZ 10055ae6 f i LIBCMT:undname.obj
 0001:00054af1       ?doTypeOnly@UnDecorator@@SAHXZ 10055af1 f i LIBCMT:undname.obj
 0001:00054afc       ?haveTemplateParameters@UnDecorator@@SAHXZ 10055afc f i LIBCMT:undname.obj
 0001:00054b07       ?doEcsu@UnDecorator@@SAHXZ 10055b07 f i LIBCMT:undname.obj
 0001:00054b15       ?doNoIdentCharCheck@UnDecorator@@SAHXZ 10055b15 f i LIBCMT:undname.obj
 0001:00054b20       ?doEllipsis@UnDecorator@@SAHXZ 10055b20 f i LIBCMT:undname.obj
 0001:00054b2e       ?UScore@UnDecorator@@SAPBDW4Tokens@@@Z 10055b2e f   LIBCMT:undname.obj
 0001:00054b4c       ?getMemory@HeapManager@@QAEPAXIH@Z 10055b4c f   LIBCMT:undname.obj
 0001:00054bd4       ??0DName@@QAE@XZ           10055bd4 f i LIBCMT:undname.obj
 0001:00054be5       ??0DName@@QAE@ABV0@@Z      10055be5 f i LIBCMT:undname.obj
 0001:00054bfd       ?isValid@DName@@QBEHXZ     10055bfd f i LIBCMT:undname.obj
 0001:00054c07       ?isEmpty@DName@@QBEHXZ     10055c07 f i LIBCMT:undname.obj
 0001:00054c0f       ?status@DName@@QBE?AW4DNameStatus@@XZ 10055c0f f i LIBCMT:undname.obj
 0001:00054c14       ?setPtrRef@DName@@QAEAAV1@XZ 10055c14 f i LIBCMT:undname.obj
 0001:00054c1e       ?isPtrRef@DName@@QBEHXZ    10055c1e f i LIBCMT:undname.obj
 0001:00054c28       ?isUDC@DName@@QBEHXZ       10055c28 f i LIBCMT:undname.obj
 0001:00054c39       ?setIsUDC@DName@@QAEXXZ    10055c39 f i LIBCMT:undname.obj
 0001:00054c46       ?isUDTThunk@DName@@QBEHXZ  10055c46 f i LIBCMT:undname.obj
 0001:00054c57       ?setIsArray@DName@@QAEXXZ  10055c57 f i LIBCMT:undname.obj
 0001:00054c5f       ?isArray@DName@@QBEHXZ     10055c5f f i LIBCMT:undname.obj
 0001:00054c69       ?isNoTE@DName@@QBEHXZ      10055c69 f i LIBCMT:undname.obj
 0001:00054c73       ?setIsNoTE@DName@@QAEXXZ   10055c73 f i LIBCMT:undname.obj
 0001:00054c7b       ?isPinPtr@DName@@QBEHXZ    10055c7b f i LIBCMT:undname.obj
 0001:00054c85       ?setIsPinPtr@DName@@QAEXXZ 10055c85 f i LIBCMT:undname.obj
 0001:00054c8d       ?isComArray@DName@@QBEHXZ  10055c8d f i LIBCMT:undname.obj
 0001:00054c97       ?setIsComArray@DName@@QAEXXZ 10055c97 f i LIBCMT:undname.obj
 0001:00054c9f       ?isVCallThunk@DName@@QBEHXZ 10055c9f f i LIBCMT:undname.obj
 0001:00054ca9       ?setIsVCallThunk@DName@@QAEXXZ 10055ca9 f i LIBCMT:undname.obj
 0001:00054cb1       ?length@DName@@QBEHXZ      10055cb1 f i LIBCMT:undname.obj
 0001:00054cbe       ?getLastChar@DName@@QBEDXZ 10055cbe f i LIBCMT:undname.obj
 0001:00054ccc       ?getString@DName@@QBEPADPAD0@Z 10055ccc f i LIBCMT:undname.obj
 0001:00054ce4       ??_5DName@@QAEAAV0@ABV0@@Z 10055ce4 f   LIBCMT:undname.obj
 0001:00054d03       ??4DName@@QAEAAV0@ABV0@@Z  10055d03 f   LIBCMT:undname.obj
 0001:00054d1b       ?isFull@Replicator@@QBEHXZ 10055d1b f i LIBCMT:undname.obj
 0001:00054d24       ??0Replicator@@QAE@XZ      10055d24 f i LIBCMT:undname.obj
 0001:00054d2a       ??0DNameNode@@IAE@XZ       10055d2a f   LIBCMT:undname.obj
 0001:00054d33       ??0charNode@@QAE@D@Z       10055d33 f   LIBCMT:undname.obj
 0001:00054d4a       ?length@charNode@@UBEHXZ   10055d4a f i LIBCMT:undname.obj
 0001:00054d4e       ?getLastChar@charNode@@UBEDXZ 10055d4e f i LIBCMT:undname.obj
 0001:00054d52       ?getString@charNode@@UBEPADPAD0@Z 10055d52 f i LIBCMT:undname.obj
 0001:00054d69       ??0pDNameNode@@QAE@PAVDName@@@Z 10055d69 f   LIBCMT:undname.obj
 0001:00054d93       ?length@pDNameNode@@UBEHXZ 10055d93 f i LIBCMT:undname.obj
 0001:00054da9       ?getLastChar@pDNameNode@@UBEDXZ 10055da9 f i LIBCMT:undname.obj
 0001:00054dc0       ?getString@pDNameNode@@UBEPADPAD0@Z 10055dc0 f i LIBCMT:undname.obj
 0001:00054dd9       ??0DNameStatusNode@@AAE@W4DNameStatus@@@Z 10055dd9 f   LIBCMT:undname.obj
 0001:00054dfe       ?length@DNameStatusNode@@UBEHXZ 10055dfe f i LIBCMT:undname.obj
 0001:00054e02       ?getLastChar@DNameStatusNode@@UBEDXZ 10055e02 f i LIBCMT:undname.obj
 0001:00054e0e       ?make@DNameStatusNode@@SAPAV1@W4DNameStatus@@@Z 10055e0e f i LIBCMT:undname.obj
 0001:00054e94       ??0pairNode@@QAE@PAVDNameNode@@0@Z 10055e94 f   LIBCMT:undname.obj
 0001:00054eb5       ?length@pairNode@@UBEHXZ   10055eb5 f i LIBCMT:undname.obj
 0001:00054ee0       ?getLastChar@pairNode@@UBEDXZ 10055ee0 f i LIBCMT:undname.obj
 0001:00054efc       ?getString@pairNode@@UBEPADPAD0@Z 10055efc f i LIBCMT:undname.obj
 0001:00054f76       ??0UnDecorator@@QAE@PADPBDHP6APADJ@ZK@Z 10055f76 f i LIBCMT:undname.obj
 0001:00054fe5       ?getDataIndirectType@UnDecorator@@CA?AVDName@@XZ 10055fe5 f i LIBCMT:undname.obj
 0001:0005501a       ?getThisType@UnDecorator@@CA?AVDName@@XZ 1005601a f i LIBCMT:undname.obj
 0001:00055050       ??2@YAPAXIAAVHeapManager@@H@Z 10056050 f i LIBCMT:undname.obj
 0001:00055067       ?getStringHelper@@YAPADPAD00H@Z 10056067 f i LIBCMT:undname.obj
 0001:0005509e       ??0DName@@QAE@PAV0@@Z      1005609e f   LIBCMT:undname.obj
 0001:000550f1       ??0DName@@QAE@W4DNameStatus@@@Z 100560f1 f   LIBCMT:undname.obj
 0001:00055136       ?getString@DName@@QBEPADPADH@Z 10056136 f i LIBCMT:undname.obj
 0001:0005518e       ?append@DName@@AAEXPAVDNameNode@@@Z 1005618e f   LIBCMT:undname.obj
 0001:000551cd       ??4DName@@QAEAAV0@PAV0@@Z  100561cd f   LIBCMT:undname.obj
 0001:0005521a       ??4DName@@QAEAAV0@W4DNameStatus@@@Z 1005621a f   LIBCMT:undname.obj
 0001:00055251       ??YReplicator@@QAEAAV0@ABVDName@@@Z 10056251 f   LIBCMT:undname.obj
 0001:0005529b       ??AReplicator@@QBE?AVDName@@H@Z 1005629b f   LIBCMT:undname.obj
 0001:000552db       ??0pcharNode@@QAE@PBDH@Z   100562db f   LIBCMT:undname.obj
 0001:00055332       ?length@pcharNode@@UBEHXZ  10056332 f i LIBCMT:undname.obj
 0001:00055336       ?getLastChar@pcharNode@@UBEDXZ 10056336 f i LIBCMT:undname.obj
 0001:00055348       ?getString@pcharNode@@UBEPADPAD0@Z 10056348 f i LIBCMT:undname.obj
 0001:00055365       ?getString@DNameStatusNode@@UBEPADPAD0@Z 10056365 f i LIBCMT:undname.obj
 0001:0005538e       ?getReturnType@UnDecorator@@CA?AVDName@@PAV2@@Z 1005638e f   LIBCMT:undname.obj
 0001:000553bf       ?getStorageConvention@UnDecorator@@CA?AVDName@@XZ 100563bf f i LIBCMT:undname.obj
 0001:000553d2       ??YDName@@QAEAAV0@W4DNameStatus@@@Z 100563d2 f   LIBCMT:undname.obj
 0001:00055414       ?doPchar@DName@@AAEXPBDH@Z 10056414 f   LIBCMT:undname.obj
 0001:00055490       ??0DName@@QAE@D@Z          10056490 f   LIBCMT:undname.obj
 0001:000554bd       ??0DName@@QAE@PBD@Z        100564bd f   LIBCMT:undname.obj
 0001:000554f6       ??0DName@@QAE@AAPBDD@Z     100564f6 f   LIBCMT:undname.obj
 0001:000555b5       ??0DName@@QAE@_K@Z         100565b5 f   LIBCMT:undname.obj
 0001:00055623       ??0DName@@QAE@_J@Z         10056623 f   LIBCMT:undname.obj
 0001:000556be       ??HDName@@QBE?AV0@W4DNameStatus@@@Z 100566be f   LIBCMT:undname.obj
 0001:000556e2       ??YDName@@QAEAAV0@ABV0@@Z  100566e2 f   LIBCMT:undname.obj
 0001:00055725       ??YDName@@QAEAAV0@PAV0@@Z  10056725 f   LIBCMT:undname.obj
 0001:0005578c       ??4DName@@QAEAAV0@D@Z      1005678c f i LIBCMT:undname.obj
 0001:000557b9       ??4DName@@QAEAAV0@PBD@Z    100567b9 f   LIBCMT:undname.obj
 0001:000557ee       ?getCallingConvention@UnDecorator@@CA?AVDName@@XZ 100567ee f   LIBCMT:undname.obj
 0001:00055898       ?getVCallThunkType@UnDecorator@@CA?AVDName@@XZ 10056898 f i LIBCMT:undname.obj
 0001:000558d1       ??HDName@@QBE?AV0@ABV0@@Z  100568d1 f   LIBCMT:undname.obj
 0001:000558f5       ??HDName@@QBE?AV0@PAV0@@Z  100568f5 f   LIBCMT:undname.obj
 0001:00055919       ??YDName@@QAEAAV0@D@Z      10056919 f   LIBCMT:undname.obj
 0001:0005596b       ??YDName@@QAEAAV0@PBD@Z    1005696b f   LIBCMT:undname.obj
 0001:000559cf       ?getArgumentList@UnDecorator@@CA?AVDName@@XZ 100569cf f   LIBCMT:undname.obj
 0001:00055ad1       ?getVdispMapType@UnDecorator@@CA?AVDName@@ABV2@@Z 10056ad1 f i LIBCMT:undname.obj
 0001:00055b25       ??H@YA?AVDName@@DABV0@@Z   10056b25 f i LIBCMT:undname.obj
 0001:00055b49       ??H@YA?AVDName@@W4DNameStatus@@ABV0@@Z 10056b49 f i LIBCMT:undname.obj
 0001:00055b6d       ??H@YA?AVDName@@PBDABV0@@Z 10056b6d f i LIBCMT:undname.obj
 0001:00055b91       ??HDName@@QBE?AV0@D@Z      10056b91 f   LIBCMT:undname.obj
 0001:00055bb5       ??HDName@@QBE?AV0@PBD@Z    10056bb5 f   LIBCMT:undname.obj
 0001:00055bd9       ?getDimension@UnDecorator@@CA?AVDName@@_N@Z 10056bd9 f   LIBCMT:undname.obj
 0001:00055d2b       ?getEnumType@UnDecorator@@CA?AVDName@@XZ 10056d2b f i LIBCMT:undname.obj
 0001:00055dff       ?getArgumentTypes@UnDecorator@@CA?AVDName@@XZ 10056dff f   LIBCMT:undname.obj
 0001:00055edb       ?getThrowTypes@UnDecorator@@CA?AVDName@@XZ 10056edb f   LIBCMT:undname.obj
 0001:00055f5a       ?getExtendedDataIndirectType@UnDecorator@@CA?AVDName@@AADAA_NH@Z 10056f5a f   LIBCMT:undname.obj
 0001:000560d7       ?getArrayType@UnDecorator@@CA?AVDName@@ABV2@@Z 100570d7 f i LIBCMT:undname.obj
 0001:00056251       ?getLexicalFrame@UnDecorator@@CA?AVDName@@XZ 10057251 f i LIBCMT:undname.obj
 0001:00056284       ?getDisplacement@UnDecorator@@CA?AVDName@@XZ 10057284 f i LIBCMT:undname.obj
 0001:0005629a       ?getCallIndex@UnDecorator@@CA?AVDName@@XZ 1005729a f i LIBCMT:undname.obj
 0001:000562b0       ?getGuardNumber@UnDecorator@@CA?AVDName@@XZ 100572b0 f i LIBCMT:undname.obj
 0001:000562c6       ?getVfTableType@UnDecorator@@CA?AVDName@@ABV2@@Z 100572c6 f i LIBCMT:undname.obj
 0001:000563fd       ?getStringEncoding@UnDecorator@@CA?AVDName@@PADH@Z 100573fd f   LIBCMT:undname.obj
 0001:000564a1       ?getSignedDimension@UnDecorator@@CA?AVDName@@XZ 100574a1 f   LIBCMT:undname.obj
 0001:000564f3       ?getTemplateConstant@UnDecorator@@CA?AVDName@@XZ 100574f3 f   LIBCMT:undname.obj
 0001:000567c0       ?getPtrRefDataType@UnDecorator@@CA?AVDName@@ABV2@H@Z 100577c0 f i LIBCMT:undname.obj
 0001:0005689e       ?getVbTableType@UnDecorator@@CA?AVDName@@ABV2@@Z 1005789e f i LIBCMT:undname.obj
 0001:000568b5       ?getTemplateArgumentList@UnDecorator@@CA?AVDName@@XZ 100578b5 f   LIBCMT:undname.obj
 0001:00056a79       ?getOperatorName@UnDecorator@@CA?AVDName@@_NPA_N@Z 10057a79 f i LIBCMT:undname.obj
 0001:00057016       ?getTemplateName@UnDecorator@@CA?AVDName@@_N@Z 10058016 f   LIBCMT:undname.obj
 0001:0005715d       ?getZName@UnDecorator@@CA?AVDName@@_N0@Z 1005815d f   LIBCMT:undname.obj
 0001:00057353       ?getScopedName@UnDecorator@@CA?AVDName@@XZ 10058353 f   LIBCMT:undname.obj
 0001:00057424       ?getECSUName@UnDecorator@@CA?AVDName@@XZ 10058424 f i LIBCMT:undname.obj
 0001:00057437       ?getECSUDataType@UnDecorator@@CA?AVDName@@XZ 10058437 f   LIBCMT:undname.obj
 0001:0005753e       ?getSymbolName@UnDecorator@@CA?AVDName@@XZ 1005853e f i LIBCMT:undname.obj
 0001:00057588       ?getBasedType@UnDecorator@@CA?AVDName@@XZ 10058588 f   LIBCMT:undname.obj
 0001:00057620       ?composeDeclaration@UnDecorator@@CA?AVDName@@ABV2@@Z 10058620 f i LIBCMT:undname.obj
 0001:000581bb       ?getDecoratedName@UnDecorator@@CA?AVDName@@XZ 100591bb f   LIBCMT:undname.obj
 0001:000583d3       ?getScope@UnDecorator@@CA?AVDName@@XZ 100593d3 f   LIBCMT:undname.obj
 0001:00058643       ?getFunctionIndirectType@UnDecorator@@CA?AVDName@@ABV2@@Z 10059643 f   LIBCMT:undname.obj
 0001:00058997       ?getDataIndirectType@UnDecorator@@CA?AVDName@@ABV2@D0H@Z 10059997 f   LIBCMT:undname.obj
 0001:00058e5e       ??BUnDecorator@@QAEPADXZ   10059e5e f i LIBCMT:undname.obj
 0001:00058f8f       ?getPtrRefType@UnDecorator@@CA?AVDName@@ABV2@0D@Z 10059f8f f   LIBCMT:undname.obj
 0001:00059088       ?getPointerType@UnDecorator@@CA?AVDName@@ABV2@0@Z 1005a088 f i LIBCMT:undname.obj
 0001:000590a5       ?getPointerTypeArray@UnDecorator@@CA?AVDName@@ABV2@0@Z 1005a0a5 f i LIBCMT:undname.obj
 0001:000590c2       ?getReferenceType@UnDecorator@@CA?AVDName@@ABV2@0@Z 1005a0c2 f i LIBCMT:undname.obj
 0001:000590df       ___unDName                 1005a0df f   LIBCMT:undname.obj
 0001:00059179       ___unDNameEx               1005a179 f   LIBCMT:undname.obj
 0001:00059213       ?getBasicDataType@UnDecorator@@CA?AVDName@@ABV2@@Z 1005a213 f   LIBCMT:undname.obj
 0001:000595ca       ?getPrimaryDataType@UnDecorator@@CA?AVDName@@ABV2@@Z 1005a5ca f   LIBCMT:undname.obj
 0001:00059702       ?getDataType@UnDecorator@@CA?AVDName@@PAV2@@Z 1005a702 f   LIBCMT:undname.obj
 0001:000597c2       ?getExternalDataType@UnDecorator@@CA?AVDName@@ABV2@@Z 1005a7c2 f i LIBCMT:undname.obj
 0001:00059830       ?_ValidateRead@@YAHPBXI@Z  1005a830 f   LIBCMT:validate.obj
 0001:00059842       ?_ValidateWrite@@YAHPAXI@Z 1005a842 f   LIBCMT:validate.obj
 0001:00059854       ?_ValidateExecute@@YAHP6GHXZ@Z 1005a854 f   LIBCMT:validate.obj
 0001:00059868       __global_unwind2           1005a868 f   LIBCMT:exsup.obj
 0001:000598cd       __local_unwind2            1005a8cd f   LIBCMT:exsup.obj
 0001:00059951       __abnormal_termination     1005a951 f   LIBCMT:exsup.obj
 0001:00059974       __NLG_Notify1              1005a974 f   LIBCMT:exsup.obj
 0001:0005997d       __NLG_Notify               1005a97d f   LIBCMT:exsup.obj
 0001:00059994       __NLG_Dispatch2            1005a994     LIBCMT:exsup.obj
 0001:00059994       __NLG_Dispatch             1005a994     LIBCMT:exsup.obj
 0001:0005999c       __NLG_Call                 1005a99c f   LIBCMT:exsup.obj
 0001:0005999e       __NLG_Return2              1005a99e     LIBCMT:exsup.obj
 0001:0005999f       __lseeki64_nolock          1005a99f f   LIBCMT:lseeki64.obj
 0001:00059a24       __lseeki64                 1005aa24 f   LIBCMT:lseeki64.obj
 0001:00059b3d       __getbuf                   1005ab3d f   LIBCMT:_getbuf.obj
 0001:00059b86       __isatty                   1005ab86 f   LIBCMT:isatty.obj
 0001:00059bea       __wctomb_s_l               1005abea f   LIBCMT:wctomb.obj
 0001:00059d56       _wctomb_s                  1005ad56 f   LIBCMT:wctomb.obj
 0001:00059d73       __wctomb_l                 1005ad73 f   LIBCMT:wctomb.obj
 0001:00059dc4       _wctomb                    1005adc4 f   LIBCMT:wctomb.obj
 0001:00059e00       __aulldvrm                 1005ae00 f   LIBCMT:ulldvrm.obj
 0001:00059f3b       __output_s_l               1005af3b f   LIBCMT:outputs.obj
 0001:0005ab0b       __ZeroTail                 1005bb0b f i LIBCMT:_intrncvt_.obj
 0001:0005ab54       __IncMan                   1005bb54 f i LIBCMT:_intrncvt_.obj
 0001:0005abc1       __RoundMan                 1005bbc1 f i LIBCMT:_intrncvt_.obj
 0001:0005acb1       __CopyMan                  1005bcb1 f i LIBCMT:_intrncvt_.obj
 0001:0005acd0       __FillZeroMan              1005bcd0 f i LIBCMT:_intrncvt_.obj
 0001:0005ace1       __IsZeroMan                1005bce1 f i LIBCMT:_intrncvt_.obj
 0001:0005ad00       __ShrMan                   1005bd00 f i LIBCMT:_intrncvt_.obj
 0001:0005ad9a       __ld12cvt                  1005bd9a f i LIBCMT:_intrncvt_.obj
 0001:0005b2c5       __ld12tod                  1005c2c5 f   LIBCMT:_intrncvt_.obj
 0001:0005b809       __ld12tof                  1005c809 f   LIBCMT:_intrncvt_.obj
 0001:0005bd4d       __ld12told                 1005cd4d f   LIBCMT:_intrncvt_.obj
 0001:0005be14       ___add_12                  1005ce14 f i LIBCMT:_mantold_.obj
 0001:0005be85       ___mtold12                 1005ce85 f   LIBCMT:_mantold_.obj
 0001:0005c053       __mbsnbcpy_s_l             1005d053 f   LIBCMT:mbsnbcpy_s_l.obj
 0001:0005c262       __mbsdec_l                 1005d262 f   LIBCMT:mbsdec.obj
 0001:0005c2fb       __mbsdec                   1005d2fb f   LIBCMT:mbsdec.obj
 0001:0005c312       __commit                   1005d312 f   LIBCMT:commit.obj
 0001:0005c3f3       __fcloseall                1005d3f3 f   LIBCMT:closeall.obj
 0001:0005cbb1       __open                     1005dbb1 f   LIBCMT:open.obj
 0001:0005cc67       __sopen_helper             1005dc67 f   LIBCMT:open.obj
 0001:0005cd33       __sopen                    1005dd33 f   LIBCMT:open.obj
 0001:0005cd65       __sopen_s                  1005dd65 f   LIBCMT:open.obj
 0001:0005cd85       __mbsnbicmp_l              1005dd85 f   LIBCMT:mbsnbicm.obj
 0001:0005cfb0       __mbsnbicmp                1005dfb0 f   LIBCMT:mbsnbicm.obj
 0001:0005cfca       __mbsnbcmp_l               1005dfca f   LIBCMT:mbsnbcmp.obj
 0001:0005d134       __mbsnbcmp                 1005e134 f   LIBCMT:mbsnbcmp.obj
 0001:0005d14e       __matherr                  1005e14e f   LIBCMT:_matherr_.obj
 0001:0005d151       __putwch_nolock            1005e151 f   LIBCMT:putwch.obj
 0001:0005d216       __cputws                   1005e216 f   LIBCMT:putwch.obj
 0001:0005d2b5       __putwch                   1005e2b5 f   LIBCMT:putwch.obj
 0001:0005d2fb       __mbtowc_l                 1005e2fb f   LIBCMT:mbtowc.obj
 0001:0005d412       _mbtowc                    1005e412 f   LIBCMT:mbtowc.obj
 0001:0005d42c       ___ansicp                  1005e42c f   LIBCMT:convrtcp.obj
 0001:0005d475       ___convertcp               1005e475 f   LIBCMT:convrtcp.obj
 0001:0005d630       __alloca_probe_16          1005e630 f   LIBCMT:alloca16.obj
 0001:0005d646       __alloca_probe_8           1005e646     LIBCMT:alloca16.obj
 0001:0005d65c       __iswctype_l               1005e65c f   LIBCMT:iswctype.obj
 0001:0005d6e6       _iswctype                  1005e6e6 f   LIBCMT:iswctype.obj
 0001:0005d75c       _is_wctype                 1005e75c f   LIBCMT:iswctype.obj
 0001:0005d780       ___crtGetLocaleInfoW       1005e780 f   LIBCMT:w_loc.obj
 0001:0005d8f3       ___crtGetLocaleInfoA       1005e8f3 f   LIBCMT:a_loc.obj
 0001:0005d930       _$I10_OUTPUT               1005e930 f   LIBCMT:_x10fout_.obj
 0001:0005e254       __set_controlfp            1005f254 f   LIBCMT:_ieee87_.obj
 0001:0005e5c8       __statusfp                 1005f5c8 f   LIBCMT:_ieee87_.obj
 0001:0005e65a       __fpreset                  1005f65a f   LIBCMT:_ieee87_.obj
 0001:0005e893       __statusfp2                1005f893 f   LIBCMT:_ieee87_.obj
 0001:0005e8ed       __clearfp                  1005f8ed f   LIBCMT:_ieee87_.obj
 0001:0005e9c6       ___control87_2             1005f9c6 f   LIBCMT:_ieee87_.obj
 0001:0005ecda       __control87                1005fcda f i LIBCMT:_ieee87_.obj
 0001:0005efe9       __controlfp                1005ffe9 f   LIBCMT:_ieee87_.obj
 0001:0005f2fb       __get_daylight             100602fb f   LIBCMT:timeset.obj
 0001:0005f334       __get_dstbias              10060334 f   LIBCMT:timeset.obj
 0001:0005f36d       __get_timezone             1006036d f   LIBCMT:timeset.obj
 0001:0005f3a6       __get_tzname               100603a6 f   LIBCMT:timeset.obj
 0001:0005f44a       ___daylight                1006044a f   LIBCMT:timeset.obj
 0001:0005f450       ___dstbias                 10060450 f   LIBCMT:timeset.obj
 0001:0005f456       ___timezone                10060456 f   LIBCMT:timeset.obj
 0001:0005f45c       ___tzname                  1006045c f   LIBCMT:timeset.obj
 0001:0005f462       __set_daylight             10060462 f i LIBCMT:tzset.obj
 0001:0005f473       __set_dstbias              10060473 f i LIBCMT:tzset.obj
 0001:0005f484       __set_timezone             10060484 f i LIBCMT:tzset.obj
 0001:0005fbaa       ___tzset                   10060baa f   LIBCMT:tzset.obj
 0001:0005fbf9       __tzset                    10060bf9 f   LIBCMT:tzset.obj
 0001:0005fc31       __isindst                  10060c31 f   LIBCMT:tzset.obj
 0001:0005fc72       __strnicmp_l               10060c72 f   LIBCMT:strnicmp.obj
 0001:0005fd64       __strnicmp                 10060d64 f   LIBCMT:strnicmp.obj
 0001:0005fe9f       __itoa_s                   10060e9f f   LIBCMT:xtoas.obj
 0001:0005fec9       __ltoa_s                   10060ec9 f   LIBCMT:xtoas.obj
 0001:0005fef0       __ultoa_s                  10060ef0 f   LIBCMT:xtoas.obj
 0001:00060002       __i64toa_s                 10061002 f   LIBCMT:xtoas.obj
 0001:00060037       __ui64toa_s                10061037 f   LIBCMT:xtoas.obj
 0001:00060056       __purecall                 10061056 f   LIBCMT:purevirt.obj
 0001:00060080       __set_purecall_handler     10061080 f   LIBCMT:purevirt.obj
 0001:000600a7       __get_purecall_handler     100610a7 f   LIBCMT:purevirt.obj
 0001:000600b4       __chsize_nolock            100610b4 f   LIBCMT:chsize.obj
 0001:0006026a       __chsize_s                 1006126a f   LIBCMT:chsize.obj
 0001:00060357       __chsize                   10061357 f   LIBCMT:chsize.obj
 0001:00060373       __setmode_nolock           10061373 f   LIBCMT:setmode.obj
 0001:0006042f       __set_fmode                1006142f f   LIBCMT:setmode.obj
 0001:0006047b       __get_fmode                1006147b f   LIBCMT:setmode.obj
 0001:000604b4       __setmode                  100614b4 f   LIBCMT:setmode.obj
 0001:000605ab       ___initconin               100615ab f   LIBCMT:initcon.obj
 0001:000605ca       ___initconout              100615ca f   LIBCMT:initcon.obj
 0001:000605e9       ___termcon                 100615e9 f   LIBCMT:initcon.obj
 0001:00060616       _wcslen                    10061616 f   LIBCMT:wcslen.obj
 0001:00060653       ___crtGetStringTypeW       10061653 f   LIBCMT:w_str.obj
 0001:00060691       __getenv_helper_nolock     10061691 f   LIBCMT:getenv.obj
 0001:00060851       _getenv                    10061851 f   LIBCMT:getenv.obj
 0001:000608d4       _getenv_s                  100618d4 f   LIBCMT:getenv.obj
 0001:000609ac       __dupenv_s                 100619ac f   LIBCMT:getenv.obj
 0001:00060aa0       ___ascii_strnicmp          10061aa0 f   LIBCMT:_strnicm.obj
 0001:00060b01       __mbsnbicoll_l             10061b01 f   LIBCMT:mbsnbico.obj
 0001:00060bef       __mbsnbicoll               10061bef f   LIBCMT:mbsnbico.obj
 0001:00060c09       ___wtomb_environ           10061c09 f   LIBCMT:wtombenv.obj
 0001:00060ca0       _strnlen                   10061ca0 f   LIBCMT:strlen_s.obj
 0001:0006104b       ___crtCompareStringA       1006204b f   LIBCMT:a_cmp.obj
 0001:0006108d       __strnicoll_l              1006208d f   LIBCMT:strnicol.obj
 0001:00061187       __strnicoll                10062187 f   LIBCMT:strnicol.obj
 0001:0006125c       ___crtsetenv               1006225c f   LIBCMT:setenv.obj
 0001:000614a7       __strdup                   100624a7 f   LIBCMT:strdup.obj
 0001:000614fc       __mbschr_l                 100624fc f   LIBCMT:mbschr.obj
 0001:000615b8       __mbschr                   100625b8 f   LIBCMT:mbschr.obj
 0001:0006c3db       _aliases_lookup            1006d3db f   iconv:iconv.obj
 0001:0006c51a       _aliases2_lookup           1006d51a f   iconv:iconv.obj
 0001:0006c54a       _libiconv_open             1006d54a f   iconv:iconv.obj
 0001:0006d1ba       _libiconv                  1006e1ba f   iconv:iconv.obj
 0001:0006d1f0       _libiconv_close            1006e1f0 f   iconv:iconv.obj
 0001:0006d1fd       _libiconvctl               1006e1fd f   iconv:iconv.obj
 0001:0006d2e0       _libiconvlist              1006e2e0 f   iconv:iconv.obj
 0001:0006d440       _locale_charset            1006e440 f   iconv:localcharset.obj
 0001:0006d4e0       __tcsstr                   1006e4e0 f i wzFilePacker_static:wzFilePacker.obj
 0001:0006d4f0       ?_tcsstr@@YAPADPADPBD@Z    1006e4f0 f i wzFilePacker_static:wzFilePacker.obj
 0001:0006d500       ??0CAutoFree@@QAE@XZ       1006e500 f i wzFilePacker_static:wzFilePacker.obj
 0001:0006d510       ??1CAutoFree@@QAE@XZ       1006e510 f   wzFilePacker_static:wzFilePacker.obj
 0001:0006d520       ?CONVERT_PATHCHAR@CPackFile@@CAXPAD@Z 1006e520 f i wzFilePacker_static:wzFilePacker.obj
 0001:0006d580       ??0CPackFile@@QAE@XZ       1006e580 f   wzFilePacker_static:wzFilePacker.obj
 0001:0006d5b0       ?Close@CPackFile@@QAEXXZ   1006e5b0 f   wzFilePacker_static:wzFilePacker.obj
 0001:0006d5d0       ?CreateFinder@CPackFile@@AAEPAXPAXPBD@Z 1006e5d0 f   wzFilePacker_static:wzFilePacker.obj
 0001:0006d5e0       ?DestroyFinder@CPackFile@@AAEXPAX@Z 1006e5e0 f   wzFilePacker_static:wzFilePacker.obj
 0001:0006d5f0       ?FinderGetNextFile@CPackFile@@AAEHPAX@Z 1006e5f0 f   wzFilePacker_static:wzFilePacker.obj
 0001:0006d600       ?FinderGetProperties@CPackFile@@AAEHPAXPAUFileProperties@@@Z 1006e600 f   wzFilePacker_static:wzFilePacker.obj
 0001:0006d6b0       ?CreateFileA@CPackFile@@QAEPAXPBD_K@Z 1006e6b0 f   wzFilePacker_static:wzFilePacker.obj
 0001:0006d6e0       ?OpenFile@CPackFile@@QAEPAXPBDK@Z 1006e6e0 f   wzFilePacker_static:wzFilePacker.obj
 0001:0006d710       ?DeleteFileA@CPackFile@@QAEHPBD@Z 1006e710 f   wzFilePacker_static:wzFilePacker.obj
 0001:0006d730       ?FileExists@CPackFile@@QAEHPBD@Z 1006e730 f   wzFilePacker_static:wzFilePacker.obj
 0001:0006d750       ?RenameFile@CPackFile@@QAEHPBD0@Z 1006e750 f   wzFilePacker_static:wzFilePacker.obj
 0001:0006d780       ?RemoveDirectoryA@CPackFile@@QAEHPBD@Z 1006e780 f   wzFilePacker_static:wzFilePacker.obj
 0001:0006d7a0       ?CreateDirectoryA@CPackFile@@QAEHPBD@Z 1006e7a0 f   wzFilePacker_static:wzFilePacker.obj
 0001:0006d7d0       ?CloseFile@CPackFile@@QAEXPAX@Z 1006e7d0 f   wzFilePacker_static:wzFilePacker.obj
 0001:0006d7e0       ?GetFileProperties@CPackFile@@QAEHPAXPAUFileProperties@@@Z 1006e7e0 f   wzFilePacker_static:wzFilePacker.obj
 0001:0006d890       ?ReadFile@CPackFile@@QAEHPAX0K@Z 1006e890 f   wzFilePacker_static:wzFilePacker.obj
 0001:0006d8b0       ?WriteFile@CPackFile@@QAEHPAXPBXK@Z 1006e8b0 f   wzFilePacker_static:wzFilePacker.obj
 0001:0006d8d0       ?GetFileSize@CPackFile@@QAEHPAXPA_K@Z 1006e8d0 f   wzFilePacker_static:wzFilePacker.obj
 0001:0006d8e0       ?GetFilePointer@CPackFile@@QAEHPAXPA_K@Z 1006e8e0 f   wzFilePacker_static:wzFilePacker.obj
 0001:0006d8f0       ?SetFilePointer@CPackFile@@QAEHPAX_KK@Z 1006e8f0 f   wzFilePacker_static:wzFilePacker.obj
 0001:0006d910       ?IsEOF@CPackFile@@QAEHPAX@Z 1006e910 f   wzFilePacker_static:wzFilePacker.obj
 0001:0006d920       ?AddFile@CPackFile@@QAEHPBD0@Z 1006e920 f   wzFilePacker_static:wzFilePacker.obj
 0001:0006da30       ?SetHwnd@CPackFile@@QAEXPAUHWND__@@@Z 1006ea30 f   wzFilePacker_static:wzFilePacker.obj
 0001:0006da40       ?GetFindFileNameInPackFile@CPackFile@@SAHPBDPAD@Z 1006ea40 f   wzFilePacker_static:wzFilePacker.obj
 0001:0006db80       ?ExtractFile@CPackFile@@QAEHPAXPBD1@Z 1006eb80 f   wzFilePacker_static:wzFilePacker.obj
 0001:0006dc70       ?EncryptHdr@CPackFile@@SAHPAD@Z 1006ec70 f   wzFilePacker_static:wzFilePacker.obj
 0001:0006dd50       ?WriteHeader@CPackFile@@QAEXPADHH@Z 1006ed50 f   wzFilePacker_static:wzFilePacker.obj
 0001:0006def0       ?length@?$basic_string@DU?$char_traits@D@std@@V?$allocator@D@2@@std@@QBEIXZ 1006eef0 f i wzFilePacker_static:wzFilePacker.obj
 0001:0006df00       ??D?$_Vector_const_iterator@V?$basic_string@DU?$char_traits@D@std@@V?$allocator@D@2@@std@@V?$allocator@V?$basic_string@DU?$char_traits@D@std@@V?$allocator@D@2@@std@@@2@@std@@QBEABV?$basic_string@DU?$char_traits@D@std@@V?$allocator@D@2@@1@XZ 1006ef00 f i wzFilePacker_static:wzFilePacker.obj
 0001:0006df30       ??E?$_Vector_const_iterator@V?$basic_string@DU?$char_traits@D@std@@V?$allocator@D@2@@std@@V?$allocator@V?$basic_string@DU?$char_traits@D@std@@V?$allocator@D@2@@std@@@2@@std@@QAEAAV01@XZ 1006ef30 f i wzFilePacker_static:wzFilePacker.obj
 0001:0006df60       ??1CPackFile@@QAE@XZ       1006ef60 f   wzFilePacker_static:wzFilePacker.obj
 0001:0006df70       ?Open@CPackFile@@QAEPAXPBD0K@Z 1006ef70 f   wzFilePacker_static:wzFilePacker.obj
 0001:0006e040       ??D?$_Vector_iterator@V?$basic_string@DU?$char_traits@D@std@@V?$allocator@D@2@@std@@V?$allocator@V?$basic_string@DU?$char_traits@D@std@@V?$allocator@D@2@@std@@@2@@std@@QBEAAV?$basic_string@DU?$char_traits@D@std@@V?$allocator@D@2@@1@XZ 1006f040 f i wzFilePacker_static:wzFilePacker.obj
 0001:0006e070       ?find_last_of@?$basic_string@DU?$char_traits@D@std@@V?$allocator@D@2@@std@@QBEIPBDII@Z 1006f070 f i wzFilePacker_static:wzFilePacker.obj
 0001:0006e110       ??E?$_Vector_iterator@V?$basic_string@DU?$char_traits@D@std@@V?$allocator@D@2@@std@@V?$allocator@V?$basic_string@DU?$char_traits@D@std@@V?$allocator@D@2@@std@@@2@@std@@QAEAAV01@XZ 1006f110 f i wzFilePacker_static:wzFilePacker.obj
 0001:0006e140       ?find_last_of@?$basic_string@DU?$char_traits@D@std@@V?$allocator@D@2@@std@@QBEIPBDI@Z 1006f140 f i wzFilePacker_static:wzFilePacker.obj
 0001:0006e170       ??E?$_Vector_iterator@V?$basic_string@DU?$char_traits@D@std@@V?$allocator@D@2@@std@@V?$allocator@V?$basic_string@DU?$char_traits@D@std@@V?$allocator@D@2@@std@@@2@@std@@QAE?AV01@H@Z 1006f170 f i wzFilePacker_static:wzFilePacker.obj
 0001:0006e1b0       ?FindFile@CPackFile@@QAEHPAXPBDAAV?$vector@V?$basic_string@DU?$char_traits@D@std@@V?$allocator@D@2@@std@@V?$allocator@V?$basic_string@DU?$char_traits@D@std@@V?$allocator@D@2@@std@@@2@@std@@2H@Z 1006f1b0 f   wzFilePacker_static:wzFilePacker.obj
 0001:0006e510       ?ExtractAll@CPackFile@@QAEHPAXPBD@Z 1006f510 f   wzFilePacker_static:wzFilePacker.obj
 0001:0006ed40       ?MurgeFile@CPackFile@@QAEHPAXH@Z 1006fd40 f   wzFilePacker_static:wzFilePacker.obj
 0001:0006f760       @geVFile_CloseAPI@0        10070760 f   wzFilePacker_static:vfile.obj
 0001:0006f7f0       @geVFile_RegisterFileSystem@8 100707f0 f   wzFilePacker_static:vfile.obj
 0001:0006f840       @geVFile_UpdateContext@12  10070840 f   wzFilePacker_static:vfile.obj
 0001:0006f860       @geVFile_Open_Detail@20    10070860 f   wzFilePacker_static:vfile.obj
 0001:0006f950       @geVFile_Open@12           10070950 f   wzFilePacker_static:vfile.obj
 0001:0006fa40       @geVFile_GetContext@4      10070a40 f   wzFilePacker_static:vfile.obj
 0001:0006fad0       @geVFile_AddPath@12        10070ad0 f   wzFilePacker_static:vfile.obj
 0001:0006fb40       @geVFile_DeleteFile@8      10070b40 f   wzFilePacker_static:vfile.obj
 0001:0006fb50       @geVFile_RenameFile@12     10070b50 f   wzFilePacker_static:vfile.obj
 0001:0006fb70       @geVFile_FileExists@8      10070b70 f   wzFilePacker_static:vfile.obj
 0001:0006fb80       @geVFile_Close@4           10070b80 f   wzFilePacker_static:vfile.obj
 0001:0006fbd0       @geVFile_GetS@12           10070bd0 f   wzFilePacker_static:vfile.obj
 0001:0006fbf0       @geVFile_Read@12           10070bf0 f   wzFilePacker_static:vfile.obj
 0001:0006fc20       @geVFile_Write@12          10070c20 f   wzFilePacker_static:vfile.obj
 0001:0006fc50       @geVFile_Seek@16           10070c50 f   wzFilePacker_static:vfile.obj
 0001:0006fc70       _geVFile_Printf            10070c70 f   wzFilePacker_static:vfile.obj
 0001:0006fcf0       @geVFile_EOF@4             10070cf0 f   wzFilePacker_static:vfile.obj
 0001:0006fd00       @geVFile_Tell@8            10070d00 f   wzFilePacker_static:vfile.obj
 0001:0006fd10       @geVFile_Size@8            10070d10 f   wzFilePacker_static:vfile.obj
 0001:0006fd20       @geVFile_GetProperties@8   10070d20 f   wzFilePacker_static:vfile.obj
 0001:0006fd30       @geVFile_SetSize@12        10070d30 f   wzFilePacker_static:vfile.obj
 0001:0006fd50       @geVFile_SetAttributes@8   10070d50 f   wzFilePacker_static:vfile.obj
 0001:0006fd60       @geVFile_SetTime@8         10070d60 f   wzFilePacker_static:vfile.obj
 0001:0006fd70       @geVFile_SetHints@8        10070d70 f   wzFilePacker_static:vfile.obj
 0001:0006fd80       @geVFile_EnlargeDirectorySize@8 10070d80 f   wzFilePacker_static:vfile.obj
 0001:0006fd90       @geVFile_CreateFinder@8    10070d90 f   wzFilePacker_static:vfile.obj
 0001:0006fde0       @geVFile_DestroyFinder@4   10070de0 f   wzFilePacker_static:vfile.obj
 0001:0006fe10       @geVFile_FinderGetNextFile@4 10070e10 f   wzFilePacker_static:vfile.obj
 0001:0006fe20       @geVFile_FinderGetProperties@8 10070e20 f   wzFilePacker_static:vfile.obj
 0001:0006fe30       @geVFile_TimeToWin32FileTime@8 10070e30 f   wzFilePacker_static:vfile.obj
 0001:0006fe40       @geVFile_SetVersion@8      10070e40 f   wzFilePacker_static:vfile.obj
 0001:0006fe50       @geVFile_IsPrevVersion@4   10070e50 f   wzFilePacker_static:vfile.obj
 0001:0006fe60       @geVFile_OpenNewSystem@20  10070e60 f   wzFilePacker_static:vfile.obj
 0001:0006ffa0       @geVFile_UpdateSystem@4    10070fa0 f   wzFilePacker_static:vfile.obj
 0001:000700e0       _EmptyDirectory            100710e0 f   wzFilePacker_static:vFile_util.obj
 0001:000702a0       _SetupDirectory            100712a0 f   wzFilePacker_static:vFile_util.obj
 0001:000702c0       _ExplorerVFS               100712c0 f   wzFilePacker_static:vFile_util.obj
 0001:000704b0       _CopyVFile                 100714b0 f   wzFilePacker_static:vFile_util.obj
 0001:00070620       _CopyOneFile               10071620 f   wzFilePacker_static:vFile_util.obj
 0001:000706a0       _GetFiles                  100716a0 f   wzFilePacker_static:vFile_util.obj
 0001:00070b70       _MakeDirectory             10071b70 f   wzFilePacker_static:vFile_util.obj
 0001:00070c40       _ExtractVFS                10071c40 f   wzFilePacker_static:vFile_util.obj
 0001:00070ea0       _GetDir                    10071ea0 f   wzFilePacker_static:vFile_util.obj
 0001:00071200       _geRam_EnableCriticalCallback 10072200 f   wzFilePacker_static:Ram.obj
 0001:00071210       _geRam_SetCriticalCallback 10072210 f   wzFilePacker_static:Ram.obj
 0001:00071240       _geRam_Allocate            10072240 f   wzFilePacker_static:Ram.obj
 0001:00071260       _geRam_Free_               10072260 f   wzFilePacker_static:Ram.obj
 0001:00071270       _geRam_Realloc             10072270 f   wzFilePacker_static:Ram.obj
 0001:000712d0       _geRam_AllocateClear       100722d0 f   wzFilePacker_static:Ram.obj
 0001:00071300       _Encrypt                   10072300 f   wzFilePacker_static:fsvfs.obj
 0001:00071340       _Decrypt                   10072340 f   wzFilePacker_static:fsvfs.obj
 0001:00072d50       @FSVFS_GetAPIs@0           10073d50 f   wzFilePacker_static:fsvfs.obj
 0001:000735c0       @FSMemory_GetAPIs@0        100745c0 f   wzFilePacker_static:FSMEMORY.obj
 0001:00074280       @FSDos_GetAPIs@0           10075280 f   wzFilePacker_static:fsdos.obj
 0001:00074290       _DirTree_Create            10075290 f   wzFilePacker_static:dirtree.obj
 0001:000742e0       _DirTree_Destroy           100752e0 f   wzFilePacker_static:dirtree.obj
 0001:00074580       _DirTree_SetFileSize       10075580 f   wzFilePacker_static:dirtree.obj
 0001:000745a0       _DirTree_GetFileSize       100755a0 f   wzFilePacker_static:dirtree.obj
 0001:000745c0       _DirTree_WriteToFile       100755c0 f   wzFilePacker_static:dirtree.obj
 0001:000745f0       _DirTree_GetSize           100755f0 f   wzFilePacker_static:dirtree.obj
 0001:00074a10       _DirTree_CreateFromFile    10075a10 f   wzFilePacker_static:dirtree.obj
 0001:00074d90       _DirTree_FindExact         10075d90 f   wzFilePacker_static:dirtree.obj
 0001:00074df0       _DirTree_FindPartial       10075df0 f   wzFilePacker_static:dirtree.obj
 0001:00074e70       _DirTree_AddFile           10075e70 f   wzFilePacker_static:dirtree.obj
 0001:00074f40       _DirTree_Remove            10075f40 f   wzFilePacker_static:dirtree.obj
 0001:00074fd0       _DirTree_SetFileAttributes 10075fd0 f   wzFilePacker_static:dirtree.obj
 0001:00074ff0       _DirTree_GetFileAttributes 10075ff0 f   wzFilePacker_static:dirtree.obj
 0001:00075000       _DirTree_SetFileOffset     10076000 f   wzFilePacker_static:dirtree.obj
 0001:00075020       _DirTree_GetFileOffset     10076020 f   wzFilePacker_static:dirtree.obj
 0001:00075040       _DirTree_SetFileTime       10076040 f   wzFilePacker_static:dirtree.obj
 0001:00075060       _DirTree_GetFileTime       10076060 f   wzFilePacker_static:dirtree.obj
 0001:00075080       _DirTree_SetFileHints      10076080 f   wzFilePacker_static:dirtree.obj
 0001:000750f0       _DirTree_GetFileHints      100760f0 f   wzFilePacker_static:dirtree.obj
 0001:00075110       _DirTree_GetName           10076110 f   wzFilePacker_static:dirtree.obj
 0001:00075150       _DirTree_FileExists        10076150 f   wzFilePacker_static:dirtree.obj
 0001:00075170       _DirTree_CreateFinder      10076170 f   wzFilePacker_static:dirtree.obj
 0001:000752a0       _DirTree_DestroyFinder     100762a0 f   wzFilePacker_static:dirtree.obj
 0001:000752e0       _DirTree_FinderGetNextFile 100762e0 f   wzFilePacker_static:dirtree.obj
 0001:000753a0       _DirTree_SetAllFileOffset  100763a0 f   wzFilePacker_static:dirtree.obj
 0001:00075450       _DuplicateString           10076450 f   wzFilePacker_static:dirtree-common.obj
 0001:00075490       _GetNextDir                10076490 f   wzFilePacker_static:dirtree-common.obj
 0001:000754c0       _MatchPattern              100764c0 f   wzFilePacker_static:dirtree-common.obj
 0001:00075520       _PathHasDir                10076520 f   wzFilePacker_static:dirtree-common.obj
 0001:00075536       _timeKillEvent@4           10076536 f   winmm:WINMM.dll
 0001:0007553c       _mmioClose@8               1007653c f   winmm:WINMM.dll
 0001:00075542       _mmioSeek@12               10076542 f   winmm:WINMM.dll
 0001:00075548       _mmioRead@12               10076548 f   winmm:WINMM.dll
 0001:0007554e       _timeSetEvent@20           1007654e f   winmm:WINMM.dll
 0001:00075554       _timeEndPeriod@4           10076554 f   winmm:WINMM.dll
 0001:0007555a       _timeGetTime@0             1007655a f   winmm:WINMM.dll
 0001:00075560       _timeBeginPeriod@4         10076560 f   winmm:WINMM.dll
 0001:00075566       _mixerClose@4              10076566 f   winmm:WINMM.dll
 0001:0007556c       _mixerGetLineInfoA@12      1007656c f   winmm:WINMM.dll
 0001:00075572       _mixerGetDevCapsA@12       10076572 f   winmm:WINMM.dll
 0001:00075578       _mixerOpen@20              10076578 f   winmm:WINMM.dll
 0001:0007557e       _mixerGetNumDevs@0         1007657e f   winmm:WINMM.dll
 0001:00075584       _mixerGetLineControlsA@12  10076584 f   winmm:WINMM.dll
 0001:0007558a       _mixerGetControlDetailsA@12 1007658a f   winmm:WINMM.dll
 0001:00075590       _mixerSetControlDetails@12 10076590 f   winmm:WINMM.dll
 0001:00075596       _MakeSureDirectoryPathExists@4 10076596 f   Dbghelp:dbghelp.dll
 0001:0007559c       _HeapFree@12               1007659c f   kernel32:KERNEL32.dll
 0001:000755a2       _HeapAlloc@12              100765a2 f   kernel32:KERNEL32.dll
 0001:000755a8       _TerminateProcess@8        100765a8 f   kernel32:KERNEL32.dll
 0001:000755ae       _GetCurrentProcess@0       100765ae f   kernel32:KERNEL32.dll
 0001:000755b4       _UnhandledExceptionFilter@4 100765b4 f   kernel32:KERNEL32.dll
 0001:000755ba       _SetUnhandledExceptionFilter@4 100765ba f   kernel32:KERNEL32.dll
 0001:000755c0       _IsDebuggerPresent@0       100765c0 f   kernel32:KERNEL32.dll
 0001:000755c6       _RaiseException@16         100765c6 f   kernel32:KERNEL32.dll
 0001:000755cc       _RtlUnwind@16              100765cc f   kernel32:KERNEL32.dll
 0001:000755d2       _HeapReAlloc@16            100765d2 f   kernel32:KERNEL32.dll
 0001:000755d8       _GetCurrentThreadId@0      100765d8 f   kernel32:KERNEL32.dll
 0001:000755de       _GetCommandLineA@0         100765de f   kernel32:KERNEL32.dll
 0001:000755e4       _GetModuleHandleW@4        100765e4 f   kernel32:KERNEL32.dll
 0001:000755ea       _ExitProcess@4             100765ea f   kernel32:KERNEL32.dll
 0001:000755f0       _GetModuleHandleA@4        100765f0 f   kernel32:KERNEL32.dll
 0001:000755f6       _HeapCreate@12             100765f6 f   kernel32:KERNEL32.dll
 0001:000755fc       _HeapDestroy@4             100765fc f   kernel32:KERNEL32.dll
 0001:00075602       _VirtualFree@12            10076602 f   kernel32:KERNEL32.dll
 0001:00075608       _FatalAppExitA@8           10076608 f   kernel32:KERNEL32.dll
 0001:0007560e       _VirtualAlloc@16           1007660e f   kernel32:KERNEL32.dll
 0001:00075614       _GetCPInfo@8               10076614 f   kernel32:KERNEL32.dll
 0001:0007561a       _InterlockedIncrement@4    1007661a f   kernel32:KERNEL32.dll
 0001:00075620       _InterlockedDecrement@4    10076620 f   kernel32:KERNEL32.dll
 0001:00075626       _GetACP@0                  10076626 f   kernel32:KERNEL32.dll
 0001:0007562c       _GetOEMCP@0                1007662c f   kernel32:KERNEL32.dll
 0001:00075632       _IsValidCodePage@4         10076632 f   kernel32:KERNEL32.dll
 0001:00075638       _TlsGetValue@4             10076638 f   kernel32:KERNEL32.dll
 0001:0007563e       _TlsAlloc@0                1007663e f   kernel32:KERNEL32.dll
 0001:00075644       _TlsSetValue@8             10076644 f   kernel32:KERNEL32.dll
 0001:0007564a       _TlsFree@4                 1007664a f   kernel32:KERNEL32.dll
 0001:00075650       _SetLastError@4            10076650 f   kernel32:KERNEL32.dll
 0001:00075656       _GetCurrentThread@0        10076656 f   kernel32:KERNEL32.dll
 0001:0007565c       _WriteFile@20              1007665c f   kernel32:KERNEL32.dll
 0001:00075662       _GetStdHandle@4            10076662 f   kernel32:KERNEL32.dll
 0001:00075668       _HeapSize@12               10076668 f   kernel32:KERNEL32.dll
 0001:0007566e       _SetFilePointer@16         1007666e f   kernel32:KERNEL32.dll
 0001:00075674       _MultiByteToWideChar@24    10076674 f   kernel32:KERNEL32.dll
 0001:0007567a       _ReadFile@20               1007667a f   kernel32:KERNEL32.dll
 0001:00075680       _CloseHandle@4             10076680 f   kernel32:KERNEL32.dll
 0001:00075686       _WideCharToMultiByte@32    10076686 f   kernel32:KERNEL32.dll
 0001:0007568c       _GetConsoleCP@0            1007668c f   kernel32:KERNEL32.dll
 0001:00075692       _GetConsoleMode@8          10076692 f   kernel32:KERNEL32.dll
 0001:00075698       _SetHandleCount@4          10076698 f   kernel32:KERNEL32.dll
 0001:0007569e       _GetFileType@4             1007669e f   kernel32:KERNEL32.dll
 0001:000756a4       _GetStartupInfoA@4         100766a4 f   kernel32:KERNEL32.dll
 0001:000756aa       _FreeEnvironmentStringsA@4 100766aa f   kernel32:KERNEL32.dll
 0001:000756b0       _GetEnvironmentStrings@0   100766b0 f   kernel32:KERNEL32.dll
 0001:000756b6       _FreeEnvironmentStringsW@4 100766b6 f   kernel32:KERNEL32.dll
 0001:000756bc       _GetEnvironmentStringsW@0  100766bc f   kernel32:KERNEL32.dll
 0001:000756c2       _QueryPerformanceCounter@4 100766c2 f   kernel32:KERNEL32.dll
 0001:000756c8       _GetTickCount@0            100766c8 f   kernel32:KERNEL32.dll
 0001:000756ce       _GetCurrentProcessId@0     100766ce f   kernel32:KERNEL32.dll
 0001:000756d4       _GetSystemTimeAsFileTime@4 100766d4 f   kernel32:KERNEL32.dll
 0001:000756da       _LCMapStringA@24           100766da f   kernel32:KERNEL32.dll
 0001:000756e0       _LCMapStringW@24           100766e0 f   kernel32:KERNEL32.dll
 0001:000756e6       _SetStdHandle@8            100766e6 f   kernel32:KERNEL32.dll
 0001:000756ec       _SetConsoleCtrlHandler@8   100766ec f   kernel32:KERNEL32.dll
 0001:000756f2       _InitializeCriticalSectionAndSpinCount@8 100766f2 f   kernel32:KERNEL32.dll
 0001:000756f8       _GetStringTypeA@20         100766f8 f   kernel32:KERNEL32.dll
 0001:000756fe       _GetStringTypeW@16         100766fe f   kernel32:KERNEL32.dll
 0001:00075704       _GetTimeFormatA@24         10076704 f   kernel32:KERNEL32.dll
 0001:0007570a       _GetDateFormatA@24         1007670a f   kernel32:KERNEL32.dll
 0001:00075710       _GetUserDefaultLCID@0      10076710 f   kernel32:KERNEL32.dll
 0001:00075716       _GetLocaleInfoA@16         10076716 f   kernel32:KERNEL32.dll
 0001:0007571c       _EnumSystemLocalesA@8      1007671c f   kernel32:KERNEL32.dll
 0001:00075722       _IsValidLocale@8           10076722 f   kernel32:KERNEL32.dll
 0001:00075728       _FlushFileBuffers@4        10076728 f   kernel32:KERNEL32.dll
 0001:0007572e       _CreateFileA@28            1007672e f   kernel32:KERNEL32.dll
 0001:00075734       _WriteConsoleA@20          10076734 f   kernel32:KERNEL32.dll
 0001:0007573a       _GetConsoleOutputCP@0      1007673a f   kernel32:KERNEL32.dll
 0001:00075740       _WriteConsoleW@20          10076740 f   kernel32:KERNEL32.dll
 0001:00075746       _GetLocaleInfoW@16         10076746 f   kernel32:KERNEL32.dll
 0001:0007574c       _GetTimeZoneInformation@4  1007674c f   kernel32:KERNEL32.dll
 0001:00075752       _SetEndOfFile@4            10076752 f   kernel32:KERNEL32.dll
 0001:00075758       _GetProcessHeap@0          10076758 f   kernel32:KERNEL32.dll
 0001:0007575e       _CompareStringA@24         1007675e f   kernel32:KERNEL32.dll
 0001:00075764       _CompareStringW@24         10076764 f   kernel32:KERNEL32.dll
 0001:0007576a       _SetEnvironmentVariableA@8 1007676a f   kernel32:KERNEL32.dll
 0001:00075770       _lstrlenA@4                10076770 f   kernel32:KERNEL32.dll
 0001:00075776       _lstrcpyA@8                10076776 f   kernel32:KERNEL32.dll
 0001:0007577c       _FindNextFileA@8           1007677c f   kernel32:KERNEL32.dll
 0001:00075782       _FindFirstFileA@8          10076782 f   kernel32:KERNEL32.dll
 0001:00075788       _FindClose@4               10076788 f   kernel32:KERNEL32.dll
 0001:0007578e       _RemoveDirectoryA@4        1007678e f   kernel32:KERNEL32.dll
 0001:00075794       _GetSystemDirectoryA@8     10076794 f   kernel32:KERNEL32.dll
 0001:0007579a       _CreateDirectoryA@8        1007679a f   kernel32:KERNEL32.dll
 0001:000757a0       _SetFilePointerEx@20       100767a0 f   kernel32:KERNEL32.dll
 0001:000757a6       _GetFileSizeEx@8           100767a6 f   kernel32:KERNEL32.dll
 0001:000757ac       _GetFileInformationByHandle@8 100767ac f   kernel32:KERNEL32.dll
 0001:000757b2       _SetFileAttributesA@8      100767b2 f   kernel32:KERNEL32.dll
 0001:000757b8       _SetFileTime@16            100767b8 f   kernel32:KERNEL32.dll
 0001:000757be       _DeleteFileA@4             100767be f   kernel32:KERNEL32.dll
 0001:000757c4       _MoveFileA@8               100767c4 f   kernel32:KERNEL32.dll
 0001:000757ca       _SendMessageA@16           100767ca f   user32:USER32.dll
 0001:000757d0       _wsprintfA                 100767d0 f   user32:USER32.dll
 0001:000757e0       _ogg_page_version          100767e0 f   ogg_static:framing.obj
 0001:000757f0       _ogg_page_continued        100767f0 f   ogg_static:framing.obj
 0001:00075800       _ogg_page_bos              10076800 f   ogg_static:framing.obj
 0001:00075810       _ogg_page_eos              10076810 f   ogg_static:framing.obj
 0001:00075820       _ogg_page_granulepos       10076820 f   ogg_static:framing.obj
 0001:00075900       _ogg_page_serialno         10076900 f   ogg_static:framing.obj
 0001:00075930       _ogg_page_pageno           10076930 f   ogg_static:framing.obj
 0001:00075960       _ogg_page_packets          10076960 f   ogg_static:framing.obj
 0001:00075990       _ogg_stream_init           10076990 f   ogg_static:framing.obj
 0001:00075a00       _ogg_stream_clear          10076a00 f   ogg_static:framing.obj
 0001:00075a50       _ogg_stream_destroy        10076a50 f   ogg_static:framing.obj
 0001:00075a70       _ogg_page_checksum_set     10076a70 f   ogg_static:framing.obj
 0001:00075b20       _ogg_stream_packetin       10076b20 f   ogg_static:framing.obj
 0001:00075d00       _ogg_stream_flush          10076d00 f   ogg_static:framing.obj
 0001:00075f00       _ogg_stream_pageout        10076f00 f   ogg_static:framing.obj
 0001:00075f50       _ogg_stream_eos            10076f50 f   ogg_static:framing.obj
 0001:00075f60       _ogg_sync_init             10076f60 f   ogg_static:framing.obj
 0001:00075f80       _ogg_sync_clear            10076f80 f   ogg_static:framing.obj
 0001:00075fb0       _ogg_sync_destroy          10076fb0 f   ogg_static:framing.obj
 0001:00075fd0       _ogg_sync_buffer           10076fd0 f   ogg_static:framing.obj
 0001:00076050       _ogg_sync_wrote            10077050 f   ogg_static:framing.obj
 0001:00076070       _ogg_sync_pageseek         10077070 f   ogg_static:framing.obj
 0001:000761c0       _ogg_sync_pageout          100771c0 f   ogg_static:framing.obj
 0001:00076200       _ogg_stream_pagein         10077200 f   ogg_static:framing.obj
 0001:000764f0       _ogg_sync_reset            100774f0 f   ogg_static:framing.obj
 0001:00076510       _ogg_stream_reset          10077510 f   ogg_static:framing.obj
 0001:00076560       _ogg_stream_reset_serialno 10077560 f   ogg_static:framing.obj
 0001:00076580       _ogg_stream_packetout      10077580 f   ogg_static:framing.obj
 0001:000766d0       _ogg_stream_packetpeek     100776d0 f   ogg_static:framing.obj
 0001:000766f0       _ogg_packet_clear          100776f0 f   ogg_static:framing.obj
 0001:00076710       _oggpack_writeinit         10077710 f   ogg_static:bitwise.obj
 0001:00076750       _oggpackB_writeinit        10077750 f   ogg_static:bitwise.obj
 0001:00076760       _oggpack_writetrunc        10077760 f   ogg_static:bitwise.obj
 0001:000767a0       _oggpackB_writetrunc       100777a0 f   ogg_static:bitwise.obj
 0001:000767e0       _oggpack_write             100777e0 f   ogg_static:bitwise.obj
 0001:000768e0       _oggpackB_write            100778e0 f   ogg_static:bitwise.obj
 0001:000769d0       _oggpack_writealign        100779d0 f   ogg_static:bitwise.obj
 0001:000769f0       _oggpackB_writealign       100779f0 f   ogg_static:bitwise.obj
 0001:00076a10       _oggpack_writecopy         10077a10 f   ogg_static:bitwise.obj
 0001:00076b10       _oggpackB_writecopy        10077b10 f   ogg_static:bitwise.obj
 0001:00076b30       _oggpack_reset             10077b30 f   ogg_static:bitwise.obj
 0001:00076b50       _oggpackB_reset            10077b50 f   ogg_static:bitwise.obj
 0001:00076b60       _oggpack_writeclear        10077b60 f   ogg_static:bitwise.obj
 0001:00076b90       _oggpackB_writeclear       10077b90 f   ogg_static:bitwise.obj
 0001:00076ba0       _oggpack_readinit          10077ba0 f   ogg_static:bitwise.obj
 0001:00076bd0       _oggpackB_readinit         10077bd0 f   ogg_static:bitwise.obj
 0001:00076bf0       _oggpack_look              10077bf0 f   ogg_static:bitwise.obj
 0001:00076ca0       _oggpackB_look             10077ca0 f   ogg_static:bitwise.obj
 0001:00076d50       _oggpack_look1             10077d50 f   ogg_static:bitwise.obj
 0001:00076d80       _oggpackB_look1            10077d80 f   ogg_static:bitwise.obj
 0001:00076db0       _oggpack_adv               10077db0 f   ogg_static:bitwise.obj
 0001:00076de0       _oggpackB_adv              10077de0 f   ogg_static:bitwise.obj
 0001:00076e00       _oggpack_adv1              10077e00 f   ogg_static:bitwise.obj
 0001:00076e30       _oggpackB_adv1             10077e30 f   ogg_static:bitwise.obj
 0001:00076e40       _oggpack_read              10077e40 f   ogg_static:bitwise.obj
 0001:00076f10       _oggpackB_read             10077f10 f   ogg_static:bitwise.obj
 0001:00076fe0       _oggpack_read1             10077fe0 f   ogg_static:bitwise.obj
 0001:00077030       _oggpackB_read1            10078030 f   ogg_static:bitwise.obj
 0001:00077080       _oggpack_bytes             10078080 f   ogg_static:bitwise.obj
 0001:000770a0       _oggpack_bits              100780a0 f   ogg_static:bitwise.obj
 0001:000770b0       _oggpackB_bytes            100780b0 f   ogg_static:bitwise.obj
 0001:000770c0       _oggpackB_bits             100780c0 f   ogg_static:bitwise.obj
 0001:000770d0       _oggpack_get_buffer        100780d0 f   ogg_static:bitwise.obj
 0001:000770e0       _oggpackB_get_buffer       100780e0 f   ogg_static:bitwise.obj
 0001:000770f0       _filelength                100780f0 f   LIBCMT:flength.obj
 0001:000770f0       __filelength               100780f0 f   LIBCMT:flength.obj
 0001:000771ef       __mbsstr_l                 100781ef f   LIBCMT:mbsstr.obj
 0001:00077330       __mbsstr                   10078330 f   LIBCMT:mbsstr.obj
 0001:00077347       _remove                    10078347 f   LIBCMT:unlink.obj
 0001:00077377       __unlink                   10078377 f   LIBCMT:unlink.obj
 0001:00077382       __findclose                10078382 f   LIBCMT:findfile.obj
 0001:000773a8       ___timet_from_ft           100783a8 f   LIBCMT:findfile.obj
 0001:0007740e       __findfirst32              1007840e f   LIBCMT:findfile.obj
 0001:00077535       __findnext32               10078535 f   LIBCMT:findfile.obj
 0001:0007765b       ___time64_t_from_ft        1007865b f   LIBCMT:findfi32.obj
 0001:000776c3       __findfirst64i32           100786c3 f   LIBCMT:findfi32.obj
 0001:000777f3       __findnext64i32            100787f3 f   LIBCMT:findfi32.obj
 0001:00077930       __allshl                   10078930 f   LIBCMT:llshl.obj
 0001:0007794f       ___loctotime32_t           1007894f f   LIBCMT:dtoxtime.obj
 0001:00077b55       ___loctotime64_t           10078b55 f   LIBCMT:dtoxtm64.obj
 0001:00077dc0       _FileTimeToSystemTime@8    10078dc0 f   kernel32:KERNEL32.dll
 0001:00077dc6       _FileTimeToLocalFileTime@8 10078dc6 f   kernel32:KERNEL32.dll
 0002:00000000       __imp__InitializeCriticalSection@4 1007a000     kernel32:KERNEL32.dll
 0002:00000004       __imp__DeleteCriticalSection@4 1007a004     kernel32:KERNEL32.dll
 0002:00000008       __imp__LeaveCriticalSection@4 1007a008     kernel32:KERNEL32.dll
 0002:0000000c       __imp__EnterCriticalSection@4 1007a00c     kernel32:KERNEL32.dll
 0002:00000010       __imp__GetCurrentDirectoryA@8 1007a010     kernel32:KERNEL32.dll
 0002:00000014       __imp__InterlockedExchange@8 1007a014     kernel32:KERNEL32.dll
 0002:00000018       __imp__GetProcAddress@8    1007a018     kernel32:KERNEL32.dll
 0002:0000001c       __imp__LoadLibraryA@4      1007a01c     kernel32:KERNEL32.dll
 0002:00000020       __imp__FreeLibrary@4       1007a020     kernel32:KERNEL32.dll
 0002:00000024       __imp__Sleep@4             1007a024     kernel32:KERNEL32.dll
 0002:00000028       __imp__GetLastError@0      1007a028     kernel32:KERNEL32.dll
 0002:0000002c       __imp__LocalFree@4         1007a02c     kernel32:KERNEL32.dll
 0002:00000030       __imp__LocalAlloc@8        1007a030     kernel32:KERNEL32.dll
 0002:00000034       __imp__OutputDebugStringA@4 1007a034     kernel32:KERNEL32.dll
 0002:00000038       __imp__GetFileAttributesA@4 1007a038     kernel32:KERNEL32.dll
 0002:0000003c       __imp__GetModuleFileNameA@12 1007a03c     kernel32:KERNEL32.dll
 0002:00000040       __imp__GetDriveTypeA@4     1007a040     kernel32:KERNEL32.dll
 0002:00000044       __imp__MulDiv@12           1007a044     kernel32:KERNEL32.dll
 0002:00000048       __imp__FileTimeToSystemTime@8 1007a048     kernel32:KERNEL32.dll
 0002:0000004c       __imp__MoveFileA@8         1007a04c     kernel32:KERNEL32.dll
 0002:00000050       __imp__DeleteFileA@4       1007a050     kernel32:KERNEL32.dll
 0002:00000054       __imp__SetFileTime@16      1007a054     kernel32:KERNEL32.dll
 0002:00000058       __imp__SetFileAttributesA@8 1007a058     kernel32:KERNEL32.dll
 0002:0000005c       __imp__GetFileInformationByHandle@8 1007a05c     kernel32:KERNEL32.dll
 0002:00000060       __imp__GetFileSizeEx@8     1007a060     kernel32:KERNEL32.dll
 0002:00000064       __imp__SetFilePointerEx@20 1007a064     kernel32:KERNEL32.dll
 0002:00000068       __imp__CreateDirectoryA@8  1007a068     kernel32:KERNEL32.dll
 0002:0000006c       __imp__GetSystemDirectoryA@8 1007a06c     kernel32:KERNEL32.dll
 0002:00000070       __imp__RemoveDirectoryA@4  1007a070     kernel32:KERNEL32.dll
 0002:00000074       __imp__FindClose@4         1007a074     kernel32:KERNEL32.dll
 0002:00000078       __imp__FindFirstFileA@8    1007a078     kernel32:KERNEL32.dll
 0002:0000007c       __imp__FindNextFileA@8     1007a07c     kernel32:KERNEL32.dll
 0002:00000080       __imp__lstrcpyA@8          1007a080     kernel32:KERNEL32.dll
 0002:00000084       __imp__lstrlenA@4          1007a084     kernel32:KERNEL32.dll
 0002:00000088       __imp__SetEnvironmentVariableA@8 1007a088     kernel32:KERNEL32.dll
 0002:0000008c       __imp__CompareStringW@24   1007a08c     kernel32:KERNEL32.dll
 0002:00000090       __imp__CompareStringA@24   1007a090     kernel32:KERNEL32.dll
 0002:00000094       __imp__GetProcessHeap@0    1007a094     kernel32:KERNEL32.dll
 0002:00000098       __imp__SetEndOfFile@4      1007a098     kernel32:KERNEL32.dll
 0002:0000009c       __imp__GetTimeZoneInformation@4 1007a09c     kernel32:KERNEL32.dll
 0002:000000a0       __imp__GetLocaleInfoW@16   1007a0a0     kernel32:KERNEL32.dll
 0002:000000a4       __imp__WriteConsoleW@20    1007a0a4     kernel32:KERNEL32.dll
 0002:000000a8       __imp__HeapFree@12         1007a0a8     kernel32:KERNEL32.dll
 0002:000000ac       __imp__HeapAlloc@12        1007a0ac     kernel32:KERNEL32.dll
 0002:000000b0       __imp__TerminateProcess@8  1007a0b0     kernel32:KERNEL32.dll
 0002:000000b4       __imp__GetCurrentProcess@0 1007a0b4     kernel32:KERNEL32.dll
 0002:000000b8       __imp__UnhandledExceptionFilter@4 1007a0b8     kernel32:KERNEL32.dll
 0002:000000bc       __imp__SetUnhandledExceptionFilter@4 1007a0bc     kernel32:KERNEL32.dll
 0002:000000c0       __imp__IsDebuggerPresent@0 1007a0c0     kernel32:KERNEL32.dll
 0002:000000c4       __imp__RaiseException@16   1007a0c4     kernel32:KERNEL32.dll
 0002:000000c8       __imp__RtlUnwind@16        1007a0c8     kernel32:KERNEL32.dll
 0002:000000cc       __imp__HeapReAlloc@16      1007a0cc     kernel32:KERNEL32.dll
 0002:000000d0       __imp__GetCurrentThreadId@0 1007a0d0     kernel32:KERNEL32.dll
 0002:000000d4       __imp__GetCommandLineA@0   1007a0d4     kernel32:KERNEL32.dll
 0002:000000d8       __imp__GetModuleHandleW@4  1007a0d8     kernel32:KERNEL32.dll
 0002:000000dc       __imp__ExitProcess@4       1007a0dc     kernel32:KERNEL32.dll
 0002:000000e0       __imp__GetModuleHandleA@4  1007a0e0     kernel32:KERNEL32.dll
 0002:000000e4       __imp__HeapCreate@12       1007a0e4     kernel32:KERNEL32.dll
 0002:000000e8       __imp__HeapDestroy@4       1007a0e8     kernel32:KERNEL32.dll
 0002:000000ec       __imp__VirtualFree@12      1007a0ec     kernel32:KERNEL32.dll
 0002:000000f0       __imp__FatalAppExitA@8     1007a0f0     kernel32:KERNEL32.dll
 0002:000000f4       __imp__VirtualAlloc@16     1007a0f4     kernel32:KERNEL32.dll
 0002:000000f8       __imp__GetCPInfo@8         1007a0f8     kernel32:KERNEL32.dll
 0002:000000fc       __imp__InterlockedIncrement@4 1007a0fc     kernel32:KERNEL32.dll
 0002:00000100       __imp__InterlockedDecrement@4 1007a100     kernel32:KERNEL32.dll
 0002:00000104       __imp__GetACP@0            1007a104     kernel32:KERNEL32.dll
 0002:00000108       __imp__GetOEMCP@0          1007a108     kernel32:KERNEL32.dll
 0002:0000010c       __imp__IsValidCodePage@4   1007a10c     kernel32:KERNEL32.dll
 0002:00000110       __imp__TlsGetValue@4       1007a110     kernel32:KERNEL32.dll
 0002:00000114       __imp__TlsAlloc@0          1007a114     kernel32:KERNEL32.dll
 0002:00000118       __imp__TlsSetValue@8       1007a118     kernel32:KERNEL32.dll
 0002:0000011c       __imp__TlsFree@4           1007a11c     kernel32:KERNEL32.dll
 0002:00000120       __imp__SetLastError@4      1007a120     kernel32:KERNEL32.dll
 0002:00000124       __imp__GetCurrentThread@0  1007a124     kernel32:KERNEL32.dll
 0002:00000128       __imp__WriteFile@20        1007a128     kernel32:KERNEL32.dll
 0002:0000012c       __imp__GetStdHandle@4      1007a12c     kernel32:KERNEL32.dll
 0002:00000130       __imp__HeapSize@12         1007a130     kernel32:KERNEL32.dll
 0002:00000134       __imp__SetFilePointer@16   1007a134     kernel32:KERNEL32.dll
 0002:00000138       __imp__MultiByteToWideChar@24 1007a138     kernel32:KERNEL32.dll
 0002:0000013c       __imp__ReadFile@20         1007a13c     kernel32:KERNEL32.dll
 0002:00000140       __imp__CloseHandle@4       1007a140     kernel32:KERNEL32.dll
 0002:00000144       __imp__WideCharToMultiByte@32 1007a144     kernel32:KERNEL32.dll
 0002:00000148       __imp__GetConsoleCP@0      1007a148     kernel32:KERNEL32.dll
 0002:0000014c       __imp__GetConsoleMode@8    1007a14c     kernel32:KERNEL32.dll
 0002:00000150       __imp__SetHandleCount@4    1007a150     kernel32:KERNEL32.dll
 0002:00000154       __imp__GetFileType@4       1007a154     kernel32:KERNEL32.dll
 0002:00000158       __imp__GetStartupInfoA@4   1007a158     kernel32:KERNEL32.dll
 0002:0000015c       __imp__FreeEnvironmentStringsA@4 1007a15c     kernel32:KERNEL32.dll
 0002:00000160       __imp__GetEnvironmentStrings@0 1007a160     kernel32:KERNEL32.dll
 0002:00000164       __imp__FreeEnvironmentStringsW@4 1007a164     kernel32:KERNEL32.dll
 0002:00000168       __imp__GetEnvironmentStringsW@0 1007a168     kernel32:KERNEL32.dll
 0002:0000016c       __imp__QueryPerformanceCounter@4 1007a16c     kernel32:KERNEL32.dll
 0002:00000170       __imp__GetTickCount@0      1007a170     kernel32:KERNEL32.dll
 0002:00000174       __imp__GetCurrentProcessId@0 1007a174     kernel32:KERNEL32.dll
 0002:00000178       __imp__GetSystemTimeAsFileTime@4 1007a178     kernel32:KERNEL32.dll
 0002:0000017c       __imp__LCMapStringA@24     1007a17c     kernel32:KERNEL32.dll
 0002:00000180       __imp__LCMapStringW@24     1007a180     kernel32:KERNEL32.dll
 0002:00000184       __imp__SetStdHandle@8      1007a184     kernel32:KERNEL32.dll
 0002:00000188       __imp__SetConsoleCtrlHandler@8 1007a188     kernel32:KERNEL32.dll
 0002:0000018c       __imp__InitializeCriticalSectionAndSpinCount@8 1007a18c     kernel32:KERNEL32.dll
 0002:00000190       __imp__GetStringTypeA@20   1007a190     kernel32:KERNEL32.dll
 0002:00000194       __imp__GetStringTypeW@16   1007a194     kernel32:KERNEL32.dll
 0002:00000198       __imp__GetTimeFormatA@24   1007a198     kernel32:KERNEL32.dll
 0002:0000019c       __imp__GetDateFormatA@24   1007a19c     kernel32:KERNEL32.dll
 0002:000001a0       __imp__GetUserDefaultLCID@0 1007a1a0     kernel32:KERNEL32.dll
 0002:000001a4       __imp__GetLocaleInfoA@16   1007a1a4     kernel32:KERNEL32.dll
 0002:000001a8       __imp__EnumSystemLocalesA@8 1007a1a8     kernel32:KERNEL32.dll
 0002:000001ac       __imp__IsValidLocale@8     1007a1ac     kernel32:KERNEL32.dll
 0002:000001b0       __imp__FlushFileBuffers@4  1007a1b0     kernel32:KERNEL32.dll
 0002:000001b4       __imp__CreateFileA@28      1007a1b4     kernel32:KERNEL32.dll
 0002:000001b8       __imp__WriteConsoleA@20    1007a1b8     kernel32:KERNEL32.dll
 0002:000001bc       __imp__GetConsoleOutputCP@0 1007a1bc     kernel32:KERNEL32.dll
 0002:000001c0       __imp__FileTimeToLocalFileTime@8 1007a1c0     kernel32:KERNEL32.dll
 0002:000001c4       \177KERNEL32_NULL_THUNK_DATA 1007a1c4     kernel32:KERNEL32.dll
 0002:000001c8       __imp__GetDesktopWindow@0  1007a1c8     user32:USER32.dll
 0002:000001cc       __imp__SendMessageA@16     1007a1cc     user32:USER32.dll
 0002:000001d0       __imp__wsprintfA           1007a1d0     user32:USER32.dll
 0002:000001d4       \177USER32_NULL_THUNK_DATA 1007a1d4     user32:USER32.dll
 0002:000001d8       __imp__mixerGetLineControlsA@12 1007a1d8     winmm:WINMM.dll
 0002:000001dc       __imp__mixerGetNumDevs@0   1007a1dc     winmm:WINMM.dll
 0002:000001e0       __imp__mixerOpen@20        1007a1e0     winmm:WINMM.dll
 0002:000001e4       __imp__mixerGetDevCapsA@12 1007a1e4     winmm:WINMM.dll
 0002:000001e8       __imp__mixerGetLineInfoA@12 1007a1e8     winmm:WINMM.dll
 0002:000001ec       __imp__mixerClose@4        1007a1ec     winmm:WINMM.dll
 0002:000001f0       __imp__mixerGetControlDetailsA@12 1007a1f0     winmm:WINMM.dll
 0002:000001f4       __imp__timeGetTime@0       1007a1f4     winmm:WINMM.dll
 0002:000001f8       __imp__timeEndPeriod@4     1007a1f8     winmm:WINMM.dll
 0002:000001fc       __imp__timeSetEvent@20     1007a1fc     winmm:WINMM.dll
 0002:00000200       __imp__mmioRead@12         1007a200     winmm:WINMM.dll
 0002:00000204       __imp__mmioSeek@12         1007a204     winmm:WINMM.dll
 0002:00000208       __imp__mmioClose@8         1007a208     winmm:WINMM.dll
 0002:0000020c       __imp__timeKillEvent@4     1007a20c     winmm:WINMM.dll
 0002:00000210       __imp__mixerSetControlDetails@12 1007a210     winmm:WINMM.dll
 0002:00000214       __imp__timeBeginPeriod@4   1007a214     winmm:WINMM.dll
 0002:00000218       \177WINMM_NULL_THUNK_DATA  1007a218     winmm:WINMM.dll
 0002:0000021c       __imp__MakeSureDirectoryPathExists@4 1007a21c     Dbghelp:dbghelp.dll
 0002:00000220       \177dbghelp_NULL_THUNK_DATA 1007a220     Dbghelp:dbghelp.dll
 0002:00000224       __imp__CoInitialize@4      1007a224     ole32:ole32.dll
 0002:00000228       __imp__CoUninitialize@0    1007a228     ole32:ole32.dll
 0002:0000022c       \177ole32_NULL_THUNK_DATA  1007a22c     ole32:ole32.dll
 0002:00000230       ___xc_a                    1007a230     LIBCMT:crt0init.obj
 0002:00000268       ___xc_z                    1007a268     LIBCMT:crt0init.obj
 0002:0000026c       ___xi_a                    1007a26c     LIBCMT:crt0init.obj
 0002:00000284       ___xi_z                    1007a284     LIBCMT:crt0init.obj
 0002:00000288       ___xp_a                    1007a288     LIBCMT:crt0init.obj
 0002:00000294       ___xp_z                    1007a294     LIBCMT:crt0init.obj
 0002:00000298       ___xt_a                    1007a298     LIBCMT:crt0init.obj
 0002:0000029c       ___xt_z                    1007a29c     LIBCMT:crt0init.obj
 0002:000002bc       ??_C@_0P@GHFPNOJB@bad?5allocation?$AA@ 1007a2bc     audiostr.obj
 0002:000002cb       ?_Value@?$_Is_swap_move@U_Swap_move_tag@std@@@std@@2_NB 1007a2cb     audiostr.obj
 0002:000002cc       ?value@?$integral_constant@_N$0A@@tr1@std@@2_NB 1007a2cc     audiostr.obj
 0002:000002cd       ?value@?$integral_constant@_N$00@tr1@std@@2_NB 1007a2cd     audiostr.obj
 0002:000002d0       ??_C@_0BN@JACENBPF@?$CB?$CB?5is?5not?5Ogg?5BitStream?5file?$AA@ 1007a2d0     audiostr.obj
 0002:000002f0       ??_C@_0CH@CAKNHALN@?1?1?5not?5an?5OGG?5so?5assume?5that?5it?8@ 1007a2f0     audiostr.obj
 0002:00000318       ??_C@_0CN@FMOCCFFO@?$CFd?5time?5error?5for?5reading?5data?5f@ 1007a318     audiostr.obj
 0002:00000348       ??_C@_0CH@NMNFIPJD@?$CI?$CFs?$CJ?5ov_open_callbacks?9?5?5?$CIch?5?$CFd?$CJ@ 1007a348     audiostr.obj
 0002:00000370       ??_C@_0ED@MLJAHFGD@AUDIOSTR?5?$DN?$DO?5OGG?5reading?5error?3?5?5@ 1007a370     audiostr.obj
 0002:000003b4       ??_C@_0CO@OCLMGODK@?$EAERROR?3?5could?5not?5find?5file?5?$CFs?5i@ 1007a3b4     audiostr.obj
 0002:000003e4       ??_C@_0DA@GCGHODBF@?$CDOPEN?5streaming?5file?5?5?$CI?$CFs?$CJ?5in?5lo@ 1007a3e4     audiostr.obj
 0002:00000414       ??_C@_01KICIPPFI@?2?$AA@   1007a414     audiostr.obj
 0002:00000418       ??_C@_02JDPG@rb?$AA@       1007a418     audiostr.obj
 0002:0000041c       ??_C@_0CH@HBBDHBGP@?$CDOPEN?5streaming?5file?5?5?$CI?$CFs?$CJ?5in?5pa@ 1007a41c     audiostr.obj
 0002:00000444       ??_C@_03NKNKOHHD@ogg?$AA@  1007a444     audiostr.obj
 0002:00000448       ??_C@_07BDCAJABG@Destroy?$AA@ 1007a448     audiostr.obj
 0002:00000450       __real@bf800000            1007a450     audiostr.obj
 0002:00000454       _CLSID_DirectSound         1007a454     ds.obj
 0002:00000464       _CLSID_DirectSound8        1007a464     ds.obj
 0002:00000474       _CLSID_DirectSoundCapture  1007a474     ds.obj
 0002:00000484       _CLSID_DirectSoundCapture8 1007a484     ds.obj
 0002:00000494       _CLSID_DirectSoundFullDuplex 1007a494     ds.obj
 0002:000004a4       _DSDEVID_DefaultPlayback   1007a4a4     ds.obj
 0002:000004b4       _DSDEVID_DefaultCapture    1007a4b4     ds.obj
 0002:000004c4       _DSDEVID_DefaultVoicePlayback 1007a4c4     ds.obj
 0002:000004d4       _DSDEVID_DefaultVoiceCapture 1007a4d4     ds.obj
 0002:000004e4       _IID_IReferenceClock       1007a4e4     ds.obj
 0002:000004f4       _IID_IDirectSound          1007a4f4     ds.obj
 0002:00000504       _IID_IDirectSound8         1007a504     ds.obj
 0002:00000514       _IID_IDirectSoundBuffer    1007a514     ds.obj
 0002:00000524       _IID_IDirectSoundBuffer8   1007a524     ds.obj
 0002:00000534       _GUID_All_Objects          1007a534     ds.obj
 0002:00000544       _IID_IDirectSound3DListener 1007a544     ds.obj
 0002:00000554       _IID_IDirectSound3DBuffer  1007a554     ds.obj
 0002:00000564       _IID_IDirectSoundCapture   1007a564     ds.obj
 0002:00000574       _IID_IDirectSoundCaptureBuffer 1007a574     ds.obj
 0002:00000584       _IID_IDirectSoundCaptureBuffer8 1007a584     ds.obj
 0002:00000594       _IID_IDirectSoundNotify    1007a594     ds.obj
 0002:000005a4       _IID_IKsPropertySet        1007a5a4     ds.obj
 0002:000005b4       _IID_IDirectSoundFXGargle  1007a5b4     ds.obj
 0002:000005c4       _IID_IDirectSoundFXChorus  1007a5c4     ds.obj
 0002:000005d4       _IID_IDirectSoundFXFlanger 1007a5d4     ds.obj
 0002:000005e4       _IID_IDirectSoundFXEcho    1007a5e4     ds.obj
 0002:000005f4       _IID_IDirectSoundFXDistortion 1007a5f4     ds.obj
 0002:00000604       _IID_IDirectSoundFXCompressor 1007a604     ds.obj
 0002:00000614       _IID_IDirectSoundFXParamEq 1007a614     ds.obj
 0002:00000624       _IID_IDirectSoundFXI3DL2Reverb 1007a624     ds.obj
 0002:00000634       _IID_IDirectSoundFXWavesReverb 1007a634     ds.obj
 0002:00000644       _IID_IDirectSoundCaptureFXAec 1007a644     ds.obj
 0002:00000654       _IID_IDirectSoundCaptureFXNoiseSuppress 1007a654     ds.obj
 0002:00000664       _IID_IDirectSoundFullDuplex 1007a664     ds.obj
 0002:00000674       _DS3DALG_NO_VIRTUALIZATION 1007a674     ds.obj
 0002:00000684       _DS3DALG_HRTF_FULL         1007a684     ds.obj
 0002:00000694       _DS3DALG_HRTF_LIGHT        1007a694     ds.obj
 0002:000006a4       _GUID_DSFX_STANDARD_GARGLE 1007a6a4     ds.obj
 0002:000006b4       _GUID_DSFX_STANDARD_CHORUS 1007a6b4     ds.obj
 0002:000006c4       _GUID_DSFX_STANDARD_FLANGER 1007a6c4     ds.obj
 0002:000006d4       _GUID_DSFX_STANDARD_ECHO   1007a6d4     ds.obj
 0002:000006e4       _GUID_DSFX_STANDARD_DISTORTION 1007a6e4     ds.obj
 0002:000006f4       _GUID_DSFX_STANDARD_COMPRESSOR 1007a6f4     ds.obj
 0002:00000704       _GUID_DSFX_STANDARD_PARAMEQ 1007a704     ds.obj
 0002:00000714       _GUID_DSFX_STANDARD_I3DL2REVERB 1007a714     ds.obj
 0002:00000724       _GUID_DSFX_WAVES_REVERB    1007a724     ds.obj
 0002:00000734       _GUID_DSCFX_CLASS_AEC      1007a734     ds.obj
 0002:00000744       _GUID_DSCFX_MS_AEC         1007a744     ds.obj
 0002:00000754       _GUID_DSCFX_SYSTEM_AEC     1007a754     ds.obj
 0002:00000764       _GUID_DSCFX_CLASS_NS       1007a764     ds.obj
 0002:00000774       _GUID_DSCFX_MS_NS          1007a774     ds.obj
 0002:00000784       _GUID_DSCFX_SYSTEM_NS      1007a784     ds.obj
 0002:00000794       _DSPROPSETID_EAX_ReverbProperties 1007a794     ds.obj
 0002:000007a4       _DSPROPSETID_EAXBUFFER_ReverbProperties 1007a7a4     ds.obj
 0002:000007b8       __real@408f400000000000    1007a7b8     ds.obj
 0002:000007c0       __real@4059000000000000    1007a7c0     ds.obj
 0002:000007c8       __real@4000000000000000    1007a7c8     ds.obj
 0002:000007d0       ??_C@_0CP@ICFBJNML@?8can?8t?5find?5free?5Software?5buffer@ 1007a7d0     ds.obj
 0002:00000800       ??_C@_0CP@PCCLABBK@?8can?8t?5find?5free?5Hardware?5buffer@ 1007a800     ds.obj
 0002:00000830       ??_C@_0BD@PPENOOPJ@DirectSoundCreate8?$AA@ 1007a830     ds.obj
 0002:00000844       ??_C@_0L@ELNNJJJ@dsound?4dll?$AA@ 1007a844     ds.obj
 0002:00000850       ??_C@_05FOGCOAPK@DS_OK?$AA@ 1007a850     ds.obj
 0002:00000858       ??_C@_07CIFAGBMG@unknown?$AA@ 1007a858     ds.obj
 0002:00000860       ??_C@_0BE@BMJCAPGM@DSERR_UNINITIALIZED?$AA@ 1007a860     ds.obj
 0002:00000874       ??_C@_0BB@MLKAOHBD@DSERR_BUFFERLOST?$AA@ 1007a874     ds.obj
 0002:00000888       ??_C@_0BG@JFJBCEJM@DSERR_OTHERAPPHASPRIO?$AA@ 1007a888     ds.obj
 0002:000008a0       ??_C@_0BJ@PODLOCNP@DSERR_ALREADYINITIALIZED?$AA@ 1007a8a0     ds.obj
 0002:000008bc       ??_C@_0BG@FGFOLLAI@DSERR_PRIOLEVELNEEDED?$AA@ 1007a8bc     ds.obj
 0002:000008d4       ??_C@_0P@HJFILJLC@DSERR_NODRIVER?$AA@ 1007a8d4     ds.obj
 0002:000008e4       ??_C@_0BC@NMCDDLDP@DSERR_INVALIDCALL?$AA@ 1007a8e4     ds.obj
 0002:000008f8       ??_C@_0BF@KBGGCPDE@DSERR_CONTROLUNAVAIL?$AA@ 1007a8f8     ds.obj
 0002:00000910       ??_C@_0BA@ECKDOBJD@DSERR_BADFORMAT?$AA@ 1007a910     ds.obj
 0002:00000920       ??_C@_0BA@COPOGMBA@DSERR_ALLOCATED?$AA@ 1007a920     ds.obj
 0002:00000930       ??_C@_0BC@KCMPJMLN@DSERR_OUTOFMEMORY?$AA@ 1007a930     ds.obj
 0002:00000944       ??_C@_0BD@MODBPMIE@DSERR_INVALIDPARAM?$AA@ 1007a944     ds.obj
 0002:00000958       ??_C@_0BE@FNFJCFJP@DSERR_NOAGGREGATION?$AA@ 1007a958     ds.obj
 0002:0000096c       ??_C@_0BC@IMOOOGNJ@DSERR_UNSUPPORTED?$AA@ 1007a96c     ds.obj
 0002:00000980       ??_C@_0O@PDIJJBF@DSERR_GENERIC?$AA@ 1007a980     ds.obj
 0002:00000990       __real@00000000            1007a990     ds.obj
 0002:00000998       ??_C@_0EE@EJANCIKG@?$FLCritical?5Error?$FN?5Unable?5to?5alloc@ 1007a998     ds.obj
 0002:000009dc       __real@3f800000            1007a9dc     ds.obj
 0002:000009e0       __real@41a00000            1007a9e0     ds.obj
 0002:000009e4       __real@3dcccccd            1007a9e4     ds.obj
 0002:000009e8       __real@3fb99999a0000000    1007a9e8     ds.obj
 0002:000009f0       __real@40000000            1007a9f0     ds.obj
 0002:000009f4       ??_C@_0BK@LFIIOGNJ@ds_set_volume?3?5?$CFf?$CK?$CFf?5?$DN?5?$CFf?$AA@ 1007a9f4     ds.obj
 0002:00000a14       ??_7bad_alloc@std@@6B@     1007aa14     sound.obj
 0002:00000a20       ??_C@_0JE@HFKFCDEG@DirectSound?5could?5not?5be?5initial@ 1007aa20     sound.obj
 0002:00000ab8       __real@4097700000000000    1007aab8     sound.obj
 0002:00000ac4       ??_7logic_error@std@@6B@   1007aac4     sound.obj
 0002:00000ad0       ??_7length_error@std@@6B@  1007aad0     sound.obj
 0002:00000adc       ??_7out_of_range@std@@6B@  1007aadc     sound.obj
 0002:00000ae4       ??_C@_0BE@JONHPENG@map?1set?$DMT?$DO?5too?5long?$AA@ 1007aae4     sound.obj
 0002:00000af8       ??_C@_0BM@PAPJHAGI@invalid?5map?1set?$DMT?$DO?5iterator?$AA@ 1007aaf8     sound.obj
 0002:00000b18       __real@3fc0000000000000    1007ab18     sound.obj
 0002:00000b20       __real@4f800000            1007ab20     sound.obj
 0002:00000b28       __real@3fd3333333333333    1007ab28     sound.obj
 0002:00000b30       __real@3fe0000000000000    1007ab30     sound.obj
 0002:00000b38       ??_C@_0BO@DBKAIMCB@can?8t?5play?5ambient?5sound?5?3?5?$CFd?$AA@ 1007ab38     ambientsnd.obj
 0002:00000b58       ??_C@_08LPEFNMAG@none?4wav?$AA@ 1007ab58     gamesnd.obj
 0002:00000b64       ??_C@_0BG@LOBOAFMF@can?8t?5play?5sound?5?3?5?$CFd?$AA@ 1007ab64     gamesnd.obj
 0002:00000b7c       ??_C@_05OCFELOIJ@1?40?40?$AA@ 1007ab7c     scriptparser.obj
 0002:00000b84       ?collate@?$_Locbase@H@std@@2HB 1007ab84     scriptparser.obj
 0002:00000b88       ?ctype@?$_Locbase@H@std@@2HB 1007ab88     scriptparser.obj
 0002:00000b8c       ?monetary@?$_Locbase@H@std@@2HB 1007ab8c     scriptparser.obj
 0002:00000b90       ?numeric@?$_Locbase@H@std@@2HB 1007ab90     scriptparser.obj
 0002:00000b94       ?time@?$_Locbase@H@std@@2HB 1007ab94     scriptparser.obj
 0002:00000b98       ?messages@?$_Locbase@H@std@@2HB 1007ab98     scriptparser.obj
 0002:00000b9c       ?all@?$_Locbase@H@std@@2HB 1007ab9c     scriptparser.obj
 0002:00000ba0       ?none@?$_Locbase@H@std@@2HB 1007aba0     scriptparser.obj
 0002:00000ba4       ?table_size@?$ctype@D@std@@2IB 1007aba4     scriptparser.obj
 0002:00000ba8       ?skipws@?$_Iosb@H@std@@2W4_Fmtflags@12@B 1007aba8     scriptparser.obj
 0002:00000bac       ?unitbuf@?$_Iosb@H@std@@2W4_Fmtflags@12@B 1007abac     scriptparser.obj
 0002:00000bb0       ?uppercase@?$_Iosb@H@std@@2W4_Fmtflags@12@B 1007abb0     scriptparser.obj
 0002:00000bb4       ?showbase@?$_Iosb@H@std@@2W4_Fmtflags@12@B 1007abb4     scriptparser.obj
 0002:00000bb8       ?showpoint@?$_Iosb@H@std@@2W4_Fmtflags@12@B 1007abb8     scriptparser.obj
 0002:00000bbc       ?showpos@?$_Iosb@H@std@@2W4_Fmtflags@12@B 1007abbc     scriptparser.obj
 0002:00000bc0       ?left@?$_Iosb@H@std@@2W4_Fmtflags@12@B 1007abc0     scriptparser.obj
 0002:00000bc4       ?right@?$_Iosb@H@std@@2W4_Fmtflags@12@B 1007abc4     scriptparser.obj
 0002:00000bc8       ?internal@?$_Iosb@H@std@@2W4_Fmtflags@12@B 1007abc8     scriptparser.obj
 0002:00000bcc       ?dec@?$_Iosb@H@std@@2W4_Fmtflags@12@B 1007abcc     scriptparser.obj
 0002:00000bd0       ?oct@?$_Iosb@H@std@@2W4_Fmtflags@12@B 1007abd0     scriptparser.obj
 0002:00000bd4       ?hex@?$_Iosb@H@std@@2W4_Fmtflags@12@B 1007abd4     scriptparser.obj
 0002:00000bd8       ?scientific@?$_Iosb@H@std@@2W4_Fmtflags@12@B 1007abd8     scriptparser.obj
 0002:00000bdc       ?fixed@?$_Iosb@H@std@@2W4_Fmtflags@12@B 1007abdc     scriptparser.obj
 0002:00000be0       ?hexfloat@?$_Iosb@H@std@@2W4_Fmtflags@12@B 1007abe0     scriptparser.obj
 0002:00000be4       ?boolalpha@?$_Iosb@H@std@@2W4_Fmtflags@12@B 1007abe4     scriptparser.obj
 0002:00000be8       ?_Stdio@?$_Iosb@H@std@@2W4_Fmtflags@12@B 1007abe8     scriptparser.obj
 0002:00000bec       ?adjustfield@?$_Iosb@H@std@@2W4_Fmtflags@12@B 1007abec     scriptparser.obj
 0002:00000bf0       ?basefield@?$_Iosb@H@std@@2W4_Fmtflags@12@B 1007abf0     scriptparser.obj
 0002:00000bf4       ?floatfield@?$_Iosb@H@std@@2W4_Fmtflags@12@B 1007abf4     scriptparser.obj
 0002:00000bf8       ?goodbit@?$_Iosb@H@std@@2W4_Iostate@12@B 1007abf8     scriptparser.obj
 0002:00000bfc       ?eofbit@?$_Iosb@H@std@@2W4_Iostate@12@B 1007abfc     scriptparser.obj
 0002:00000c00       ?failbit@?$_Iosb@H@std@@2W4_Iostate@12@B 1007ac00     scriptparser.obj
 0002:00000c04       ?badbit@?$_Iosb@H@std@@2W4_Iostate@12@B 1007ac04     scriptparser.obj
 0002:00000c08       ?_Hardfail@?$_Iosb@H@std@@2W4_Iostate@12@B 1007ac08     scriptparser.obj
 0002:00000c0c       ?in@?$_Iosb@H@std@@2W4_Openmode@12@B 1007ac0c     scriptparser.obj
 0002:00000c10       ?out@?$_Iosb@H@std@@2W4_Openmode@12@B 1007ac10     scriptparser.obj
 0002:00000c14       ?ate@?$_Iosb@H@std@@2W4_Openmode@12@B 1007ac14     scriptparser.obj
 0002:00000c18       ?app@?$_Iosb@H@std@@2W4_Openmode@12@B 1007ac18     scriptparser.obj
 0002:00000c1c       ?trunc@?$_Iosb@H@std@@2W4_Openmode@12@B 1007ac1c     scriptparser.obj
 0002:00000c20       ?_Nocreate@?$_Iosb@H@std@@2W4_Openmode@12@B 1007ac20     scriptparser.obj
 0002:00000c24       ?_Noreplace@?$_Iosb@H@std@@2W4_Openmode@12@B 1007ac24     scriptparser.obj
 0002:00000c28       ?binary@?$_Iosb@H@std@@2W4_Openmode@12@B 1007ac28     scriptparser.obj
 0002:00000c2c       ?beg@?$_Iosb@H@std@@2W4_Seekdir@12@B 1007ac2c     scriptparser.obj
 0002:00000c30       ?cur@?$_Iosb@H@std@@2W4_Seekdir@12@B 1007ac30     scriptparser.obj
 0002:00000c34       ?end@?$_Iosb@H@std@@2W4_Seekdir@12@B 1007ac34     scriptparser.obj
 0002:00000c38       ??_C@_07GDJHAFNB@doppler?$AA@ 1007ac38     scriptparser.obj
 0002:00000c40       ??_C@_07DGBKEDPM@rolloff?$AA@ 1007ac40     scriptparser.obj
 0002:00000c48       ??_C@_0BD@CAKBHHCG@doppler_factor?3?5?$CFf?$AA@ 1007ac48     scriptparser.obj
 0002:00000c5c       ??_C@_0BD@HENBNIKL@rolloff_factor?3?5?$CFf?$AA@ 1007ac5c     scriptparser.obj
 0002:00000c70       ??_C@_01IPJKGB@?$CD?$AA@   1007ac70     scriptparser.obj
 0002:00000c74       ??_C@_06LLCHJONG@Config?$AA@ 1007ac74     scriptparser.obj
 0002:00000c7c       ??_C@_0BL@LGAAMPPI@can?8t?5read?5config?5file?3?5?$CFs?$AA@ 1007ac7c     scriptparser.obj
 0002:00000c98       ??_C@_06DFLDJKHK@euc?9kr?$AA@ 1007ac98     scriptparser.obj
 0002:00000ca0       ??_C@_0BD@OLBABOEK@vector?$DMT?$DO?5too?5long?$AA@ 1007aca0     scriptparser.obj
 0002:00000cb4       ??_C@_0BC@IFKMNIFL@END_AMBIENT_SOUND?$AA@ 1007acb4     scriptparser.obj
 0002:00000cc8       ??_C@_0BE@LACDJGHH@BEGIN_AMBIENT_SOUND?$AA@ 1007acc8     scriptparser.obj
 0002:00000cdc       ??_C@_0N@DOAEGMLI@END_UI_SOUND?$AA@ 1007acdc     scriptparser.obj
 0002:00000cec       ??_C@_0P@LHKPHOON@BEGIN_UI_SOUND?$AA@ 1007acec     scriptparser.obj
 0002:00000cfc       ??_C@_0BD@KKFLLHDM@END_GAMEPLAY_SOUND?$AA@ 1007acfc     scriptparser.obj
 0002:00000d10       ??_C@_0BF@JILGFEJB@BEGIN_GAMEPLAY_SOUND?$AA@ 1007ad10     scriptparser.obj
 0002:00000d28       ??_C@_0BD@GABPLJEN@ambient?5?$FLID?3?$CFd?$FN?5?$CFs?$AA@ 1007ad28     scriptparser.obj
 0002:00000d3c       ??_C@_0BE@HIGDCMN@gameplay?5?$FLID?3?$CFd?$FN?5?$CFs?$AA@ 1007ad3c     scriptparser.obj
 0002:00000d50       ??_C@_05BMGBEOOC@?$CFs?2?$CFs?$AA@ 1007ad50     scriptparser.obj
 0002:00000d58       ??_C@_0DF@CGCGHMDD@xls?5parsing?5error?3?5invalid?5?$CD?5?5in@ 1007ad58     scriptparser.obj
 0002:00000d90       ??_C@_0M@ONKGKIJL@sound_table?$AA@ 1007ad90     scriptparser.obj
 0002:00000d9c       ??_C@_0CI@JDGBAAMP@can?8t?5read?5sound?5configuration?5f@ 1007ad9c     scriptparser.obj
 0002:00000dc4       ??_C@_0N@ECONFPOO@END_UI_MUSIC?$AA@ 1007adc4     scriptparser.obj
 0002:00000dd4       ??_C@_0BN@BOIGPPOH@music?5?$FLID?3?$CFd?$FN?5?$CFs?5?5?$CISlot?3?5?$CFd?$CJ?$AA@ 1007add4     scriptparser.obj
 0002:00000df4       ??_C@_0P@MLEGENLL@BEGIN_UI_MUSIC?$AA@ 1007adf4     scriptparser.obj
 0002:00000e04       ??_C@_0M@CHGMBOKB@music_table?$AA@ 1007ae04     scriptparser.obj
 0002:00000e10       ??_C@_0CI@JFEFIBLK@can?8t?5read?5music?5configuration?5f@ 1007ae10     scriptparser.obj
 0002:00000e38       ??_C@_0BA@PDNJFCMA@END_VOICE_SOUND?$AA@ 1007ae38     scriptparser.obj
 0002:00000e48       ??_C@_0BN@OMFHFOAG@voice?5?$FLID?3?$CFd?$FN?5?$CFs?5?5?$CISlot?3?5?$CFd?$CJ?$AA@ 1007ae48     scriptparser.obj
 0002:00000e68       ??_C@_0BC@KAFOLEKB@BEGIN_VOICE_SOUND?$AA@ 1007ae68     scriptparser.obj
 0002:00000e7c       ??_C@_0M@GNEDICNM@Voice_table?$AA@ 1007ae7c     scriptparser.obj
 0002:00000e88       ??_C@_0CI@GHJECAFL@can?8t?5read?5voice?5configuration?5f@ 1007ae88     scriptparser.obj
 0002:00000eb0       ??_C@_00CNPNBAHC@?$AA@     1007aeb0     scriptparser.obj
 0002:00000eb4       ??_C@_04HGIPLDBL@?$CFd?$AN?6?$AA@ 1007aeb4     scriptparser.obj
 0002:00000ebc       ??_C@_0BE@NEJEJMDJ@amdInitialize?5Error?$AA@ 1007aebc     util_audiomixer.obj
 0002:00000ed0       ??_C@_0EJ@LGHDPJPO@?$FL?$CFd?$FN?5found?5MIXERLINE_COMPONENTTY@ 1007aed0     util_audiomixer.obj
 0002:00000f1c       ??_C@_0BP@FDGPJNDL@Failed?5to?5get?5the?5line?5control?$AA@ 1007af1c     util_audiomixer.obj
 0002:00000f3c       ??_C@_0BK@JKDLHODC@Unable?5to?5get?5source?5line?$AA@ 1007af3c     util_audiomixer.obj
 0002:00000f58       ??_C@_0BH@HDMPOKNM@Got?5the?5source?5line?5id?$AA@ 1007af58     util_audiomixer.obj
 0002:00000f70       ??_C@_06IALFDLEA@?$LI?$LG?$MA?L?E?$KJ?$AA@ 1007af70     util_audiomixer.obj
 0002:00000f78       ??_C@_02LMMGGCAJ@?3?5?$AA@ 1007af78     util_debug.obj
 0002:00000f7c       ??_C@_01LFCBOECM@?4?$AA@   1007af7c     util_shwapi.obj
 0002:00000f80       ??_C@_0CG@DDKLCEHK@?$CI?$CFx?$CJ?5?$CK?$CK?$CK?$CK?$CK?$CK?$CK?$CK?$CK?$CK?$CKREAD?5ERROR?5?$CK?$CK?$CK?$CK?$CK@ 1007af80     cfile.obj
 0002:00000fa8       ??_C@_0CK@DIPHEHCA@get_cfile_block?5succeessfully?5re@ 1007afa8     cfile.obj
 0002:00000fd4       ??_C@_0CE@IDJGCCPI@get_cfile_block?5succeessfully?5st@ 1007afd4     cfile.obj
 0002:00000ff8       ??_C@_0CL@CHGEIBMF@free_cfile_block?5succeessfully?5r@ 1007aff8     cfile.obj
 0002:00001024       ??_C@_0CF@KDJOPKIN@free_cfile_block?5succeessfully?5s@ 1007b024     cfile.obj
 0002:0000104c       ??_C@_0BN@EIJID@can?8t?5find?5?5?$CI?$CFs?$CJ?5in?5packFile?$AA@ 1007b04c     cfile.obj
 0002:0000106c       ??_C@_0BG@GCMJPKEN@cfopen?5file_path?5?3?5?$CFs?$AA@ 1007b06c     cfile.obj
 0002:00001088       __real@3ff0000000000000    1007b088     floating.obj
 0002:00001090       __real@40dfffc000000000    1007b090     floating.obj
 0002:00001098       __real@400921fb60000000    1007b098     vecmat.obj
 0002:000010a0       __real@bfc90fdb            1007b0a0     vecmat.obj
 0002:000010a4       __real@3fc90fdb            1007b0a4     vecmat.obj
 0002:000010a8       __real@3fd5555560000000    1007b0a8     vecmat.obj
 0002:000010b0       __real@3fd0000000000000    1007b0b0     vecmat.obj
 0002:000010b8       __real@3f1a36e2eb1c432d    1007b0b8     vecmat.obj
 0002:000010c0       __real@0000000000000000    1007b0c0     vecmat.obj
 0002:000010c8       __real@40c3880000000000    1007b0c8     vecmat.obj
 0002:000010d0       __real@3c23d70a            1007b0d0     vecmat.obj
 0002:000010d4       __real@461c3f9a            1007b0d4     vecmat.obj
 0002:000010d8       __real@3ba3d70a            1007b0d8     vecmat.obj
 0002:000010dc       __real@350637bd            1007b0dc     vecmat.obj
 0002:000010e0       __real@401921fb60000000    1007b0e0     vecmat.obj
 0002:000010e8       __real@40490fdb            1007b0e8     vecmat.obj
 0002:000010f0       __real@bfefffffc0000000    1007b0f0     vecmat.obj
 0002:000010f8       __real@3fefffffc0000000    1007b0f8     vecmat.obj
 0002:00001100       __real@3ffe666660000000    1007b100     vecmat.obj
 0002:00001108       __real@3ff0ccccc0000000    1007b108     vecmat.obj
 0002:00001110       __real@4000ccccc0000000    1007b110     vecmat.obj
 0002:00001118       __real@3ee4f8b588e368f1    1007b118     vecmat.obj
 0002:00001120       __real@3e7ad7f29abcaf48    1007b120     vecmat.obj
 0002:00001128       __real@4010000000000000    1007b128     vecmat.obj
 0002:00001130       __real@3727c5ac            1007b130     vecmat.obj
 0002:00001138       __real@3bc79ca10c924223    1007b138     vecmat.obj
 0002:00001140       __real@3f91df3300000000    1007b140     vecmat.obj
 0002:00001148       __real@ccbebc20            1007b148     vecmat.obj
 0002:0000114c       __real@4cbebc20            1007b14c     vecmat.obj
 0002:00001150       __real@4066800000000000    1007b150     vecmat.obj
 0002:00001158       __real@400921fa00000000    1007b158     vecmat.obj
 0002:00001160       __real@43b38000            1007b160     vecmat.obj
 0002:00001164       ??_C@_06CPFLJKI@KOI8?9R?$AA@ 1007b164     ole.obj
 0002:0000116c       ??_C@_0BC@KPKIOBLF@Fat?5Size?3?7?$CFi?0?$CFX?5?6?$AA@ 1007b16c     ole.obj
 0002:00001180       ??_C@_0BA@OOOJGKBM@Count?5Dif?3?7?$CFi?5?6?$AA@ 1007b180     ole.obj
 0002:00001190       ??_C@_0BA@CBEFDILE@Dif?5start?3?7?$CFX?5?6?$AA@ 1007b190     ole.obj
 0002:000011a0       ??_C@_0BB@NEENJNCK@Count?5MFat?3?7?$CFi?5?6?$AA@ 1007b1a0     ole.obj
 0002:000011b4       ??_C@_0BF@EGFHLFAK@MiniFat?5Start?3?7?$CFXh?5?6?$AA@ 1007b1b4     ole.obj
 0002:000011cc       ??_C@_0BC@GOIPDEMO@Mini?5Cutoff?3?7?$CFi?5?6?$AA@ 1007b1cc     ole.obj
 0002:000011e0       ??_C@_0BA@OPNMPPP@Dir?5Start?3?7?$CFi?5?6?$AA@ 1007b1e0     ole.obj
 0002:000011f0       ??_C@_0BA@HKFGOLOH@Fat?5sect?4?3?7?$CFi?5?6?$AA@ 1007b1f0     ole.obj
 0002:00001200       ??_C@_0BE@JMAHHPDC@mini?5len?3?7?$CFXh?5?$CI?$CFi?$CJ?6?$AA@ 1007b200     ole.obj
 0002:00001214       ??_C@_0BE@HDLEHKJD@sect?5len?3?7?$CFXh?5?$CI?$CFi?$CJ?6?$AA@ 1007b214     ole.obj
 0002:00001228       ??_C@_0BC@JPPGKHGD@Byte?5order?3?7?$CFXh?5?6?$AA@ 1007b228     ole.obj
 0002:0000123c       ??_C@_0P@DGOHBIAG@verdll?3?7?7?$CFXh?5?6?$AA@ 1007b23c     ole.obj
 0002:0000124c       ??_C@_0BA@HJDGMJB@verminor?3?7?$CFXh?5?6?$AA@ 1007b24c     ole.obj
 0002:0000125c       ??_C@_0BE@JNLNCLIE@verminor?3?7?$CFXh?5?5?$CFXh?6?$AA@ 1007b25c     ole.obj
 0002:00001270       ??_C@_0BC@LAGGPEPB@Header?5Size?3?7?$CFi?5?6?$AA@ 1007b270     ole.obj
 0002:00001284       ??_C@_0O@FHCIHLBD@xls_appendSST?$AA@ 1007b284     xls.obj
 0002:00001298       __real@41f0000000000000    1007b298     xls.obj
 0002:000012a0       ??_C@_0N@FIFEHJKH@xls_addSheet?$AA@ 1007b2a0     xls.obj
 0002:000012b0       ??_C@_0L@MOINHILE@xls_addRow?$AA@ 1007b2b0     xls.obj
 0002:000012bc       ??_C@_0O@BLICHBLC@xls_makeTable?$AA@ 1007b2bc     xls.obj
 0002:000012cc       ??_C@_0M@CHMEMMIB@xls_addCell?$AA@ 1007b2cc     xls.obj
 0002:000012d8       ??_C@_0M@BAGOPKC@xls_addFont?$AA@ 1007b2d8     xls.obj
 0002:000012e4       ??_C@_09GLCMNFNF@xls_addXF?$AA@ 1007b2e4     xls.obj
 0002:000012f0       ??_C@_0P@COHHPIP@xls_addColinfo?$AA@ 1007b2f0     xls.obj
 0002:00001300       ??_C@_0N@EOHHCEII@Merged?5Cells?$AA@ 1007b300     xls.obj
 0002:00001310       ??_C@_0BG@OJBMAAEK@xls_PreParseWorkSheet?$AA@ 1007b310     xls.obj
 0002:00001328       ??_C@_0BD@HMLKICGH@xls_ParseWorkSheet?$AA@ 1007b328     xls.obj
 0002:0000133c       ??_C@_0BB@FENKFBFK@xls_getWorkSheet?$AA@ 1007b33c     xls.obj
 0002:00001350       ??_C@_09ELCEGGHO@xls_close?$AA@ 1007b350     xls.obj
 0002:0000135c       ??_C@_0L@OFOJHEEE@xls_addSST?$AA@ 1007b35c     xls.obj
 0002:00001368       ??_C@_0BC@GCEGELDI@xls_ParseWorkBook?$AA@ 1007b368     xls.obj
 0002:0000137c       ??_C@_0BE@FNMMGAFK@Workbook?5not?5found?6?$AA@ 1007b37c     xls.obj
 0002:00001390       ??_C@_08FKPPLGGL@Workbook?$AA@ 1007b390     xls.obj
 0002:0000139c       ??_C@_0BF@IDMBKBIK@File?5?$CC?$CFs?$CC?5not?5found?6?$AA@ 1007b39c     xls.obj
 0002:000013b4       ??_C@_08DAKOEABO@xls_open?$AA@ 1007b3b4     xls.obj
 0002:000013c0       ??_C@_01BJJEKLCA@?$CC?$AA@ 1007b3c0     xls.obj
 0002:000013c4       ??_C@_01GPOEFGEJ@?7?$AA@   1007b3c4     xls.obj
 0002:000013c8       ??_C@_01EEMJAFIK@?6?$AA@   1007b3c8     xls.obj
 0002:000013cc       ??_C@_01KDCPPGHE@r?$AA@    1007b3cc     xls.obj
 0002:000013d0       ??_C@_0O@PIDLJLCH@BOF?9BIFF5?17?18?$AA@ 1007b3d0     xlstool.obj
 0002:000013e0       ??_C@_0DI@GKNCGAB@Formula?5related?0?5always?5before?5t@ 1007b3e0     xlstool.obj
 0002:00001418       ??_C@_0CA@EHLGNKAC@?$DPFORMULA?9RELATED?$DN?$DP?$CIBC?$DNSHRFMLA?$CJ?$CJ?$AA@ 1007b418     xlstool.obj
 0002:00001438       ??_C@_0O@DLHEJDKI@Number?5Format?$AA@ 1007b438     xlstool.obj
 0002:00001448       ??_C@_06DPGELLJH@FORMAT?$AA@ 1007b448     xlstool.obj
 0002:00001450       ??_C@_09KALIILMP@BOF?9BIFF4?$AA@ 1007b450     xlstool.obj
 0002:0000145c       ??_C@_0BC@IKFIIKPN@Style?5Information?$AA@ 1007b45c     xlstool.obj
 0002:00001470       ??_C@_05ELDPMCMC@STYLE?$AA@ 1007b470     xlstool.obj
 0002:00001478       ??_C@_0BG@PLOGDDG@Cell?5Value?0?5RK?5Number?$AA@ 1007b478     xlstool.obj
 0002:00001490       ??_C@_02HMALEKPN@RK?$AA@   1007b490     xlstool.obj
 0002:00001494       ??_C@_0BJ@EEGJJKEB@Sheet?5Window?5Information?$AA@ 1007b494     xlstool.obj
 0002:000014b0       ??_C@_07MLHIFLFJ@WINDOW2?$AA@ 1007b4b0     xlstool.obj
 0002:000014b8       ??_C@_0L@EJFKMGGC@Data?5Table?$AA@ 1007b4b8     xlstool.obj
 0002:000014c4       ??_C@_05HJCCDKBG@TABLE?$AA@ 1007b4c4     xlstool.obj
 0002:000014cc       ??_C@_0BD@ENMCJLHN@Default?5Row?5Height?$AA@ 1007b4cc     xlstool.obj
 0002:000014e0       ??_C@_0BB@KJEDNAAB@DEFAULTROWHEIGHT?$AA@ 1007b4e0     xlstool.obj
 0002:000014f4       ??_C@_0BL@FEMIGKAO@Externally?5Referenced?5Name?$AA@ 1007b4f4     xlstool.obj
 0002:00001510       ??_C@_0L@GHFIAONA@EXTERNNAME?$AA@ 1007b510     xlstool.obj
 0002:0000151c       ??_C@_0BG@IOFJKILA@Array?9Entered?5Formula?$AA@ 1007b51c     xlstool.obj
 0002:00001534       ??_C@_05LDMPNNPN@ARRAY?$AA@ 1007b534     xlstool.obj
 0002:0000153c       ??_C@_0N@OAPOACGP@Defined?5Name?$AA@ 1007b53c     xlstool.obj
 0002:0000154c       ??_C@_04IPKHEEB@NAME?$AA@  1007b54c     xlstool.obj
 0002:00001554       ??_C@_0N@GJHOCKBP@Index?5Record?$AA@ 1007b554     xlstool.obj
 0002:00001564       ??_C@_05JBOMLEMN@INDEX?$AA@ 1007b564     xlstool.obj
 0002:0000156c       ??_C@_09OPPJBNAI@BOF?9BIFF3?$AA@ 1007b56c     xlstool.obj
 0002:00001578       ??_C@_0BA@DAHBIKNA@Describes?5a?5Row?$AA@ 1007b578     xlstool.obj
 0002:00001588       ??_C@_03DBIDOGKE@ROW?$AA@  1007b588     xlstool.obj
 0002:0000158c       ??_C@_0BK@CLLBFEAC@String?5Value?5of?5a?5Formula?$AA@ 1007b58c     xlstool.obj
 0002:000015a8       ??_C@_06IGECGLFO@STRING?$AA@ 1007b5a8     xlstool.obj
 0002:000015b0       ??_C@_0BN@CIJBIJIM@Cell?5Value?0?5Boolean?5or?5Error?$AA@ 1007b5b0     xlstool.obj
 0002:000015d0       ??_C@_07GLFEIAGA@BOOLERR?$AA@ 1007b5d0     xlstool.obj
 0002:000015d8       ??_C@_0BM@HLNPLKH@Cell?5Value?0?5String?5Constant?$AA@ 1007b5d8     xlstool.obj
 0002:000015f4       ??_C@_05EILEDKCG@LABEL?$AA@ 1007b5f4     xlstool.obj
 0002:000015fc       ??_C@_0CC@LHEBHFNC@Cell?5Value?0?5Floating?9Point?5Numbe@ 1007b5fc     xlstool.obj
 0002:00001620       ??_C@_06EFEGMLFC@NUMBER?$AA@ 1007b620     xlstool.obj
 0002:00001628       ??_C@_0BH@FLCLNAMO@Cell?5Value?0?5Blank?5Cell?$AA@ 1007b628     xlstool.obj
 0002:00001640       ??_C@_05NLIPEJCP@BLANK?$AA@ 1007b640     xlstool.obj
 0002:00001648       ??_C@_0BA@OKNLGPCP@Cell?5Table?5Size?$AA@ 1007b648     xlstool.obj
 0002:00001658       ??_C@_0L@DNMOIILO@DIMENSIONS?$AA@ 1007b658     xlstool.obj
 0002:00001664       ??_C@_0BJ@JIHHEGCD@Data?5Validation?5Criteria?$AA@ 1007b664     xlstool.obj
 0002:00001680       ??_C@_02JLMMPJCD@DV?$AA@   1007b680     xlstool.obj
 0002:00001684       ??_C@_0CE@DMOHDJIH@Shared?5Workbook?5Protection?5Passw@ 1007b684     xlstool.obj
 0002:000016a8       ??_C@_0N@JAODDLDI@PROT4REVPASS?$AA@ 1007b6a8     xlstool.obj
 0002:000016b8       ??_C@_0BI@IDDCBFDO@SQL?5Datatype?5Identifier?$AA@ 1007b6b8     xlstool.obj
 0002:000016d0       ??_C@_09NOMEBI@SXFDBTYPE?$AA@ 1007b6d0     xlstool.obj
 0002:000016dc       ??_C@_09CAIAINMI@Hyperlink?$AA@ 1007b6dc     xlstool.obj
 0002:000016e8       ??_C@_05LPKAECKG@HLINK?$AA@ 1007b6e8     xlstool.obj
 0002:000016f0       ??_C@_0N@CNEFMFII@Refresh?5Flag?$AA@ 1007b6f0     xlstool.obj
 0002:00001700       ??_C@_0L@IEPMBANO@REFRESHALL?$AA@ 1007b700     xlstool.obj
 0002:0000170c       ??_C@_0M@CLEFNON@Text?5Object?$AA@ 1007b70c     xlstool.obj
 0002:00001718       ??_C@_03IPJKJENE@TXO?$AA@  1007b718     xlstool.obj
 0002:0000171c       ??_C@_07HLIIJJIG@DCONBIN?$AA@ 1007b71c     xlstool.obj
 0002:00001724       ??_C@_0BM@JOGMPBEG@Data?5Validation?5Information?$AA@ 1007b724     xlstool.obj
 0002:00001740       ??_C@_04FHFMEBOL@DVAL?$AA@ 1007b740     xlstool.obj
 0002:00001748       ??_C@_0CC@KPOLKMHC@Conditional?5Formatting?5Condition@ 1007b748     xlstool.obj
 0002:0000176c       ??_C@_02NEEBPNPH@CF?$AA@   1007b76c     xlstool.obj
 0002:00001770       ??_C@_0CJ@JIOCPNPK@Conditional?5Formatting?5Range?5Inf@ 1007b770     xlstool.obj
 0002:0000179c       ??_C@_07PEHPELP@CONDFMT?$AA@ 1007b79c     xlstool.obj
 0002:000017a4       ??_C@_0CA@OGEGLJOH@Shared?5Workbook?5Protection?5Flag?$AA@ 1007b7a4     xlstool.obj
 0002:000017c4       ??_C@_08PGOOHNHL@PROT4REV?$AA@ 1007b7c4     xlstool.obj
 0002:000017d0       ??_C@_0BE@LGCJFLBD@Supporting?5Workbook?$AA@ 1007b7d0     xlstool.obj
 0002:000017e4       ??_C@_07LFBIAFCF@SUPBOOK?$AA@ 1007b7e4     xlstool.obj
 0002:000017ec       ??_C@_0BE@PNGFHGNP@External?5Data?5Range?$AA@ 1007b7ec     xlstool.obj
 0002:00001800       ??_C@_03OCELCMIB@QSI?$AA@  1007b800     xlstool.obj
 0002:00001804       ??_C@_0BL@OHACEHBE@End?5of?5Custom?5View?5Records?$AA@ 1007b804     xlstool.obj
 0002:00001820       ??_C@_0N@CLENOLKD@USERSVIEWEND?$AA@ 1007b820     xlstool.obj
 0002:00001830       ??_C@_0BF@OCLGIKDB@Custom?5View?5Settings?$AA@ 1007b830     xlstool.obj
 0002:00001848       ??_C@_0P@NLCDIFBE@USERSVIEWBEGIN?$AA@ 1007b848     xlstool.obj
 0002:00001858       ??_C@_0BO@NLBEOBLC@Workbook?5Custom?5View?5Settings?$AA@ 1007b858     xlstool.obj
 0002:00001878       ??_C@_09ENNEJBCC@USERBVIEW?$AA@ 1007b878     xlstool.obj
 0002:00001884       ??_C@_0CK@CGCEAJJE@File?9Sharing?5Information?5for?5Sha@ 1007b884     xlstool.obj
 0002:000018b0       ??_C@_0N@EAPIJEHO@FILESHARING2?$AA@ 1007b8b0     xlstool.obj
 0002:000018c0       ??_C@_0N@NANFKDCO@Flag?5for?5DSF?$AA@ 1007b8c0     xlstool.obj
 0002:000018d0       ??_C@_09MMOOKOGO@XL5MODIFY?$AA@ 1007b8d0     xlstool.obj
 0002:000018dc       ??_C@_0BD@NKBDHPPM@Double?5Stream?5File?$AA@ 1007b8dc     xlstool.obj
 0002:000018f0       ??_C@_03CBEJHOD@DSF?$AA@   1007b8f0     xlstool.obj
 0002:000018f4       ??_C@_0BP@LKNLLGHM@Natural?5Language?5Formulas?5Flag?$AA@ 1007b8f4     xlstool.obj
 0002:00001914       ??_C@_08MCODPEJD@USESELFS?$AA@ 1007b914     xlstool.obj
 0002:00001920       ??_C@_0BG@CPBHDFPB@Sheet?5Tab?5Index?5Array?$AA@ 1007b920     xlstool.obj
 0002:00001938       ??_C@_05GGPCMJLM@TABID?$AA@ 1007b938     xlstool.obj
 0002:00001940       ??_C@_06ICOKPHJ@SXDBEX?$AA@ 1007b940     xlstool.obj
 0002:00001948       ??_C@_0BK@FBJABKPN@PivotTable?5Formula?5Record?$AA@ 1007b948     xlstool.obj
 0002:00001964       ??_C@_09FHHJEHCC@SXFORMULA?$AA@ 1007b964     xlstool.obj
 0002:00001970       ??_C@_0CA@JGCGFBAL@Extended?5PivotTable?5View?5Fields?$AA@ 1007b970     xlstool.obj
 0002:00001990       ??_C@_06DHGFDEEH@SXVDEX?$AA@ 1007b990     xlstool.obj
 0002:00001998       ??_C@_0BN@DAOPNBMK@Extended?5Shared?5String?5Table?$AA@ 1007b998     xlstool.obj
 0002:000019b8       ??_C@_06DAHLDBDL@EXTSST?$AA@ 1007b9b8     xlstool.obj
 0002:000019c0       ??_C@_0CA@IMCGOIPL@Cell?5Value?0?5String?5Constant?1SST?$AA@ 1007b9c0     xlstool.obj
 0002:000019e0       ??_C@_08LMPADLAD@LABELSST?$AA@ 1007b9e0     xlstool.obj
 0002:000019ec       ??_C@_0BE@HEBIOEHI@Shared?5String?5Table?$AA@ 1007b9ec     xlstool.obj
 0002:00001a00       ??_C@_03LHCOIIBG@SST?$AA@  1007ba00     xlstool.obj
 0002:00001a04       ??_C@_0BJ@HHNHFIAD@PivotTable?5Format?5Record?$AA@ 1007ba04     xlstool.obj
 0002:00001a20       ??_C@_08IJBNOFIH@SXFORMAT?$AA@ 1007ba20     xlstool.obj
 0002:00001a2c       ??_C@_0BN@MOCOCIMO@PivotTable?5Parsed?5Expression?$AA@ 1007ba2c     xlstool.obj
 0002:00001a4c       ??_C@_06LOFMHONI@SXFMLA?$AA@ 1007ba4c     xlstool.obj
 0002:00001a54       ??_C@_0BF@KCEHDELL@PivotTable?5Name?5Pair?$AA@ 1007ba54     xlstool.obj
 0002:00001a6c       ??_C@_06HMAOCADL@SXPAIR?$AA@ 1007ba6c     xlstool.obj
 0002:00001a74       ??_C@_0CB@GBFGJLBN@PivotTable?5Selection?5Information@ 1007ba74     xlstool.obj
 0002:00001a98       ??_C@_08EIAKAOK@SXSELECT?$AA@ 1007ba98     xlstool.obj
 0002:00001aa4       ??_C@_0BA@BCFOGJME@PivotTable?5Name?$AA@ 1007baa4     xlstool.obj
 0002:00001ab4       ??_C@_06KBFECFJC@SXNAME?$AA@ 1007bab4     xlstool.obj
 0002:00001abc       ??_C@_0BH@IILJLEAB@PivotTable?5Rule?5Filter?$AA@ 1007babc     xlstool.obj
 0002:00001ad4       ??_C@_06GILAPJL@SXFILT?$AA@ 1007bad4     xlstool.obj
 0002:00001adc       ??_C@_0CF@HDGAOEBG@PivotTable?5View?5Extended?5Informa@ 1007badc     xlstool.obj
 0002:00001b04       ??_C@_04EMOEACMD@SXEX?$AA@ 1007bb04     xlstool.obj
 0002:00001b0c       ??_C@_0BF@ECCCAGMN@PivotTable?5Rule?5Data?$AA@ 1007bb0c     xlstool.obj
 0002:00001b24       ??_C@_06NKPNPFOO@SXRULE?$AA@ 1007bb24     xlstool.obj
 0002:00001b2c       ??_C@_0CD@OLENPAAJ@Microsoft?5Office?5Drawing?5Selecti@ 1007bb2c     xlstool.obj
 0002:00001b50       ??_C@_0BE@JHHNICAI@MSODRAWINGSELECTION?$AA@ 1007bb50     xlstool.obj
 0002:00001b64       ??_C@_0BJ@JDOHKHOD@Microsoft?5Office?5Drawing?$AA@ 1007bb64     xlstool.obj
 0002:00001b80       ??_C@_0L@KOCGHLEC@MSODRAWING?$AA@ 1007bb80     xlstool.obj
 0002:00001b8c       ??_C@_0BP@KGJINBHN@Microsoft?5Office?5Drawing?5Group?$AA@ 1007bb8c     xlstool.obj
 0002:00001bac       ??_C@_0BA@NBHMNIJK@MSODRAWINGGROUP?$AA@ 1007bbac     xlstool.obj
 0002:00001bbc       ??_C@_0CB@FPBMADKA@Sheet?5Tab?5ID?5of?5Conflict?5History@ 1007bbbc     xlstool.obj
 0002:00001be0       ??_C@_09ELICDJAE@TABIDCONF?$AA@ 1007bbe0     xlstool.obj
 0002:00001bec       ??_C@_0L@GMAFCLLA@Cells?5span?$AA@ 1007bbec     xlstool.obj
 0002:00001bf8       ??_C@_05GMONBJFL@CSPAN?$AA@ 1007bbf8     xlstool.obj
 0002:00001c00       ??_C@_0M@GPAPMOCJ@View?5Source?$AA@ 1007bc00     xlstool.obj
 0002:00001c0c       ??_C@_04LBHAMGCB@SXVS?$AA@ 1007bc0c     xlstool.obj
 0002:00001c14       ??_C@_0BO@DNFGNONP@End?5of?5User?5Interface?5Records?$AA@ 1007bc14     xlstool.obj
 0002:00001c34       ??_C@_0N@KJBLNFPK@INTERFACEEND?$AA@ 1007bc34     xlstool.obj
 0002:00001c44       ??_C@_0CE@POHKOLGI@Beginning?5of?5User?5Interface?5Reco@ 1007bc44     xlstool.obj
 0002:00001c68       ??_C@_0N@EKHODNCG@INTERFACEHDR?$AA@ 1007bc68     xlstool.obj
 0002:00001c78       ??_C@_0BA@BGJBIHEA@Extended?5Format?$AA@ 1007bc78     xlstool.obj
 0002:00001c88       ??_C@_02MEDCLBGG@XF?$AA@   1007bc88     xlstool.obj
 0002:00001c8c       ??_C@_0CI@NDMFHPMC@Description?5String?5for?5Chart?5Aut@ 1007bc8c     xlstool.obj
 0002:00001cb4       ??_C@_06DDKAHEEC@UDDESC?$AA@ 1007bcb4     xlstool.obj
 0002:00001cbc       ??_C@_0BD@LDIKAJKJ@Size?5of?5OLE?5Object?$AA@ 1007bcbc     xlstool.obj
 0002:00001cd0       ??_C@_07MDNEMGIP@OLESIZE?$AA@ 1007bcd0     xlstool.obj
 0002:00001cd8       ??_C@_0BE@NNPIJIHK@Scenario?5Protection?$AA@ 1007bcd8     xlstool.obj
 0002:00001cec       ??_C@_0M@DMJGADNP@SCENPROTECT?$AA@ 1007bcec     xlstool.obj
 0002:00001cf8       ??_C@_0CN@MMCFABNL@Query?5Parameters?9External?5Source@ 1007bcf8     xlstool.obj
 0002:00001d28       ??_C@_0P@NJHFKGND@PARAMQRY?9SXEXT?$AA@ 1007bd28     xlstool.obj
 0002:00001d38       ??_C@_0BF@PIAIHKBM@Workbook?5Option?5Flag?$AA@ 1007bd38     xlstool.obj
 0002:00001d50       ??_C@_08ILNGGBI@BOOKBOOL?$AA@ 1007bd50     xlstool.obj
 0002:00001d5c       ??_C@_0P@DKPGOKAP@Stream?5Offsets?$AA@ 1007bd5c     xlstool.obj
 0002:00001d6c       ??_C@_06GJCCELH@DBCELL?$AA@ 1007bd6c     xlstool.obj
 0002:00001d74       ??_C@_0BP@KFDECKG@Cell?5with?5Character?5Formatting?$AA@ 1007bd74     xlstool.obj
 0002:00001d94       ??_C@_07GJAPJPPC@RSTRING?$AA@ 1007bd94     xlstool.obj
 0002:00001d9c       ??_C@_09DNIEDBMH@Stream?5ID?$AA@ 1007bd9c     xlstool.obj
 0002:00001da8       ??_C@_07CDLAMBCG@SXIDSTM?$AA@ 1007bda8     xlstool.obj
 0002:00001db0       ??_C@_0BF@IOIBILBJ@Visual?5Basic?5Project?$AA@ 1007bdb0     xlstool.obj
 0002:00001dc8       ??_C@_06LKAHOLOG@OBPROJ?$AA@ 1007bdc8     xlstool.obj
 0002:00001dd0       ??_C@_0BC@NBLKJAJG@Page?5Item?5Indexes?$AA@ 1007bdd0     xlstool.obj
 0002:00001de4       ??_C@_06LPHJFHPO@SXTBPG?$AA@ 1007bde4     xlstool.obj
 0002:00001dec       ??_C@_0BF@OGNMNNEA@Page?5Item?5Name?5Count?$AA@ 1007bdec     xlstool.obj
 0002:00001e04       ??_C@_0L@KAGLLOIB@SXTBRGIITM?$AA@ 1007be04     xlstool.obj
 0002:00001e10       ??_C@_0CD@MICIJHFA@Multiple?5Consolidation?5Source?5In@ 1007be10     xlstool.obj
 0002:00001e34       ??_C@_05KHPJGBFN@SXTBL?$AA@ 1007be34     xlstool.obj
 0002:00001e3c       ??_C@_06ENNEIMBA@String?$AA@ 1007be3c     xlstool.obj
 0002:00001e44       ??_C@_08DADLDFEO@SXSTRING?$AA@ 1007be44     xlstool.obj
 0002:00001e50       ??_C@_0BG@GNKNFHKE@PivotTable?5Cache?5Data?$AA@ 1007be50     xlstool.obj
 0002:00001e68       ??_C@_04PNALJCCP@SXDB?$AA@ 1007be68     xlstool.obj
 0002:00001e70       ??_C@_09ONLKGJGL@Data?5Item?$AA@ 1007be70     xlstool.obj
 0002:00001e7c       ??_C@_04BOPPELOE@SXDI?$AA@ 1007be7c     xlstool.obj
 0002:00001e84       ??_C@_0O@DHEDFKLG@Menu?5Deletion?$AA@ 1007be84     xlstool.obj
 0002:00001e94       ??_C@_07OIMCEBGE@DELMENU?$AA@ 1007be94     xlstool.obj
 0002:00001e9c       ??_C@_0O@PFFDJBHL@Menu?5Addition?$AA@ 1007be9c     xlstool.obj
 0002:00001eac       ??_C@_07OKAGMGNJ@ADDMENU?$AA@ 1007beac     xlstool.obj
 0002:00001eb4       ??_C@_0CD@EKGJLPIE@ADDMENU?1DELMENU?5Record?5Group?5Cou@ 1007beb4     xlstool.obj
 0002:00001ed8       ??_C@_03FOBBLAAH@MMS?$AA@  1007bed8     xlstool.obj
 0002:00001edc       ??_C@_0BF@LMOHNADE@Multiple?5Blank?5Cells?$AA@ 1007bedc     xlstool.obj
 0002:00001ef4       ??_C@_08DNPEPKNN@MULBLANK?$AA@ 1007bef4     xlstool.obj
 0002:00001f00       ??_C@_0BC@IDLNAGGK@Multiple?5RK?5Cells?$AA@ 1007bf00     xlstool.obj
 0002:00001f14       ??_C@_05KAHPIMMA@MULRK?$AA@ 1007bf14     xlstool.obj
 0002:00001f1c       ??_C@_0P@LMKIDDHD@Shared?5Formula?$AA@ 1007bf1c     xlstool.obj
 0002:00001f2c       ??_C@_07FJPJGBLI@SHRFMLA?$AA@ 1007bf2c     xlstool.obj
 0002:00001f34       ??_C@_0P@CDJNODAM@Recipient?5Name?$AA@ 1007bf34     xlstool.obj
 0002:00001f44       ??_C@_09HOLJAGEE@RECIPNAME?$AA@ 1007bf44     xlstool.obj
 0002:00001f50       ??_C@_0BJ@MIECCOEA@Routing?5Slip?5Information?$AA@ 1007bf50     xlstool.obj
 0002:00001f6c       ??_C@_08JOFLKCCH@DOCROUTE?$AA@ 1007bf6c     xlstool.obj
 0002:00001f78       ??_C@_09MFIEFKCC@Page?5Item?$AA@ 1007bf78     xlstool.obj
 0002:00001f84       ??_C@_04FNAEAEI@SXPI?$AA@  1007bf84     xlstool.obj
 0002:00001f8c       ??_C@_0BA@BDDHIAEE@Line?5Item?5Array?$AA@ 1007bf8c     xlstool.obj
 0002:00001f9c       ??_C@_04BAOMBKFM@SXLI?$AA@ 1007bf9c     xlstool.obj
 0002:00001fa4       ??_C@_0BF@IBHIAPIO@Row?1Column?5Field?5IDs?$AA@ 1007bfa4     xlstool.obj
 0002:00001fbc       ??_C@_05NGHMGPLL@SXIVD?$AA@ 1007bfbc     xlstool.obj
 0002:00001fc4       ??_C@_09MBCGACOH@View?5Item?$AA@ 1007bfc4     xlstool.obj
 0002:00001fd0       ??_C@_04BFNDMPK@SXVI?$AA@  1007bfd0     xlstool.obj
 0002:00001fd8       ??_C@_0M@EFEBIKCB@View?5Fields?$AA@ 1007bfd8     xlstool.obj
 0002:00001fe4       ??_C@_04LEPDECLH@SXVD?$AA@ 1007bfe4     xlstool.obj
 0002:00001fec       ??_C@_0BA@NMHBLMLJ@View?5Definition?$AA@ 1007bfec     xlstool.obj
 0002:00001ffc       ??_C@_06ECJHPAFF@SXVIEW?$AA@ 1007bffc     xlstool.obj
 0002:00002004       ??_C@_0O@CADFIKPK@Scenario?5Data?$AA@ 1007c004     xlstool.obj
 0002:00002014       ??_C@_08NKGHDBHL@SCENARIO?$AA@ 1007c014     xlstool.obj
 0002:00002020       ??_C@_0BF@JIBMBFOL@Scenario?5Output?5Data?$AA@ 1007c020     xlstool.obj
 0002:00002038       ??_C@_07PKBNMDDM@SCENMAN?$AA@ 1007c038     xlstool.obj
 0002:00002040       ??_C@_0BK@HOGLFCFN@Global?5Column?9Width?5Flags?$AA@ 1007c040     xlstool.obj
 0002:0000205c       ??_C@_03FPFOLIGN@GCW?$AA@  1007c05c     xlstool.obj
 0002:00002060       ??_C@_0CC@OLPJONIL@Polygon?5Object?5Vertex?5Coordinate@ 1007c060     xlstool.obj
 0002:00002084       ??_C@_09HDNPCNBP@COORDLIST?$AA@ 1007c084     xlstool.obj
 0002:00002090       ??_C@_0L@PPMHOBLF@Page?5Setup?$AA@ 1007c090     xlstool.obj
 0002:0000209c       ??_C@_05MAJHNKMG@SETUP?$AA@ 1007c09c     xlstool.obj
 0002:000020a4       ??_C@_0BK@BOFDFAOI@Window?5Zoom?5Magnification?$AA@ 1007c0a4     xlstool.obj
 0002:000020c0       ??_C@_03CJBDLDDP@SCL?$AA@  1007c0c0     xlstool.obj
 0002:000020c4       ??_C@_0BA@LDNNGDH@AutoFilter?5Data?$AA@ 1007c0c4     xlstool.obj
 0002:000020d4       ??_C@_0L@CLLMEDKM@AUTOFILTER?$AA@ 1007c0d4     xlstool.obj
 0002:000020e0       ??_C@_0BG@KKJLAHJN@Drop?9Down?5Arrow?5Count?$AA@ 1007c0e0     xlstool.obj
 0002:000020f8       ??_C@_0P@LMHDDKFO@AUTOFILTERINFO?$AA@ 1007c0f8     xlstool.obj
 0002:00002108       ??_C@_0BO@FOJGNDJA@Built?9in?5Function?5Group?5Count?$AA@ 1007c108     xlstool.obj
 0002:00002128       ??_C@_0N@ECHEGBGP@FNGROUPCOUNT?$AA@ 1007c128     xlstool.obj
 0002:00002138       ??_C@_0BN@JJNICPAL@Sheet?5Contains?5Filtered?5List?$AA@ 1007c138     xlstool.obj
 0002:00002158       ??_C@_0L@OPBMAFBH@FILTERMODE?$AA@ 1007c158     xlstool.obj
 0002:00002164       ??_C@_0BE@GNOHNEDP@Function?5Group?5Name?$AA@ 1007c164     xlstool.obj
 0002:00002178       ??_C@_0M@EDHBAOEF@FNGROUPNAME?$AA@ 1007c178     xlstool.obj
 0002:00002184       ??_C@_0CD@BENNHFGO@Sheet?5Was?5Printed?5Using?5LINE?4PRI@ 1007c184     xlstool.obj
 0002:000021a8       ??_C@_03OLEINGAA@LPR?$AA@  1007c1a8     xlstool.obj
 0002:000021ac       ??_C@_0BG@LPJPDLLC@Standard?5Column?5Width?$AA@ 1007c1ac     xlstool.obj
 0002:000021c4       ??_C@_0O@GJBBGHNM@STANDARDWIDTH?$AA@ 1007c1c4     xlstool.obj
 0002:000021d4       ??_C@_0L@JNDMKNAL@Sound?5Note?$AA@ 1007c1d4     xlstool.obj
 0002:000021e0       ??_C@_05MEGDOMG@SOUND?$AA@ 1007c1e0     xlstool.obj
 0002:000021e8       ??_C@_0BI@COCINNBI@Named?5Graph?5Information?$AA@ 1007c1e8     xlstool.obj
 0002:00002200       ??_C@_08OICGLOKE@LHNGRAPH?$AA@ 1007c200     xlstool.obj
 0002:0000220c       ??_C@_0CB@HIGDDHHF@?4WK?$DP?5File?5Conversion?5Information@ 1007c20c     xlstool.obj
 0002:00002230       ??_C@_08BHPOLLHG@LHRECORD?$AA@ 1007c230     xlstool.obj
 0002:0000223c       ??_C@_0BJ@NMNKOKDA@Color?5Palette?5Definition?$AA@ 1007c23c     xlstool.obj
 0002:00002258       ??_C@_07GHNKBFGK@PALETTE?$AA@ 1007c258     xlstool.obj
 0002:00002260       ??_C@_0L@JPKCEGAC@Subscriber?$AA@ 1007c260     xlstool.obj
 0002:0000226c       ??_C@_03KPDLEBHD@SUB?$AA@  1007c26c     xlstool.obj
 0002:00002270       ??_C@_0BA@KOOGCIHO@Sorting?5Options?$AA@ 1007c270     xlstool.obj
 0002:00002280       ??_C@_04DEPGJHBM@SORT?$AA@ 1007c280     xlstool.obj
 0002:00002288       ??_C@_0BH@PLDAHLCG@Object?5Display?5Options?$AA@ 1007c288     xlstool.obj
 0002:000022a0       ??_C@_07PBDOAGN@HIDEOBJ?$AA@ 1007c2a0     xlstool.obj
 0002:000022a8       ??_C@_0CE@PLKFDKOL@Default?5Country?5and?5WIN?4INI?5Coun@ 1007c2a8     xlstool.obj
 0002:000022cc       ??_C@_07HECCBLFC@COUNTRY?$AA@ 1007c2cc     xlstool.obj
 0002:000022d4       ??_C@_09PNIDBPNC@Publisher?$AA@ 1007c2d4     xlstool.obj
 0002:000022e0       ??_C@_03LNIOOOJN@PUB?$AA@  1007c2e0     xlstool.obj
 0002:000022e4       ??_C@_0BA@FPLEKHGK@Edition?5Globals?$AA@ 1007c2e4     xlstool.obj
 0002:000022f4       ??_C@_03LKNKHEDC@EDG?$AA@  1007c2f4     xlstool.obj
 0002:000022f8       ??_C@_0BM@CHMJICNB@Workbook?5Is?5an?5Add?9in?5Macro?$AA@ 1007c2f8     xlstool.obj
 0002:00002314       ??_C@_05CCINGCLC@ADDIN?$AA@ 1007c314     xlstool.obj
 0002:0000231c       ??_C@_0BM@NHLAGNGI@Workbook?5Is?5Write?9Protected?$AA@ 1007c31c     xlstool.obj
 0002:00002338       ??_C@_09FJMCLGLK@WRITEPROT?$AA@ 1007c338     xlstool.obj
 0002:00002344       ??_C@_0BC@MENLFMPC@Sheet?5Information?$AA@ 1007c344     xlstool.obj
 0002:00002358       ??_C@_0L@CHKOCBDJ@BOUNDSHEET?$AA@ 1007c358     xlstool.obj
 0002:00002364       ??_C@_0CA@MEGLPMBK@Center?5Between?5Vertical?5Margins?$AA@ 1007c364     xlstool.obj
 0002:00002384       ??_C@_07HOJCCAMM@VCENTER?$AA@ 1007c384     xlstool.obj
 0002:0000238c       ??_C@_0CC@HAAMBINM@Center?5Between?5Horizontal?5Margin@ 1007c38c     xlstool.obj
 0002:000023b0       ??_C@_07BHKDADNF@HCENTER?$AA@ 1007c3b0     xlstool.obj
 0002:000023b8       ??_C@_0CB@MOHOIANN@State?5Change?5of?5Gridlines?5Option@ 1007c3b8     xlstool.obj
 0002:000023dc       ??_C@_07PJNFMBOG@GRIDSET?$AA@ 1007c3dc     xlstool.obj
 0002:000023e4       ??_C@_0CB@EECHJNEB@Additional?5Workspace?5Information@ 1007c3e4     xlstool.obj
 0002:00002408       ??_C@_06MILFAEFH@WSBOOL?$AA@ 1007c408     xlstool.obj
 0002:00002410       ??_C@_0BP@LHDCPFBC@Size?5of?5Row?5and?5Column?5Gutters?$AA@ 1007c410     xlstool.obj
 0002:00002430       ??_C@_04NFPOPLNA@GUTS?$AA@ 1007c430     xlstool.obj
 0002:00002438       ??_C@_0L@FDIHEIAN@Image?5Data?$AA@ 1007c438     xlstool.obj
 0002:00002444       ??_C@_06MMKDAGA@IMDATA?$AA@ 1007c444     xlstool.obj
 0002:0000244c       ??_C@_0BO@LPPDCKPI@Column?5Formatting?5Information?$AA@ 1007c44c     xlstool.obj
 0002:0000246c       ??_C@_07NKMIJNJB@COLINFO?$AA@ 1007c46c     xlstool.obj
 0002:00002474       ??_C@_0BG@OEMHPNPG@Objects?5Are?5Protected?$AA@ 1007c474     xlstool.obj
 0002:0000248c       ??_C@_0L@NCALCEBC@OBJPROTECT?$AA@ 1007c48c     xlstool.obj
 0002:00002498       ??_C@_0BH@MOFCLFE@Workbook?5Is?5a?5Template?$AA@ 1007c498     xlstool.obj
 0002:000024b0       ??_C@_08CGHHJMNA@TEMPLATE?$AA@ 1007c4b0     xlstool.obj
 0002:000024bc       ??_C@_0BI@LOBGLAAM@Recalculate?5Before?5Save?$AA@ 1007c4bc     xlstool.obj
 0002:000024d4       ??_C@_0L@BBJJHLDP@SAVERECALC?$AA@ 1007c4d4     xlstool.obj
 0002:000024e0       ??_C@_0BF@ECFCHJAO@Recalculation?5Status?$AA@ 1007c4e0     xlstool.obj
 0002:000024f8       ??_C@_08FKCFAOCL@UNCALCED?$AA@ 1007c4f8     xlstool.obj
 0002:00002504       ??_C@_0BL@HINCONPP@Describes?5a?5Graphic?5Object?$AA@ 1007c504     xlstool.obj
 0002:00002520       ??_C@_03GEEEJGKJ@OBJ?$AA@  1007c520     xlstool.obj
 0002:00002524       ??_C@_0BH@GHPLOPBH@Write?5Access?5User?5Name?$AA@ 1007c524     xlstool.obj
 0002:0000253c       ??_C@_0M@OHDCAMII@WRITEACCESS?$AA@ 1007c53c     xlstool.obj
 0002:00002548       ??_C@_0BJ@IKDEJCF@File?9Sharing?5Information?$AA@ 1007c548     xlstool.obj
 0002:00002564       ??_C@_0M@OPEIEJGK@FILESHARING?$AA@ 1007c564     xlstool.obj
 0002:00002570       ??_C@_0BF@PMLKJHIP@Nonresident?5Operands?$AA@ 1007c570     xlstool.obj
 0002:00002588       ??_C@_03FGNIEPGF@CRN?$AA@  1007c588     xlstool.obj
 0002:0000258c       ??_C@_0BB@CPDIBOKF@CRN?5Record?5Count?$AA@ 1007c58c     xlstool.obj
 0002:000025a0       ??_C@_03HMAJKMGH@XCT?$AA@  1007c5a0     xlstool.obj
 0002:000025a4       ??_C@_0BK@CJCNCOLA@Default?5Width?5for?5Columns?$AA@ 1007c5a4     xlstool.obj
 0002:000025c0       ??_C@_0M@BEPGAJKH@DEFCOLWIDTH?$AA@ 1007c5c0     xlstool.obj
 0002:000025cc       ??_C@_0CE@GHCJMDPM@Data?5Consolidation?5Named?5Referen@ 1007c5cc     xlstool.obj
 0002:000025f0       ??_C@_08ILKMGOHL@DCONNAME?$AA@ 1007c5f0     xlstool.obj
 0002:000025fc       ??_C@_0BO@FAMBKCOJ@Data?5Consolidation?5References?$AA@ 1007c5fc     xlstool.obj
 0002:0000261c       ??_C@_07OKFCLNHF@DCONREF?$AA@ 1007c61c     xlstool.obj
 0002:00002624       ??_C@_0BP@KGOOMLPD@Data?5Consolidation?5Information?$AA@ 1007c624     xlstool.obj
 0002:00002644       ??_C@_04IDDKJMO@DCON?$AA@  1007c644     xlstool.obj
 0002:0000264c       ??_C@_0CC@POJCMGJM@Environment?9Specific?5Print?5Recor@ 1007c64c     xlstool.obj
 0002:00002670       ??_C@_03PNKAFFHC@PLS?$AA@  1007c670     xlstool.obj
 0002:00002674       ??_C@_0BC@PGIFPKOG@Default?5Code?5Page?$AA@ 1007c674     xlstool.obj
 0002:00002688       ??_C@_08COFBOPB@CODEPAGE?$AA@ 1007c688     xlstool.obj
 0002:00002694       ??_C@_0CD@LKKAKHOC@Number?5of?5Panes?5and?5Their?5Positi@ 1007c694     xlstool.obj
 0002:000026b8       ??_C@_04NFGMODPL@PANE?$AA@ 1007c6b8     xlstool.obj
 0002:000026c0       ??_C@_0CA@FBCJEFHH@Save?5Backup?5Version?5of?5the?5File?$AA@ 1007c6c0     xlstool.obj
 0002:000026e0       ??_C@_06PGIJNBLC@BACKUP?$AA@ 1007c6e0     xlstool.obj
 0002:000026e8       ??_C@_0BD@BOOOFJEK@Window?5Information?$AA@ 1007c6e8     xlstool.obj
 0002:000026fc       ??_C@_07OAFFAIJK@WINDOW1?$AA@ 1007c6fc     xlstool.obj
 0002:00002704       ??_C@_0BH@MHADBKD@Continues?5Long?5Records?$AA@ 1007c704     xlstool.obj
 0002:0000271c       ??_C@_08EECOACDK@CONTINUE?$AA@ 1007c71c     xlstool.obj
 0002:00002728       ??_C@_0BB@PHLPIPJJ@Font?5Description?$AA@ 1007c728     xlstool.obj
 0002:0000273c       ??_C@_04IJMKNFPK@FONT?$AA@ 1007c73c     xlstool.obj
 0002:00002744       ??_C@_0BL@PGFCJACG@File?5Is?5Password?9Protected?$AA@ 1007c744     xlstool.obj
 0002:00002760       ??_C@_08LKEFKCCF@FILEPASS?$AA@ 1007c760     xlstool.obj
 0002:0000276c       ??_C@_0BF@NDMBCKGD@Print?5Gridlines?5Flag?$AA@ 1007c76c     xlstool.obj
 0002:00002784       ??_C@_0P@FMNMCFAJ@PRINTGRIDLINES?$AA@ 1007c784     xlstool.obj
 0002:00002794       ??_C@_0BI@NKJEHJHL@Print?5Row?1Column?5Labels?$AA@ 1007c794     xlstool.obj
 0002:000027ac       ??_C@_0N@PMNBLCBM@PRINTHEADERS?$AA@ 1007c7ac     xlstool.obj
 0002:000027bc       ??_C@_0BK@PCHGMHFE@Bottom?5Margin?5Measurement?$AA@ 1007c7bc     xlstool.obj
 0002:000027d8       ??_C@_0N@BAPPMDPJ@BOTTOMMARGIN?$AA@ 1007c7d8     xlstool.obj
 0002:000027e8       ??_C@_0BH@DIEFLONO@Top?5Margin?5Measurement?$AA@ 1007c7e8     xlstool.obj
 0002:00002800       ??_C@_09EMPOGLDA@TOPMARGIN?$AA@ 1007c800     xlstool.obj
 0002:0000280c       ??_C@_0BJ@FJAGNKJL@Right?5Margin?5Measurement?$AA@ 1007c80c     xlstool.obj
 0002:00002828       ??_C@_0M@IFFGHPAI@RIGHTMARGIN?$AA@ 1007c828     xlstool.obj
 0002:00002834       ??_C@_0BI@FAIFCOJF@Left?5Margin?5Measurement?$AA@ 1007c834     xlstool.obj
 0002:0000284c       ??_C@_0L@PICEGLPF@LEFTMARGIN?$AA@ 1007c84c     xlstool.obj
 0002:00002858       ??_C@_0BB@CBOLFMMO@1904?5Date?5System?$AA@ 1007c858     xlstool.obj
 0002:0000286c       ??_C@_04LHPODIJI@1904?$AA@ 1007c86c     xlstool.obj
 0002:00002874       ??_C@_0BC@JFKGCGKO@Current?5Selection?$AA@ 1007c874     xlstool.obj
 0002:00002888       ??_C@_09FCNMPPO@SELECTION?$AA@ 1007c888     xlstool.obj
 0002:00002894       ??_C@_0BP@OLBKMJIP@Comment?5Associated?5with?5a?5Cell?$AA@ 1007c894     xlstool.obj
 0002:000028b4       ??_C@_04PLNCJLIN@NOTE?$AA@ 1007c8b4     xlstool.obj
 0002:000028bc       ??_C@_0BJ@DEIEHEOP@Explicit?5Row?5Page?5Breaks?$AA@ 1007c8bc     xlstool.obj
 0002:000028d8       ??_C@_0BF@MEHFGKNN@HORIZONTALPAGEBREAKS?$AA@ 1007c8d8     xlstool.obj
 0002:000028f0       ??_C@_0BM@BMECJPIB@Explicit?5Column?5Page?5Breaks?$AA@ 1007c8f0     xlstool.obj
 0002:0000290c       ??_C@_0BD@PAAOEFGK@VERTICALPAGEBREAKS?$AA@ 1007c90c     xlstool.obj
 0002:00002920       ??_C@_0BE@LNENCDOK@?5?$CIbiffview?5guessed?$CJ?$AA@ 1007c920     xlstool.obj
 0002:00002934       ??_C@_0P@NMKMMDHH@?$DPWINDOWPROTECT?$AA@ 1007c934     xlstool.obj
 0002:00002944       ??_C@_0BD@LHBAKOMG@External?5Reference?$AA@ 1007c944     xlstool.obj
 0002:00002958       ??_C@_0M@CPIPEJFB@EXTERNSHEET?$AA@ 1007c958     xlstool.obj
 0002:00002964       ??_C@_0BO@DNMMENKF@Number?5of?5External?5References?$AA@ 1007c964     xlstool.obj
 0002:00002984       ??_C@_0M@MCDFCPKE@EXTERNCOUNT?$AA@ 1007c984     xlstool.obj
 0002:00002990       ??_C@_0BK@FBEDLBNB@Print?5Footer?5on?5Each?5Page?$AA@ 1007c990     xlstool.obj
 0002:000029ac       ??_C@_06NLFGPPOL@FOOTER?$AA@ 1007c9ac     xlstool.obj
 0002:000029b4       ??_C@_0BK@DLNCGKDG@Print?5Header?5on?5Each?5Page?$AA@ 1007c9b4     xlstool.obj
 0002:000029d0       ??_C@_06MFNLEOCO@HEADER?$AA@ 1007c9d0     xlstool.obj
 0002:000029d8       ??_C@_0BE@BCNHAOOL@Protection?5Password?$AA@ 1007c9d8     xlstool.obj
 0002:000029ec       ??_C@_08KENNMKEI@PASSWORD?$AA@ 1007c9ec     xlstool.obj
 0002:000029f8       ??_C@_0BA@LDGCPKLO@Protection?5Flag?$AA@ 1007c9f8     xlstool.obj
 0002:00002a08       ??_C@_07EIONPJLK@PROTECT?$AA@ 1007ca08     xlstool.obj
 0002:00002a10       ??_C@_0P@GDGPIGLN@Iteration?5Mode?$AA@ 1007ca10     xlstool.obj
 0002:00002a20       ??_C@_09HOOEJAIN@ITERATION?$AA@ 1007ca20     xlstool.obj
 0002:00002a2c       ??_C@_0BE@KHGLPOKH@Iteration?5Increment?$AA@ 1007ca2c     xlstool.obj
 0002:00002a40       ??_C@_05BJPCNOLC@DELTA?$AA@ 1007ca40     xlstool.obj
 0002:00002a48       ??_C@_0P@JLPGOML@Reference?5Mode?$AA@ 1007ca48     xlstool.obj
 0002:00002a58       ??_C@_07NLGFCNEN@REFMODE?$AA@ 1007ca58     xlstool.obj
 0002:00002a60       ??_C@_09DGDDLEAF@Precision?$AA@ 1007ca60     xlstool.obj
 0002:00002a6c       ??_C@_09EJJPIKCC@PRECISION?$AA@ 1007ca6c     xlstool.obj
 0002:00002a78       ??_C@_0BB@NLFNIAA@Calculation?5Mode?$AA@ 1007ca78     xlstool.obj
 0002:00002a8c       ??_C@_08IIDADLOA@CALCMODE?$AA@ 1007ca8c     xlstool.obj
 0002:00002a98       ??_C@_0BA@CABKKCCO@Iteration?5Count?$AA@ 1007ca98     xlstool.obj
 0002:00002aa8       ??_C@_09KAKPPEHI@CALCCOUNT?$AA@ 1007caa8     xlstool.obj
 0002:00002ab4       ??_C@_0M@FKGOBENP@End?5of?5File?$AA@ 1007cab4     xlstool.obj
 0002:00002ac0       ??_C@_03KPJEKKJC@EOF?$AA@  1007cac0     xlstool.obj
 0002:00002ac4       ??_C@_0BC@MLBJLLNP@Beginning?5of?5File?$AA@ 1007cac4     xlstool.obj
 0002:00002ad8       ??_C@_09PGOCCMEJ@BOF?9BIFF2?$AA@ 1007cad8     xlstool.obj
 0002:00002ae4       ??_C@_0N@IHFHONPO@Cell?5Formula?$AA@ 1007cae4     xlstool.obj
 0002:00002af4       ??_C@_07EKHICOBI@FORMULA?$AA@ 1007caf4     xlstool.obj
 0002:00002afc       ??_C@_06DHGOCNPL@Unknow?$AA@ 1007cafc     xlstool.obj
 0002:00002be8       ??_C@_02GMLFBBN@wb?$AA@    1007cbe8     xlstool.obj
 0002:00002bec       ??_C@_0M@NHJCAKFC@xlslib?3?5?$CFs?6?$AA@ 1007cbec     xlstool.obj
 0002:00002bf8       ??_C@_08NBDJLNFA@UTF?916LE?$AA@ 1007cbf8     xlstool.obj
 0002:00002c04       ??_C@_0BJ@BMFAGEFF@BIFF4W?5Workbook?5globals?6?$AA@ 1007cc04     xlstool.obj
 0002:00002c20       ??_C@_0BD@JHININMK@BIFF4?5Macro?5sheet?6?$AA@ 1007cc20     xlstool.obj
 0002:00002c34       ??_C@_06DPKENMLO@Chart?6?$AA@ 1007cc34     xlstool.obj
 0002:00002c3c       ??_C@_0L@HLNPBOHM@Worksheet?6?$AA@ 1007cc3c     xlstool.obj
 0002:00002c48       ??_C@_0BF@NGAOKHGL@Visual?5Basic?5module?6?$AA@ 1007cc48     xlstool.obj
 0002:00002c60       ??_C@_0DA@HHHLHLBD@?9?9?9?9?9?9?9?9?9?9?9?9?9?9?9?9?9?9?9?9?9?9?9?9?9?9?9?9?9?9?9?9@ 1007cc60     xlstool.obj
 0002:00002c90       ??_C@_0BC@EAKPEBCJ@Workbook?5globals?6?$AA@ 1007cc90     xlstool.obj
 0002:00002ca4       ??_C@_0BA@MKHIBCHP@?5?5?5?5type?3?5?$CF?44X?5?$AA@ 1007cca4     xlstool.obj
 0002:00002cb4       ??_C@_0O@NHININF@codepage?3?5?$CFi?6?$AA@ 1007ccb4     xlstool.obj
 0002:00002cc4       ??_C@_0O@CCNPAHGG@?5?5is5ver?3?5?$CFi?6?$AA@ 1007ccc4     xlstool.obj
 0002:00002cd4       ??_C@_08NPLBMLKA@BookInfo?$AA@ 1007ccd4     xlstool.obj
 0002:00002ce0       ??_C@_0N@NFIAAOOP@?5?5?5Size?3?5?$CFi?6?$AA@ 1007cce0     xlstool.obj
 0002:00002cf0       ??_C@_0BI@NEKFOAN@?5?5?5?5?5ID?3?5?$CF?44Xh?5?$CFs?5?$CI?$CFs?$CJ?6?$AA@ 1007ccf0     xlstool.obj
 0002:00002d08       ??_C@_03DCEDJCCL@BOF?$AA@  1007cd08     xlstool.obj
 0002:00002d0c       ??_C@_0BA@LPPHNKEK@?5?5flags?3?5?$CF?44Xh?6?$AA@ 1007cd0c     xlstool.obj
 0002:00002d1c       ??_C@_0O@GGOOLFHF@?5?5?5?5Pos?3?5?$CFXh?6?$AA@ 1007cd1c     xlstool.obj
 0002:00002d2c       ??_C@_0BH@FPIMGIGN@85?3?5Visual?5Basic?5sheet?$AA@ 1007cd2c     xlstool.obj
 0002:00002d44       ??_C@_0BA@CDIOGFPL@85?3?5Chart?5sheet?$AA@ 1007cd44     xlstool.obj
 0002:00002d54       ??_C@_0CE@DHNJIPFM@85?3?5Microsoft?5Excel?54?40?5macro?5sh@ 1007cd54     xlstool.obj
 0002:00002d78       ??_C@_0BO@JKEOEODC@85?3?5Worksheet?5or?5dialog?5sheet?$AA@ 1007cd78     xlstool.obj
 0002:00002d98       ??_C@_0BA@PILJBENH@?5?5?5?5?5?5?5xf?3?5?$CFi?5?6?$AA@ 1007cd98     xlstool.obj
 0002:00002da8       ??_C@_0BC@PEFPHADI@?5?5?5?5Flags?3?5?$CF?44X?5?6?$AA@ 1007cda8     xlstool.obj
 0002:00002dbc       ??_C@_0BJ@JHNDDLIK@?5?5?5Height?3?5?$CFi?5?$CI1?120?5px?$CJ?6?$AA@ 1007cdbc     xlstool.obj
 0002:00002dd8       ??_C@_0BA@IEBFFLEI@?5Last?5col?3?5?$CFi?5?6?$AA@ 1007cdd8     xlstool.obj
 0002:00002de8       ??_C@_0BA@EPFECGIJ@First?5col?3?5?$CFi?5?6?$AA@ 1007cde8     xlstool.obj
 0002:00002df8       ??_C@_0BA@GKJDFBEC@?5?5?5?5Index?3?5?$CFi?5?6?$AA@ 1007cdf8     xlstool.obj
 0002:00002e08       ??_C@_02MNMNLDAI@?$CJ?6?$AA@ 1007ce08     xlstool.obj
 0002:00002e0c       ??_C@_0L@OICLGHD@collapsed?5?$AA@ 1007ce0c     xlstool.obj
 0002:00002e18       ??_C@_08INMOLJKM@outline?5?$AA@ 1007ce18     xlstool.obj
 0002:00002e24       ??_C@_07KHJCLHGE@hiddeh?5?$AA@ 1007ce24     xlstool.obj
 0002:00002e2c       ??_C@_0BA@HCGMMOEG@?5?5?5?5Flags?3?5?$CFi?5?$CI?$AA@ 1007ce2c     xlstool.obj
 0002:00002e3c       ??_C@_0BA@IDDOPECC@?5?5?5?5?5?5?5XF?3?5?$CFi?5?6?$AA@ 1007ce3c     xlstool.obj
 0002:00002e4c       ??_C@_0BK@KIGJCBGO@?5?5?5?5Width?3?5?$CFi?5?$CI1?1256?5px?$CJ?6?$AA@ 1007ce4c     xlstool.obj
 0002:00002e68       ??_C@_0N@FHFCGOEP@?5?5?5?5str?3?5?$CFs?6?$AA@ 1007ce68     xlstool.obj
 0002:00002e78       ??_C@_0N@FAAMIACI@?5?5?5long?3?5?$CFi?6?$AA@ 1007ce78     xlstool.obj
 0002:00002e88       ??_C@_0N@NCMLPNJC@?5double?3?5?$CFf?6?$AA@ 1007ce88     xlstool.obj
 0002:00002e98       ??_C@_0N@MJACJIMI@?5?5?5?5?5xf?3?5?$CFi?6?$AA@ 1007ce98     xlstool.obj
 0002:00002ea8       ??_C@_0P@LBEHJAIH@?5?5?5Cell?3?5?$CFc?$CFi?6?$AA@ 1007cea8     xlstool.obj
 0002:00002eb8       ??_C@_0BA@LIHMNALL@?5?5?5charset?3?5?$CFi?6?$AA@ 1007ceb8     xlstool.obj
 0002:00002ec8       ??_C@_0BA@MANJJGKB@?5?5?5?5family?3?5?$CFi?6?$AA@ 1007cec8     xlstool.obj
 0002:00002ed8       ??_C@_0BA@MHMCHPJH@?5underline?3?5?$CFi?6?$AA@ 1007ced8     xlstool.obj
 0002:00002ee8       ??_C@_0BA@MAODAHDF@escapement?3?5?$CFi?6?$AA@ 1007cee8     xlstool.obj
 0002:00002ef8       ??_C@_0BA@IMFJJNJH@?5?5?5?5?5?5bold?3?5?$CFi?6?$AA@ 1007cef8     xlstool.obj
 0002:00002f08       ??_C@_0BC@ELDHDBMN@?5?5?5?5?5color?3?5?$CF?46X?6?$AA@ 1007cf08     xlstool.obj
 0002:00002f1c       ??_C@_0BC@IEEOAJDP@?5?5?5?5?5?5flag?3?5?$CF?44X?6?$AA@ 1007cf1c     xlstool.obj
 0002:00002f30       ??_C@_0BA@LNIFCCOP@?5?5?5?5height?3?5?$CFi?6?$AA@ 1007cf30     xlstool.obj
 0002:00002f40       ??_C@_0BA@CFMLILAH@?5?5?5?5?5?5name?3?5?$CFs?6?$AA@ 1007cf40     xlstool.obj
 0002:00002f50       ??_C@_0BB@FNDBDGBI@GroundColor?3?5?$CFi?6?$AA@ 1007cf50     xlstool.obj
 0002:00002f64       ??_C@_0BB@IJHJMKEE@?5?5Linecolor?3?5?$CFi?6?$AA@ 1007cf64     xlstool.obj
 0002:00002f78       ??_C@_0BB@LEPMFJNK@?5?5LineStyle?3?5?$CFi?6?$AA@ 1007cf78     xlstool.obj
 0002:00002f8c       ??_C@_0BB@LCNMNOIK@?5?5?5UsedAttr?3?5?$CFi?6?$AA@ 1007cf8c     xlstool.obj
 0002:00002fa0       ??_C@_0BB@BBPMNMFC@?5?5?5?5?5?5Ident?3?5?$CFi?6?$AA@ 1007cfa0     xlstool.obj
 0002:00002fb4       ??_C@_0BB@ENLMFBCH@?5?5?5Rotation?3?5?$CFi?6?$AA@ 1007cfb4     xlstool.obj
 0002:00002fc8       ??_C@_0BB@ICDNFGFM@?5?5?5?5?5?5Align?3?5?$CFi?6?$AA@ 1007cfc8     xlstool.obj
 0002:00002fdc       ??_C@_0BB@LAPKPDNB@?5?5?5?5?5?5?5Type?3?5?$CFi?6?$AA@ 1007cfdc     xlstool.obj
 0002:00002ff0       ??_C@_0BB@PAPCBBDF@?5?5?5?5?5Format?3?5?$CFi?6?$AA@ 1007cff0     xlstool.obj
 0002:00003004       ??_C@_0BB@OEODCNJM@?5?5?5?5?5?5?5Font?3?5?$CFi?6?$AA@ 1007d004     xlstool.obj
 0002:00003018       ??_C@_06ODLOODK@?$CGnbsp?$DL?$AA@ 1007d018     xlstool.obj
 0002:00003020       ??_C@_02DKCKIIND@?$CFs?$AA@ 1007d020     xlstool.obj
 0002:00003024       ??_C@_04GEFJINEE@?$CF?42f?$AA@ 1007d024     xlstool.obj
 0002:0000302c       ??_C@_04GHNNFJCK@?$CF?40f?$AA@ 1007d02c     xlstool.obj
 0002:00003034       ??_C@_04ENDCGANO@?$CF?41e?$AA@ 1007d034     xlstool.obj
 0002:0000303c       ??_C@_05JJCGAMOD@?$CF?42f?$CF?$AA@ 1007d03c     xlstool.obj
 0002:00003044       ??_C@_03OGKCFPKH@?$CFi?$CF?$AA@ 1007d044     xlstool.obj
 0002:00003048       ??_C@_04GGBPDDBN@?$CF?41f?$AA@ 1007d048     xlstool.obj
 0002:00003050       ??_C@_02IKAHHCAI@?$CFi?$AA@ 1007d050     xlstool.obj
 0002:00003058       ??_C@_0GM@FBOJAFED@?4xf?$CFi?$HL?5font?9size?3?$CFipt?$DLfont?9famil@ 1007d058     xlstool.obj
 0002:000030c4       ??_C@_05MPFIAJAP@Arial?$AA@ 1007d0c4     xlstool.obj
 0002:000030cc       ??_C@_0BM@NGALAKNG@text?9decoration?3?5underline?$DL?$AA@ 1007d0cc     xlstool.obj
 0002:000030e8       ??_C@_0BD@DHCJFIDP@font?9weight?3?5bold?$DL?$AA@ 1007d0e8     xlstool.obj
 0002:000030fc       ??_C@_0BE@NEKNFFJM@font?9style?3?5italic?$DL?$AA@ 1007d0fc     xlstool.obj
 0002:00003110       ??_C@_0N@PFJGBCNM@color?3?$CD?$CF?46X?$DL?$AA@ 1007d110     xlstool.obj
 0002:00003120       ??_C@_0CA@EKOMNFAF@border?9bottom?3?51px?5solid?5Black?$DL?$AA@ 1007d120     xlstool.obj
 0002:00003140       ??_C@_0BN@ONIOGKCE@border?9top?3?51px?5solid?5black?$DL?$AA@ 1007d140     xlstool.obj
 0002:00003160       ??_C@_0BP@FLGEPMPK@border?9right?3?51px?5solid?5black?$DL?$AA@ 1007d160     xlstool.obj
 0002:00003180       ??_C@_01LOCGONAA@?$AA?$AA@ 1007d180     xlstool.obj
 0002:00003184       ??_C@_0BO@BBFHCOLK@border?9left?3?51px?5solid?5black?$DL?$AA@ 1007d184     xlstool.obj
 0002:000031a4       ??_C@_04GOOOJOPP@left?$AA@ 1007d1a4     xlstool.obj
 0002:000031ac       ??_C@_06BBLOAEEI@center?$AA@ 1007d1ac     xlstool.obj
 0002:000031b4       ??_C@_05DHJDAOHK@right?$AA@ 1007d1b4     xlstool.obj
 0002:000031bc       ??_C@_03FGFCOCMD@top?$AA@  1007d1bc     xlstool.obj
 0002:000031c0       ??_C@_06PMMPCIPB@bottom?$AA@ 1007d1c0     xlstool.obj
 0002:000031c8       ??_C@_06CGLIEPEJ@middle?$AA@ 1007d1c8     xlstool.obj
 0002:000031d0       ??_C@_0CF@DAJPCBAO@audiomixer?5device?5is?5not?5support@ 1007d1d0     wzSound.obj
 0002:000031f8       ??_C@_0CM@BPAMFFI@secure?5file?5system?5opened?5succes@ 1007d1f8     wzSound.obj
 0002:00003224       ??_C@_0CD@EAONBBBE@can?8t?5open?5secure?5file?5system?5?3?5@ 1007d224     wzSound.obj
 0002:00003248       ??_C@_0BI@HKDHILJF@pack?5Encryption?5SUCCESS?$AA@ 1007d248     wzSound.obj
 0002:00003260       ??_C@_0CC@BPKMBLEF@ERROR?9?5amdGetMicOutputMuteContro@ 1007d260     wzSound.obj
 0002:00003284       ??_C@_0CE@JOGKBPJD@ERROR?9?5amdGetMicOutputVolumeCont@ 1007d284     wzSound.obj
 0002:000032a8       ??_C@_0CD@PJFOFAKL@ERROR?9?5amdGetMicInputVolumeContr@ 1007d2a8     wzSound.obj
 0002:000032cc       ??_C@_0BM@MOHFIGFN@ERROR?9?5amdGetWavMuteControl?$AA@ 1007d2cc     wzSound.obj
 0002:000032e8       ??_C@_0BO@JCMPLJOK@ERROR?9?5amdGetWavVolumeControl?$AA@ 1007d2e8     wzSound.obj
 0002:00003308       ??_C@_0BP@MJOOLGGL@ERROR?9?5amdGetMasterMuteControl?$AA@ 1007d308     wzSound.obj
 0002:00003328       ??_C@_0CB@DNAKBPKI@ERROR?9?5amdGetMasterVolumeControl@ 1007d328     wzSound.obj
 0002:0000334c       ??_C@_0BF@MFBLIFPP@CoInitialize?5Failed?$CB?$AA@ 1007d34c     wzSound.obj
 0002:00003364       ??_C@_0BP@DEPCNHLF@wzsnd?5is?5already?5initialized?5?$CB?$AA@ 1007d364     wzSound.obj
 0002:00003384       ??_C@_0BL@PLGBJAMA@wzsnd?5is?5not?5initialized?5?$CB?$AA@ 1007d384     wzSound.obj
 0002:000033a0       ??_C@_0BE@OIPLICFJ@?$CD?$FL4?$FN?5CoUninitialize?$AA@ 1007d3a0     wzSound.obj
 0002:000033b4       ??_C@_0CA@DAAJGADE@?$CD?$FL3?$FN?5uninitialize?5speaker?5mixer?$AA@ 1007d3b4     wzSound.obj
 0002:000033d4       ??_C@_0CD@FDLOJCBC@?$CD?$FL2?$FN?5uninitialize?5microphone?5mix@ 1007d3d4     wzSound.obj
 0002:000033f8       ??_C@_0BL@FNKMOFKH@?$CD?$FL1?$FN?5close?5packFile?5system?$AA@ 1007d3f8     wzSound.obj
 0002:00003414       ??_C@_0CA@FFAAANEL@?$CD?$FL0?$FN?5destroy?5all?5sound?5channels?$AA@ 1007d414     wzSound.obj
 0002:00003434       ??_C@_0P@MNMNFJJ@?$CD?$FL?9?9?9?9?9?9?9?9?9?9?9?$FN?$AA@ 1007d434     wzSound.obj
 0002:00003444       __real@40400000            1007d444     wzSound.obj
 0002:00003448       ??_C@_07MGFEJOAL@?$FL?$CFd?$FN?5?$CFs?$AA@ 1007d448     wzSound.obj
 0002:00003450       ??_C@_0CN@NCCLHEBG@index?$FL?$CFd?$FN?5invalid?5Listener?5or?5Po@ 1007d450     wzSound.obj
 0002:00003480       _GUID_NULL                 1007d480     uuid:cguid_i.obj
 0002:00003490       _CATID_MARSHALER           1007d490     uuid:cguid_i.obj
 0002:000034a0       _IID_IRpcChannel           1007d4a0     uuid:cguid_i.obj
 0002:000034b0       _IID_IRpcStub              1007d4b0     uuid:cguid_i.obj
 0002:000034c0       _IID_IStubManager          1007d4c0     uuid:cguid_i.obj
 0002:000034d0       _IID_IRpcProxy             1007d4d0     uuid:cguid_i.obj
 0002:000034e0       _IID_IProxyManager         1007d4e0     uuid:cguid_i.obj
 0002:000034f0       _IID_IPSFactory            1007d4f0     uuid:cguid_i.obj
 0002:00003500       _IID_IInternalMoniker      1007d500     uuid:cguid_i.obj
 0002:00003510       _IID_IDfReserved1          1007d510     uuid:cguid_i.obj
 0002:00003520       _IID_IDfReserved2          1007d520     uuid:cguid_i.obj
 0002:00003530       _IID_IDfReserved3          1007d530     uuid:cguid_i.obj
 0002:00003540       _CLSID_StdMarshal          1007d540     uuid:cguid_i.obj
 0002:00003550       _IID_IStub                 1007d550     uuid:cguid_i.obj
 0002:00003560       _IID_IProxy                1007d560     uuid:cguid_i.obj
 0002:00003570       _IID_IEnumGeneric          1007d570     uuid:cguid_i.obj
 0002:00003580       _IID_IEnumHolder           1007d580     uuid:cguid_i.obj
 0002:00003590       _IID_IEnumCallback         1007d590     uuid:cguid_i.obj
 0002:000035a0       _IID_IOleManager           1007d5a0     uuid:cguid_i.obj
 0002:000035b0       _IID_IOlePresObj           1007d5b0     uuid:cguid_i.obj
 0002:000035c0       _IID_IDebug                1007d5c0     uuid:cguid_i.obj
 0002:000035d0       _IID_IDebugStream          1007d5d0     uuid:cguid_i.obj
 0002:000035e0       _CLSID_PSGenObject         1007d5e0     uuid:cguid_i.obj
 0002:000035f0       _CLSID_PSClientSite        1007d5f0     uuid:cguid_i.obj
 0002:00003600       _CLSID_PSClassObject       1007d600     uuid:cguid_i.obj
 0002:00003610       _CLSID_PSInPlaceActive     1007d610     uuid:cguid_i.obj
 0002:00003620       _CLSID_PSInPlaceFrame      1007d620     uuid:cguid_i.obj
 0002:00003630       _CLSID_PSDragDrop          1007d630     uuid:cguid_i.obj
 0002:00003640       _CLSID_PSBindCtx           1007d640     uuid:cguid_i.obj
 0002:00003650       _CLSID_PSEnumerators       1007d650     uuid:cguid_i.obj
 0002:00003660       _CLSID_StaticMetafile      1007d660     uuid:cguid_i.obj
 0002:00003670       _CLSID_StaticDib           1007d670     uuid:cguid_i.obj
 0002:00003680       _CLSID_Picture_Metafile    1007d680     uuid:cguid_i.obj
 0002:00003690       _CLSID_Picture_EnhMetafile 1007d690     uuid:cguid_i.obj
 0002:000036a0       _CLSID_Picture_Dib         1007d6a0     uuid:cguid_i.obj
 0002:000036b0       _CLSID_DCOMAccessControl   1007d6b0     uuid:cguid_i.obj
 0002:000036c0       _CLSID_StdGlobalInterfaceTable 1007d6c0     uuid:cguid_i.obj
 0002:000036d0       _CLSID_ManualResetEvent    1007d6d0     uuid:cguid_i.obj
 0002:000036e0       _CLSID_StdEvent            1007d6e0     uuid:cguid_i.obj
 0002:000036f0       _CLSID_SynchronizeContainer 1007d6f0     uuid:cguid_i.obj
 0002:00003700       _CLSID_ComBinding          1007d700     uuid:cguid_i.obj
 0002:00003710       _CLSID_StdAsyncActManager  1007d710     uuid:cguid_i.obj
 0002:00003720       _CLSID_InProcFreeMarshaler 1007d720     uuid:cguid_i.obj
 0002:00003730       _CLSID_RemoteUnknownPSFactory 1007d730     uuid:cguid_i.obj
 0002:00003740       _IID_IRichEditOle          1007d740     uuid:cguid_i.obj
 0002:00003750       _IID_IRichEditOleCallback  1007d750     uuid:cguid_i.obj
 0002:00003760       _CLSID_AllClasses          1007d760     uuid:cguid_i.obj
 0002:00003770       _CLSID_LocalMachineClasses 1007d770     uuid:cguid_i.obj
 0002:00003780       _CLSID_CurrentUserClasses  1007d780     uuid:cguid_i.obj
 0002:00003790       _CLSID_AddrControl         1007d790     uuid:cguid_i.obj
 0002:000037a0       _CLSID_GlobalOptions       1007d7a0     uuid:cguid_i.obj
 0002:000037b0       _CLSID_SurrogateManager    1007d7b0     uuid:cguid_i.obj
 0002:000037c0       _CLSID_ContextSwitcher     1007d7c0     uuid:cguid_i.obj
 0002:000037d0       _IID_IPropertyFrame        1007d7d0     uuid:cguid_i.obj
 0002:000037e0       _CLSID_CFontPropPage       1007d7e0     uuid:cguid_i.obj
 0002:000037f0       _CLSID_CColorPropPage      1007d7f0     uuid:cguid_i.obj
 0002:00003800       _CLSID_CPicturePropPage    1007d800     uuid:cguid_i.obj
 0002:00003810       _CLSID_StockFontPage       1007d810     uuid:cguid_i.obj
 0002:00003820       _CLSID_StockColorPage      1007d820     uuid:cguid_i.obj
 0002:00003830       _CLSID_StockPicturePage    1007d830     uuid:cguid_i.obj
 0002:00003840       _CLSID_PersistPropset      1007d840     uuid:cguid_i.obj
 0002:00003850       _CLSID_ConvertVBX          1007d850     uuid:cguid_i.obj
 0002:00003860       _CLSID_StdFont             1007d860     uuid:cguid_i.obj
 0002:00003870       _CLSID_StdPicture          1007d870     uuid:cguid_i.obj
 0002:00003880       _GUID_HIMETRIC             1007d880     uuid:cguid_i.obj
 0002:00003890       _GUID_COLOR                1007d890     uuid:cguid_i.obj
 0002:000038a0       _GUID_XPOSPIXEL            1007d8a0     uuid:cguid_i.obj
 0002:000038b0       _GUID_YPOSPIXEL            1007d8b0     uuid:cguid_i.obj
 0002:000038c0       _GUID_XSIZEPIXEL           1007d8c0     uuid:cguid_i.obj
 0002:000038d0       _GUID_YSIZEPIXEL           1007d8d0     uuid:cguid_i.obj
 0002:000038e0       _GUID_XPOS                 1007d8e0     uuid:cguid_i.obj
 0002:000038f0       _GUID_YPOS                 1007d8f0     uuid:cguid_i.obj
 0002:00003900       _GUID_XSIZE                1007d900     uuid:cguid_i.obj
 0002:00003910       _GUID_YSIZE                1007d910     uuid:cguid_i.obj
 0002:00003920       _GUID_TRISTATE             1007d920     uuid:cguid_i.obj
 0002:00003930       _GUID_OPTIONVALUEEXCLUSIVE 1007d930     uuid:cguid_i.obj
 0002:00003940       _GUID_CHECKVALUEEXCLUSIVE  1007d940     uuid:cguid_i.obj
 0002:00003950       _GUID_FONTNAME             1007d950     uuid:cguid_i.obj
 0002:00003960       _GUID_FONTSIZE             1007d960     uuid:cguid_i.obj
 0002:00003970       _GUID_FONTBOLD             1007d970     uuid:cguid_i.obj
 0002:00003980       _GUID_FONTITALIC           1007d980     uuid:cguid_i.obj
 0002:00003990       _GUID_FONTUNDERSCORE       1007d990     uuid:cguid_i.obj
 0002:000039a0       _GUID_FONTSTRIKETHROUGH    1007d9a0     uuid:cguid_i.obj
 0002:000039b0       _GUID_HANDLE               1007d9b0     uuid:cguid_i.obj
 0002:000039c0       _IID_StdOle                1007d9c0     uuid:cguid_i.obj
 0002:000039d0       _IID_ICursor               1007d9d0     uuid:cguid_i.obj
 0002:000039e0       _IID_ICursorMove           1007d9e0     uuid:cguid_i.obj
 0002:000039f0       _IID_ICursorScroll         1007d9f0     uuid:cguid_i.obj
 0002:00003a00       _IID_ICursorUpdateARow     1007da00     uuid:cguid_i.obj
 0002:00003a10       _IID_INotifyDBEvents       1007da10     uuid:cguid_i.obj
 0002:00003a20       _IID_ICursorFind           1007da20     uuid:cguid_i.obj
 0002:00003a30       _IID_IEntryID              1007da30     uuid:cguid_i.obj
 0002:00003a40       __GUID_NAMEONLY            1007da40     uuid:cguid_i.obj
 0002:00003a50       __DBBMKGUID                1007da50     uuid:cguid_i.obj
 0002:00003a60       __DBCIDGUID                1007da60     uuid:cguid_i.obj
 0002:00003a70       _IID_IBoundObject          1007da70     uuid:cguid_i.obj
 0002:00003a80       _IID_IBoundObjectSite      1007da80     uuid:cguid_i.obj
 0002:00003a90       _CLSID_GblComponentCategoriesMgr 1007da90     uuid:cguid_i.obj
 0002:00003aa0       _CLSID_ThumbnailFCNHandler 1007daa0     uuid:cguid_i.obj
 0002:00003ab0       _CLSID_ThumbnailUpdater    1007dab0     uuid:cguid_i.obj
 0002:00003ac0       _GUID_DEVCLASS_1394        1007dac0     uuid:cguid_i.obj
 0002:00003ad0       _GUID_DEVCLASS_1394DEBUG   1007dad0     uuid:cguid_i.obj
 0002:00003ae0       _GUID_DEVCLASS_61883       1007dae0     uuid:cguid_i.obj
 0002:00003af0       _GUID_DEVCLASS_ADAPTER     1007daf0     uuid:cguid_i.obj
 0002:00003b00       _GUID_DEVCLASS_APMSUPPORT  1007db00     uuid:cguid_i.obj
 0002:00003b10       _GUID_DEVCLASS_AVC         1007db10     uuid:cguid_i.obj
 0002:00003b20       _GUID_DEVCLASS_BATTERY     1007db20     uuid:cguid_i.obj
 0002:00003b30       _GUID_DEVCLASS_BIOMETRIC   1007db30     uuid:cguid_i.obj
 0002:00003b40       _GUID_DEVCLASS_BLUETOOTH   1007db40     uuid:cguid_i.obj
 0002:00003b50       _GUID_DEVCLASS_CDROM       1007db50     uuid:cguid_i.obj
 0002:00003b60       _GUID_DEVCLASS_COMPUTER    1007db60     uuid:cguid_i.obj
 0002:00003b70       _GUID_DEVCLASS_DECODER     1007db70     uuid:cguid_i.obj
 0002:00003b80       _GUID_DEVCLASS_DISKDRIVE   1007db80     uuid:cguid_i.obj
 0002:00003b90       _GUID_DEVCLASS_DISPLAY     1007db90     uuid:cguid_i.obj
 0002:00003ba0       _GUID_DEVCLASS_DOT4        1007dba0     uuid:cguid_i.obj
 0002:00003bb0       _GUID_DEVCLASS_DOT4PRINT   1007dbb0     uuid:cguid_i.obj
 0002:00003bc0       _GUID_DEVCLASS_ENUM1394    1007dbc0     uuid:cguid_i.obj
 0002:00003bd0       _GUID_DEVCLASS_FDC         1007dbd0     uuid:cguid_i.obj
 0002:00003be0       _GUID_DEVCLASS_FLOPPYDISK  1007dbe0     uuid:cguid_i.obj
 0002:00003bf0       _GUID_DEVCLASS_GPS         1007dbf0     uuid:cguid_i.obj
 0002:00003c00       _GUID_DEVCLASS_HDC         1007dc00     uuid:cguid_i.obj
 0002:00003c10       _GUID_DEVCLASS_HIDCLASS    1007dc10     uuid:cguid_i.obj
 0002:00003c20       _GUID_DEVCLASS_IMAGE       1007dc20     uuid:cguid_i.obj
 0002:00003c30       _GUID_DEVCLASS_INFINIBAND  1007dc30     uuid:cguid_i.obj
 0002:00003c40       _GUID_DEVCLASS_INFRARED    1007dc40     uuid:cguid_i.obj
 0002:00003c50       _GUID_DEVCLASS_KEYBOARD    1007dc50     uuid:cguid_i.obj
 0002:00003c60       _GUID_DEVCLASS_LEGACYDRIVER 1007dc60     uuid:cguid_i.obj
 0002:00003c70       _GUID_DEVCLASS_MEDIA       1007dc70     uuid:cguid_i.obj
 0002:00003c80       _GUID_DEVCLASS_MEDIUM_CHANGER 1007dc80     uuid:cguid_i.obj
 0002:00003c90       _GUID_DEVCLASS_MODEM       1007dc90     uuid:cguid_i.obj
 0002:00003ca0       _GUID_DEVCLASS_MONITOR     1007dca0     uuid:cguid_i.obj
 0002:00003cb0       _GUID_DEVCLASS_MOUSE       1007dcb0     uuid:cguid_i.obj
 0002:00003cc0       _GUID_DEVCLASS_MTD         1007dcc0     uuid:cguid_i.obj
 0002:00003cd0       _GUID_DEVCLASS_MULTIFUNCTION 1007dcd0     uuid:cguid_i.obj
 0002:00003ce0       _GUID_DEVCLASS_MULTIPORTSERIAL 1007dce0     uuid:cguid_i.obj
 0002:00003cf0       _GUID_DEVCLASS_NET         1007dcf0     uuid:cguid_i.obj
 0002:00003d00       _GUID_DEVCLASS_NETCLIENT   1007dd00     uuid:cguid_i.obj
 0002:00003d10       _GUID_DEVCLASS_NETSERVICE  1007dd10     uuid:cguid_i.obj
 0002:00003d20       _GUID_DEVCLASS_NETTRANS    1007dd20     uuid:cguid_i.obj
 0002:00003d30       _GUID_DEVCLASS_NODRIVER    1007dd30     uuid:cguid_i.obj
 0002:00003d40       _GUID_DEVCLASS_PCMCIA      1007dd40     uuid:cguid_i.obj
 0002:00003d50       _GUID_DEVCLASS_PNPPRINTERS 1007dd50     uuid:cguid_i.obj
 0002:00003d60       _GUID_DEVCLASS_PORTS       1007dd60     uuid:cguid_i.obj
 0002:00003d70       _GUID_DEVCLASS_PRINTER     1007dd70     uuid:cguid_i.obj
 0002:00003d80       _GUID_DEVCLASS_PRINTERUPGRADE 1007dd80     uuid:cguid_i.obj
 0002:00003d90       _GUID_DEVCLASS_PROCESSOR   1007dd90     uuid:cguid_i.obj
 0002:00003da0       _GUID_DEVCLASS_SBP2        1007dda0     uuid:cguid_i.obj
 0002:00003db0       _GUID_DEVCLASS_SCSIADAPTER 1007ddb0     uuid:cguid_i.obj
 0002:00003dc0       _GUID_DEVCLASS_SECURITYACCELERATOR 1007ddc0     uuid:cguid_i.obj
 0002:00003dd0       _GUID_DEVCLASS_SIDESHOW    1007ddd0     uuid:cguid_i.obj
 0002:00003de0       _GUID_DEVCLASS_SMARTCARDREADER 1007dde0     uuid:cguid_i.obj
 0002:00003df0       _GUID_DEVCLASS_SOUND       1007ddf0     uuid:cguid_i.obj
 0002:00003e00       _GUID_DEVCLASS_SYSTEM      1007de00     uuid:cguid_i.obj
 0002:00003e10       _GUID_DEVCLASS_TAPEDRIVE   1007de10     uuid:cguid_i.obj
 0002:00003e20       _GUID_DEVCLASS_UNKNOWN     1007de20     uuid:cguid_i.obj
 0002:00003e30       _GUID_DEVCLASS_USB         1007de30     uuid:cguid_i.obj
 0002:00003e40       _GUID_DEVCLASS_VOLUME      1007de40     uuid:cguid_i.obj
 0002:00003e50       _GUID_DEVCLASS_VOLUMESNAPSHOT 1007de50     uuid:cguid_i.obj
 0002:00003e60       _GUID_DEVCLASS_WCEUSBS     1007de60     uuid:cguid_i.obj
 0002:00003e70       _GUID_DEVCLASS_WPD         1007de70     uuid:cguid_i.obj
 0002:00003e80       _GUID_DEVCLASS_FSFILTER_ACTIVITYMONITOR 1007de80     uuid:cguid_i.obj
 0002:00003e90       _GUID_DEVCLASS_FSFILTER_UNDELETE 1007de90     uuid:cguid_i.obj
 0002:00003ea0       _GUID_DEVCLASS_FSFILTER_ANTIVIRUS 1007dea0     uuid:cguid_i.obj
 0002:00003eb0       _GUID_DEVCLASS_FSFILTER_REPLICATION 1007deb0     uuid:cguid_i.obj
 0002:00003ec0       _GUID_DEVCLASS_FSFILTER_CONTINUOUSBACKUP 1007dec0     uuid:cguid_i.obj
 0002:00003ed0       _GUID_DEVCLASS_FSFILTER_CONTENTSCREENER 1007ded0     uuid:cguid_i.obj
 0002:00003ee0       _GUID_DEVCLASS_FSFILTER_QUOTAMANAGEMENT 1007dee0     uuid:cguid_i.obj
 0002:00003ef0       _GUID_DEVCLASS_FSFILTER_SYSTEMRECOVERY 1007def0     uuid:cguid_i.obj
 0002:00003f00       _GUID_DEVCLASS_FSFILTER_CFSMETADATASERVER 1007df00     uuid:cguid_i.obj
 0002:00003f10       _GUID_DEVCLASS_FSFILTER_HSM 1007df10     uuid:cguid_i.obj
 0002:00003f20       _GUID_DEVCLASS_FSFILTER_COMPRESSION 1007df20     uuid:cguid_i.obj
 0002:00003f30       _GUID_DEVCLASS_FSFILTER_ENCRYPTION 1007df30     uuid:cguid_i.obj
 0002:00003f40       _GUID_DEVCLASS_FSFILTER_PHYSICALQUOTAMANAGEMENT 1007df40     uuid:cguid_i.obj
 0002:00003f50       _GUID_DEVCLASS_FSFILTER_OPENFILEBACKUP 1007df50     uuid:cguid_i.obj
 0002:00003f60       _GUID_DEVCLASS_FSFILTER_SECURITYENHANCER 1007df60     uuid:cguid_i.obj
 0002:00003f70       _GUID_DEVCLASS_FSFILTER_COPYPROTECTION 1007df70     uuid:cguid_i.obj
 0002:00003f80       _GUID_DEVCLASS_FSFILTER_SYSTEM 1007df80     uuid:cguid_i.obj
 0002:00003f90       _GUID_DEVCLASS_FSFILTER_INFRASTRUCTURE 1007df90     uuid:cguid_i.obj
 0002:00003fa0       _GUID_DEVINTERFACE_DISK    1007dfa0     uuid:cguid_i.obj
 0002:00003fb0       _GUID_DEVINTERFACE_CDROM   1007dfb0     uuid:cguid_i.obj
 0002:00003fc0       _GUID_DEVINTERFACE_PARTITION 1007dfc0     uuid:cguid_i.obj
 0002:00003fd0       _GUID_DEVINTERFACE_TAPE    1007dfd0     uuid:cguid_i.obj
 0002:00003fe0       _GUID_DEVINTERFACE_WRITEONCEDISK 1007dfe0     uuid:cguid_i.obj
 0002:00003ff0       _GUID_DEVINTERFACE_VOLUME  1007dff0     uuid:cguid_i.obj
 0002:00004000       _GUID_DEVINTERFACE_MEDIUMCHANGER 1007e000     uuid:cguid_i.obj
 0002:00004010       _GUID_DEVINTERFACE_FLOPPY  1007e010     uuid:cguid_i.obj
 0002:00004020       _GUID_DEVINTERFACE_CDCHANGER 1007e020     uuid:cguid_i.obj
 0002:00004030       _GUID_DEVINTERFACE_STORAGEPORT 1007e030     uuid:cguid_i.obj
 0002:00004040       _GUID_DEVINTERFACE_COMPORT 1007e040     uuid:cguid_i.obj
 0002:00004050       _GUID_DEVINTERFACE_SERENUM_BUS_ENUMERATOR 1007e050     uuid:cguid_i.obj
 0002:00004064       ??_7invalid_argument@std@@6B@ 1007e064     libcpmt:string.obj
 0002:0000406c       ??_C@_0BA@JFNIOLAK@string?5too?5long?$AA@ 1007e06c     libcpmt:string.obj
 0002:0000407c       ??_C@_0BI@CFPLBAOH@invalid?5string?5position?$AA@ 1007e07c     libcpmt:string.obj
 0002:00004094       ??_C@_0BI@ILCMCLF@invalid?5string?5argument?$AA@ 1007e094     libcpmt:string.obj
 0002:000040b0       __real@8@3ffe8000000000000000 1007e0b0     vorbisfile_static:vorbisfile.obj
 0002:000040b8       __real@4@3ffe8000000000000000 1007e0b8     vorbisfile_static:vorbisfile.obj
 0002:000040c0       __real@8@00000000000000000000 1007e0c0     vorbisfile_static:vorbisfile.obj
 0002:000040c8       __real@8@c0068300000000000000 1007e0c8     vorbisfile_static:vorbisfile.obj
 0002:000040d0       __real@4@400e8000000000000000 1007e0d0     vorbisfile_static:vorbisfile.obj
 0002:000040d4       __real@4@40068000000000000000 1007e0d4     vorbisfile_static:vorbisfile.obj
 0002:000040d8       __real@8@3fff8000000000000000 1007e0d8     vorbisfile_static:vorbisfile.obj
 0002:000040e0       __real@8@bfff8000000000000000 1007e0e0     vorbisfile_static:info.obj
 0002:000040e8       __real@4@c0068c00000000000000 1007e0e8     vorbisfile_static:analysis.obj
 0002:000040f0       __real@8@3ff283126e978d4fe000 1007e0f0     vorbisfile_static:analysis.obj
 0002:000040f8       __real@8@3ff1d1b7170000000000 1007e0f8     vorbisfile_static:analysis.obj
 0002:00004100       __real@8@4002d1999a0000000000 1007e100     vorbisfile_static:analysis.obj
 0002:00004108       __real@8@3ff4c1fc8f0000000000 1007e108     vorbisfile_static:analysis.obj
 0002:00004110       __real@8@40008f5c290000000000 1007e110     vorbisfile_static:analysis.obj
 0002:00004118       __real@8@3fe59ee9ee0000000000 1007e118     vorbisfile_static:analysis.obj
 0002:00004120       __real@8@3ffd8000000000000000 1007e120     vorbisfile_static:analysis.obj
 0002:00004128       __real@4@400afa00000000000000 1007e128     vorbisfile_static:analysis.obj
 0002:0000412c       __real@4@4008bf115b0000000000 1007e12c     vorbisfile_static:analysis.obj
 0002:00004130       __real@4@3feac0a8c10000000000 1007e130     vorbisfile_static:analysis.obj
 0002:00004134       __real@4@40038000000000000000 1007e134     vorbisfile_static:psy.obj
 0002:00004138       __real@4@00000000000000000000 1007e138     vorbisfile_static:psy.obj
 0002:0000413c       __real@4@3ff1d1b7170000000000 1007e13c     vorbisfile_static:psy.obj
 0002:00004140       __real@4@3ff4c1fc8f0000000000 1007e140     vorbisfile_static:psy.obj
 0002:00004144       __real@4@3fe59ee9ee0000000000 1007e144     vorbisfile_static:psy.obj
 0002:00004148       __real@8@4005c800000000000000 1007e148     vorbisfile_static:psy.obj
 0002:00004150       __real@8@3ffeb172150000000000 1007e150     vorbisfile_static:psy.obj
 0002:00004158       __real@8@3ffc8000000000000000 1007e158     vorbisfile_static:psy.obj
 0002:00004160       __real@8@4001bee7b40000000000 1007e160     vorbisfile_static:psy.obj
 0002:00004168       __real@8@3fffb8aa3b0000000000 1007e168     vorbisfile_static:psy.obj
 0002:00004170       __real@4@3ffd8000000000000000 1007e170     vorbisfile_static:psy.obj
 0002:00004178       __real@8@40008000000000000000 1007e178     vorbisfile_static:psy.obj
 0002:00004180       __real@4@40028000000000000000 1007e180     vorbisfile_static:psy.obj
 0002:00004184       __real@4@c006c800000000000000 1007e184     vorbisfile_static:psy.obj
 0002:00004188       __real@8@3ffff800000000000000 1007e188     vorbisfile_static:psy.obj
 0002:00004190       __real@8@40008400000000000000 1007e190     vorbisfile_static:psy.obj
 0002:00004198       __real@4@3fff8000000000000000 1007e198     vorbisfile_static:psy.obj
 0002:0000419c       __real@4@4002a000000000000000 1007e19c     vorbisfile_static:psy.obj
 0002:000041a0       __real@8@4003f000000000000000 1007e1a0     vorbisfile_static:psy.obj
 0002:000041a8       __real@8@4002a000000000000000 1007e1a8     vorbisfile_static:psy.obj
 0002:000041b0       __real@4@4008f9c0000000000000 1007e1b0     vorbisfile_static:psy.obj
 0002:000041b4       __real@4@4001c000000000000000 1007e1b4     vorbisfile_static:psy.obj
 0002:000041b8       __real@8@3ffbcccccd0000000000 1007e1b8     vorbisfile_static:psy.obj
 0002:000041c0       __real@4@c00c9c3c000000000000 1007e1c0     vorbisfile_static:psy.obj
 0002:000041c8       __real@8@c0008000000000000000 1007e1c8     vorbisfile_static:psy.obj
 0002:000041d0       __real@8@3ffffffcb90000000000 1007e1d0     vorbisfile_static:psy.obj
 0002:000041d8       __real@8@4001f000000000000000 1007e1d8     vorbisfile_static:bitrate.obj
 0002:000041e0       __real@8@4000c90fdb0000000000 1007e1e0     vorbisfile_static:envelope.obj
 0002:000041e8       __real@8@3ff9caa5254a952a5000 1007e1e8     vorbisfile_static:envelope.obj
 0002:000041f0       __real@4@400fc34f800000000000 1007e1f0     vorbisfile_static:envelope.obj
 0002:000041f8       __real@8@40028000000000000000 1007e1f8     vorbisfile_static:envelope.obj
 0002:00004200       __real@8@4002f000000000000000 1007e200     vorbisfile_static:envelope.obj
 0002:00004208       __real@8@3ffb8000000000000000 1007e208     vorbisfile_static:envelope.obj
 0002:00004210       __real@8@3ffeb333333333333000 1007e210     vorbisfile_static:envelope.obj
 0002:00004218       __real@8@3ffcccccccccccccd000 1007e218     vorbisfile_static:envelope.obj
 0002:00004220       __real@4@40018000000000000000 1007e220     vorbisfile_static:mdct.obj
 0002:00004228       __real@8@bffe8000000000000000 1007e228     vorbisfile_static:mdct.obj
 0002:00004230       __real@4@4000c90fdb0000000000 1007e230     vorbisfile_static:mdct.obj
 0002:00004234       __real@4@3ffeb504f30000000000 1007e234     vorbisfile_static:mdct.obj
 0002:00004238       __real@4@3ffdc3ef150000000000 1007e238     vorbisfile_static:mdct.obj
 0002:0000423c       __real@4@3ffeec835e0000000000 1007e23c     vorbisfile_static:mdct.obj
 0002:00004240       __real@4@4008ffe0000000000000 1007e240     vorbisfile_static:floor1.obj
 0002:00004244       __real@4@4001ea0ea10000000000 1007e244     vorbisfile_static:floor1.obj
 0002:00004248       __real@8@4004a2f9838f1632f000 1007e248     vorbisfile_static:lsp.obj
 0002:00004250       __real@4@40048000000000000000 1007e250     vorbisfile_static:lsp.obj
 0002:00004254       __real@4@40058000000000000000 1007e254     vorbisfile_static:lsp.obj
 0002:00004258       __real@4@c0028000000000000000 1007e258     vorbisfile_static:lsp.obj
 0002:00004260       __real@8@3fdaafebff0bcb24a800 1007e260     vorbisfile_static:lsp.obj
 0002:00004268       __real@8@bfeb8637bd05af6c6800 1007e268     vorbisfile_static:lsp.obj
 0002:00004270       __real@8@3feb8637bd05af6c6800 1007e270     vorbisfile_static:lsp.obj
 0002:00004278       __real@8@3fbcbce5086492111800 1007e278     vorbisfile_static:lsp.obj
 0002:00004280       __FPinit                   1007e280     LIBCMT:_fpinit_.obj
 0002:00004284       __FPmtinit                 1007e284     LIBCMT:_fpinit_.obj
 0002:00004288       __FPmtterm                 1007e288     LIBCMT:_fpinit_.obj
 0002:0000428c       ?ProcessDetach@NativeDll@<CrtImplementationDetails>@@0IB 1007e28c     LIBCMT:stricmp.obj
 0002:00004290       ?ProcessAttach@NativeDll@<CrtImplementationDetails>@@0IB 1007e290     LIBCMT:stricmp.obj
 0002:00004294       ?ThreadAttach@NativeDll@<CrtImplementationDetails>@@0IB 1007e294     LIBCMT:stricmp.obj
 0002:00004298       ?ThreadDetach@NativeDll@<CrtImplementationDetails>@@0IB 1007e298     LIBCMT:stricmp.obj
 0002:0000429c       ?ProcessVerifier@NativeDll@<CrtImplementationDetails>@@0IB 1007e29c     LIBCMT:stricmp.obj
 0002:000042a4       ??_7exception@std@@6B@     1007e2a4     LIBCMT:stdexcpt.obj
 0002:000042ac       ??_C@_0BC@EOODALEL@Unknown?5exception?$AA@ 1007e2ac     LIBCMT:stdexcpt.obj
 0002:000042c4       ??_7bad_cast@std@@6B@      1007e2c4     LIBCMT:stdexcpt.obj
 0002:000042d0       ??_7bad_typeid@std@@6B@    1007e2d0     LIBCMT:stdexcpt.obj
 0002:000042dc       ??_7__non_rtti_object@std@@6B@ 1007e2dc     LIBCMT:stdexcpt.obj
 0002:000042e8       ??_7type_info@@6B@         1007e2e8     LIBCMT:typinfo.obj
 0002:0000430c       __pRawDllMain              1007e30c     LIBCMT:dllcrt0.obj
 0002:0000430c       __pDefaultRawDllMain       1007e30c     LIBCMT:dllcrt0.obj
 0002:000043a8       ??_C@_0P@MIGLKIOC@CorExitProcess?$AA@ 1007e3a8     LIBCMT:crt0dat.obj
 0002:000043b8       ??_C@_1BI@BGOHAHKC@?$AAm?$AAs?$AAc?$AAo?$AAr?$AAe?$AAe?$AA?4?$AAd?$AAl?$AAl?$AA?$AA@ 1007e3b8     LIBCMT:crt0dat.obj
 0002:000043d0       ??_C@_05KLBDPFGC@e?$CL000?$AA@ 1007e3d0     LIBCMT:cvt.obj
 0002:000043d8       __real@4150017ec0000000    1007e3d8     LIBCMT:_testfdiv_.obj
 0002:000043e0       __real@4147ffff80000000    1007e3e0     LIBCMT:_testfdiv_.obj
 0002:000043e8       ??_C@_0BK@NHEOCAHP@IsProcessorFeaturePresent?$AA@ 1007e3e8     LIBCMT:_testfdiv_.obj
 0002:00004404       ??_C@_08CPNIBGIE@KERNEL32?$AA@ 1007e404     LIBCMT:_testfdiv_.obj
 0002:00004410       ??_C@_07LCBHPJJN@LC_TIME?$AA@ 1007e410     LIBCMT:setlocal.obj
 0002:00004418       ??_C@_0L@DLHIECNL@LC_NUMERIC?$AA@ 1007e418     LIBCMT:setlocal.obj
 0002:00004424       ??_C@_0M@MIENIKLA@LC_MONETARY?$AA@ 1007e424     LIBCMT:setlocal.obj
 0002:00004430       ??_C@_08EADHIDAD@LC_CTYPE?$AA@ 1007e430     LIBCMT:setlocal.obj
 0002:0000443c       ??_C@_0L@KFJHEKIK@LC_COLLATE?$AA@ 1007e43c     LIBCMT:setlocal.obj
 0002:00004448       ??_C@_06NEFDFEKB@LC_ALL?$AA@ 1007e448     LIBCMT:setlocal.obj
 0002:00004450       ___lc_category             1007e450     LIBCMT:setlocal.obj
 0002:00004518       ??_C@_03EGDHDPFD@_?4?0?$AA@ 1007e518     LIBCMT:setlocal.obj
 0002:0000451c       ??_C@_01IDAFKMJL@_?$AA@    1007e51c     LIBCMT:setlocal.obj
 0002:00004520       ??_C@_01ICJEACDI@?$DL?$AA@ 1007e520     LIBCMT:setlocal.obj
 0002:00004524       ??_C@_01NEMOKFLO@?$DN?$AA@ 1007e524     LIBCMT:setlocal.obj
 0002:00004528       ??_C@_01GFHCPBMG@C?$AA@    1007e528     LIBCMT:setlocal.obj
 0002:0000452c       ??_C@_02BALPLPBG@?$DN?$DL?$AA@ 1007e52c     LIBCMT:setlocal.obj
 0002:00004530       ??_C@_0O@NLDKAIKN@EncodePointer?$AA@ 1007e530     LIBCMT:tidtable.obj
 0002:00004540       ??_C@_1BK@DBDEIDLH@?$AAK?$AAE?$AAR?$AAN?$AAE?$AAL?$AA3?$AA2?$AA?4?$AAD?$AAL?$AAL?$AA?$AA@ 1007e540     LIBCMT:tidtable.obj
 0002:0000455c       ??_C@_0O@KBPMFGHI@DecodePointer?$AA@ 1007e55c     LIBCMT:tidtable.obj
 0002:0000456c       ??_C@_07PEJMOBNF@FlsFree?$AA@ 1007e56c     LIBCMT:tidtable.obj
 0002:00004574       ??_C@_0M@JCPCPOEF@FlsSetValue?$AA@ 1007e574     LIBCMT:tidtable.obj
 0002:00004580       ??_C@_0M@GDNOONDI@FlsGetValue?$AA@ 1007e580     LIBCMT:tidtable.obj
 0002:0000458c       ??_C@_08KNHFBNJ@FlsAlloc?$AA@ 1007e58c     LIBCMT:tidtable.obj
 0002:000045a0       ??_C@_0P@GGKDKEEG@runtime?5error?5?$AA@ 1007e5a0     LIBCMT:crt0msg.obj
 0002:000045b0       ??_C@_02PCIJFNDE@?$AN?6?$AA@ 1007e5b0     LIBCMT:crt0msg.obj
 0002:000045b4       ??_C@_0O@MJNIPGOH@TLOSS?5error?$AN?6?$AA@ 1007e5b4     LIBCMT:crt0msg.obj
 0002:000045c4       ??_C@_0N@BONNPDHF@SING?5error?$AN?6?$AA@ 1007e5c4     LIBCMT:crt0msg.obj
 0002:000045d4       ??_C@_0P@MBDAJNE@DOMAIN?5error?$AN?6?$AA@ 1007e5d4     LIBCMT:crt0msg.obj
 0002:000045e8       ??_C@_0JL@DFDOOABL@R6034?$AN?6An?5application?5has?5made?5a@ 1007e5e8     LIBCMT:crt0msg.obj
 0002:00004688       ??_C@_0PH@EPAFIJ@R6033?$AN?6?9?5Attempt?5to?5use?5MSIL?5cod@ 1007e688     LIBCMT:crt0msg.obj
 0002:00004780       ??_C@_0DD@BKEEABMM@R6032?$AN?6?9?5not?5enough?5space?5for?5lo@ 1007e780     LIBCMT:crt0msg.obj
 0002:000047b8       ??_C@_0GD@OFKILIED@R6031?$AN?6?9?5Attempt?5to?5initialize?5t@ 1007e7b8     LIBCMT:crt0msg.obj
 0002:0000481c       ??_C@_0BP@LPMHJOKI@R6030?$AN?6?9?5CRT?5not?5initialized?$AN?6?$AA@ 1007e81c     LIBCMT:crt0msg.obj
 0002:0000483c       ??_C@_0CF@KJDAIALP@R6028?$AN?6?9?5unable?5to?5initialize?5he@ 1007e83c     LIBCMT:crt0msg.obj
 0002:00004864       ??_C@_0DF@GAKBPDFP@R6027?$AN?6?9?5not?5enough?5space?5for?5lo@ 1007e864     LIBCMT:crt0msg.obj
 0002:0000489c       ??_C@_0DF@IBLNNAIG@R6026?$AN?6?9?5not?5enough?5space?5for?5st@ 1007e89c     LIBCMT:crt0msg.obj
 0002:000048d4       ??_C@_0CG@IOHKGFNJ@R6025?$AN?6?9?5pure?5virtual?5function?5c@ 1007e8d4     LIBCMT:crt0msg.obj
 0002:000048fc       ??_C@_0DF@JIJJFJDC@R6024?$AN?6?9?5not?5enough?5space?5for?5_o@ 1007e8fc     LIBCMT:crt0msg.obj
 0002:00004934       ??_C@_0CJ@EGEJHFME@R6019?$AN?6?9?5unable?5to?5open?5console?5@ 1007e934     LIBCMT:crt0msg.obj
 0002:00004960       ??_C@_0CB@GNHNIELH@R6018?$AN?6?9?5unexpected?5heap?5error?$AN?6@ 1007e960     LIBCMT:crt0msg.obj
 0002:00004984       ??_C@_0CN@FOLDKNG@R6017?$AN?6?9?5unexpected?5multithread?5@ 1007e984     LIBCMT:crt0msg.obj
 0002:000049b4       ??_C@_0CM@FAHFJNHO@R6016?$AN?6?9?5not?5enough?5space?5for?5th@ 1007e9b4     LIBCMT:crt0msg.obj
 0002:000049e0       ??_C@_0JG@LBKMGKLD@?$AN?6This?5application?5has?5requested@ 1007e9e0     LIBCMT:crt0msg.obj
 0002:00004a78       ??_C@_0CM@FLCNIPKK@R6009?$AN?6?9?5not?5enough?5space?5for?5en@ 1007ea78     LIBCMT:crt0msg.obj
 0002:00004aa4       ??_C@_0CK@KMMJOAPP@R6008?$AN?6?9?5not?5enough?5space?5for?5ar@ 1007eaa4     LIBCMT:crt0msg.obj
 0002:00004ad0       ??_C@_0CN@LEKKICBM@R6002?$AN?6?9?5floating?5point?5support?5@ 1007ead0     LIBCMT:crt0msg.obj
 0002:00004b00       ??_C@_0CF@GOGNBNAK@Microsoft?5Visual?5C?$CL?$CL?5Runtime?5Lib@ 1007eb00     LIBCMT:crt0msg.obj
 0002:00004b28       ??_C@_02PHMGELLB@?6?6?$AA@ 1007eb28     LIBCMT:crt0msg.obj
 0002:00004b2c       ??_C@_03KHICJKCI@?4?4?4?$AA@ 1007eb2c     LIBCMT:crt0msg.obj
 0002:00004b30       ??_C@_0BH@DNAGHKFM@?$DMprogram?5name?5unknown?$DO?$AA@ 1007eb30     LIBCMT:crt0msg.obj
 0002:00004b48       ??_C@_0BK@OFGJDLJJ@Runtime?5Error?$CB?6?6Program?3?5?$AA@ 1007eb48     LIBCMT:crt0msg.obj
 0002:00005478       __DEFAULT_CW_in_mem        1007f478     LIBCMT:_common_.obj
 0002:0000547a       __pi_by_2_to_61            1007f47a     LIBCMT:_common_.obj
 0002:00008e00       __pDestructExceptionObject 10082e00     LIBCMT:frame.obj
 0002:00008e08       ??_7bad_exception@std@@6B@ 10082e08     LIBCMT:frame.obj
 0002:00008e10       ??_C@_0O@DPKOEFFH@bad?5exception?$AA@ 10082e10     LIBCMT:frame.obj
 0002:00008e20       ??_C@_1O@CEDCILHN@?$AA?$CI?$AAn?$AAu?$AAl?$AAl?$AA?$CJ?$AA?$AA@ 10082e20     LIBCMT:output.obj
 0002:00008e30       ??_C@_06OJHGLDPL@?$CInull?$CJ?$AA@ 10082e30     LIBCMT:output.obj
 0002:00008e38       ___lookuptable             10082e38     LIBCMT:output.obj
 0002:0000d160       ??_C@_0L@KDOEJCKC@_nextafter?$AA@ 10087160     LIBCMT:_fpexcept_.obj
 0002:0000d16c       ??_C@_05JGDBENOH@_logb?$AA@ 1008716c     LIBCMT:_fpexcept_.obj
 0002:0000d174       ??_C@_03ONILCKOB@_yn?$AA@  10087174     LIBCMT:_fpexcept_.obj
 0002:0000d178       ??_C@_03NAKIGLHK@_y1?$AA@  10087178     LIBCMT:_fpexcept_.obj
 0002:0000d17c       ??_C@_03MJLDFKDL@_y0?$AA@  1008717c     LIBCMT:_fpexcept_.obj
 0002:0000d180       ??_C@_05GKKHEGJL@frexp?$AA@ 10087180     LIBCMT:_fpexcept_.obj
 0002:0000d188       ??_C@_04KEPJIHGP@fmod?$AA@ 10087188     LIBCMT:_fpexcept_.obj
 0002:0000d190       ??_C@_06MEIMCGCF@_hypot?$AA@ 10087190     LIBCMT:_fpexcept_.obj
 0002:0000d198       ??_C@_05KBKMEMPO@_cabs?$AA@ 10087198     LIBCMT:_fpexcept_.obj
 0002:0000d1a0       ??_C@_05CEJMAHNP@ldexp?$AA@ 100871a0     LIBCMT:_fpexcept_.obj
 0002:0000d1a8       ??_C@_04EHEDPDJG@modf?$AA@ 100871a8     LIBCMT:_fpexcept_.obj
 0002:0000d1b0       ??_C@_04ODHECPBC@fabs?$AA@ 100871b0     LIBCMT:_fpexcept_.obj
 0002:0000d1b8       ??_C@_05PBJFFIGL@floor?$AA@ 100871b8     LIBCMT:_fpexcept_.obj
 0002:0000d1c0       ??_C@_04GFPJNGEK@ceil?$AA@ 100871c0     LIBCMT:_fpexcept_.obj
 0002:0000d1c8       ??_C@_03IIINPABG@tan?$AA@  100871c8     LIBCMT:_fpexcept_.obj
 0002:0000d1cc       ??_C@_03LALBNOCG@cos?$AA@  100871cc     LIBCMT:_fpexcept_.obj
 0002:0000d1d0       ??_C@_03BLEJJJBH@sin?$AA@  100871d0     LIBCMT:_fpexcept_.obj
 0002:0000d1d4       ??_C@_04EIAKFFMI@sqrt?$AA@ 100871d4     LIBCMT:_fpexcept_.obj
 0002:0000d1dc       ??_C@_05KNGEOGJB@atan2?$AA@ 100871dc     LIBCMT:_fpexcept_.obj
 0002:0000d1e4       ??_C@_04MLLJIGOK@atan?$AA@ 100871e4     LIBCMT:_fpexcept_.obj
 0002:0000d1ec       ??_C@_04PDIFKINK@acos?$AA@ 100871ec     LIBCMT:_fpexcept_.obj
 0002:0000d1f4       ??_C@_04FIHNOPOL@asin?$AA@ 100871f4     LIBCMT:_fpexcept_.obj
 0002:0000d1fc       ??_C@_04FJHINJAO@tanh?$AA@ 100871fc     LIBCMT:_fpexcept_.obj
 0002:0000d204       ??_C@_04HPJJNFIM@cosh?$AA@ 10087204     LIBCMT:_fpexcept_.obj
 0002:0000d20c       ??_C@_04COOMCNPB@sinh?$AA@ 1008720c     LIBCMT:_fpexcept_.obj
 0002:0000d214       ??_C@_05HGHHAHAP@log10?$AA@ 10087214     LIBCMT:_fpexcept_.obj
 0002:0000d21c       ??_C@_03MGHMBJCF@log?$AA@  1008721c     LIBCMT:_fpexcept_.obj
 0002:0000d220       ??_C@_03JGHBODFD@pow?$AA@  10087220     LIBCMT:_fpexcept_.obj
 0002:0000d224       ??_C@_03KHJOGHMM@exp?$AA@  10087224     LIBCMT:_fpexcept_.obj
 0002:0000d228       __XcptActTab               10087228     LIBCMT:winxfltr.obj
 0002:0000d308       ??_C@_05EOHGHCHD@exp10?$AA@ 10087308     LIBCMT:_libm_error_.obj
 0002:0000d310       ??_C@_13NOLLCAOD@?$AA?$AA?$AA?$AA@ 10087310     LIBCMT:a_map.obj
 0002:0000d314       ??_C@_0BG@KLEAJEFJ@Illegal?5byte?5sequence?$AA@ 10087314     LIBCMT:syserr.obj
 0002:0000d32c       ??_C@_0BE@ICMCHPHH@Directory?5not?5empty?$AA@ 1008732c     LIBCMT:syserr.obj
 0002:0000d340       ??_C@_0BJ@IHEHINLI@Function?5not?5implemented?$AA@ 10087340     LIBCMT:syserr.obj
 0002:0000d35c       ??_C@_0BD@CLHBCGPB@No?5locks?5available?$AA@ 1008735c     LIBCMT:syserr.obj
 0002:0000d370       ??_C@_0BC@BEDIHIDK@Filename?5too?5long?$AA@ 10087370     LIBCMT:syserr.obj
 0002:0000d384       ??_C@_0BK@JAEBMJJM@Resource?5deadlock?5avoided?$AA@ 10087384     LIBCMT:syserr.obj
 0002:0000d3a0       ??_C@_0BB@FCBJFCAJ@Result?5too?5large?$AA@ 100873a0     LIBCMT:syserr.obj
 0002:0000d3b4       ??_C@_0N@MMJPGLJK@Domain?5error?$AA@ 100873b4     LIBCMT:syserr.obj
 0002:0000d3c4       ??_C@_0M@LHEPIIOM@Broken?5pipe?$AA@ 100873c4     LIBCMT:syserr.obj
 0002:0000d3d0       ??_C@_0P@PKCJJLLM@Too?5many?5links?$AA@ 100873d0     LIBCMT:syserr.obj
 0002:0000d3e0       ??_C@_0BG@DDBFNKBH@Read?9only?5file?5system?$AA@ 100873e0     LIBCMT:syserr.obj
 0002:0000d3f8       ??_C@_0N@FEHLOILP@Invalid?5seek?$AA@ 100873f8     LIBCMT:syserr.obj
 0002:0000d408       ??_C@_0BI@FEALHKLD@No?5space?5left?5on?5device?$AA@ 10087408     LIBCMT:syserr.obj
 0002:0000d420       ??_C@_0P@LFMMIPAE@File?5too?5large?$AA@ 10087420     LIBCMT:syserr.obj
 0002:0000d430       ??_C@_0CE@ONOKNLPF@Inappropriate?5I?1O?5control?5operat@ 10087430     LIBCMT:syserr.obj
 0002:0000d454       ??_C@_0BE@INBJMKGG@Too?5many?5open?5files?$AA@ 10087454     LIBCMT:syserr.obj
 0002:0000d468       ??_C@_0BO@IIFBODJE@Too?5many?5open?5files?5in?5system?$AA@ 10087468     LIBCMT:syserr.obj
 0002:0000d488       ??_C@_0BB@HMGGCEBG@Invalid?5argument?$AA@ 10087488     LIBCMT:syserr.obj
 0002:0000d49c       ??_C@_0P@NDHGCGKE@Is?5a?5directory?$AA@ 1008749c     LIBCMT:syserr.obj
 0002:0000d4ac       ??_C@_0BA@CJBACOOL@Not?5a?5directory?$AA@ 100874ac     LIBCMT:syserr.obj
 0002:0000d4bc       ??_C@_0P@NLEIANHE@No?5such?5device?$AA@ 100874bc     LIBCMT:syserr.obj
 0002:0000d4cc       ??_C@_0O@OAMDNOCP@Improper?5link?$AA@ 100874cc     LIBCMT:syserr.obj
 0002:0000d4dc       ??_C@_0M@NAAJNNGH@File?5exists?$AA@ 100874dc     LIBCMT:syserr.obj
 0002:0000d4e8       ??_C@_0BA@BIBLIOEK@Resource?5device?$AA@ 100874e8     LIBCMT:syserr.obj
 0002:0000d4f8       ??_C@_0O@NIPGCINC@Unknown?5error?$AA@ 100874f8     LIBCMT:syserr.obj
 0002:0000d508       ??_C@_0M@LOEHLCJD@Bad?5address?$AA@ 10087508     LIBCMT:syserr.obj
 0002:0000d514       ??_C@_0BC@HFNFNKAI@Permission?5denied?$AA@ 10087514     LIBCMT:syserr.obj
 0002:0000d528       ??_C@_0BB@IMDKMPFB@Not?5enough?5space?$AA@ 10087528     LIBCMT:syserr.obj
 0002:0000d53c       ??_C@_0CB@EPFKGNAK@Resource?5temporarily?5unavailable@ 1008753c     LIBCMT:syserr.obj
 0002:0000d560       ??_C@_0BD@LOHELEP@No?5child?5processes?$AA@ 10087560     LIBCMT:syserr.obj
 0002:0000d574       ??_C@_0BE@NFGDDCEF@Bad?5file?5descriptor?$AA@ 10087574     LIBCMT:syserr.obj
 0002:0000d588       ??_C@_0BC@HKPNECK@Exec?5format?5error?$AA@ 10087588     LIBCMT:syserr.obj
 0002:0000d59c       ??_C@_0BC@MFFGCDFL@Arg?5list?5too?5long?$AA@ 1008759c     LIBCMT:syserr.obj
 0002:0000d5b0       ??_C@_0BK@DPKMCKJ@No?5such?5device?5or?5address?$AA@ 100875b0     LIBCMT:syserr.obj
 0002:0000d5cc       ??_C@_0BD@KKNFOBBD@Input?1output?5error?$AA@ 100875cc     LIBCMT:syserr.obj
 0002:0000d5e0       ??_C@_0BK@FJBOAFDK@Interrupted?5function?5call?$AA@ 100875e0     LIBCMT:syserr.obj
 0002:0000d5fc       ??_C@_0BA@FKIAIBGA@No?5such?5process?$AA@ 100875fc     LIBCMT:syserr.obj
 0002:0000d60c       ??_C@_0BK@FMDHKPNF@No?5such?5file?5or?5directory?$AA@ 1008760c     LIBCMT:syserr.obj
 0002:0000d628       ??_C@_0BI@BJFCGOHL@Operation?5not?5permitted?$AA@ 10087628     LIBCMT:syserr.obj
 0002:0000d640       ??_C@_08INEPGKHH@No?5error?$AA@ 10087640     LIBCMT:syserr.obj
 0002:0000d64c       ??_C@_0BC@JEAENNKH@SystemFunction036?$AA@ 1008764c     LIBCMT:rand_s.obj
 0002:0000d660       ??_C@_0N@JJPEKNFO@ADVAPI32?4DLL?$AA@ 10087660     LIBCMT:rand_s.obj
 0002:0000d670       ___newctype                10087670     LIBCMT:ctype.obj
 0002:0000d970       __wctype                   10087970     LIBCMT:ctype.obj
 0002:0000db78       ___newclmap                10087b78     LIBCMT:ctype.obj
 0002:0000dcf8       ___newcumap                10087cf8     LIBCMT:ctype.obj
 0002:0000de78       ??_C@_08JCCMCCIL@HH?3mm?3ss?$AA@ 10087e78     LIBCMT:strftime.obj
 0002:0000de84       ??_C@_0BE@CKGJFCPC@dddd?0?5MMMM?5dd?0?5yyyy?$AA@ 10087e84     LIBCMT:strftime.obj
 0002:0000de98       ??_C@_08BPBNCDIB@MM?1dd?1yy?$AA@ 10087e98     LIBCMT:strftime.obj
 0002:0000dea4       ??_C@_02CJNFDJBF@PM?$AA@   10087ea4     LIBCMT:strftime.obj
 0002:0000dea8       ??_C@_02DEDBPAFC@AM?$AA@   10087ea8     LIBCMT:strftime.obj
 0002:0000deac       ??_C@_08EDHMEBNP@December?$AA@ 10087eac     LIBCMT:strftime.obj
 0002:0000deb8       ??_C@_08HCHEGEOA@November?$AA@ 10087eb8     LIBCMT:strftime.obj
 0002:0000dec4       ??_C@_07JJNFCEND@October?$AA@ 10087ec4     LIBCMT:strftime.obj
 0002:0000decc       ??_C@_09BHHEALKD@September?$AA@ 10087ecc     LIBCMT:strftime.obj
 0002:0000ded8       ??_C@_06LBBHFDDG@August?$AA@ 10087ed8     LIBCMT:strftime.obj
 0002:0000dee0       ??_C@_04MIEPOIFP@July?$AA@ 10087ee0     LIBCMT:strftime.obj
 0002:0000dee8       ??_C@_04CNLMGBGM@June?$AA@ 10087ee8     LIBCMT:strftime.obj
 0002:0000def0       ??_C@_05DMJDNLEJ@April?$AA@ 10087ef0     LIBCMT:strftime.obj
 0002:0000def8       ??_C@_05HPCKOFNC@March?$AA@ 10087ef8     LIBCMT:strftime.obj
 0002:0000df00       ??_C@_08GNJGEPFN@February?$AA@ 10087f00     LIBCMT:strftime.obj
 0002:0000df0c       ??_C@_07CGJPFGJA@January?$AA@ 10087f0c     LIBCMT:strftime.obj
 0002:0000df14       ??_C@_03MKABNOCG@Dec?$AA@  10087f14     LIBCMT:strftime.obj
 0002:0000df18       ??_C@_03JPJOFNIA@Nov?$AA@  10087f18     LIBCMT:strftime.obj
 0002:0000df1c       ??_C@_03BMAOKBAD@Oct?$AA@  10087f1c     LIBCMT:strftime.obj
 0002:0000df20       ??_C@_03GGCAPAJC@Sep?$AA@  10087f20     LIBCMT:strftime.obj
 0002:0000df24       ??_C@_03IFJFEIGA@Aug?$AA@  10087f24     LIBCMT:strftime.obj
 0002:0000df28       ??_C@_03LBGABGKK@Jul?$AA@  10087f28     LIBCMT:strftime.obj
 0002:0000df2c       ??_C@_03IDFGHECI@Jun?$AA@  10087f2c     LIBCMT:strftime.obj
 0002:0000df30       ??_C@_03CNMDKL@May?$AA@    10087f30     LIBCMT:strftime.obj
 0002:0000df34       ??_C@_03LEOLGMJP@Apr?$AA@  10087f34     LIBCMT:strftime.obj
 0002:0000df38       ??_C@_03ODNJBKGA@Mar?$AA@  10087f38     LIBCMT:strftime.obj
 0002:0000df3c       ??_C@_03HJBDCHOM@Feb?$AA@  10087f3c     LIBCMT:strftime.obj
 0002:0000df40       ??_C@_03JIHJHPIE@Jan?$AA@  10087f40     LIBCMT:strftime.obj
 0002:0000df44       ??_C@_08INBOOONO@Saturday?$AA@ 10087f44     LIBCMT:strftime.obj
 0002:0000df50       ??_C@_06JECMNKMI@Friday?$AA@ 10087f50     LIBCMT:strftime.obj
 0002:0000df58       ??_C@_08HACCIKIA@Thursday?$AA@ 10087f58     LIBCMT:strftime.obj
 0002:0000df64       ??_C@_09DLIGFAKA@Wednesday?$AA@ 10087f64     LIBCMT:strftime.obj
 0002:0000df70       ??_C@_07BAAGCFCM@Tuesday?$AA@ 10087f70     LIBCMT:strftime.obj
 0002:0000df78       ??_C@_06JLEDEDGH@Monday?$AA@ 10087f78     LIBCMT:strftime.obj
 0002:0000df80       ??_C@_06OOPIFAJ@Sunday?$AA@ 10087f80     LIBCMT:strftime.obj
 0002:0000df88       ??_C@_03FEFJNEK@Sat?$AA@   10087f88     LIBCMT:strftime.obj
 0002:0000df8c       ??_C@_03IDIOELNC@Fri?$AA@  10087f8c     LIBCMT:strftime.obj
 0002:0000df90       ??_C@_03IOFIKPDN@Thu?$AA@  10087f90     LIBCMT:strftime.obj
 0002:0000df94       ??_C@_03MHOMLAJA@Wed?$AA@  10087f94     LIBCMT:strftime.obj
 0002:0000df98       ??_C@_03NAGEINEP@Tue?$AA@  10087f98     LIBCMT:strftime.obj
 0002:0000df9c       ??_C@_03PDAGKDH@Mon?$AA@   10087f9c     LIBCMT:strftime.obj
 0002:0000dfa0       ??_C@_03KOEHGMDN@Sun?$AA@  10087fa0     LIBCMT:strftime.obj
 0002:0000dfa4       ??_C@_03EBAPMIKO@a?1p?$AA@ 10087fa4     LIBCMT:strftime.obj
 0002:0000dfa8       ??_C@_05JAMEPDIN@am?1pm?$AA@ 10087fa8     LIBCMT:strftime.obj
 0002:0000dfb0       ??_C@_0O@FMJNFNKE@united?9states?$AA@ 10087fb0     LIBCMT:getqloc.obj
 0002:0000dfc0       ??_C@_0P@NDHFFKCA@united?9kingdom?$AA@ 10087fc0     LIBCMT:getqloc.obj
 0002:0000dfd0       ??_C@_0BC@HHDADLGF@trinidad?5?$CG?5tobago?$AA@ 10087fd0     LIBCMT:getqloc.obj
 0002:0000dfe4       ??_C@_0M@IOAEBDAC@south?9korea?$AA@ 10087fe4     LIBCMT:getqloc.obj
 0002:0000dff0       ??_C@_0N@FIELFKIJ@south?9africa?$AA@ 10087ff0     LIBCMT:getqloc.obj
 0002:0000e000       ??_C@_0M@OPNDHCMC@south?5korea?$AA@ 10088000     LIBCMT:getqloc.obj
 0002:0000e00c       ??_C@_0N@MDEOEPFI@south?5africa?$AA@ 1008800c     LIBCMT:getqloc.obj
 0002:0000e01c       ??_C@_06FKAPCJLB@slovak?$AA@ 1008801c     LIBCMT:getqloc.obj
 0002:0000e024       ??_C@_0M@EFJANOAL@puerto?9rico?$AA@ 10088024     LIBCMT:getqloc.obj
 0002:0000e030       ??_C@_08PGOJKDAI@pr?9china?$AA@ 10088030     LIBCMT:getqloc.obj
 0002:0000e03c       ??_C@_08JHDOMCMI@pr?5china?$AA@ 1008803c     LIBCMT:getqloc.obj
 0002:0000e048       ??_C@_02JHCHFBLL@nz?$AA@   10088048     LIBCMT:getqloc.obj
 0002:0000e04c       ??_C@_0M@LINHDHKP@new?9zealand?$AA@ 1008804c     LIBCMT:getqloc.obj
 0002:0000e058       ??_C@_09IIIPPBDB@hong?9kong?$AA@ 10088058     LIBCMT:getqloc.obj
 0002:0000e064       ??_C@_07HJLCKBG@holland?$AA@ 10088064     LIBCMT:getqloc.obj
 0002:0000e06c       ??_C@_0O@LEHGMHAG@great?5britain?$AA@ 1008806c     LIBCMT:getqloc.obj
 0002:0000e07c       ??_C@_07FACOMELA@england?$AA@ 1008807c     LIBCMT:getqloc.obj
 0002:0000e084       ??_C@_05JIHCEICB@czech?$AA@ 10088084     LIBCMT:getqloc.obj
 0002:0000e08c       ??_C@_05BBJOBLGB@china?$AA@ 1008808c     LIBCMT:getqloc.obj
 0002:0000e094       ??_C@_07GPKPHICP@britain?$AA@ 10088094     LIBCMT:getqloc.obj
 0002:0000e09c       ??_C@_07MHIPBHMG@america?$AA@ 1008809c     LIBCMT:getqloc.obj
 0002:0000e0a4       ??_C@_03KIALPMKC@usa?$AA@  100880a4     LIBCMT:getqloc.obj
 0002:0000e0a8       ??_C@_02FGJGKGGD@us?$AA@   100880a8     LIBCMT:getqloc.obj
 0002:0000e0ac       ??_C@_02NEINDODK@uk?$AA@   100880ac     LIBCMT:getqloc.obj
 0002:0000e0b0       ??_C@_05JMPCFJFJ@swiss?$AA@ 100880b0     LIBCMT:getqloc.obj
 0002:0000e0b8       ??_C@_0BA@HLOCPIOD@swedish?9finland?$AA@ 100880b8     LIBCMT:getqloc.obj
 0002:0000e0c8       ??_C@_0BC@PKCNIABK@spanish?9venezuela?$AA@ 100880c8     LIBCMT:getqloc.obj
 0002:0000e0dc       ??_C@_0BA@GBHHMIJI@spanish?9uruguay?$AA@ 100880dc     LIBCMT:getqloc.obj
 0002:0000e0ec       ??_C@_0BE@BHDOHPMC@spanish?9puerto?5rico?$AA@ 100880ec     LIBCMT:getqloc.obj
 0002:0000e100       ??_C@_0N@KMOIDGGN@spanish?9peru?$AA@ 10088100     LIBCMT:getqloc.obj
 0002:0000e110       ??_C@_0BB@HMHLPGPH@spanish?9paraguay?$AA@ 10088110     LIBCMT:getqloc.obj
 0002:0000e124       ??_C@_0P@MCPKNGFD@spanish?9panama?$AA@ 10088124     LIBCMT:getqloc.obj
 0002:0000e134       ??_C@_0BC@IHOHGAIL@spanish?9nicaragua?$AA@ 10088134     LIBCMT:getqloc.obj
 0002:0000e148       ??_C@_0P@KLMJDNFJ@spanish?9modern?$AA@ 10088148     LIBCMT:getqloc.obj
 0002:0000e158       ??_C@_0BA@BPAPGBCM@spanish?9mexican?$AA@ 10088158     LIBCMT:getqloc.obj
 0002:0000e168       ??_C@_0BB@PDECHHHE@spanish?9honduras?$AA@ 10088168     LIBCMT:getqloc.obj
 0002:0000e17c       ??_C@_0BC@KLHKFGDB@spanish?9guatemala?$AA@ 1008817c     LIBCMT:getqloc.obj
 0002:0000e190       ??_C@_0BE@MFOOKJAI@spanish?9el?5salvador?$AA@ 10088190     LIBCMT:getqloc.obj
 0002:0000e1a4       ??_C@_0BA@FCOKFPFC@spanish?9ecuador?$AA@ 100881a4     LIBCMT:getqloc.obj
 0002:0000e1b4       ??_C@_0BL@PLMGIMOO@spanish?9dominican?5republic?$AA@ 100881b4     LIBCMT:getqloc.obj
 0002:0000e1d0       ??_C@_0BD@HLGDNMHB@spanish?9costa?5rica?$AA@ 100881d0     LIBCMT:getqloc.obj
 0002:0000e1e4       ??_C@_0BB@PKCBKCPE@spanish?9colombia?$AA@ 100881e4     LIBCMT:getqloc.obj
 0002:0000e1f8       ??_C@_0O@MCBIJGNE@spanish?9chile?$AA@ 100881f8     LIBCMT:getqloc.obj
 0002:0000e208       ??_C@_0BA@BEFEIGJJ@spanish?9bolivia?$AA@ 10088208     LIBCMT:getqloc.obj
 0002:0000e218       ??_C@_0BC@EMECMPD@spanish?9argentina?$AA@ 10088218     LIBCMT:getqloc.obj
 0002:0000e22c       ??_C@_0BF@EALFLENP@portuguese?9brazilian?$AA@ 1008822c     LIBCMT:getqloc.obj
 0002:0000e244       ??_C@_0BC@HBLEBLNN@norwegian?9nynorsk?$AA@ 10088244     LIBCMT:getqloc.obj
 0002:0000e258       ??_C@_0BB@HMACDDCK@norwegian?9bokmal?$AA@ 10088258     LIBCMT:getqloc.obj
 0002:0000e26c       ??_C@_09BAFFPPHE@norwegian?$AA@ 1008826c     LIBCMT:getqloc.obj
 0002:0000e278       ??_C@_0O@EAJFJDFG@italian?9swiss?$AA@ 10088278     LIBCMT:getqloc.obj
 0002:0000e288       ??_C@_0O@CNOMPGD@irish?9english?$AA@ 10088288     LIBCMT:getqloc.obj
 0002:0000e298       ??_C@_0N@EDHBGCKG@german?9swiss?$AA@ 10088298     LIBCMT:getqloc.obj
 0002:0000e2a8       ??_C@_0BC@JACMHNBP@german?9luxembourg?$AA@ 100882a8     LIBCMT:getqloc.obj
 0002:0000e2bc       ??_C@_0BE@HBGMGFEG@german?9lichtenstein?$AA@ 100882bc     LIBCMT:getqloc.obj
 0002:0000e2d0       ??_C@_0BA@HKKBIBKL@german?9austrian?$AA@ 100882d0     LIBCMT:getqloc.obj
 0002:0000e2e0       ??_C@_0N@GCAEPEBK@french?9swiss?$AA@ 100882e0     LIBCMT:getqloc.obj
 0002:0000e2f0       ??_C@_0BC@DJFJJCK@french?9luxembourg?$AA@ 100882f0     LIBCMT:getqloc.obj
 0002:0000e304       ??_C@_0BA@NNCEDFIC@french?9canadian?$AA@ 10088304     LIBCMT:getqloc.obj
 0002:0000e314       ??_C@_0P@CMPOCLM@french?9belgian?$AA@ 10088314     LIBCMT:getqloc.obj
 0002:0000e324       ??_C@_0M@GHHDJOK@english?9usa?$AA@ 10088324     LIBCMT:getqloc.obj
 0002:0000e330       ??_C@_0L@PLDJKEIL@english?9us?$AA@ 10088330     LIBCMT:getqloc.obj
 0002:0000e33c       ??_C@_0L@HJCCDMNC@english?9uk?$AA@ 1008833c     LIBCMT:getqloc.obj
 0002:0000e348       ??_C@_0BK@CKLIAGJB@english?9trinidad?5y?5tobago?$AA@ 10088348     LIBCMT:getqloc.obj
 0002:0000e364       ??_C@_0BF@JMJMGNNF@english?9south?5africa?$AA@ 10088364     LIBCMT:getqloc.obj
 0002:0000e37c       ??_C@_0L@DKIIFDFD@english?9nz?$AA@ 1008837c     LIBCMT:getqloc.obj
 0002:0000e388       ??_C@_0BA@ONHGJCLH@english?9jamaica?$AA@ 10088388     LIBCMT:getqloc.obj
 0002:0000e398       ??_C@_0M@HJBGHOPO@english?9ire?$AA@ 10088398     LIBCMT:getqloc.obj
 0002:0000e3a4       ??_C@_0BC@LFEKMIFB@english?9caribbean?$AA@ 100883a4     LIBCMT:getqloc.obj
 0002:0000e3b8       ??_C@_0M@OLDPFKHI@english?9can?$AA@ 100883b8     LIBCMT:getqloc.obj
 0002:0000e3c4       ??_C@_0P@OMDEHBMP@english?9belize?$AA@ 100883c4     LIBCMT:getqloc.obj
 0002:0000e3d4       ??_C@_0M@KFHFPFED@english?9aus?$AA@ 100883d4     LIBCMT:getqloc.obj
 0002:0000e3e0       ??_C@_0BB@MNMBKDFE@english?9american?$AA@ 100883e0     LIBCMT:getqloc.obj
 0002:0000e3f4       ??_C@_0O@KIDLNNBA@dutch?9belgian?$AA@ 100883f4     LIBCMT:getqloc.obj
 0002:0000e404       ??_C@_0BE@JBKABBMH@chinese?9traditional?$AA@ 10088404     LIBCMT:getqloc.obj
 0002:0000e418       ??_C@_0BC@MJJMPKCG@chinese?9singapore?$AA@ 10088418     LIBCMT:getqloc.obj
 0002:0000e42c       ??_C@_0BD@FDKADDCP@chinese?9simplified?$AA@ 1008842c     LIBCMT:getqloc.obj
 0002:0000e440       ??_C@_0BB@DBEFDDME@chinese?9hongkong?$AA@ 10088440     LIBCMT:getqloc.obj
 0002:0000e454       ??_C@_07DHNMFMCI@chinese?$AA@ 10088454     LIBCMT:getqloc.obj
 0002:0000e45c       ??_C@_03FNDDCHI@chi?$AA@   1008845c     LIBCMT:getqloc.obj
 0002:0000e460       ??_C@_03BMMIADDJ@chh?$AA@  10088460     LIBCMT:getqloc.obj
 0002:0000e464       ??_C@_08OAIPJDGI@canadian?$AA@ 10088464     LIBCMT:getqloc.obj
 0002:0000e470       ??_C@_07HBPMNPNJ@belgian?$AA@ 10088470     LIBCMT:getqloc.obj
 0002:0000e478       ??_C@_0L@OEKOPBEL@australian?$AA@ 10088478     LIBCMT:getqloc.obj
 0002:0000e484       ??_C@_0BB@MEIMBEDG@american?9english?$AA@ 10088484     LIBCMT:getqloc.obj
 0002:0000e498       ??_C@_0BB@DFMDPDGB@american?5english?$AA@ 10088498     LIBCMT:getqloc.obj
 0002:0000e4ac       ??_C@_08IJLOKOLL@american?$AA@ 100884ac     LIBCMT:getqloc.obj
 0002:0000e4b8       ___rg_language             100884b8     LIBCMT:getqloc.obj
 0002:0000e6c0       ___rg_country              100886c0     LIBCMT:getqloc.obj
 0002:0000e778       ___rglangidNotDefault      10088778     LIBCMT:getqloc.obj
 0002:0000e78c       ??_C@_01GBGANLPD@0?$AA@    1008878c     LIBCMT:getqloc.obj
 0002:0000e790       ??_C@_03NFKLAGEF@OCP?$AA@  10088790     LIBCMT:getqloc.obj
 0002:0000e794       ??_C@_03DFHEHBHG@ACP?$AA@  10088794     LIBCMT:getqloc.obj
 0002:0000e798       ??_C@_0BC@NFIEMBLL@Norwegian?9Nynorsk?$AA@ 10088798     LIBCMT:getqloc.obj
 0002:0000e7ac       ??_C@_0BI@DFKBFLJE@GetProcessWindowStation?$AA@ 100887ac     LIBCMT:crtmbox.obj
 0002:0000e7c4       ??_C@_0BK@CIDNPOGP@GetUserObjectInformationA?$AA@ 100887c4     LIBCMT:crtmbox.obj
 0002:0000e7e0       ??_C@_0BD@HHGDFDBJ@GetLastActivePopup?$AA@ 100887e0     LIBCMT:crtmbox.obj
 0002:0000e7f4       ??_C@_0BA@HNOPNCHB@GetActiveWindow?$AA@ 100887f4     LIBCMT:crtmbox.obj
 0002:0000e804       ??_C@_0M@CHKKJDAI@MessageBoxA?$AA@ 10088804     LIBCMT:crtmbox.obj
 0002:0000e810       ??_C@_0L@NDEGIDAG@USER32?4DLL?$AA@ 10088810     LIBCMT:crtmbox.obj
 0002:0000e81c       ??_C@_0BK@CFCOFLF@?5Complete?5Object?5Locator?8?$AA@ 1008881c     LIBCMT:undname.obj
 0002:0000e838       ??_C@_0BN@MECKDCOJ@?5Class?5Hierarchy?5Descriptor?8?$AA@ 10088838     LIBCMT:undname.obj
 0002:0000e858       ??_C@_0BD@LGICGFMM@?5Base?5Class?5Array?8?$AA@ 10088858     LIBCMT:undname.obj
 0002:0000e86c       ??_C@_0BM@LDKODKLH@?5Base?5Class?5Descriptor?5at?5?$CI?$AA@ 1008886c     LIBCMT:undname.obj
 0002:0000e888       ??_C@_0BC@DAFEJGAK@?5Type?5Descriptor?8?$AA@ 10088888     LIBCMT:undname.obj
 0002:0000e89c       ??_C@_0BM@PMGGMLDN@?$GAlocal?5static?5thread?5guard?8?$AA@ 1008889c     LIBCMT:undname.obj
 0002:0000e8b8       ??_C@_0CL@FGIJHLCE@?$GAmanaged?5vector?5copy?5constructor@ 100888b8     LIBCMT:undname.obj
 0002:0000e8e4       ??_C@_0CJ@GJELGAMM@?$GAvector?5vbase?5copy?5constructor?5i@ 100888e4     LIBCMT:undname.obj
 0002:0000e910       ??_C@_0CD@CGAJBKEJ@?$GAvector?5copy?5constructor?5iterato@ 10088910     LIBCMT:undname.obj
 0002:0000e934       ??_C@_0CB@PDBIFEP@?$GAdynamic?5atexit?5destructor?5for?5?8@ 10088934     LIBCMT:undname.obj
 0002:0000e958       ??_C@_0BL@CLIPGLGB@?$GAdynamic?5initializer?5for?5?8?$AA@ 10088958     LIBCMT:undname.obj
 0002:0000e974       ??_C@_0CM@FCBBDIGB@?$GAeh?5vector?5vbase?5copy?5constructo@ 10088974     LIBCMT:undname.obj
 0002:0000e9a0       ??_C@_0CG@HLDDJMAG@?$GAeh?5vector?5copy?5constructor?5iter@ 100889a0     LIBCMT:undname.obj
 0002:0000e9c8       ??_C@_0CF@IMGKMJNO@?$GAmanaged?5vector?5destructor?5itera@ 100889c8     LIBCMT:undname.obj
 0002:0000e9f0       ??_C@_0CG@CFDHKGGD@?$GAmanaged?5vector?5constructor?5iter@ 100889f0     LIBCMT:undname.obj
 0002:0000ea18       ??_C@_0BN@CKNJLHMB@?$GAplacement?5delete?$FL?$FN?5closure?8?$AA@ 10088a18     LIBCMT:undname.obj
 0002:0000ea38       ??_C@_0BL@CNOONJFP@?$GAplacement?5delete?5closure?8?$AA@ 10088a38     LIBCMT:undname.obj
 0002:0000ea54       ??_C@_0P@HJKNJFNN@?$GAomni?5callsig?8?$AA@ 10088a54     LIBCMT:undname.obj
 0002:0000ea64       ??_C@_09LBNFPBCA@?5delete?$FL?$FN?$AA@ 10088a64     LIBCMT:undname.obj
 0002:0000ea70       ??_C@_06FHBGPFGH@?5new?$FL?$FN?$AA@ 10088a70     LIBCMT:undname.obj
 0002:0000ea78       ??_C@_0CE@IIHCMGGL@?$GAlocal?5vftable?5constructor?5closu@ 10088a78     LIBCMT:undname.obj
 0002:0000ea9c       ??_C@_0BA@KKLDJDLB@?$GAlocal?5vftable?8?$AA@ 10088a9c     LIBCMT:undname.obj
 0002:0000eaac       ??_C@_05KHLCHHI@?$GARTTI?$AA@ 10088aac     LIBCMT:undname.obj
 0002:0000eab4       ??_C@_03KLGMFNMG@?$GAEH?$AA@ 10088ab4     LIBCMT:undname.obj
 0002:0000eab8       ??_C@_0BA@KBCDOMBN@?$GAudt?5returning?8?$AA@ 10088ab8     LIBCMT:undname.obj
 0002:0000eac8       ??_C@_0BL@LLKPOHJI@?$GAcopy?5constructor?5closure?8?$AA@ 10088ac8     LIBCMT:undname.obj
 0002:0000eae4       ??_C@_0CH@OOJPLCPH@?$GAeh?5vector?5vbase?5constructor?5ite@ 10088ae4     LIBCMT:undname.obj
 0002:0000eb0c       ??_C@_0CA@GCEOPDGL@?$GAeh?5vector?5destructor?5iterator?8?$AA@ 10088b0c     LIBCMT:undname.obj
 0002:0000eb2c       ??_C@_0CB@JONCMFFK@?$GAeh?5vector?5constructor?5iterator?8@ 10088b2c     LIBCMT:undname.obj
 0002:0000eb50       ??_C@_0BL@NILFHHPC@?$GAvirtual?5displacement?5map?8?$AA@ 10088b50     LIBCMT:undname.obj
 0002:0000eb6c       ??_C@_0CE@IKBNEHA@?$GAvector?5vbase?5constructor?5iterat@ 10088b6c     LIBCMT:undname.obj
 0002:0000eb90       ??_C@_0BN@LFPFMEDL@?$GAvector?5destructor?5iterator?8?$AA@ 10088b90     LIBCMT:undname.obj
 0002:0000ebb0       ??_C@_0BO@PFGOCPJJ@?$GAvector?5constructor?5iterator?8?$AA@ 10088bb0     LIBCMT:undname.obj
 0002:0000ebd0       ??_C@_0BN@IMDCHIKM@?$GAscalar?5deleting?5destructor?8?$AA@ 10088bd0     LIBCMT:undname.obj
 0002:0000ebf0       ??_C@_0BO@OBMKPJIG@?$GAdefault?5constructor?5closure?8?$AA@ 10088bf0     LIBCMT:undname.obj
 0002:0000ec10       ??_C@_0BN@DEGPLNFK@?$GAvector?5deleting?5destructor?8?$AA@ 10088c10     LIBCMT:undname.obj
 0002:0000ec30       ??_C@_0BD@JDLKDPAB@?$GAvbase?5destructor?8?$AA@ 10088c30     LIBCMT:undname.obj
 0002:0000ec44       ??_C@_08OBABFOLI@?$GAstring?8?$AA@ 10088c44     LIBCMT:undname.obj
 0002:0000ec50       ??_C@_0BF@KDPPACIK@?$GAlocal?5static?5guard?8?$AA@ 10088c50     LIBCMT:undname.obj
 0002:0000ec68       ??_C@_08LLFFHHDJ@?$GAtypeof?8?$AA@ 10088c68     LIBCMT:undname.obj
 0002:0000ec74       ??_C@_07FEEIOKP@?$GAvcall?8?$AA@ 10088c74     LIBCMT:undname.obj
 0002:0000ec7c       ??_C@_09BLBHBJP@?$GAvbtable?8?$AA@ 10088c7c     LIBCMT:undname.obj
 0002:0000ec88       ??_C@_09IFPLHPGF@?$GAvftable?8?$AA@ 10088c88     LIBCMT:undname.obj
 0002:0000ec94       ??_C@_02MHEGNOJ@?$FO?$DN?$AA@ 10088c94     LIBCMT:undname.obj
 0002:0000ec98       ??_C@_02DHLNPPGH@?$HM?$DN?$AA@ 10088c98     LIBCMT:undname.obj
 0002:0000ec9c       ??_C@_02FGJGFEAB@?$CG?$DN?$AA@ 10088c9c     LIBCMT:undname.obj
 0002:0000eca0       ??_C@_03CDNPDDLA@?$DM?$DM?$DN?$AA@ 10088ca0     LIBCMT:undname.obj
 0002:0000eca4       ??_C@_03IKFCCPFF@?$DO?$DO?$DN?$AA@ 10088ca4     LIBCMT:undname.obj
 0002:0000eca8       ??_C@_02FENAOKFI@?$CF?$DN?$AA@ 10088ca8     LIBCMT:undname.obj
 0002:0000ecac       ??_C@_02FJEHGPIO@?1?$DN?$AA@ 10088cac     LIBCMT:undname.obj
 0002:0000ecb0       ??_C@_02FKMDLLOA@?9?$DN?$AA@ 10088cb0     LIBCMT:undname.obj
 0002:0000ecb4       ??_C@_02FOEOMHFC@?$CL?$DN?$AA@ 10088cb4     LIBCMT:undname.obj
 0002:0000ecb8       ??_C@_02FPIMKNGF@?$CK?$DN?$AA@ 10088cb8     LIBCMT:undname.obj
 0002:0000ecbc       ??_C@_02NONPIBCD@?$HM?$HM?$AA@ 10088cbc     LIBCMT:undname.obj
 0002:0000ecc0       ??_C@_02PPKAJPJL@?$CG?$CG?$AA@ 10088cc0     LIBCMT:undname.obj
 0002:0000ecc4       ??_C@_01DNKMNLPK@?$HM?$AA@ 10088cc4     LIBCMT:undname.obj
 0002:0000ecc8       ??_C@_01JKBOJNNK@?$FO?$AA@ 10088cc8     LIBCMT:undname.obj
 0002:0000eccc       ??_C@_01PJKLJHI@?$HO?$AA@  10088ccc     LIBCMT:undname.obj
 0002:0000ecd0       ??_C@_02HCKGKOFO@?$CI?$CJ?$AA@ 10088cd0     LIBCMT:undname.obj
 0002:0000ecd4       ??_C@_01IHBHIGKO@?0?$AA@   10088cd4     LIBCMT:undname.obj
 0002:0000ecd8       ??_C@_02EEKDKGMJ@?$DO?$DN?$AA@ 10088cd8     LIBCMT:undname.obj
 0002:0000ecdc       ??_C@_01PPODPGHN@?$DO?$AA@ 10088cdc     LIBCMT:undname.obj
 0002:0000ece0       ??_C@_02EHCHHCKH@?$DM?$DN?$AA@ 10088ce0     LIBCMT:undname.obj
 0002:0000ece4       ??_C@_01MNNFJEPP@?$DM?$AA@ 10088ce4     LIBCMT:undname.obj
 0002:0000ece8       ??_C@_01FGNFDNOH@?$CF?$AA@ 10088ce8     LIBCMT:undname.obj
 0002:0000ecec       ??_C@_01KMDKNFGN@?1?$AA@   10088cec     LIBCMT:undname.obj
 0002:0000ecf0       ??_C@_03MNHNFDLC@?9?$DO?$CK?$AA@ 10088cf0     LIBCMT:undname.obj
 0002:0000ecf4       ??_C@_01HNPIGOCE@?$CG?$AA@ 10088cf4     LIBCMT:undname.obj
 0002:0000ecf8       ??_C@_01MIFGBAGJ@?$CL?$AA@ 10088cf8     LIBCMT:undname.obj
 0002:0000ecfc       ??_C@_01JOAMLHOP@?9?$AA@   10088cfc     LIBCMT:undname.obj
 0002:0000ed00       ??_C@_02BAABKJLB@?9?9?$AA@ 10088d00     LIBCMT:undname.obj
 0002:0000ed04       ??_C@_02ECNGHCIF@?$CL?$CL?$AA@ 10088d04     LIBCMT:undname.obj
 0002:0000ed08       ??_C@_01NBENCBCI@?$CK?$AA@ 10088d08     LIBCMT:undname.obj
 0002:0000ed0c       ??_C@_02HBOOOICD@?9?$DO?$AA@ 10088d0c     LIBCMT:undname.obj
 0002:0000ed10       ??_C@_08LHJFAFGD@operator?$AA@ 10088d10     LIBCMT:undname.obj
 0002:0000ed1c       ??_C@_02GPECMEKF@?$FL?$FN?$AA@ 10088d1c     LIBCMT:undname.obj
 0002:0000ed20       ??_C@_02FDNJECIE@?$CB?$DN?$AA@ 10088d20     LIBCMT:undname.obj
 0002:0000ed24       ??_C@_02EGOFBIJA@?$DN?$DN?$AA@ 10088d24     LIBCMT:undname.obj
 0002:0000ed28       ??_C@_01DCLJPIOD@?$CB?$AA@ 10088d28     LIBCMT:undname.obj
 0002:0000ed2c       ??_C@_02FODMEDOG@?$DM?$DM?$AA@ 10088d2c     LIBCMT:undname.obj
 0002:0000ed30       ??_C@_02GPIOPFAK@?$DO?$DO?$AA@ 10088d30     LIBCMT:undname.obj
 0002:0000ed34       ??_C@_07FPCDHGMM@?5delete?$AA@ 10088d34     LIBCMT:undname.obj
 0002:0000ed3c       ??_C@_04NIHEBCM@?5new?$AA@ 10088d3c     LIBCMT:undname.obj
 0002:0000ed44       ??_C@_0M@GFIIJFMG@__unaligned?$AA@ 10088d44     LIBCMT:undname.obj
 0002:0000ed50       ??_C@_0L@PILCLIHE@__restrict?$AA@ 10088d50     LIBCMT:undname.obj
 0002:0000ed5c       ??_C@_07JOMMBBKO@__ptr64?$AA@ 10088d5c     LIBCMT:undname.obj
 0002:0000ed64       ??_C@_09HIJEGCPM@__clrcall?$AA@ 10088d64     LIBCMT:undname.obj
 0002:0000ed70       ??_C@_0L@JMKHOMEK@__fastcall?$AA@ 10088d70     LIBCMT:undname.obj
 0002:0000ed7c       ??_C@_0L@NPHFGOKO@__thiscall?$AA@ 10088d7c     LIBCMT:undname.obj
 0002:0000ed88       ??_C@_09IFJBGAPI@__stdcall?$AA@ 10088d88     LIBCMT:undname.obj
 0002:0000ed94       ??_C@_08GHMPAG@__pascal?$AA@ 10088d94     LIBCMT:undname.obj
 0002:0000eda0       ??_C@_07KOLFKCDI@__cdecl?$AA@ 10088da0     LIBCMT:undname.obj
 0002:0000eda8       ??_C@_08EHJDFFNH@__based?$CI?$AA@ 10088da8     LIBCMT:undname.obj
 0002:0000ef38       ??_7DNameNode@@6B@         10088f38     LIBCMT:undname.obj
 0002:0000ef44       ??_7charNode@@6B@          10088f44     LIBCMT:undname.obj
 0002:0000ef50       ??_7pDNameNode@@6B@        10088f50     LIBCMT:undname.obj
 0002:0000ef5c       ??_7DNameStatusNode@@6B@   10088f5c     LIBCMT:undname.obj
 0002:0000ef68       ??_7pairNode@@6B@          10088f68     LIBCMT:undname.obj
 0002:0000ef74       ??_7pcharNode@@6B@         10088f74     LIBCMT:undname.obj
 0002:0000ef80       ??_C@_04OKOHEJBO@?5?$DP?$DP?5?$AA@ 10088f80     LIBCMT:undname.obj
 0002:0000ef88       ??_C@_06EEGAIFAK@?$HLflat?$HN?$AA@ 10088f88     LIBCMT:undname.obj
 0002:0000ef90       ??_C@_05JIBOFOHK@?$HLfor?5?$AA@ 10088f90     LIBCMT:undname.obj
 0002:0000ef98       ??_C@_0BN@IBLMMFAP@?$GAnon?9type?9template?9parameter?$AA@ 10088f98     LIBCMT:undname.obj
 0002:0000efb8       ??_C@_09EBBEKKIH@unsigned?5?$AA@ 10088fb8     LIBCMT:undname.obj
 0002:0000efc4       ??_C@_05CJIMAING@long?5?$AA@ 10088fc4     LIBCMT:undname.obj
 0002:0000efcc       ??_C@_04LAHKHJMA@int?5?$AA@ 10088fcc     LIBCMT:undname.obj
 0002:0000efd4       ??_C@_06EHJMALKF@short?5?$AA@ 10088fd4     LIBCMT:undname.obj
 0002:0000efdc       ??_C@_05CIHEBHNO@char?5?$AA@ 10088fdc     LIBCMT:undname.obj
 0002:0000efe4       ??_C@_04GKJNKENE@void?$AA@ 10088fe4     LIBCMT:undname.obj
 0002:0000efec       ??_C@_0L@EGPHHEKN@?$DMellipsis?$DO?$AA@ 10088fec     LIBCMT:undname.obj
 0002:0000eff8       ??_C@_0M@ELJOJFFH@?0?$DMellipsis?$DO?$AA@ 10088ff8     LIBCMT:undname.obj
 0002:0000f004       ??_C@_04EENFHACM@?0?4?4?4?$AA@ 10089004     LIBCMT:undname.obj
 0002:0000f00c       ??_C@_07HDJPLPEK@?5throw?$CI?$AA@ 1008900c     LIBCMT:undname.obj
 0002:0000f014       ??_C@_02GOGNNPBN@?$CJ?$FL?$AA@ 10089014     LIBCMT:undname.obj
 0002:0000f018       ??_C@_02MDINNEEG@s?5?$AA@  10089018     LIBCMT:undname.obj
 0002:0000f01c       ??_C@_0BE@EODMJLIF@?$GAtemplate?9parameter?$AA@ 1008901c     LIBCMT:undname.obj
 0002:0000f030       ??_C@_01GEODFPGF@?8?$AA@   10089030     LIBCMT:undname.obj
 0002:0000f034       ??_C@_04HIBGFPH@NULL?$AA@  10089034     LIBCMT:undname.obj
 0002:0000f03c       ??_C@_0O@GKABPPIF@cli?3?3pin_ptr?$DM?$AA@ 1008903c     LIBCMT:undname.obj
 0002:0000f04c       ??_C@_0M@EALIELKG@cli?3?3array?$DM?$AA@ 1008904c     LIBCMT:undname.obj
 0002:0000f058       ??_C@_05BEFAKPML@void?5?$AA@ 10089058     LIBCMT:undname.obj
 0002:0000f060       ??_C@_02OHHJMEON@?8?8?$AA@ 10089060     LIBCMT:undname.obj
 0002:0000f064       ??_C@_0BG@JNJLAMPM@?$GAanonymous?5namespace?8?$AA@ 10089064     LIBCMT:undname.obj
 0002:0000f07c       ??_C@_01NLNLIGKH@?$GA?$AA@ 1008907c     LIBCMT:undname.obj
 0002:0000f080       ??_C@_0O@KHGCOMHP@generic?9type?9?$AA@ 10089080     LIBCMT:undname.obj
 0002:0000f090       ??_C@_0BE@JAEOCHPE@template?9parameter?9?$AA@ 10089090     LIBCMT:undname.obj
 0002:0000f0a4       ??_C@_02MOLJINC@?3?3?$AA@  100890a4     LIBCMT:undname.obj
 0002:0000f0a8       ??_C@_0P@GCIFDJCJ@?$GAunknown?5ecsu?8?$AA@ 100890a8     LIBCMT:undname.obj
 0002:0000f0b8       ??_C@_06MOJHIBMG@union?5?$AA@ 100890b8     LIBCMT:undname.obj
 0002:0000f0c0       ??_C@_07DIBCDNGL@struct?5?$AA@ 100890c0     LIBCMT:undname.obj
 0002:0000f0c8       ??_C@_06LJBABKPM@class?5?$AA@ 100890c8     LIBCMT:undname.obj
 0002:0000f0d0       ??_C@_05LJGMCFOG@enum?5?$AA@ 100890d0     LIBCMT:undname.obj
 0002:0000f0d8       ??_C@_08KOFANOFK@coclass?5?$AA@ 100890d8     LIBCMT:undname.obj
 0002:0000f0e4       ??_C@_0N@DLIEFKNA@cointerface?5?$AA@ 100890e4     LIBCMT:undname.obj
 0002:0000f0f4       ??_C@_02KCKGHPCA@?$CJ?5?$AA@ 100890f4     LIBCMT:undname.obj
 0002:0000f0f8       ??_C@_0M@DHNBOJMP@extern?5?$CCC?$CC?5?$AA@ 100890f8     LIBCMT:undname.obj
 0002:0000f104       ??_C@_08KJLFOPNE@?$FLthunk?$FN?3?$AA@ 10089104     LIBCMT:undname.obj
 0002:0000f110       ??_C@_08GPDDCMKI@public?3?5?$AA@ 10089110     LIBCMT:undname.obj
 0002:0000f11c       ??_C@_0M@GAIFPFIP@protected?3?5?$AA@ 1008911c     LIBCMT:undname.obj
 0002:0000f128       ??_C@_09LAPHOOG@private?3?5?$AA@ 10089128     LIBCMT:undname.obj
 0002:0000f134       ??_C@_08NIEOINHE@virtual?5?$AA@ 10089134     LIBCMT:undname.obj
 0002:0000f140       ??_C@_07PGOEDBHP@static?5?$AA@ 10089140     LIBCMT:undname.obj
 0002:0000f148       ??_C@_0DA@HGFJFBBE@?$GAtemplate?5static?5data?5member?5des@ 10089148     LIBCMT:undname.obj
 0002:0000f178       ??_C@_0DB@ILEFOCIJ@?$GAtemplate?5static?5data?5member?5con@ 10089178     LIBCMT:undname.obj
 0002:0000f1ac       ??_C@_0CB@KJDOOODE@?$GAlocal?5static?5destructor?5helper?8@ 100891ac     LIBCMT:undname.obj
 0002:0000f1d0       ??_C@_0L@HNGCOGAE@?$GAadjustor?$HL?$AA@ 100891d0     LIBCMT:undname.obj
 0002:0000f1dc       ??_C@_0L@GHPFDFH@?$GAvtordisp?$HL?$AA@ 100891dc     LIBCMT:undname.obj
 0002:0000f1e8       ??_C@_0N@CBHHHENL@?$GAvtordispex?$HL?$AA@ 100891e8     LIBCMT:undname.obj
 0002:0000f1f8       ??_C@_01CLKCMJKC@?5?$AA@   100891f8     LIBCMT:undname.obj
 0002:0000f1fc       ??_C@_02IGFCGPIL@?$HN?8?$AA@ 100891fc     LIBCMT:undname.obj
 0002:0000f200       ??_C@_03OPGICMGF@?$HN?8?5?$AA@ 10089200     LIBCMT:undname.obj
 0002:0000f204       ??_C@_06LIJLOJAG@const?5?$AA@ 10089204     LIBCMT:undname.obj
 0002:0000f20c       ??_C@_09GAIEOBLP@volatile?5?$AA@ 1008920c     LIBCMT:undname.obj
 0002:0000f218       ??_C@_04HEJADOOB@CV?3?5?$AA@ 10089218     LIBCMT:undname.obj
 0002:0000f220       ??_C@_08PABEKFH@volatile?$AA@ 10089220     LIBCMT:undname.obj
 0002:0000f22c       ??_C@_09EFNPDFFP@?5volatile?$AA@ 1008922c     LIBCMT:undname.obj
 0002:0000f238       ??_C@_05BNCCCJPP@const?$AA@ 10089238     LIBCMT:undname.obj
 0002:0000f240       ??_C@_07EDHNAJHC@signed?5?$AA@ 10089240     LIBCMT:undname.obj
 0002:0000f248       ??_C@_06BNJCAIGJ@double?$AA@ 10089248     LIBCMT:undname.obj
 0002:0000f250       ??_C@_07NFANNNEC@UNKNOWN?$AA@ 10089250     LIBCMT:undname.obj
 0002:0000f258       ??_C@_08GAHOLHEO@__int128?$AA@ 10089258     LIBCMT:undname.obj
 0002:0000f264       ??_C@_04DDKJGDCM@bool?$AA@ 10089264     LIBCMT:undname.obj
 0002:0000f26c       ??_C@_07CLGGIAMF@wchar_t?$AA@ 1008926c     LIBCMT:undname.obj
 0002:0000f274       ??_C@_07LFCOJCAC@__int64?$AA@ 10089274     LIBCMT:undname.obj
 0002:0000f27c       ??_C@_07ICFHOGAF@__int16?$AA@ 1008927c     LIBCMT:undname.obj
 0002:0000f284       ??_C@_07OFLPPHGP@__int32?$AA@ 10089284     LIBCMT:undname.obj
 0002:0000f28c       ??_C@_06EBGKOKIG@__int8?$AA@ 1008928c     LIBCMT:undname.obj
 0002:0000f294       ??_C@_06GCICPBLB@__w64?5?$AA@ 10089294     LIBCMT:undname.obj
 0002:0000f29c       ??_C@_05KNFBNCOH@float?$AA@ 1008929c     LIBCMT:undname.obj
 0002:0000f2a4       ??_C@_04GOKPGOLB@long?$AA@ 100892a4     LIBCMT:undname.obj
 0002:0000f2ac       ??_C@_03JBIPMCLC@int?$AA@  100892ac     LIBCMT:undname.obj
 0002:0000f2b0       ??_C@_05BFKKPKCG@short?$AA@ 100892b0     LIBCMT:undname.obj
 0002:0000f2b8       ??_C@_04ENMBGAPA@char?$AA@ 100892b8     LIBCMT:undname.obj
 0002:0000f2c0       ___lookuptable_s           100892c0     LIBCMT:outputs.obj
 0002:0000f320       __atan_table               10089320     LIBCMT:_atan_table_.obj
 0002:00010b30       ??_C@_06IMKFLFPG@1?$CDQNAN?$AA@ 1008ab30     LIBCMT:_x10fout_.obj
 0002:00010b38       ??_C@_05DNEBIAHO@1?$CDINF?$AA@ 1008ab38     LIBCMT:_x10fout_.obj
 0002:00010b40       ??_C@_05PHHOCPM@1?$CDIND?$AA@ 1008ab40     LIBCMT:_x10fout_.obj
 0002:00010b48       ??_C@_06PGGFOGJG@1?$CDSNAN?$AA@ 1008ab48     LIBCMT:_x10fout_.obj
 0002:00010b50       ___dnames                  1008ab50     LIBCMT:timeset.obj
 0002:00010b68       ___mnames                  1008ab68     LIBCMT:timeset.obj
 0002:00010b90       ??_C@_02CLFPBFFP@TZ?$AA@   1008ab90     LIBCMT:tzset.obj
 0002:00010b94       ??_C@_06GDENEHCP@CONIN$?$AA@ 1008ab94     LIBCMT:initcon.obj
 0002:00010b9c       ??_C@_07GPDNMNG@CONOUT$?$AA@ 1008ab9c     LIBCMT:initcon.obj
 0002:000d85b8       ??_C@_05LCOLKLHA@?$CK?4wpk?$AA@ 101525b8     wzFilePacker_static:wzFilePacker.obj
 0002:000d85c0       ??_C@_03HMFOOINA@r?$CLb?$AA@ 101525c0     wzFilePacker_static:wzFilePacker.obj
 0002:000d85c4       ??_C@_04FGAJMCLA@?2?$CK?4?$CK?$AA@ 101525c4     wzFilePacker_static:wzFilePacker.obj
 0002:000d85cc       ??_C@_03EMIMMIHL@?$CK?4?$CK?$AA@ 101525cc     wzFilePacker_static:wzFilePacker.obj
 0002:000d8a00       ??_C@_02DJGKEECL@?4?4?$AA@ 10152a00     wzFilePacker_static:vFile_util.obj
 0002:000d8a04       ??_C@_0L@IMPLNOCC@?2wz_sound?2?$AA@ 10152a04     wzFilePacker_static:vFile_util.obj
 0002:000d8e40       ??_C@_0BI@LCBABOGN@header?5is?5Final?5Version?$AA@ 10152e40     wzFilePacker_static:fsvfs.obj
 0002:000d8e58       ??_C@_0P@FOHJAHFG@header?5invalid?$AA@ 10152e58     wzFilePacker_static:fsvfs.obj
 0002:000d8e68       ??_C@_0DM@MLIJDPNB@Now?5Packing?5File?5Version?5?3?5?$CFd?0?5P@ 10152e68     wzFilePacker_static:fsvfs.obj
 0002:000d8ea4       ??_C@_0DA@JPDHOIDD@?$CK?$CK?$CK?$CK?$CK?$CK?$CK?$CK?$CK?$CK?$CK?$CK?$CK?$CK?$CK?$CK?5N2_UpdateFilePo@ 10152ea4     wzFilePacker_static:fsvfs.obj
 0002:000d8ed4       ??_C@_0CO@LGMGIONK@?$CK?$CK?$CK?$CK?$CK?$CK?$CK?$CK?$CK?$CK?$CK?$CK?$CK?$CK?$CK?$CK?5N2_SetFilePoint@ 10152ed4     wzFilePacker_static:fsvfs.obj
 0002:000d8f04       ??_C@_0DF@IHAPMOPK@?$CL?$CL?$CL?$CL?$CL?$CL?$CL?$CL?$CL?$CL?5ReadFail_4_Error?5?3?5?G?O@ 10152f04     wzFilePacker_static:fsvfs.obj
 0002:000d8f3c       ??_C@_0DH@HABJGGNC@?$CL?$CL?$CL?$CL?$CL?$CL?$CL?$CL?$CL?$CL?5ReadFail_3_Error?5?3?5?$MA?P@ 10152f3c     wzFilePacker_static:fsvfs.obj
 0002:000d8f74       ??_C@_0DG@LCJJILDN@?$CL?$CL?$CL?$CL?$CL?$CL?$CL?$CL?$CL?$CL?5ReadFail_2_Error?5?3?5?$LP?$MA@ 10152f74     wzFilePacker_static:fsvfs.obj
 0002:000d8fac       ??_C@_0CG@GENKINJN@?$CL?$CL?$CL?$CL?$CL?$CL?$CL?$CL?$CL?$CL?5ReadFail_1_ErrorCode?5@ 10152fac     wzFilePacker_static:fsvfs.obj
 0002:000d8fd4       ??_C@_0BH@MMBDGEON@Remove?5Fsvfs?5Tree?5Fail?$AA@ 10152fd4     wzFilePacker_static:fsvfs.obj
 0002:000d8fec       ??_C@_0BK@PKGCLKLI@Remove?5Fsvfs?5Tree?5SUCCESS?$AA@ 10152fec     wzFilePacker_static:fsvfs.obj
 0002:000d9008       ??_C@_0BM@OPDJPMGP@Not?5File?5SameName?5Tree?9Node?$AA@ 10153008     wzFilePacker_static:fsvfs.obj
 0002:000d9458       ??_C@_02CEGDFPFP@?4?2?$AA@ 10153458     wzFilePacker_static:fsdos.obj
 0002:000d945c       ??_C@_0BP@PFJFMKGH@Win32_SetFilePointer_Error?3?$CFd?6?$AA@ 1015345c     wzFilePacker_static:fsdos.obj
 0002:000d9910       ??_R4bad_alloc@std@@6B@    10153910     sound.obj
 0002:000d9924       ??_R3bad_alloc@std@@8      10153924     sound.obj
 0002:000d9934       ??_R2bad_alloc@std@@8      10153934     sound.obj
 0002:000d9940       ??_R1A@?0A@EA@bad_alloc@std@@8 10153940     sound.obj
 0002:000d995c       ??_R1A@?0A@EA@exception@std@@8 1015395c     sound.obj
 0002:000d9978       ??_R3exception@std@@8      10153978     sound.obj
 0002:000d9988       ??_R2exception@std@@8      10153988     sound.obj
 0002:000d9990       ??_R4logic_error@std@@6B@  10153990     sound.obj
 0002:000d99a4       ??_R3logic_error@std@@8    101539a4     sound.obj
 0002:000d99b4       ??_R2logic_error@std@@8    101539b4     sound.obj
 0002:000d99c0       ??_R1A@?0A@EA@logic_error@std@@8 101539c0     sound.obj
 0002:000d99dc       ??_R4length_error@std@@6B@ 101539dc     sound.obj
 0002:000d99f0       ??_R3length_error@std@@8   101539f0     sound.obj
 0002:000d9a00       ??_R2length_error@std@@8   10153a00     sound.obj
 0002:000d9a10       ??_R1A@?0A@EA@length_error@std@@8 10153a10     sound.obj
 0002:000d9a2c       ??_R4out_of_range@std@@6B@ 10153a2c     sound.obj
 0002:000d9a40       ??_R3out_of_range@std@@8   10153a40     sound.obj
 0002:000d9a50       ??_R2out_of_range@std@@8   10153a50     sound.obj
 0002:000d9a60       ??_R1A@?0A@EA@out_of_range@std@@8 10153a60     sound.obj
 0002:000d9a7c       ??_R4invalid_argument@std@@6B@ 10153a7c     libcpmt:string.obj
 0002:000d9a90       ??_R3invalid_argument@std@@8 10153a90     libcpmt:string.obj
 0002:000d9aa0       ??_R2invalid_argument@std@@8 10153aa0     libcpmt:string.obj
 0002:000d9ab0       ??_R1A@?0A@EA@invalid_argument@std@@8 10153ab0     libcpmt:string.obj
 0002:000d9acc       ??_R4exception@std@@6B@    10153acc     LIBCMT:stdexcpt.obj
 0002:000d9ae0       ??_R4bad_cast@std@@6B@     10153ae0     LIBCMT:stdexcpt.obj
 0002:000d9af4       ??_R3bad_cast@std@@8       10153af4     LIBCMT:stdexcpt.obj
 0002:000d9b04       ??_R2bad_cast@std@@8       10153b04     LIBCMT:stdexcpt.obj
 0002:000d9b10       ??_R1A@?0A@EA@bad_cast@std@@8 10153b10     LIBCMT:stdexcpt.obj
 0002:000d9b2c       ??_R4bad_typeid@std@@6B@   10153b2c     LIBCMT:stdexcpt.obj
 0002:000d9b40       ??_R3bad_typeid@std@@8     10153b40     LIBCMT:stdexcpt.obj
 0002:000d9b50       ??_R2bad_typeid@std@@8     10153b50     LIBCMT:stdexcpt.obj
 0002:000d9b5c       ??_R1A@?0A@EA@bad_typeid@std@@8 10153b5c     LIBCMT:stdexcpt.obj
 0002:000d9b78       ??_R4__non_rtti_object@std@@6B@ 10153b78     LIBCMT:stdexcpt.obj
 0002:000d9b8c       ??_R3__non_rtti_object@std@@8 10153b8c     LIBCMT:stdexcpt.obj
 0002:000d9b9c       ??_R2__non_rtti_object@std@@8 10153b9c     LIBCMT:stdexcpt.obj
 0002:000d9bac       ??_R1A@?0A@EA@__non_rtti_object@std@@8 10153bac     LIBCMT:stdexcpt.obj
 0002:000d9bc8       ??_R4type_info@@6B@        10153bc8     LIBCMT:typinfo.obj
 0002:000d9bdc       ??_R3type_info@@8          10153bdc     LIBCMT:typinfo.obj
 0002:000d9bec       ??_R2type_info@@8          10153bec     LIBCMT:typinfo.obj
 0002:000d9bf4       ??_R1A@?0A@EA@type_info@@8 10153bf4     LIBCMT:typinfo.obj
 0002:000d9c10       ??_R4bad_exception@std@@6B@ 10153c10     LIBCMT:frame.obj
 0002:000d9c24       ??_R3bad_exception@std@@8  10153c24     LIBCMT:frame.obj
 0002:000d9c34       ??_R2bad_exception@std@@8  10153c34     LIBCMT:frame.obj
 0002:000d9c40       ??_R1A@?0A@EA@bad_exception@std@@8 10153c40     LIBCMT:frame.obj
 0002:000d9c5c       ___rtc_iaa                 10153c5c     LIBCMT:_initsect_.obj
 0002:000d9c60       ___rtc_izz                 10153c60     LIBCMT:_initsect_.obj
 0002:000d9c64       ___rtc_taa                 10153c64     LIBCMT:_initsect_.obj
 0002:000d9c68       ___rtc_tzz                 10153c68     LIBCMT:_initsect_.obj
 0002:000d9c70       __TI2?AVbad_alloc@std@@    10153c70     sound.obj
 0002:000d9c80       __CTA2?AVbad_alloc@std@@   10153c80     sound.obj
 0002:000d9c8c       __CT??_R0?AVbad_alloc@std@@@8??0bad_alloc@std@@QAE@ABV01@@Z12 10153c8c     sound.obj
 0002:000d9ca8       __CT??_R0?AVexception@std@@@8??0exception@std@@QAE@ABV01@@Z12 10153ca8     sound.obj
 0002:000d9d7c       __TI3?AVlength_error@std@@ 10153d7c     sound.obj
 0002:000d9db8       __CTA3?AVlength_error@std@@ 10153db8     sound.obj
 0002:000d9dc8       __CT??_R0?AVlength_error@std@@@8??0length_error@std@@QAE@ABV01@@Z40 10153dc8     sound.obj
 0002:000d9de4       __CT??_R0?AVlogic_error@std@@@8??0logic_error@std@@QAE@ABV01@@Z40 10153de4     sound.obj
 0002:000d9e2c       __TI3?AVout_of_range@std@@ 10153e2c     sound.obj
 0002:000d9e68       __CTA3?AVout_of_range@std@@ 10153e68     sound.obj
 0002:000d9e78       __CT??_R0?AVout_of_range@std@@@8??0out_of_range@std@@QAE@ABV01@@Z40 10153e78     sound.obj
 0002:000da834       __TI3?AVinvalid_argument@std@@ 10154834     libcpmt:string.obj
 0002:000da870       __CTA3?AVinvalid_argument@std@@ 10154870     libcpmt:string.obj
 0002:000da880       __CT??_R0?AVinvalid_argument@std@@@8??0invalid_argument@std@@QAE@ABV01@@Z40 10154880     libcpmt:string.obj
 0002:000daedc       __TI2?AVbad_exception@std@@ 10154edc     LIBCMT:frame.obj
 0002:000daeec       __CTA2?AVbad_exception@std@@ 10154eec     LIBCMT:frame.obj
 0002:000daef8       __CT??_R0?AVbad_exception@std@@@8??0bad_exception@std@@QAE@ABV01@@Z12 10154ef8     LIBCMT:frame.obj
 0002:000db4dc       __IMPORT_DESCRIPTOR_KERNEL32 101554dc     kernel32:KERNEL32.dll
 0002:000db4f0       __IMPORT_DESCRIPTOR_USER32 101554f0     user32:USER32.dll
 0002:000db504       __IMPORT_DESCRIPTOR_ole32  10155504     ole32:ole32.dll
 0002:000db518       __IMPORT_DESCRIPTOR_WINMM  10155518     winmm:WINMM.dll
 0002:000db52c       __IMPORT_DESCRIPTOR_dbghelp 1015552c     Dbghelp:dbghelp.dll
 0002:000db540       __NULL_IMPORT_DESCRIPTOR   10155540     kernel32:KERNEL32.dll
 0003:0000000c       ?MAX_CHANNELS@@3HA         1015700c     ds.obj
 0003:00000018       ?Ds_eax_presets@@3PAUEAX_REVERBPROPERTIES@@A 10157018     ds.obj
 0003:000001b8       ?DSPROPSETID_EAX_ReverbProperties_Def@@3U_GUID@@A 101571b8     ds.obj
 0003:000001c8       ?DSPROPSETID_EAXBUFFER_ReverbProperties_Def@@3U_GUID@@A 101571c8     ds.obj
 0003:000001dc       ?DSPROPSETID_VoiceManager_Def@@3U_GUID@@A 101571dc     ds3d.obj
 0003:000001f0       ?Sound_enabled@@3HA        101571f0     sound.obj
 0003:000001f4       ?Master_sound_volume@@3MA  101571f4     sound.obj
 0003:000001f8       ?Master_voice_volume@@3MA  101571f8     sound.obj
 0003:000001fc       ?Sound_cache_maintain_milliseconds@@3HA 101571fc     sound.obj
 0003:00000200       ??_R0?AVbad_alloc@std@@@8  10157200     sound.obj
 0003:0000021c       ??_R0?AVexception@std@@@8  1015721c     sound.obj
 0003:00000238       ??_R0?AVlogic_error@std@@@8 10157238     sound.obj
 0003:00000258       ??_R0?AVlength_error@std@@@8 10157258     sound.obj
 0003:00000278       ??_R0?AVout_of_range@std@@@8 10157278     sound.obj
 0003:000002b8       ?timestamp_ticker@@3HA     101572b8     timer.obj
 0003:000002d0       ?fl_magic@@3HA             101572d0     floating.obj
 0003:000002d4       ?p_fl_magic@@3PBMB         101572d4     floating.obj
 0003:000002dc       ?vmd_x_vector@@3Uvector@@A 101572dc     vecmat.obj
 0003:000002e8       ?vmd_y_vector@@3Uvector@@A 101572e8     vecmat.obj
 0003:000002f4       ?vmd_z_vector@@3Uvector@@A 101572f4     vecmat.obj
 0003:00000300       ?vmd_identity_matrix@@3Umatrix@@A 10157300     vecmat.obj
 0003:0000032c       ?libxls_major_version@@3HA 1015732c     version.obj
 0003:00000338       ?brdb@@3PAUstr_brdb@@A     10157338     xlstool.obj
 0003:00000b88       ?nMixerControlID_master_vol@@3HA 10157b88     wzSound.obj
 0003:00000b8c       ?nMixerControlID_master_pan@@3HA 10157b8c     wzSound.obj
 0003:00000b90       ?nMixerControlID_master_mute@@3HA 10157b90     wzSound.obj
 0003:00000b94       ?nMixerControlID_wav_vol@@3HA 10157b94     wzSound.obj
 0003:00000b98       ?nMixerControlID_wav_pan@@3HA 10157b98     wzSound.obj
 0003:00000b9c       ?nMixerControlID_wav_mute@@3HA 10157b9c     wzSound.obj
 0003:00000ba0       ?nMixerControlID_mic_input_vol@@3PAHA 10157ba0     wzSound.obj
 0003:00000bb4       ?nMixerControlID_mic_output_vol@@3HA 10157bb4     wzSound.obj
 0003:00000bb8       ?nMixerControlID_mic_output_mute@@3HA 10157bb8     wzSound.obj
 0003:00000bbc       ?_rolloff_factor@@3MA      10157bbc     wzSound.obj
 0003:00000bc4       ??_R0?AVinvalid_argument@std@@@8 10157bc4     libcpmt:string.obj
 0003:00000be8       ??_C@_04EFJP@pcmR?$AA@     10157be8     vorbisfile_static:vorbisfile.obj
 0003:00000bf0       ??_C@_04EHCF@pcmL?$AA@     10157bf0     vorbisfile_static:vorbisfile.obj
 0003:00000bf8       ??_C@_01KPOD@?$DN?$AA@     10157bf8     vorbisfile_static:info.obj
 0003:00000bfc       ??_C@_06GIBB@vorbis?$AA@   10157bfc     vorbisfile_static:info.obj
 0003:00000c04       ??_C@_0BO@KFNF@Xiph?4Org?5libVorbis?5I?520030909?$AA@ 10157c04     vorbisfile_static:info.obj
 0003:00000c24       _analysis_noisy            10157c24     vorbisfile_static:analysis.obj
 0003:00000c28       ??_C@_03FBAH@?$CFf?6?$AA@  10157c28     vorbisfile_static:analysis.obj
 0003:00000c2c       ??_C@_03CHB@?$CFf?5?$AA@   10157c2c     vorbisfile_static:analysis.obj
 0003:00000c30       ??_C@_0BO@NFHP@failed?5to?5open?5data?5dump?5file?$AA@ 10157c30     vorbisfile_static:analysis.obj
 0003:00000c50       ??_C@_01LLF@w?$AA@         10157c50     vorbisfile_static:analysis.obj
 0003:00000c54       ??_C@_07DFJO@?$CFs_?$CFd?4m?$AA@ 10157c54     vorbisfile_static:analysis.obj
 0003:00006bc8       __floor_P                  1015dbc8     vorbisfile_static:registry.obj
 0003:00006bd0       __residue_P                1015dbd0     vorbisfile_static:registry.obj
 0003:00006bdc       __mapping_P                1015dbdc     vorbisfile_static:registry.obj
 0003:0000ebb0       _mapping0_exportbundle     10165bb0     vorbisfile_static:mapping0.obj
 0003:0000ebc8       _residue0_exportbundle     10165bc8     vorbisfile_static:res0.obj
 0003:0000ebe8       _residue1_exportbundle     10165be8     vorbisfile_static:res0.obj
 0003:0000ec08       _residue2_exportbundle     10165c08     vorbisfile_static:res0.obj
 0003:0000f028       _floor1_exportbundle       10166028     vorbisfile_static:floor1.obj
 0003:0000f048       _floor0_exportbundle       10166048     vorbisfile_static:floor0.obj
 0003:0000f4fc       __fltused                  101664fc     LIBCMT:_fpinit_.obj
 0003:0000f500       __ldused                   10166500     LIBCMT:_fpinit_.obj
 0003:0000f510       ___security_cookie         10166510     LIBCMT:gs_cookie.obj
 0003:0000f514       ___security_cookie_complement 10166514     LIBCMT:gs_cookie.obj
 0003:0000f530       __half                     10166530     LIBCMT:_pow_.obj
 0003:0000f540       ??_R0?AVbad_cast@std@@@8   10166540     LIBCMT:stdexcpt.obj
 0003:0000f55c       ??_R0?AVbad_typeid@std@@@8 1016655c     LIBCMT:stdexcpt.obj
 0003:0000f57c       ??_R0?AV__non_rtti_object@std@@@8 1016657c     LIBCMT:stdexcpt.obj
 0003:0000f5a4       ??_R0?AVtype_info@@@8      101665a4     LIBCMT:typinfo.obj
 0003:0000f790       __aexit_rtn                10166790     LIBCMT:crt0dat.obj
 0003:0000f794       __cfltcvt_tab              10166794     LIBCMT:cmiscdat.obj
 0003:0000f7bc       __amblksiz                 101667bc     LIBCMT:heapinit.obj
 0003:0000f8e0       ___initialmbcinfo          101668e0     LIBCMT:mbctype.obj
 0003:0000fb00       __mbctype                  10166b00     LIBCMT:mbctype.obj
 0003:0000fc08       __mbcasemap                10166c08     LIBCMT:mbctype.obj
 0003:0000fd08       ___ptmbcinfo               10166d08     LIBCMT:mbctype.obj
 0003:0000fe04       ___globallocalestatus      10166e04     LIBCMT:glstatus.obj
 0003:0000fe08       ___clocalestr              10166e08     LIBCMT:nlsdata2.obj
 0003:0000fe10       ___initiallocinfo          10166e10     LIBCMT:nlsdata2.obj
 0003:0000fee8       ___ptlocinfo               10166ee8     LIBCMT:nlsdata2.obj
 0003:0000feec       ___lc_clike                10166eec     LIBCMT:nlsdata2.obj
 0003:0000fef0       ___initiallocalestructinfo 10166ef0     LIBCMT:nlsdata2.obj
 0003:0000fef8       ___flsindex                10166ef8     LIBCMT:tidtable.obj
 0003:0000fefc       ___getvalueindex           10166efc     LIBCMT:tidtable.obj
 0003:0000ffc0       __infinity                 10166fc0     LIBCMT:_87tran_.obj
 0003:0000ffca       __minfinity                10166fca     LIBCMT:_87tran_.obj
 0003:0000ffd4       __logemax                  10166fd4     LIBCMT:_87tran_.obj
 0003:0000fffa       __OP_EXPjmptab             10166ffa     LIBCMT:_87tran_.obj
 0003:00010020       __indefinite               10167020     LIBCMT:_87disp_.obj
 0003:0001002a       __piby2                    1016702a     LIBCMT:_87disp_.obj
 0003:00010064       ??_R0?AVbad_exception@std@@@8 10167064     LIBCMT:frame.obj
 0003:00010090       ___nullstring              10167090     LIBCMT:output.obj
 0003:00010094       ___wnullstring             10167094     LIBCMT:output.obj
 0003:00010098       __iob                      10167098     LIBCMT:_file.obj
 0003:00010318       __lookuptrailbytes         10167318     LIBCMT:read.obj
 0003:00010420       __d_inf                    10167420     LIBCMT:_util_.obj
 0003:00010428       __d_ind                    10167428     LIBCMT:_util_.obj
 0003:00010430       __d_max                    10167430     LIBCMT:_util_.obj
 0003:00010438       __d_min                    10167438     LIBCMT:_util_.obj
 0003:00010440       __d_mzero                  10167440     LIBCMT:_util_.obj
 0003:00010550       ___badioinfo               10167550     LIBCMT:ioinit.obj
 0003:00010590       __First_FPE_Indx           10167590     LIBCMT:winxfltr.obj
 0003:00010594       __Num_FPE                  10167594     LIBCMT:winxfltr.obj
 0003:00010598       __XcptActTabSize           10167598     LIBCMT:winxfltr.obj
 0003:0001059c       __XcptActTabCount          1016759c     LIBCMT:winxfltr.obj
 0003:000105a8       __sys_errlist              101675a8     LIBCMT:syserr.obj
 0003:00010658       __sys_nerr                 10167658     LIBCMT:syserr.obj
 0003:00010660       __pctype                   10167660     LIBCMT:ctype.obj
 0003:00010664       __pwctype                  10167664     LIBCMT:ctype.obj
 0003:00010668       ___lc_time_c               10167668     LIBCMT:strftime.obj
 0003:00010720       ___lc_time_curr            10167720     LIBCMT:strftime.obj
 0003:00010724       ___lconv_static_decimal    10167724     LIBCMT:lconv.obj
 0003:00010728       ___lconv_c                 10167728     LIBCMT:lconv.obj
 0003:00010758       ___lconv                   10167758     LIBCMT:lconv.obj
 0003:0001075c       ___mb_cur_max              1016775c     LIBCMT:nlsdata1.obj
 0003:00010760       ___decimal_point           10167760     LIBCMT:nlsdata1.obj
 0003:00010764       ___decimal_point_length    10167764     LIBCMT:nlsdata1.obj
 0003:00010770       ___abort_behavior          10167770     LIBCMT:abort.obj
 0003:000108e0       __NLG_Destination          101678e0     LIBCMT:exsup.obj
 0003:00010920       __pow10pos                 10167920     LIBCMT:_constpow_.obj
 0003:00010a80       __pow10neg                 10167a80     LIBCMT:_constpow_.obj
 0003:00010bdc       __matherr_flag             10167bdc     LIBCMT:_matherr_.obj
 0003:00010bf0       __timezone                 10167bf0     LIBCMT:timeset.obj
 0003:00010bf4       __daylight                 10167bf4     LIBCMT:timeset.obj
 0003:00010bf8       __dstbias                  10167bf8     LIBCMT:timeset.obj
 0003:00010c80       __tzname                   10167c80     LIBCMT:timeset.obj
 0003:00010ca0       __coninpfh                 10167ca0     LIBCMT:initcon.obj
 0003:00010ca4       __confh                    10167ca4     LIBCMT:initcon.obj
 0003:00010ca8       __lpdays                   10167ca8     LIBCMT:days.obj
 0003:00010cdc       __days                     10167cdc     LIBCMT:days.obj
 0003:00010d10       __libiconv_version         10167d10     iconv:iconv.obj
 0003:00010d14       ??_C@_08KIEN@?1?1IGNORE?$AA@ 10167d14     iconv:iconv.obj
 0003:00010d20       ??_C@_0L@CMOP@?1?1TRANSLIT?$AA@ 10167d20     iconv:iconv.obj
 0003:00010d2c       ??_C@_05OGAG@ASCII?$AA@    10167d2c     iconv:localcharset.obj
 0003:00010d34       ??_C@_04FIHK@CP?$CFu?$AA@  10167d34     iconv:localcharset.obj
 0003:00010d3c       ??_C@_0BAE@GMIJ@CP936?$AAGBK?$AACP1361?$AAJOHAB?$AACP20127?$AAA@ 10167d3c     iconv:localcharset.obj
 0003:00010e54       _cchCurDir                 10167e54     wzFilePacker_static:vFile_util.obj
 0003:0001139c       ??_C@_04BABO@OggS?$AA@     1016839c     ogg_static:framing.obj
 0003:00011460       ?Compressed_buffer@@3PAEA  10168460     audiostr.obj
 0003:00026d4c       ?Global_service_lock@@3U_RTL_CRITICAL_SECTION@@A 1017dd4c     audiostr.obj
 0003:00026d64       ?m_ass@@3VAudioStreamServices@@A 1017dd64     audiostr.obj
 0003:00026d68       ?Wavedata_service_buffer@@3PAEA 1017dd68     audiostr.obj
 0003:00052c88       ?Compressed_service_buffer@@3PAEA 101a9c88     audiostr.obj
 0003:00068578       ?Wavedata_load_buffer@@3PAEA 101bf578     audiostr.obj
 0003:00094498       ?Audiostream_inited@@3HA   101eb498     audiostr.obj
 0003:000944a0       ?Audio_streams@@3PAVAudioStream@@A 101eb4a0     audiostr.obj
 0003:00095b28       ?ds_hardware_buffers@@3PAUds_sound_buffer@@A 101ecb28     ds.obj
 0003:000962a8       ?ds_software_buffers@@3PAUds_sound_buffer@@A 101ed2a8     ds.obj
 0003:000a52a8       ?ds_vol_lookup@@3PAHA      101fc2a8     ds.obj
 0003:000a54a0       ?pfn_DirectSoundCreate8@@3P6GJPAU_GUID@@PAPAUIDirectSound8@@PAUIUnknown@@@ZA 101fc4a0     ds.obj
 0003:000a54a4       ?Ds_dll_loaded@@3HA        101fc4a4     ds.obj
 0003:000a54a8       ?Ds_dll_handle@@3PAUHINSTANCE__@@A 101fc4a8     ds.obj
 0003:000a54ac       ?pDirectSound8@@3PAUIDirectSound8@@A 101fc4ac     ds.obj
 0003:000a54b0       ?pPrimaryBuffer@@3PAUIDirectSoundBuffer@@A 101fc4b0     ds.obj
 0003:000a54c4       ?Channels@@3PAUchannel@@A  101fc4c4     ds.obj
 0003:000a54dc       ?ds_initialized@@3HA       101fc4dc     ds.obj
 0003:000a54e4       ?DS3D_inited@@3HA          101fc4e4     ds3d.obj
 0003:000a54e8       ?pDS3D_listener@@3PAUIDirectSound3DListener@@A 101fc4e8     ds3d.obj
 0003:000a54ec       ?UserSampleBits@@3GA       101fc4ec     sound.obj
 0003:000a54f4       ?UserSampleRate@@3GA       101fc4f4     sound.obj
 0003:000a54fc       ?View_matrix@@3Umatrix@@A  101fc4fc     sound.obj
 0003:000a5520       ?Snd_hram@@3HA             101fc520     sound.obj
 0003:000a5524       ?Snd_sram@@3HA             101fc524     sound.obj
 0003:000a5528       ?View_position@@3Uvector@@A 101fc528     sound.obj
 0003:000a553c       ?Is_sound_cache@@3_NA      101fc53c     sound.obj
 0003:000a5540       ?map_sounds@@3V?$map@HUsound@@U?$less@H@std@@V?$allocator@U?$pair@$$CBHUsound@@@std@@@3@@std@@A 101fc540     sound.obj
 0003:000a5560       ?cfile_callbacks@@3Uov_callbacks@@A 101fc560     ogg.obj
 0003:000a5570       ?mmio_callbacks@@3Uov_callbacks@@A 101fc570     ogg.obj
 0003:000a5580       ?ogg_inited@@3HA           101fc580     ogg.obj
 0003:000a5584       ?ambi_handles@@3V?$map@HHU?$less@H@std@@V?$allocator@U?$pair@$$CBHH@std@@@2@@std@@A 101fc584     ambientsnd.obj
 0003:000a55a8       ?Event_music@@3PAUEventMusic@@A 101fc5a8     eventmusic.obj
 0003:000abe58       ?Num_music_files@@3HA      10202e58     eventmusic.obj
 0003:000abe5c       ?music_handles@@3V?$map@HHU?$less@H@std@@V?$allocator@U?$pair@$$CBHH@std@@@2@@std@@A 10202e5c     eventmusic.obj
 0003:000abe80       ?index_table_event_music@@3V?$map@HHU?$less@H@std@@V?$allocator@U?$pair@$$CBHH@std@@@2@@std@@A 10202e80     scriptparser.obj
 0003:000abea0       ?Snds@@3V?$map@HUgame_snd@@U?$less@H@std@@V?$allocator@U?$pair@$$CBHUgame_snd@@@std@@@3@@std@@A 10202ea0     scriptparser.obj
 0003:000abec0       ?index_table_voice_sound@@3V?$map@HHU?$less@H@std@@V?$allocator@U?$pair@$$CBHH@std@@@2@@std@@A 10202ec0     scriptparser.obj
 0003:000abee0       ?Snds_iface@@3V?$map@HUgame_snd@@U?$less@H@std@@V?$allocator@U?$pair@$$CBHUgame_snd@@@std@@@3@@std@@A 10202ee0     scriptparser.obj
 0003:000abf00       ?VoiceTbl@@3V?$map@HUVoiceSnd@@U?$less@H@std@@V?$allocator@U?$pair@$$CBHUVoiceSnd@@@std@@@3@@std@@A 10202f00     scriptparser.obj
 0003:000abf20       ?AmbientTbl@@3V?$map@HUAmbientSnd@@U?$less@H@std@@V?$allocator@U?$pair@$$CBHUAmbientSnd@@@std@@@3@@std@@A 10202f20     scriptparser.obj
 0003:000abf40       ?voice_snd@@3PAUVoiceSnd@@A 10202f40     voicesnd.obj
 0003:000eef40       ?Num_voice_files@@3HA      10245f40     voicesnd.obj
 0003:000eef44       ?voice_handles@@3V?$map@HHU?$less@H@std@@V?$allocator@U?$pair@$$CBHH@std@@@2@@std@@A 10245f44     voicesnd.obj
 0003:000eef9c       _enable_debugLog           10245f9c     util_debug.obj
 0003:000eefa0       ?hVFS@@3PAXA               10245fa0     util_packfile.obj
 0003:000eefa8       ?packFile@@3VCPackFile@@A  10245fa8     util_packfile.obj
 0003:000ef3b0       ?Cfile_list@@3PAUCFILE@@A  102463b0     cfile.obj
 0003:000ef9b0       ?cfile_inited@@3HA         102469b0     cfile.obj
 0003:000ef9b4       ?fi@@3T_flint@@A           102469b4     floating.obj
 0003:000ef9b8       ?fo@@3T_flint@@A           102469b8     floating.obj
 0003:000ef9c0       ?vmd_zero_vector@@3Uvector@@A 102469c0     vecmat.obj
 0003:000ef9d0       ?Rand_count@@3HA           102469d0     systemvars.obj
 0003:000ef9d8       ?libxls_minor_version@@3HA 102469d8     version.obj
 0003:000ef9dc       ?libxls_micro_version@@3HA 102469dc     version.obj
 0003:000ef9e8       ?dwMaxMicVol_output@@3KA   102469e8     wzSound.obj
 0003:000ef9ec       ?dwMinMicVol_output@@3KA   102469ec     wzSound.obj
 0003:000ef9f0       ?isInitialized@@3HA        102469f0     wzSound.obj
 0003:000ef9f4       ?g_mixer_speaker@@3PAUHMIXER__@@A 102469f4     wzSound.obj
 0003:000ef9f8       ?g_mixer_microphone@@3PAUHMIXER__@@A 102469f8     wzSound.obj
 0003:000ef9fc       ?dwMinMasterVol@@3KA       102469fc     wzSound.obj
 0003:000efa00       ?dwMaxMasterVol@@3KA       10246a00     wzSound.obj
 0003:000efa04       ?lMinMasterPan@@3JA        10246a04     wzSound.obj
 0003:000efa08       ?lMaxMasterPan@@3JA        10246a08     wzSound.obj
 0003:000efa0c       ?dwMinWavVol@@3KA          10246a0c     wzSound.obj
 0003:000efa10       ?dwMaxWavVol@@3KA          10246a10     wzSound.obj
 0003:000efa14       ?lMinWavPan@@3JA           10246a14     wzSound.obj
 0003:000efa18       ?lMaxWavPan@@3JA           10246a18     wzSound.obj
 0003:000efa1c       ?dwMinMicVol_input@@3PAKA  10246a1c     wzSound.obj
 0003:000efa30       ?dwMaxMicVol_input@@3PAKA  10246a30     wzSound.obj
 0003:000efa44       ?dwMicCount_input@@3KA     10246a44     wzSound.obj
 0003:000efa48       ?lMinMicPan@@3JA           10246a48     wzSound.obj
 0003:000efa4c       ?lMaxMicPan@@3JA           10246a4c     wzSound.obj
 0003:000efa50       ?psz_ConfigFile@@3PADA     10246a50     wzSound.obj
 0003:000efb54       ?use_secure_filesystem@@3HA 10246b54     wzSound.obj
 0003:000efb58       ?psz_VoiceFile@@3PADA      10246b58     wzSound.obj
 0003:000efc5c       ?_doppler_factor@@3MA      10246c5c     wzSound.obj
 0003:000efc60       ?psz_MusicFile@@3PADA      10246c60     wzSound.obj
 0003:000efd64       ?_3DQuality@@3KA           10246d64     wzSound.obj
 0003:000efd68       ?psz_SoundFile@@3PADA      10246d68     wzSound.obj
 0003:000efe70       ?psz_secure_filesystem@@3PADA 10246e70     wzSound.obj
 0003:000eff78       ?psz_local_filesystem@@3PADA 10246f78     wzSound.obj
 0003:000f0084       ___fastflag                10247084     LIBCMT:_fpinit_.obj
 0003:000f0088       __adjust_fdiv              10247088     LIBCMT:_fpinit_.obj
 0003:000f008c       ___pInvalidArgHandler      1024708c     LIBCMT:invarg.obj
 0003:000f00a8       __aenvptr                  102470a8     LIBCMT:dllcrt0.obj
 0003:000f00ac       __wenvptr                  102470ac     LIBCMT:dllcrt0.obj
 0003:000f00b0       ___error_mode              102470b0     LIBCMT:dllcrt0.obj
 0003:000f00b4       ___app_type                102470b4     LIBCMT:dllcrt0.obj
 0003:000f00b8       __umaskval                 102470b8     LIBCMT:crt0dat.obj
 0003:000f00bc       ___argc                    102470bc     LIBCMT:crt0dat.obj
 0003:000f00c0       ___argv                    102470c0     LIBCMT:crt0dat.obj
 0003:000f00c4       ___wargv                   102470c4     LIBCMT:crt0dat.obj
 0003:000f00c8       __environ                  102470c8     LIBCMT:crt0dat.obj
 0003:000f00cc       ___initenv                 102470cc     LIBCMT:crt0dat.obj
 0003:000f00d0       __wenviron                 102470d0     LIBCMT:crt0dat.obj
 0003:000f00d4       ___winitenv                102470d4     LIBCMT:crt0dat.obj
 0003:000f00d8       __pgmptr                   102470d8     LIBCMT:crt0dat.obj
 0003:000f00dc       __wpgmptr                  102470dc     LIBCMT:crt0dat.obj
 0003:000f00e0       __exitflag                 102470e0     LIBCMT:crt0dat.obj
 0003:000f00e4       __C_Termination_Done       102470e4     LIBCMT:crt0dat.obj
 0003:000f00e8       __C_Exit_Done              102470e8     LIBCMT:crt0dat.obj
 0003:000f00ec       __crtheap                  102470ec     LIBCMT:heapinit.obj
 0003:000f0240       ___sbh_pHeaderDefer        10247240     LIBCMT:sbheap.obj
 0003:000f0248       ___mbulinfo                10247248     LIBCMT:mbctype.obj
 0003:000f0254       ___mbcodepage              10247254     LIBCMT:mbctype.obj
 0003:000f0258       ___ismbcodepage            10247258     LIBCMT:mbctype.obj
 0003:000f025c       ___mblcid                  1024725c     LIBCMT:mbctype.obj
 0003:000f0260       ___locale_changed          10247260     LIBCMT:setlocal.obj
 0003:000f0264       ___lc_handle               10247264     LIBCMT:nlsdata2.obj
 0003:000f027c       ___lc_codepage             1024727c     LIBCMT:nlsdata2.obj
 0003:000f0280       ___lc_collate_cp           10247280     LIBCMT:nlsdata2.obj
 0003:000f0284       _gpFlsAlloc                10247284     LIBCMT:tidtable.obj
 0003:000f0288       _gpFlsGetValue             10247288     LIBCMT:tidtable.obj
 0003:000f028c       _gpFlsSetValue             1024728c     LIBCMT:tidtable.obj
 0003:000f0290       _gpFlsFree                 10247290     LIBCMT:tidtable.obj
 0003:000f08d4       ?_pnhHeap@@3P6AHI@ZA       102478d4     LIBCMT:handler.obj
 0003:000f08d8       __newmode                  102478d8     LIBCMT:_newmode.obj
 0003:000f08dc       __maxwait                  102478dc     LIBCMT:crtheap.obj
 0003:000f08e0       ?__pInconsistency@@3P6AXXZA 102478e0     LIBCMT:hooks.obj
 0003:000f08ec       __cflush                   102478ec     LIBCMT:_file.obj
 0003:000f08f0       __stdbuf                   102478f0     LIBCMT:_sftbuf.obj
 0003:000f0a2c       ___pPurecall               10247a2c     LIBCMT:inithelp.obj
 0003:000f0a34       __outputformat             10247a34     LIBCMT:outputformat.obj
 0003:000f0a3c       ___lconv_static_null       10247a3c     LIBCMT:lconv.obj
 0003:000f0a68       ?pArgList@UnDecorator@@0PAVReplicator@@A 10247a68     LIBCMT:undname.obj
 0003:000f0a6c       ?pZNameList@UnDecorator@@0PAVReplicator@@A 10247a6c     LIBCMT:undname.obj
 0003:000f0a70       ?pTemplateArgList@UnDecorator@@0PAVReplicator@@A 10247a70     LIBCMT:undname.obj
 0003:000f0a74       ?gName@UnDecorator@@0PBDB  10247a74     LIBCMT:undname.obj
 0003:000f0a78       ?name@UnDecorator@@0PBDB   10247a78     LIBCMT:undname.obj
 0003:000f0a7c       ?outputString@UnDecorator@@0PADA 10247a7c     LIBCMT:undname.obj
 0003:000f0a80       ?maxStringLength@UnDecorator@@0HA 10247a80     LIBCMT:undname.obj
 0003:000f0a84       ?disableFlags@UnDecorator@@0KA 10247a84     LIBCMT:undname.obj
 0003:000f0a88       ?m_pGetParameter@UnDecorator@@0P6APADJ@ZA 10247a88     LIBCMT:undname.obj
 0003:000f0a8c       ?fExplicitTemplateParams@UnDecorator@@0_NA 10247a8c     LIBCMT:undname.obj
 0003:000f0a8d       ?fGetTemplateArgumentList@UnDecorator@@0_NA 10247a8d     LIBCMT:undname.obj
 0003:000f0a90       ?nodes@?1??make@DNameStatusNode@@SAPAV2@W4DNameStatus@@@Z@4PAV2@A 10247a90     LIBCMT:undname.obj
 0003:000f0ac0       ??_B?1??make@DNameStatusNode@@SAPAV1@W4DNameStatus@@@Z@51 10247ac0     LIBCMT:undname.obj
 0003:000f0ac4       __commode                  10247ac4     LIBCMT:ncommode.obj
 0003:000f0b88       __fmode                    10247b88     LIBCMT:txtmode.obj
 0003:000f0b90       ??_C@_00A@?$AA@            10247b90     iconv:localcharset.obj
 0003:000f0ba8       ?autofree@@3VCAutoFree@@A  10247ba8     wzFilePacker_static:wzFilePacker.obj
 0003:000f0bb8       _dwTreeCount               10247bb8     wzFilePacker_static:vfile.obj
 0003:000f0bbc       _g_nTreeArrayCount         10247bbc     wzFilePacker_static:vfile.obj
 0003:000f0bc0       _g_ulStartBinaryOffset     10247bc0     wzFilePacker_static:vfile.obj
 0003:000f0bc8       _g_ulTatalBinarySize       10247bc8     wzFilePacker_static:vfile.obj
 0003:000f0bd4       _bCurDirCreated            10247bd4     wzFilePacker_static:vFile_util.obj
 0003:000f14e4       __pmatherr                 102484e4     <common>
 0003:000f14e8       __nhandle                  102484e8     <common>
 0003:000f1500       ___pioinfo                 10248500     <common>
 0003:000f1600       ___piob                    10248600     <common>
 0003:000f1620       __bufin                    10248620     <common>
 0003:000f2620       __nstream                  10249620     <common>
 0003:000f2624       __debugger_hook_dummy      10249624     <common>
 0003:000f2628       ___use_sse2_mathfcns       10249628     <common>
 0003:000f262c       ___setlc_active            1024962c     <common>
 0003:000f2630       ___unguarded_readlc_active 10249630     <common>
 0003:000f2634       ___sse2_available          10249634     <common>
 0003:000f2638       ___sbh_initialized         10249638     <common>
 0003:000f263c       ___sbh_cntHeaderList       1024963c     <common>
 0003:000f2640       ___sbh_pHeaderList         10249640     <common>
 0003:000f2644       ___sbh_threshold           10249644     <common>
 0003:000f2648       ___sbh_pHeaderScan         10249648     <common>
 0003:000f264c       ___sbh_sizeHeaderList      1024964c     <common>
 0003:000f2650       ___sbh_indGroupDefer       10249650     <common>
 0003:000f2654       ___active_heap             10249654     <common>
 0003:000f2658       ___env_initialized         10249658     <common>
 0003:000f265c       ___onexitend               1024965c     <common>
 0003:000f2660       ___onexitbegin             10249660     <common>
 0003:000f2664       ___mbctype_initialized     10249664     <common>
 0003:000f2668       ___dyn_tls_init_callback   10249668     <common>
 0003:000f266c       __acmdln                   1024966c     <common>
 0003:000f2670       _StupidUnusedPointer       10249670     <common>
 0003:000f2680       _lpszCurDir                10249680     <common>
 0003:000f2a80       _g_TreeList                10249a80     <common>

 entry point at        0001:0003a067

 Static symbols

 0001:fffff000       __unwindfunclet$??0?$_Tree@V?$_Tmap_traits@HHU?$less@H@std@@V?$allocator@U?$pair@$$CBHH@std@@@2@$0A@@std@@@std@@QAE@ABU?$less@H@1@ABV?$allocator@U?$pair@$$CBHH@std@@@1@@Z$0 10000000 f   eventmusic.obj
 0001:fffff000       __ehhandler$?_Copy@?$basic_string@DU?$char_traits@D@std@@V?$allocator@D@2@@std@@IAEXII@Z 10000000 f   scriptparser.obj
 0001:fffff000       __ehhandler$?_Copy@?$basic_string@DU?$char_traits@D@std@@V?$allocator@D@2@@std@@IAEXII@Z 10000000 f   wzSound.obj
 0001:fffff000       __unwindfunclet$??0logic_error@std@@QAE@ABV?$basic_string@DU?$char_traits@D@std@@V?$allocator@D@2@@1@@Z$0 10000000 f   wzSound.obj
 0001:fffff000       __unwindfunclet$??0logic_error@std@@QAE@ABV01@@Z$0 10000000 f   scriptparser.obj
 0001:fffff000       __unwindfunclet$?_Insert@?$_Tree@V?$_Tmap_traits@HHU?$less@H@std@@V?$allocator@U?$pair@$$CBHH@std@@@2@$0A@@std@@@std@@IAE?AViterator@12@_NPAU_Node@?$_Tree_nod@V?$_Tmap_traits@HHU?$less@H@std@@V?$allocator@U?$pair@$$CBHH@std@@@2@$0A@@std@@@2@ABU?$pair@$$CBHH@2@@Z$0 10000000 f   wzSound.obj
 0001:fffff000       __unwindfunclet$??1?$_Tree@V?$_Tmap_traits@HHU?$less@H@std@@V?$allocator@U?$pair@$$CBHH@std@@@2@$0A@@std@@@std@@QAE@XZ$0 10000000 f   voicesnd.obj
 0001:fffff000       __unwindfunclet$??0logic_error@std@@QAE@ABV01@@Z$0 10000000 f   wzSound.obj
 0001:fffff000       __unwindfunclet$?_Insert@?$_Tree@V?$_Tmap_traits@HHU?$less@H@std@@V?$allocator@U?$pair@$$CBHH@std@@@2@$0A@@std@@@std@@IAE?AViterator@12@_NPAU_Node@?$_Tree_nod@V?$_Tmap_traits@HHU?$less@H@std@@V?$allocator@U?$pair@$$CBHH@std@@@2@$0A@@std@@@2@ABU?$pair@$$CBHH@2@@Z$0 10000000 f   voicesnd.obj
 0001:fffff000       __unwindfunclet$??0?$_Tree@V?$_Tmap_traits@HHU?$less@H@std@@V?$allocator@U?$pair@$$CBHH@std@@@2@$0A@@std@@@std@@QAE@ABU?$less@H@1@ABV?$allocator@U?$pair@$$CBHH@std@@@1@@Z$0 10000000 f   voicesnd.obj
 0001:fffff000       __unwindfunclet$??0logic_error@std@@QAE@ABV01@@Z$0 10000000 f   libcpmt:string.obj
 0001:fffff000       __unwindfunclet$??0logic_error@std@@QAE@ABV01@@Z$0 10000000 f   voicesnd.obj
 0001:fffff000       __unwindfunclet$?erase@?$_Tree@V?$_Tmap_traits@HHU?$less@H@std@@V?$allocator@U?$pair@$$CBHH@std@@@2@$0A@@std@@@std@@QAE?AViterator@12@Vconst_iterator@12@@Z$0 10000000 f   voicesnd.obj
 0001:fffff000       __ehhandler$?_Copy@?$basic_string@DU?$char_traits@D@std@@V?$allocator@D@2@@std@@IAEXII@Z 10000000 f   xls.obj
 0001:fffff000       __unwindfunclet$?_Insert@?$_Tree@V?$_Tmap_traits@HUAmbientSnd@@U?$less@H@std@@V?$allocator@U?$pair@$$CBHUAmbientSnd@@@std@@@3@$0A@@std@@@std@@IAE?AViterator@12@_NPAU_Node@?$_Tree_nod@V?$_Tmap_traits@HUAmbientSnd@@U?$less@H@std@@V?$allocator@U?$pair@$$CBHUAmbientSnd@@@std@@@3@$0A@@std@@@2@ABU?$pair@$$CBHUAmbientSnd@@@2@@Z$0 10000000 f   scriptparser.obj
 0001:fffff000       __unwindfunclet$??0logic_error@std@@QAE@ABV?$basic_string@DU?$char_traits@D@std@@V?$allocator@D@2@@1@@Z$0 10000000 f   voicesnd.obj
 0001:fffff000       __unwindfunclet$??0logic_error@std@@QAE@ABV?$basic_string@DU?$char_traits@D@std@@V?$allocator@D@2@@1@@Z$0 10000000 f   xls.obj
 0001:fffff000       __ehhandler$?_Copy@?$basic_string@DU?$char_traits@D@std@@V?$allocator@D@2@@std@@IAEXII@Z 10000000 f   voicesnd.obj
 0001:fffff000       __unwindfunclet$??0logic_error@std@@QAE@ABV?$basic_string@DU?$char_traits@D@std@@V?$allocator@D@2@@1@@Z$0 10000000 f   libcpmt:string.obj
 0001:fffff000       __unwindfunclet$?_Insert_n@?$vector@V?$basic_string@DU?$char_traits@D@std@@V?$allocator@D@2@@std@@V?$allocator@V?$basic_string@DU?$char_traits@D@std@@V?$allocator@D@2@@std@@@2@@std@@IAEXV?$_Vector_const_iterator@V?$basic_string@DU?$char_traits@D@std@@V?$allocator@D@2@@std@@V?$allocator@V?$basic_string@DU?$char_traits@D@std@@V?$allocator@D@2@@std@@@2@@2@IABV?$basic_string@DU?$char_traits@D@std@@V?$allocator@D@2@@2@@Z$4 10000000 f   wzFilePacker_static:wzFilePacker.obj
 0001:fffff000       __unwindfunclet$??0logic_error@std@@QAE@ABV01@@Z$0 10000000 f   xls.obj
 0001:fffff000       __unwindfunclet$??0?$_Tree@V?$_Tmap_traits@HHU?$less@H@std@@V?$allocator@U?$pair@$$CBHH@std@@@2@$0A@@std@@@std@@QAE@ABU?$less@H@1@ABV?$allocator@U?$pair@$$CBHH@std@@@1@@Z$0 10000000 f   scriptparser.obj
 0001:fffff000       __unwindfunclet$?_Xlen@?$vector@UST_CELLS@@V?$allocator@UST_CELLS@@@std@@@std@@KAXXZ$0 10000000 f   xls.obj
 0001:fffff000       __unwindfunclet$?_Insert@?$_Tree@V?$_Tmap_traits@HHU?$less@H@std@@V?$allocator@U?$pair@$$CBHH@std@@@2@$0A@@std@@@std@@IAE?AViterator@12@_NPAU_Node@?$_Tree_nod@V?$_Tmap_traits@HHU?$less@H@std@@V?$allocator@U?$pair@$$CBHH@std@@@2@$0A@@std@@@2@ABU?$pair@$$CBHH@2@@Z$0 10000000 f   scriptparser.obj
 0001:fffff000       __unwindfunclet$?erase@?$_Tree@V?$_Tmap_traits@HHU?$less@H@std@@V?$allocator@U?$pair@$$CBHH@std@@@2@$0A@@std@@@std@@QAE?AViterator@12@Vconst_iterator@12@@Z$0 10000000 f   scriptparser.obj
 0001:fffff000       __ehhandler$?_Copy@?$basic_string@DU?$char_traits@D@std@@V?$allocator@D@2@@std@@IAEXII@Z 10000000 f   libcpmt:string.obj
 0001:fffff000       __unwindfunclet$??1?$_Tree@V?$_Tmap_traits@HHU?$less@H@std@@V?$allocator@U?$pair@$$CBHH@std@@@2@$0A@@std@@@std@@QAE@XZ$0 10000000 f   scriptparser.obj
 0001:fffff000       __ehhandler$?_Copy@?$basic_string@DU?$char_traits@D@std@@V?$allocator@D@2@@std@@IAEXII@Z 10000000 f   eventmusic.obj
 0001:fffff000       __unwindfunclet$??0logic_error@std@@QAE@ABV?$basic_string@DU?$char_traits@D@std@@V?$allocator@D@2@@1@@Z$0 10000000 f   eventmusic.obj
 0001:fffff000       __unwindfunclet$??$_Uninit_move@PAV?$basic_string@DU?$char_traits@D@std@@V?$allocator@D@2@@std@@PAV12@V?$allocator@V?$basic_string@DU?$char_traits@D@std@@V?$allocator@D@2@@std@@@2@@std@@YAPAV?$basic_string@DU?$char_traits@D@std@@V?$allocator@D@2@@0@PAV10@00AAV?$allocator@V?$basic_string@DU?$char_traits@D@std@@V?$allocator@D@2@@std@@@0@U_Swap_move_tag@0@U_Range_checked_iterator_tag@0@@Z$2 10000000 f   wzFilePacker_static:wzFilePacker.obj
 0001:fffff000       __unwindfunclet$?erase@?$_Tree@V?$_Tmap_traits@HHU?$less@H@std@@V?$allocator@U?$pair@$$CBHH@std@@@2@$0A@@std@@@std@@QAE?AViterator@12@Vconst_iterator@12@@Z$0 10000000 f   eventmusic.obj
 0001:fffff000       __unwindfunclet$??0logic_error@std@@QAE@ABV01@@Z$0 10000000 f   eventmusic.obj
 0001:fffff000       __unwindfunclet$?_Insert@?$_Tree@V?$_Tmap_traits@HHU?$less@H@std@@V?$allocator@U?$pair@$$CBHH@std@@@2@$0A@@std@@@std@@IAE?AViterator@12@_NPAU_Node@?$_Tree_nod@V?$_Tmap_traits@HHU?$less@H@std@@V?$allocator@U?$pair@$$CBHH@std@@@2@$0A@@std@@@2@ABU?$pair@$$CBHH@2@@Z$0 10000000 f   eventmusic.obj
 0001:fffff000       __unwindfunclet$??0?$vector@V?$basic_string@DU?$char_traits@D@std@@V?$allocator@D@2@@std@@V?$allocator@V?$basic_string@DU?$char_traits@D@std@@V?$allocator@D@2@@std@@@2@@std@@QAE@XZ$0 10000000 f   wzFilePacker_static:wzFilePacker.obj
 0001:fffff000       __unwindfunclet$??1?$_Tree@V?$_Tmap_traits@HHU?$less@H@std@@V?$allocator@U?$pair@$$CBHH@std@@@2@$0A@@std@@@std@@QAE@XZ$0 10000000 f   eventmusic.obj
 0001:fffff000       __unwindfunclet$??0logic_error@std@@QAE@ABV?$basic_string@DU?$char_traits@D@std@@V?$allocator@D@2@@1@@Z$0 10000000 f   scriptparser.obj
 0001:fffff000       __unwindfunclet$??$_Uninit_fill_n@PAV?$basic_string@DU?$char_traits@D@std@@V?$allocator@D@2@@std@@IV12@V?$allocator@V?$basic_string@DU?$char_traits@D@std@@V?$allocator@D@2@@std@@@2@@std@@YAXPAV?$basic_string@DU?$char_traits@D@std@@V?$allocator@D@2@@0@IABV10@AAV?$allocator@V?$basic_string@DU?$char_traits@D@std@@V?$allocator@D@2@@std@@@0@U_Nonscalar_ptr_iterator_tag@0@U_Range_checked_iterator_tag@0@@Z$2 10000000 f   wzFilePacker_static:wzFilePacker.obj
 0001:fffff000       __ehhandler$?_Copy@?$basic_string@DU?$char_traits@D@std@@V?$allocator@D@2@@std@@IAEXII@Z 10000000 f   ambientsnd.obj
 0001:fffff000       __ehhandler$?_Copy@?$basic_string@DU?$char_traits@D@std@@V?$allocator@D@2@@std@@IAEXII@Z 10000000 f   wzFilePacker_static:wzFilePacker.obj
 0001:fffff000       __unwindfunclet$??0logic_error@std@@QAE@ABV01@@Z$0 10000000 f   wzFilePacker_static:wzFilePacker.obj
 0001:fffff000       __unwindfunclet$??0logic_error@std@@QAE@ABV01@@Z$0 10000000 f   ambientsnd.obj
 0001:fffff000       __unwindfunclet$??$_Construct@V?$basic_string@DU?$char_traits@D@std@@V?$allocator@D@2@@std@@V12@@std@@YAXPAV?$basic_string@DU?$char_traits@D@std@@V?$allocator@D@2@@0@ABV10@@Z$0 10000000 f   wzFilePacker_static:wzFilePacker.obj
 0001:fffff000       __unwindfunclet$?_Xlen@?$vector@V?$basic_string@DU?$char_traits@D@std@@V?$allocator@D@2@@std@@V?$allocator@V?$basic_string@DU?$char_traits@D@std@@V?$allocator@D@2@@std@@@2@@std@@KAXXZ$0 10000000 f   wzFilePacker_static:wzFilePacker.obj
 0001:fffff000       __unwindfunclet$??0logic_error@std@@QAE@ABV?$basic_string@DU?$char_traits@D@std@@V?$allocator@D@2@@1@@Z$0 10000000 f   ambientsnd.obj
 0001:fffff000       __unwindfunclet$??0logic_error@std@@QAE@ABV?$basic_string@DU?$char_traits@D@std@@V?$allocator@D@2@@1@@Z$0 10000000 f   wzFilePacker_static:wzFilePacker.obj
 0001:fffff008       __unwindfunclet$?_Insert_n@?$vector@V?$basic_string@DU?$char_traits@D@std@@V?$allocator@D@2@@std@@V?$allocator@V?$basic_string@DU?$char_traits@D@std@@V?$allocator@D@2@@std@@@2@@std@@IAEXV?$_Vector_const_iterator@V?$basic_string@DU?$char_traits@D@std@@V?$allocator@D@2@@std@@V?$allocator@V?$basic_string@DU?$char_traits@D@std@@V?$allocator@D@2@@std@@@2@@2@IABV?$basic_string@DU?$char_traits@D@std@@V?$allocator@D@2@@2@@Z$5 10000008 f   wzFilePacker_static:wzFilePacker.obj
 0001:fffff008       __ehhandler$??0logic_error@std@@QAE@ABV?$basic_string@DU?$char_traits@D@std@@V?$allocator@D@2@@1@@Z 10000008 f   ambientsnd.obj
 0001:fffff008       __ehhandler$??0logic_error@std@@QAE@ABV?$basic_string@DU?$char_traits@D@std@@V?$allocator@D@2@@1@@Z 10000008 f   wzFilePacker_static:wzFilePacker.obj
 0001:fffff008       __ehhandler$?_Xlen@?$vector@V?$basic_string@DU?$char_traits@D@std@@V?$allocator@D@2@@std@@V?$allocator@V?$basic_string@DU?$char_traits@D@std@@V?$allocator@D@2@@std@@@2@@std@@KAXXZ 10000008 f   wzFilePacker_static:wzFilePacker.obj
 0001:fffff008       __ehhandler$??0logic_error@std@@QAE@ABV01@@Z 10000008 f   wzFilePacker_static:wzFilePacker.obj
 0001:fffff008       __ehhandler$??0logic_error@std@@QAE@ABV01@@Z 10000008 f   ambientsnd.obj
 0001:fffff008       __ehhandler$??0logic_error@std@@QAE@ABV?$basic_string@DU?$char_traits@D@std@@V?$allocator@D@2@@1@@Z 10000008 f   scriptparser.obj
 0001:fffff008       __ehhandler$??0logic_error@std@@QAE@ABV?$basic_string@DU?$char_traits@D@std@@V?$allocator@D@2@@1@@Z 10000008 f   wzSound.obj
 0001:fffff008       __ehhandler$??0logic_error@std@@QAE@ABV01@@Z 10000008 f   scriptparser.obj
 0001:fffff008       __ehhandler$??1?$_Tree@V?$_Tmap_traits@HHU?$less@H@std@@V?$allocator@U?$pair@$$CBHH@std@@@2@$0A@@std@@@std@@QAE@XZ 10000008 f   voicesnd.obj
 0001:fffff008       __ehhandler$??1?$_Tree@V?$_Tmap_traits@HHU?$less@H@std@@V?$allocator@U?$pair@$$CBHH@std@@@2@$0A@@std@@@std@@QAE@XZ 10000008 f   eventmusic.obj
 0001:fffff008       __ehhandler$??0logic_error@std@@QAE@ABV?$basic_string@DU?$char_traits@D@std@@V?$allocator@D@2@@1@@Z 10000008 f   xls.obj
 0001:fffff008       __ehhandler$?_Insert@?$_Tree@V?$_Tmap_traits@HHU?$less@H@std@@V?$allocator@U?$pair@$$CBHH@std@@@2@$0A@@std@@@std@@IAE?AViterator@12@_NPAU_Node@?$_Tree_nod@V?$_Tmap_traits@HHU?$less@H@std@@V?$allocator@U?$pair@$$CBHH@std@@@2@$0A@@std@@@2@ABU?$pair@$$CBHH@2@@Z 10000008 f   eventmusic.obj
 0001:fffff008       __ehhandler$??0?$vector@V?$basic_string@DU?$char_traits@D@std@@V?$allocator@D@2@@std@@V?$allocator@V?$basic_string@DU?$char_traits@D@std@@V?$allocator@D@2@@std@@@2@@std@@QAE@XZ 10000008 f   wzFilePacker_static:wzFilePacker.obj
 0001:fffff008       __ehhandler$??0?$_Tree@V?$_Tmap_traits@HHU?$less@H@std@@V?$allocator@U?$pair@$$CBHH@std@@@2@$0A@@std@@@std@@QAE@ABU?$less@H@1@ABV?$allocator@U?$pair@$$CBHH@std@@@1@@Z 10000008 f   eventmusic.obj
 0001:fffff008       __ehhandler$?_Insert@?$_Tree@V?$_Tmap_traits@HHU?$less@H@std@@V?$allocator@U?$pair@$$CBHH@std@@@2@$0A@@std@@@std@@IAE?AViterator@12@_NPAU_Node@?$_Tree_nod@V?$_Tmap_traits@HHU?$less@H@std@@V?$allocator@U?$pair@$$CBHH@std@@@2@$0A@@std@@@2@ABU?$pair@$$CBHH@2@@Z 10000008 f   wzSound.obj
 0001:fffff008       __ehhandler$??0logic_error@std@@QAE@ABV01@@Z 10000008 f   eventmusic.obj
 0001:fffff008       __ehhandler$?_Insert@?$_Tree@V?$_Tmap_traits@HHU?$less@H@std@@V?$allocator@U?$pair@$$CBHH@std@@@2@$0A@@std@@@std@@IAE?AViterator@12@_NPAU_Node@?$_Tree_nod@V?$_Tmap_traits@HHU?$less@H@std@@V?$allocator@U?$pair@$$CBHH@std@@@2@$0A@@std@@@2@ABU?$pair@$$CBHH@2@@Z 10000008 f   voicesnd.obj
 0001:fffff008       __ehhandler$?erase@?$_Tree@V?$_Tmap_traits@HHU?$less@H@std@@V?$allocator@U?$pair@$$CBHH@std@@@2@$0A@@std@@@std@@QAE?AViterator@12@Vconst_iterator@12@@Z 10000008 f   eventmusic.obj
 0001:fffff008       __unwindfunclet$??$_Uninit_move@PAV?$basic_string@DU?$char_traits@D@std@@V?$allocator@D@2@@std@@PAV12@V?$allocator@V?$basic_string@DU?$char_traits@D@std@@V?$allocator@D@2@@std@@@2@@std@@YAPAV?$basic_string@DU?$char_traits@D@std@@V?$allocator@D@2@@0@PAV10@00AAV?$allocator@V?$basic_string@DU?$char_traits@D@std@@V?$allocator@D@2@@std@@@0@U_Swap_move_tag@0@U_Range_checked_iterator_tag@0@@Z$3 10000008 f   wzFilePacker_static:wzFilePacker.obj
 0001:fffff008       __ehhandler$??0logic_error@std@@QAE@ABV?$basic_string@DU?$char_traits@D@std@@V?$allocator@D@2@@1@@Z 10000008 f   eventmusic.obj
 0001:fffff008       __ehhandler$??0logic_error@std@@QAE@ABV01@@Z 10000008 f   wzSound.obj
 0001:fffff008       __ehhandler$??0?$_Tree@V?$_Tmap_traits@HHU?$less@H@std@@V?$allocator@U?$pair@$$CBHH@std@@@2@$0A@@std@@@std@@QAE@ABU?$less@H@1@ABV?$allocator@U?$pair@$$CBHH@std@@@1@@Z 10000008 f   voicesnd.obj
 0001:fffff008       __ehhandler$??0logic_error@std@@QAE@ABV01@@Z 10000008 f   libcpmt:string.obj
 0001:fffff008       __ehhandler$??0logic_error@std@@QAE@ABV01@@Z 10000008 f   voicesnd.obj
 0001:fffff008       __ehhandler$??1?$_Tree@V?$_Tmap_traits@HHU?$less@H@std@@V?$allocator@U?$pair@$$CBHH@std@@@2@$0A@@std@@@std@@QAE@XZ 10000008 f   scriptparser.obj
 0001:fffff008       __ehhandler$?erase@?$_Tree@V?$_Tmap_traits@HHU?$less@H@std@@V?$allocator@U?$pair@$$CBHH@std@@@2@$0A@@std@@@std@@QAE?AViterator@12@Vconst_iterator@12@@Z 10000008 f   voicesnd.obj
 0001:fffff008       __ehhandler$?erase@?$_Tree@V?$_Tmap_traits@HHU?$less@H@std@@V?$allocator@U?$pair@$$CBHH@std@@@2@$0A@@std@@@std@@QAE?AViterator@12@Vconst_iterator@12@@Z 10000008 f   scriptparser.obj
 0001:fffff008       __ehhandler$??0logic_error@std@@QAE@ABV?$basic_string@DU?$char_traits@D@std@@V?$allocator@D@2@@1@@Z 10000008 f   voicesnd.obj
 0001:fffff008       __ehhandler$?_Insert@?$_Tree@V?$_Tmap_traits@HHU?$less@H@std@@V?$allocator@U?$pair@$$CBHH@std@@@2@$0A@@std@@@std@@IAE?AViterator@12@_NPAU_Node@?$_Tree_nod@V?$_Tmap_traits@HHU?$less@H@std@@V?$allocator@U?$pair@$$CBHH@std@@@2@$0A@@std@@@2@ABU?$pair@$$CBHH@2@@Z 10000008 f   scriptparser.obj
 0001:fffff008       __ehhandler$?_Xlen@?$vector@UST_CELLS@@V?$allocator@UST_CELLS@@@std@@@std@@KAXXZ 10000008 f   xls.obj
 0001:fffff008       __ehhandler$??0?$_Tree@V?$_Tmap_traits@HHU?$less@H@std@@V?$allocator@U?$pair@$$CBHH@std@@@2@$0A@@std@@@std@@QAE@ABU?$less@H@1@ABV?$allocator@U?$pair@$$CBHH@std@@@1@@Z 10000008 f   scriptparser.obj
 0001:fffff008       __ehhandler$??0logic_error@std@@QAE@ABV01@@Z 10000008 f   xls.obj
 0001:fffff008       __ehhandler$?_Insert@?$_Tree@V?$_Tmap_traits@HUAmbientSnd@@U?$less@H@std@@V?$allocator@U?$pair@$$CBHUAmbientSnd@@@std@@@3@$0A@@std@@@std@@IAE?AViterator@12@_NPAU_Node@?$_Tree_nod@V?$_Tmap_traits@HUAmbientSnd@@U?$less@H@std@@V?$allocator@U?$pair@$$CBHUAmbientSnd@@@std@@@3@$0A@@std@@@2@ABU?$pair@$$CBHUAmbientSnd@@@2@@Z 10000008 f   scriptparser.obj
 0001:fffff008       __ehhandler$??0logic_error@std@@QAE@ABV?$basic_string@DU?$char_traits@D@std@@V?$allocator@D@2@@1@@Z 10000008 f   libcpmt:string.obj
 0001:fffff010       __ehhandler$?_Insert_n@?$vector@V?$basic_string@DU?$char_traits@D@std@@V?$allocator@D@2@@std@@V?$allocator@V?$basic_string@DU?$char_traits@D@std@@V?$allocator@D@2@@std@@@2@@std@@IAEXV?$_Vector_const_iterator@V?$basic_string@DU?$char_traits@D@std@@V?$allocator@D@2@@std@@V?$allocator@V?$basic_string@DU?$char_traits@D@std@@V?$allocator@D@2@@std@@@2@@2@IABV?$basic_string@DU?$char_traits@D@std@@V?$allocator@D@2@@2@@Z 10000010 f   wzFilePacker_static:wzFilePacker.obj
 0001:fffff011       __ehhandler$??$_Uninit_fill_n@PAV?$basic_string@DU?$char_traits@D@std@@V?$allocator@D@2@@std@@IV12@V?$allocator@V?$basic_string@DU?$char_traits@D@std@@V?$allocator@D@2@@std@@@2@@std@@YAXPAV?$basic_string@DU?$char_traits@D@std@@V?$allocator@D@2@@0@IABV10@AAV?$allocator@V?$basic_string@DU?$char_traits@D@std@@V?$allocator@D@2@@std@@@0@U_Nonscalar_ptr_iterator_tag@0@U_Range_checked_iterator_tag@0@@Z 10000011 f   wzFilePacker_static:wzFilePacker.obj
 0001:fffff011       __ehhandler$??$_Construct@V?$basic_string@DU?$char_traits@D@std@@V?$allocator@D@2@@std@@V12@@std@@YAXPAV?$basic_string@DU?$char_traits@D@std@@V?$allocator@D@2@@0@ABV10@@Z 10000011 f   wzFilePacker_static:wzFilePacker.obj
 0001:fffff019       __ehhandler$??$_Uninit_move@PAV?$basic_string@DU?$char_traits@D@std@@V?$allocator@D@2@@std@@PAV12@V?$allocator@V?$basic_string@DU?$char_traits@D@std@@V?$allocator@D@2@@std@@@2@@std@@YAPAV?$basic_string@DU?$char_traits@D@std@@V?$allocator@D@2@@0@PAV10@00AAV?$allocator@V?$basic_string@DU?$char_traits@D@std@@V?$allocator@D@2@@std@@@0@U_Swap_move_tag@0@U_Range_checked_iterator_tag@0@@Z 10000019 f   wzFilePacker_static:wzFilePacker.obj
 0001:fffff059       __catch$?_Copy@?$basic_string@DU?$char_traits@D@std@@V?$allocator@D@2@@std@@IAEXII@Z$0 10000059 f   libcpmt:string.obj
 0001:fffff079       __catch$??$_Uninit_fill_n@PAV?$basic_string@DU?$char_traits@D@std@@V?$allocator@D@2@@std@@IV12@V?$allocator@V?$basic_string@DU?$char_traits@D@std@@V?$allocator@D@2@@std@@@2@@std@@YAXPAV?$basic_string@DU?$char_traits@D@std@@V?$allocator@D@2@@0@IABV10@AAV?$allocator@V?$basic_string@DU?$char_traits@D@std@@V?$allocator@D@2@@std@@@0@U_Nonscalar_ptr_iterator_tag@0@U_Range_checked_iterator_tag@0@@Z$0 10000079 f   wzFilePacker_static:wzFilePacker.obj
 0001:fffff07d       __catch$?_Copy@?$basic_string@DU?$char_traits@D@std@@V?$allocator@D@2@@std@@IAEXII@Z$0 1000007d f   scriptparser.obj
 0001:fffff07d       __catch$?_Copy@?$basic_string@DU?$char_traits@D@std@@V?$allocator@D@2@@std@@IAEXII@Z$0 1000007d f   xls.obj
 0001:fffff07d       __catch$?_Copy@?$basic_string@DU?$char_traits@D@std@@V?$allocator@D@2@@std@@IAEXII@Z$0 1000007d f   wzSound.obj
 0001:fffff07d       __catch$?_Copy@?$basic_string@DU?$char_traits@D@std@@V?$allocator@D@2@@std@@IAEXII@Z$0 1000007d f   eventmusic.obj
 0001:fffff07d       __catch$?_Copy@?$basic_string@DU?$char_traits@D@std@@V?$allocator@D@2@@std@@IAEXII@Z$0 1000007d f   ambientsnd.obj
 0001:fffff07d       __catch$?_Copy@?$basic_string@DU?$char_traits@D@std@@V?$allocator@D@2@@std@@IAEXII@Z$0 1000007d f   voicesnd.obj
 0001:fffff07d       __catch$?_Copy@?$basic_string@DU?$char_traits@D@std@@V?$allocator@D@2@@std@@IAEXII@Z$0 1000007d f   wzFilePacker_static:wzFilePacker.obj
 0001:fffff095       __catch$??$_Uninit_move@PAV?$basic_string@DU?$char_traits@D@std@@V?$allocator@D@2@@std@@PAV12@V?$allocator@V?$basic_string@DU?$char_traits@D@std@@V?$allocator@D@2@@std@@@2@@std@@YAPAV?$basic_string@DU?$char_traits@D@std@@V?$allocator@D@2@@0@PAV10@00AAV?$allocator@V?$basic_string@DU?$char_traits@D@std@@V?$allocator@D@2@@std@@@0@U_Swap_move_tag@0@U_Range_checked_iterator_tag@0@@Z$0 10000095 f   wzFilePacker_static:wzFilePacker.obj
 0001:fffff0ca       __catch$?_Copy@?$basic_string@DU?$char_traits@D@std@@V?$allocator@D@2@@std@@IAEXII@Z$1 100000ca f   libcpmt:string.obj
 0001:fffff10e       __catch$?_Copy@?$basic_string@DU?$char_traits@D@std@@V?$allocator@D@2@@std@@IAEXII@Z$1 1000010e f   ambientsnd.obj
 0001:fffff10e       __catch$?_Copy@?$basic_string@DU?$char_traits@D@std@@V?$allocator@D@2@@std@@IAEXII@Z$1 1000010e f   wzFilePacker_static:wzFilePacker.obj
 0001:fffff10e       __catch$?_Copy@?$basic_string@DU?$char_traits@D@std@@V?$allocator@D@2@@std@@IAEXII@Z$1 1000010e f   eventmusic.obj
 0001:fffff10e       __catch$?_Copy@?$basic_string@DU?$char_traits@D@std@@V?$allocator@D@2@@std@@IAEXII@Z$1 1000010e f   scriptparser.obj
 0001:fffff10e       __catch$?_Copy@?$basic_string@DU?$char_traits@D@std@@V?$allocator@D@2@@std@@IAEXII@Z$1 1000010e f   xls.obj
 0001:fffff10e       __catch$?_Copy@?$basic_string@DU?$char_traits@D@std@@V?$allocator@D@2@@std@@IAEXII@Z$1 1000010e f   voicesnd.obj
 0001:fffff10e       __catch$?_Copy@?$basic_string@DU?$char_traits@D@std@@V?$allocator@D@2@@std@@IAEXII@Z$1 1000010e f   wzSound.obj
 0001:fffff1e8       __catch$?_Insert_n@?$vector@V?$basic_string@DU?$char_traits@D@std@@V?$allocator@D@2@@std@@V?$allocator@V?$basic_string@DU?$char_traits@D@std@@V?$allocator@D@2@@std@@@2@@std@@IAEXV?$_Vector_const_iterator@V?$basic_string@DU?$char_traits@D@std@@V?$allocator@D@2@@std@@V?$allocator@V?$basic_string@DU?$char_traits@D@std@@V?$allocator@D@2@@std@@@2@@2@IABV?$basic_string@DU?$char_traits@D@std@@V?$allocator@D@2@@2@@Z$0 100001e8 f   wzFilePacker_static:wzFilePacker.obj
 0001:fffff2f2       __catch$?_Insert_n@?$vector@V?$basic_string@DU?$char_traits@D@std@@V?$allocator@D@2@@std@@V?$allocator@V?$basic_string@DU?$char_traits@D@std@@V?$allocator@D@2@@std@@@2@@std@@IAEXV?$_Vector_const_iterator@V?$basic_string@DU?$char_traits@D@std@@V?$allocator@D@2@@std@@V?$allocator@V?$basic_string@DU?$char_traits@D@std@@V?$allocator@D@2@@std@@@2@@2@IABV?$basic_string@DU?$char_traits@D@std@@V?$allocator@D@2@@2@@Z$2 100002f2 f   wzFilePacker_static:wzFilePacker.obj
 0001:00005a2d       __catch$?_Copy@?$basic_string@DU?$char_traits@D@std@@V?$allocator@D@2@@std@@IAEXII@Z$0 10006a2d f i sound.obj
 0001:00005abe       __catch$?_Copy@?$basic_string@DU?$char_traits@D@std@@V?$allocator@D@2@@std@@IAEXII@Z$1 10006abe f i sound.obj
 0001:00009310       ?check_AmbiHandle@@YAHH@Z  1000a310 f   ambientsnd.obj
 0001:0000a730       ?check_MusicHandle@@YAHH@Z 1000b730 f   eventmusic.obj
 0001:0000af80       ?gamesnd_init_struct@@YAXPAUgame_snd@@@Z 1000bf80 f   scriptparser.obj
 0001:00010ad0       ?check_VoiceHandle@@YAHH@Z 10011ad0 f   voicesnd.obj
 0001:00010da0       ?timer_get@@YAIXZ          10011da0 f   timer.obj
 0001:00011050       ?open_mixer@@YAHIH@Z       10012050 f   util_audiomixer.obj
 0001:00012f70       _ascii_width               10013f70 f   util_shwapi.obj
 0001:00012f80       _ascii_cwidth              10013f80 f   util_shwapi.obj
 0001:00012f90       __getc                     10013f90 f   util_shwapi.obj
 0001:00012fa0       __getx                     10013fa0 f   util_shwapi.obj
 0001:00012fb0       __setc                     10013fb0 f   util_shwapi.obj
 0001:0001c1a9       __catch$??$_Uninit_copy@PBV?$basic_string@DU?$char_traits@D@std@@V?$allocator@D@2@@std@@PAV12@V?$allocator@V?$basic_string@DU?$char_traits@D@std@@V?$allocator@D@2@@std@@@2@@std@@YAPAV?$basic_string@DU?$char_traits@D@std@@V?$allocator@D@2@@0@PBV10@0PAV10@AAV?$allocator@V?$basic_string@DU?$char_traits@D@std@@V?$allocator@D@2@@std@@@0@U_Nonscalar_ptr_iterator_tag@0@U_Range_checked_iterator_tag@0@@Z$0 1001d1a9 f i xls.obj
 0001:0001c2d9       __catch$??$_Uninit_copy@PAV?$basic_string@DU?$char_traits@D@std@@V?$allocator@D@2@@std@@PAV12@V?$allocator@V?$basic_string@DU?$char_traits@D@std@@V?$allocator@D@2@@std@@@2@@std@@YAPAV?$basic_string@DU?$char_traits@D@std@@V?$allocator@D@2@@0@PAV10@00AAV?$allocator@V?$basic_string@DU?$char_traits@D@std@@V?$allocator@D@2@@std@@@0@U_Nonscalar_ptr_iterator_tag@0@U_Range_checked_iterator_tag@0@@Z$0 1001d2d9 f i xls.obj
 0001:0001c429       __catch$??$_Uninit_fill_n@PAV?$basic_string@DU?$char_traits@D@std@@V?$allocator@D@2@@std@@IV12@V?$allocator@V?$basic_string@DU?$char_traits@D@std@@V?$allocator@D@2@@std@@@2@@std@@YAXPAV?$basic_string@DU?$char_traits@D@std@@V?$allocator@D@2@@0@IABV10@AAV?$allocator@V?$basic_string@DU?$char_traits@D@std@@V?$allocator@D@2@@std@@@0@U_Nonscalar_ptr_iterator_tag@0@U_Range_checked_iterator_tag@0@@Z$0 1001d429 f i xls.obj
 0001:0001c705       __catch$??$_Uninit_move@PAV?$basic_string@DU?$char_traits@D@std@@V?$allocator@D@2@@std@@PAV12@V?$allocator@V?$basic_string@DU?$char_traits@D@std@@V?$allocator@D@2@@std@@@2@@std@@YAPAV?$basic_string@DU?$char_traits@D@std@@V?$allocator@D@2@@0@PAV10@00AAV?$allocator@V?$basic_string@DU?$char_traits@D@std@@V?$allocator@D@2@@std@@@0@U_Swap_move_tag@0@U_Range_checked_iterator_tag@0@@Z$0 1001d705 f i xls.obj
 0001:0001c8e0       __catch$??0?$vector@V?$basic_string@DU?$char_traits@D@std@@V?$allocator@D@2@@std@@V?$allocator@V?$basic_string@DU?$char_traits@D@std@@V?$allocator@D@2@@std@@@2@@std@@QAE@ABV01@@Z$0 1001d8e0 f i xls.obj
 0001:0001ce38       __catch$?_Insert_n@?$vector@V?$basic_string@DU?$char_traits@D@std@@V?$allocator@D@2@@std@@V?$allocator@V?$basic_string@DU?$char_traits@D@std@@V?$allocator@D@2@@std@@@2@@std@@IAEXV?$_Vector_const_iterator@V?$basic_string@DU?$char_traits@D@std@@V?$allocator@D@2@@std@@V?$allocator@V?$basic_string@DU?$char_traits@D@std@@V?$allocator@D@2@@std@@@2@@2@IABV?$basic_string@DU?$char_traits@D@std@@V?$allocator@D@2@@2@@Z$0 1001de38 f i xls.obj
 0001:0001cf42       __catch$?_Insert_n@?$vector@V?$basic_string@DU?$char_traits@D@std@@V?$allocator@D@2@@std@@V?$allocator@V?$basic_string@DU?$char_traits@D@std@@V?$allocator@D@2@@std@@@2@@std@@IAEXV?$_Vector_const_iterator@V?$basic_string@DU?$char_traits@D@std@@V?$allocator@D@2@@std@@V?$allocator@V?$basic_string@DU?$char_traits@D@std@@V?$allocator@D@2@@std@@@2@@2@IABV?$basic_string@DU?$char_traits@D@std@@V?$allocator@D@2@@2@@Z$2 1001df42 f i xls.obj
 0001:0001d329       __catch$??$_Uninit_copy@PAUST_CELLS@@PAU1@V?$allocator@UST_CELLS@@@std@@@std@@YAPAUST_CELLS@@PAU1@00AAV?$allocator@UST_CELLS@@@0@U_Nonscalar_ptr_iterator_tag@0@U_Range_checked_iterator_tag@0@@Z$0 1001e329 f i xls.obj
 0001:0001d3f9       __catch$??$_Uninit_fill_n@PAUST_CELLS@@IU1@V?$allocator@UST_CELLS@@@std@@@std@@YAXPAUST_CELLS@@IABU1@AAV?$allocator@UST_CELLS@@@0@U_Nonscalar_ptr_iterator_tag@0@U_Range_checked_iterator_tag@0@@Z$0 1001e3f9 f i xls.obj
 0001:0001d72e       __catch$?_Insert_n@?$vector@UST_CELLS@@V?$allocator@UST_CELLS@@@std@@@std@@IAEXV?$_Vector_const_iterator@UST_CELLS@@V?$allocator@UST_CELLS@@@std@@@2@IABUST_CELLS@@@Z$0 1001e72e f i xls.obj
 0001:0001d84d       __catch$?_Insert_n@?$vector@UST_CELLS@@V?$allocator@UST_CELLS@@@std@@@std@@IAEXV?$_Vector_const_iterator@UST_CELLS@@V?$allocator@UST_CELLS@@@std@@@2@IABUST_CELLS@@@Z$2 1001e84d f i xls.obj
 0001:0001dfc0       ?get_brbdnum@@YAHH@Z       1001efc0 f   xlstool.obj
 0001:0001e050       ?convert@@YAPADPBDHPAH00@Z 1001f050 f   xlstool.obj
 0001:00020bc0       __ov_open1                 10021bc0 f   vorbisfile_static:vorbisfile.obj
 0001:00020ce0       __fetch_headers            10021ce0 f   vorbisfile_static:vorbisfile.obj
 0001:00020e30       __get_next_page            10021e30 f   vorbisfile_static:vorbisfile.obj
 0001:00020ef0       __get_data                 10021ef0 f   vorbisfile_static:vorbisfile.obj
 0001:00020f60       __ov_open2                 10021f60 f   vorbisfile_static:vorbisfile.obj
 0001:00020fb0       __open_seekable2           10021fb0 f   vorbisfile_static:vorbisfile.obj
 0001:000210b0       __get_prev_page            100220b0 f   vorbisfile_static:vorbisfile.obj
 0001:000211d0       __seek_helper              100221d0 f   vorbisfile_static:vorbisfile.obj
 0001:00021210       __bisect_forward_serialno  10022210 f   vorbisfile_static:vorbisfile.obj
 0001:00021430       __prefetch_all_headers     10022430 f   vorbisfile_static:vorbisfile.obj
 0001:00021760       __fseek64_wrap             10022760 f   vorbisfile_static:vorbisfile.obj
 0001:00021810       __decode_clear             10022810 f   vorbisfile_static:vorbisfile.obj
 0001:000228d0       __make_decode_ready        100238d0 f   vorbisfile_static:vorbisfile.obj
 0001:00022950       __fetch_and_process_packet 10023950 f   vorbisfile_static:vorbisfile.obj
 0001:00023330       _host_is_big_endian        10024330 f   vorbisfile_static:vorbisfile.obj
 0001:000235b0       __ov_splice                100245b0 f   vorbisfile_static:vorbisfile.obj
 0001:00023690       __ov_initset               10024690 f   vorbisfile_static:vorbisfile.obj
 0001:000236c0       __ov_initprime             100246c0 f   vorbisfile_static:vorbisfile.obj
 0001:00023710       __ov_getlap                10024710 f   vorbisfile_static:vorbisfile.obj
 0001:000238d0       __ov_64_seek_lap           100248d0 f   vorbisfile_static:vorbisfile.obj
 0001:00023a80       __ov_d_seek_lap            10024a80 f   vorbisfile_static:vorbisfile.obj
 0001:00023e60       _tagcompare                10024e60 f   vorbisfile_static:info.obj
 0001:000242a0       __v_readstring             100252a0 f   vorbisfile_static:info.obj
 0001:000242d0       __vorbis_unpack_info       100252d0 f   vorbisfile_static:info.obj
 0001:000243b0       __vorbis_unpack_comment    100253b0 f   vorbisfile_static:info.obj
 0001:00024490       __vorbis_unpack_books      10025490 f   vorbisfile_static:info.obj
 0001:000247a0       __vorbis_pack_comment      100257a0 f   vorbisfile_static:info.obj
 0001:00024870       __v_writestring            10025870 f   vorbisfile_static:info.obj
 0001:00024b00       __vorbis_pack_info         10025b00 f   vorbisfile_static:info.obj
 0001:00024bc0       _ilog2                     10025bc0 f   vorbisfile_static:info.obj
 0001:00024be0       __vorbis_pack_books        10025be0 f   vorbisfile_static:info.obj
 0001:00025000       __vds_shared_init          10026000 f   vorbisfile_static:block.obj
 0001:000253a0       _ilog2                     100263a0 f   vorbisfile_static:block.obj
 0001:00025810       __preextrapolate_helper    10026810 f   vorbisfile_static:block.obj
 0001:00026b20       _todB                      10027b20 f   vorbisfile_static:analysis.obj
 0001:00027130       _setup_tone_curves         10028130 f   vorbisfile_static:psy.obj
 0001:000278b0       _min_curve                 100288b0 f   vorbisfile_static:psy.obj
 0001:000278e0       _max_curve                 100288e0 f   vorbisfile_static:psy.obj
 0001:00027910       _attenuate_curve           10028910 f   vorbisfile_static:psy.obj
 0001:00027b40       _bark_noise_hybridmp       10028b40 f   vorbisfile_static:psy.obj
 0001:000281b0       _seed_loop                 100291b0 f   vorbisfile_static:psy.obj
 0001:00028290       _seed_curve                10029290 f   vorbisfile_static:psy.obj
 0001:00028360       _max_seeds                 10029360 f   vorbisfile_static:psy.obj
 0001:000284a0       _seed_chase                100294a0 f   vorbisfile_static:psy.obj
 0001:00028830       _dipole_hypot              10029830 f   vorbisfile_static:psy.obj
 0001:00028900       _round_hypot               10029900 f   vorbisfile_static:psy.obj
 0001:00028af0       _apsort                    10029af0 f   vorbisfile_static:psy.obj
 0001:00028e60       _unitnorm                  10029e60 f   vorbisfile_static:psy.obj
 0001:00029270       _couple_lossless           1002a270 f   vorbisfile_static:psy.obj
 0001:00029340       _precomputed_couple_point  1002a340 f   vorbisfile_static:psy.obj
 0001:00029e00       _bitreverse                1002ae00 f   vorbisfile_static:sharedbook.obj
 0001:00029e60       _sort32a                   1002ae60 f   vorbisfile_static:sharedbook.obj
 0001:00029ff0       __dist                     1002aff0 f   vorbisfile_static:sharedbook.obj
 0001:0002a700       _bitreverse                1002b700 f   vorbisfile_static:codebook.obj
 0001:0002bde0       _BINBYTES                  1002cde0 f   vorbisfile_static:bitrate.obj
 0001:0002be00       _LACING_ADJUST             1002ce00 f   vorbisfile_static:bitrate.obj
 0001:0002be20       _floater_interpolate       1002ce20 f   vorbisfile_static:bitrate.obj
 0001:0002bf00       _limit_sum                 1002cf00 f   vorbisfile_static:bitrate.obj
 0001:0002c4b0       __ve_amp                   1002d4b0 f   vorbisfile_static:envelope.obj
 0001:0002c820       _todB                      1002d820 f   vorbisfile_static:envelope.obj
 0001:0002c9c0       _drftf1                    1002d9c0 f   vorbisfile_static:smallft.obj
 0001:0002cb70       _dradf2                    1002db70 f   vorbisfile_static:smallft.obj
 0001:0002cd30       _dradf4                    1002dd30 f   vorbisfile_static:smallft.obj
 0001:0002d1a0       _dradfg                    1002e1a0 f   vorbisfile_static:smallft.obj
 0001:0002dd80       _drftb1                    1002ed80 f   vorbisfile_static:smallft.obj
 0001:0002df40       _dradb2                    1002ef40 f   vorbisfile_static:smallft.obj
 0001:0002e0f0       _dradb3                    1002f0f0 f   vorbisfile_static:smallft.obj
 0001:0002e3c0       _dradb4                    1002f3c0 f   vorbisfile_static:smallft.obj
 0001:0002e8b0       _dradbg                    1002f8b0 f   vorbisfile_static:smallft.obj
 0001:0002f3a0       _fdrffti                   100303a0 f   vorbisfile_static:smallft.obj
 0001:0002f3c0       _drfti1                    100303c0 f   vorbisfile_static:smallft.obj
 0001:0002fcc0       _mdct_butterfly_32         10030cc0 f   vorbisfile_static:mdct.obj
 0001:000301c0       _mdct_butterfly_8          100311c0 f   vorbisfile_static:mdct.obj
 0001:00030250       _mdct_butterfly_generic    10031250 f   vorbisfile_static:mdct.obj
 0001:00030bb0       _mapping0_free_info        10031bb0 f   vorbisfile_static:mapping0.obj
 0001:00030bd0       _mapping0_pack             10031bd0 f   vorbisfile_static:mapping0.obj
 0001:00030d20       _ilog                      10031d20 f   vorbisfile_static:mapping0.obj
 0001:00030d40       _mapping0_unpack           10031d40 f   vorbisfile_static:mapping0.obj
 0001:00030f10       _mapping0_forward          10031f10 f   vorbisfile_static:mapping0.obj
 0001:00031890       _todB                      10032890 f   vorbisfile_static:mapping0.obj
 0001:000318c0       _mapping0_inverse          100328c0 f   vorbisfile_static:mapping0.obj
 0001:00031dc0       _ilog                      10032dc0 f   vorbisfile_static:res0.obj
 0001:00031dd0       _icount                    10032dd0 f   vorbisfile_static:res0.obj
 0001:00032170       __01inverse                10033170 f   vorbisfile_static:res0.obj
 0001:000324b0       __encodepart               100334b0 f   vorbisfile_static:res0.obj
 0001:00032510       _local_book_besterror      10033510 f   vorbisfile_static:res0.obj
 0001:000326d0       __01forward                100336d0 f   vorbisfile_static:res0.obj
 0001:000329a0       __01class                  100339a0 f   vorbisfile_static:res0.obj
 0001:00032c70       __2class                   10033c70 f   vorbisfile_static:res0.obj
 0001:00033110       _floor1_free_info          10034110 f   vorbisfile_static:floor1.obj
 0001:00033130       _floor1_free_look          10034130 f   vorbisfile_static:floor1.obj
 0001:00033150       _floor1_pack               10034150 f   vorbisfile_static:floor1.obj
 0001:00033310       _ilog2                     10034310 f   vorbisfile_static:floor1.obj
 0001:00033330       _floor1_unpack             10034330 f   vorbisfile_static:floor1.obj
 0001:00033560       _floor1_look               10034560 f   vorbisfile_static:floor1.obj
 0001:00033780       _icomp                     10034780 f   vorbisfile_static:floor1.obj
 0001:00033c60       _render_point              10034c60 f   vorbisfile_static:floor1.obj
 0001:00033cb0       _accumulate_fit            10034cb0 f   vorbisfile_static:floor1.obj
 0001:00033ea0       _vorbis_dBquant            10034ea0 f   vorbisfile_static:floor1.obj
 0001:00033ed0       _fit_line                  10034ed0 f   vorbisfile_static:floor1.obj
 0001:000340e0       _inspect_error             100350e0 f   vorbisfile_static:floor1.obj
 0001:00034310       _post_Y                    10035310 f   vorbisfile_static:floor1.obj
 0001:000349e0       _ilog                      100359e0 f   vorbisfile_static:floor1.obj
 0001:000349f0       _render_line0              100359f0 f   vorbisfile_static:floor1.obj
 0001:00034a80       _floor1_inverse1           10035a80 f   vorbisfile_static:floor1.obj
 0001:00034d70       _floor1_inverse2           10035d70 f   vorbisfile_static:floor1.obj
 0001:00034e80       _render_line               10035e80 f   vorbisfile_static:floor1.obj
 0001:00034f40       _floor0_free_info          10035f40 f   vorbisfile_static:floor0.obj
 0001:00034f60       _floor0_free_look          10035f60 f   vorbisfile_static:floor0.obj
 0001:00034fc0       _floor0_unpack             10035fc0 f   vorbisfile_static:floor0.obj
 0001:00035080       _floor0_look               10036080 f   vorbisfile_static:floor0.obj
 0001:000350b0       _floor0_inverse1           100360b0 f   vorbisfile_static:floor0.obj
 0001:000351f0       _floor0_inverse2           100361f0 f   vorbisfile_static:floor0.obj
 0001:00035270       _floor0_map_lazy_init      10036270 f   vorbisfile_static:floor0.obj
 0001:00035860       _cheby                     10036860 f   vorbisfile_static:lsp.obj
 0001:000358b0       _comp                      100368b0 f   vorbisfile_static:lsp.obj
 0001:000358f0       _Laguerre_With_Deflation   100368f0 f   vorbisfile_static:lsp.obj
 0001:00035a80       _Newton_Raphson            10036a80 f   vorbisfile_static:lsp.obj
 0001:00036434       __onexit_nolock            10037434 f   LIBCMT:onexit.obj
 0001:000365d7       ?ArrayUnwindFilter@@YAHPAU_EXCEPTION_POINTERS@@@Z 100375d7 f   LIBCMT:ehvecdtr.obj
 0001:0003739d       ?CatchGuardHandler@@YA?AW4_EXCEPTION_DISPOSITION@@PAUEHExceptionRecord@@PAUCatchGuardRN@@PAX2@Z 1003839d f   LIBCMT:_trnsctrl_.obj
 0001:000374a7       ?TranslatorGuardHandler@@YA?AW4_EXCEPTION_DISPOSITION@@PAUEHExceptionRecord@@PAUTranslatorGuardRN@@PAX2@Z 100384a7 f   LIBCMT:_trnsctrl_.obj
 0001:00037e5e       __splitpath_helper         10038e5e f   LIBCMT:splitpat.obj
 0001:00039f71       ___DllMainCRTStartup       1003af71 f   LIBCMT:dllcrt0.obj
 0001:0003aad0       _swap                      1003bad0 f   LIBCMT:qsort.obj
 0001:0003ab00       _shortsort                 1003bb00 f   LIBCMT:qsort.obj
 0001:0003b03d       __initterm                 1003c03d f   LIBCMT:crt0dat.obj
 0001:0003b17b       _doexit                    1003c17b f   LIBCMT:crt0dat.obj
 0001:0003b5b9       __shift                    1003c5b9 f   LIBCMT:cvt.obj
 0001:0003b5fe       __cftoe2_l                 1003c5fe f   LIBCMT:cvt.obj
 0001:0003bbf0       __cftof2_l                 1003cbf0 f   LIBCMT:cvt.obj
 0001:0003d330       _ValidateLocalCookies      1003e330 f   LIBCMT:chandler4.obj
 0001:0003d4ec       _fastcopy_I                1003e4ec f   LIBCMT:p4_memcpy.obj
 0001:0003d656       _has_osfxsr_set            1003e656 f   LIBCMT:cpu_disp.obj
 0001:0003d715       _fastzero_I                1003e715 f   LIBCMT:p4_memset.obj
 0001:0003d7fb       ?CPtoLCID@@YAHH@Z          1003e7fb f   LIBCMT:mbctype.obj
 0001:0003d82a       ?setSBCS@@YAXPAUthreadmbcinfostruct@@@Z 1003e82a f   LIBCMT:mbctype.obj
 0001:0003d88e       ?setSBUpLow@@YAXPAUthreadmbcinfostruct@@@Z 1003e88e f   LIBCMT:mbctype.obj
 0001:0003dac5       ?getSystemCP@@YAHH@Z       1003eac5 f   LIBCMT:mbctype.obj
 0001:0003e199       __copytlocinfo_nolock      1003f199 f   LIBCMT:setlocal.obj
 0001:0003e1bf       __updatetlocinfoEx_nolock  1003f1bf f   LIBCMT:setlocal.obj
 0001:0003e2dd       _sync_legacy_variables_lk  1003f2dd f   LIBCMT:setlocal.obj
 0001:0003e68a       __setlocale_get_all        1003f68a f   LIBCMT:setlocal.obj
 0001:0003ea38       __setlocale_set_cat        1003fa38 f   LIBCMT:setlocal.obj
 0001:0003ed3a       __setlocale_nolock         1003fd3a f   LIBCMT:setlocal.obj
 0001:00041b71       ?ExFilterRethrow@@YAHPAU_EXCEPTION_POINTERS@@@Z 10042b71 f   LIBCMT:frame.obj
 0001:00041f65       ?IsInExceptionSpec@@YAEPAUEHExceptionRecord@@PBU_s_ESTypeList@@@Z 10042f65 f   LIBCMT:frame.obj
 0001:00041fe0       ?CallUnexpected@@YAXPBU_s_ESTypeList@@@Z 10042fe0 f   LIBCMT:frame.obj
 0001:00042011       __catch$?CallUnexpected@@YAXPBU_s_ESTypeList@@@Z$0 10043011 f   LIBCMT:frame.obj
 0001:00042029       ?Is_bad_exception_allowed@@YAEPBU_s_ESTypeList@@@Z 10043029 f   LIBCMT:frame.obj
 0001:000420e1       ?CallCatchBlock@@YAPAXPAUEHExceptionRecord@@PAUEHRegistrationNode@@PAU_CONTEXT@@PBU_s_FuncInfo@@PAXHK@Z 100430e1 f   LIBCMT:frame.obj
 0001:000425d3       ?CatchIt@@YAXPAUEHExceptionRecord@@PAUEHRegistrationNode@@PAU_CONTEXT@@PAXPBU_s_FuncInfo@@PBU_s_HandlerType@@PBU_s_CatchableType@@PBU_s_TryBlockMapEntry@@H1E@Z 100435d3 f   LIBCMT:frame.obj
 0001:00042641       ?FindHandlerForForeignException@@YAXPAUEHExceptionRecord@@PAUEHRegistrationNode@@PAU_CONTEXT@@PAXPBU_s_FuncInfo@@HH1@Z 10043641 f   LIBCMT:frame.obj
 0001:00042735       ?FindHandler@@YAXPAUEHExceptionRecord@@PAUEHRegistrationNode@@PAU_CONTEXT@@PAXPBU_s_FuncInfo@@EH1@Z 10043735 f   LIBCMT:frame.obj
 0001:00042d30       _write_char                10043d30 f   LIBCMT:output.obj
 0001:00042d63       _write_multi_char          10043d63 f   LIBCMT:output.obj
 0001:00042d89       _write_string              10043d89 f   LIBCMT:output.obj
 0001:00043ce6       ?strtoxl@@YAKPAUlocaleinfo_struct@@PBDPAPBDHH@Z 10044ce6 f   LIBCMT:strtol.obj
 0001:00043fa6       ?strtoxq@@YA_KPAUlocaleinfo_struct@@PBDPAPBDHH@Z 10044fa6 f   LIBCMT:strtoq.obj
 0001:000452e6       _write_char                100462e6 f   LIBCMT:outputp.obj
 0001:00045319       _write_multi_char          10046319 f   LIBCMT:outputp.obj
 0001:0004533f       _write_string              1004633f f   LIBCMT:outputp.obj
 0001:00046661       ?x_ismbbtype_l@@YAHPAUlocaleinfo_struct@@IHH@Z 10047661 f   LIBCMT:ismbbyte.obj
 0001:00046c77       _flsall                    10047c77 f   LIBCMT:fflush.obj
 0001:00047d78       __unwind_handler4          10048d78 f   LIBCMT:exsup4.obj
 0001:0004966a       __get_fname                1004a66a f   LIBCMT:_fpexcept_.obj
 0001:0004a930       _parse_cmdline             1004b930 f   LIBCMT:stdargv.obj
 0001:0004ad09       _xcptlookup                1004bd09 f   LIBCMT:winxfltr.obj
 0001:0004b45b       ?strncnt@@YAHPBDH@Z        1004c45b f   LIBCMT:a_map.obj
 0001:0004b479       ?__crtLCMapStringA_stat@@YAHPAUlocaleinfo_struct@@KKPBDHPADHHH@Z 1004c479 f   LIBCMT:a_map.obj
 0001:0004c46b       _ctrlevent_capture@4       1004d46b f   LIBCMT:winsig.obj
 0001:0004c506       _siglookup                 1004d506 f   LIBCMT:winsig.obj
 0001:0004d8d4       ?__crtGetStringTypeA_stat@@YAHPAUlocaleinfo_struct@@KPBDHPAGHHH@Z 1004e8d4 f   LIBCMT:a_str.obj
 0001:0004daff       __get_lc_time              1004eaff f   LIBCMT:inittime.obj
 0001:0004e128       _fix_grouping              1004f128 f   LIBCMT:initnum.obj
 0001:0004e36a       _fix_grouping              1004f36a f   LIBCMT:initmon.obj
 0001:0004f0bf       ?_store_str@@YAXPADPAPADPAI@Z 100500bf f   LIBCMT:strftime.obj
 0001:0004f0df       ?_store_number@@YAXHPAPADPAI@Z 100500df f   LIBCMT:strftime.obj
 0001:0004f115       ?_store_num@@YAXHHPAPADPAII@Z 10050115 f   LIBCMT:strftime.obj
 0001:0004f190       ?_expandtime@@YAHPAUlocaleinfo_struct@@DPBUtm@@PAPADPAIPAU__lc_time_data@@I@Z 10050190 f   LIBCMT:strftime.obj
 0001:0004f578       ?_store_winword@@YAHPAUlocaleinfo_struct@@HPBUtm@@PAPADPAIPAU__lc_time_data@@@Z 10050578 f   LIBCMT:strftime.obj
 0001:0004fd7b       _TranslateName             10050d7b f   LIBCMT:getqloc.obj
 0001:0004fddd       _GetLcidFromDefault        10050ddd f   LIBCMT:getqloc.obj
 0001:0004fdf1       _ProcessCodePage           10050df1 f   LIBCMT:getqloc.obj
 0001:0004fe95       _TestDefaultCountry        10050e95 f   LIBCMT:getqloc.obj
 0001:0004feb9       _LcidFromHexString         10050eb9 f   LIBCMT:getqloc.obj
 0001:0004feed       _GetPrimaryLen             10050eed f   LIBCMT:getqloc.obj
 0001:0004ff08       _CountryEnumProc@4         10050f08 f   LIBCMT:getqloc.obj
 0001:0004ffa0       _TestDefaultLanguage       10050fa0 f   LIBCMT:getqloc.obj
 0001:00050014       _LangCountryEnumProc@4     10051014 f   LIBCMT:getqloc.obj
 0001:000501e6       _LanguageEnumProc@4        100511e6 f   LIBCMT:getqloc.obj
 0001:000502a7       _GetLcidFromCountry        100512a7 f   LIBCMT:getqloc.obj
 0001:000502d3       _GetLcidFromLangCountry    100512d3 f   LIBCMT:getqloc.obj
 0001:0005033a       _GetLcidFromLanguage       1005133a f   LIBCMT:getqloc.obj
 0001:00050567       _cmpResult                 10051567 f   LIBCMT:memcmp.obj
 0001:00050579       _cmpBYTE                   10051579 f   LIBCMT:memcmp.obj
 0001:00050591       _cmpWORD                   10051591 f   LIBCMT:memcmp.obj
 0001:000505d1       _cmpDWORD                  100515d1 f   LIBCMT:memcmp.obj
 0001:00050649       _unaligned_memcmp          10051649 f   LIBCMT:memcmp.obj
 0001:00054f28       ?und_strlen@@YAIPBD@Z      10055f28 f   LIBCMT:undname.obj
 0001:00054f36       ?und_memcpy@@YAXPADPBDI@Z  10055f36 f   LIBCMT:undname.obj
 0001:00054f4c       ?und_strncmp@@YAIPBD0I@Z   10055f4c f   LIBCMT:undname.obj
 0001:00059888       __unwind_handler           1005a888 f   LIBCMT:exsup.obj
 0001:00059e95       _write_char                1005ae95 f   LIBCMT:outputs.obj
 0001:00059ec8       _write_multi_char          1005aec8 f   LIBCMT:outputs.obj
 0001:00059eee       _write_string              1005aeee f   LIBCMT:outputs.obj
 0001:0005c492       __tsopen_nolock            1005d492 f   LIBCMT:open.obj
 0001:0005d767       ?__crtGetLocaleInfoW_stat@@YAHPAUlocaleinfo_struct@@KKPA_WHH@Z 1005e767 f   LIBCMT:w_loc.obj
 0001:0005d7b4       ?__crtGetLocaleInfoA_stat@@YAHPAUlocaleinfo_struct@@KKPADHH@Z 1005e7b4 f   LIBCMT:a_loc.obj
 0001:0005e2c9       __abstract_cw              1005f2c9 f   LIBCMT:_ieee87_.obj
 0001:0005e368       __hw_cw                    1005f368 f   LIBCMT:_ieee87_.obj
 0001:0005e3f6       __abstract_sw              1005f3f6 f   LIBCMT:_ieee87_.obj
 0001:0005e439       ___abstract_cw_sse2        1005f439 f   LIBCMT:_ieee87_.obj
 0001:0005e4d9       ___hw_cw_sse2              1005f4d9 f   LIBCMT:_ieee87_.obj
 0001:0005e579       ___abstract_sw_sse2        1005f579 f   LIBCMT:_ieee87_.obj
 0001:0005e5bc       ___fpreset_sse2            1005f5bc f   LIBCMT:_ieee87_.obj
 0001:0005e692       ___statusfp_sse2           1005f692 f   LIBCMT:_ieee87_.obj
 0001:0005e6cd       ___clearfp_sse2            1005f6cd f   LIBCMT:_ieee87_.obj
 0001:0005e71d       ___control87_sse2          1005f71d f   LIBCMT:_ieee87_.obj
 0001:0005f495       __tzset_nolock             10060495 f   LIBCMT:tzset.obj
 0001:0005f7db       _cvtdate                   100607db f   LIBCMT:tzset.obj
 0001:0005f9d2       __isindst_nolock           100609d2 f   LIBCMT:tzset.obj
 0001:0005fdc2       _xtoa_s@20                 10060dc2 f   LIBCMT:xtoas.obj
 0001:0005ff0a       @x64toa_s@24               10060f0a f   LIBCMT:xtoas.obj
 0001:00060630       ?__crtGetStringTypeW_stat@@YAHPAUlocaleinfo_struct@@KPB_WHPAGHH@Z 10061630 f   LIBCMT:w_str.obj
 0001:00060718       __getenv_s_helper          10061718 f   LIBCMT:getenv.obj
 0001:000607ad       __dupenv_s_helper          100617ad f   LIBCMT:getenv.obj
 0001:00060cbd       ?strncnt@@YAHPBDH@Z        10061cbd f   LIBCMT:a_cmp.obj
 0001:00060cdb       ?__crtCompareStringA_stat@@YAHPAUlocaleinfo_struct@@KKPBDH1HH@Z 10061cdb f   LIBCMT:a_cmp.obj
 0001:000611b0       _findenv                   100621b0 f   LIBCMT:setenv.obj
 0001:00061202       _copy_environ              10062202 f   LIBCMT:setenv.obj
 0001:000615cf       _ascii_mbtowc              100625cf f   iconv:iconv.obj
 0001:000615ea       _ascii_wctomb              100625ea f   iconv:iconv.obj
 0001:00061603       _utf8_mbtowc               10062603 f   iconv:iconv.obj
 0001:00061898       _utf8_wctomb               10062898 f   iconv:iconv.obj
 0001:00061995       _ucs2_mbtowc               10062995 f   iconv:iconv.obj
 0001:00061a17       _ucs2_wctomb               10062a17 f   iconv:iconv.obj
 0001:00061a5c       _ucs2be_mbtowc             10062a5c f   iconv:iconv.obj
 0001:00061a91       _ucs2be_wctomb             10062a91 f   iconv:iconv.obj
 0001:00061ace       _ucs2le_mbtowc             10062ace f   iconv:iconv.obj
 0001:00061b03       _ucs2le_wctomb             10062b03 f   iconv:iconv.obj
 0001:00061b3b       _ucs4_mbtowc               10062b3b f   iconv:iconv.obj
 0001:00061bdb       _ucs4_wctomb               10062bdb f   iconv:iconv.obj
 0001:00061c18       _ucs4be_mbtowc             10062c18 f   iconv:iconv.obj
 0001:00061c4f       _ucs4be_wctomb             10062c4f f   iconv:iconv.obj
 0001:00061c80       _ucs4le_mbtowc             10062c80 f   iconv:iconv.obj
 0001:00061cb7       _ucs4le_wctomb             10062cb7 f   iconv:iconv.obj
 0001:00061ce6       _utf16_mbtowc              10062ce6 f   iconv:iconv.obj
 0001:00061dbf       _utf16_wctomb              10062dbf f   iconv:iconv.obj
 0001:00061e87       _utf16be_mbtowc            10062e87 f   iconv:iconv.obj
 0001:00061f07       _utf16be_wctomb            10062f07 f   iconv:iconv.obj
 0001:00061f8b       _utf16le_mbtowc            10062f8b f   iconv:iconv.obj
 0001:0006200b       _utf16le_wctomb            1006300b f   iconv:iconv.obj
 0001:00062086       _utf32_mbtowc              10063086 f   iconv:iconv.obj
 0001:00062134       _utf32_wctomb              10063134 f   iconv:iconv.obj
 0001:000621b5       _utf32be_mbtowc            100631b5 f   iconv:iconv.obj
 0001:00062205       _utf32be_wctomb            10063205 f   iconv:iconv.obj
 0001:0006224e       _utf32le_mbtowc            1006324e f   iconv:iconv.obj
 0001:0006229e       _utf32le_wctomb            1006329e f   iconv:iconv.obj
 0001:000622e2       _utf7_mbtowc               100632e2 f   iconv:iconv.obj
 0001:00062509       _utf7_wctomb               10063509 f   iconv:iconv.obj
 0001:00062781       _utf7_reset                10063781 f   iconv:iconv.obj
 0001:000627ec       _ucs2internal_mbtowc       100637ec f   iconv:iconv.obj
 0001:0006281b       _ucs2internal_wctomb       1006381b f   iconv:iconv.obj
 0001:0006284e       _ucs2swapped_mbtowc        1006384e f   iconv:iconv.obj
 0001:00062885       _ucs2swapped_wctomb        10063885 f   iconv:iconv.obj
 0001:000628be       _ucs4internal_mbtowc       100638be f   iconv:iconv.obj
 0001:000628d8       _ucs4internal_wctomb       100638d8 f   iconv:iconv.obj
 0001:000628f0       _ucs4swapped_mbtowc        100638f0 f   iconv:iconv.obj
 0001:0006292f       _ucs4swapped_wctomb        1006392f f   iconv:iconv.obj
 0001:0006296c       _c99_mbtowc                1006396c f   iconv:iconv.obj
 0001:00062ab4       _c99_wctomb                10063ab4 f   iconv:iconv.obj
 0001:00062b28       _java_mbtowc               10063b28 f   iconv:iconv.obj
 0001:00062c7c       _java_wctomb               10063c7c f   iconv:iconv.obj
 0001:00062e08       _iso8859_1_mbtowc          10063e08 f   iconv:iconv.obj
 0001:00062e19       _iso8859_1_wctomb          10063e19 f   iconv:iconv.obj
 0001:00062e32       _iso8859_2_mbtowc          10063e32 f   iconv:iconv.obj
 0001:00062e51       _iso8859_2_wctomb          10063e51 f   iconv:iconv.obj
 0001:00062e91       _iso8859_3_mbtowc          10063e91 f   iconv:iconv.obj
 0001:00062ebd       _iso8859_3_wctomb          10063ebd f   iconv:iconv.obj
 0001:00062f13       _iso8859_4_mbtowc          10063f13 f   iconv:iconv.obj
 0001:00062f32       _iso8859_4_wctomb          10063f32 f   iconv:iconv.obj
 0001:00062f72       _iso8859_5_mbtowc          10063f72 f   iconv:iconv.obj
 0001:00062f91       _iso8859_5_wctomb          10063f91 f   iconv:iconv.obj
 0001:00062fdc       _iso8859_6_mbtowc          10063fdc f   iconv:iconv.obj
 0001:00063008       _iso8859_6_wctomb          10064008 f   iconv:iconv.obj
 0001:00063048       _iso8859_7_mbtowc          10064048 f   iconv:iconv.obj
 0001:00063074       _iso8859_7_wctomb          10064074 f   iconv:iconv.obj
 0001:000630ca       _iso8859_8_mbtowc          100640ca f   iconv:iconv.obj
 0001:000630f6       _iso8859_8_wctomb          100640f6 f   iconv:iconv.obj
 0001:0006314c       _iso8859_9_mbtowc          1006414c f   iconv:iconv.obj
 0001:0006316b       _iso8859_9_wctomb          1006416b f   iconv:iconv.obj
 0001:000631ab       _iso8859_10_mbtowc         100641ab f   iconv:iconv.obj
 0001:000631ca       _iso8859_10_wctomb         100641ca f   iconv:iconv.obj
 0001:000631ff       _iso8859_13_mbtowc         100641ff f   iconv:iconv.obj
 0001:0006321e       _iso8859_13_wctomb         1006421e f   iconv:iconv.obj
 0001:0006325e       _iso8859_14_mbtowc         1006425e f   iconv:iconv.obj
 0001:0006327d       _iso8859_14_wctomb         1006427d f   iconv:iconv.obj
 0001:000632ff       _iso8859_15_mbtowc         100642ff f   iconv:iconv.obj
 0001:00063327       _iso8859_15_wctomb         10064327 f   iconv:iconv.obj
 0001:00063379       _iso8859_16_mbtowc         10064379 f   iconv:iconv.obj
 0001:00063398       _iso8859_16_wctomb         10064398 f   iconv:iconv.obj
 0001:000633f9       _koi8_r_mbtowc             100643f9 f   iconv:iconv.obj
 0001:00063418       _koi8_r_wctomb             10064418 f   iconv:iconv.obj
 0001:000634a1       _koi8_u_mbtowc             100644a1 f   iconv:iconv.obj
 0001:000634c0       _koi8_u_wctomb             100644c0 f   iconv:iconv.obj
 0001:00063549       _koi8_ru_mbtowc            10064549 f   iconv:iconv.obj
 0001:00063568       _koi8_ru_wctomb            10064568 f   iconv:iconv.obj
 0001:000635f1       _cp1250_mbtowc             100645f1 f   iconv:iconv.obj
 0001:0006361d       _cp1250_wctomb             1006461d f   iconv:iconv.obj
 0001:00063690       _cp1251_mbtowc             10064690 f   iconv:iconv.obj
 0001:000636bc       _cp1251_wctomb             100646bc f   iconv:iconv.obj
 0001:0006373a       _cp1252_mbtowc             1006473a f   iconv:iconv.obj
 0001:0006376f       _cp1252_wctomb             1006476f f   iconv:iconv.obj
 0001:000637f0       _cp1253_mbtowc             100647f0 f   iconv:iconv.obj
 0001:0006381c       _cp1253_wctomb             1006481c f   iconv:iconv.obj
 0001:0006389a       _cp1254_mbtowc             1006489a f   iconv:iconv.obj
 0001:000638f8       _cp1254_wctomb             100648f8 f   iconv:iconv.obj
 0001:00063995       _normal_flushwc            10064995 f   iconv:iconv.obj
 0001:000639b1       _cp1255_mbtowc             100649b1 f   iconv:iconv.obj
 0001:00063b26       _cp1255_wctomb             10064b26 f   iconv:iconv.obj
 0001:00063cc8       _cp1256_mbtowc             10064cc8 f   iconv:iconv.obj
 0001:00063ce7       _cp1256_wctomb             10064ce7 f   iconv:iconv.obj
 0001:00063d7b       _cp1257_mbtowc             10064d7b f   iconv:iconv.obj
 0001:00063da7       _cp1257_wctomb             10064da7 f   iconv:iconv.obj
 0001:00063e1a       _cp1258_mbtowc             10064e1a f   iconv:iconv.obj
 0001:00063f38       _cp1258_wctomb             10064f38 f   iconv:iconv.obj
 0001:000640e6       _cp850_mbtowc              100650e6 f   iconv:iconv.obj
 0001:00064105       _cp850_wctomb              10065105 f   iconv:iconv.obj
 0001:0006416d       _cp862_mbtowc              1006516d f   iconv:iconv.obj
 0001:0006418c       _cp862_wctomb              1006518c f   iconv:iconv.obj
 0001:00064259       _cp866_mbtowc              10065259 f   iconv:iconv.obj
 0001:00064288       _cp866_wctomb              10065288 f   iconv:iconv.obj
 0001:00064306       _mac_roman_mbtowc          10065306 f   iconv:iconv.obj
 0001:00064332       _mac_roman_wctomb          10065332 f   iconv:iconv.obj
 0001:00064407       _mac_centraleurope_mbtowc  10065407 f   iconv:iconv.obj
 0001:00064426       _mac_centraleurope_wctomb  10065426 f   iconv:iconv.obj
 0001:000644ba       _mac_iceland_mbtowc        100654ba f   iconv:iconv.obj
 0001:000644e6       _mac_iceland_wctomb        100654e6 f   iconv:iconv.obj
 0001:000645a2       _mac_croatian_mbtowc       100655a2 f   iconv:iconv.obj
 0001:000645ce       _mac_croatian_wctomb       100655ce f   iconv:iconv.obj
 0001:00064671       _mac_romania_mbtowc        10065671 f   iconv:iconv.obj
 0001:0006469d       _mac_romania_wctomb        1006569d f   iconv:iconv.obj
 0001:00064740       _mac_cyrillic_mbtowc       10065740 f   iconv:iconv.obj
 0001:0006475f       _mac_cyrillic_wctomb       1006575f f   iconv:iconv.obj
 0001:00064802       _mac_ukraine_mbtowc        10065802 f   iconv:iconv.obj
 0001:00064821       _mac_ukraine_wctomb        10065821 f   iconv:iconv.obj
 0001:000648c4       _mac_greek_mbtowc          100658c4 f   iconv:iconv.obj
 0001:000648f0       _mac_greek_wctomb          100658f0 f   iconv:iconv.obj
 0001:00064979       _mac_turkish_mbtowc        10065979 f   iconv:iconv.obj
 0001:000649a5       _mac_turkish_wctomb        100659a5 f   iconv:iconv.obj
 0001:00064a61       _mac_hebrew_mbtowc         10065a61 f   iconv:iconv.obj
 0001:00064a8d       _mac_hebrew_wctomb         10065a8d f   iconv:iconv.obj
 0001:00064b0b       _mac_arabic_mbtowc         10065b0b f   iconv:iconv.obj
 0001:00064b37       _mac_arabic_wctomb         10065b37 f   iconv:iconv.obj
 0001:00064b89       _mac_thai_mbtowc           10065b89 f   iconv:iconv.obj
 0001:00064bb5       _mac_thai_wctomb           10065bb5 f   iconv:iconv.obj
 0001:00064c3e       _hp_roman8_mbtowc          10065c3e f   iconv:iconv.obj
 0001:00064c6a       _hp_roman8_wctomb          10065c6a f   iconv:iconv.obj
 0001:00064ce1       _nextstep_mbtowc           10065ce1 f   iconv:iconv.obj
 0001:00064d0d       _nextstep_wctomb           10065d0d f   iconv:iconv.obj
 0001:00064d96       _armscii_8_mbtowc          10065d96 f   iconv:iconv.obj
 0001:00064dc2       _armscii_8_wctomb          10065dc2 f   iconv:iconv.obj
 0001:00064e2a       _georgian_academy_mbtowc   10065e2a f   iconv:iconv.obj
 0001:00064e64       _georgian_academy_wctomb   10065e64 f   iconv:iconv.obj
 0001:00064f06       _georgian_ps_mbtowc        10065f06 f   iconv:iconv.obj
 0001:00064f43       _georgian_ps_wctomb        10065f43 f   iconv:iconv.obj
 0001:00064fe9       _koi8_t_mbtowc             10065fe9 f   iconv:iconv.obj
 0001:00065015       _koi8_t_wctomb             10066015 f   iconv:iconv.obj
 0001:00065088       _mulelao_mbtowc            10066088 f   iconv:iconv.obj
 0001:000650b4       _mulelao_wctomb            100660b4 f   iconv:iconv.obj
 0001:000650f3       _cp1133_mbtowc             100660f3 f   iconv:iconv.obj
 0001:00065139       _cp1133_wctomb             10066139 f   iconv:iconv.obj
 0001:00065184       _tis620_mbtowc             10066184 f   iconv:iconv.obj
 0001:000651b9       _tis620_wctomb             100661b9 f   iconv:iconv.obj
 0001:000651f0       _cp874_mbtowc              100661f0 f   iconv:iconv.obj
 0001:0006521c       _cp874_wctomb              1006621c f   iconv:iconv.obj
 0001:00065279       _viscii_mbtowc             10066279 f   iconv:iconv.obj
 0001:000652a9       _viscii_wctomb             100662a9 f   iconv:iconv.obj
 0001:00065306       _tcvn_mbtowc               10066306 f   iconv:iconv.obj
 0001:00065429       _tcvn_wctomb               10066429 f   iconv:iconv.obj
 0001:0006556f       _iso646_jp_mbtowc          1006656f f   iconv:iconv.obj
 0001:000655aa       _iso646_jp_wctomb          100665aa f   iconv:iconv.obj
 0001:000655ed       _jisx0201_mbtowc           100665ed f   iconv:iconv.obj
 0001:0006563b       _jisx0201_wctomb           1006663b f   iconv:iconv.obj
 0001:0006568f       _jisx0208_mbtowc           1006668f f   iconv:iconv.obj
 0001:0006570d       _jisx0208_wctomb           1006670d f   iconv:iconv.obj
 0001:00065870       _jisx0212_mbtowc           10066870 f   iconv:iconv.obj
 0001:00065930       _jisx0212_wctomb           10066930 f   iconv:iconv.obj
 0001:00065a39       _iso646_cn_mbtowc          10066a39 f   iconv:iconv.obj
 0001:00065a74       _iso646_cn_wctomb          10066a74 f   iconv:iconv.obj
 0001:00065ab7       _gb2312_mbtowc             10066ab7 f   iconv:iconv.obj
 0001:00065b35       _gb2312_wctomb             10066b35 f   iconv:iconv.obj
 0001:00065c79       _isoir165_mbtowc           10066c79 f   iconv:iconv.obj
 0001:00065d20       _isoir165ext_mbtowc        10066d20 f   iconv:iconv.obj
 0001:00065d9e       _isoir165_wctomb           10066d9e f   iconv:iconv.obj
 0001:00065e30       _isoir165ext_wctomb        10066e30 f   iconv:iconv.obj
 0001:00065ff0       _ksc5601_mbtowc            10066ff0 f   iconv:iconv.obj
 0001:00066090       _ksc5601_wctomb            10067090 f   iconv:iconv.obj
 0001:000661f3       _euc_jp_mbtowc             100671f3 f   iconv:iconv.obj
 0001:00066360       _euc_jp_wctomb             10067360 f   iconv:iconv.obj
 0001:000664e6       _sjis_mbtowc               100674e6 f   iconv:iconv.obj
 0001:000665ef       _sjis_wctomb               100675ef f   iconv:iconv.obj
 0001:00066714       _cp932_mbtowc              10067714 f   iconv:iconv.obj
 0001:00066866       _cp932ext_mbtowc           10067866 f   iconv:iconv.obj
 0001:00066931       _cp932_wctomb              10067931 f   iconv:iconv.obj
 0001:00066ab7       _cp932ext_wctomb           10067ab7 f   iconv:iconv.obj
 0001:00066cfa       _iso2022_jp_mbtowc         10067cfa f   iconv:iconv.obj
 0001:00066e3f       _iso2022_jp_wctomb         10067e3f f   iconv:iconv.obj
 0001:00066f73       _iso2022_jp_reset          10067f73 f   iconv:iconv.obj
 0001:00066f9e       _iso2022_jp1_mbtowc        10067f9e f   iconv:iconv.obj
 0001:00067186       _iso2022_jp1_wctomb        10068186 f   iconv:iconv.obj
 0001:0006731b       _iso2022_jp1_reset         1006831b f   iconv:iconv.obj
 0001:00067346       _iso2022_jp2_mbtowc        10068346 f   iconv:iconv.obj
 0001:00067768       _iso2022_jp2_wctomb        10068768 f   iconv:iconv.obj
 0001:00067cd7       _iso2022_jp2_reset         10068cd7 f   iconv:iconv.obj
 0001:00067d02       _euc_cn_mbtowc             10068d02 f   iconv:iconv.obj
 0001:00067d66       _euc_cn_wctomb             10068d66 f   iconv:iconv.obj
 0001:00067dcb       _ces_gbk_mbtowc            10068dcb f   iconv:iconv.obj
 0001:00067e13       _gbk_mbtowc                10068e13 f   iconv:iconv.obj
 0001:00067f1d       _gbkext1_mbtowc            10068f1d f   iconv:iconv.obj
 0001:00067f8d       _gbkext2_mbtowc            10068f8d f   iconv:iconv.obj
 0001:00068004       _cp936ext_mbtowc           10069004 f   iconv:iconv.obj
 0001:0006809a       _ces_gbk_wctomb            1006909a f   iconv:iconv.obj
 0001:000680f9       _gbk_wctomb                100690f9 f   iconv:iconv.obj
 0001:000681fb       _gbkext_inv_wctomb         100691fb f   iconv:iconv.obj
 0001:00068384       _cp936ext_wctomb           10069384 f   iconv:iconv.obj
 0001:000683f3       _gb18030_mbtowc            100693f3 f   iconv:iconv.obj
 0001:000684ed       _gb18030ext_mbtowc         100694ed f   iconv:iconv.obj
 0001:000685b5       _gb18030uni_mbtowc         100695b5 f   iconv:iconv.obj
 0001:0006869f       _gb18030_wctomb            1006969f f   iconv:iconv.obj
 0001:0006877a       _gb18030ext_wctomb         1006977a f   iconv:iconv.obj
 0001:000689d6       _gb18030uni_wctomb         100699d6 f   iconv:iconv.obj
 0001:00068a94       _iso2022_cn_mbtowc         10069a94 f   iconv:iconv.obj
 0001:00068ccb       _cns11643_1_mbtowc         10069ccb f   iconv:iconv.obj
 0001:00068d9c       _cns11643_2_mbtowc         10069d9c f   iconv:iconv.obj
 0001:00068df8       _iso2022_cn_wctomb         10069df8 f   iconv:iconv.obj
 0001:0006900e       _cns11643_inv_wctomb       1006a00e f   iconv:iconv.obj
 0001:000691bf       _iso2022_cn_reset          1006a1bf f   iconv:iconv.obj
 0001:000691e1       _iso2022_cn_ext_mbtowc     1006a1e1 f   iconv:iconv.obj
 0001:0006963d       _cns11643_3_mbtowc         1006a63d f   iconv:iconv.obj
 0001:000696cd       _cns11643_4_mbtowc         1006a6cd f   iconv:iconv.obj
 0001:00069762       _cns11643_5_mbtowc         1006a762 f   iconv:iconv.obj
 0001:000697d0       _cns11643_6_mbtowc         1006a7d0 f   iconv:iconv.obj
 0001:0006983e       _cns11643_7_mbtowc         1006a83e f   iconv:iconv.obj
 0001:000698ac       _iso2022_cn_ext_wctomb     1006a8ac f   iconv:iconv.obj
 0001:00069d2d       _iso2022_cn_ext_reset      1006ad2d f   iconv:iconv.obj
 0001:00069d4f       _hz_mbtowc                 1006ad4f f   iconv:iconv.obj
 0001:00069e40       _hz_wctomb                 1006ae40 f   iconv:iconv.obj
 0001:00069f06       _hz_reset                  1006af06 f   iconv:iconv.obj
 0001:00069f2d       _euc_tw_mbtowc             1006af2d f   iconv:iconv.obj
 0001:0006a0d3       _cns11643_15_mbtowc        1006b0d3 f   iconv:iconv.obj
 0001:0006a141       _euc_tw_wctomb             1006b141 f   iconv:iconv.obj
 0001:0006a1d1       _ces_big5_mbtowc           1006b1d1 f   iconv:iconv.obj
 0001:0006a22c       _big5_mbtowc               1006b22c f   iconv:iconv.obj
 0001:0006a2c1       _ces_big5_wctomb           1006b2c1 f   iconv:iconv.obj
 0001:0006a320       _big5_wctomb               1006b320 f   iconv:iconv.obj
 0001:0006a4a2       _cp950_mbtowc              1006b4a2 f   iconv:iconv.obj
 0001:0006a580       _cp950ext_mbtowc           1006b580 f   iconv:iconv.obj
 0001:0006a5e8       _cp950_wctomb              1006b5e8 f   iconv:iconv.obj
 0001:0006a844       _cp950ext_wctomb           1006b844 f   iconv:iconv.obj
 0001:0006a9cd       _big5hkscs_mbtowc          1006b9cd f   iconv:iconv.obj
 0001:0006aa4d       _hkscs_mbtowc              1006ba4d f   iconv:iconv.obj
 0001:0006ab49       _big5hkscs_wctomb          1006bb49 f   iconv:iconv.obj
 0001:0006abc4       _hkscs_wctomb              1006bbc4 f   iconv:iconv.obj
 0001:0006aef8       _euc_kr_mbtowc             1006bef8 f   iconv:iconv.obj
 0001:0006af5c       _euc_kr_wctomb             1006bf5c f   iconv:iconv.obj
 0001:0006afc1       _cp949_mbtowc              1006bfc1 f   iconv:iconv.obj
 0001:0006b051       _uhc_1_mbtowc              1006c051 f   iconv:iconv.obj
 0001:0006b0f0       _uhc_2_mbtowc              1006c0f0 f   iconv:iconv.obj
 0001:0006b18c       _cp949_wctomb              1006c18c f   iconv:iconv.obj
 0001:0006b222       _uhc_1_wctomb              1006c222 f   iconv:iconv.obj
 0001:0006b2ee       _uhc_2_wctomb              1006c2ee f   iconv:iconv.obj
 0001:0006b3ba       _johab_mbtowc              1006c3ba f   iconv:iconv.obj
 0001:0006b48e       _johab_hangul_mbtowc       1006c48e f   iconv:iconv.obj
 0001:0006b581       _johab_wctomb              1006c581 f   iconv:iconv.obj
 0001:0006b67d       _johab_hangul_wctomb       1006c67d f   iconv:iconv.obj
 0001:0006b730       _iso2022_kr_mbtowc         1006c730 f   iconv:iconv.obj
 0001:0006b866       _iso2022_kr_wctomb         1006c866 f   iconv:iconv.obj
 0001:0006b967       _iso2022_kr_reset          1006c967 f   iconv:iconv.obj
 0001:0006b989       _cp437_mbtowc              1006c989 f   iconv:iconv.obj
 0001:0006b9a8       _cp437_wctomb              1006c9a8 f   iconv:iconv.obj
 0001:0006ba56       _cp737_mbtowc              1006ca56 f   iconv:iconv.obj
 0001:0006ba75       _cp737_wctomb              1006ca75 f   iconv:iconv.obj
 0001:0006bafe       _cp775_mbtowc              1006cafe f   iconv:iconv.obj
 0001:0006bb1d       _cp775_wctomb              1006cb1d f   iconv:iconv.obj
 0001:0006bb85       _cp852_mbtowc              1006cb85 f   iconv:iconv.obj
 0001:0006bba4       _cp852_wctomb              1006cba4 f   iconv:iconv.obj
 0001:0006bc01       _cp853_mbtowc              1006cc01 f   iconv:iconv.obj
 0001:0006bc2d       _cp853_wctomb              1006cc2d f   iconv:iconv.obj
 0001:0006bcab       _cp855_mbtowc              1006ccab f   iconv:iconv.obj
 0001:0006bcca       _cp855_wctomb              1006ccca f   iconv:iconv.obj
 0001:0006bd32       _cp857_mbtowc              1006cd32 f   iconv:iconv.obj
 0001:0006bd5e       _cp857_wctomb              1006cd5e f   iconv:iconv.obj
 0001:0006bdbb       _cp858_mbtowc              1006cdbb f   iconv:iconv.obj
 0001:0006bdef       _cp858_wctomb              1006cdef f   iconv:iconv.obj
 0001:0006be57       _cp860_mbtowc              1006ce57 f   iconv:iconv.obj
 0001:0006be76       _cp860_wctomb              1006ce76 f   iconv:iconv.obj
 0001:0006bf15       _cp861_mbtowc              1006cf15 f   iconv:iconv.obj
 0001:0006bf34       _cp861_wctomb              1006cf34 f   iconv:iconv.obj
 0001:0006bfe2       _cp863_mbtowc              1006cfe2 f   iconv:iconv.obj
 0001:0006c001       _cp863_wctomb              1006d001 f   iconv:iconv.obj
 0001:0006c0af       _cp864_mbtowc              1006d0af f   iconv:iconv.obj
 0001:0006c0f8       _cp864_wctomb              1006d0f8 f   iconv:iconv.obj
 0001:0006c1cd       _cp865_mbtowc              1006d1cd f   iconv:iconv.obj
 0001:0006c1ec       _cp865_wctomb              1006d1ec f   iconv:iconv.obj
 0001:0006c29a       _cp869_mbtowc              1006d29a f   iconv:iconv.obj
 0001:0006c2c6       _cp869_wctomb              1006d2c6 f   iconv:iconv.obj
 0001:0006c339       _cp1125_mbtowc             1006d339 f   iconv:iconv.obj
 0001:0006c368       _cp1125_wctomb             1006d368 f   iconv:iconv.obj
 0001:0006c43c       _aliases_hash              1006d43c f   iconv:iconv.obj
 0001:0006c7b9       _unicode_loop_convert      1006d7b9 f   iconv:iconv.obj
 0001:0006c966       _unicode_transliterate     1006d966 f   iconv:iconv.obj
 0001:0006cf99       _johab_hangul_decompose    1006df99 f   iconv:iconv.obj
 0001:0006d056       _unicode_loop_reset        1006e056 f   iconv:iconv.obj
 0001:0006d288       _wchar_id_loop_convert     1006e288 f   iconv:iconv.obj
 0001:0006d3e1       _compare_by_index          1006e3e1 f   iconv:iconv.obj
 0001:0006d3f0       _compare_by_name           1006e3f0 f   iconv:iconv.obj
 0001:0006d4bd       _get_charset_aliases       1006e4bd f   iconv:localcharset.obj
 0001:0006f710       @geVFile_RegisterFileSystemInternal@8 10070710 f   wzFilePacker_static:vfile.obj
 0001:0006f780       _RegisterBuiltInAPIs       10070780 f   wzFilePacker_static:vfile.obj
 0001:0006f810       @CheckOpenFlags@4          10070810 f   wzFilePacker_static:vfile.obj
 0001:0006fa50       _DestroySearchList         10070a50 f   wzFilePacker_static:vfile.obj
 0001:0006fa80       _CopySearchList            10070a80 f   wzFilePacker_static:vfile.obj
 0001:00071220       _geRam_DoCriticalCallback  10072220 f   wzFilePacker_static:Ram.obj
 0001:00071380       @FSVFS_FinderCreate@12     10072380 f   wzFilePacker_static:fsvfs.obj
 0001:000713f0       @FSVFS_FinderGetNextFile@4 100723f0 f   wzFilePacker_static:fsvfs.obj
 0001:00071410       @FSVFS_FinderGetProperties@8 10072410 f   wzFilePacker_static:fsvfs.obj
 0001:00071470       @FSVFS_FinderDestroy@4     10072470 f   wzFilePacker_static:fsvfs.obj
 0001:000714a0       @FSVFS_OpenNewSystem@16    100724a0 f   wzFilePacker_static:fsvfs.obj
 0001:00071b80       @FSVFS_UpdateContext@16    10072b80 f   wzFilePacker_static:fsvfs.obj
 0001:00071b90       @FSVFS_MakeSpace@24        10072b90 f   wzFilePacker_static:fsvfs.obj
 0001:00071e30       @FSVFS_EnlargeDirectorySize@8 10072e30 f   wzFilePacker_static:fsvfs.obj
 0001:00071f10       @FSVFS_Close@4             10072f10 f   wzFilePacker_static:fsvfs.obj
 0001:00072080       @ForceFilePos@4            10073080 f   wzFilePacker_static:fsvfs.obj
 0001:000720a0       _ClampOperationSize        100730a0 f   wzFilePacker_static:fsvfs.obj
 0001:000720e0       @UpdateFilePos@4           100730e0 f   wzFilePacker_static:fsvfs.obj
 0001:000721c0       @FSVFS_GetS@12             100731c0 f   wzFilePacker_static:fsvfs.obj
 0001:00072210       @FSVFS_Read@12             10073210 f   wzFilePacker_static:fsvfs.obj
 0001:00072380       @FSVFS_Write@12            10073380 f   wzFilePacker_static:fsvfs.obj
 0001:000723e0       @FSVFS_Seek@16             100733e0 f   wzFilePacker_static:fsvfs.obj
 0001:00072470       @FSVFS_EOF@4               10073470 f   wzFilePacker_static:fsvfs.obj
 0001:00072490       @FSVFS_Tell@8              10073490 f   wzFilePacker_static:fsvfs.obj
 0001:000724b0       @FSVFS_Size@8              100734b0 f   wzFilePacker_static:fsvfs.obj
 0001:000724d0       @FSVFS_GetProperties@8     100734d0 f   wzFilePacker_static:fsvfs.obj
 0001:00072520       @FSVFS_SetSize@12          10073520 f   wzFilePacker_static:fsvfs.obj
 0001:00072530       @FSVFS_SetAttributes@8     10073530 f   wzFilePacker_static:fsvfs.obj
 0001:00072550       @FSVFS_SetTime@8           10073550 f   wzFilePacker_static:fsvfs.obj
 0001:00072560       @FSVFS_SetHints@8          10073560 f   wzFilePacker_static:fsvfs.obj
 0001:00072570       @FSVFS_FileExists@12       10073570 f   wzFilePacker_static:fsvfs.obj
 0001:00072590       @FSVFS_Disperse@16         10073590 f   wzFilePacker_static:fsvfs.obj
 0001:000725a0       _FSVFS_GetVoidSpace        100735a0 f   wzFilePacker_static:fsvfs.obj
 0001:00072a30       _FSVFS_SetVoidSpace        10073a30 f   wzFilePacker_static:fsvfs.obj
 0001:00072d40       @FSVFS_RenameFile@16       10073d40 f   wzFilePacker_static:fsvfs.obj
 0001:00072d60       @FSVFS_Open@20             10073d60 f   wzFilePacker_static:fsvfs.obj
 0001:00072f20       @FSVFS_DeleteFile@12       10073f20 f   wzFilePacker_static:fsvfs.obj
 0001:00073060       @FSMemory_FinderCreate@12  10074060 f   wzFilePacker_static:FSMEMORY.obj
 0001:00073070       @FSMemory_FinderGetNextFile@4 10074070 f   wzFilePacker_static:FSMEMORY.obj
 0001:00073080       @FSMemory_FinderGetProperties@8 10074080 f   wzFilePacker_static:FSMEMORY.obj
 0001:00073090       @FSMemory_FinderDestroy@4  10074090 f   wzFilePacker_static:FSMEMORY.obj
 0001:000730a0       @FSMemory_Open@20          100740a0 f   wzFilePacker_static:FSMEMORY.obj
 0001:000730b0       @FSMemory_OpenNewSystem@16 100740b0 f   wzFilePacker_static:FSMEMORY.obj
 0001:00073170       @FSMemory_UpdateContext@16 10074170 f   wzFilePacker_static:FSMEMORY.obj
 0001:000731a0       @FSMemory_Close@4          100741a0 f   wzFilePacker_static:FSMEMORY.obj
 0001:000731e0       @ClampOperationSize@12     100741e0 f   wzFilePacker_static:FSMEMORY.obj
 0001:00073220       @DataPtr@4                 10074220 f   wzFilePacker_static:FSMEMORY.obj
 0001:00073230       @FSMemory_GetS@12          10074230 f   wzFilePacker_static:FSMEMORY.obj
 0001:00073290       @FSMemory_Read@12          10074290 f   wzFilePacker_static:FSMEMORY.obj
 0001:000732f0       @TestForExpansion@12       100742f0 f   wzFilePacker_static:FSMEMORY.obj
 0001:00073370       @FSMemory_Write@12         10074370 f   wzFilePacker_static:FSMEMORY.obj
 0001:000733f0       @FSMemory_Seek@16          100743f0 f   wzFilePacker_static:FSMEMORY.obj
 0001:000734c0       @FSMemory_EOF@4            100744c0 f   wzFilePacker_static:FSMEMORY.obj
 0001:000734e0       @FSMemory_Tell@8           100744e0 f   wzFilePacker_static:FSMEMORY.obj
 0001:00073500       @FSMemory_Size@8           10074500 f   wzFilePacker_static:FSMEMORY.obj
 0001:00073520       @FSMemory_GetProperties@8  10074520 f   wzFilePacker_static:FSMEMORY.obj
 0001:00073530       @FSMemory_SetSize@12       10074530 f   wzFilePacker_static:FSMEMORY.obj
 0001:00073540       @FSMemory_SetAttributes@8  10074540 f   wzFilePacker_static:FSMEMORY.obj
 0001:00073550       @FSMemory_SetTime@8        10074550 f   wzFilePacker_static:FSMEMORY.obj
 0001:00073560       @FSMemory_SetHints@8       10074560 f   wzFilePacker_static:FSMEMORY.obj
 0001:00073570       @FSMemory_FileExists@12    10074570 f   wzFilePacker_static:FSMEMORY.obj
 0001:00073580       @FSMemory_Disperse@16      10074580 f   wzFilePacker_static:FSMEMORY.obj
 0001:00073590       @FSMemory_DeleteFile@12    10074590 f   wzFilePacker_static:FSMEMORY.obj
 0001:000735a0       @FSMemory_RenameFile@16    100745a0 f   wzFilePacker_static:FSMEMORY.obj
 0001:000735b0       @FSMemory_EnlargeDirectorySize@8 100745b0 f   wzFilePacker_static:FSMEMORY.obj
 0001:000735d0       _BuildFileName             100745d0 f   wzFilePacker_static:fsdos.obj
 0001:000736a0       @FSDos_FinderCreate@12     100746a0 f   wzFilePacker_static:fsdos.obj
 0001:00073770       @FSDos_FinderGetNextFile@4 10074770 f   wzFilePacker_static:fsdos.obj
 0001:000737e0       @FSDos_FinderGetProperties@8 100747e0 f   wzFilePacker_static:fsdos.obj
 0001:00073860       @FSDos_FinderDestroy@4     10074860 f   wzFilePacker_static:fsdos.obj
 0001:00073890       _IsRootDirectory           10074890 f   wzFilePacker_static:fsdos.obj
 0001:000738e0       @FSDos_Open@20             100748e0 f   wzFilePacker_static:fsdos.obj
 0001:00073ae0       @FSDos_OpenNewSystem@16    10074ae0 f   wzFilePacker_static:fsdos.obj
 0001:00073b00       @FSDos_UpdateContext@16    10074b00 f   wzFilePacker_static:fsdos.obj
 0001:00073b10       @FSDos_Close@4             10074b10 f   wzFilePacker_static:fsdos.obj
 0001:00073b60       @FSDos_GetS@12             10074b60 f   wzFilePacker_static:fsdos.obj
 0001:00073c40       @FSDos_Read@12             10074c40 f   wzFilePacker_static:fsdos.obj
 0001:00073ca0       @FSDos_Write@12            10074ca0 f   wzFilePacker_static:fsdos.obj
 0001:00073ce0       @FSDos_Seek@16             10074ce0 f   wzFilePacker_static:fsdos.obj
 0001:00073da0       @FSDos_EOF@4               10074da0 f   wzFilePacker_static:fsdos.obj
 0001:00073e30       @FSDos_Tell@8              10074e30 f   wzFilePacker_static:fsdos.obj
 0001:00073ea0       @FSDos_Size@8              10074ea0 f   wzFilePacker_static:fsdos.obj
 0001:00073f10       @FSDos_GetProperties@8     10074f10 f   wzFilePacker_static:fsdos.obj
 0001:00073fd0       @FSDos_SetSize@12          10074fd0 f   wzFilePacker_static:fsdos.obj
 0001:00074020       @FSDos_SetAttributes@8     10075020 f   wzFilePacker_static:fsdos.obj
 0001:00074050       @FSDos_SetTime@8           10075050 f   wzFilePacker_static:fsdos.obj
 0001:00074080       @FSDos_SetHints@8          10075080 f   wzFilePacker_static:fsdos.obj
 0001:00074090       @FSDos_FileExists@12       10075090 f   wzFilePacker_static:fsdos.obj
 0001:00074120       @FSDos_Disperse@16         10075120 f   wzFilePacker_static:fsdos.obj
 0001:00074130       @FSDos_DeleteFile@12       10075130 f   wzFilePacker_static:fsdos.obj
 0001:000741c0       @FSDos_RenameFile@16       100751c0 f   wzFilePacker_static:fsdos.obj
 0001:00074270       @FSDos_EnlargeDirectorySize@8 10075270 f   wzFilePacker_static:fsdos.obj
 0001:00074340       _WriteTree                 10075340 f   wzFilePacker_static:dirtree.obj
 0001:000744c0       _DirTree_WriteToFile1      100754c0 f   wzFilePacker_static:dirtree.obj
 0001:00074660       _ReadTree                  10075660 f   wzFilePacker_static:dirtree.obj
 0001:000748b0       _ReadTreeCount             100758b0 f   wzFilePacker_static:dirtree.obj
 0001:00075c80       __os_body_expand           10076c80 f   ogg_static:framing.obj
 0001:00075cb0       __os_lacing_expand         10076cb0 f   ogg_static:framing.obj
 0001:000765a0       __packetout                100775a0 f   ogg_static:framing.obj
 0001:00076a30       _oggpack_writecopy_helper  10077a30 f   ogg_static:bitwise.obj
 0001:00077dd0       __ehhandler$?_Copy@?$basic_string@DU?$char_traits@D@std@@V?$allocator@D@2@@std@@IAEXII@Z 10078dd0 f   sound.obj
 0001:00077df0       __unwindfunclet$??0logic_error@std@@QAE@ABV?$basic_string@DU?$char_traits@D@std@@V?$allocator@D@2@@1@@Z$0 10078df0 f   sound.obj
 0001:00077df8       __ehhandler$??0logic_error@std@@QAE@ABV?$basic_string@DU?$char_traits@D@std@@V?$allocator@D@2@@1@@Z 10078df8 f   sound.obj
 0001:00077e20       __unwindfunclet$?_Insert@?$_Tree@V?$_Tmap_traits@HUsound@@U?$less@H@std@@V?$allocator@U?$pair@$$CBHUsound@@@std@@@3@$0A@@std@@@std@@IAE?AViterator@12@_NPAU_Node@?$_Tree_nod@V?$_Tmap_traits@HUsound@@U?$less@H@std@@V?$allocator@U?$pair@$$CBHUsound@@@std@@@3@$0A@@std@@@2@ABU?$pair@$$CBHUsound@@@2@@Z$0 10078e20 f   sound.obj
 0001:00077e28       __ehhandler$?_Insert@?$_Tree@V?$_Tmap_traits@HUsound@@U?$less@H@std@@V?$allocator@U?$pair@$$CBHUsound@@@std@@@3@$0A@@std@@@std@@IAE?AViterator@12@_NPAU_Node@?$_Tree_nod@V?$_Tmap_traits@HUsound@@U?$less@H@std@@V?$allocator@U?$pair@$$CBHUsound@@@std@@@3@$0A@@std@@@2@ABU?$pair@$$CBHUsound@@@2@@Z 10078e28 f   sound.obj
 0001:00077e50       __unwindfunclet$??0logic_error@std@@QAE@ABV01@@Z$0 10078e50 f   sound.obj
 0001:00077e58       __ehhandler$??0logic_error@std@@QAE@ABV01@@Z 10078e58 f   sound.obj
 0001:00077e80       __unwindfunclet$?erase@?$_Tree@V?$_Tmap_traits@HUsound@@U?$less@H@std@@V?$allocator@U?$pair@$$CBHUsound@@@std@@@3@$0A@@std@@@std@@QAE?AViterator@12@Vconst_iterator@12@@Z$0 10078e80 f   sound.obj
 0001:00077e88       __ehhandler$?erase@?$_Tree@V?$_Tmap_traits@HUsound@@U?$less@H@std@@V?$allocator@U?$pair@$$CBHUsound@@@std@@@3@$0A@@std@@@std@@QAE?AViterator@12@Vconst_iterator@12@@Z 10078e88 f   sound.obj
 0001:00077eb0       __unwindfunclet$??0?$_Tree@V?$_Tmap_traits@HUsound@@U?$less@H@std@@V?$allocator@U?$pair@$$CBHUsound@@@std@@@3@$0A@@std@@@std@@QAE@ABU?$less@H@1@ABV?$allocator@U?$pair@$$CBHUsound@@@std@@@1@@Z$0 10078eb0 f   sound.obj
 0001:00077eb8       __ehhandler$??0?$_Tree@V?$_Tmap_traits@HUsound@@U?$less@H@std@@V?$allocator@U?$pair@$$CBHUsound@@@std@@@3@$0A@@std@@@std@@QAE@ABU?$less@H@1@ABV?$allocator@U?$pair@$$CBHUsound@@@std@@@1@@Z 10078eb8 f   sound.obj
 0001:00077ee0       __unwindfunclet$??1?$_Tree@V?$_Tmap_traits@HUsound@@U?$less@H@std@@V?$allocator@U?$pair@$$CBHUsound@@@std@@@3@$0A@@std@@@std@@QAE@XZ$0 10078ee0 f   sound.obj
 0001:00077ee8       __ehhandler$??1?$_Tree@V?$_Tmap_traits@HUsound@@U?$less@H@std@@V?$allocator@U?$pair@$$CBHUsound@@@std@@@3@$0A@@std@@@std@@QAE@XZ 10078ee8 f   sound.obj
 0001:00077f10       __unwindfunclet$?erase@?$_Tree@V?$_Tmap_traits@HHU?$less@H@std@@V?$allocator@U?$pair@$$CBHH@std@@@2@$0A@@std@@@std@@QAE?AViterator@12@Vconst_iterator@12@@Z$0 10078f10 f   ambientsnd.obj
 0001:00077f18       __ehhandler$?erase@?$_Tree@V?$_Tmap_traits@HHU?$less@H@std@@V?$allocator@U?$pair@$$CBHH@std@@@2@$0A@@std@@@std@@QAE?AViterator@12@Vconst_iterator@12@@Z 10078f18 f   ambientsnd.obj
 0001:00077f40       __unwindfunclet$??0?$_Tree@V?$_Tmap_traits@HHU?$less@H@std@@V?$allocator@U?$pair@$$CBHH@std@@@2@$0A@@std@@@std@@QAE@ABU?$less@H@1@ABV?$allocator@U?$pair@$$CBHH@std@@@1@@Z$0 10078f40 f   ambientsnd.obj
 0001:00077f48       __ehhandler$??0?$_Tree@V?$_Tmap_traits@HHU?$less@H@std@@V?$allocator@U?$pair@$$CBHH@std@@@2@$0A@@std@@@std@@QAE@ABU?$less@H@1@ABV?$allocator@U?$pair@$$CBHH@std@@@1@@Z 10078f48 f   ambientsnd.obj
 0001:00077f70       __unwindfunclet$?_Insert@?$_Tree@V?$_Tmap_traits@HHU?$less@H@std@@V?$allocator@U?$pair@$$CBHH@std@@@2@$0A@@std@@@std@@IAE?AViterator@12@_NPAU_Node@?$_Tree_nod@V?$_Tmap_traits@HHU?$less@H@std@@V?$allocator@U?$pair@$$CBHH@std@@@2@$0A@@std@@@2@ABU?$pair@$$CBHH@2@@Z$0 10078f70 f   ambientsnd.obj
 0001:00077f78       __ehhandler$?_Insert@?$_Tree@V?$_Tmap_traits@HHU?$less@H@std@@V?$allocator@U?$pair@$$CBHH@std@@@2@$0A@@std@@@std@@IAE?AViterator@12@_NPAU_Node@?$_Tree_nod@V?$_Tmap_traits@HHU?$less@H@std@@V?$allocator@U?$pair@$$CBHH@std@@@2@$0A@@std@@@2@ABU?$pair@$$CBHH@2@@Z 10078f78 f   ambientsnd.obj
 0001:00077fa0       __unwindfunclet$?_Insert@?$_Tree@V?$_Tmap_traits@HUAmbientSnd@@U?$less@H@std@@V?$allocator@U?$pair@$$CBHUAmbientSnd@@@std@@@3@$0A@@std@@@std@@IAE?AViterator@12@_NPAU_Node@?$_Tree_nod@V?$_Tmap_traits@HUAmbientSnd@@U?$less@H@std@@V?$allocator@U?$pair@$$CBHUAmbientSnd@@@std@@@3@$0A@@std@@@2@ABU?$pair@$$CBHUAmbientSnd@@@2@@Z$0 10078fa0 f   ambientsnd.obj
 0001:00077fa8       __ehhandler$?_Insert@?$_Tree@V?$_Tmap_traits@HUAmbientSnd@@U?$less@H@std@@V?$allocator@U?$pair@$$CBHUAmbientSnd@@@std@@@3@$0A@@std@@@std@@IAE?AViterator@12@_NPAU_Node@?$_Tree_nod@V?$_Tmap_traits@HUAmbientSnd@@U?$less@H@std@@V?$allocator@U?$pair@$$CBHUAmbientSnd@@@std@@@3@$0A@@std@@@2@ABU?$pair@$$CBHUAmbientSnd@@@2@@Z 10078fa8 f   ambientsnd.obj
 0001:00077fd0       __unwindfunclet$??1?$_Tree@V?$_Tmap_traits@HHU?$less@H@std@@V?$allocator@U?$pair@$$CBHH@std@@@2@$0A@@std@@@std@@QAE@XZ$0 10078fd0 f   ambientsnd.obj
 0001:00077fd8       __ehhandler$??1?$_Tree@V?$_Tmap_traits@HHU?$less@H@std@@V?$allocator@U?$pair@$$CBHH@std@@@2@$0A@@std@@@std@@QAE@XZ 10078fd8 f   ambientsnd.obj
 0001:00078000       __unwindfunclet$??0?$_Tree@V?$_Tmap_traits@HUgame_snd@@U?$less@H@std@@V?$allocator@U?$pair@$$CBHUgame_snd@@@std@@@3@$0A@@std@@@std@@QAE@ABU?$less@H@1@ABV?$allocator@U?$pair@$$CBHUgame_snd@@@std@@@1@@Z$0 10079000 f   scriptparser.obj
 0001:00078008       __ehhandler$??0?$_Tree@V?$_Tmap_traits@HUgame_snd@@U?$less@H@std@@V?$allocator@U?$pair@$$CBHUgame_snd@@@std@@@3@$0A@@std@@@std@@QAE@ABU?$less@H@1@ABV?$allocator@U?$pair@$$CBHUgame_snd@@@std@@@1@@Z 10079008 f   scriptparser.obj
 0001:00078030       __unwindfunclet$?_Insert@?$_Tree@V?$_Tmap_traits@HUgame_snd@@U?$less@H@std@@V?$allocator@U?$pair@$$CBHUgame_snd@@@std@@@3@$0A@@std@@@std@@IAE?AViterator@12@_NPAU_Node@?$_Tree_nod@V?$_Tmap_traits@HUgame_snd@@U?$less@H@std@@V?$allocator@U?$pair@$$CBHUgame_snd@@@std@@@3@$0A@@std@@@2@ABU?$pair@$$CBHUgame_snd@@@2@@Z$0 10079030 f   scriptparser.obj
 0001:00078038       __ehhandler$?_Insert@?$_Tree@V?$_Tmap_traits@HUgame_snd@@U?$less@H@std@@V?$allocator@U?$pair@$$CBHUgame_snd@@@std@@@3@$0A@@std@@@std@@IAE?AViterator@12@_NPAU_Node@?$_Tree_nod@V?$_Tmap_traits@HUgame_snd@@U?$less@H@std@@V?$allocator@U?$pair@$$CBHUgame_snd@@@std@@@3@$0A@@std@@@2@ABU?$pair@$$CBHUgame_snd@@@2@@Z 10079038 f   scriptparser.obj
 0001:00078060       __unwindfunclet$??0?$_Tree@V?$_Tmap_traits@HUAmbientSnd@@U?$less@H@std@@V?$allocator@U?$pair@$$CBHUAmbientSnd@@@std@@@3@$0A@@std@@@std@@QAE@ABU?$less@H@1@ABV?$allocator@U?$pair@$$CBHUAmbientSnd@@@std@@@1@@Z$0 10079060 f   scriptparser.obj
 0001:00078068       __ehhandler$??0?$_Tree@V?$_Tmap_traits@HUAmbientSnd@@U?$less@H@std@@V?$allocator@U?$pair@$$CBHUAmbientSnd@@@std@@@3@$0A@@std@@@std@@QAE@ABU?$less@H@1@ABV?$allocator@U?$pair@$$CBHUAmbientSnd@@@std@@@1@@Z 10079068 f   scriptparser.obj
 0001:00078090       __unwindfunclet$??0?$_Tree@V?$_Tmap_traits@HUVoiceSnd@@U?$less@H@std@@V?$allocator@U?$pair@$$CBHUVoiceSnd@@@std@@@3@$0A@@std@@@std@@QAE@ABU?$less@H@1@ABV?$allocator@U?$pair@$$CBHUVoiceSnd@@@std@@@1@@Z$0 10079090 f   scriptparser.obj
 0001:00078098       __ehhandler$??0?$_Tree@V?$_Tmap_traits@HUVoiceSnd@@U?$less@H@std@@V?$allocator@U?$pair@$$CBHUVoiceSnd@@@std@@@3@$0A@@std@@@std@@QAE@ABU?$less@H@1@ABV?$allocator@U?$pair@$$CBHUVoiceSnd@@@std@@@1@@Z 10079098 f   scriptparser.obj
 0001:000780c0       __unwindfunclet$?_Xlen@?$vector@UST_CELLS@@V?$allocator@UST_CELLS@@@std@@@std@@KAXXZ$0 100790c0 f   scriptparser.obj
 0001:000780c8       __ehhandler$?_Xlen@?$vector@UST_CELLS@@V?$allocator@UST_CELLS@@@std@@@std@@KAXXZ 100790c8 f   scriptparser.obj
 0001:000780f0       __unwindfunclet$?erase@?$_Tree@V?$_Tmap_traits@HUgame_snd@@U?$less@H@std@@V?$allocator@U?$pair@$$CBHUgame_snd@@@std@@@3@$0A@@std@@@std@@QAE?AViterator@12@Vconst_iterator@12@@Z$0 100790f0 f   scriptparser.obj
 0001:000780f8       __ehhandler$?erase@?$_Tree@V?$_Tmap_traits@HUgame_snd@@U?$less@H@std@@V?$allocator@U?$pair@$$CBHUgame_snd@@@std@@@3@$0A@@std@@@std@@QAE?AViterator@12@Vconst_iterator@12@@Z 100790f8 f   scriptparser.obj
 0001:00078120       __unwindfunclet$?erase@?$_Tree@V?$_Tmap_traits@HUAmbientSnd@@U?$less@H@std@@V?$allocator@U?$pair@$$CBHUAmbientSnd@@@std@@@3@$0A@@std@@@std@@QAE?AViterator@12@Vconst_iterator@12@@Z$0 10079120 f   scriptparser.obj
 0001:00078128       __ehhandler$?erase@?$_Tree@V?$_Tmap_traits@HUAmbientSnd@@U?$less@H@std@@V?$allocator@U?$pair@$$CBHUAmbientSnd@@@std@@@3@$0A@@std@@@std@@QAE?AViterator@12@Vconst_iterator@12@@Z 10079128 f   scriptparser.obj
 0001:00078150       __unwindfunclet$?erase@?$_Tree@V?$_Tmap_traits@HUVoiceSnd@@U?$less@H@std@@V?$allocator@U?$pair@$$CBHUVoiceSnd@@@std@@@3@$0A@@std@@@std@@QAE?AViterator@12@Vconst_iterator@12@@Z$0 10079150 f   scriptparser.obj
 0001:00078158       __ehhandler$?erase@?$_Tree@V?$_Tmap_traits@HUVoiceSnd@@U?$less@H@std@@V?$allocator@U?$pair@$$CBHUVoiceSnd@@@std@@@3@$0A@@std@@@std@@QAE?AViterator@12@Vconst_iterator@12@@Z 10079158 f   scriptparser.obj
 0001:00078180       __unwindfunclet$??0?$vector@UST_CELLS@@V?$allocator@UST_CELLS@@@std@@@std@@QAE@XZ$0 10079180 f   scriptparser.obj
 0001:00078188       __ehhandler$??0?$vector@UST_CELLS@@V?$allocator@UST_CELLS@@@std@@@std@@QAE@XZ 10079188 f   scriptparser.obj
 0001:000781b0       __unwindfunclet$??1?$_Tree@V?$_Tmap_traits@HUgame_snd@@U?$less@H@std@@V?$allocator@U?$pair@$$CBHUgame_snd@@@std@@@3@$0A@@std@@@std@@QAE@XZ$0 100791b0 f   scriptparser.obj
 0001:000781b8       __ehhandler$??1?$_Tree@V?$_Tmap_traits@HUgame_snd@@U?$less@H@std@@V?$allocator@U?$pair@$$CBHUgame_snd@@@std@@@3@$0A@@std@@@std@@QAE@XZ 100791b8 f   scriptparser.obj
 0001:000781e0       __unwindfunclet$??1?$_Tree@V?$_Tmap_traits@HUAmbientSnd@@U?$less@H@std@@V?$allocator@U?$pair@$$CBHUAmbientSnd@@@std@@@3@$0A@@std@@@std@@QAE@XZ$0 100791e0 f   scriptparser.obj
 0001:000781e8       __ehhandler$??1?$_Tree@V?$_Tmap_traits@HUAmbientSnd@@U?$less@H@std@@V?$allocator@U?$pair@$$CBHUAmbientSnd@@@std@@@3@$0A@@std@@@std@@QAE@XZ 100791e8 f   scriptparser.obj
 0001:00078210       __unwindfunclet$??1?$_Tree@V?$_Tmap_traits@HUVoiceSnd@@U?$less@H@std@@V?$allocator@U?$pair@$$CBHUVoiceSnd@@@std@@@3@$0A@@std@@@std@@QAE@XZ$0 10079210 f   scriptparser.obj
 0001:00078218       __ehhandler$??1?$_Tree@V?$_Tmap_traits@HUVoiceSnd@@U?$less@H@std@@V?$allocator@U?$pair@$$CBHUVoiceSnd@@@std@@@3@$0A@@std@@@std@@QAE@XZ 10079218 f   scriptparser.obj
 0001:00078240       __unwindfunclet$?gamesnd_parse_musictxt@@YAXPAD@Z$0 10079240 f   scriptparser.obj
 0001:00078248       __unwindfunclet$?gamesnd_parse_musictxt@@YAXPAD@Z$1 10079248 f   scriptparser.obj
 0001:00078250       __ehhandler$?gamesnd_parse_musictxt@@YAXPAD@Z 10079250 f   scriptparser.obj
 0001:00078280       __unwindfunclet$?gamesnd_parse_voicetxt@@YAXPAD@Z$0 10079280 f   scriptparser.obj
 0001:00078288       __unwindfunclet$?gamesnd_parse_voicetxt@@YAXPAD@Z$1 10079288 f   scriptparser.obj
 0001:00078290       __ehhandler$?gamesnd_parse_voicetxt@@YAXPAD@Z 10079290 f   scriptparser.obj
 0001:000782c0       __unwindfunclet$?gamesnd_parse_configtxt@@YAXPAD@Z$0 100792c0 f   scriptparser.obj
 0001:000782cb       __unwindfunclet$?gamesnd_parse_configtxt@@YAXPAD@Z$1 100792cb f   scriptparser.obj
 0001:000782d3       __ehhandler$?gamesnd_parse_configtxt@@YAXPAD@Z 100792d3 f   scriptparser.obj
 0001:00078310       __unwindfunclet$?gamesnd_parse_soundtxt@@YAXPAD@Z$0 10079310 f   scriptparser.obj
 0001:0007831b       __unwindfunclet$?gamesnd_parse_soundtxt@@YAXPAD@Z$1 1007931b f   scriptparser.obj
 0001:00078326       __ehhandler$?gamesnd_parse_soundtxt@@YAXPAD@Z 10079326 f   scriptparser.obj
 0001:00078360       __unwindfunclet$??$_Construct@V?$basic_string@DU?$char_traits@D@std@@V?$allocator@D@2@@std@@V12@@std@@YAXPAV?$basic_string@DU?$char_traits@D@std@@V?$allocator@D@2@@0@ABV10@@Z$0 10079360 f   xls.obj
 0001:00078371       __ehhandler$??$_Construct@V?$basic_string@DU?$char_traits@D@std@@V?$allocator@D@2@@std@@V12@@std@@YAXPAV?$basic_string@DU?$char_traits@D@std@@V?$allocator@D@2@@0@ABV10@@Z 10079371 f   xls.obj
 0001:00078390       __unwindfunclet$?_Xlen@?$vector@V?$basic_string@DU?$char_traits@D@std@@V?$allocator@D@2@@std@@V?$allocator@V?$basic_string@DU?$char_traits@D@std@@V?$allocator@D@2@@std@@@2@@std@@KAXXZ$0 10079390 f   xls.obj
 0001:00078398       __ehhandler$?_Xlen@?$vector@V?$basic_string@DU?$char_traits@D@std@@V?$allocator@D@2@@std@@V?$allocator@V?$basic_string@DU?$char_traits@D@std@@V?$allocator@D@2@@std@@@2@@std@@KAXXZ 10079398 f   xls.obj
 0001:000783c0       __unwindfunclet$??$_Uninit_copy@PBV?$basic_string@DU?$char_traits@D@std@@V?$allocator@D@2@@std@@PAV12@V?$allocator@V?$basic_string@DU?$char_traits@D@std@@V?$allocator@D@2@@std@@@2@@std@@YAPAV?$basic_string@DU?$char_traits@D@std@@V?$allocator@D@2@@0@PBV10@0PAV10@AAV?$allocator@V?$basic_string@DU?$char_traits@D@std@@V?$allocator@D@2@@std@@@0@U_Nonscalar_ptr_iterator_tag@0@U_Range_checked_iterator_tag@0@@Z$2 100793c0 f   xls.obj
 0001:000783d1       __ehhandler$??$_Uninit_copy@PBV?$basic_string@DU?$char_traits@D@std@@V?$allocator@D@2@@std@@PAV12@V?$allocator@V?$basic_string@DU?$char_traits@D@std@@V?$allocator@D@2@@std@@@2@@std@@YAPAV?$basic_string@DU?$char_traits@D@std@@V?$allocator@D@2@@0@PBV10@0PAV10@AAV?$allocator@V?$basic_string@DU?$char_traits@D@std@@V?$allocator@D@2@@std@@@0@U_Nonscalar_ptr_iterator_tag@0@U_Range_checked_iterator_tag@0@@Z 100793d1 f   xls.obj
 0001:000783f0       __unwindfunclet$??$_Uninit_copy@PAV?$basic_string@DU?$char_traits@D@std@@V?$allocator@D@2@@std@@PAV12@V?$allocator@V?$basic_string@DU?$char_traits@D@std@@V?$allocator@D@2@@std@@@2@@std@@YAPAV?$basic_string@DU?$char_traits@D@std@@V?$allocator@D@2@@0@PAV10@00AAV?$allocator@V?$basic_string@DU?$char_traits@D@std@@V?$allocator@D@2@@std@@@0@U_Nonscalar_ptr_iterator_tag@0@U_Range_checked_iterator_tag@0@@Z$2 100793f0 f   xls.obj
 0001:00078401       __ehhandler$??$_Uninit_copy@PAV?$basic_string@DU?$char_traits@D@std@@V?$allocator@D@2@@std@@PAV12@V?$allocator@V?$basic_string@DU?$char_traits@D@std@@V?$allocator@D@2@@std@@@2@@std@@YAPAV?$basic_string@DU?$char_traits@D@std@@V?$allocator@D@2@@0@PAV10@00AAV?$allocator@V?$basic_string@DU?$char_traits@D@std@@V?$allocator@D@2@@std@@@0@U_Nonscalar_ptr_iterator_tag@0@U_Range_checked_iterator_tag@0@@Z 10079401 f   xls.obj
 0001:00078420       __unwindfunclet$??$_Uninit_fill_n@PAV?$basic_string@DU?$char_traits@D@std@@V?$allocator@D@2@@std@@IV12@V?$allocator@V?$basic_string@DU?$char_traits@D@std@@V?$allocator@D@2@@std@@@2@@std@@YAXPAV?$basic_string@DU?$char_traits@D@std@@V?$allocator@D@2@@0@IABV10@AAV?$allocator@V?$basic_string@DU?$char_traits@D@std@@V?$allocator@D@2@@std@@@0@U_Nonscalar_ptr_iterator_tag@0@U_Range_checked_iterator_tag@0@@Z$2 10079420 f   xls.obj
 0001:00078431       __ehhandler$??$_Uninit_fill_n@PAV?$basic_string@DU?$char_traits@D@std@@V?$allocator@D@2@@std@@IV12@V?$allocator@V?$basic_string@DU?$char_traits@D@std@@V?$allocator@D@2@@std@@@2@@std@@YAXPAV?$basic_string@DU?$char_traits@D@std@@V?$allocator@D@2@@0@IABV10@AAV?$allocator@V?$basic_string@DU?$char_traits@D@std@@V?$allocator@D@2@@std@@@0@U_Nonscalar_ptr_iterator_tag@0@U_Range_checked_iterator_tag@0@@Z 10079431 f   xls.obj
 0001:00078450       __unwindfunclet$??0?$vector@V?$basic_string@DU?$char_traits@D@std@@V?$allocator@D@2@@std@@V?$allocator@V?$basic_string@DU?$char_traits@D@std@@V?$allocator@D@2@@std@@@2@@std@@QAE@XZ$0 10079450 f   xls.obj
 0001:00078458       __ehhandler$??0?$vector@V?$basic_string@DU?$char_traits@D@std@@V?$allocator@D@2@@std@@V?$allocator@V?$basic_string@DU?$char_traits@D@std@@V?$allocator@D@2@@std@@@2@@std@@QAE@XZ 10079458 f   xls.obj
 0001:00078480       __unwindfunclet$??$_Uninit_move@PAV?$basic_string@DU?$char_traits@D@std@@V?$allocator@D@2@@std@@PAV12@V?$allocator@V?$basic_string@DU?$char_traits@D@std@@V?$allocator@D@2@@std@@@2@@std@@YAPAV?$basic_string@DU?$char_traits@D@std@@V?$allocator@D@2@@0@PAV10@00AAV?$allocator@V?$basic_string@DU?$char_traits@D@std@@V?$allocator@D@2@@std@@@0@U_Swap_move_tag@0@U_Range_checked_iterator_tag@0@@Z$2 10079480 f   xls.obj
 0001:00078488       __unwindfunclet$??$_Uninit_move@PAV?$basic_string@DU?$char_traits@D@std@@V?$allocator@D@2@@std@@PAV12@V?$allocator@V?$basic_string@DU?$char_traits@D@std@@V?$allocator@D@2@@std@@@2@@std@@YAPAV?$basic_string@DU?$char_traits@D@std@@V?$allocator@D@2@@0@PAV10@00AAV?$allocator@V?$basic_string@DU?$char_traits@D@std@@V?$allocator@D@2@@std@@@0@U_Swap_move_tag@0@U_Range_checked_iterator_tag@0@@Z$3 10079488 f   xls.obj
 0001:00078499       __ehhandler$??$_Uninit_move@PAV?$basic_string@DU?$char_traits@D@std@@V?$allocator@D@2@@std@@PAV12@V?$allocator@V?$basic_string@DU?$char_traits@D@std@@V?$allocator@D@2@@std@@@2@@std@@YAPAV?$basic_string@DU?$char_traits@D@std@@V?$allocator@D@2@@0@PAV10@00AAV?$allocator@V?$basic_string@DU?$char_traits@D@std@@V?$allocator@D@2@@std@@@0@U_Swap_move_tag@0@U_Range_checked_iterator_tag@0@@Z 10079499 f   xls.obj
 0001:000784c0       __unwindfunclet$??0?$vector@V?$basic_string@DU?$char_traits@D@std@@V?$allocator@D@2@@std@@V?$allocator@V?$basic_string@DU?$char_traits@D@std@@V?$allocator@D@2@@std@@@2@@std@@QAE@ABV01@@Z$2 100794c0 f   xls.obj
 0001:000784c8       __ehhandler$??0?$vector@V?$basic_string@DU?$char_traits@D@std@@V?$allocator@D@2@@std@@V?$allocator@V?$basic_string@DU?$char_traits@D@std@@V?$allocator@D@2@@std@@@2@@std@@QAE@ABV01@@Z 100794c8 f   xls.obj
 0001:000784f0       __unwindfunclet$??$_Construct@UST_CELLS@@U1@@std@@YAXPAUST_CELLS@@ABU1@@Z$0 100794f0 f   xls.obj
 0001:00078501       __ehhandler$??$_Construct@UST_CELLS@@U1@@std@@YAXPAUST_CELLS@@ABU1@@Z 10079501 f   xls.obj
 0001:00078520       __unwindfunclet$?_Insert_n@?$vector@V?$basic_string@DU?$char_traits@D@std@@V?$allocator@D@2@@std@@V?$allocator@V?$basic_string@DU?$char_traits@D@std@@V?$allocator@D@2@@std@@@2@@std@@IAEXV?$_Vector_const_iterator@V?$basic_string@DU?$char_traits@D@std@@V?$allocator@D@2@@std@@V?$allocator@V?$basic_string@DU?$char_traits@D@std@@V?$allocator@D@2@@std@@@2@@2@IABV?$basic_string@DU?$char_traits@D@std@@V?$allocator@D@2@@2@@Z$4 10079520 f   xls.obj
 0001:00078528       __unwindfunclet$?_Insert_n@?$vector@V?$basic_string@DU?$char_traits@D@std@@V?$allocator@D@2@@std@@V?$allocator@V?$basic_string@DU?$char_traits@D@std@@V?$allocator@D@2@@std@@@2@@std@@IAEXV?$_Vector_const_iterator@V?$basic_string@DU?$char_traits@D@std@@V?$allocator@D@2@@std@@V?$allocator@V?$basic_string@DU?$char_traits@D@std@@V?$allocator@D@2@@std@@@2@@2@IABV?$basic_string@DU?$char_traits@D@std@@V?$allocator@D@2@@2@@Z$5 10079528 f   xls.obj
 0001:00078530       __ehhandler$?_Insert_n@?$vector@V?$basic_string@DU?$char_traits@D@std@@V?$allocator@D@2@@std@@V?$allocator@V?$basic_string@DU?$char_traits@D@std@@V?$allocator@D@2@@std@@@2@@std@@IAEXV?$_Vector_const_iterator@V?$basic_string@DU?$char_traits@D@std@@V?$allocator@D@2@@std@@V?$allocator@V?$basic_string@DU?$char_traits@D@std@@V?$allocator@D@2@@std@@@2@@2@IABV?$basic_string@DU?$char_traits@D@std@@V?$allocator@D@2@@2@@Z 10079530 f   xls.obj
 0001:00078560       __unwindfunclet$??$_Uninit_copy@PAUST_CELLS@@PAU1@V?$allocator@UST_CELLS@@@std@@@std@@YAPAUST_CELLS@@PAU1@00AAV?$allocator@UST_CELLS@@@0@U_Nonscalar_ptr_iterator_tag@0@U_Range_checked_iterator_tag@0@@Z$2 10079560 f   xls.obj
 0001:00078571       __ehhandler$??$_Uninit_copy@PAUST_CELLS@@PAU1@V?$allocator@UST_CELLS@@@std@@@std@@YAPAUST_CELLS@@PAU1@00AAV?$allocator@UST_CELLS@@@0@U_Nonscalar_ptr_iterator_tag@0@U_Range_checked_iterator_tag@0@@Z 10079571 f   xls.obj
 0001:00078590       __unwindfunclet$??$_Uninit_fill_n@PAUST_CELLS@@IU1@V?$allocator@UST_CELLS@@@std@@@std@@YAXPAUST_CELLS@@IABU1@AAV?$allocator@UST_CELLS@@@0@U_Nonscalar_ptr_iterator_tag@0@U_Range_checked_iterator_tag@0@@Z$2 10079590 f   xls.obj
 0001:000785a1       __ehhandler$??$_Uninit_fill_n@PAUST_CELLS@@IU1@V?$allocator@UST_CELLS@@@std@@@std@@YAXPAUST_CELLS@@IABU1@AAV?$allocator@UST_CELLS@@@0@U_Nonscalar_ptr_iterator_tag@0@U_Range_checked_iterator_tag@0@@Z 100795a1 f   xls.obj
 0001:000785c0       __unwindfunclet$?_Insert_n@?$vector@UST_CELLS@@V?$allocator@UST_CELLS@@@std@@@std@@IAEXV?$_Vector_const_iterator@UST_CELLS@@V?$allocator@UST_CELLS@@@std@@@2@IABUST_CELLS@@@Z$4 100795c0 f   xls.obj
 0001:000785c8       __unwindfunclet$?_Insert_n@?$vector@UST_CELLS@@V?$allocator@UST_CELLS@@@std@@@std@@IAEXV?$_Vector_const_iterator@UST_CELLS@@V?$allocator@UST_CELLS@@@std@@@2@IABUST_CELLS@@@Z$5 100795c8 f   xls.obj
 0001:000785d0       __ehhandler$?_Insert_n@?$vector@UST_CELLS@@V?$allocator@UST_CELLS@@@std@@@std@@IAEXV?$_Vector_const_iterator@UST_CELLS@@V?$allocator@UST_CELLS@@@std@@@2@IABUST_CELLS@@@Z 100795d0 f   xls.obj
 0001:000785f0       __unwindfunclet$?SetRow@@YAXV?$basic_string@DU?$char_traits@D@std@@V?$allocator@D@2@@std@@PAUST_ROWS@@@Z$0 100795f0 f   xls.obj
 0001:000785f8       __unwindfunclet$?SetRow@@YAXV?$basic_string@DU?$char_traits@D@std@@V?$allocator@D@2@@std@@PAUST_ROWS@@@Z$1 100795f8 f   xls.obj
 0001:00078600       __unwindfunclet$?SetRow@@YAXV?$basic_string@DU?$char_traits@D@std@@V?$allocator@D@2@@std@@PAUST_ROWS@@@Z$2 10079600 f   xls.obj
 0001:00078608       __unwindfunclet$?SetRow@@YAXV?$basic_string@DU?$char_traits@D@std@@V?$allocator@D@2@@std@@PAUST_ROWS@@@Z$3 10079608 f   xls.obj
 0001:00078610       __ehhandler$?SetRow@@YAXV?$basic_string@DU?$char_traits@D@std@@V?$allocator@D@2@@std@@PAUST_ROWS@@@Z 10079610 f   xls.obj
 0001:00078630       __unwindfunclet$?SetRows@@YAXAAV?$basic_string@DU?$char_traits@D@std@@V?$allocator@D@2@@std@@PAUST_ROWS@@@Z$0 10079630 f   xls.obj
 0001:00078638       __unwindfunclet$?SetRows@@YAXAAV?$basic_string@DU?$char_traits@D@std@@V?$allocator@D@2@@std@@PAUST_ROWS@@@Z$1 10079638 f   xls.obj
 0001:00078640       __ehhandler$?SetRows@@YAXAAV?$basic_string@DU?$char_traits@D@std@@V?$allocator@D@2@@std@@PAUST_ROWS@@@Z 10079640 f   xls.obj
 0001:00078670       __unwindfunclet$?GetTxtFile@@YAHPADPAUST_ROWS@@@Z$0 10079670 f   xls.obj
 0001:0007867b       __ehhandler$?GetTxtFile@@YAHPADPAUST_ROWS@@@Z 1007967b f   xls.obj
 0001:000786a9       __unwindfunclet$?_Xlen@_String_base@std@@SAXXZ$0 100796a9 f   libcpmt:string.obj
 0001:000786b1       __ehhandler$?_Xlen@_String_base@std@@SAXXZ 100796b1 f   libcpmt:string.obj
 0001:000786cc       __unwindfunclet$?_Xran@_String_base@std@@SAXXZ$0 100796cc f   libcpmt:string.obj
 0001:000786d4       __ehhandler$?_Xran@_String_base@std@@SAXXZ 100796d4 f   libcpmt:string.obj
 0001:000786ef       __unwindfunclet$?_Xinvarg@_String_base@std@@SAXXZ$0 100796ef f   libcpmt:string.obj
 0001:000786f7       __ehhandler$?_Xinvarg@_String_base@std@@SAXXZ 100796f7 f   libcpmt:string.obj
 0001:00078712       __ehhandler$?CallUnexpected@@YAXPBU_s_ESTypeList@@@Z 10079712 f   LIBCMT:frame.obj
 0001:00078730       __unwindfunclet$?FindFile@CPackFile@@QAEHPAXPBDAAV?$vector@V?$basic_string@DU?$char_traits@D@std@@V?$allocator@D@2@@std@@V?$allocator@V?$basic_string@DU?$char_traits@D@std@@V?$allocator@D@2@@std@@@2@@std@@2H@Z$0 10079730 f   wzFilePacker_static:wzFilePacker.obj
 0001:0007873b       __unwindfunclet$?FindFile@CPackFile@@QAEHPAXPBDAAV?$vector@V?$basic_string@DU?$char_traits@D@std@@V?$allocator@D@2@@std@@V?$allocator@V?$basic_string@DU?$char_traits@D@std@@V?$allocator@D@2@@std@@@2@@std@@2H@Z$1 1007973b f   wzFilePacker_static:wzFilePacker.obj
 0001:00078746       __ehhandler$?FindFile@CPackFile@@QAEHPAXPBDAAV?$vector@V?$basic_string@DU?$char_traits@D@std@@V?$allocator@D@2@@std@@V?$allocator@V?$basic_string@DU?$char_traits@D@std@@V?$allocator@D@2@@std@@@2@@std@@2H@Z 10079746 f   wzFilePacker_static:wzFilePacker.obj
 0001:00078780       __unwindfunclet$?ExtractAll@CPackFile@@QAEHPAXPBD@Z$0 10079780 f   wzFilePacker_static:wzFilePacker.obj
 0001:0007878b       __unwindfunclet$?ExtractAll@CPackFile@@QAEHPAXPBD@Z$1 1007978b f   wzFilePacker_static:wzFilePacker.obj
 0001:00078796       __unwindfunclet$?ExtractAll@CPackFile@@QAEHPAXPBD@Z$2 10079796 f   wzFilePacker_static:wzFilePacker.obj
 0001:0007879e       __unwindfunclet$?ExtractAll@CPackFile@@QAEHPAXPBD@Z$3 1007979e f   wzFilePacker_static:wzFilePacker.obj
 0001:000787a6       __unwindfunclet$?ExtractAll@CPackFile@@QAEHPAXPBD@Z$4 100797a6 f   wzFilePacker_static:wzFilePacker.obj
 0001:000787ae       __unwindfunclet$?ExtractAll@CPackFile@@QAEHPAXPBD@Z$5 100797ae f   wzFilePacker_static:wzFilePacker.obj
 0001:000787b6       __unwindfunclet$?ExtractAll@CPackFile@@QAEHPAXPBD@Z$6 100797b6 f   wzFilePacker_static:wzFilePacker.obj
 0001:000787be       __unwindfunclet$?ExtractAll@CPackFile@@QAEHPAXPBD@Z$7 100797be f   wzFilePacker_static:wzFilePacker.obj
 0001:000787c9       __unwindfunclet$?ExtractAll@CPackFile@@QAEHPAXPBD@Z$8 100797c9 f   wzFilePacker_static:wzFilePacker.obj
 0001:000787d4       __unwindfunclet$?ExtractAll@CPackFile@@QAEHPAXPBD@Z$9 100797d4 f   wzFilePacker_static:wzFilePacker.obj
 0001:000787dc       __ehhandler$?ExtractAll@CPackFile@@QAEHPAXPBD@Z 100797dc f   wzFilePacker_static:wzFilePacker.obj
 0001:00078810       __unwindfunclet$?MurgeFile@CPackFile@@QAEHPAXH@Z$0 10079810 f   wzFilePacker_static:wzFilePacker.obj
 0001:0007881b       __unwindfunclet$?MurgeFile@CPackFile@@QAEHPAXH@Z$1 1007981b f   wzFilePacker_static:wzFilePacker.obj
 0001:00078826       __ehhandler$?MurgeFile@CPackFile@@QAEHPAXH@Z 10079826 f   wzFilePacker_static:wzFilePacker.obj
 0001:00078860       ??__EAudio_streams@@YAXXZ  10079860 f   audiostr.obj
 0001:00078890       ??__Emap_sounds@@YAXXZ     10079890 f   sound.obj
 0001:000788c0       ??__Eambi_handles@@YAXXZ   100798c0 f   ambientsnd.obj
 0001:000788f0       ??__Emusic_handles@@YAXXZ  100798f0 f   eventmusic.obj
 0001:00078920       ??__ESnds@@YAXXZ           10079920 f   scriptparser.obj
 0001:00078950       ??__ESnds_iface@@YAXXZ     10079950 f   scriptparser.obj
 0001:00078980       ??__EAmbientTbl@@YAXXZ     10079980 f   scriptparser.obj
 0001:000789b0       ??__EVoiceTbl@@YAXXZ       100799b0 f   scriptparser.obj
 0001:000789e0       ??__Eindex_table_event_music@@YAXXZ 100799e0 f   scriptparser.obj
 0001:00078a10       ??__Eindex_table_voice_sound@@YAXXZ 10079a10 f   scriptparser.obj
 0001:00078a40       ??__Evoice_handles@@YAXXZ  10079a40 f   voicesnd.obj
 0001:00078a70       ??__EpackFile@@YAXXZ       10079a70 f   util_packfile.obj
 0001:00078a90       ??__Eautofree@@YAXXZ       10079a90 f   wzFilePacker_static:wzFilePacker.obj
 0001:00078aa0       ??__FAudio_streams@@YAXXZ  10079aa0 f   audiostr.obj
 0001:00078ac0       ??__Fmap_sounds@@YAXXZ     10079ac0 f   sound.obj
 0001:00078ad0       ??__Fambi_handles@@YAXXZ   10079ad0 f   ambientsnd.obj
 0001:00078ae0       ??__Fmusic_handles@@YAXXZ  10079ae0 f   eventmusic.obj
 0001:00078af0       ??__FSnds_iface@@YAXXZ     10079af0 f   scriptparser.obj
 0001:00078b00       ??__Findex_table_voice_sound@@YAXXZ 10079b00 f   scriptparser.obj
 0001:00078b10       ??__FSnds@@YAXXZ           10079b10 f   scriptparser.obj
 0001:00078b20       ??__FAmbientTbl@@YAXXZ     10079b20 f   scriptparser.obj
 0001:00078b30       ??__FVoiceTbl@@YAXXZ       10079b30 f   scriptparser.obj
 0001:00078b40       ??__Findex_table_event_music@@YAXXZ 10079b40 f   scriptparser.obj
 0001:00078b50       ??__Fvoice_handles@@YAXXZ  10079b50 f   voicesnd.obj
 0001:00078b60       ??__FpackFile@@YAXXZ       10079b60 f   util_packfile.obj
 0001:00078b6a       ??__Fnomem@?5???2@YAPAXI@Z@YAXXZ 10079b6a f   LIBCMT:new.obj
 0001:00078b80       ??__Fautofree@@YAXXZ       10079b80 f   wzFilePacker_static:wzFilePacker.obj

 Exports

  ordinal    name

        1    ?wzsnd_cache_is@@YA_NXZ (bool __cdecl wzsnd_cache_is(void))
               exported name: wzsnd_cache_is
        2    ?wzsnd_cache_maintain_milliseconds_get@@YAHXZ (int __cdecl wzsnd_cache_maintain_milliseconds_get(void))
               exported name: wzsnd_cache_maintain_milliseconds_get
        3    ?wzsnd_cache_maintain_milliseconds_set@@YAXH@Z (void __cdecl wzsnd_cache_maintain_milliseconds_set(int))
               exported name: wzsnd_cache_maintain_milliseconds_set
        4    ?wzsnd_cache_off@@YAXXZ (void __cdecl wzsnd_cache_off(void))
               exported name: wzsnd_cache_off
        5    ?wzsnd_cache_on@@YAXXZ (void __cdecl wzsnd_cache_on(void))
               exported name: wzsnd_cache_on
        6    ?wzsnd_cache_size@@YAHXZ (int __cdecl wzsnd_cache_size(void))
               exported name: wzsnd_cache_size
        7    ?wzsnd_check_channel@@YAXXZ (void __cdecl wzsnd_check_channel(void))
               exported name: wzsnd_check_channel
        8    ?wzsnd_env_disable@@YAXXZ (void __cdecl wzsnd_env_disable(void))
               exported name: wzsnd_env_disable
        9    ?wzsnd_env_get@@YAXPAUsound_env@@@Z (void __cdecl wzsnd_env_get(struct sound_env *))
               exported name: wzsnd_env_get
       10    ?wzsnd_env_set@@YAXPAUsound_env@@@Z (void __cdecl wzsnd_env_set(struct sound_env *))
               exported name: wzsnd_env_set
       11    ?wzsnd_env_set_preset@@YAXK@Z (void __cdecl wzsnd_env_set_preset(unsigned long))
               exported name: wzsnd_env_set_preset
       12    ?wzsnd_env_supported@@YAHXZ (int __cdecl wzsnd_env_supported(void))
               exported name: wzsnd_env_supported
       13    ?wzsnd_getState_ambi@@YAHH@Z (int __cdecl wzsnd_getState_ambi(int))
               exported name: wzsnd_getState_ambi
       14    ?wzsnd_getState_bgm@@YAHH@Z (int __cdecl wzsnd_getState_bgm(int))
               exported name: wzsnd_getState_bgm
       15    ?wzsnd_getState_sound@@YAHH@Z (int __cdecl wzsnd_getState_sound(int))
               exported name: wzsnd_getState_sound
       16    ?wzsnd_getState_voice@@YAHH@Z (int __cdecl wzsnd_getState_voice(int))
               exported name: wzsnd_getState_voice
       17    ?wzsnd_get_ambienttable@@YAHPAUsoundEntry@@@Z (int __cdecl wzsnd_get_ambienttable(struct soundEntry *))
               exported name: wzsnd_get_ambienttable
       18    ?wzsnd_get_interfacesoundtable@@YAHPAUsoundEntry@@@Z (int __cdecl wzsnd_get_interfacesoundtable(struct soundEntry *))
               exported name: wzsnd_get_interfacesoundtable
       19    ?wzsnd_get_master_mute@@YA_NXZ (bool __cdecl wzsnd_get_master_mute(void))
               exported name: wzsnd_get_master_mute
       20    ?wzsnd_get_master_vol@@YAXPAH0@Z (void __cdecl wzsnd_get_master_vol(int *,int *))
               exported name: wzsnd_get_master_vol
       21    ?wzsnd_get_mic_input_vol@@YAXPAK@Z (void __cdecl wzsnd_get_mic_input_vol(unsigned long *))
               exported name: wzsnd_get_mic_input_vol
       22    ?wzsnd_get_mic_output_mute@@YA_NXZ (bool __cdecl wzsnd_get_mic_output_mute(void))
               exported name: wzsnd_get_mic_output_mute
       23    ?wzsnd_get_mic_output_vol@@YAXPAK@Z (void __cdecl wzsnd_get_mic_output_vol(unsigned long *))
               exported name: wzsnd_get_mic_output_vol
       24    ?wzsnd_get_soundtable@@YAHPAUsoundEntry@@@Z (int __cdecl wzsnd_get_soundtable(struct soundEntry *))
               exported name: wzsnd_get_soundtable
       25    ?wzsnd_get_soundtableArray@@YAHPAUsoundEntry@@@Z (int __cdecl wzsnd_get_soundtableArray(struct soundEntry *))
               exported name: wzsnd_get_soundtableArray
       26    ?wzsnd_get_wav_mute@@YA_NXZ (bool __cdecl wzsnd_get_wav_mute(void))
               exported name: wzsnd_get_wav_mute
       27    ?wzsnd_get_wav_vol@@YAXPAH0@Z (void __cdecl wzsnd_get_wav_vol(int *,int *))
               exported name: wzsnd_get_wav_vol
       28    ?wzsnd_init@@YAHPAUWZSNDINFO@@@Z (int __cdecl wzsnd_init(struct WZSNDINFO *))
               exported name: wzsnd_init
       29    ?wzsnd_load_gameplay@@YAXXZ (void __cdecl wzsnd_load_gameplay(void))
               exported name: wzsnd_load_gameplay
       30    ?wzsnd_load_ui@@YAXXZ (void __cdecl wzsnd_load_ui(void))
               exported name: wzsnd_load_ui
       31    ?wzsnd_pause@@YAXH@Z (void __cdecl wzsnd_pause(int))
               exported name: wzsnd_pause
       32    ?wzsnd_pause_all@@YAXXZ (void __cdecl wzsnd_pause_all(void))
               exported name: wzsnd_pause_all
       33    ?wzsnd_pause_all_ambi@@YAXXZ (void __cdecl wzsnd_pause_all_ambi(void))
               exported name: wzsnd_pause_all_ambi
       34    ?wzsnd_pause_all_bgm@@YAXXZ (void __cdecl wzsnd_pause_all_bgm(void))
               exported name: wzsnd_pause_all_bgm
       35    ?wzsnd_pause_all_voice@@YAXXZ (void __cdecl wzsnd_pause_all_voice(void))
               exported name: wzsnd_pause_all_voice
       36    ?wzsnd_pause_ambi@@YAXH@Z (void __cdecl wzsnd_pause_ambi(int))
               exported name: wzsnd_pause_ambi
       37    ?wzsnd_pause_bgm@@YAXH@Z (void __cdecl wzsnd_pause_bgm(int))
               exported name: wzsnd_pause_bgm
       38    ?wzsnd_pause_voice@@YAXH@Z (void __cdecl wzsnd_pause_voice(int))
               exported name: wzsnd_pause_voice
       39    ?wzsnd_play@@YAHHHHMH@Z (int __cdecl wzsnd_play(int,int,int,float,int))
               exported name: wzsnd_play
       40    ?wzsnd_play_3d@@YAHHPAU_D3DVECTOR@@00HHPAUSND_SOURCEDESC@@@Z (int __cdecl wzsnd_play_3d(int,struct _D3DVECTOR *,struct _D3DVECTOR *,struct _D3DVECTOR *,int,int,struct SND_SOURCEDESC *))
               exported name: wzsnd_play_3d
       41    ?wzsnd_play_ambi@@YAHHHHMHH@Z (int __cdecl wzsnd_play_ambi(int,int,int,float,int,int))
               exported name: wzsnd_play_ambi
       42    ?wzsnd_play_bgm@@YAHHHMH@Z (int __cdecl wzsnd_play_bgm(int,int,float,int))
               exported name: wzsnd_play_bgm
       43    ?wzsnd_play_ui@@YAHHM@Z (int __cdecl wzsnd_play_ui(int,float))
               exported name: wzsnd_play_ui
       44    ?wzsnd_play_voice@@YAHHHMH@Z (int __cdecl wzsnd_play_voice(int,int,float,int))
               exported name: wzsnd_play_voice
       45    ?wzsnd_reload_soundtable@@YAXXZ (void __cdecl wzsnd_reload_soundtable(void))
               exported name: wzsnd_reload_soundtable
       46    ?wzsnd_set_loop_ambi@@YAXHH@Z (void __cdecl wzsnd_set_loop_ambi(int,int))
               exported name: wzsnd_set_loop_ambi
       47    ?wzsnd_set_loop_bgm@@YAXHH@Z (void __cdecl wzsnd_set_loop_bgm(int,int))
               exported name: wzsnd_set_loop_bgm
       48    ?wzsnd_set_loop_voice@@YAXHH@Z (void __cdecl wzsnd_set_loop_voice(int,int))
               exported name: wzsnd_set_loop_voice
       49    ?wzsnd_set_master_mute@@YAX_N@Z (void __cdecl wzsnd_set_master_mute(bool))
               exported name: wzsnd_set_master_mute
       50    ?wzsnd_set_master_vol@@YAXHH@Z (void __cdecl wzsnd_set_master_vol(int,int))
               exported name: wzsnd_set_master_vol
       51    ?wzsnd_set_mic_input_vol@@YAXK@Z (void __cdecl wzsnd_set_mic_input_vol(unsigned long))
               exported name: wzsnd_set_mic_input_vol
       52    ?wzsnd_set_mic_output_mute@@YAX_N@Z (void __cdecl wzsnd_set_mic_output_mute(bool))
               exported name: wzsnd_set_mic_output_mute
       53    ?wzsnd_set_mic_output_vol@@YAXK@Z (void __cdecl wzsnd_set_mic_output_vol(unsigned long))
               exported name: wzsnd_set_mic_output_vol
       54    ?wzsnd_set_volume@@YAXHM@Z (void __cdecl wzsnd_set_volume(int,float))
               exported name: wzsnd_set_volume
       55    ?wzsnd_set_volume_all@@YAXM@Z (void __cdecl wzsnd_set_volume_all(float))
               exported name: wzsnd_set_volume_all
       56    ?wzsnd_set_volume_all_ambi@@YAXM@Z (void __cdecl wzsnd_set_volume_all_ambi(float))
               exported name: wzsnd_set_volume_all_ambi
       57    ?wzsnd_set_volume_all_bgm@@YAXM@Z (void __cdecl wzsnd_set_volume_all_bgm(float))
               exported name: wzsnd_set_volume_all_bgm
       58    ?wzsnd_set_volume_all_voice@@YAXM@Z (void __cdecl wzsnd_set_volume_all_voice(float))
               exported name: wzsnd_set_volume_all_voice
       59    ?wzsnd_set_volume_ambi@@YAXHM@Z (void __cdecl wzsnd_set_volume_ambi(int,float))
               exported name: wzsnd_set_volume_ambi
       60    ?wzsnd_set_volume_bgm@@YAXHM@Z (void __cdecl wzsnd_set_volume_bgm(int,float))
               exported name: wzsnd_set_volume_bgm
       61    ?wzsnd_set_volume_voice@@YAXHM@Z (void __cdecl wzsnd_set_volume_voice(int,float))
               exported name: wzsnd_set_volume_voice
       62    ?wzsnd_set_wav_mute@@YAX_N@Z (void __cdecl wzsnd_set_wav_mute(bool))
               exported name: wzsnd_set_wav_mute
       63    ?wzsnd_set_wav_vol@@YAXHH@Z (void __cdecl wzsnd_set_wav_vol(int,int))
               exported name: wzsnd_set_wav_vol
       64    ?wzsnd_stop@@YAXH@Z (void __cdecl wzsnd_stop(int))
               exported name: wzsnd_stop
       65    ?wzsnd_stop_all@@YAXXZ (void __cdecl wzsnd_stop_all(void))
               exported name: wzsnd_stop_all
       66    ?wzsnd_stop_all_ambi@@YAXH@Z (void __cdecl wzsnd_stop_all_ambi(int))
               exported name: wzsnd_stop_all_ambi
       67    ?wzsnd_stop_all_bgm@@YAXH@Z (void __cdecl wzsnd_stop_all_bgm(int))
               exported name: wzsnd_stop_all_bgm
       68    ?wzsnd_stop_all_voice@@YAXH@Z (void __cdecl wzsnd_stop_all_voice(int))
               exported name: wzsnd_stop_all_voice
       69    ?wzsnd_stop_ambi@@YAXHH@Z (void __cdecl wzsnd_stop_ambi(int,int))
               exported name: wzsnd_stop_ambi
       70    ?wzsnd_stop_bgm@@YAXHH@Z (void __cdecl wzsnd_stop_bgm(int,int))
               exported name: wzsnd_stop_bgm
       71    ?wzsnd_stop_ui@@YAXH@Z (void __cdecl wzsnd_stop_ui(int))
               exported name: wzsnd_stop_ui
       72    ?wzsnd_stop_voice@@YAXHH@Z (void __cdecl wzsnd_stop_voice(int,int))
               exported name: wzsnd_stop_voice
       73    ?wzsnd_uninit@@YAXXZ (void __cdecl wzsnd_uninit(void))
               exported name: wzsnd_uninit
       74    ?wzsnd_unload_gameplay@@YAXXZ (void __cdecl wzsnd_unload_gameplay(void))
               exported name: wzsnd_unload_gameplay
       75    ?wzsnd_unload_ui@@YAXXZ (void __cdecl wzsnd_unload_ui(void))
               exported name: wzsnd_unload_ui
       76    ?wzsnd_unpause@@YAXH@Z (void __cdecl wzsnd_unpause(int))
               exported name: wzsnd_unpause
       77    ?wzsnd_unpause_all@@YAXXZ (void __cdecl wzsnd_unpause_all(void))
               exported name: wzsnd_unpause_all
       78    ?wzsnd_unpause_all_ambi@@YAXXZ (void __cdecl wzsnd_unpause_all_ambi(void))
               exported name: wzsnd_unpause_all_ambi
       79    ?wzsnd_unpause_all_bgm@@YAXXZ (void __cdecl wzsnd_unpause_all_bgm(void))
               exported name: wzsnd_unpause_all_bgm
       80    ?wzsnd_unpause_all_voice@@YAXXZ (void __cdecl wzsnd_unpause_all_voice(void))
               exported name: wzsnd_unpause_all_voice
       81    ?wzsnd_unpause_ambi@@YAXH@Z (void __cdecl wzsnd_unpause_ambi(int))
               exported name: wzsnd_unpause_ambi
       82    ?wzsnd_unpause_bgm@@YAXH@Z (void __cdecl wzsnd_unpause_bgm(int))
               exported name: wzsnd_unpause_bgm
       83    ?wzsnd_unpause_voice@@YAXH@Z (void __cdecl wzsnd_unpause_voice(int))
               exported name: wzsnd_unpause_voice
       84    ?wzsnd_update_3d_source@@YAXHPAU_D3DVECTOR@@0PAUSND_SOURCEDESC@@@Z (void __cdecl wzsnd_update_3d_source(int,struct _D3DVECTOR *,struct _D3DVECTOR *,struct SND_SOURCEDESC *))
               exported name: wzsnd_update_3d_source
       85    ?wzsnd_update_cache@@YAXXZ (void __cdecl wzsnd_update_cache(void))
               exported name: wzsnd_update_cache
       86    ?wzsnd_update_listener@@YAXPAU_D3DVECTOR@@000@Z (void __cdecl wzsnd_update_listener(struct _D3DVECTOR *,struct _D3DVECTOR *,struct _D3DVECTOR *,struct _D3DVECTOR *))
               exported name: wzsnd_update_listener
